 config_alm_process

 Timestamp is 614c8062 (Thu Sep 23 13:25:54 2021)

 Preferred load address is 10000000

 Start         Length     Name                   Class
 0001:00000000 000002a0H .text$di                CODE
 0001:000002a0 0001e21aH .text$mn                CODE
 0001:0001e4ba 00004791H .text$x                 CODE
 0001:00022c4b 0000011eH .text$yd                CODE
 0002:00000000 00001740H .idata$5                DATA
 0002:00001740 00000004H .CRT$XCA                DATA
 0002:00001744 00000054H .CRT$XCU                DATA
 0002:00001798 00000004H .CRT$XCZ                DATA
 0002:0000179c 00000004H .CRT$XIA                DATA
 0002:000017a0 00000004H .CRT$XIAA               DATA
 0002:000017a4 00000004H .CRT$XIC                DATA
 0002:000017a8 00000004H .CRT$XIZ                DATA
 0002:000017b0 0000acb0H .rdata                  DATA
 0002:0000c460 00001ee8H .rdata$r                DATA
 0002:0000e348 00000004H .rtc$IAA                DATA
 0002:0000e34c 00000004H .rtc$IZZ                DATA
 0002:0000e350 00000004H .rtc$TAA                DATA
 0002:0000e354 00000004H .rtc$TZZ                DATA
 0002:0000e358 00004234H .xdata$x                DATA
 0002:00012590 00000b9eH .edata                  DATA
 0002:00013130 00000078H .idata$2                DATA
 0002:000131a8 00000014H .idata$3                DATA
 0002:000131bc 00001740H .idata$4                DATA
 0002:000148fc 0000f308H .idata$6                DATA
 0003:00000000 0000037cH .data                   DATA
 0003:0000037c 0000098cH .data$r                 DATA
 0003:00000d08 000004ccH .bss                    DATA
 0004:00000000 000000a0H .rsrc$01                DATA
 0004:000000a0 00000628H .rsrc$02                DATA

  Address         Publics by Value              Rva+Base       Lib:Object

 0000:00000000       ___guard_flags             00000000     <absolute>
 0000:00000000       ___guard_fids_table        00000000     <absolute>
 0000:00000000       ___safe_se_handler_table   00000000     <absolute>
 0000:00000000       ___guard_fids_count        00000000     <absolute>
 0000:00000000       __except_list              00000000     <absolute>
 0000:00000000       ___safe_se_handler_count   00000000     <absolute>
 0000:00009876       __fltused                  00009876     <absolute>
 0000:00009876       __ldused                   00009876     <absolute>
 0000:00000000       ___ImageBase               10000000     <linker-defined>
 0001:000002a0       ??$_Allocate@U?$_Tree_node@U?$pair@$$CBVQString@@PAVcProcess@@@std@@PAX@std@@@std@@YAPAU?$_Tree_node@U?$pair@$$CBVQString@@PAVcProcess@@@std@@PAX@0@IPAU10@@Z 100012a0 f i alm_process.obj
 0001:000002cd       ??$_Buynode@ABUpiecewise_construct_t@std@@V?$tuple@$$QAVQString@@@2@V?$tuple@$$$V@2@@?$_Tree_buy@U?$pair@$$CBVQString@@PAVcProcess@@@std@@V?$allocator@U?$pair@$$CBVQString@@PAVcProcess@@@std@@@2@@std@@QAEPAU?$_Tree_node@U?$pair@$$CBVQString@@PAVcProcess@@@std@@PAX@1@ABUpiecewise_construct_t@1@$$QAV?$tuple@$$QAVQString@@@1@$$QAV?$tuple@$$$V@1@@Z 100012cd f i alm_process.obj
 0001:000002cd       ??$_Buynode@ABUpiecewise_construct_t@std@@V?$tuple@ABVQString@@@2@V?$tuple@$$$V@2@@?$_Tree_buy@U?$pair@$$CBVQString@@PAVcProcess@@@std@@V?$allocator@U?$pair@$$CBVQString@@PAVcProcess@@@std@@@2@@std@@QAEPAU?$_Tree_node@U?$pair@$$CBVQString@@PAVcProcess@@@std@@PAX@1@ABUpiecewise_construct_t@1@$$QAV?$tuple@ABVQString@@@1@$$QAV?$tuple@$$$V@1@@Z 100012cd f i alm_process.obj
 0001:0000031e       ??$_Buynode@U?$pair@VQString@@PAVcProcess@@@std@@@?$_Tree_buy@U?$pair@$$CBVQString@@PAVcProcess@@@std@@V?$allocator@U?$pair@$$CBVQString@@PAVcProcess@@@std@@@2@@std@@QAEPAU?$_Tree_node@U?$pair@$$CBVQString@@PAVcProcess@@@std@@PAX@1@$$QAU?$pair@VQString@@PAVcProcess@@@1@@Z 1000131e f i alm_process.obj
 0001:00000369       ??$_Insert_at@AAU?$pair@$$CBVQString@@PAVcProcess@@@std@@PAU?$_Tree_node@U?$pair@$$CBVQString@@PAVcProcess@@@std@@PAX@2@@?$_Tree@V?$_Tmap_traits@VQString@@PAVcProcess@@U?$less@VQString@@@std@@V?$allocator@U?$pair@$$CBVQString@@PAVcProcess@@@std@@@4@$0A@@std@@@std@@IAE?AV?$_Tree_iterator@V?$_Tree_val@U?$_Tree_simple_types@U?$pair@$$CBVQString@@PAVcProcess@@@std@@@std@@@std@@@1@_NPAU?$_Tree_node@U?$pair@$$CBVQString@@PAVcProcess@@@std@@PAX@1@AAU?$pair@$$CBVQString@@PAVcProcess@@@1@1@Z 10001369 f i alm_process.obj
 0001:00000496       ??$_Insert_hint@AAU?$pair@$$CBVQString@@PAVcProcess@@@std@@PAU?$_Tree_node@U?$pair@$$CBVQString@@PAVcProcess@@@std@@PAX@2@@?$_Tree@V?$_Tmap_traits@VQString@@PAVcProcess@@U?$less@VQString@@@std@@V?$allocator@U?$pair@$$CBVQString@@PAVcProcess@@@std@@@4@$0A@@std@@@std@@IAE?AV?$_Tree_iterator@V?$_Tree_val@U?$_Tree_simple_types@U?$pair@$$CBVQString@@PAVcProcess@@@std@@@std@@@std@@@1@V?$_Tree_const_iterator@V?$_Tree_val@U?$_Tree_simple_types@U?$pair@$$CBVQString@@PAVcProcess@@@std@@@std@@@std@@@1@AAU?$pair@$$CBVQString@@PAVcProcess@@@1@PAU?$_Tree_node@U?$pair@$$CBVQString@@PAVcProcess@@@std@@PAX@1@@Z 10001496 f i alm_process.obj
 0001:00000608       ??$_Insert_nohint@AAU?$pair@$$CBVQString@@PAVcProcess@@@std@@PAU?$_Tree_node@U?$pair@$$CBVQString@@PAVcProcess@@@std@@PAX@2@@?$_Tree@V?$_Tmap_traits@VQString@@PAVcProcess@@U?$less@VQString@@@std@@V?$allocator@U?$pair@$$CBVQString@@PAVcProcess@@@std@@@4@$0A@@std@@@std@@IAE?AU?$pair@V?$_Tree_iterator@V?$_Tree_val@U?$_Tree_simple_types@U?$pair@$$CBVQString@@PAVcProcess@@@std@@@std@@@std@@@std@@_N@1@_NAAU?$pair@$$CBVQString@@PAVcProcess@@@1@PAU?$_Tree_node@U?$pair@$$CBVQString@@PAVcProcess@@@std@@PAX@1@@Z 10001608 f i alm_process.obj
 0001:00000700       ??$construct@U?$pair@$$CBVQString@@PAVcProcess@@@std@@ABUpiecewise_construct_t@2@V?$tuple@ABVQString@@@2@V?$tuple@$$$V@2@@?$allocator@U?$_Tree_node@U?$pair@$$CBVQString@@PAVcProcess@@@std@@PAX@std@@@std@@QAEXPAU?$pair@$$CBVQString@@PAVcProcess@@@1@ABUpiecewise_construct_t@1@$$QAV?$tuple@ABVQString@@@1@$$QAV?$tuple@$$$V@1@@Z 10001700 f i alm_process.obj
 0001:00000700       ??$construct@U?$pair@$$CBVQString@@PAVcProcess@@@std@@ABUpiecewise_construct_t@2@V?$tuple@$$QAVQString@@@2@V?$tuple@$$$V@2@@?$allocator@U?$_Tree_node@U?$pair@$$CBVQString@@PAVcProcess@@@std@@PAX@std@@@std@@QAEXPAU?$pair@$$CBVQString@@PAVcProcess@@@1@ABUpiecewise_construct_t@1@$$QAV?$tuple@$$QAVQString@@@1@$$QAV?$tuple@$$$V@1@@Z 10001700 f i alm_process.obj
 0001:00000733       ??$construct@U?$pair@$$CBVQString@@PAVcProcess@@@std@@U?$pair@VQString@@PAVcProcess@@@2@@?$allocator@U?$_Tree_node@U?$pair@$$CBVQString@@PAVcProcess@@@std@@PAX@std@@@std@@QAEXPAU?$pair@$$CBVQString@@PAVcProcess@@@1@$$QAU?$pair@VQString@@PAVcProcess@@@1@@Z 10001733 f i alm_process.obj
 0001:00000767       ??$insert@U?$pair@VQString@@PAVcProcess@@@std@@@?$_Tree@V?$_Tmap_traits@VQString@@PAVcProcess@@U?$less@VQString@@@std@@V?$allocator@U?$pair@$$CBVQString@@PAVcProcess@@@std@@@4@$0A@@std@@@std@@QAE?AU?$pair@V?$_Tree_iterator@V?$_Tree_val@U?$_Tree_simple_types@U?$pair@$$CBVQString@@PAVcProcess@@@std@@@std@@@std@@@std@@_N@1@$$QAU?$pair@VQString@@PAVcProcess@@@1@@Z 10001767 f i alm_process.obj
 0001:0000078e       ??0?$QGuardedPtr@VQDockWindow@@@@QAE@XZ 1000178e f i alm_process.obj
 0001:0000078e       ??0?$QGuardedPtr@VQPopupMenu@@@@QAE@XZ 1000178e f i alm_process.obj
 0001:000007cf       ??0ProcessListView@@QAE@PAVQWidget@@PBDI@Z 100017cf f   alm_process.obj
 0001:00000814       ??0ProcessListViewItem@@QAE@PAVQListView@@PAVcProcess@@@Z 10001814 f   alm_process.obj
 0001:000008e7       ??0alm_process@@QAE@ABVQString@@00@Z 100018e7 f   alm_process.obj
 0001:00002721       ??0config_plugin_base@@QAE@ABVQString@@00@Z 10003721 f i alm_process.obj
 0001:000027ae       ??1?$QGuardedPtr@VQPopupMenu@@@@QAE@XZ 100037ae f i alm_process.obj
 0001:000027ae       ??1?$QGuardedPtr@VQDockWindow@@@@QAE@XZ 100037ae f i alm_process.obj
 0001:000027b3       ??1?$QPtrList@VQListViewItem@@@@UAE@XZ 100037b3 f i alm_process.obj
 0001:000027e6       ??1?$QPtrList@VQPopupMenu@@@@UAE@XZ 100037e6 f i alm_process.obj
 0001:00002819       ??1?$QPtrList@VcProcess@@@@UAE@XZ 10003819 f i alm_process.obj
 0001:0000284c       ??1?$_Tree@V?$_Tmap_traits@VQString@@PAVcProcess@@U?$less@VQString@@@std@@V?$allocator@U?$pair@$$CBVQString@@PAVcProcess@@@std@@@4@$0A@@std@@@std@@QAE@XZ 1000384c f i alm_process.obj
 0001:0000286e       ??1?$pair@VQString@@PAVcProcess@@@std@@QAE@XZ 1000386e f i alm_process.obj
 0001:00002874       ??1ProcessListView@@UAE@XZ 10003874 f   alm_process.obj
 0001:00002887       ??1ProcessListViewItem@@UAE@XZ 10003887 f   alm_process.obj
 0001:00002893       ??1QDockWindowList@@UAE@XZ 10003893 f i alm_process.obj
 0001:000028dc       ??1QPopupMenuList@@UAE@XZ  100038dc f i alm_process.obj
 0001:0000290e       ??1alm_process@@UAE@XZ     1000390e f   alm_process.obj
 0001:00002ab8       ??1config_plugin_base@@UAE@XZ 10003ab8 f i alm_process.obj
 0001:00002b12       ??4?$QGuardedPtr@VQDockWindow@@@@QAEAAV0@PAVQDockWindow@@@Z 10003b12 f i alm_process.obj
 0001:00002b12       ??4?$QGuardedPtr@VQPopupMenu@@@@QAEAAV0@PAVQPopupMenu@@@Z 10003b12 f i alm_process.obj
 0001:00002b70       ??A?$map@VQString@@PAVcProcess@@U?$less@VQString@@@std@@V?$allocator@U?$pair@$$CBVQString@@PAVcProcess@@@std@@@4@@std@@QAEAAPAVcProcess@@$$QAVQString@@@Z 10003b70 f i alm_process.obj
 0001:00002b70       ??A?$map@VQString@@PAVcProcess@@U?$less@VQString@@@std@@V?$allocator@U?$pair@$$CBVQString@@PAVcProcess@@@std@@@4@@std@@QAEAAPAVcProcess@@ABVQString@@@Z 10003b70 f i alm_process.obj
 0001:00002bd0       ??E?$_Tree_unchecked_const_iterator@V?$_Tree_val@U?$_Tree_simple_types@U?$pair@$$CBVQString@@PAVcProcess@@@std@@@std@@@std@@U_Iterator_base0@2@@std@@QAEAAV01@XZ 10003bd0 f i alm_process.obj
 0001:00002c0a       ??F?$_Tree_unchecked_const_iterator@V?$_Tree_val@U?$_Tree_simple_types@U?$pair@$$CBVQString@@PAVcProcess@@@std@@@std@@@std@@U_Iterator_base0@2@@std@@QAEAAV01@XZ 10003c0a f i alm_process.obj
 0001:00002c4e       ??_ECAlm_sys_select@@WCI@AEPAXI@Z 10003c4e f i alm_process.obj
 0001:00002c56       ??_EProcessListView@@WCI@AEPAXI@Z 10003c56 f i alm_process.obj
 0001:00002c5e       ??_EQDockWindow@@WCI@AEPAXI@Z 10003c5e f i alm_process.obj
 0001:00002c66       ??_EQHBoxLayout@@WCI@AEPAXI@Z 10003c66 f i alm_process.obj
 0001:00002c6e       ??_EQLabel@@WCI@AEPAXI@Z   10003c6e f i alm_process.obj
 0001:00002c76       ??_EQLineEdit@@WCI@AEPAXI@Z 10003c76 f i alm_process.obj
 0001:00002c7e       ??_EQPopupMenu@@WCI@AEPAXI@Z 10003c7e f i alm_process.obj
 0001:00002c86       ??_EQPopupMenu@@WIM@AEPAXI@Z 10003c86 f i alm_process.obj
 0001:00002c91       ??_EQPushButton@@WCI@AEPAXI@Z 10003c91 f i alm_process.obj
 0001:00002c99       ??_EQTabWidget@@WCI@AEPAXI@Z 10003c99 f i alm_process.obj
 0001:00002ca1       ??_EQToolBar@@WCI@AEPAXI@Z 10003ca1 f i alm_process.obj
 0001:00002ca9       ??_EQVBoxLayout@@WCI@AEPAXI@Z 10003ca9 f i alm_process.obj
 0001:00002cb1       ??_EQWidget@@WCI@AEPAXI@Z  10003cb1 f i alm_process.obj
 0001:00002cb9       ??_Ealm_process@@WCI@AEPAXI@Z 10003cb9 f i alm_process.obj
 0001:00002cc1       ??_Econfig_plugin_base@@WCI@AEPAXI@Z 10003cc1 f i alm_process.obj
 0001:00002cc9       ??_E?$QPtrList@VQListViewItem@@@@UAEPAXI@Z 10003cc9 f i alm_process.obj
 0001:00002cc9       ??_G?$QPtrList@VQListViewItem@@@@UAEPAXI@Z 10003cc9 f i alm_process.obj
 0001:00002ce8       ??_G?$QPtrList@VQPopupMenu@@@@UAEPAXI@Z 10003ce8 f i alm_process.obj
 0001:00002ce8       ??_E?$QPtrList@VQPopupMenu@@@@UAEPAXI@Z 10003ce8 f i alm_process.obj
 0001:00002d07       ??_G?$QPtrList@VcProcess@@@@UAEPAXI@Z 10003d07 f i alm_process.obj
 0001:00002d07       ??_E?$QPtrList@VcProcess@@@@UAEPAXI@Z 10003d07 f i alm_process.obj
 0001:00002d26       ??_GCAlm_sys_select@@UAEPAXI@Z 10003d26 f i alm_process.obj
 0001:00002d26       ??_ECAlm_sys_select@@UAEPAXI@Z 10003d26 f i alm_process.obj
 0001:00002d46       ??_GProcessListView@@UAEPAXI@Z 10003d46 f i alm_process.obj
 0001:00002d46       ??_EProcessListView@@UAEPAXI@Z 10003d46 f i alm_process.obj
 0001:00002d65       ??_GProcessListViewItem@@UAEPAXI@Z 10003d65 f i alm_process.obj
 0001:00002d65       ??_EProcessListViewItem@@UAEPAXI@Z 10003d65 f i alm_process.obj
 0001:00002d84       ??_EQAction@@UAEPAXI@Z     10003d84 f i alm_process.obj
 0001:00002d84       ??_GQAction@@UAEPAXI@Z     10003d84 f i alm_process.obj
 0001:00002da4       ??_GQDockWindow@@UAEPAXI@Z 10003da4 f i alm_process.obj
 0001:00002da4       ??_EQDockWindow@@UAEPAXI@Z 10003da4 f i alm_process.obj
 0001:00002dc4       ??_EQDockWindowList@@UAEPAXI@Z 10003dc4 f i alm_process.obj
 0001:00002dc4       ??_GQDockWindowList@@UAEPAXI@Z 10003dc4 f i alm_process.obj
 0001:00002de3       ??_EQGuardedPtrPrivate@@UAEPAXI@Z 10003de3 f i alm_process.obj
 0001:00002de3       ??_GQGuardedPtrPrivate@@UAEPAXI@Z 10003de3 f i alm_process.obj
 0001:00002e03       ??_EQHBoxLayout@@UAEPAXI@Z 10003e03 f i alm_process.obj
 0001:00002e03       ??_GQHBoxLayout@@UAEPAXI@Z 10003e03 f i alm_process.obj
 0001:00002e23       ??_GQLabel@@UAEPAXI@Z      10003e23 f i alm_process.obj
 0001:00002e23       ??_EQLabel@@UAEPAXI@Z      10003e23 f i alm_process.obj
 0001:00002e43       ??_EQLineEdit@@UAEPAXI@Z   10003e43 f i alm_process.obj
 0001:00002e43       ??_GQLineEdit@@UAEPAXI@Z   10003e43 f i alm_process.obj
 0001:00002e63       ??_GQListViewItem@@UAEPAXI@Z 10003e63 f i alm_process.obj
 0001:00002e63       ??_EQListViewItem@@UAEPAXI@Z 10003e63 f i alm_process.obj
 0001:00002e83       ??_EQPopupMenu@@UAEPAXI@Z  10003e83 f i alm_process.obj
 0001:00002e83       ??_GQPopupMenu@@UAEPAXI@Z  10003e83 f i alm_process.obj
 0001:00002ea3       ??_GQPopupMenuList@@UAEPAXI@Z 10003ea3 f i alm_process.obj
 0001:00002ea3       ??_EQPopupMenuList@@UAEPAXI@Z 10003ea3 f i alm_process.obj
 0001:00002ec2       ??_EQPushButton@@UAEPAXI@Z 10003ec2 f i alm_process.obj
 0001:00002ec2       ??_GQPushButton@@UAEPAXI@Z 10003ec2 f i alm_process.obj
 0001:00002ee2       ??_EQSpacerItem@@UAEPAXI@Z 10003ee2 f i alm_process.obj
 0001:00002ee2       ??_GQSpacerItem@@UAEPAXI@Z 10003ee2 f i alm_process.obj
 0001:00002f02       ??_GQTabWidget@@UAEPAXI@Z  10003f02 f i alm_process.obj
 0001:00002f02       ??_EQTabWidget@@UAEPAXI@Z  10003f02 f i alm_process.obj
 0001:00002f22       ??_GQToolBar@@UAEPAXI@Z    10003f22 f i alm_process.obj
 0001:00002f22       ??_EQToolBar@@UAEPAXI@Z    10003f22 f i alm_process.obj
 0001:00002f42       ??_GQVBoxLayout@@UAEPAXI@Z 10003f42 f i alm_process.obj
 0001:00002f42       ??_EQVBoxLayout@@UAEPAXI@Z 10003f42 f i alm_process.obj
 0001:00002f62       ??_GQWidget@@UAEPAXI@Z     10003f62 f i alm_process.obj
 0001:00002f62       ??_EQWidget@@UAEPAXI@Z     10003f62 f i alm_process.obj
 0001:00002f82       ??_Ealm_process@@UAEPAXI@Z 10003f82 f i alm_process.obj
 0001:00002f82       ??_Galm_process@@UAEPAXI@Z 10003f82 f i alm_process.obj
 0001:00002fa1       ??_Econfig_plugin_base@@UAEPAXI@Z 10003fa1 f i alm_process.obj
 0001:00002fa1       ??_Gconfig_plugin_base@@UAEPAXI@Z 10003fa1 f i alm_process.obj
 0001:00002fc0       ?_Buyheadnode@?$_Tree_alloc@$0A@U?$_Tree_base_types@U?$pair@$$CBVQString@@PAVcProcess@@@std@@V?$allocator@U?$pair@$$CBVQString@@PAVcProcess@@@std@@@2@@std@@@std@@QAEPAU?$_Tree_node@U?$pair@$$CBVQString@@PAVcProcess@@@std@@PAX@2@XZ 10003fc0 f i alm_process.obj
 0001:00002fea       ?_Buynode0@?$_Tree_buy@U?$pair@$$CBVQString@@PAVcProcess@@@std@@V?$allocator@U?$pair@$$CBVQString@@PAVcProcess@@@std@@@2@@std@@QAEPAU?$_Tree_node@U?$pair@$$CBVQString@@PAVcProcess@@@std@@PAX@2@XZ 10003fea f i alm_process.obj
 0001:0000301c       ?_Erase@?$_Tree@V?$_Tmap_traits@VQString@@PAVcProcess@@U?$less@VQString@@@std@@V?$allocator@U?$pair@$$CBVQString@@PAVcProcess@@@std@@@4@$0A@@std@@@std@@IAEXPAU?$_Tree_node@U?$pair@$$CBVQString@@PAVcProcess@@@std@@PAX@2@@Z 1000401c f i alm_process.obj
 0001:0000305a       ?_Lrotate@?$_Tree@V?$_Tmap_traits@VQString@@PAVcProcess@@U?$less@VQString@@@std@@V?$allocator@U?$pair@$$CBVQString@@PAVcProcess@@@std@@@4@$0A@@std@@@std@@IAEXPAU?$_Tree_node@U?$pair@$$CBVQString@@PAVcProcess@@@std@@PAX@2@@Z 1000405a f i alm_process.obj
 0001:0000309e       ?_Rrotate@?$_Tree@V?$_Tmap_traits@VQString@@PAVcProcess@@U?$less@VQString@@@std@@V?$allocator@U?$pair@$$CBVQString@@PAVcProcess@@@std@@@4@$0A@@std@@@std@@IAEXPAU?$_Tree_node@U?$pair@$$CBVQString@@PAVcProcess@@@std@@PAX@2@@Z 1000409e f i alm_process.obj
 0001:000030e4       ?about@alm_process@@EAE?AVQString@@XZ 100040e4 f   alm_process.obj
 0001:0000317b       ?about@config_plugin_base@@UAE?AVQString@@XZ 1000417b f i alm_process.obj
 0001:000031d1       ?activate@alm_process@@UAEX_N@Z 100041d1 f   alm_process.obj
 0001:00003315       ?addMultiInputs@alm_process@@AAEXXZ 10004315 f   alm_process.obj
 0001:0000339c       ?addSingleInputs@alm_process@@AAEXXZ 1000439c f   alm_process.obj
 0001:00003436       ?apply@alm_process@@EAEXXZ 10004436 f   alm_process.obj
 0001:0000355b       ?apply@config_plugin_base@@UAEXXZ 1000455b f i alm_process.obj
 0001:0000355b       ??3@YAXPAX0@Z              1000455b f i alm_process.obj
 0001:0000355c       ?changeMask@alm_process@@AAEXXZ 1000455c f   alm_process.obj
 0001:000035ea       ?checkProcessContributors@alm_process@@AAEXXZ 100045ea f   alm_process.obj
 0001:00003f74       ?checkReferences@alm_process@@AAEXXZ 10004f74 f   alm_process.obj
 0001:00004032       ?clear@?$QPtrList@VcProcess@@@@UAEXXZ 10005032 f i alm_process.obj
 0001:00004032       ?clear@?$QPtrList@VQPopupMenu@@@@UAEXXZ 10005032 f i alm_process.obj
 0001:00004032       ?clear@?$QPtrList@VQListViewItem@@@@UAEXXZ 10005032 f i alm_process.obj
 0001:00004038       ?clear@?$_Tree@V?$_Tmap_traits@VQString@@PAVcProcess@@U?$less@VQString@@@std@@V?$allocator@U?$pair@$$CBVQString@@PAVcProcess@@@std@@@4@$0A@@std@@@std@@QAEXXZ 10005038 f i alm_process.obj
 0001:00004059       ?clearFilter@alm_process@@AAEXXZ 10005059 f   alm_process.obj
 0001:00004067       ?clearMask@alm_process@@AAEXXZ 10005067 f   alm_process.obj
 0001:000041d0       ?closeEvent@alm_process@@UAEXPAVQCloseEvent@@@Z 100051d0 f   alm_process.obj
 0001:00004254       ?closeEvent@config_plugin_base@@UAEXPAVQCloseEvent@@@Z 10005254 f i alm_process.obj
 0001:00004262       ?copyProcessUsingTemplate@alm_process@@AAEXXZ 10005262 f   alm_process.obj
 0001:00004443       ?count@?$QPtrList@VQListViewItem@@@@UBEIXZ 10005443 f i alm_process.obj
 0001:00004443       ?count@?$QPtrList@VcProcess@@@@UBEIXZ 10005443 f i alm_process.obj
 0001:00004443       ?count@?$QPtrList@VQPopupMenu@@@@UBEIXZ 10005443 f i alm_process.obj
 0001:00004447       ?countSelections@alm_process@@AAEHPAPAVQListViewItem@@@Z 10005447 f   alm_process.obj
 0001:000044b1       ?deleteGroup@alm_process@@AAEXXZ 100054b1 f   alm_process.obj
 0001:00004658       ?deleteItem@?$QPtrList@VQPopupMenu@@@@EAEXPAX@Z 10005658 f i alm_process.obj
 0001:00004673       ?deleteItem@?$QPtrList@VcProcess@@@@EAEXPAX@Z 10005673 f i alm_process.obj
 0001:00004673       ?deleteItem@?$QPtrList@VQListViewItem@@@@EAEXPAX@Z 10005673 f i alm_process.obj
 0001:0000468d       ?deleteProcess@alm_process@@AAEXXZ 1000568d f   alm_process.obj
 0001:0000498c       ?deref@?$QGuardedPtr@VQDockWindow@@@@AAEXXZ 1000598c f i alm_process.obj
 0001:0000498c       ?deref@?$QGuardedPtr@VQPopupMenu@@@@AAEXXZ 1000598c f i alm_process.obj
 0001:000049a1       ?displayEnd@ProcessListView@@AAEX_N@Z 100059a1 f   alm_process.obj
 0001:00004a1e       ?displayHome@ProcessListView@@AAEX_N@Z 10005a1e f   alm_process.obj
 0001:00004a8b       ?duplicateProcess@alm_process@@AAEXXZ 10005a8b f   alm_process.obj
 0001:00004d79       ?erase@?$_Tree@V?$_Tmap_traits@VQString@@PAVcProcess@@U?$less@VQString@@@std@@V?$allocator@U?$pair@$$CBVQString@@PAVcProcess@@@std@@@4@$0A@@std@@@std@@QAE?AV?$_Tree_iterator@V?$_Tree_val@U?$_Tree_simple_types@U?$pair@$$CBVQString@@PAVcProcess@@@std@@@std@@@std@@@2@V?$_Tree_const_iterator@V?$_Tree_val@U?$_Tree_simple_types@U?$pair@$$CBVQString@@PAVcProcess@@@std@@@std@@@std@@@2@0@Z 10005d79 f i alm_process.obj
 0001:00004dc8       ?erase@?$_Tree@V?$_Tmap_traits@VQString@@PAVcProcess@@U?$less@VQString@@@std@@V?$allocator@U?$pair@$$CBVQString@@PAVcProcess@@@std@@@4@$0A@@std@@@std@@QAE?AV?$_Tree_iterator@V?$_Tree_val@U?$_Tree_simple_types@U?$pair@$$CBVQString@@PAVcProcess@@@std@@@std@@@std@@@2@V?$_Tree_const_iterator@V?$_Tree_val@U?$_Tree_simple_types@U?$pair@$$CBVQString@@PAVcProcess@@@std@@@std@@@std@@@2@@Z 10005dc8 f i alm_process.obj
 0001:00005016       ?filterChange@alm_process@@AAEXABVQString@@@Z 10006016 f   alm_process.obj
 0001:00005110       ?isDirty@alm_process@@UAE_NXZ 10006110 f   alm_process.obj
 0001:0000512a       ?keyPressEvent@ProcessListView@@EAEXPAVQKeyEvent@@@Z 1000612a f   alm_process.obj
 0001:0000516f       ?loadProcesses@alm_process@@AAE_NVQString@@@Z 1000616f f   alm_process.obj
 0001:0000588e       ?markDirty@alm_process@@AAEXXZ 1000688e f   alm_process.obj
 0001:00005a50       ?menus@alm_process@@UAE?AVQPopupMenuList@@XZ 10006a50 f   alm_process.obj
 0001:00005aab       ?menus@config_plugin_base@@UAE?AVQPopupMenuList@@XZ 10006aab f i alm_process.obj
 0001:00005ace       ?metaObject@alm_process@@UBEPAVQMetaObject@@XZ 10006ace f i alm_process.obj
 0001:00005ad3       ?navToAck@alm_process@@AAEXVQString@@00@Z 10006ad3 f   alm_process.obj
 0001:00005baf       ?navToOutput@alm_process@@AAEXVQString@@0@Z 10006baf f   alm_process.obj
 0001:00005c9d       ?navigate@alm_process@@UAEXABVQString@@0@Z 10006c9d f   alm_process.obj
 0001:00005d49       ?navigate@config_plugin_base@@UAEXABVQString@@0@Z 10006d49 f i alm_process.obj
 0001:00005d4c       ?newGate@alm_process@@AAEXXZ 10006d4c f   alm_process.obj
 0001:000062d8       ?newGroup@alm_process@@AAEXXZ 100072d8 f   alm_process.obj
 0001:000063df       ?newProcess@alm_process@@AAEXVQString@@AAVQStringList@@@Z 100073df f   alm_process.obj
 0001:0000652c       ?newProcess@alm_process@@AAEXXZ 1000752c f   alm_process.obj
 0001:00006684       ?paintCell@ProcessListViewItem@@EAEXPAVQPainter@@ABVQColorGroup@@HHH@Z 10007684 f   alm_process.obj
 0001:00006753       ?procListContextMenu@alm_process@@AAEXPAVQListViewItem@@ABVQPoint@@H@Z 10007753 f   alm_process.obj
 0001:00006772       ?renameGroup@alm_process@@AAEXXZ 10007772 f   alm_process.obj
 0001:00006abd       ?renameProcess@alm_process@@AAEXPAVQListViewItem@@HABVQString@@@Z 10007abd f   alm_process.obj
 0001:00006d8a       ?reply@alm_process@@UAEXPAVresponse@@@Z 10007d8a f   alm_process.obj
 0001:00007732       ?reply@config_plugin_base@@UAEXPAVresponse@@@Z 10008732 f i alm_process.obj
 0001:00007732       ?activate@config_plugin_base@@UAEX_N@Z 10008732 f i alm_process.obj
 0001:00007735       ?resizeEvent@alm_process@@UAEXPAVQResizeEvent@@@Z 10008735 f   alm_process.obj
 0001:0000776a       ?saveProcesses@alm_process@@AAE_NVQString@@@Z 1000876a f   alm_process.obj
 0001:00007a0f       ?selectProcess@alm_process@@AAEXPAVQListViewItem@@@Z 10008a0f f   alm_process.obj
 0001:000080b9       ?selectProcess@alm_process@@AAEXVQString@@@Z 100090b9 f   alm_process.obj
 0001:000081cb       ?selectProcess@alm_process@@AAEXXZ 100091cb f   alm_process.obj
 0001:00008217       ?selectSystem@alm_process@@AAEXABVQString@@@Z 10009217 f   alm_process.obj
 0001:00008863       ?setLatchAck@alm_process@@AAEXXZ 10009863 f   alm_process.obj
 0001:00008a53       ?setMask@alm_process@@AAEXXZ 10009a53 f   alm_process.obj
 0001:00008c2a       ?setProcessGroup@alm_process@@AAEXXZ 10009c2a f   alm_process.obj
 0001:00008e06       ?startRename@alm_process@@AAEXPAVQListViewItem@@@Z 10009e06 f   alm_process.obj
 0001:00008e1b       ?startRenameProc@alm_process@@AAEXXZ 10009e1b f   alm_process.obj
 0001:00008e34       ?sysCommand@alm_process@@AAEXABVQString@@0@Z 10009e34 f   alm_process.obj
 0001:00008e74       ?text@ProcessListViewItem@@UBE?AVQString@@H@Z 10009e74 f   alm_process.obj
 0001:00008eb4       ?toolbars@alm_process@@UAE?AVQDockWindowList@@XZ 10009eb4 f   alm_process.obj
 0001:00008f0f       ?toolbars@config_plugin_base@@UAE?AVQDockWindowList@@XZ 10009f0f f i alm_process.obj
 0001:00008f32       ?updateProcList@alm_process@@AAEXPAVcProcess@@@Z 10009f32 f   alm_process.obj
 0001:00008f9c       ?qt_static_property@cfg_Table@@SA_NPAVQObject@@HHPAVQVariant@@@Z 10009f9c f i cfg_widgets001:moc_cfg_Table.obj
 0001:00008f9c       ?validate@config_plugin_base@@UAE_NXZ 10009f9c f i alm_process.obj
 0001:00008f9c       ?qt_static_property@cfg_ListView@@SA_NPAVQObject@@HHPAVQVariant@@@Z 10009f9c f i cfg_widgets001:moc_cfg_ListView.obj
 0001:00008f9c       ?isDirty@config_plugin_base@@UAE_NXZ 10009f9c f i alm_process.obj
 0001:00008f9f       ??0cAcqFileData@@QAE@VQString@@@Z 10009f9f f   cAcqFileData.obj
 0001:00009033       ??1cAcqFileData@@UAE@XZ    1000a033 f   cAcqFileData.obj
 0001:000090a1       ??_EcAcqFileData@@UAEPAXI@Z 1000a0a1 f i cAcqFileData.obj
 0001:000090a1       ??_GcAcqFileData@@UAEPAXI@Z 1000a0a1 f i cAcqFileData.obj
 0001:000090c0       ?findSlot@cAcqFileData@@QAE?AVQString@@H@Z 1000a0c0 f   cAcqFileData.obj
 0001:00009183       ?findSlot@cAcqFileData@@QAEHVQString@@@Z 1000a183 f   cAcqFileData.obj
 0001:000091d3       ?loadDetails@cAcqFileData@@QAE_NXZ 1000a1d3 f   cAcqFileData.obj
 0001:000096a7       ??0CheckContDialog@@QAE@XZ 1000a6a7 f   checkContDialogImpl.obj
 0001:000096c6       ??1CheckContDialog@@UAE@XZ 1000a6c6 f   checkContDialogImpl.obj
 0001:000096d8       ??_ECheckContDialog@@WCI@AEPAXI@Z 1000a6d8 f i checkContDialogImpl.obj
 0001:000096e0       ??_ECheckContDialog@@UAEPAXI@Z 1000a6e0 f i checkContDialogImpl.obj
 0001:000096e0       ??_GCheckContDialog@@UAEPAXI@Z 1000a6e0 f i checkContDialogImpl.obj
 0001:000096ff       ?accept@CheckContDialog@@UAEXXZ 1000a6ff f   checkContDialogImpl.obj
 0001:000097ff       ?metaObject@CheckContDialog@@UBEPAVQMetaObject@@XZ 1000a7ff f i checkContDialogImpl.obj
 0001:00009804       ?rbContribDiag_clicked@CheckContDialog@@UAEXXZ 1000a804 f   checkContDialogImpl.obj
 0001:0000987c       ?rbInputDiag_clicked@CheckContDialog@@UAEXXZ 1000a87c f   checkContDialogImpl.obj
 0001:000098f3       ??0?$QMap@HPAVcAcqFileData@@@@QAE@XZ 1000a8f3 f i cProc_dialog.obj
 0001:00009926       ??0?$QMapPrivate@HPAVcAcqFileData@@@@QAE@PBV0@@Z 1000a926 f i cProc_dialog.obj
 0001:000099b1       ??0?$QMapPrivate@HPAVcAcqFileData@@@@QAE@XZ 1000a9b1 f i cProc_dialog.obj
 0001:000099e6       ??0ContributorListBoxItem@@QAE@PAVQListBox@@ABVQString@@_N@Z 1000a9e6 f   cProc_dialog.obj
 0001:00009a0b       ??0cProc_dialog@@QAE@QAVQStringList@@PAVQWidget@@PBDI@Z 1000aa0b f   cProc_dialog.obj
 0001:00009e77       ??1ContributorListBoxItem@@UAE@XZ 1000ae77 f   cProc_dialog.obj
 0001:00009e83       ??1cProc_dialog@@UAE@XZ    1000ae83 f   cProc_dialog.obj
 0001:00009f93       ??A?$QMap@HPAVcAcqFileData@@@@QAEAAPAVcAcqFileData@@ABH@Z 1000af93 f i cProc_dialog.obj
 0001:00009fe3       ??_EcProc_dialog@@WCI@AEPAXI@Z 1000afe3 f i cProc_dialog.obj
 0001:00009feb       ??_G?$QMapPrivate@HPAVcAcqFileData@@@@QAEPAXI@Z 1000afeb f i cProc_dialog.obj
 0001:0000a013       ??_EContributorListBoxItem@@UAEPAXI@Z 1000b013 f i cProc_dialog.obj
 0001:0000a013       ??_GContributorListBoxItem@@UAEPAXI@Z 1000b013 f i cProc_dialog.obj
 0001:0000a032       ??_EQDoubleValidator@@UAEPAXI@Z 1000b032 f i cProc_dialog.obj
 0001:0000a032       ??_GQDoubleValidator@@UAEPAXI@Z 1000b032 f i cProc_dialog.obj
 0001:0000a052       ??_EcProc_dialog@@UAEPAXI@Z 1000b052 f i cProc_dialog.obj
 0001:0000a052       ??_GcProc_dialog@@UAEPAXI@Z 1000b052 f i cProc_dialog.obj
 0001:0000a071       ?addTruthColumn@cProc_dialog@@IAEXXZ 1000b071 f   cProc_dialog.obj
 0001:0000a0bf       ?applyProc@cProc_dialog@@QAE_NXZ 1000b0bf f   cProc_dialog.obj
 0001:0000a63c       ?changeFunction@cProc_dialog@@IAEXABVQString@@@Z 1000b63c f   cProc_dialog.obj
 0001:0000a811       ?changeGroup@cProc_dialog@@IAEXABVQString@@@Z 1000b811 f   cProc_dialog.obj
 0001:0000a849       ?changeHoldoff@cProc_dialog@@IAEXABVQString@@@Z 1000b849 f   cProc_dialog.obj
 0001:0000a8a7       ?clear@?$QMapPrivate@HPAVcAcqFileData@@@@QAEXPAU?$QMapNode@HPAVcAcqFileData@@@@@Z 1000b8a7 f i cProc_dialog.obj
 0001:0000a8d6       ?clear@?$QMapPrivate@HPAVcAcqFileData@@@@QAEXXZ 1000b8d6 f i cProc_dialog.obj
 0001:0000a905       ?clear@cProc_dialog@@QAEX_N@Z 1000b905 f   cProc_dialog.obj
 0001:0000aa13       ?copy@?$QMapPrivate@HPAVcAcqFileData@@@@QAEPAU?$QMapNode@HPAVcAcqFileData@@@@PAU2@@Z 1000ba13 f i cProc_dialog.obj
 0001:0000aa87       ?dec@?$QMapIterator@HPAVcAcqFileData@@@@AAEHXZ 1000ba87 f i cProc_dialog.obj
 0001:0000aac6       ?deleteTruthColumn@cProc_dialog@@IAEXXZ 1000bac6 f   cProc_dialog.obj
 0001:0000aaf1       ?detachInternal@?$QMap@HPAVcAcqFileData@@@@AAEXXZ 1000baf1 f i cProc_dialog.obj
 0001:0000ab28       ?editAcqSlot@cProc_dialog@@QAEXXZ 1000bb28 f   cProc_dialog.obj
 0001:0000ac46       ?enableNavigate@cProc_dialog@@IAEXXZ 1000bc46 f   cProc_dialog.obj
 0001:0000ac99       ?enableTruthDeleteCol@cProc_dialog@@IAEXHH@Z 1000bc99 f   cProc_dialog.obj
 0001:0000acbc       ?endTimeChanged@cProc_dialog@@IAEXABVQTime@@@Z 1000bcbc f   cProc_dialog.obj
 0001:0000ad49       ?find@?$QMap@HPAVcAcqFileData@@@@QAE?AV?$QMapIterator@HPAVcAcqFileData@@@@ABH@Z 1000bd49 f i cProc_dialog.obj
 0001:0000ad75       ?find@?$QMapPrivate@HPAVcAcqFileData@@@@QBE?AV?$QMapConstIterator@HPAVcAcqFileData@@@@ABH@Z 1000bd75 f i cProc_dialog.obj
 0001:0000adba       ?inc@?$QMapIterator@HPAVcAcqFileData@@@@AAEHXZ 1000bdba f i cProc_dialog.obj
 0001:0000adba       ?inc@?$QMapIterator@VQString@@H@@AAEHXZ 1000bdba f i cAcqFileData.obj
 0001:0000adeb       ?inputBlockChange@cProc_dialog@@IAEXABVQString@@@Z 1000bdeb f   cProc_dialog.obj
 0001:0000ae9c       ?inputSlotChange@cProc_dialog@@IAEXABVQString@@@Z 1000be9c f   cProc_dialog.obj
 0001:0000afa3       ?insert@?$QMap@HPAVcAcqFileData@@@@QAE?AV?$QMapIterator@HPAVcAcqFileData@@@@ABHABQAVcAcqFileData@@_N@Z 1000bfa3 f i cProc_dialog.obj
 0001:0000afe8       ?insert@?$QMapPrivate@HPAVcAcqFileData@@@@QAE?AV?$QMapIterator@HPAVcAcqFileData@@@@PAUQMapNodeBase@@0ABH@Z 1000bfe8 f i cProc_dialog.obj
 0001:0000b06d       ?insertSingle@?$QMapPrivate@HPAVcAcqFileData@@@@QAE?AV?$QMapIterator@HPAVcAcqFileData@@@@ABH@Z 1000c06d f i cProc_dialog.obj
 0001:0000b0e5       ?isDirty@cProc_dialog@@QBE_NXZ 1000c0e5 f   cProc_dialog.obj
 0001:0000b0ec       ?itemChanged@cProc_dialog@@IAEXHH@Z 1000c0ec f   cProc_dialog.obj
 0001:0000b0fb       ?loadAcqFiles@cProc_dialog@@QAE_NVQString@@@Z 1000c0fb f   cProc_dialog.obj
 0001:0000b491       ?loadOutputModules@cProc_dialog@@QAE_NVQString@@@Z 1000c491 f   cProc_dialog.obj
 0001:0000b86f       ?metaObject@cProc_dialog@@UBEPAVQMetaObject@@XZ 1000c86f f i cProc_dialog.obj
 0001:0000b874       ?navContributesTo@cProc_dialog@@IAEXXZ 1000c874 f   cProc_dialog.obj
 0001:0000b8a4       ?navOutputModule@cProc_dialog@@IAEXXZ 1000c8a4 f   cProc_dialog.obj
 0001:0000b8f6       ?paint@ContributorListBoxItem@@EAEXPAVQPainter@@@Z 1000c8f6 f   cProc_dialog.obj
 0001:0000b9ee       ?reloadInputList@cProc_dialog@@QAEXXZ 1000c9ee f   cProc_dialog.obj
 0001:0000bbb4       ?remove@?$QMap@HPAVcAcqFileData@@@@QAEXABH@Z 1000cbb4 f i cProc_dialog.obj
 0001:0000bc00       ?remove@?$QMapPrivate@HPAVcAcqFileData@@@@QAEXV?$QMapIterator@HPAVcAcqFileData@@@@@Z 1000cc00 f i cProc_dialog.obj
 0001:0000bc2a       ?setMask@cProc_dialog@@QAEXVQString@@@Z 1000cc2a f   cProc_dialog.obj
 0001:0000bd11       ?setProcess@cProc_dialog@@QAEXPAVcProcess@@_N@Z 1000cd11 f   cProc_dialog.obj
 0001:0000c00a       ?setReadOnly@cProc_dialog@@QAEX_N@Z 1000d00a f   cProc_dialog.obj
 0001:0000c05a       ?showAnd@cProc_dialog@@AAEXXZ 1000d05a f   cProc_dialog.obj
 0001:0000c101       ?showHoldoff@cProc_dialog@@AAEXXZ 1000d101 f   cProc_dialog.obj
 0001:0000c1b1       ?showInput@cProc_dialog@@AAEXXZ 1000d1b1 f   cProc_dialog.obj
 0001:0000c386       ?showNot@cProc_dialog@@AAEXXZ 1000d386 f   cProc_dialog.obj
 0001:0000c402       ?showOr@cProc_dialog@@AAEXXZ 1000d402 f   cProc_dialog.obj
 0001:0000c4d7       ?showTime@cProc_dialog@@AAEXXZ 1000d4d7 f   cProc_dialog.obj
 0001:0000c5bc       ?showTruth@cProc_dialog@@AAEXXZ 1000d5bc f   cProc_dialog.obj
 0001:0000c7c8       ?startTimeChanged@cProc_dialog@@IAEXABVQTime@@@Z 1000d7c8 f   cProc_dialog.obj
 0001:0000c855       ?updateProcessCount@cProc_dialog@@QAEXH@Z 1000d855 f   cProc_dialog.obj
 0001:0000c8af       ??0cProcess@@QAE@ABVQString@@@Z 1000d8af f   cProcess.obj
 0001:0000c997       ??1?$QDict@VQString@@@@UAE@XZ 1000d997 f i cProcess.obj
 0001:0000c9ca       ??1cProcess@@UAE@XZ        1000d9ca f   cProcess.obj
 0001:0000ca8b       ??_G?$QDict@VQString@@@@UAEPAXI@Z 1000da8b f i cProcess.obj
 0001:0000ca8b       ??_E?$QDict@VQString@@@@UAEPAXI@Z 1000da8b f i cProcess.obj
 0001:0000caaa       ??_GcProcess@@UAEPAXI@Z    1000daaa f i cProcess.obj
 0001:0000caaa       ??_EcProcess@@UAEPAXI@Z    1000daaa f i cProcess.obj
 0001:0000cac9       ?FindEntry@cProcess@@AAE?AVQString@@AAV?$QDict@VQString@@@@ABV2@@Z 1000dac9 f   cProcess.obj
 0001:0000cb1e       ?Index@cProcess@@AAEXABVQStringList@@AAV?$QDict@VQString@@@@@Z 1000db1e f   cProcess.obj
 0001:0000cc22       ?LoadSettings@cProcess@@QAE_NABVQStringList@@@Z 1000dc22 f   cProcess.obj
 0001:0000d550       ?LoadTruth@cProcess@@AAEHAAV?$QDict@VQString@@@@@Z 1000e550 f   cProcess.obj
 0001:0000d63c       ?_Lbound@?$_Tree@V?$_Tmap_traits@VQString@@PAVcProcess@@U?$less@VQString@@@std@@V?$allocator@U?$pair@$$CBVQString@@PAVcProcess@@@std@@@4@$0A@@std@@@std@@IAEPAU?$_Tree_node@U?$pair@$$CBVQString@@PAVcProcess@@@std@@PAX@2@ABVQString@@@Z 1000e63c f i alm_process.obj
 0001:0000d63c       ?_Lbound@?$_Tree@V?$_Tmap_traits@VQString@@PAVcProcess@@U?$less@VQString@@@std@@V?$allocator@U?$pair@$$CBVQString@@PAVcProcess@@@std@@@4@$0A@@std@@@std@@IBEPAU?$_Tree_node@U?$pair@$$CBVQString@@PAVcProcess@@@std@@PAX@2@ABVQString@@@Z 1000e63c f i cProcess.obj
 0001:0000d672       ?addEntry@cProcess@@AAEXAAVQStringList@@ABVQString@@1@Z 1000e672 f   cProcess.obj
 0001:0000d6ee       ?checkInputs@cProcess@@QAE_N_N0ABV?$map@VQString@@PAVcProcess@@U?$less@VQString@@@std@@V?$allocator@U?$pair@$$CBVQString@@PAVcProcess@@@std@@@4@@std@@@Z 1000e6ee f   cProcess.obj
 0001:0000d77f       ?clear@?$QDict@VQString@@@@UAEXXZ 1000e77f f i cProcess.obj
 0001:0000d785       ?count@?$QDict@VQString@@@@UBEIXZ 1000e785 f i cProcess.obj
 0001:0000d789       ?countOutputs@cProcess@@AAEXABV?$map@VQString@@PAVcProcess@@U?$less@VQString@@@std@@V?$allocator@U?$pair@$$CBVQString@@PAVcProcess@@@std@@@4@@std@@@Z 1000e789 f   cProcess.obj
 0001:0000d89c       ?countProcessOutputs@cProcess@@SAXAAV?$map@VQString@@PAVcProcess@@U?$less@VQString@@@std@@V?$allocator@U?$pair@$$CBVQString@@PAVcProcess@@@std@@@4@@std@@@Z 1000e89c f   cProcess.obj
 0001:0000d951       ?deleteItem@?$QDict@VQString@@@@EAEXPAX@Z 1000e951 f i cProcess.obj
 0001:0000d976       ?find@?$_Tree@V?$_Tmap_traits@VQString@@PAVcProcess@@U?$less@VQString@@@std@@V?$allocator@U?$pair@$$CBVQString@@PAVcProcess@@@std@@@4@$0A@@std@@@std@@QAE?AV?$_Tree_iterator@V?$_Tree_val@U?$_Tree_simple_types@U?$pair@$$CBVQString@@PAVcProcess@@@std@@@std@@@std@@@2@ABVQString@@@Z 1000e976 f i alm_process.obj
 0001:0000d976       ?find@?$_Tree@V?$_Tmap_traits@VQString@@PAVcProcess@@U?$less@VQString@@@std@@V?$allocator@U?$pair@$$CBVQString@@PAVcProcess@@@std@@@4@$0A@@std@@@std@@QBE?AV?$_Tree_const_iterator@V?$_Tree_val@U?$_Tree_simple_types@U?$pair@$$CBVQString@@PAVcProcess@@@std@@@std@@@std@@@2@ABVQString@@@Z 1000e976 f i cProcess.obj
 0001:0000d9b8       ?getName@cProcess@@QBE?AVQString@@XZ 1000e9b8 f   cProcess.obj
 0001:0000d9d6       ?getValid@cProcess@@SA_NABVQString@@@Z 1000e9d6 f   cProcess.obj
 0001:0000da29       ?saveSettings@cProcess@@QAE?AVQStringList@@XZ 1000ea29 f   cProcess.obj
 0001:0000e11e       ?setName@cProcess@@QAE_NABVQString@@@Z 1000f11e f   cProcess.obj
 0001:0000e1ea       ??0multiInputBase@@QAE@PAVQWidget@@PBD_NI@Z 1000f1ea f   multiinput.obj
 0001:0000e989       ??1multiInputBase@@UAE@XZ  1000f989 f   multiinput.obj
 0001:0000e9c9       ??_EQListView@@WCI@AEPAXI@Z 1000f9c9 f i multiinput.obj
 0001:0000e9d1       ??_EmultiInputBase@@WCI@AEPAXI@Z 1000f9d1 f i multiinput.obj
 0001:0000e9d9       ??_EQListView@@UAEPAXI@Z   1000f9d9 f i multiinput.obj
 0001:0000e9d9       ??_GQListView@@UAEPAXI@Z   1000f9d9 f i multiinput.obj
 0001:0000e9f9       ??_EmultiInputBase@@UAEPAXI@Z 1000f9f9 f i multiinput.obj
 0001:0000e9f9       ??_GmultiInputBase@@UAEPAXI@Z 1000f9f9 f i multiinput.obj
 0001:0000ea18       ?languageChange@multiInputBase@@MAEXXZ 1000fa18 f   multiinput.obj
 0001:0000ed66       ?metaObject@multiInputBase@@UBEPAVQMetaObject@@XZ 1000fd66 f i multiinput.obj
 0001:0000ed6b       ??0MultiInputInvalidListViewItem@@QAE@PAVQListView@@ABVQString@@@Z 1000fd6b f   multiinputimpl.obj
 0001:0000ee24       ??0multiInput@@QAE@ABV?$map@VQString@@PAVcProcess@@U?$less@VQString@@@std@@V?$allocator@U?$pair@$$CBVQString@@PAVcProcess@@@std@@@4@@std@@QBVcProcess@@PAVQWidget@@PBD_NI@Z 1000fe24 f   multiinputimpl.obj
 0001:0000f3a8       ??1MultiInputInvalidListViewItem@@UAE@XZ 100103a8 f   multiinputimpl.obj
 0001:0000f3b4       ??1multiInput@@UAE@XZ      100103b4 f   multiinputimpl.obj
 0001:0000f4ec       ??_EmultiInput@@WCI@AEPAXI@Z 100104ec f i multiinputimpl.obj
 0001:0000f4f4       ??_GMultiInputInvalidListViewItem@@UAEPAXI@Z 100104f4 f i multiinputimpl.obj
 0001:0000f4f4       ??_EMultiInputInvalidListViewItem@@UAEPAXI@Z 100104f4 f i multiinputimpl.obj
 0001:0000f513       ??_GmultiInput@@UAEPAXI@Z  10010513 f i multiinputimpl.obj
 0001:0000f513       ??_EmultiInput@@UAEPAXI@Z  10010513 f i multiinputimpl.obj
 0001:0000f532       ?addProcesses@multiInput@@QAEXPAVQListViewItem@@@Z 10010532 f   multiinputimpl.obj
 0001:0000f5bc       ?changeInputs@multiInput@@QAEXQAVcProcess@@@Z 100105bc f   multiinputimpl.obj
 0001:0000f63c       ?enableAdd@multiInput@@QAEXXZ 1001063c f   multiinputimpl.obj
 0001:0000f6a2       ?enableRemove@multiInput@@QAEXXZ 100106a2 f   multiinputimpl.obj
 0001:0000f725       ?filterChange@multiInput@@QAEXABVQString@@@Z 10010725 f   multiinputimpl.obj
 0001:0000f8a8       ?metaObject@multiInput@@UBEPAVQMetaObject@@XZ 100108a8 f i multiinputimpl.obj
 0001:0000f8ad       ?paintCell@MultiInputInvalidListViewItem@@EAEXPAVQPainter@@ABVQColorGroup@@HHH@Z 100108ad f   multiinputimpl.obj
 0001:0000f976       ?removeProcesses@multiInput@@QAEXPAVQListViewItem@@@Z 10010976 f   multiinputimpl.obj
 0001:0000fa1b       ?resizeEvent@multiInput@@MAEXPAVQResizeEvent@@@Z 10010a1b f   multiinputimpl.obj
 0001:0000fa3c       ??_Eplugindesc@@UAEPAXI@Z  10010a3c f i plugindesc.obj
 0001:0000fa3c       ??_Gconfig_plugin_desc_base@@UAEPAXI@Z 10010a3c f i plugindesc.obj
 0001:0000fa3c       ??_Gplugindesc@@UAEPAXI@Z  10010a3c f i plugindesc.obj
 0001:0000fa3c       ??_Econfig_plugin_desc_base@@UAEPAXI@Z 10010a3c f i plugindesc.obj
 0001:0000fa5c       ?create@plugindesc@@UAEPAVconfig_plugin_base@@ABVQString@@00@Z 10010a5c f   plugindesc.obj
 0001:0000fa97       ?keys@plugindesc@@UAE?AVQStringList@@ABVQString@@0@Z 10010a97 f   plugindesc.obj
 0001:0000faf2       ?pixmap@plugindesc@@UAE?AVQPixmap@@ABVQString@@@Z 10010af2 f   plugindesc.obj
 0001:0000fb11       _load_bncs_config_plugin_desc 10010b11 f   plugindesc.obj
 0001:0000fb27       ??0singleInputBase@@QAE@PAVQWidget@@PBD_NI@Z 10010b27 f   singleinput.obj
 0001:0000ff7c       ??1singleInputBase@@UAE@XZ 10010f7c f   singleinput.obj
 0001:0000ff8f       ??_EsingleInputBase@@WCI@AEPAXI@Z 10010f8f f i singleinput.obj
 0001:0000ff97       ??_GsingleInputBase@@UAEPAXI@Z 10010f97 f i singleinput.obj
 0001:0000ff97       ??_EsingleInputBase@@UAEPAXI@Z 10010f97 f i singleinput.obj
 0001:0000ffb6       ?languageChange@singleInputBase@@MAEXXZ 10010fb6 f   singleinput.obj
 0001:00010140       ?metaObject@singleInputBase@@UBEPAVQMetaObject@@XZ 10011140 f i singleinput.obj
 0001:00010145       ??0singleInput@@QAE@ABV?$map@VQString@@PAVcProcess@@U?$less@VQString@@@std@@V?$allocator@U?$pair@$$CBVQString@@PAVcProcess@@@std@@@4@@std@@QBVcProcess@@W4ESingleType@0@PAVQWidget@@PBD_NI@Z 10011145 f   singleinputimpl.obj
 0001:00010527       ??1singleInput@@UAE@XZ     10011527 f   singleinputimpl.obj
 0001:00010539       ??_EsingleInput@@WCI@AEPAXI@Z 10011539 f i singleinputimpl.obj
 0001:00010541       ??_GsingleInput@@UAEPAXI@Z 10011541 f i singleinputimpl.obj
 0001:00010541       ??_EsingleInput@@UAEPAXI@Z 10011541 f i singleinputimpl.obj
 0001:00010560       ?changeInputs@singleInput@@QAE_NQAVcProcess@@@Z 10011560 f   singleinputimpl.obj
 0001:000105d0       ?changeMask@singleInput@@QAE_NPAVcProc_dialog@@@Z 100115d0 f   singleinputimpl.obj
 0001:00010605       ?clearFilter@singleInput@@AAEXXZ 10011605 f   singleinputimpl.obj
 0001:00010610       ?filterChange@singleInput@@AAEXABVQString@@@Z 10011610 f   singleinputimpl.obj
 0001:0001070a       ?metaObject@singleInput@@UBEPAVQMetaObject@@XZ 1001170a f i singleinputimpl.obj
 0001:0001070f       ?selectinChanged@singleInput@@QAEXPAVQListViewItem@@@Z 1001170f f   singleinputimpl.obj
 0001:0001071f       ??0template_dialogBase@@QAE@PAVQWidget@@PBD_NI@Z 1001171f f   template_dialog.obj
 0001:00011470       ??1template_dialogBase@@UAE@XZ 10012470 f   template_dialog.obj
 0001:00011483       ??_EQButtonGroup@@WCI@AEPAXI@Z 10012483 f i template_dialog.obj
 0001:0001148b       ??_EQGridLayout@@WCI@AEPAXI@Z 1001248b f i template_dialog.obj
 0001:00011493       ??_EQCheckBox@@WCI@AEPAXI@Z 10012493 f i template_dialog.obj
 0001:00011493       ??_EQRadioButton@@WCI@AEPAXI@Z 10012493 f i template_dialog.obj
 0001:0001149b       ??_EQSpinBox@@WCI@AEPAXI@Z 1001249b f i template_dialog.obj
 0001:000114a3       ??_EQSpinBox@@WGM@AEPAXI@Z 100124a3 f i template_dialog.obj
 0001:000114ab       ??_Etemplate_dialogBase@@WCI@AEPAXI@Z 100124ab f i template_dialog.obj
 0001:000114b3       ??_GQButtonGroup@@UAEPAXI@Z 100124b3 f i template_dialog.obj
 0001:000114b3       ??_EQButtonGroup@@UAEPAXI@Z 100124b3 f i template_dialog.obj
 0001:000114d3       ??_GQGridLayout@@UAEPAXI@Z 100124d3 f i template_dialog.obj
 0001:000114d3       ??_EQGridLayout@@UAEPAXI@Z 100124d3 f i template_dialog.obj
 0001:000114f3       ??_EQCheckBox@@UAEPAXI@Z   100124f3 f i template_dialog.obj
 0001:000114f3       ??_EQRadioButton@@UAEPAXI@Z 100124f3 f i template_dialog.obj
 0001:000114f3       ??_GQCheckBox@@UAEPAXI@Z   100124f3 f i template_dialog.obj
 0001:000114f3       ??_GQRadioButton@@UAEPAXI@Z 100124f3 f i template_dialog.obj
 0001:00011513       ??_EQSpinBox@@UAEPAXI@Z    10012513 f i template_dialog.obj
 0001:00011513       ??_GQSpinBox@@UAEPAXI@Z    10012513 f i template_dialog.obj
 0001:00011533       ??_Gtemplate_dialogBase@@UAEPAXI@Z 10012533 f i template_dialog.obj
 0001:00011533       ??_Etemplate_dialogBase@@UAEPAXI@Z 10012533 f i template_dialog.obj
 0001:00011552       ?languageChange@template_dialogBase@@MAEXXZ 10012552 f   template_dialog.obj
 0001:000119b8       ?metaObject@template_dialogBase@@UBEPAVQMetaObject@@XZ 100129b8 f i template_dialog.obj
 0001:000119bd       ??$make_pair@AAVQString@@AAPAVcProcess@@@std@@YA?AU?$pair@VQString@@PAVcProcess@@@0@AAVQString@@AAPAVcProcess@@@Z 100129bd f i template_dialogimpl.obj
 0001:000119e3       ??0template_dialog@@QAE@ABV?$QPtrList@VcProcess@@@@ABVQStringList@@PAVQWidget@@PBD_NI@Z 100129e3 f   template_dialogimpl.obj
 0001:00011be0       ??1?$QPtrListIterator@VcProcess@@@@QAE@XZ 10012be0 f i template_dialogimpl.obj
 0001:00011be6       ??1template_dialog@@UAE@XZ 10012be6 f   template_dialogimpl.obj
 0001:00011bf8       ??_Etemplate_dialog@@WCI@AEPAXI@Z 10012bf8 f i template_dialogimpl.obj
 0001:00011c00       ??_Gtemplate_dialog@@UAEPAXI@Z 10012c00 f i template_dialogimpl.obj
 0001:00011c00       ??_Etemplate_dialog@@UAEPAXI@Z 10012c00 f i template_dialogimpl.obj
 0001:00011c1f       ?copyProcesses@template_dialog@@QAEXAAV?$QPtrList@VcProcess@@@@AAV?$map@VQString@@PAVcProcess@@U?$less@VQString@@@std@@V?$allocator@U?$pair@$$CBVQString@@PAVcProcess@@@std@@@4@@std@@PAVQListView@@@Z 10012c1f f   template_dialogimpl.obj
 0001:00012086       ?getThisPrefix@template_dialog@@QAE?AVQString@@H@Z 10013086 f   template_dialogimpl.obj
 0001:00012210       ?metaObject@template_dialog@@UBEPAVQMetaObject@@XZ 10013210 f i template_dialogimpl.obj
 0001:00012215       ?numCopies@template_dialog@@QAEXH@Z 10013215 f   template_dialogimpl.obj
 0001:0001225d       ?oldPrefixChanged@template_dialog@@QAEXABVQString@@@Z 1001325d f   template_dialogimpl.obj
 0001:00012265       ?setOldPrefix@template_dialog@@QAEXVQString@@@Z 10013265 f   template_dialogimpl.obj
 0001:000122b7       ?setSelectionData@template_dialog@@AAEXHQBVcProcess@@@Z 100132b7 f   template_dialogimpl.obj
 0001:00012336       ?showExample@template_dialog@@QAEXXZ 10013336 f   template_dialogimpl.obj
 0001:00012475       ??0CheckContDialogBase@@QAE@PAVQWidget@@PBD_NI@Z 10013475 f   checkcontributiondialog.obj
 0001:000130ab       ??1CheckContDialogBase@@UAE@XZ 100140ab f   checkcontributiondialog.obj
 0001:000130be       ??_ECheckContDialogBase@@WCI@AEPAXI@Z 100140be f i checkcontributiondialog.obj
 0001:000130c6       ??_GCheckContDialogBase@@UAEPAXI@Z 100140c6 f i checkcontributiondialog.obj
 0001:000130c6       ??_ECheckContDialogBase@@UAEPAXI@Z 100140c6 f i checkcontributiondialog.obj
 0001:000130e5       ?languageChange@CheckContDialogBase@@MAEXXZ 100140e5 f   checkcontributiondialog.obj
 0001:00013447       ?metaObject@CheckContDialogBase@@UBEPAVQMetaObject@@XZ 10014447 f i checkcontributiondialog.obj
 0001:0001344c       ?rbContribDiag_clicked@CheckContDialogBase@@UAEXXZ 1001444c f   checkcontributiondialog.obj
 0001:00013459       ?rbInputDiag_clicked@CheckContDialogBase@@UAEXXZ 10014459 f   checkcontributiondialog.obj
 0001:00013466       ??0LatchAckDialogBase@@QAE@PAVQWidget@@PBD_NI@Z 10014466 f   latchackdialog.obj
 0001:00013822       ??1LatchAckDialogBase@@UAE@XZ 10014822 f   latchackdialog.obj
 0001:00013835       ??_ELatchAckDialogBase@@WCI@AEPAXI@Z 10014835 f i latchackdialog.obj
 0001:0001383d       ??_GLatchAckDialogBase@@UAEPAXI@Z 1001483d f i latchackdialog.obj
 0001:0001383d       ??_ELatchAckDialogBase@@UAEPAXI@Z 1001483d f i latchackdialog.obj
 0001:0001385c       ?languageChange@LatchAckDialogBase@@MAEXXZ 1001485c f   latchackdialog.obj
 0001:00013a4c       ?metaObject@LatchAckDialogBase@@UBEPAVQMetaObject@@XZ 10014a4c f i latchackdialog.obj
 0001:00013a51       ??0LatchAckDialog@@QAE@PAVQWidget@@PBD_NI@Z 10014a51 f   latchackdialogimpl.obj
 0001:00013a7c       ??1LatchAckDialog@@UAE@XZ  10014a7c f   latchackdialogimpl.obj
 0001:00013a8e       ??_ELatchAckDialog@@WCI@AEPAXI@Z 10014a8e f i latchackdialogimpl.obj
 0001:00013a96       ??_ELatchAckDialog@@UAEPAXI@Z 10014a96 f i latchackdialogimpl.obj
 0001:00013a96       ??_GLatchAckDialog@@UAEPAXI@Z 10014a96 f i latchackdialogimpl.obj
 0001:00013ab5       ?metaObject@LatchAckDialog@@UBEPAVQMetaObject@@XZ 10014ab5 f i latchackdialogimpl.obj
 0001:00013aba       ?className@alm_process@@UBEPBDXZ 10014aba f   moc_alm_process.obj
 0001:00013ac0       ?command@alm_process@@IAEXVQString@@0@Z 10014ac0 f   moc_alm_process.obj
 0001:00013b80       ?qt_cast@alm_process@@UAEPAXPBD@Z 10014b80 f   moc_alm_process.obj
 0001:00013bae       ?qt_emit@alm_process@@UAE_NHPAUQUObject@@@Z 10014bae f   moc_alm_process.obj
 0001:00013c12       ?qt_invoke@alm_process@@UAE_NHPAUQUObject@@@Z 10014c12 f   moc_alm_process.obj
 0001:00013ece       ?staticMetaObject@alm_process@@SAPAVQMetaObject@@XZ 10014ece f   moc_alm_process.obj
 0001:000141c4       ?className@CheckContDialog@@UBEPBDXZ 100151c4 f   moc_checkContDialogImpl.obj
 0001:000141ca       ?qt_cast@CheckContDialog@@UAEPAXPBD@Z 100151ca f   moc_checkContDialogImpl.obj
 0001:000141f7       ?qt_invoke@CheckContDialog@@UAE_NHPAUQUObject@@@Z 100151f7 f   moc_checkContDialogImpl.obj
 0001:00014249       ?staticMetaObject@CheckContDialog@@SAPAVQMetaObject@@XZ 10015249 f   moc_checkContDialogImpl.obj
 0001:00014292       ?className@CheckContDialogBase@@UBEPBDXZ 10015292 f   moc_checkcontributiondialog.obj
 0001:00014298       ?qt_cast@CheckContDialogBase@@UAEPAXPBD@Z 10015298 f   moc_checkcontributiondialog.obj
 0001:000142c6       ?qt_invoke@CheckContDialogBase@@UAE_NHPAUQUObject@@@Z 100152c6 f   moc_checkcontributiondialog.obj
 0001:00014319       ?staticMetaObject@CheckContDialogBase@@SAPAVQMetaObject@@XZ 10015319 f   moc_checkcontributiondialog.obj
 0001:00014363       ?tr@CheckContDialogBase@@SA?AVQString@@PBD0@Z 10015363 f   moc_checkcontributiondialog.obj
 0001:000143a6       ?className@cProc_dialog@@UBEPBDXZ 100153a6 f   moc_cProc_dialog.obj
 0001:000143ac       ?itemsChanged@cProc_dialog@@IAEXXZ 100153ac f   moc_cProc_dialog.obj
 0001:000143c3       ?navToAck@cProc_dialog@@IAEXVQString@@00@Z 100153c3 f   moc_cProc_dialog.obj
 0001:000144a6       ?navToOutput@cProc_dialog@@IAEXVQString@@0@Z 100154a6 f   moc_cProc_dialog.obj
 0001:0001456e       ?navToProc@cProc_dialog@@IAEXVQString@@@Z 1001556e f   moc_cProc_dialog.obj
 0001:000145c1       ?qt_cast@cProc_dialog@@UAEPAXPBD@Z 100155c1 f   moc_cProc_dialog.obj
 0001:000145ee       ?qt_emit@cProc_dialog@@UAE_NHPAUQUObject@@@Z 100155ee f   moc_cProc_dialog.obj
 0001:000146da       ?qt_invoke@cProc_dialog@@UAE_NHPAUQUObject@@@Z 100156da f   moc_cProc_dialog.obj
 0001:00014866       ?qt_property@cProc_dialog@@UAE_NHHPAVQVariant@@@Z 10015866 f   moc_cProc_dialog.obj
 0001:0001486f       ?staticMetaObject@cProc_dialog@@SAPAVQMetaObject@@XZ 1001586f f   moc_cProc_dialog.obj
 0001:00014b80       ?updateProc@cProc_dialog@@IAEXPAVcProcess@@@Z 10015b80 f   moc_cProc_dialog.obj
 0001:00014c0b       ?className@LatchAckDialogBase@@UBEPBDXZ 10015c0b f   moc_latchackdialog.obj
 0001:00014c11       ?qt_cast@LatchAckDialogBase@@UAEPAXPBD@Z 10015c11 f   moc_latchackdialog.obj
 0001:00014c3f       ?qt_invoke@LatchAckDialogBase@@UAE_NHPAUQUObject@@@Z 10015c3f f   moc_latchackdialog.obj
 0001:00014c71       ?staticMetaObject@LatchAckDialogBase@@SAPAVQMetaObject@@XZ 10015c71 f   moc_latchackdialog.obj
 0001:00014cbb       ?tr@LatchAckDialogBase@@SA?AVQString@@PBD0@Z 10015cbb f   moc_latchackdialog.obj
 0001:00014cfe       ?className@LatchAckDialog@@UBEPBDXZ 10015cfe f   moc_latchackdialogimpl.obj
 0001:00014d04       ?qt_cast@LatchAckDialog@@UAEPAXPBD@Z 10015d04 f   moc_latchackdialogimpl.obj
 0001:00014d31       ?qt_invoke@LatchAckDialog@@UAE_NHPAUQUObject@@@Z 10015d31 f   moc_latchackdialogimpl.obj
 0001:00014d3a       ?qt_property@LatchAckDialog@@UAE_NHHPAVQVariant@@@Z 10015d3a f   moc_latchackdialogimpl.obj
 0001:00014d3a       ?qt_property@CheckContDialog@@UAE_NHHPAVQVariant@@@Z 10015d3a f   moc_checkContDialogImpl.obj
 0001:00014d3a       ?qt_property@multiInput@@UAE_NHHPAVQVariant@@@Z 10015d3a f   moc_multiinputimpl.obj
 0001:00014d3a       ?qt_property@singleInput@@UAE_NHHPAVQVariant@@@Z 10015d3a f   moc_singleinputimpl.obj
 0001:00014d3a       ?qt_property@template_dialog@@UAE_NHHPAVQVariant@@@Z 10015d3a f   moc_template_dialogimpl.obj
 0001:00014d43       ?staticMetaObject@LatchAckDialog@@SAPAVQMetaObject@@XZ 10015d43 f   moc_latchackdialogimpl.obj
 0001:00014d87       ?className@multiInputBase@@UBEPBDXZ 10015d87 f   moc_multiinput.obj
 0001:00014d8d       ?qt_cast@multiInputBase@@UAEPAXPBD@Z 10015d8d f   moc_multiinput.obj
 0001:00014dbb       ?qt_invoke@multiInputBase@@UAE_NHPAUQUObject@@@Z 10015dbb f   moc_multiinput.obj
 0001:00014ded       ?staticMetaObject@multiInputBase@@SAPAVQMetaObject@@XZ 10015ded f   moc_multiinput.obj
 0001:00014e37       ?tr@multiInputBase@@SA?AVQString@@PBD0@Z 10015e37 f   moc_multiinput.obj
 0001:00014e7a       ?className@multiInput@@UBEPBDXZ 10015e7a f   moc_multiinputimpl.obj
 0001:00014e80       ?qt_cast@multiInput@@UAEPAXPBD@Z 10015e80 f   moc_multiinputimpl.obj
 0001:00014ead       ?qt_invoke@multiInput@@UAE_NHPAUQUObject@@@Z 10015ead f   moc_multiinputimpl.obj
 0001:00014f2d       ?staticMetaObject@multiInput@@SAPAVQMetaObject@@XZ 10015f2d f   moc_multiinputimpl.obj
 0001:00014ff5       ?className@proc_config@@UBEPBDXZ 10015ff5 f   moc_proc_config.obj
 0001:00014ffb       ?qt_cast@proc_config@@UAEPAXPBD@Z 10015ffb f   moc_proc_config.obj
 0001:00015029       ?qt_emit@proc_config@@UAE_NHPAUQUObject@@@Z 10016029 f   moc_proc_config.obj
 0001:00015033       ?qt_invoke@proc_config@@UAE_NHPAUQUObject@@@Z 10016033 f   moc_proc_config.obj
 0001:00015065       ?qt_property@alm_process@@UAE_NHHPAVQVariant@@@Z 10016065 f   moc_alm_process.obj
 0001:00015065       ?qt_property@proc_config@@UAE_NHHPAVQVariant@@@Z 10016065 f   moc_proc_config.obj
 0001:0001506f       ?staticMetaObject@proc_config@@SAPAVQMetaObject@@XZ 1001606f f   moc_proc_config.obj
 0001:000150b9       ?tr@proc_config@@SA?AVQString@@PBD0@Z 100160b9 f   moc_proc_config.obj
 0001:000150fc       ?className@singleInputBase@@UBEPBDXZ 100160fc f   moc_singleinput.obj
 0001:00015102       ?qt_cast@singleInputBase@@UAEPAXPBD@Z 10016102 f   moc_singleinput.obj
 0001:00015130       ?qt_invoke@singleInputBase@@UAE_NHPAUQUObject@@@Z 10016130 f   moc_singleinput.obj
 0001:00015162       ?staticMetaObject@singleInputBase@@SAPAVQMetaObject@@XZ 10016162 f   moc_singleinput.obj
 0001:000151ac       ?tr@singleInputBase@@SA?AVQString@@PBD0@Z 100161ac f   moc_singleinput.obj
 0001:000151ef       ?className@singleInput@@UBEPBDXZ 100161ef f   moc_singleinputimpl.obj
 0001:000151f5       ?qt_cast@singleInput@@UAEPAXPBD@Z 100161f5 f   moc_singleinputimpl.obj
 0001:00015222       ?qt_invoke@singleInput@@UAE_NHPAUQUObject@@@Z 10016222 f   moc_singleinputimpl.obj
 0001:00015273       ?staticMetaObject@singleInput@@SAPAVQMetaObject@@XZ 10016273 f   moc_singleinputimpl.obj
 0001:0001531c       ?className@template_dialogBase@@UBEPBDXZ 1001631c f   moc_template_dialog.obj
 0001:00015322       ?qt_cast@template_dialogBase@@UAEPAXPBD@Z 10016322 f   moc_template_dialog.obj
 0001:00015350       ?qt_invoke@template_dialogBase@@UAE_NHPAUQUObject@@@Z 10016350 f   moc_template_dialog.obj
 0001:00015382       ?staticMetaObject@template_dialogBase@@SAPAVQMetaObject@@XZ 10016382 f   moc_template_dialog.obj
 0001:000153cc       ?tr@template_dialogBase@@SA?AVQString@@PBD0@Z 100163cc f   moc_template_dialog.obj
 0001:0001540f       ?className@template_dialog@@UBEPBDXZ 1001640f f   moc_template_dialogimpl.obj
 0001:00015415       ?qt_cast@template_dialog@@UAEPAXPBD@Z 10016415 f   moc_template_dialogimpl.obj
 0001:00015442       ?qt_emit@multiInput@@UAE_NHPAUQUObject@@@Z 10016442 f   moc_multiinputimpl.obj
 0001:00015442       ?qt_emit@singleInput@@UAE_NHPAUQUObject@@@Z 10016442 f   moc_singleinputimpl.obj
 0001:00015442       ?qt_emit@template_dialog@@UAE_NHPAUQUObject@@@Z 10016442 f   moc_template_dialogimpl.obj
 0001:00015442       ?qt_emit@CheckContDialog@@UAE_NHPAUQUObject@@@Z 10016442 f   moc_checkContDialogImpl.obj
 0001:00015442       ?qt_emit@LatchAckDialog@@UAE_NHPAUQUObject@@@Z 10016442 f   moc_latchackdialogimpl.obj
 0001:0001544b       ?qt_invoke@template_dialog@@UAE_NHPAUQUObject@@@Z 1001644b f   moc_template_dialogimpl.obj
 0001:0001549c       ?staticMetaObject@template_dialog@@SAPAVQMetaObject@@XZ 1001649c f   moc_template_dialogimpl.obj
 0001:00015542       ??0proc_config@@QAE@PAVQWidget@@PBDI@Z 10016542 f   proc_config.obj
 0001:000184b2       ??1proc_config@@UAE@XZ     100194b2 f   proc_config.obj
 0001:00018505       ??_EQComboBox@@WCI@AEPAXI@Z 10019505 f i proc_config.obj
 0001:0001850d       ??_EQGroupBox@@WCI@AEPAXI@Z 1001950d f i proc_config.obj
 0001:00018515       ??_EQListBox@@WCI@AEPAXI@Z 10019515 f i proc_config.obj
 0001:0001851d       ??_EQSplitter@@WCI@AEPAXI@Z 1001951d f i proc_config.obj
 0001:00018525       ??_EQTextEdit@@WCI@AEPAXI@Z 10019525 f i proc_config.obj
 0001:0001852d       ??_EQTimeEdit@@WCI@AEPAXI@Z 1001952d f i proc_config.obj
 0001:00018535       ??_EQWidgetStack@@WCI@AEPAXI@Z 10019535 f i proc_config.obj
 0001:0001853d       ??_Eproc_config@@WCI@AEPAXI@Z 1001953d f i proc_config.obj
 0001:00018545       ??_EQComboBox@@UAEPAXI@Z   10019545 f i proc_config.obj
 0001:00018545       ??_GQComboBox@@UAEPAXI@Z   10019545 f i proc_config.obj
 0001:00018565       ??_EQGroupBox@@UAEPAXI@Z   10019565 f i proc_config.obj
 0001:00018565       ??_GQGroupBox@@UAEPAXI@Z   10019565 f i proc_config.obj
 0001:00018585       ??_GQListBox@@UAEPAXI@Z    10019585 f i proc_config.obj
 0001:00018585       ??_EQListBox@@UAEPAXI@Z    10019585 f i proc_config.obj
 0001:000185a5       ??_GQSplitter@@UAEPAXI@Z   100195a5 f i proc_config.obj
 0001:000185a5       ??_EQSplitter@@UAEPAXI@Z   100195a5 f i proc_config.obj
 0001:000185c5       ??_EQTextEdit@@UAEPAXI@Z   100195c5 f i proc_config.obj
 0001:000185c5       ??_GQTextEdit@@UAEPAXI@Z   100195c5 f i proc_config.obj
 0001:000185e5       ??_EQTimeEdit@@UAEPAXI@Z   100195e5 f i proc_config.obj
 0001:000185e5       ??_GQTimeEdit@@UAEPAXI@Z   100195e5 f i proc_config.obj
 0001:00018605       ??_GQWidgetStack@@UAEPAXI@Z 10019605 f i proc_config.obj
 0001:00018605       ??_EQWidgetStack@@UAEPAXI@Z 10019605 f i proc_config.obj
 0001:00018625       ??_Eproc_config@@UAEPAXI@Z 10019625 f i proc_config.obj
 0001:00018625       ??_Gproc_config@@UAEPAXI@Z 10019625 f i proc_config.obj
 0001:00018644       ?languageChange@proc_config@@MAEXXZ 10019644 f   proc_config.obj
 0001:00019833       ?metaObject@proc_config@@UBEPAVQMetaObject@@XZ 1001a833 f i proc_config.obj
 0001:00019838       ?setName@QWidget@@UAEXPBD@Z 1001a838 f   qt-mt323:qt-mt323.dll
 0001:0001983e       ?setCaption@QWidget@@UAEXABVQString@@@Z 1001a83e f   qt-mt323:qt-mt323.dll
 0001:00019844       ?setFocusPolicy@QWidget@@UAEXW4FocusPolicy@1@@Z 1001a844 f   qt-mt323:qt-mt323.dll
 0001:0001984a       ?text@QListViewItem@@UBE?AVQString@@H@Z 1001a84a f   qt-mt323:qt-mt323.dll
 0001:00019850       ?paintCell@QListViewItem@@UAEXPAVQPainter@@ABVQColorGroup@@HHH@Z 1001a850 f   qt-mt323:qt-mt323.dll
 0001:00019856       ?setRenameEnabled@QListViewItem@@UAEXH_N@Z 1001a856 f   qt-mt323:qt-mt323.dll
 0001:0001985c       ?keyPressEvent@QListView@@MAEXPAVQKeyEvent@@@Z 1001a85c f   qt-mt323:qt-mt323.dll
 0001:00019862       ?acceptDrop@QListViewItem@@UBE_NPBVQMimeSource@@@Z 1001a862 f   qt-mt323:qt-mt323.dll
 0001:00019868       ?activate@QListViewItem@@MAEXXZ 1001a868 f   qt-mt323:qt-mt323.dll
 0001:0001986e       ?activateItemAt@QPopupMenu@@UAEXH@Z 1001a86e f   qt-mt323:qt-mt323.dll
 0001:00019874       ?addChild@QScrollView@@UAEXPAVQWidget@@HH@Z 1001a874 f   qt-mt323:qt-mt323.dll
 0001:0001987a       ?addColumn@QListView@@UAEHABVQIconSet@@ABVQString@@H@Z 1001a87a f   qt-mt323:qt-mt323.dll
 0001:00019880       ?addColumn@QListView@@UAEHABVQString@@H@Z 1001a880 f   qt-mt323:qt-mt323.dll
 0001:00019886       ?addItem@QBoxLayout@@UAEXPAVQLayoutItem@@@Z 1001a886 f   qt-mt323:qt-mt323.dll
 0001:0001988c       ?addTab@QTabWidget@@UAEXPAVQWidget@@ABVQIconSet@@ABVQString@@@Z 1001a88c f   qt-mt323:qt-mt323.dll
 0001:00019892       ?addTab@QTabWidget@@UAEXPAVQWidget@@ABVQString@@@Z 1001a892 f   qt-mt323:qt-mt323.dll
 0001:00019898       ?addTab@QTabWidget@@UAEXPAVQWidget@@PAVQTab@@@Z 1001a898 f   qt-mt323:qt-mt323.dll
 0001:0001989e       ?addTo@QAction@@UAE_NPAVQWidget@@@Z 1001a89e f   qt-mt323:qt-mt323.dll
 0001:000198a4       ?addedTo@QAction@@MAEXHPAVQPopupMenu@@@Z 1001a8a4 f   qt-mt323:qt-mt323.dll
 0001:000198aa       ?addedTo@QAction@@MAEXPAVQWidget@@0@Z 1001a8aa f   qt-mt323:qt-mt323.dll
 0001:000198b0       ?adjustSize@QWidget@@UAEXXZ 1001a8b0 f   qt-mt323:qt-mt323.dll
 0001:000198b6       ?cancelRename@QListViewItem@@MAEXH@Z 1001a8b6 f   qt-mt323:qt-mt323.dll
 0001:000198bc       ?checkConnectArgs@QObject@@MAE_NPBDPBV1@0@Z 1001a8bc f   qt-mt323:qt-mt323.dll
 0001:000198c2       ?childEvent@QLayout@@MAEXPAVQChildEvent@@@Z 1001a8c2 f   qt-mt323:qt-mt323.dll
 0001:000198c8       ?childEvent@QObject@@MAEXPAVQChildEvent@@@Z 1001a8c8 f   qt-mt323:qt-mt323.dll
 0001:000198ce       ?className@QAction@@UBEPBDXZ 1001a8ce f   qt-mt323:qt-mt323.dll
 0001:000198d4       ?className@QDockWindow@@UBEPBDXZ 1001a8d4 f   qt-mt323:qt-mt323.dll
 0001:000198da       ?className@QGuardedPtrPrivate@@UBEPBDXZ 1001a8da f   qt-mt323:qt-mt323.dll
 0001:000198e0       ?className@QHBoxLayout@@UBEPBDXZ 1001a8e0 f   qt-mt323:qt-mt323.dll
 0001:000198e6       ?className@QLabel@@UBEPBDXZ 1001a8e6 f   qt-mt323:qt-mt323.dll
 0001:000198ec       ?className@QLineEdit@@UBEPBDXZ 1001a8ec f   qt-mt323:qt-mt323.dll
 0001:000198f2       ?className@QListView@@UBEPBDXZ 1001a8f2 f   qt-mt323:qt-mt323.dll
 0001:000198f8       ?className@QPopupMenu@@UBEPBDXZ 1001a8f8 f   qt-mt323:qt-mt323.dll
 0001:000198fe       ?className@QPushButton@@UBEPBDXZ 1001a8fe f   qt-mt323:qt-mt323.dll
 0001:00019904       ?className@QTabWidget@@UBEPBDXZ 1001a904 f   qt-mt323:qt-mt323.dll
 0001:0001990a       ?className@QToolBar@@UBEPBDXZ 1001a90a f   qt-mt323:qt-mt323.dll
 0001:00019910       ?className@QVBoxLayout@@UBEPBDXZ 1001a910 f   qt-mt323:qt-mt323.dll
 0001:00019916       ?className@QWidget@@UBEPBDXZ 1001a916 f   qt-mt323:qt-mt323.dll
 0001:0001991c       ?clear@?$QPtrList@VQDockWindow@@@@UAEXXZ 1001a91c f   qt-mt323:qt-mt323.dll
 0001:00019922       ?clear@QLineEdit@@UAEXXZ   1001a922 f   qt-mt323:qt-mt323.dll
 0001:00019928       ?clear@QListView@@UAEXXZ   1001a928 f   qt-mt323:qt-mt323.dll
 0001:0001992e       ?clear@QToolBar@@UAEXXZ    1001a92e f   qt-mt323:qt-mt323.dll
 0001:00019934       ?clearSelection@QListView@@UAEXXZ 1001a934 f   qt-mt323:qt-mt323.dll
 0001:0001993a       ?clearValidator@QLineEdit@@UAEXXZ 1001a93a f   qt-mt323:qt-mt323.dll
 0001:00019940       ?close@QWidget@@UAE_N_N@Z  1001a940 f   qt-mt323:qt-mt323.dll
 0001:00019946       ?closeEvent@QPopupMenu@@MAEXPAVQCloseEvent@@@Z 1001a946 f   qt-mt323:qt-mt323.dll
 0001:0001994c       ?closeEvent@QWidget@@MAEXPAVQCloseEvent@@@Z 1001a94c f   qt-mt323:qt-mt323.dll
 0001:00019952       ?cmd@QPaintDevice@@MAE_NHPAVQPainter@@PATQPDevCmdParam@@@Z 1001a952 f   qt-mt323:qt-mt323.dll
 0001:00019958       ?compare@QListViewItem@@UBEHPAV1@H_N@Z 1001a958 f   qt-mt323:qt-mt323.dll
 0001:0001995e       ?compareItems@QGList@@MAEHPAX0@Z 1001a95e f   qt-mt323:qt-mt323.dll
 0001:00019964       ?connectNotify@QObject@@MAEXPBD@Z 1001a964 f   qt-mt323:qt-mt323.dll
 0001:0001996a       ?contentsContextMenuEvent@QListView@@MAEXPAVQContextMenuEvent@@@Z 1001a96a f   qt-mt323:qt-mt323.dll
 0001:00019970       ?contentsDragEnterEvent@QListView@@MAEXPAVQDragEnterEvent@@@Z 1001a970 f   qt-mt323:qt-mt323.dll
 0001:00019976       ?contentsDragLeaveEvent@QListView@@MAEXPAVQDragLeaveEvent@@@Z 1001a976 f   qt-mt323:qt-mt323.dll
 0001:0001997c       ?contentsDragMoveEvent@QListView@@MAEXPAVQDragMoveEvent@@@Z 1001a97c f   qt-mt323:qt-mt323.dll
 0001:00019982       ?contentsDropEvent@QListView@@MAEXPAVQDropEvent@@@Z 1001a982 f   qt-mt323:qt-mt323.dll
 0001:00019988       ?contentsMouseDoubleClickEvent@QListView@@MAEXPAVQMouseEvent@@@Z 1001a988 f   qt-mt323:qt-mt323.dll
 0001:0001998e       ?contentsMouseMoveEvent@QListView@@MAEXPAVQMouseEvent@@@Z 1001a98e f   qt-mt323:qt-mt323.dll
 0001:00019994       ?contentsMousePressEvent@QListView@@MAEXPAVQMouseEvent@@@Z 1001a994 f   qt-mt323:qt-mt323.dll
 0001:0001999a       ?contentsMouseReleaseEvent@QListView@@MAEXPAVQMouseEvent@@@Z 1001a99a f   qt-mt323:qt-mt323.dll
 0001:000199a0       ?contentsWheelEvent@QScrollView@@MAEXPAVQWheelEvent@@@Z 1001a9a0 f   qt-mt323:qt-mt323.dll
 0001:000199a6       ?contextMenuEvent@QDockWindow@@MAEXPAVQContextMenuEvent@@@Z 1001a9a6 f   qt-mt323:qt-mt323.dll
 0001:000199ac       ?contextMenuEvent@QLineEdit@@MAEXPAVQContextMenuEvent@@@Z 1001a9ac f   qt-mt323:qt-mt323.dll
 0001:000199b2       ?contextMenuEvent@QScrollView@@MAEXPAVQContextMenuEvent@@@Z 1001a9b2 f   qt-mt323:qt-mt323.dll
 0001:000199b8       ?contextMenuEvent@QWidget@@MAEXPAVQContextMenuEvent@@@Z 1001a9b8 f   qt-mt323:qt-mt323.dll
 0001:000199be       ?copy@QLineEdit@@UBEXXZ    1001a9be f   qt-mt323:qt-mt323.dll
 0001:000199c4       ?count@?$QPtrList@VQDockWindow@@@@UBEIXZ 1001a9c4 f   qt-mt323:qt-mt323.dll
 0001:000199ca       ?create@QWidget@@MAEXPAUHWND__@@_N1@Z 1001a9ca f   qt-mt323:qt-mt323.dll
 0001:000199d0       ?createPopupMenu@QLineEdit@@MAEPAVQPopupMenu@@XZ 1001a9d0 f   qt-mt323:qt-mt323.dll
 0001:000199d6       ?customEvent@QObject@@MAEXPAVQCustomEvent@@@Z 1001a9d6 f   qt-mt323:qt-mt323.dll
 0001:000199dc       ?customWhatsThis@QPopupMenu@@UBE_NXZ 1001a9dc f   qt-mt323:qt-mt323.dll
 0001:000199e2       ?customWhatsThis@QWidget@@UBE_NXZ 1001a9e2 f   qt-mt323:qt-mt323.dll
 0001:000199e8       ?cut@QLineEdit@@UAEXXZ     1001a9e8 f   qt-mt323:qt-mt323.dll
 0001:000199ee       ?deleteItem@?$QPtrList@VQDockWindow@@@@EAEXPAX@Z 1001a9ee f   qt-mt323:qt-mt323.dll
 0001:000199f4       ?deselect@QLineEdit@@UAEXXZ 1001a9f4 f   qt-mt323:qt-mt323.dll
 0001:000199fa       ?destroy@QWidget@@MAEX_N0@Z 1001a9fa f   qt-mt323:qt-mt323.dll
 0001:00019a00       ?disconnectNotify@QObject@@MAEXPBD@Z 1001aa00 f   qt-mt323:qt-mt323.dll
 0001:00019a06       ?dock@QDockWindow@@UAEXXZ  1001aa06 f   qt-mt323:qt-mt323.dll
 0001:00019a0c       ?dragEnterEvent@QLineEdit@@MAEXPAVQDragEnterEvent@@@Z 1001aa0c f   qt-mt323:qt-mt323.dll
 0001:00019a12       ?dragEnterEvent@QWidget@@MAEXPAVQDragEnterEvent@@@Z 1001aa12 f   qt-mt323:qt-mt323.dll
 0001:00019a18       ?dragEntered@QListViewItem@@MAEXXZ 1001aa18 f   qt-mt323:qt-mt323.dll
 0001:00019a1e       ?dragLeaveEvent@QLineEdit@@MAEXPAVQDragLeaveEvent@@@Z 1001aa1e f   qt-mt323:qt-mt323.dll
 0001:00019a24       ?dragLeaveEvent@QWidget@@MAEXPAVQDragLeaveEvent@@@Z 1001aa24 f   qt-mt323:qt-mt323.dll
 0001:00019a2a       ?dragLeft@QListViewItem@@MAEXXZ 1001aa2a f   qt-mt323:qt-mt323.dll
 0001:00019a30       ?dragMoveEvent@QLineEdit@@MAEXPAVQDragMoveEvent@@@Z 1001aa30 f   qt-mt323:qt-mt323.dll
 0001:00019a36       ?dragMoveEvent@QWidget@@MAEXPAVQDragMoveEvent@@@Z 1001aa36 f   qt-mt323:qt-mt323.dll
 0001:00019a3c       ?dragObject@QListView@@MAEPAVQDragObject@@XZ 1001aa3c f   qt-mt323:qt-mt323.dll
 0001:00019a42       ?drawButton@QPushButton@@MAEXPAVQPainter@@@Z 1001aa42 f   qt-mt323:qt-mt323.dll
 0001:00019a48       ?drawButtonLabel@QPushButton@@MAEXPAVQPainter@@@Z 1001aa48 f   qt-mt323:qt-mt323.dll
 0001:00019a4e       ?drawContents@QDockWindow@@MAEXPAVQPainter@@@Z 1001aa4e f   qt-mt323:qt-mt323.dll
 0001:00019a54       ?drawContents@QFrame@@MAEXPAVQPainter@@@Z 1001aa54 f   qt-mt323:qt-mt323.dll
 0001:00019a5a       ?drawContents@QLabel@@MAEXPAVQPainter@@@Z 1001aa5a f   qt-mt323:qt-mt323.dll
 0001:00019a60       ?drawContents@QLineEdit@@MAEXPAVQPainter@@@Z 1001aa60 f   qt-mt323:qt-mt323.dll
 0001:00019a66       ?drawContents@QPopupMenu@@MAEXPAVQPainter@@@Z 1001aa66 f   qt-mt323:qt-mt323.dll
 0001:00019a6c       ?drawContents@QScrollView@@EAEXPAVQPainter@@@Z 1001aa6c f   qt-mt323:qt-mt323.dll
 0001:00019a72       ?drawContents@QScrollView@@MAEXPAVQPainter@@HHHH@Z 1001aa72 f   qt-mt323:qt-mt323.dll
 0001:00019a78       ?drawContentsOffset@QListView@@MAEXPAVQPainter@@HHHHHH@Z 1001aa78 f   qt-mt323:qt-mt323.dll
 0001:00019a7e       ?drawFrame@QDockWindow@@MAEXPAVQPainter@@@Z 1001aa7e f   qt-mt323:qt-mt323.dll
 0001:00019a84       ?drawFrame@QFrame@@MAEXPAVQPainter@@@Z 1001aa84 f   qt-mt323:qt-mt323.dll
 0001:00019a8a       ?dropEvent@QLineEdit@@MAEXPAVQDropEvent@@@Z 1001aa8a f   qt-mt323:qt-mt323.dll
 0001:00019a90       ?dropEvent@QWidget@@MAEXPAVQDropEvent@@@Z 1001aa90 f   qt-mt323:qt-mt323.dll
 0001:00019a96       ?dropped@QListViewItem@@MAEXPAVQDropEvent@@@Z 1001aa96 f   qt-mt323:qt-mt323.dll
 0001:00019a9c       ?enabledChange@QButton@@MAEX_N@Z 1001aa9c f   qt-mt323:qt-mt323.dll
 0001:00019aa2       ?enabledChange@QPopupMenu@@MAEX_N@Z 1001aaa2 f   qt-mt323:qt-mt323.dll
 0001:00019aa8       ?enabledChange@QWidget@@MAEX_N@Z 1001aaa8 f   qt-mt323:qt-mt323.dll
 0001:00019aae       ?enforceSortOrder@QListViewItem@@MBEXXZ 1001aaae f   qt-mt323:qt-mt323.dll
 0001:00019ab4       ?enterEvent@QWidget@@MAEXPAVQEvent@@@Z 1001aab4 f   qt-mt323:qt-mt323.dll
 0001:00019aba       ?event@QDockWindow@@MAE_NPAVQEvent@@@Z 1001aaba f   qt-mt323:qt-mt323.dll
 0001:00019ac0       ?event@QLineEdit@@MAE_NPAVQEvent@@@Z 1001aac0 f   qt-mt323:qt-mt323.dll
 0001:00019ac6       ?event@QObject@@UAE_NPAVQEvent@@@Z 1001aac6 f   qt-mt323:qt-mt323.dll
 0001:00019acc       ?event@QToolBar@@UAE_NPAVQEvent@@@Z 1001aacc f   qt-mt323:qt-mt323.dll
 0001:00019ad2       ?event@QWidget@@MAE_NPAVQEvent@@@Z 1001aad2 f   qt-mt323:qt-mt323.dll
 0001:00019ad8       ?eventFilter@QDockWindow@@UAE_NPAVQObject@@PAVQEvent@@@Z 1001aad8 f   qt-mt323:qt-mt323.dll
 0001:00019ade       ?eventFilter@QLayout@@MAE_NPAVQObject@@PAVQEvent@@@Z 1001aade f   qt-mt323:qt-mt323.dll
 0001:00019ae4       ?eventFilter@QListView@@UAE_NPAVQObject@@PAVQEvent@@@Z 1001aae4 f   qt-mt323:qt-mt323.dll
 0001:00019aea       ?eventFilter@QObject@@UAE_NPAV1@PAVQEvent@@@Z 1001aaea f   qt-mt323:qt-mt323.dll
 0001:00019af0       ?eventFilter@QTabWidget@@MAE_NPAVQObject@@PAVQEvent@@@Z 1001aaf0 f   qt-mt323:qt-mt323.dll
 0001:00019af6       ?expanding@QBoxLayout@@UBE?AW4ExpandData@QSizePolicy@@XZ 1001aaf6 f   qt-mt323:qt-mt323.dll
 0001:00019afc       ?expanding@QSpacerItem@@UBE?AW4ExpandData@QSizePolicy@@XZ 1001aafc f   qt-mt323:qt-mt323.dll
 0001:00019b02       ?focusInEvent@QLineEdit@@MAEXPAVQFocusEvent@@@Z 1001ab02 f   qt-mt323:qt-mt323.dll
 0001:00019b08       ?focusInEvent@QListView@@MAEXPAVQFocusEvent@@@Z 1001ab08 f   qt-mt323:qt-mt323.dll
 0001:00019b0e       ?focusInEvent@QPopupMenu@@MAEXPAVQFocusEvent@@@Z 1001ab0e f   qt-mt323:qt-mt323.dll
 0001:00019b14       ?focusInEvent@QPushButton@@MAEXPAVQFocusEvent@@@Z 1001ab14 f   qt-mt323:qt-mt323.dll
 0001:00019b1a       ?focusInEvent@QWidget@@MAEXPAVQFocusEvent@@@Z 1001ab1a f   qt-mt323:qt-mt323.dll
 0001:00019b20       ?focusNextPrevChild@QPopupMenu@@MAE_N_N@Z 1001ab20 f   qt-mt323:qt-mt323.dll
 0001:00019b26       ?focusNextPrevChild@QScrollView@@MAE_N_N@Z 1001ab26 f   qt-mt323:qt-mt323.dll
 0001:00019b2c       ?focusNextPrevChild@QWidget@@MAE_N_N@Z 1001ab2c f   qt-mt323:qt-mt323.dll
 0001:00019b32       ?focusOutEvent@QLineEdit@@MAEXPAVQFocusEvent@@@Z 1001ab32 f   qt-mt323:qt-mt323.dll
 0001:00019b38       ?focusOutEvent@QListView@@MAEXPAVQFocusEvent@@@Z 1001ab38 f   qt-mt323:qt-mt323.dll
 0001:00019b3e       ?focusOutEvent@QPopupMenu@@MAEXPAVQFocusEvent@@@Z 1001ab3e f   qt-mt323:qt-mt323.dll
 0001:00019b44       ?focusOutEvent@QPushButton@@MAEXPAVQFocusEvent@@@Z 1001ab44 f   qt-mt323:qt-mt323.dll
 0001:00019b4a       ?focusOutEvent@QWidget@@MAEXPAVQFocusEvent@@@Z 1001ab4a f   qt-mt323:qt-mt323.dll
 0001:00019b50       ?fontChange@QLabel@@MAEXABVQFont@@@Z 1001ab50 f   qt-mt323:qt-mt323.dll
 0001:00019b56       ?fontChange@QScrollView@@MAEXABVQFont@@@Z 1001ab56 f   qt-mt323:qt-mt323.dll
 0001:00019b5c       ?fontChange@QWidget@@MAEXABVQFont@@@Z 1001ab5c f   qt-mt323:qt-mt323.dll
 0001:00019b62       ?fontInf@QPaintDevice@@MBEHPAVQFont@@H@Z 1001ab62 f   qt-mt323:qt-mt323.dll
 0001:00019b68       ?fontMet@QPaintDevice@@MBEHPAVQFont@@HPBDH@Z 1001ab68 f   qt-mt323:qt-mt323.dll
 0001:00019b6e       ?frameChanged@QFrame@@MAEXXZ 1001ab6e f   qt-mt323:qt-mt323.dll
 0001:00019b74       ?frameChanged@QHBox@@MAEXXZ 1001ab74 f   qt-mt323:qt-mt323.dll
 0001:00019b7a       ?frameChanged@QPopupMenu@@EAEXXZ 1001ab7a f   qt-mt323:qt-mt323.dll
 0001:00019b80       ?frameChanged@QScrollView@@MAEXXZ 1001ab80 f   qt-mt323:qt-mt323.dll
 0001:00019b86       ?geometry@QLayout@@UBE?AVQRect@@XZ 1001ab86 f   qt-mt323:qt-mt323.dll
 0001:00019b8c       ?geometry@QSpacerItem@@UBE?AVQRect@@XZ 1001ab8c f   qt-mt323:qt-mt323.dll
 0001:00019b92       ?handle@QPaintDevice@@UBEPAUHDC__@@XZ 1001ab92 f   qt-mt323:qt-mt323.dll
 0001:00019b98       ?hasHeightForWidth@QBoxLayout@@UBE_NXZ 1001ab98 f   qt-mt323:qt-mt323.dll
 0001:00019b9e       ?hasHeightForWidth@QLayoutItem@@UBE_NXZ 1001ab9e f   qt-mt323:qt-mt323.dll
 0001:00019ba4       ?heightForWidth@QBoxLayout@@UBEHH@Z 1001aba4 f   qt-mt323:qt-mt323.dll
 0001:00019baa       ?heightForWidth@QLabel@@UBEHH@Z 1001abaa f   qt-mt323:qt-mt323.dll
 0001:00019bb0       ?heightForWidth@QLayoutItem@@UBEHH@Z 1001abb0 f   qt-mt323:qt-mt323.dll
 0001:00019bb6       ?heightForWidth@QWidget@@UBEHH@Z 1001abb6 f   qt-mt323:qt-mt323.dll
 0001:00019bbc       ?hide@QPopupMenu@@UAEXXZ   1001abbc f   qt-mt323:qt-mt323.dll
 0001:00019bc2       ?hide@QToolBar@@UAEXXZ     1001abc2 f   qt-mt323:qt-mt323.dll
 0001:00019bc8       ?hide@QWidget@@UAEXXZ      1001abc8 f   qt-mt323:qt-mt323.dll
 0001:00019bce       ?hideEvent@QDockWindow@@MAEXPAVQHideEvent@@@Z 1001abce f   qt-mt323:qt-mt323.dll
 0001:00019bd4       ?hideEvent@QWidget@@MAEXPAVQHideEvent@@@Z 1001abd4 f   qt-mt323:qt-mt323.dll
 0001:00019bda       ?hitButton@QButton@@MBE_NABVQPoint@@@Z 1001abda f   qt-mt323:qt-mt323.dll
 0001:00019be0       ?imComposeEvent@QLineEdit@@MAEXPAVQIMEvent@@@Z 1001abe0 f   qt-mt323:qt-mt323.dll
 0001:00019be6       ?imComposeEvent@QWidget@@MAEXPAVQIMEvent@@@Z 1001abe6 f   qt-mt323:qt-mt323.dll
 0001:00019bec       ?imEndEvent@QLineEdit@@MAEXPAVQIMEvent@@@Z 1001abec f   qt-mt323:qt-mt323.dll
 0001:00019bf2       ?imEndEvent@QWidget@@MAEXPAVQIMEvent@@@Z 1001abf2 f   qt-mt323:qt-mt323.dll
 0001:00019bf8       ?imStartEvent@QLineEdit@@MAEXPAVQIMEvent@@@Z 1001abf8 f   qt-mt323:qt-mt323.dll
 0001:00019bfe       ?imStartEvent@QWidget@@MAEXPAVQIMEvent@@@Z 1001abfe f   qt-mt323:qt-mt323.dll
 0001:00019c04       ?insert@QLineEdit@@UAEXABVQString@@@Z 1001ac04 f   qt-mt323:qt-mt323.dll
 0001:00019c0a       ?insertChild@QObject@@UAEXPAV1@@Z 1001ac0a f   qt-mt323:qt-mt323.dll
 0001:00019c10       ?insertItem@QListView@@UAEXPAVQListViewItem@@@Z 1001ac10 f   qt-mt323:qt-mt323.dll
 0001:00019c16       ?insertItem@QListViewItem@@UAEXPAV1@@Z 1001ac16 f   qt-mt323:qt-mt323.dll
 0001:00019c1c       ?insertTab@QTabWidget@@UAEXPAVQWidget@@ABVQIconSet@@ABVQString@@H@Z 1001ac1c f   qt-mt323:qt-mt323.dll
 0001:00019c22       ?insertTab@QTabWidget@@UAEXPAVQWidget@@ABVQString@@H@Z 1001ac22 f   qt-mt323:qt-mt323.dll
 0001:00019c28       ?insertTab@QTabWidget@@UAEXPAVQWidget@@PAVQTab@@H@Z 1001ac28 f   qt-mt323:qt-mt323.dll
 0001:00019c2e       ?invalidate@QBoxLayout@@UAEXXZ 1001ac2e f   qt-mt323:qt-mt323.dll
 0001:00019c34       ?invalidate@QLayoutItem@@UAEXXZ 1001ac34 f   qt-mt323:qt-mt323.dll
 0001:00019c3a       ?invalidateHeight@QListViewItem@@UAEXXZ 1001ac3a f   qt-mt323:qt-mt323.dll
 0001:00019c40       ?invertSelection@QListView@@UAEXXZ 1001ac40 f   qt-mt323:qt-mt323.dll
 0001:00019c46       ?isEmpty@QLayout@@UBE_NXZ  1001ac46 f   qt-mt323:qt-mt323.dll
 0001:00019c4c       ?isEmpty@QSpacerItem@@UBE_NXZ 1001ac4c f   qt-mt323:qt-mt323.dll
 0001:00019c52       ?iterator@QBoxLayout@@UAE?AVQLayoutIterator@@XZ 1001ac52 f   qt-mt323:qt-mt323.dll
 0001:00019c58       ?iterator@QLayoutItem@@UAE?AVQLayoutIterator@@XZ 1001ac58 f   qt-mt323:qt-mt323.dll
 0001:00019c5e       ?key@QListViewItem@@UBE?AVQString@@H_N@Z 1001ac5e f   qt-mt323:qt-mt323.dll
 0001:00019c64       ?keyPressEvent@QButton@@MAEXPAVQKeyEvent@@@Z 1001ac64 f   qt-mt323:qt-mt323.dll
 0001:00019c6a       ?keyPressEvent@QLineEdit@@MAEXPAVQKeyEvent@@@Z 1001ac6a f   qt-mt323:qt-mt323.dll
 0001:00019c70       ?keyPressEvent@QPopupMenu@@MAEXPAVQKeyEvent@@@Z 1001ac70 f   qt-mt323:qt-mt323.dll
 0001:00019c76       ?keyPressEvent@QWidget@@MAEXPAVQKeyEvent@@@Z 1001ac76 f   qt-mt323:qt-mt323.dll
 0001:00019c7c       ?keyReleaseEvent@QButton@@MAEXPAVQKeyEvent@@@Z 1001ac7c f   qt-mt323:qt-mt323.dll
 0001:00019c82       ?keyReleaseEvent@QWidget@@MAEXPAVQKeyEvent@@@Z 1001ac82 f   qt-mt323:qt-mt323.dll
 0001:00019c88       ?layout@QLayout@@UAEPAV1@XZ 1001ac88 f   qt-mt323:qt-mt323.dll
 0001:00019c8e       ?layout@QLayoutItem@@UAEPAVQLayout@@XZ 1001ac8e f   qt-mt323:qt-mt323.dll
 0001:00019c94       ?leaveEvent@QPopupMenu@@MAEXPAVQEvent@@@Z 1001ac94 f   qt-mt323:qt-mt323.dll
 0001:00019c9a       ?leaveEvent@QWidget@@MAEXPAVQEvent@@@Z 1001ac9a f   qt-mt323:qt-mt323.dll
 0001:00019ca0       ?maximumSize@QBoxLayout@@UBE?AVQSize@@XZ 1001aca0 f   qt-mt323:qt-mt323.dll
 0001:00019ca6       ?maximumSize@QSpacerItem@@UBE?AVQSize@@XZ 1001aca6 f   qt-mt323:qt-mt323.dll
 0001:00019cac       ?menuContentsChanged@QPopupMenu@@EAEXXZ 1001acac f   qt-mt323:qt-mt323.dll
 0001:00019cb2       ?menuDelPopup@QPopupMenu@@EAEXPAV1@@Z 1001acb2 f   qt-mt323:qt-mt323.dll
 0001:00019cb8       ?menuInsPopup@QPopupMenu@@EAEXPAV1@@Z 1001acb8 f   qt-mt323:qt-mt323.dll
 0001:00019cbe       ?menuStateChanged@QPopupMenu@@EAEXXZ 1001acbe f   qt-mt323:qt-mt323.dll
 0001:00019cc4       ?metaObject@QAction@@UBEPAVQMetaObject@@XZ 1001acc4 f   qt-mt323:qt-mt323.dll
 0001:00019cca       ?metaObject@QDockWindow@@UBEPAVQMetaObject@@XZ 1001acca f   qt-mt323:qt-mt323.dll
 0001:00019cd0       ?metaObject@QGuardedPtrPrivate@@UBEPAVQMetaObject@@XZ 1001acd0 f   qt-mt323:qt-mt323.dll
 0001:00019cd6       ?metaObject@QHBoxLayout@@UBEPAVQMetaObject@@XZ 1001acd6 f   qt-mt323:qt-mt323.dll
 0001:00019cdc       ?metaObject@QLabel@@UBEPAVQMetaObject@@XZ 1001acdc f   qt-mt323:qt-mt323.dll
 0001:00019ce2       ?metaObject@QLineEdit@@UBEPAVQMetaObject@@XZ 1001ace2 f   qt-mt323:qt-mt323.dll
 0001:00019ce8       ?metaObject@QListView@@UBEPAVQMetaObject@@XZ 1001ace8 f   qt-mt323:qt-mt323.dll
 0001:00019cee       ?metaObject@QPopupMenu@@UBEPAVQMetaObject@@XZ 1001acee f   qt-mt323:qt-mt323.dll
 0001:00019cf4       ?metaObject@QPushButton@@UBEPAVQMetaObject@@XZ 1001acf4 f   qt-mt323:qt-mt323.dll
 0001:00019cfa       ?metaObject@QTabWidget@@UBEPAVQMetaObject@@XZ 1001acfa f   qt-mt323:qt-mt323.dll
 0001:00019d00       ?metaObject@QToolBar@@UBEPAVQMetaObject@@XZ 1001ad00 f   qt-mt323:qt-mt323.dll
 0001:00019d06       ?metaObject@QVBoxLayout@@UBEPAVQMetaObject@@XZ 1001ad06 f   qt-mt323:qt-mt323.dll
 0001:00019d0c       ?metaObject@QWidget@@UBEPAVQMetaObject@@XZ 1001ad0c f   qt-mt323:qt-mt323.dll
 0001:00019d12       ?metric@QWidget@@MBEHH@Z   1001ad12 f   qt-mt323:qt-mt323.dll
 0001:00019d18       ?minimumSize@QBoxLayout@@UBE?AVQSize@@XZ 1001ad18 f   qt-mt323:qt-mt323.dll
 0001:00019d1e       ?minimumSize@QSpacerItem@@UBE?AVQSize@@XZ 1001ad1e f   qt-mt323:qt-mt323.dll
 0001:00019d24       ?minimumSizeHint@QDockWindow@@UBE?AVQSize@@XZ 1001ad24 f   qt-mt323:qt-mt323.dll
 0001:00019d2a       ?minimumSizeHint@QLabel@@UBE?AVQSize@@XZ 1001ad2a f   qt-mt323:qt-mt323.dll
 0001:00019d30       ?minimumSizeHint@QLineEdit@@UBE?AVQSize@@XZ 1001ad30 f   qt-mt323:qt-mt323.dll
 0001:00019d36       ?minimumSizeHint@QListView@@UBE?AVQSize@@XZ 1001ad36 f   qt-mt323:qt-mt323.dll
 0001:00019d3c       ?minimumSizeHint@QTabWidget@@UBE?AVQSize@@XZ 1001ad3c f   qt-mt323:qt-mt323.dll
 0001:00019d42       ?minimumSizeHint@QToolBar@@UBE?AVQSize@@XZ 1001ad42 f   qt-mt323:qt-mt323.dll
 0001:00019d48       ?minimumSizeHint@QWidget@@UBE?AVQSize@@XZ 1001ad48 f   qt-mt323:qt-mt323.dll
 0001:00019d4e       ?mouseDoubleClickEvent@QLineEdit@@MAEXPAVQMouseEvent@@@Z 1001ad4e f   qt-mt323:qt-mt323.dll
 0001:00019d54       ?mouseDoubleClickEvent@QScrollView@@MAEXPAVQMouseEvent@@@Z 1001ad54 f   qt-mt323:qt-mt323.dll
 0001:00019d5a       ?mouseDoubleClickEvent@QWidget@@MAEXPAVQMouseEvent@@@Z 1001ad5a f   qt-mt323:qt-mt323.dll
 0001:00019d60       ?mouseMoveEvent@QButton@@MAEXPAVQMouseEvent@@@Z 1001ad60 f   qt-mt323:qt-mt323.dll
 0001:00019d66       ?mouseMoveEvent@QLineEdit@@MAEXPAVQMouseEvent@@@Z 1001ad66 f   qt-mt323:qt-mt323.dll
 0001:00019d6c       ?mouseMoveEvent@QPopupMenu@@MAEXPAVQMouseEvent@@@Z 1001ad6c f   qt-mt323:qt-mt323.dll
 0001:00019d72       ?mouseMoveEvent@QScrollView@@MAEXPAVQMouseEvent@@@Z 1001ad72 f   qt-mt323:qt-mt323.dll
 0001:00019d78       ?mouseMoveEvent@QWidget@@MAEXPAVQMouseEvent@@@Z 1001ad78 f   qt-mt323:qt-mt323.dll
 0001:00019d7e       ?mousePressEvent@QButton@@MAEXPAVQMouseEvent@@@Z 1001ad7e f   qt-mt323:qt-mt323.dll
 0001:00019d84       ?mousePressEvent@QLineEdit@@MAEXPAVQMouseEvent@@@Z 1001ad84 f   qt-mt323:qt-mt323.dll
 0001:00019d8a       ?mousePressEvent@QPopupMenu@@MAEXPAVQMouseEvent@@@Z 1001ad8a f   qt-mt323:qt-mt323.dll
 0001:00019d90       ?mousePressEvent@QScrollView@@MAEXPAVQMouseEvent@@@Z 1001ad90 f   qt-mt323:qt-mt323.dll
 0001:00019d96       ?mousePressEvent@QWidget@@MAEXPAVQMouseEvent@@@Z 1001ad96 f   qt-mt323:qt-mt323.dll
 0001:00019d9c       ?mouseReleaseEvent@QButton@@MAEXPAVQMouseEvent@@@Z 1001ad9c f   qt-mt323:qt-mt323.dll
 0001:00019da2       ?mouseReleaseEvent@QLineEdit@@MAEXPAVQMouseEvent@@@Z 1001ada2 f   qt-mt323:qt-mt323.dll
 0001:00019da8       ?mouseReleaseEvent@QPopupMenu@@MAEXPAVQMouseEvent@@@Z 1001ada8 f   qt-mt323:qt-mt323.dll
 0001:00019dae       ?mouseReleaseEvent@QScrollView@@MAEXPAVQMouseEvent@@@Z 1001adae f   qt-mt323:qt-mt323.dll
 0001:00019db4       ?mouseReleaseEvent@QWidget@@MAEXPAVQMouseEvent@@@Z 1001adb4 f   qt-mt323:qt-mt323.dll
 0001:00019dba       ?move@QPushButton@@UAEXHH@Z 1001adba f   qt-mt323:qt-mt323.dll
 0001:00019dc0       ?move@QWidget@@UAEXHH@Z    1001adc0 f   qt-mt323:qt-mt323.dll
 0001:00019dc6       ?moveChild@QScrollView@@UAEXPAVQWidget@@HH@Z 1001adc6 f   qt-mt323:qt-mt323.dll
 0001:00019dcc       ?moveEvent@QWidget@@MAEXPAVQMoveEvent@@@Z 1001adcc f   qt-mt323:qt-mt323.dll
 0001:00019dd2       ?newItem@QPtrCollection@@MAEPAXPAX@Z 1001add2 f   qt-mt323:qt-mt323.dll
 0001:00019dd8       ?okRename@QListViewItem@@MAEXH@Z 1001add8 f   qt-mt323:qt-mt323.dll
 0001:00019dde       ?paintBranches@QListViewItem@@UAEXPAVQPainter@@ABVQColorGroup@@HHH@Z 1001adde f   qt-mt323:qt-mt323.dll
 0001:00019de4       ?paintEmptyArea@QListView@@MAEXPAVQPainter@@ABVQRect@@@Z 1001ade4 f   qt-mt323:qt-mt323.dll
 0001:00019dea       ?paintEvent@QButton@@MAEXPAVQPaintEvent@@@Z 1001adea f   qt-mt323:qt-mt323.dll
 0001:00019df0       ?paintEvent@QFrame@@MAEXPAVQPaintEvent@@@Z 1001adf0 f   qt-mt323:qt-mt323.dll
 0001:00019df6       ?paintEvent@QPopupMenu@@MAEXPAVQPaintEvent@@@Z 1001adf6 f   qt-mt323:qt-mt323.dll
 0001:00019dfc       ?paintEvent@QWidget@@MAEXPAVQPaintEvent@@@Z 1001adfc f   qt-mt323:qt-mt323.dll
 0001:00019e02       ?paintFocus@QListViewItem@@UAEXPAVQPainter@@ABVQColorGroup@@ABVQRect@@@Z 1001ae02 f   qt-mt323:qt-mt323.dll
 0001:00019e08       ?paletteChange@QWidget@@MAEXABVQPalette@@@Z 1001ae08 f   qt-mt323:qt-mt323.dll
 0001:00019e0e       ?paste@QLineEdit@@UAEXXZ   1001ae0e f   qt-mt323:qt-mt323.dll
 0001:00019e14       ?pixmap@QListViewItem@@UBEPBVQPixmap@@H@Z 1001ae14 f   qt-mt323:qt-mt323.dll
 0001:00019e1a       ?polish@QWidget@@UAEXXZ    1001ae1a f   qt-mt323:qt-mt323.dll
 0001:00019e20       ?property@QObject@@UBE?AVQVariant@@PBD@Z 1001ae20 f   qt-mt323:qt-mt323.dll
 0001:00019e26       ?qt_cast@QAction@@UAEPAXPBD@Z 1001ae26 f   qt-mt323:qt-mt323.dll
 0001:00019e2c       ?qt_cast@QDockWindow@@UAEPAXPBD@Z 1001ae2c f   qt-mt323:qt-mt323.dll
 0001:00019e32       ?qt_cast@QGuardedPtrPrivate@@UAEPAXPBD@Z 1001ae32 f   qt-mt323:qt-mt323.dll
 0001:00019e38       ?qt_cast@QHBoxLayout@@UAEPAXPBD@Z 1001ae38 f   qt-mt323:qt-mt323.dll
 0001:00019e3e       ?qt_cast@QLabel@@UAEPAXPBD@Z 1001ae3e f   qt-mt323:qt-mt323.dll
 0001:00019e44       ?qt_cast@QLineEdit@@UAEPAXPBD@Z 1001ae44 f   qt-mt323:qt-mt323.dll
 0001:00019e4a       ?qt_cast@QListView@@UAEPAXPBD@Z 1001ae4a f   qt-mt323:qt-mt323.dll
 0001:00019e50       ?qt_cast@QPopupMenu@@UAEPAXPBD@Z 1001ae50 f   qt-mt323:qt-mt323.dll
 0001:00019e56       ?qt_cast@QPushButton@@UAEPAXPBD@Z 1001ae56 f   qt-mt323:qt-mt323.dll
 0001:00019e5c       ?qt_cast@QTabWidget@@UAEPAXPBD@Z 1001ae5c f   qt-mt323:qt-mt323.dll
 0001:00019e62       ?qt_cast@QToolBar@@UAEPAXPBD@Z 1001ae62 f   qt-mt323:qt-mt323.dll
 0001:00019e68       ?qt_cast@QVBoxLayout@@UAEPAXPBD@Z 1001ae68 f   qt-mt323:qt-mt323.dll
 0001:00019e6e       ?qt_cast@QWidget@@UAEPAXPBD@Z 1001ae6e f   qt-mt323:qt-mt323.dll
 0001:00019e74       ?qt_emit@QAction@@UAE_NHPAUQUObject@@@Z 1001ae74 f   qt-mt323:qt-mt323.dll
 0001:00019e7a       ?qt_emit@QDockWindow@@UAE_NHPAUQUObject@@@Z 1001ae7a f   qt-mt323:qt-mt323.dll
 0001:00019e80       ?qt_emit@QGuardedPtrPrivate@@UAE_NHPAUQUObject@@@Z 1001ae80 f   qt-mt323:qt-mt323.dll
 0001:00019e86       ?qt_emit@QHBoxLayout@@UAE_NHPAUQUObject@@@Z 1001ae86 f   qt-mt323:qt-mt323.dll
 0001:00019e8c       ?qt_emit@QLabel@@UAE_NHPAUQUObject@@@Z 1001ae8c f   qt-mt323:qt-mt323.dll
 0001:00019e92       ?qt_emit@QLineEdit@@UAE_NHPAUQUObject@@@Z 1001ae92 f   qt-mt323:qt-mt323.dll
 0001:00019e98       ?qt_emit@QListView@@UAE_NHPAUQUObject@@@Z 1001ae98 f   qt-mt323:qt-mt323.dll
 0001:00019e9e       ?qt_emit@QPopupMenu@@UAE_NHPAUQUObject@@@Z 1001ae9e f   qt-mt323:qt-mt323.dll
 0001:00019ea4       ?qt_emit@QPushButton@@UAE_NHPAUQUObject@@@Z 1001aea4 f   qt-mt323:qt-mt323.dll
 0001:00019eaa       ?qt_emit@QTabWidget@@UAE_NHPAUQUObject@@@Z 1001aeaa f   qt-mt323:qt-mt323.dll
 0001:00019eb0       ?qt_emit@QToolBar@@UAE_NHPAUQUObject@@@Z 1001aeb0 f   qt-mt323:qt-mt323.dll
 0001:00019eb6       ?qt_emit@QVBoxLayout@@UAE_NHPAUQUObject@@@Z 1001aeb6 f   qt-mt323:qt-mt323.dll
 0001:00019ebc       ?qt_emit@QWidget@@UAE_NHPAUQUObject@@@Z 1001aebc f   qt-mt323:qt-mt323.dll
 0001:00019ec2       ?qt_invoke@QAction@@UAE_NHPAUQUObject@@@Z 1001aec2 f   qt-mt323:qt-mt323.dll
 0001:00019ec8       ?qt_invoke@QDockWindow@@UAE_NHPAUQUObject@@@Z 1001aec8 f   qt-mt323:qt-mt323.dll
 0001:00019ece       ?qt_invoke@QGuardedPtrPrivate@@UAE_NHPAUQUObject@@@Z 1001aece f   qt-mt323:qt-mt323.dll
 0001:00019ed4       ?qt_invoke@QHBoxLayout@@UAE_NHPAUQUObject@@@Z 1001aed4 f   qt-mt323:qt-mt323.dll
 0001:00019eda       ?qt_invoke@QLabel@@UAE_NHPAUQUObject@@@Z 1001aeda f   qt-mt323:qt-mt323.dll
 0001:00019ee0       ?qt_invoke@QLineEdit@@UAE_NHPAUQUObject@@@Z 1001aee0 f   qt-mt323:qt-mt323.dll
 0001:00019ee6       ?qt_invoke@QListView@@UAE_NHPAUQUObject@@@Z 1001aee6 f   qt-mt323:qt-mt323.dll
 0001:00019eec       ?qt_invoke@QPopupMenu@@UAE_NHPAUQUObject@@@Z 1001aeec f   qt-mt323:qt-mt323.dll
 0001:00019ef2       ?qt_invoke@QPushButton@@UAE_NHPAUQUObject@@@Z 1001aef2 f   qt-mt323:qt-mt323.dll
 0001:00019ef8       ?qt_invoke@QTabWidget@@UAE_NHPAUQUObject@@@Z 1001aef8 f   qt-mt323:qt-mt323.dll
 0001:00019efe       ?qt_invoke@QToolBar@@UAE_NHPAUQUObject@@@Z 1001aefe f   qt-mt323:qt-mt323.dll
 0001:00019f04       ?qt_invoke@QVBoxLayout@@UAE_NHPAUQUObject@@@Z 1001af04 f   qt-mt323:qt-mt323.dll
 0001:00019f0a       ?qt_invoke@QWidget@@UAE_NHPAUQUObject@@@Z 1001af0a f   qt-mt323:qt-mt323.dll
 0001:00019f10       ?qt_property@QAction@@UAE_NHHPAVQVariant@@@Z 1001af10 f   qt-mt323:qt-mt323.dll
 0001:00019f16       ?qt_property@QDockWindow@@UAE_NHHPAVQVariant@@@Z 1001af16 f   qt-mt323:qt-mt323.dll
 0001:00019f1c       ?qt_property@QGuardedPtrPrivate@@UAE_NHHPAVQVariant@@@Z 1001af1c f   qt-mt323:qt-mt323.dll
 0001:00019f22       ?qt_property@QHBoxLayout@@UAE_NHHPAVQVariant@@@Z 1001af22 f   qt-mt323:qt-mt323.dll
 0001:00019f28       ?qt_property@QLabel@@UAE_NHHPAVQVariant@@@Z 1001af28 f   qt-mt323:qt-mt323.dll
 0001:00019f2e       ?qt_property@QLineEdit@@UAE_NHHPAVQVariant@@@Z 1001af2e f   qt-mt323:qt-mt323.dll
 0001:00019f34       ?qt_property@QListView@@UAE_NHHPAVQVariant@@@Z 1001af34 f   qt-mt323:qt-mt323.dll
 0001:00019f3a       ?qt_property@QPopupMenu@@UAE_NHHPAVQVariant@@@Z 1001af3a f   qt-mt323:qt-mt323.dll
 0001:00019f40       ?qt_property@QPushButton@@UAE_NHHPAVQVariant@@@Z 1001af40 f   qt-mt323:qt-mt323.dll
 0001:00019f46       ?qt_property@QTabWidget@@UAE_NHHPAVQVariant@@@Z 1001af46 f   qt-mt323:qt-mt323.dll
 0001:00019f4c       ?qt_property@QToolBar@@UAE_NHHPAVQVariant@@@Z 1001af4c f   qt-mt323:qt-mt323.dll
 0001:00019f52       ?qt_property@QVBoxLayout@@UAE_NHHPAVQVariant@@@Z 1001af52 f   qt-mt323:qt-mt323.dll
 0001:00019f58       ?qt_property@QWidget@@UAE_NHHPAVQVariant@@@Z 1001af58 f   qt-mt323:qt-mt323.dll
 0001:00019f5e       ?read@QGList@@MAEAAVQDataStream@@AAV2@AAPAX@Z 1001af5e f   qt-mt323:qt-mt323.dll
 0001:00019f64       ?redo@QLineEdit@@UAEXXZ    1001af64 f   qt-mt323:qt-mt323.dll
 0001:00019f6a       ?removeChild@QObject@@UAEXPAV1@@Z 1001af6a f   qt-mt323:qt-mt323.dll
 0001:00019f70       ?removeChild@QScrollView@@UAEXPAVQObject@@@Z 1001af70 f   qt-mt323:qt-mt323.dll
 0001:00019f76       ?removeColumn@QListView@@UAEXH@Z 1001af76 f   qt-mt323:qt-mt323.dll
 0001:00019f7c       ?removeFrom@QAction@@UAE_NPAVQWidget@@@Z 1001af7c f   qt-mt323:qt-mt323.dll
 0001:00019f82       ?removeItem@QListView@@UAEXPAVQListViewItem@@@Z 1001af82 f   qt-mt323:qt-mt323.dll
 0001:00019f88       ?removeItem@QListViewItem@@UAEXPAV1@@Z 1001af88 f   qt-mt323:qt-mt323.dll
 0001:00019f8e       ?removePage@QTabWidget@@UAEXPAVQWidget@@@Z 1001af8e f   qt-mt323:qt-mt323.dll
 0001:00019f94       ?reparent@QWidget@@UAEXPAV1@IABVQPoint@@_N@Z 1001af94 f   qt-mt323:qt-mt323.dll
 0001:00019f9a       ?resize@QPushButton@@UAEXHH@Z 1001af9a f   qt-mt323:qt-mt323.dll
 0001:00019fa0       ?resize@QScrollView@@UAEXHH@Z 1001afa0 f   qt-mt323:qt-mt323.dll
 0001:00019fa6       ?resize@QWidget@@UAEXHH@Z  1001afa6 f   qt-mt323:qt-mt323.dll
 0001:00019fac       ?resizeContents@QScrollView@@UAEXHH@Z 1001afac f   qt-mt323:qt-mt323.dll
 0001:00019fb2       ?resizeEvent@QDockWindow@@MAEXPAVQResizeEvent@@@Z 1001afb2 f   qt-mt323:qt-mt323.dll
 0001:00019fb8       ?resizeEvent@QFrame@@MAEXPAVQResizeEvent@@@Z 1001afb8 f   qt-mt323:qt-mt323.dll
 0001:00019fbe       ?resizeEvent@QLabel@@MAEXPAVQResizeEvent@@@Z 1001afbe f   qt-mt323:qt-mt323.dll
 0001:00019fc4       ?resizeEvent@QLineEdit@@MAEXPAVQResizeEvent@@@Z 1001afc4 f   qt-mt323:qt-mt323.dll
 0001:00019fca       ?resizeEvent@QListView@@MAEXPAVQResizeEvent@@@Z 1001afca f   qt-mt323:qt-mt323.dll
 0001:00019fd0       ?resizeEvent@QPushButton@@MAEXPAVQResizeEvent@@@Z 1001afd0 f   qt-mt323:qt-mt323.dll
 0001:00019fd6       ?resizeEvent@QTabWidget@@MAEXPAVQResizeEvent@@@Z 1001afd6 f   qt-mt323:qt-mt323.dll
 0001:00019fdc       ?resizeEvent@QToolBar@@MAEXPAVQResizeEvent@@@Z 1001afdc f   qt-mt323:qt-mt323.dll
 0001:00019fe2       ?resizeEvent@QWidget@@MAEXPAVQResizeEvent@@@Z 1001afe2 f   qt-mt323:qt-mt323.dll
 0001:00019fe8       ?resolution@QPaintDevice@@UBEHXZ 1001afe8 f   qt-mt323:qt-mt323.dll
 0001:00019fee       ?rtti@QListViewItem@@UBEHXZ 1001afee f   qt-mt323:qt-mt323.dll
 0001:00019ff4       ?selectAll@QLineEdit@@UAEXXZ 1001aff4 f   qt-mt323:qt-mt323.dll
 0001:00019ffa       ?selectAll@QListView@@UAEX_N@Z 1001affa f   qt-mt323:qt-mt323.dll
 0001:0001a000       ?setAccel@QAction@@UAEXABVQKeySequence@@@Z 1001b000 f   qt-mt323:qt-mt323.dll
 0001:0001a006       ?setAccel@QButton@@UAEXABVQKeySequence@@@Z 1001b006 f   qt-mt323:qt-mt323.dll
 0001:0001a00c       ?setAcceptDrops@QWidget@@UAEX_N@Z 1001b00c f   qt-mt323:qt-mt323.dll
 0001:0001a012       ?setActiveItem@QPopupMenu@@UAEXH@Z 1001b012 f   qt-mt323:qt-mt323.dll
 0001:0001a018       ?setActiveWindow@QWidget@@UAEXXZ 1001b018 f   qt-mt323:qt-mt323.dll
 0001:0001a01e       ?setAlignment@QLabel@@UAEXH@Z 1001b01e f   qt-mt323:qt-mt323.dll
 0001:0001a024       ?setAlignment@QLayoutItem@@UAEXH@Z 1001b024 f   qt-mt323:qt-mt323.dll
 0001:0001a02a       ?setAlignment@QLineEdit@@UAEXH@Z 1001b02a f   qt-mt323:qt-mt323.dll
 0001:0001a030       ?setAllColumnsShowFocus@QListView@@UAEX_N@Z 1001b030 f   qt-mt323:qt-mt323.dll
 0001:0001a036       ?setAutoAdd@QLayout@@UAEX_N@Z 1001b036 f   qt-mt323:qt-mt323.dll
 0001:0001a03c       ?setAutoDefault@QPushButton@@UAEX_N@Z 1001b03c f   qt-mt323:qt-mt323.dll
 0001:0001a042       ?setAutoMask@QWidget@@UAEX_N@Z 1001b042 f   qt-mt323:qt-mt323.dll
 0001:0001a048       ?setAutoRepeat@QButton@@UAEX_N@Z 1001b048 f   qt-mt323:qt-mt323.dll
 0001:0001a04e       ?setAutoResize@QLabel@@UAEX_N@Z 1001b04e f   qt-mt323:qt-mt323.dll
 0001:0001a054       ?setBackgroundColor@QWidget@@UAEXABVQColor@@@Z 1001b054 f   qt-mt323:qt-mt323.dll
 0001:0001a05a       ?setBackgroundMode@QWidget@@UAEXW4BackgroundMode@Qt@@@Z 1001b05a f   qt-mt323:qt-mt323.dll
 0001:0001a060       ?setBackgroundOrigin@QWidget@@UAEXW4BackgroundOrigin@1@@Z 1001b060 f   qt-mt323:qt-mt323.dll
 0001:0001a066       ?setBackgroundPixmap@QWidget@@UAEXABVQPixmap@@@Z 1001b066 f   qt-mt323:qt-mt323.dll
 0001:0001a06c       ?setBuddy@QLabel@@UAEXPAVQWidget@@@Z 1001b06c f   qt-mt323:qt-mt323.dll
 0001:0001a072       ?setCaption@QDockWindow@@UAEXABVQString@@@Z 1001b072 f   qt-mt323:qt-mt323.dll
 0001:0001a078       ?setCheckable@QPopupMenu@@UAEX_N@Z 1001b078 f   qt-mt323:qt-mt323.dll
 0001:0001a07e       ?setCloseMode@QDockWindow@@UAEXH@Z 1001b07e f   qt-mt323:qt-mt323.dll
 0001:0001a084       ?setColumnAlignment@QListView@@UAEXHH@Z 1001b084 f   qt-mt323:qt-mt323.dll
 0001:0001a08a       ?setColumnText@QListView@@UAEXHABVQIconSet@@ABVQString@@@Z 1001b08a f   qt-mt323:qt-mt323.dll
 0001:0001a090       ?setColumnText@QListView@@UAEXHABVQString@@@Z 1001b090 f   qt-mt323:qt-mt323.dll
 0001:0001a096       ?setColumnWidth@QListView@@UAEXHH@Z 1001b096 f   qt-mt323:qt-mt323.dll
 0001:0001a09c       ?setColumnWidthMode@QListView@@UAEXHW4WidthMode@1@@Z 1001b09c f   qt-mt323:qt-mt323.dll
 0001:0001a0a2       ?setContentsPos@QListView@@UAEXHH@Z 1001b0a2 f   qt-mt323:qt-mt323.dll
 0001:0001a0a8       ?setCornerWidget@QScrollView@@UAEXPAVQWidget@@@Z 1001b0a8 f   qt-mt323:qt-mt323.dll
 0001:0001a0ae       ?setCurrentItem@QListView@@UAEXPAVQListViewItem@@@Z 1001b0ae f   qt-mt323:qt-mt323.dll
 0001:0001a0b4       ?setCursor@QWidget@@UAEXABVQCursor@@@Z 1001b0b4 f   qt-mt323:qt-mt323.dll
 0001:0001a0ba       ?setCursorPosition@QLineEdit@@UAEXH@Z 1001b0ba f   qt-mt323:qt-mt323.dll
 0001:0001a0c0       ?setDefault@QPushButton@@UAEX_N@Z 1001b0c0 f   qt-mt323:qt-mt323.dll
 0001:0001a0c6       ?setDefaultRenameAction@QListView@@UAEXW4RenameAction@1@@Z 1001b0c6 f   qt-mt323:qt-mt323.dll
 0001:0001a0cc       ?setDown@QButton@@UAEX_N@Z 1001b0cc f   qt-mt323:qt-mt323.dll
 0001:0001a0d2       ?setDragAutoScroll@QScrollView@@UAEX_N@Z 1001b0d2 f   qt-mt323:qt-mt323.dll
 0001:0001a0d8       ?setDragEnabled@QLineEdit@@UAEX_N@Z 1001b0d8 f   qt-mt323:qt-mt323.dll
 0001:0001a0de       ?setDragEnabled@QListViewItem@@UAEX_N@Z 1001b0de f   qt-mt323:qt-mt323.dll
 0001:0001a0e4       ?setDropEnabled@QListViewItem@@UAEX_N@Z 1001b0e4 f   qt-mt323:qt-mt323.dll
 0001:0001a0ea       ?setEchoMode@QLineEdit@@UAEXW4EchoMode@1@@Z 1001b0ea f   qt-mt323:qt-mt323.dll
 0001:0001a0f0       ?setEnabled@QAction@@UAEX_N@Z 1001b0f0 f   qt-mt323:qt-mt323.dll
 0001:0001a0f6       ?setEnabled@QListViewItem@@UAEX_N@Z 1001b0f6 f   qt-mt323:qt-mt323.dll
 0001:0001a0fc       ?setEnabled@QScrollView@@UAEX_N@Z 1001b0fc f   qt-mt323:qt-mt323.dll
 0001:0001a102       ?setEnabled@QWidget@@UAEX_N@Z 1001b102 f   qt-mt323:qt-mt323.dll
 0001:0001a108       ?setEraseColor@QWidget@@UAEXABVQColor@@@Z 1001b108 f   qt-mt323:qt-mt323.dll
 0001:0001a10e       ?setErasePixmap@QWidget@@UAEXABVQPixmap@@@Z 1001b10e f   qt-mt323:qt-mt323.dll
 0001:0001a114       ?setExpandable@QListViewItem@@UAEX_N@Z 1001b114 f   qt-mt323:qt-mt323.dll
 0001:0001a11a       ?setFirstItemActive@QPopupMenu@@EAEXXZ 1001b11a f   qt-mt323:qt-mt323.dll
 0001:0001a120       ?setFixedExtentHeight@QDockWindow@@UAEXH@Z 1001b120 f   qt-mt323:qt-mt323.dll
 0001:0001a126       ?setFixedExtentWidth@QDockWindow@@UAEXH@Z 1001b126 f   qt-mt323:qt-mt323.dll
 0001:0001a12c       ?setFocus@QWidget@@UAEXXZ  1001b12c f   qt-mt323:qt-mt323.dll
 0001:0001a132       ?setFocusProxy@QWidget@@UAEXPAV1@@Z 1001b132 f   qt-mt323:qt-mt323.dll
 0001:0001a138       ?setFont@QLabel@@UAEXABVQFont@@@Z 1001b138 f   qt-mt323:qt-mt323.dll
 0001:0001a13e       ?setFont@QLineEdit@@UAEXABVQFont@@@Z 1001b13e f   qt-mt323:qt-mt323.dll
 0001:0001a144       ?setFont@QListView@@UAEXABVQFont@@@Z 1001b144 f   qt-mt323:qt-mt323.dll
 0001:0001a14a       ?setFont@QPopupMenu@@UAEXABVQFont@@@Z 1001b14a f   qt-mt323:qt-mt323.dll
 0001:0001a150       ?setFont@QWidget@@UAEXABVQFont@@@Z 1001b150 f   qt-mt323:qt-mt323.dll
 0001:0001a156       ?setFrame@QLineEdit@@UAEX_N@Z 1001b156 f   qt-mt323:qt-mt323.dll
 0001:0001a15c       ?setFrameRect@QFrame@@UAEXABVQRect@@@Z 1001b15c f   qt-mt323:qt-mt323.dll
 0001:0001a162       ?setFrameStyle@QFrame@@UAEXH@Z 1001b162 f   qt-mt323:qt-mt323.dll
 0001:0001a168       ?setGeometry@QBoxLayout@@UAEXABVQRect@@@Z 1001b168 f   qt-mt323:qt-mt323.dll
 0001:0001a16e       ?setGeometry@QPushButton@@UAEXABVQRect@@@Z 1001b16e f   qt-mt323:qt-mt323.dll
 0001:0001a174       ?setGeometry@QPushButton@@UAEXHHHH@Z 1001b174 f   qt-mt323:qt-mt323.dll
 0001:0001a17a       ?setGeometry@QSpacerItem@@UAEXABVQRect@@@Z 1001b17a f   qt-mt323:qt-mt323.dll
 0001:0001a180       ?setGeometry@QWidget@@UAEXABVQRect@@@Z 1001b180 f   qt-mt323:qt-mt323.dll
 0001:0001a186       ?setGeometry@QWidget@@UAEXHHHH@Z 1001b186 f   qt-mt323:qt-mt323.dll
 0001:0001a18c       ?setGroup@QButton@@EAEXPAVQButtonGroup@@@Z 1001b18c f   qt-mt323:qt-mt323.dll
 0001:0001a192       ?setHBarGeometry@QScrollView@@MAEXAAVQScrollBar@@HHHH@Z 1001b192 f   qt-mt323:qt-mt323.dll
 0001:0001a198       ?setHScrollBarMode@QScrollView@@UAEXW4ScrollBarMode@1@@Z 1001b198 f   qt-mt323:qt-mt323.dll
 0001:0001a19e       ?setHeight@QListViewItem@@MAEXH@Z 1001b19e f   qt-mt323:qt-mt323.dll
 0001:0001a1a4       ?setHorizontallyStretchable@QDockWindow@@UAEX_N@Z 1001b1a4 f   qt-mt323:qt-mt323.dll
 0001:0001a1aa       ?setIcon@QWidget@@UAEXABVQPixmap@@@Z 1001b1aa f   qt-mt323:qt-mt323.dll
 0001:0001a1b0       ?setIconSet@QAction@@UAEXABVQIconSet@@@Z 1001b1b0 f   qt-mt323:qt-mt323.dll
 0001:0001a1b6       ?setIconText@QWidget@@UAEXABVQString@@@Z 1001b1b6 f   qt-mt323:qt-mt323.dll
 0001:0001a1bc       ?setId@QMenuData@@UAEXHH@Z 1001b1bc f   qt-mt323:qt-mt323.dll
 0001:0001a1c2       ?setIsMenuButton@QPushButton@@UAEX_N@Z 1001b1c2 f   qt-mt323:qt-mt323.dll
 0001:0001a1c8       ?setItemMargin@QListView@@UAEXH@Z 1001b1c8 f   qt-mt323:qt-mt323.dll
 0001:0001a1ce       ?setKeyCompression@QWidget@@MAEX_N@Z 1001b1ce f   qt-mt323:qt-mt323.dll
 0001:0001a1d4       ?setLabel@QToolBar@@UAEXABVQString@@@Z 1001b1d4 f   qt-mt323:qt-mt323.dll
 0001:0001a1da       ?setLineWidth@QFrame@@UAEXH@Z 1001b1da f   qt-mt323:qt-mt323.dll
 0001:0001a1e0       ?setMargin@QFrame@@UAEXH@Z 1001b1e0 f   qt-mt323:qt-mt323.dll
 0001:0001a1e6       ?setMargin@QLayout@@UAEXH@Z 1001b1e6 f   qt-mt323:qt-mt323.dll
 0001:0001a1ec       ?setMargins@QScrollView@@MAEXHHHH@Z 1001b1ec f   qt-mt323:qt-mt323.dll
 0001:0001a1f2       ?setMask@QWidget@@UAEXABVQBitmap@@@Z 1001b1f2 f   qt-mt323:qt-mt323.dll
 0001:0001a1f8       ?setMask@QWidget@@UAEXABVQRegion@@@Z 1001b1f8 f   qt-mt323:qt-mt323.dll
 0001:0001a1fe       ?setMaxLength@QLineEdit@@UAEXH@Z 1001b1fe f   qt-mt323:qt-mt323.dll
 0001:0001a204       ?setMaximumSize@QWidget@@UAEXHH@Z 1001b204 f   qt-mt323:qt-mt323.dll
 0001:0001a20a       ?setMenuBar@QLayout@@UAEXPAVQMenuBar@@@Z 1001b20a f   qt-mt323:qt-mt323.dll
 0001:0001a210       ?setMenuText@QAction@@UAEXABVQString@@@Z 1001b210 f   qt-mt323:qt-mt323.dll
 0001:0001a216       ?setMicroFocusHint@QWidget@@MAEXHHHH_NPAVQFont@@@Z 1001b216 f   qt-mt323:qt-mt323.dll
 0001:0001a21c       ?setMidLineWidth@QFrame@@UAEXH@Z 1001b21c f   qt-mt323:qt-mt323.dll
 0001:0001a222       ?setMinimumSize@QToolBar@@UAEXHH@Z 1001b222 f   qt-mt323:qt-mt323.dll
 0001:0001a228       ?setMinimumSize@QWidget@@UAEXHH@Z 1001b228 f   qt-mt323:qt-mt323.dll
 0001:0001a22e       ?setMouseTracking@QWidget@@UAEX_N@Z 1001b22e f   qt-mt323:qt-mt323.dll
 0001:0001a234       ?setMovie@QLabel@@UAEXABVQMovie@@@Z 1001b234 f   qt-mt323:qt-mt323.dll
 0001:0001a23a       ?setMovingEnabled@QDockWindow@@UAEX_N@Z 1001b23a f   qt-mt323:qt-mt323.dll
 0001:0001a240       ?setMultiLinesEnabled@QListViewItem@@UAEX_N@Z 1001b240 f   qt-mt323:qt-mt323.dll
 0001:0001a246       ?setMultiSelection@QListView@@UAEX_N@Z 1001b246 f   qt-mt323:qt-mt323.dll
 0001:0001a24c       ?setName@QObject@@UAEXPBD@Z 1001b24c f   qt-mt323:qt-mt323.dll
 0001:0001a252       ?setNewLine@QDockWindow@@UAEX_N@Z 1001b252 f   qt-mt323:qt-mt323.dll
 0001:0001a258       ?setNum@QLabel@@UAEXH@Z    1001b258 f   qt-mt323:qt-mt323.dll
 0001:0001a25e       ?setNum@QLabel@@UAEXN@Z    1001b25e f   qt-mt323:qt-mt323.dll
 0001:0001a264       ?setOffset@QDockWindow@@UAEXH@Z 1001b264 f   qt-mt323:qt-mt323.dll
 0001:0001a26a       ?setOn@QAction@@UAEX_N@Z   1001b26a f   qt-mt323:qt-mt323.dll
 0001:0001a270       ?setOn@QPushButton@@UAEX_N@Z 1001b270 f   qt-mt323:qt-mt323.dll
 0001:0001a276       ?setOpaqueMoving@QDockWindow@@UAEX_N@Z 1001b276 f   qt-mt323:qt-mt323.dll
 0001:0001a27c       ?setOpen@QListView@@UAEXPAVQListViewItem@@_N@Z 1001b27c f   qt-mt323:qt-mt323.dll
 0001:0001a282       ?setOpen@QListViewItem@@UAEX_N@Z 1001b282 f   qt-mt323:qt-mt323.dll
 0001:0001a288       ?setOrientation@QDockWindow@@UAEXW4Orientation@Qt@@@Z 1001b288 f   qt-mt323:qt-mt323.dll
 0001:0001a28e       ?setOrientation@QToolBar@@UAEXW4Orientation@Qt@@@Z 1001b28e f   qt-mt323:qt-mt323.dll
 0001:0001a294       ?setPalette@QLineEdit@@UAEXABVQPalette@@@Z 1001b294 f   qt-mt323:qt-mt323.dll
 0001:0001a29a       ?setPalette@QListView@@UAEXABVQPalette@@@Z 1001b29a f   qt-mt323:qt-mt323.dll
 0001:0001a2a0       ?setPalette@QWidget@@UAEXABVQPalette@@@Z 1001b2a0 f   qt-mt323:qt-mt323.dll
 0001:0001a2a6       ?setPaletteBackgroundColor@QWidget@@UAEXABVQColor@@@Z 1001b2a6 f   qt-mt323:qt-mt323.dll
 0001:0001a2ac       ?setPaletteBackgroundPixmap@QWidget@@UAEXABVQPixmap@@@Z 1001b2ac f   qt-mt323:qt-mt323.dll
 0001:0001a2b2       ?setPicture@QLabel@@UAEXABVQPicture@@@Z 1001b2b2 f   qt-mt323:qt-mt323.dll
 0001:0001a2b8       ?setPixmap@QButton@@UAEXABVQPixmap@@@Z 1001b2b8 f   qt-mt323:qt-mt323.dll
 0001:0001a2be       ?setPixmap@QLabel@@UAEXABVQPixmap@@@Z 1001b2be f   qt-mt323:qt-mt323.dll
 0001:0001a2c4       ?setPixmap@QListViewItem@@UAEXHABVQPixmap@@@Z 1001b2c4 f   qt-mt323:qt-mt323.dll
 0001:0001a2ca       ?setProperty@QObject@@UAE_NPBDABVQVariant@@@Z 1001b2ca f   qt-mt323:qt-mt323.dll
 0001:0001a2d0       ?setReadOnly@QLineEdit@@UAEX_N@Z 1001b2d0 f   qt-mt323:qt-mt323.dll
 0001:0001a2d6       ?setResizeEnabled@QDockWindow@@UAEX_N@Z 1001b2d6 f   qt-mt323:qt-mt323.dll
 0001:0001a2dc       ?setResizeMode@QListView@@UAEXW4ResizeMode@1@@Z 1001b2dc f   qt-mt323:qt-mt323.dll
 0001:0001a2e2       ?setResizePolicy@QScrollView@@UAEXW4ResizePolicy@1@@Z 1001b2e2 f   qt-mt323:qt-mt323.dll
 0001:0001a2e8       ?setResolution@QPaintDevice@@UAEXH@Z 1001b2e8 f   qt-mt323:qt-mt323.dll
 0001:0001a2ee       ?setRootIsDecorated@QListView@@UAEX_N@Z 1001b2ee f   qt-mt323:qt-mt323.dll
 0001:0001a2f4       ?setSelectable@QListViewItem@@UAEX_N@Z 1001b2f4 f   qt-mt323:qt-mt323.dll
 0001:0001a2fa       ?setSelected@QListView@@UAEXPAVQListViewItem@@_N@Z 1001b2fa f   qt-mt323:qt-mt323.dll
 0001:0001a300       ?setSelected@QListViewItem@@UAEX_N@Z 1001b300 f   qt-mt323:qt-mt323.dll
 0001:0001a306       ?setSelection@QLineEdit@@UAEXHH@Z 1001b306 f   qt-mt323:qt-mt323.dll
 0001:0001a30c       ?setShowSortIndicator@QListView@@UAEX_N@Z 1001b30c f   qt-mt323:qt-mt323.dll
 0001:0001a312       ?setShowToolTips@QListView@@UAEX_N@Z 1001b312 f   qt-mt323:qt-mt323.dll
 0001:0001a318       ?setSizeIncrement@QWidget@@UAEXHH@Z 1001b318 f   qt-mt323:qt-mt323.dll
 0001:0001a31e       ?setSizePolicy@QWidget@@UAEXVQSizePolicy@@@Z 1001b31e f   qt-mt323:qt-mt323.dll
 0001:0001a324       ?setSorting@QListView@@UAEXH_N@Z 1001b324 f   qt-mt323:qt-mt323.dll
 0001:0001a32a       ?setSpacing@QLayout@@UAEXH@Z 1001b32a f   qt-mt323:qt-mt323.dll
 0001:0001a330       ?setState@QButton@@MAEXW4ToggleState@1@@Z 1001b330 f   qt-mt323:qt-mt323.dll
 0001:0001a336       ?setStatusTip@QAction@@UAEXABVQString@@@Z 1001b336 f   qt-mt323:qt-mt323.dll
 0001:0001a33c       ?setStretchableWidget@QToolBar@@UAEXPAVQWidget@@@Z 1001b33c f   qt-mt323:qt-mt323.dll
 0001:0001a342       ?setText@QAction@@UAEXABVQString@@@Z 1001b342 f   qt-mt323:qt-mt323.dll
 0001:0001a348       ?setText@QButton@@UAEXABVQString@@@Z 1001b348 f   qt-mt323:qt-mt323.dll
 0001:0001a34e       ?setText@QLabel@@UAEXABVQString@@@Z 1001b34e f   qt-mt323:qt-mt323.dll
 0001:0001a354       ?setText@QLineEdit@@UAEXABVQString@@@Z 1001b354 f   qt-mt323:qt-mt323.dll
 0001:0001a35a       ?setText@QListViewItem@@UAEXHABVQString@@@Z 1001b35a f   qt-mt323:qt-mt323.dll
 0001:0001a360       ?setToggleAction@QAction@@UAEX_N@Z 1001b360 f   qt-mt323:qt-mt323.dll
 0001:0001a366       ?setToggleType@QButton@@MAEXW4ToggleType@1@@Z 1001b366 f   qt-mt323:qt-mt323.dll
 0001:0001a36c       ?setToolTip@QAction@@UAEXABVQString@@@Z 1001b36c f   qt-mt323:qt-mt323.dll
 0001:0001a372       ?setTreeStepSize@QListView@@UAEXH@Z 1001b372 f   qt-mt323:qt-mt323.dll
 0001:0001a378       ?setUpdatesEnabled@QWidget@@UAEX_N@Z 1001b378 f   qt-mt323:qt-mt323.dll
 0001:0001a37e       ?setVBarGeometry@QScrollView@@MAEXAAVQScrollBar@@HHHH@Z 1001b37e f   qt-mt323:qt-mt323.dll
 0001:0001a384       ?setVScrollBarMode@QScrollView@@UAEXW4ScrollBarMode@1@@Z 1001b384 f   qt-mt323:qt-mt323.dll
 0001:0001a38a       ?setValidator@QLineEdit@@UAEXPBVQValidator@@@Z 1001b38a f   qt-mt323:qt-mt323.dll
 0001:0001a390       ?setVerticallyStretchable@QDockWindow@@UAEX_N@Z 1001b390 f   qt-mt323:qt-mt323.dll
 0001:0001a396       ?setWFlags@QWidget@@MAEXI@Z 1001b396 f   qt-mt323:qt-mt323.dll
 0001:0001a39c       ?setWState@QWidget@@MAEXI@Z 1001b39c f   qt-mt323:qt-mt323.dll
 0001:0001a3a2       ?setWhatsThis@QAction@@UAEXABVQString@@@Z 1001b3a2 f   qt-mt323:qt-mt323.dll
 0001:0001a3a8       ?setWidget@QDockWindow@@UAEXPAVQWidget@@@Z 1001b3a8 f   qt-mt323:qt-mt323.dll
 0001:0001a3ae       ?setup@QListViewItem@@UAEXXZ 1001b3ae f   qt-mt323:qt-mt323.dll
 0001:0001a3b4       ?show@QListView@@UAEXXZ    1001b3b4 f   qt-mt323:qt-mt323.dll
 0001:0001a3ba       ?show@QPopupMenu@@UAEXXZ   1001b3ba f   qt-mt323:qt-mt323.dll
 0001:0001a3c0       ?show@QToolBar@@UAEXXZ     1001b3c0 f   qt-mt323:qt-mt323.dll
 0001:0001a3c6       ?show@QWidget@@UAEXXZ      1001b3c6 f   qt-mt323:qt-mt323.dll
 0001:0001a3cc       ?showEvent@QDockWindow@@MAEXPAVQShowEvent@@@Z 1001b3cc f   qt-mt323:qt-mt323.dll
 0001:0001a3d2       ?showEvent@QListView@@MAEXPAVQShowEvent@@@Z 1001b3d2 f   qt-mt323:qt-mt323.dll
 0001:0001a3d8       ?showEvent@QTabWidget@@MAEXPAVQShowEvent@@@Z 1001b3d8 f   qt-mt323:qt-mt323.dll
 0001:0001a3de       ?showEvent@QWidget@@MAEXPAVQShowEvent@@@Z 1001b3de f   qt-mt323:qt-mt323.dll
 0001:0001a3e4       ?showMaximized@QWidget@@UAEXXZ 1001b3e4 f   qt-mt323:qt-mt323.dll
 0001:0001a3ea       ?showMinimized@QWidget@@UAEXXZ 1001b3ea f   qt-mt323:qt-mt323.dll
 0001:0001a3f0       ?showNormal@QWidget@@UAEXXZ 1001b3f0 f   qt-mt323:qt-mt323.dll
 0001:0001a3f6       ?showPage@QTabWidget@@UAEXPAVQWidget@@@Z 1001b3f6 f   qt-mt323:qt-mt323.dll
 0001:0001a3fc       ?sizeHint@QBoxLayout@@UBE?AVQSize@@XZ 1001b3fc f   qt-mt323:qt-mt323.dll
 0001:0001a402       ?sizeHint@QDockWindow@@UBE?AVQSize@@XZ 1001b402 f   qt-mt323:qt-mt323.dll
 0001:0001a408       ?sizeHint@QHBox@@UBE?AVQSize@@XZ 1001b408 f   qt-mt323:qt-mt323.dll
 0001:0001a40e       ?sizeHint@QLabel@@UBE?AVQSize@@XZ 1001b40e f   qt-mt323:qt-mt323.dll
 0001:0001a414       ?sizeHint@QLineEdit@@UBE?AVQSize@@XZ 1001b414 f   qt-mt323:qt-mt323.dll
 0001:0001a41a       ?sizeHint@QListView@@UBE?AVQSize@@XZ 1001b41a f   qt-mt323:qt-mt323.dll
 0001:0001a420       ?sizeHint@QPopupMenu@@UBE?AVQSize@@XZ 1001b420 f   qt-mt323:qt-mt323.dll
 0001:0001a426       ?sizeHint@QPushButton@@UBE?AVQSize@@XZ 1001b426 f   qt-mt323:qt-mt323.dll
 0001:0001a42c       ?sizeHint@QSpacerItem@@UBE?AVQSize@@XZ 1001b42c f   qt-mt323:qt-mt323.dll
 0001:0001a432       ?sizeHint@QTabWidget@@UBE?AVQSize@@XZ 1001b432 f   qt-mt323:qt-mt323.dll
 0001:0001a438       ?sizeHint@QWidget@@UBE?AVQSize@@XZ 1001b438 f   qt-mt323:qt-mt323.dll
 0001:0001a43e       ?sizePolicy@QWidget@@UBE?AVQSizePolicy@@XZ 1001b43e f   qt-mt323:qt-mt323.dll
 0001:0001a444       ?sort@QListView@@UAEXXZ    1001b444 f   qt-mt323:qt-mt323.dll
 0001:0001a44a       ?sort@QListViewItem@@UAEXXZ 1001b44a f   qt-mt323:qt-mt323.dll
 0001:0001a450       ?sortChildItems@QListViewItem@@UAEXH_N@Z 1001b450 f   qt-mt323:qt-mt323.dll
 0001:0001a456       ?spacerItem@QLayoutItem@@UAEPAVQSpacerItem@@XZ 1001b456 f   qt-mt323:qt-mt323.dll
 0001:0001a45c       ?spacerItem@QSpacerItem@@UAEPAV1@XZ 1001b45c f   qt-mt323:qt-mt323.dll
 0001:0001a462       ?startDrag@QListView@@MAEXXZ 1001b462 f   qt-mt323:qt-mt323.dll
 0001:0001a468       ?startRename@QListViewItem@@UAEXH@Z 1001b468 f   qt-mt323:qt-mt323.dll
 0001:0001a46e       ?styleChange@QFrame@@MAEXAAVQStyle@@@Z 1001b46e f   qt-mt323:qt-mt323.dll
 0001:0001a474       ?styleChange@QListView@@MAEXAAVQStyle@@@Z 1001b474 f   qt-mt323:qt-mt323.dll
 0001:0001a47a       ?styleChange@QPopupMenu@@MAEXAAVQStyle@@@Z 1001b47a f   qt-mt323:qt-mt323.dll
 0001:0001a480       ?styleChange@QTabWidget@@MAEXAAVQStyle@@@Z 1001b480 f   qt-mt323:qt-mt323.dll
 0001:0001a486       ?styleChange@QToolBar@@MAEXAAVQStyle@@@Z 1001b486 f   qt-mt323:qt-mt323.dll
 0001:0001a48c       ?styleChange@QWidget@@MAEXAAVQStyle@@@Z 1001b48c f   qt-mt323:qt-mt323.dll
 0001:0001a492       ?tabletEvent@QWidget@@MAEXPAVQTabletEvent@@@Z 1001b492 f   qt-mt323:qt-mt323.dll
 0001:0001a498       ?takeItem@QListView@@UAEXPAVQListViewItem@@@Z 1001b498 f   qt-mt323:qt-mt323.dll
 0001:0001a49e       ?takeItem@QListViewItem@@UAEXPAV1@@Z 1001b49e f   qt-mt323:qt-mt323.dll
 0001:0001a4a4       ?timerEvent@QObject@@MAEXPAVQTimerEvent@@@Z 1001b4a4 f   qt-mt323:qt-mt323.dll
 0001:0001a4aa       ?timerEvent@QPopupMenu@@MAEXPAVQTimerEvent@@@Z 1001b4aa f   qt-mt323:qt-mt323.dll
 0001:0001a4b0       ?undo@QLineEdit@@UAEXXZ    1001b4b0 f   qt-mt323:qt-mt323.dll
 0001:0001a4b6       ?undock@QDockWindow@@UAEXPAVQWidget@@@Z 1001b4b6 f   qt-mt323:qt-mt323.dll
 0001:0001a4bc       ?undock@QDockWindow@@UAEXXZ 1001b4bc f   qt-mt323:qt-mt323.dll
 0001:0001a4c2       ?unsetCursor@QWidget@@UAEXXZ 1001b4c2 f   qt-mt323:qt-mt323.dll
 0001:0001a4c8       ?updateItem@QPopupMenu@@UAEXH@Z 1001b4c8 f   qt-mt323:qt-mt323.dll
 0001:0001a4ce       ?updateMask@QPushButton@@MAEXXZ 1001b4ce f   qt-mt323:qt-mt323.dll
 0001:0001a4d4       ?updateMask@QTabWidget@@MAEXXZ 1001b4d4 f   qt-mt323:qt-mt323.dll
 0001:0001a4da       ?updateMask@QWidget@@MAEXXZ 1001b4da f   qt-mt323:qt-mt323.dll
 0001:0001a4e0       ?viewportContextMenuEvent@QScrollView@@MAEXPAVQContextMenuEvent@@@Z 1001b4e0 f   qt-mt323:qt-mt323.dll
 0001:0001a4e6       ?viewportDragEnterEvent@QScrollView@@MAEXPAVQDragEnterEvent@@@Z 1001b4e6 f   qt-mt323:qt-mt323.dll
 0001:0001a4ec       ?viewportDragLeaveEvent@QScrollView@@MAEXPAVQDragLeaveEvent@@@Z 1001b4ec f   qt-mt323:qt-mt323.dll
 0001:0001a4f2       ?viewportDragMoveEvent@QScrollView@@MAEXPAVQDragMoveEvent@@@Z 1001b4f2 f   qt-mt323:qt-mt323.dll
 0001:0001a4f8       ?viewportDropEvent@QScrollView@@MAEXPAVQDropEvent@@@Z 1001b4f8 f   qt-mt323:qt-mt323.dll
 0001:0001a4fe       ?viewportMouseDoubleClickEvent@QScrollView@@MAEXPAVQMouseEvent@@@Z 1001b4fe f   qt-mt323:qt-mt323.dll
 0001:0001a504       ?viewportMouseMoveEvent@QScrollView@@MAEXPAVQMouseEvent@@@Z 1001b504 f   qt-mt323:qt-mt323.dll
 0001:0001a50a       ?viewportMousePressEvent@QScrollView@@MAEXPAVQMouseEvent@@@Z 1001b50a f   qt-mt323:qt-mt323.dll
 0001:0001a510       ?viewportMouseReleaseEvent@QScrollView@@MAEXPAVQMouseEvent@@@Z 1001b510 f   qt-mt323:qt-mt323.dll
 0001:0001a516       ?viewportPaintEvent@QScrollView@@MAEXPAVQPaintEvent@@@Z 1001b516 f   qt-mt323:qt-mt323.dll
 0001:0001a51c       ?viewportResizeEvent@QListView@@MAEXPAVQResizeEvent@@@Z 1001b51c f   qt-mt323:qt-mt323.dll
 0001:0001a522       ?viewportWheelEvent@QScrollView@@MAEXPAVQWheelEvent@@@Z 1001b522 f   qt-mt323:qt-mt323.dll
 0001:0001a528       ?wheelEvent@QScrollView@@MAEXPAVQWheelEvent@@@Z 1001b528 f   qt-mt323:qt-mt323.dll
 0001:0001a52e       ?wheelEvent@QWidget@@MAEXPAVQWheelEvent@@@Z 1001b52e f   qt-mt323:qt-mt323.dll
 0001:0001a534       ?widget@QLayoutItem@@UAEPAVQWidget@@XZ 1001b534 f   qt-mt323:qt-mt323.dll
 0001:0001a53a       ?width@QListViewItem@@UBEHABVQFontMetrics@@PBVQListView@@H@Z 1001b53a f   qt-mt323:qt-mt323.dll
 0001:0001a540       ?winEvent@QWidget@@MAE_NPAUtagMSG@@@Z 1001b540 f   qt-mt323:qt-mt323.dll
 0001:0001a546       ?windowActivationChange@QLineEdit@@MAEX_N@Z 1001b546 f   qt-mt323:qt-mt323.dll
 0001:0001a54c       ?windowActivationChange@QListView@@MAEX_N@Z 1001b54c f   qt-mt323:qt-mt323.dll
 0001:0001a552       ?windowActivationChange@QWidget@@MAEX_N@Z 1001b552 f   qt-mt323:qt-mt323.dll
 0001:0001a558       ?write@QGList@@MBEAAVQDataStream@@AAV2@PAX@Z 1001b558 f   qt-mt323:qt-mt323.dll
 0001:0001a55e       ?accept@QDialog@@MAEXXZ    1001b55e f   qt-mt323:qt-mt323.dll
 0001:0001a564       ?closeEvent@QDialog@@MAEXPAVQCloseEvent@@@Z 1001b564 f   qt-mt323:qt-mt323.dll
 0001:0001a56a       ?contextMenuEvent@QDialog@@MAEXPAVQContextMenuEvent@@@Z 1001b56a f   qt-mt323:qt-mt323.dll
 0001:0001a570       ?done@QDialog@@MAEXH@Z     1001b570 f   qt-mt323:qt-mt323.dll
 0001:0001a576       ?eventFilter@QDialog@@MAE_NPAVQObject@@PAVQEvent@@@Z 1001b576 f   qt-mt323:qt-mt323.dll
 0001:0001a57c       ?hide@QDialog@@UAEXXZ      1001b57c f   qt-mt323:qt-mt323.dll
 0001:0001a582       ?keyPressEvent@QDialog@@MAEXPAVQKeyEvent@@@Z 1001b582 f   qt-mt323:qt-mt323.dll
 0001:0001a588       ?minimumSizeHint@QDialog@@UBE?AVQSize@@XZ 1001b588 f   qt-mt323:qt-mt323.dll
 0001:0001a58e       ?move@QDialog@@UAEXHH@Z    1001b58e f   qt-mt323:qt-mt323.dll
 0001:0001a594       ?reject@QDialog@@MAEXXZ    1001b594 f   qt-mt323:qt-mt323.dll
 0001:0001a59a       ?resize@QDialog@@UAEXHH@Z  1001b59a f   qt-mt323:qt-mt323.dll
 0001:0001a5a0       ?resizeEvent@QDialog@@MAEXPAVQResizeEvent@@@Z 1001b5a0 f   qt-mt323:qt-mt323.dll
 0001:0001a5a6       ?setGeometry@QDialog@@UAEXABVQRect@@@Z 1001b5a6 f   qt-mt323:qt-mt323.dll
 0001:0001a5ac       ?setGeometry@QDialog@@UAEXHHHH@Z 1001b5ac f   qt-mt323:qt-mt323.dll
 0001:0001a5b2       ?show@QDialog@@UAEXXZ      1001b5b2 f   qt-mt323:qt-mt323.dll
 0001:0001a5b8       ?sizeHint@QDialog@@UBE?AVQSize@@XZ 1001b5b8 f   qt-mt323:qt-mt323.dll
 0001:0001a5be       ?className@QDoubleValidator@@UBEPBDXZ 1001b5be f   qt-mt323:qt-mt323.dll
 0001:0001a5c4       ?fixup@QValidator@@UBEXAAVQString@@@Z 1001b5c4 f   qt-mt323:qt-mt323.dll
 0001:0001a5ca       ?height@QListBoxText@@UBEHPBVQListBox@@@Z 1001b5ca f   qt-mt323:qt-mt323.dll
 0001:0001a5d0       ?metaObject@QDoubleValidator@@UBEPAVQMetaObject@@XZ 1001b5d0 f   qt-mt323:qt-mt323.dll
 0001:0001a5d6       ?pixmap@QListBoxItem@@UBEPBVQPixmap@@XZ 1001b5d6 f   qt-mt323:qt-mt323.dll
 0001:0001a5dc       ?qt_cast@QDoubleValidator@@UAEPAXPBD@Z 1001b5dc f   qt-mt323:qt-mt323.dll
 0001:0001a5e2       ?qt_emit@QDoubleValidator@@UAE_NHPAUQUObject@@@Z 1001b5e2 f   qt-mt323:qt-mt323.dll
 0001:0001a5e8       ?qt_invoke@QDoubleValidator@@UAE_NHPAUQUObject@@@Z 1001b5e8 f   qt-mt323:qt-mt323.dll
 0001:0001a5ee       ?qt_property@QDoubleValidator@@UAE_NHHPAVQVariant@@@Z 1001b5ee f   qt-mt323:qt-mt323.dll
 0001:0001a5f4       ?rtti@QListBoxText@@UBEHXZ 1001b5f4 f   qt-mt323:qt-mt323.dll
 0001:0001a5fa       ?setRange@QDoubleValidator@@UAEXNNH@Z 1001b5fa f   qt-mt323:qt-mt323.dll
 0001:0001a600       ?setText@QListBoxItem@@MAEXABVQString@@@Z 1001b600 f   qt-mt323:qt-mt323.dll
 0001:0001a606       ?text@QListBoxItem@@UBE?AVQString@@XZ 1001b606 f   qt-mt323:qt-mt323.dll
 0001:0001a60c       ?validate@QDoubleValidator@@UBE?AW4State@QValidator@@AAVQString@@AAH@Z 1001b60c f   qt-mt323:qt-mt323.dll
 0001:0001a612       ?width@QListBoxText@@UBEHPBVQListBox@@@Z 1001b612 f   qt-mt323:qt-mt323.dll
 0001:0001a618       ?read@QGDict@@MAEAAVQDataStream@@AAV2@AAPAX@Z 1001b618 f   qt-mt323:qt-mt323.dll
 0001:0001a61e       ?write@QGDict@@MBEAAVQDataStream@@AAV2@PAX@Z 1001b61e f   qt-mt323:qt-mt323.dll
 0001:0001a624       ?addItem@QGridLayout@@UAEXPAVQLayoutItem@@@Z 1001b624 f   qt-mt323:qt-mt323.dll
 0001:0001a62a       ?childEvent@QGroupBox@@MAEXPAVQChildEvent@@@Z 1001b62a f   qt-mt323:qt-mt323.dll
 0001:0001a630       ?className@QButtonGroup@@UBEPBDXZ 1001b630 f   qt-mt323:qt-mt323.dll
 0001:0001a636       ?className@QCheckBox@@UBEPBDXZ 1001b636 f   qt-mt323:qt-mt323.dll
 0001:0001a63c       ?className@QGridLayout@@UBEPBDXZ 1001b63c f   qt-mt323:qt-mt323.dll
 0001:0001a642       ?className@QRadioButton@@UBEPBDXZ 1001b642 f   qt-mt323:qt-mt323.dll
 0001:0001a648       ?className@QSpinBox@@UBEPBDXZ 1001b648 f   qt-mt323:qt-mt323.dll
 0001:0001a64e       ?cleanText@QSpinBox@@UBE?AVQString@@XZ 1001b64e f   qt-mt323:qt-mt323.dll
 0001:0001a654       ?drawButton@QCheckBox@@MAEXPAVQPainter@@@Z 1001b654 f   qt-mt323:qt-mt323.dll
 0001:0001a65a       ?drawButton@QRadioButton@@MAEXPAVQPainter@@@Z 1001b65a f   qt-mt323:qt-mt323.dll
 0001:0001a660       ?drawButtonLabel@QCheckBox@@MAEXPAVQPainter@@@Z 1001b660 f   qt-mt323:qt-mt323.dll
 0001:0001a666       ?drawButtonLabel@QRadioButton@@MAEXPAVQPainter@@@Z 1001b666 f   qt-mt323:qt-mt323.dll
 0001:0001a66c       ?event@QButtonGroup@@MAE_NPAVQEvent@@@Z 1001b66c f   qt-mt323:qt-mt323.dll
 0001:0001a672       ?eventFilter@QSpinBox@@MAE_NPAVQObject@@PAVQEvent@@@Z 1001b672 f   qt-mt323:qt-mt323.dll
 0001:0001a678       ?expanding@QGridLayout@@UBE?AW4ExpandData@QSizePolicy@@XZ 1001b678 f   qt-mt323:qt-mt323.dll
 0001:0001a67e       ?focusInEvent@QButton@@MAEXPAVQFocusEvent@@@Z 1001b67e f   qt-mt323:qt-mt323.dll
 0001:0001a684       ?focusInEvent@QGroupBox@@MAEXPAVQFocusEvent@@@Z 1001b684 f   qt-mt323:qt-mt323.dll
 0001:0001a68a       ?focusOutEvent@QButton@@MAEXPAVQFocusEvent@@@Z 1001b68a f   qt-mt323:qt-mt323.dll
 0001:0001a690       ?fontChange@QGroupBox@@MAEXABVQFont@@@Z 1001b690 f   qt-mt323:qt-mt323.dll
 0001:0001a696       ?hasHeightForWidth@QGridLayout@@UBE_NXZ 1001b696 f   qt-mt323:qt-mt323.dll
 0001:0001a69c       ?heightForWidth@QGridLayout@@UBEHH@Z 1001b69c f   qt-mt323:qt-mt323.dll
 0001:0001a6a2       ?hitButton@QCheckBox@@MBE_NABVQPoint@@@Z 1001b6a2 f   qt-mt323:qt-mt323.dll
 0001:0001a6a8       ?hitButton@QRadioButton@@MBE_NABVQPoint@@@Z 1001b6a8 f   qt-mt323:qt-mt323.dll
 0001:0001a6ae       ?interpretText@QSpinBox@@MAEXXZ 1001b6ae f   qt-mt323:qt-mt323.dll
 0001:0001a6b4       ?invalidate@QGridLayout@@UAEXXZ 1001b6b4 f   qt-mt323:qt-mt323.dll
 0001:0001a6ba       ?iterator@QGridLayout@@UAE?AVQLayoutIterator@@XZ 1001b6ba f   qt-mt323:qt-mt323.dll
 0001:0001a6c0       ?leaveEvent@QSpinBox@@MAEXPAVQEvent@@@Z 1001b6c0 f   qt-mt323:qt-mt323.dll
 0001:0001a6c6       ?mapTextToValue@QSpinBox@@MAEHPA_N@Z 1001b6c6 f   qt-mt323:qt-mt323.dll
 0001:0001a6cc       ?mapValueToText@QSpinBox@@MAE?AVQString@@H@Z 1001b6cc f   qt-mt323:qt-mt323.dll
 0001:0001a6d2       ?maximumSize@QGridLayout@@UBE?AVQSize@@XZ 1001b6d2 f   qt-mt323:qt-mt323.dll
 0001:0001a6d8       ?metaObject@QButtonGroup@@UBEPAVQMetaObject@@XZ 1001b6d8 f   qt-mt323:qt-mt323.dll
 0001:0001a6de       ?metaObject@QCheckBox@@UBEPAVQMetaObject@@XZ 1001b6de f   qt-mt323:qt-mt323.dll
 0001:0001a6e4       ?metaObject@QGridLayout@@UBEPAVQMetaObject@@XZ 1001b6e4 f   qt-mt323:qt-mt323.dll
 0001:0001a6ea       ?metaObject@QRadioButton@@UBEPAVQMetaObject@@XZ 1001b6ea f   qt-mt323:qt-mt323.dll
 0001:0001a6f0       ?metaObject@QSpinBox@@UBEPAVQMetaObject@@XZ 1001b6f0 f   qt-mt323:qt-mt323.dll
 0001:0001a6f6       ?minimumSize@QGridLayout@@UBE?AVQSize@@XZ 1001b6f6 f   qt-mt323:qt-mt323.dll
 0001:0001a6fc       ?minimumSizeHint@QSpinBox@@UBE?AVQSize@@XZ 1001b6fc f   qt-mt323:qt-mt323.dll
 0001:0001a702       ?moveFocus@QButtonGroup@@UAEXH@Z 1001b702 f   qt-mt323:qt-mt323.dll
 0001:0001a708       ?paintEvent@QGroupBox@@MAEXPAVQPaintEvent@@@Z 1001b708 f   qt-mt323:qt-mt323.dll
 0001:0001a70e       ?prefix@QSpinBox@@UBE?AVQString@@XZ 1001b70e f   qt-mt323:qt-mt323.dll
 0001:0001a714       ?qt_cast@QButtonGroup@@UAEPAXPBD@Z 1001b714 f   qt-mt323:qt-mt323.dll
 0001:0001a71a       ?qt_cast@QCheckBox@@UAEPAXPBD@Z 1001b71a f   qt-mt323:qt-mt323.dll
 0001:0001a720       ?qt_cast@QGridLayout@@UAEPAXPBD@Z 1001b720 f   qt-mt323:qt-mt323.dll
 0001:0001a726       ?qt_cast@QRadioButton@@UAEPAXPBD@Z 1001b726 f   qt-mt323:qt-mt323.dll
 0001:0001a72c       ?qt_cast@QSpinBox@@UAEPAXPBD@Z 1001b72c f   qt-mt323:qt-mt323.dll
 0001:0001a732       ?qt_emit@QButtonGroup@@UAE_NHPAUQUObject@@@Z 1001b732 f   qt-mt323:qt-mt323.dll
 0001:0001a738       ?qt_emit@QCheckBox@@UAE_NHPAUQUObject@@@Z 1001b738 f   qt-mt323:qt-mt323.dll
 0001:0001a73e       ?qt_emit@QGridLayout@@UAE_NHPAUQUObject@@@Z 1001b73e f   qt-mt323:qt-mt323.dll
 0001:0001a744       ?qt_emit@QRadioButton@@UAE_NHPAUQUObject@@@Z 1001b744 f   qt-mt323:qt-mt323.dll
 0001:0001a74a       ?qt_emit@QSpinBox@@UAE_NHPAUQUObject@@@Z 1001b74a f   qt-mt323:qt-mt323.dll
 0001:0001a750       ?qt_invoke@QButtonGroup@@UAE_NHPAUQUObject@@@Z 1001b750 f   qt-mt323:qt-mt323.dll
 0001:0001a756       ?qt_invoke@QCheckBox@@UAE_NHPAUQUObject@@@Z 1001b756 f   qt-mt323:qt-mt323.dll
 0001:0001a75c       ?qt_invoke@QGridLayout@@UAE_NHPAUQUObject@@@Z 1001b75c f   qt-mt323:qt-mt323.dll
 0001:0001a762       ?qt_invoke@QRadioButton@@UAE_NHPAUQUObject@@@Z 1001b762 f   qt-mt323:qt-mt323.dll
 0001:0001a768       ?qt_invoke@QSpinBox@@UAE_NHPAUQUObject@@@Z 1001b768 f   qt-mt323:qt-mt323.dll
 0001:0001a76e       ?qt_property@QButtonGroup@@UAE_NHHPAVQVariant@@@Z 1001b76e f   qt-mt323:qt-mt323.dll
 0001:0001a774       ?qt_property@QCheckBox@@UAE_NHHPAVQVariant@@@Z 1001b774 f   qt-mt323:qt-mt323.dll
 0001:0001a77a       ?qt_property@QGridLayout@@UAE_NHHPAVQVariant@@@Z 1001b77a f   qt-mt323:qt-mt323.dll
 0001:0001a780       ?qt_property@QRadioButton@@UAE_NHHPAVQVariant@@@Z 1001b780 f   qt-mt323:qt-mt323.dll
 0001:0001a786       ?qt_property@QSpinBox@@UAE_NHHPAVQVariant@@@Z 1001b786 f   qt-mt323:qt-mt323.dll
 0001:0001a78c       ?rangeChange@QSpinBox@@MAEXXZ 1001b78c f   qt-mt323:qt-mt323.dll
 0001:0001a792       ?resizeEvent@QCheckBox@@MAEXPAVQResizeEvent@@@Z 1001b792 f   qt-mt323:qt-mt323.dll
 0001:0001a798       ?resizeEvent@QGroupBox@@MAEXPAVQResizeEvent@@@Z 1001b798 f   qt-mt323:qt-mt323.dll
 0001:0001a79e       ?resizeEvent@QRadioButton@@MAEXPAVQResizeEvent@@@Z 1001b79e f   qt-mt323:qt-mt323.dll
 0001:0001a7a4       ?resizeEvent@QSpinBox@@MAEXPAVQResizeEvent@@@Z 1001b7a4 f   qt-mt323:qt-mt323.dll
 0001:0001a7aa       ?selectAll@QSpinBox@@UAEXXZ 1001b7aa f   qt-mt323:qt-mt323.dll
 0001:0001a7b0       ?setAlignment@QGroupBox@@UAEXH@Z 1001b7b0 f   qt-mt323:qt-mt323.dll
 0001:0001a7b6       ?setButton@QButtonGroup@@UAEXH@Z 1001b7b6 f   qt-mt323:qt-mt323.dll
 0001:0001a7bc       ?setButtonSymbols@QSpinBox@@UAEXW4ButtonSymbols@1@@Z 1001b7bc f   qt-mt323:qt-mt323.dll
 0001:0001a7c2       ?setChecked@QRadioButton@@UAEX_N@Z 1001b7c2 f   qt-mt323:qt-mt323.dll
 0001:0001a7c8       ?setColStretch@QGridLayout@@UAEXHH@Z 1001b7c8 f   qt-mt323:qt-mt323.dll
 0001:0001a7ce       ?setColumnLayout@QGroupBox@@UAEXHW4Orientation@Qt@@@Z 1001b7ce f   qt-mt323:qt-mt323.dll
 0001:0001a7d4       ?setEnabled@QGroupBox@@UAEX_N@Z 1001b7d4 f   qt-mt323:qt-mt323.dll
 0001:0001a7da       ?setEnabled@QSpinBox@@UAEX_N@Z 1001b7da f   qt-mt323:qt-mt323.dll
 0001:0001a7e0       ?setExclusive@QButtonGroup@@UAEX_N@Z 1001b7e0 f   qt-mt323:qt-mt323.dll
 0001:0001a7e6       ?setGeometry@QGridLayout@@UAEXABVQRect@@@Z 1001b7e6 f   qt-mt323:qt-mt323.dll
 0001:0001a7ec       ?setPrefix@QSpinBox@@UAEXABVQString@@@Z 1001b7ec f   qt-mt323:qt-mt323.dll
 0001:0001a7f2       ?setRadioButtonExclusive@QButtonGroup@@UAEX_N@Z 1001b7f2 f   qt-mt323:qt-mt323.dll
 0001:0001a7f8       ?setRowStretch@QGridLayout@@UAEXHH@Z 1001b7f8 f   qt-mt323:qt-mt323.dll
 0001:0001a7fe       ?setSpecialValueText@QSpinBox@@UAEXABVQString@@@Z 1001b7fe f   qt-mt323:qt-mt323.dll
 0001:0001a804       ?setSuffix@QSpinBox@@UAEXABVQString@@@Z 1001b804 f   qt-mt323:qt-mt323.dll
 0001:0001a80a       ?setTitle@QGroupBox@@UAEXABVQString@@@Z 1001b80a f   qt-mt323:qt-mt323.dll
 0001:0001a810       ?setValidator@QSpinBox@@UAEXPBVQValidator@@@Z 1001b810 f   qt-mt323:qt-mt323.dll
 0001:0001a816       ?setValue@QSpinBox@@UAEXH@Z 1001b816 f   qt-mt323:qt-mt323.dll
 0001:0001a81c       ?setWrapping@QSpinBox@@UAEX_N@Z 1001b81c f   qt-mt323:qt-mt323.dll
 0001:0001a822       ?sizeHint@QCheckBox@@UBE?AVQSize@@XZ 1001b822 f   qt-mt323:qt-mt323.dll
 0001:0001a828       ?sizeHint@QGridLayout@@UBE?AVQSize@@XZ 1001b828 f   qt-mt323:qt-mt323.dll
 0001:0001a82e       ?sizeHint@QGroupBox@@UBE?AVQSize@@XZ 1001b82e f   qt-mt323:qt-mt323.dll
 0001:0001a834       ?sizeHint@QRadioButton@@UBE?AVQSize@@XZ 1001b834 f   qt-mt323:qt-mt323.dll
 0001:0001a83a       ?sizeHint@QSpinBox@@UBE?AVQSize@@XZ 1001b83a f   qt-mt323:qt-mt323.dll
 0001:0001a840       ?stepChange@QRangeControl@@MAEXXZ 1001b840 f   qt-mt323:qt-mt323.dll
 0001:0001a846       ?stepDown@QSpinBox@@UAEXXZ 1001b846 f   qt-mt323:qt-mt323.dll
 0001:0001a84c       ?stepUp@QSpinBox@@UAEXXZ   1001b84c f   qt-mt323:qt-mt323.dll
 0001:0001a852       ?styleChange@QSpinBox@@MAEXAAVQStyle@@@Z 1001b852 f   qt-mt323:qt-mt323.dll
 0001:0001a858       ?suffix@QSpinBox@@UBE?AVQString@@XZ 1001b858 f   qt-mt323:qt-mt323.dll
 0001:0001a85e       ?updateDisplay@QSpinBox@@MAEXXZ 1001b85e f   qt-mt323:qt-mt323.dll
 0001:0001a864       ?updateMask@QCheckBox@@MAEXXZ 1001b864 f   qt-mt323:qt-mt323.dll
 0001:0001a86a       ?updateMask@QRadioButton@@MAEXXZ 1001b86a f   qt-mt323:qt-mt323.dll
 0001:0001a870       ?valueChange@QSpinBox@@MAEXXZ 1001b870 f   qt-mt323:qt-mt323.dll
 0001:0001a876       ?wheelEvent@QSpinBox@@MAEXPAVQWheelEvent@@@Z 1001b876 f   qt-mt323:qt-mt323.dll
 0001:0001a87c       ?addNumber@QTimeEdit@@MAEXHH@Z 1001b87c f   qt-mt323:qt-mt323.dll
 0001:0001a882       ?append@QTextEdit@@UAEXABVQString@@@Z 1001b882 f   qt-mt323:qt-mt323.dll
 0001:0001a888       ?childEvent@QSplitter@@MAEXPAVQChildEvent@@@Z 1001b888 f   qt-mt323:qt-mt323.dll
 0001:0001a88e       ?childEvent@QWidgetStack@@MAEXPAVQChildEvent@@@Z 1001b88e f   qt-mt323:qt-mt323.dll
 0001:0001a894       ?className@QComboBox@@UBEPBDXZ 1001b894 f   qt-mt323:qt-mt323.dll
 0001:0001a89a       ?className@QGroupBox@@UBEPBDXZ 1001b89a f   qt-mt323:qt-mt323.dll
 0001:0001a8a0       ?className@QListBox@@UBEPBDXZ 1001b8a0 f   qt-mt323:qt-mt323.dll
 0001:0001a8a6       ?className@QSplitter@@UBEPBDXZ 1001b8a6 f   qt-mt323:qt-mt323.dll
 0001:0001a8ac       ?className@QTextEdit@@UBEPBDXZ 1001b8ac f   qt-mt323:qt-mt323.dll
 0001:0001a8b2       ?className@QTimeEdit@@UBEPBDXZ 1001b8b2 f   qt-mt323:qt-mt323.dll
 0001:0001a8b8       ?className@QWidgetStack@@UBEPBDXZ 1001b8b8 f   qt-mt323:qt-mt323.dll
 0001:0001a8be       ?clear@QTextEdit@@UAEXXZ   1001b8be f   qt-mt323:qt-mt323.dll
 0001:0001a8c4       ?clearParagraphBackground@QTextEdit@@UAEXH@Z 1001b8c4 f   qt-mt323:qt-mt323.dll
 0001:0001a8ca       ?clearSelection@QListBox@@UAEXXZ 1001b8ca f   qt-mt323:qt-mt323.dll
 0001:0001a8d0       ?contentsContextMenuEvent@QListBox@@MAEXPAVQContextMenuEvent@@@Z 1001b8d0 f   qt-mt323:qt-mt323.dll
 0001:0001a8d6       ?contentsContextMenuEvent@QTextEdit@@MAEXPAVQContextMenuEvent@@@Z 1001b8d6 f   qt-mt323:qt-mt323.dll
 0001:0001a8dc       ?contentsDragEnterEvent@QScrollView@@MAEXPAVQDragEnterEvent@@@Z 1001b8dc f   qt-mt323:qt-mt323.dll
 0001:0001a8e2       ?contentsDragEnterEvent@QTextEdit@@MAEXPAVQDragEnterEvent@@@Z 1001b8e2 f   qt-mt323:qt-mt323.dll
 0001:0001a8e8       ?contentsDragLeaveEvent@QScrollView@@MAEXPAVQDragLeaveEvent@@@Z 1001b8e8 f   qt-mt323:qt-mt323.dll
 0001:0001a8ee       ?contentsDragLeaveEvent@QTextEdit@@MAEXPAVQDragLeaveEvent@@@Z 1001b8ee f   qt-mt323:qt-mt323.dll
 0001:0001a8f4       ?contentsDragMoveEvent@QScrollView@@MAEXPAVQDragMoveEvent@@@Z 1001b8f4 f   qt-mt323:qt-mt323.dll
 0001:0001a8fa       ?contentsDragMoveEvent@QTextEdit@@MAEXPAVQDragMoveEvent@@@Z 1001b8fa f   qt-mt323:qt-mt323.dll
 0001:0001a900       ?contentsDropEvent@QScrollView@@MAEXPAVQDropEvent@@@Z 1001b900 f   qt-mt323:qt-mt323.dll
 0001:0001a906       ?contentsDropEvent@QTextEdit@@MAEXPAVQDropEvent@@@Z 1001b906 f   qt-mt323:qt-mt323.dll
 0001:0001a90c       ?contentsMouseDoubleClickEvent@QScrollView@@MAEXPAVQMouseEvent@@@Z 1001b90c f   qt-mt323:qt-mt323.dll
 0001:0001a912       ?contentsMouseDoubleClickEvent@QTextEdit@@MAEXPAVQMouseEvent@@@Z 1001b912 f   qt-mt323:qt-mt323.dll
 0001:0001a918       ?contentsMouseMoveEvent@QScrollView@@MAEXPAVQMouseEvent@@@Z 1001b918 f   qt-mt323:qt-mt323.dll
 0001:0001a91e       ?contentsMouseMoveEvent@QTextEdit@@MAEXPAVQMouseEvent@@@Z 1001b91e f   qt-mt323:qt-mt323.dll
 0001:0001a924       ?contentsMousePressEvent@QScrollView@@MAEXPAVQMouseEvent@@@Z 1001b924 f   qt-mt323:qt-mt323.dll
 0001:0001a92a       ?contentsMousePressEvent@QTextEdit@@MAEXPAVQMouseEvent@@@Z 1001b92a f   qt-mt323:qt-mt323.dll
 0001:0001a930       ?contentsMouseReleaseEvent@QScrollView@@MAEXPAVQMouseEvent@@@Z 1001b930 f   qt-mt323:qt-mt323.dll
 0001:0001a936       ?contentsMouseReleaseEvent@QTextEdit@@MAEXPAVQMouseEvent@@@Z 1001b936 f   qt-mt323:qt-mt323.dll
 0001:0001a93c       ?contentsWheelEvent@QTextEdit@@MAEXPAVQWheelEvent@@@Z 1001b93c f   qt-mt323:qt-mt323.dll
 0001:0001a942       ?copy@QTextEdit@@UAEXXZ    1001b942 f   qt-mt323:qt-mt323.dll
 0001:0001a948       ?createPopupMenu@QTextEdit@@MAEPAVQPopupMenu@@ABVQPoint@@@Z 1001b948 f   qt-mt323:qt-mt323.dll
 0001:0001a94e       ?createPopupMenu@QTextEdit@@MAEPAVQPopupMenu@@XZ 1001b94e f   qt-mt323:qt-mt323.dll
 0001:0001a954       ?cut@QTextEdit@@UAEXXZ     1001b954 f   qt-mt323:qt-mt323.dll
 0001:0001a95a       ?del@QTextEdit@@UAEXXZ     1001b95a f   qt-mt323:qt-mt323.dll
 0001:0001a960       ?doChangeInterval@QTextEdit@@MAEXXZ 1001b960 f   qt-mt323:qt-mt323.dll
 0001:0001a966       ?doKeyboardAction@QTextEdit@@UAEXW4KeyboardAction@1@@Z 1001b966 f   qt-mt323:qt-mt323.dll
 0001:0001a96c       ?drawContents@QTextEdit@@EAEXPAVQPainter@@@Z 1001b96c f   qt-mt323:qt-mt323.dll
 0001:0001a972       ?drawContents@QTextEdit@@MAEXPAVQPainter@@HHHH@Z 1001b972 f   qt-mt323:qt-mt323.dll
 0001:0001a978       ?drawContentsOffset@QScrollView@@MAEXPAVQPainter@@HHHHHH@Z 1001b978 f   qt-mt323:qt-mt323.dll
 0001:0001a97e       ?drawSplitter@QSplitter@@MAEXPAVQPainter@@HHHH@Z 1001b97e f   qt-mt323:qt-mt323.dll
 0001:0001a984       ?emitHighlighted@QTextEdit@@EAEXABVQString@@@Z 1001b984 f   qt-mt323:qt-mt323.dll
 0001:0001a98a       ?emitLinkClicked@QTextEdit@@EAEXABVQString@@@Z 1001b98a f   qt-mt323:qt-mt323.dll
 0001:0001a990       ?ensureCurrentVisible@QListBox@@UAEXXZ 1001b990 f   qt-mt323:qt-mt323.dll
 0001:0001a996       ?ensureCursorVisible@QTextEdit@@UAEXXZ 1001b996 f   qt-mt323:qt-mt323.dll
 0001:0001a99c       ?event@QGroupBox@@MAE_NPAVQEvent@@@Z 1001b99c f   qt-mt323:qt-mt323.dll
 0001:0001a9a2       ?event@QSplitter@@MAE_NPAVQEvent@@@Z 1001b9a2 f   qt-mt323:qt-mt323.dll
 0001:0001a9a8       ?event@QTextEdit@@MAE_NPAVQEvent@@@Z 1001b9a8 f   qt-mt323:qt-mt323.dll
 0001:0001a9ae       ?event@QTimeEdit@@MAE_NPAVQEvent@@@Z 1001b9ae f   qt-mt323:qt-mt323.dll
 0001:0001a9b4       ?eventFilter@QComboBox@@UAE_NPAVQObject@@PAVQEvent@@@Z 1001b9b4 f   qt-mt323:qt-mt323.dll
 0001:0001a9ba       ?eventFilter@QListBox@@MAE_NPAVQObject@@PAVQEvent@@@Z 1001b9ba f   qt-mt323:qt-mt323.dll
 0001:0001a9c0       ?eventFilter@QTextEdit@@UAE_NPAVQObject@@PAVQEvent@@@Z 1001b9c0 f   qt-mt323:qt-mt323.dll
 0001:0001a9c6       ?find@QTextEdit@@UAE_NABVQString@@_N11PAH2@Z 1001b9c6 f   qt-mt323:qt-mt323.dll
 0001:0001a9cc       ?focusInEvent@QComboBox@@MAEXPAVQFocusEvent@@@Z 1001b9cc f   qt-mt323:qt-mt323.dll
 0001:0001a9d2       ?focusInEvent@QListBox@@MAEXPAVQFocusEvent@@@Z 1001b9d2 f   qt-mt323:qt-mt323.dll
 0001:0001a9d8       ?focusNextPrevChild@QTextEdit@@MAE_N_N@Z 1001b9d8 f   qt-mt323:qt-mt323.dll
 0001:0001a9de       ?focusOutEvent@QComboBox@@MAEXPAVQFocusEvent@@@Z 1001b9de f   qt-mt323:qt-mt323.dll
 0001:0001a9e4       ?focusOutEvent@QListBox@@MAEXPAVQFocusEvent@@@Z 1001b9e4 f   qt-mt323:qt-mt323.dll
 0001:0001a9ea       ?frameChanged@QWidgetStack@@MAEXXZ 1001b9ea f   qt-mt323:qt-mt323.dll
 0001:0001a9f0       ?getFormat@QTextEdit@@UAE_NHHPAVQFont@@PAVQColor@@PAW4VerticalAlignment@1@@Z 1001b9f0 f   qt-mt323:qt-mt323.dll
 0001:0001a9f6       ?getParagraphFormat@QTextEdit@@UAE_NHPAVQFont@@PAVQColor@@PAW4VerticalAlignment@1@PAHPAW4DisplayMode@QStyleSheetItem@@PAW4ListStyle@6@3@Z 1001b9f6 f   qt-mt323:qt-mt323.dll
 0001:0001a9fc       ?heightForWidth@QTextEdit@@UBEHH@Z 1001b9fc f   qt-mt323:qt-mt323.dll
 0001:0001aa02       ?imComposeEvent@QTextEdit@@MAEXPAVQIMEvent@@@Z 1001ba02 f   qt-mt323:qt-mt323.dll
 0001:0001aa08       ?imEndEvent@QTextEdit@@MAEXPAVQIMEvent@@@Z 1001ba08 f   qt-mt323:qt-mt323.dll
 0001:0001aa0e       ?imStartEvent@QTextEdit@@MAEXPAVQIMEvent@@@Z 1001ba0e f   qt-mt323:qt-mt323.dll
 0001:0001aa14       ?indent@QTextEdit@@UAEXXZ  1001ba14 f   qt-mt323:qt-mt323.dll
 0001:0001aa1a       ?insert@QTextEdit@@UAEXABVQString@@_N11@Z 1001ba1a f   qt-mt323:qt-mt323.dll
 0001:0001aa20       ?insertAt@QTextEdit@@UAEXABVQString@@HH@Z 1001ba20 f   qt-mt323:qt-mt323.dll
 0001:0001aa26       ?insertParagraph@QTextEdit@@UAEXABVQString@@H@Z 1001ba26 f   qt-mt323:qt-mt323.dll
 0001:0001aa2c       ?invertSelection@QListBox@@UAEXXZ 1001ba2c f   qt-mt323:qt-mt323.dll
 0001:0001aa32       ?keyPressEvent@QComboBox@@MAEXPAVQKeyEvent@@@Z 1001ba32 f   qt-mt323:qt-mt323.dll
 0001:0001aa38       ?keyPressEvent@QListBox@@MAEXPAVQKeyEvent@@@Z 1001ba38 f   qt-mt323:qt-mt323.dll
 0001:0001aa3e       ?keyPressEvent@QTextEdit@@MAEXPAVQKeyEvent@@@Z 1001ba3e f   qt-mt323:qt-mt323.dll
 0001:0001aa44       ?linksEnabled@QTextEdit@@EBE_NXZ 1001ba44 f   qt-mt323:qt-mt323.dll
 0001:0001aa4a       ?metaObject@QComboBox@@UBEPAVQMetaObject@@XZ 1001ba4a f   qt-mt323:qt-mt323.dll
 0001:0001aa50       ?metaObject@QGroupBox@@UBEPAVQMetaObject@@XZ 1001ba50 f   qt-mt323:qt-mt323.dll
 0001:0001aa56       ?metaObject@QListBox@@UBEPAVQMetaObject@@XZ 1001ba56 f   qt-mt323:qt-mt323.dll
 0001:0001aa5c       ?metaObject@QSplitter@@UBEPAVQMetaObject@@XZ 1001ba5c f   qt-mt323:qt-mt323.dll
 0001:0001aa62       ?metaObject@QTextEdit@@UBEPAVQMetaObject@@XZ 1001ba62 f   qt-mt323:qt-mt323.dll
 0001:0001aa68       ?metaObject@QTimeEdit@@UBEPAVQMetaObject@@XZ 1001ba68 f   qt-mt323:qt-mt323.dll
 0001:0001aa6e       ?metaObject@QWidgetStack@@UBEPAVQMetaObject@@XZ 1001ba6e f   qt-mt323:qt-mt323.dll
 0001:0001aa74       ?minimumSizeHint@QListBox@@UBE?AVQSize@@XZ 1001ba74 f   qt-mt323:qt-mt323.dll
 0001:0001aa7a       ?minimumSizeHint@QScrollView@@UBE?AVQSize@@XZ 1001ba7a f   qt-mt323:qt-mt323.dll
 0001:0001aa80       ?minimumSizeHint@QSplitter@@UBE?AVQSize@@XZ 1001ba80 f   qt-mt323:qt-mt323.dll
 0001:0001aa86       ?minimumSizeHint@QTimeEdit@@UBE?AVQSize@@XZ 1001ba86 f   qt-mt323:qt-mt323.dll
 0001:0001aa8c       ?minimumSizeHint@QWidgetStack@@UBE?AVQSize@@XZ 1001ba8c f   qt-mt323:qt-mt323.dll
 0001:0001aa92       ?mouseDoubleClickEvent@QComboBox@@MAEXPAVQMouseEvent@@@Z 1001ba92 f   qt-mt323:qt-mt323.dll
 0001:0001aa98       ?mouseDoubleClickEvent@QListBox@@MAEXPAVQMouseEvent@@@Z 1001ba98 f   qt-mt323:qt-mt323.dll
 0001:0001aa9e       ?mouseMoveEvent@QComboBox@@MAEXPAVQMouseEvent@@@Z 1001ba9e f   qt-mt323:qt-mt323.dll
 0001:0001aaa4       ?mouseMoveEvent@QListBox@@MAEXPAVQMouseEvent@@@Z 1001baa4 f   qt-mt323:qt-mt323.dll
 0001:0001aaaa       ?mousePressEvent@QComboBox@@MAEXPAVQMouseEvent@@@Z 1001baaa f   qt-mt323:qt-mt323.dll
 0001:0001aab0       ?mousePressEvent@QListBox@@MAEXPAVQMouseEvent@@@Z 1001bab0 f   qt-mt323:qt-mt323.dll
 0001:0001aab6       ?mouseReleaseEvent@QComboBox@@MAEXPAVQMouseEvent@@@Z 1001bab6 f   qt-mt323:qt-mt323.dll
 0001:0001aabc       ?mouseReleaseEvent@QListBox@@MAEXPAVQMouseEvent@@@Z 1001babc f   qt-mt323:qt-mt323.dll
 0001:0001aac2       ?moveCursor@QTextEdit@@UAEXW4CursorAction@1@_N@Z 1001bac2 f   qt-mt323:qt-mt323.dll
 0001:0001aac8       ?outOfRange@QTimeEdit@@MBE_NHHH@Z 1001bac8 f   qt-mt323:qt-mt323.dll
 0001:0001aace       ?paintCell@QListBox@@MAEXPAVQPainter@@HH@Z 1001bace f   qt-mt323:qt-mt323.dll
 0001:0001aad4       ?paintEvent@QComboBox@@MAEXPAVQPaintEvent@@@Z 1001bad4 f   qt-mt323:qt-mt323.dll
 0001:0001aada       ?paste@QTextEdit@@UAEXXZ   1001bada f   qt-mt323:qt-mt323.dll
 0001:0001aae0       ?pasteSubType@QTextEdit@@UAEXABVQCString@@@Z 1001bae0 f   qt-mt323:qt-mt323.dll
 0001:0001aae6       ?placeCursor@QTextEdit@@UAEXABVQPoint@@PAVQTextCursor@@@Z 1001bae6 f   qt-mt323:qt-mt323.dll
 0001:0001aaec       ?polish@QTextEdit@@UAEXXZ  1001baec f   qt-mt323:qt-mt323.dll
 0001:0001aaf2       ?popup@QComboBox@@UAEXXZ   1001baf2 f   qt-mt323:qt-mt323.dll
 0001:0001aaf8       ?qt_cast@QComboBox@@UAEPAXPBD@Z 1001baf8 f   qt-mt323:qt-mt323.dll
 0001:0001aafe       ?qt_cast@QGroupBox@@UAEPAXPBD@Z 1001bafe f   qt-mt323:qt-mt323.dll
 0001:0001ab04       ?qt_cast@QListBox@@UAEPAXPBD@Z 1001bb04 f   qt-mt323:qt-mt323.dll
 0001:0001ab0a       ?qt_cast@QSplitter@@UAEPAXPBD@Z 1001bb0a f   qt-mt323:qt-mt323.dll
 0001:0001ab10       ?qt_cast@QTextEdit@@UAEPAXPBD@Z 1001bb10 f   qt-mt323:qt-mt323.dll
 0001:0001ab16       ?qt_cast@QTimeEdit@@UAEPAXPBD@Z 1001bb16 f   qt-mt323:qt-mt323.dll
 0001:0001ab1c       ?qt_cast@QWidgetStack@@UAEPAXPBD@Z 1001bb1c f   qt-mt323:qt-mt323.dll
 0001:0001ab22       ?qt_emit@QComboBox@@UAE_NHPAUQUObject@@@Z 1001bb22 f   qt-mt323:qt-mt323.dll
 0001:0001ab28       ?qt_emit@QGroupBox@@UAE_NHPAUQUObject@@@Z 1001bb28 f   qt-mt323:qt-mt323.dll
 0001:0001ab2e       ?qt_emit@QListBox@@UAE_NHPAUQUObject@@@Z 1001bb2e f   qt-mt323:qt-mt323.dll
 0001:0001ab34       ?qt_emit@QSplitter@@UAE_NHPAUQUObject@@@Z 1001bb34 f   qt-mt323:qt-mt323.dll
 0001:0001ab3a       ?qt_emit@QTextEdit@@UAE_NHPAUQUObject@@@Z 1001bb3a f   qt-mt323:qt-mt323.dll
 0001:0001ab40       ?qt_emit@QTimeEdit@@UAE_NHPAUQUObject@@@Z 1001bb40 f   qt-mt323:qt-mt323.dll
 0001:0001ab46       ?qt_emit@QWidgetStack@@UAE_NHPAUQUObject@@@Z 1001bb46 f   qt-mt323:qt-mt323.dll
 0001:0001ab4c       ?qt_invoke@QComboBox@@UAE_NHPAUQUObject@@@Z 1001bb4c f   qt-mt323:qt-mt323.dll
 0001:0001ab52       ?qt_invoke@QGroupBox@@UAE_NHPAUQUObject@@@Z 1001bb52 f   qt-mt323:qt-mt323.dll
 0001:0001ab58       ?qt_invoke@QListBox@@UAE_NHPAUQUObject@@@Z 1001bb58 f   qt-mt323:qt-mt323.dll
 0001:0001ab5e       ?qt_invoke@QSplitter@@UAE_NHPAUQUObject@@@Z 1001bb5e f   qt-mt323:qt-mt323.dll
 0001:0001ab64       ?qt_invoke@QTextEdit@@UAE_NHPAUQUObject@@@Z 1001bb64 f   qt-mt323:qt-mt323.dll
 0001:0001ab6a       ?qt_invoke@QTimeEdit@@UAE_NHPAUQUObject@@@Z 1001bb6a f   qt-mt323:qt-mt323.dll
 0001:0001ab70       ?qt_invoke@QWidgetStack@@UAE_NHPAUQUObject@@@Z 1001bb70 f   qt-mt323:qt-mt323.dll
 0001:0001ab76       ?qt_property@QComboBox@@UAE_NHHPAVQVariant@@@Z 1001bb76 f   qt-mt323:qt-mt323.dll
 0001:0001ab7c       ?qt_property@QGroupBox@@UAE_NHHPAVQVariant@@@Z 1001bb7c f   qt-mt323:qt-mt323.dll
 0001:0001ab82       ?qt_property@QListBox@@UAE_NHHPAVQVariant@@@Z 1001bb82 f   qt-mt323:qt-mt323.dll
 0001:0001ab88       ?qt_property@QSplitter@@UAE_NHHPAVQVariant@@@Z 1001bb88 f   qt-mt323:qt-mt323.dll
 0001:0001ab8e       ?qt_property@QTextEdit@@UAE_NHHPAVQVariant@@@Z 1001bb8e f   qt-mt323:qt-mt323.dll
 0001:0001ab94       ?qt_property@QTimeEdit@@UAE_NHHPAVQVariant@@@Z 1001bb94 f   qt-mt323:qt-mt323.dll
 0001:0001ab9a       ?qt_property@QWidgetStack@@UAE_NHHPAVQVariant@@@Z 1001bb9a f   qt-mt323:qt-mt323.dll
 0001:0001aba0       ?redo@QTextEdit@@UAEXXZ    1001bba0 f   qt-mt323:qt-mt323.dll
 0001:0001aba6       ?removeLastNumber@QTimeEdit@@MAEXH@Z 1001bba6 f   qt-mt323:qt-mt323.dll
 0001:0001abac       ?removeParagraph@QTextEdit@@UAEXH@Z 1001bbac f   qt-mt323:qt-mt323.dll
 0001:0001abb2       ?removeSelectedText@QTextEdit@@UAEXH@Z 1001bbb2 f   qt-mt323:qt-mt323.dll
 0001:0001abb8       ?removeSelection@QTextEdit@@UAEXH@Z 1001bbb8 f   qt-mt323:qt-mt323.dll
 0001:0001abbe       ?resetFormat@QTextEdit@@UAEXXZ 1001bbbe f   qt-mt323:qt-mt323.dll
 0001:0001abc4       ?resizeEvent@QComboBox@@MAEXPAVQResizeEvent@@@Z 1001bbc4 f   qt-mt323:qt-mt323.dll
 0001:0001abca       ?resizeEvent@QListBox@@MAEXPAVQResizeEvent@@@Z 1001bbca f   qt-mt323:qt-mt323.dll
 0001:0001abd0       ?resizeEvent@QSplitter@@MAEXPAVQResizeEvent@@@Z 1001bbd0 f   qt-mt323:qt-mt323.dll
 0001:0001abd6       ?resizeEvent@QTextEdit@@MAEXPAVQResizeEvent@@@Z 1001bbd6 f   qt-mt323:qt-mt323.dll
 0001:0001abdc       ?resizeEvent@QTimeEdit@@MAEXPAVQResizeEvent@@@Z 1001bbdc f   qt-mt323:qt-mt323.dll
 0001:0001abe2       ?resizeEvent@QWidgetStack@@MAEXPAVQResizeEvent@@@Z 1001bbe2 f   qt-mt323:qt-mt323.dll
 0001:0001abe8       ?scrollToAnchor@QTextEdit@@UAEXABVQString@@@Z 1001bbe8 f   qt-mt323:qt-mt323.dll
 0001:0001abee       ?scrollToBottom@QTextEdit@@UAEXXZ 1001bbee f   qt-mt323:qt-mt323.dll
 0001:0001abf4       ?sectionFormattedText@QTimeEdit@@MAE?AVQString@@H@Z 1001bbf4 f   qt-mt323:qt-mt323.dll
 0001:0001abfa       ?selectAll@QListBox@@UAEX_N@Z 1001bbfa f   qt-mt323:qt-mt323.dll
 0001:0001ac00       ?selectAll@QTextEdit@@UAEX_N@Z 1001bc00 f   qt-mt323:qt-mt323.dll
 0001:0001ac06       ?setAlignment@QTextEdit@@UAEXH@Z 1001bc06 f   qt-mt323:qt-mt323.dll
 0001:0001ac0c       ?setAutoAdvance@QTimeEdit@@UAEX_N@Z 1001bc0c f   qt-mt323:qt-mt323.dll
 0001:0001ac12       ?setAutoCompletion@QComboBox@@UAEX_N@Z 1001bc12 f   qt-mt323:qt-mt323.dll
 0001:0001ac18       ?setAutoResize@QComboBox@@UAEX_N@Z 1001bc18 f   qt-mt323:qt-mt323.dll
 0001:0001ac1e       ?setBold@QTextEdit@@UAEX_N@Z 1001bc1e f   qt-mt323:qt-mt323.dll
 0001:0001ac24       ?setBottomItem@QListBox@@UAEXH@Z 1001bc24 f   qt-mt323:qt-mt323.dll
 0001:0001ac2a       ?setChildGeometries@QWidgetStack@@MAEXXZ 1001bc2a f   qt-mt323:qt-mt323.dll
 0001:0001ac30       ?setColor@QTextEdit@@UAEXABVQColor@@@Z 1001bc30 f   qt-mt323:qt-mt323.dll
 0001:0001ac36       ?setColumnMode@QListBox@@UAEXH@Z 1001bc36 f   qt-mt323:qt-mt323.dll
 0001:0001ac3c       ?setColumnMode@QListBox@@UAEXW4LayoutMode@1@@Z 1001bc3c f   qt-mt323:qt-mt323.dll
 0001:0001ac42       ?setContentsPos@QScrollView@@UAEXHH@Z 1001bc42 f   qt-mt323:qt-mt323.dll
 0001:0001ac48       ?setCurrentFont@QTextEdit@@UAEXABVQFont@@@Z 1001bc48 f   qt-mt323:qt-mt323.dll
 0001:0001ac4e       ?setCurrentItem@QComboBox@@UAEXH@Z 1001bc4e f   qt-mt323:qt-mt323.dll
 0001:0001ac54       ?setCurrentItem@QListBox@@UAEXH@Z 1001bc54 f   qt-mt323:qt-mt323.dll
 0001:0001ac5a       ?setCurrentItem@QListBox@@UAEXPAVQListBoxItem@@@Z 1001bc5a f   qt-mt323:qt-mt323.dll
 0001:0001ac60       ?setCurrentText@QComboBox@@UAEXABVQString@@@Z 1001bc60 f   qt-mt323:qt-mt323.dll
 0001:0001ac66       ?setCursorPosition@QTextEdit@@UAEXHH@Z 1001bc66 f   qt-mt323:qt-mt323.dll
 0001:0001ac6c       ?setEditText@QComboBox@@UAEXABVQString@@@Z 1001bc6c f   qt-mt323:qt-mt323.dll
 0001:0001ac72       ?setEnabled@QComboBox@@UAEX_N@Z 1001bc72 f   qt-mt323:qt-mt323.dll
 0001:0001ac78       ?setEnabled@QTextEdit@@UAEX_N@Z 1001bc78 f   qt-mt323:qt-mt323.dll
 0001:0001ac7e       ?setFamily@QTextEdit@@UAEXABVQString@@@Z 1001bc7e f   qt-mt323:qt-mt323.dll
 0001:0001ac84       ?setFocusSection@QTimeEdit@@MAE_NH@Z 1001bc84 f   qt-mt323:qt-mt323.dll
 0001:0001ac8a       ?setFont@QComboBox@@UAEXABVQFont@@@Z 1001bc8a f   qt-mt323:qt-mt323.dll
 0001:0001ac90       ?setFont@QListBox@@UAEXABVQFont@@@Z 1001bc90 f   qt-mt323:qt-mt323.dll
 0001:0001ac96       ?setFont@QTextEdit@@UAEXABVQFont@@@Z 1001bc96 f   qt-mt323:qt-mt323.dll
 0001:0001ac9c       ?setFormat@QTextEdit@@UAEXPAVQTextFormat@@H@Z 1001bc9c f   qt-mt323:qt-mt323.dll
 0001:0001aca2       ?setFrameRect@QWidgetStack@@UAEXABVQRect@@@Z 1001bca2 f   qt-mt323:qt-mt323.dll
 0001:0001aca8       ?setHour@QTimeEdit@@MAEXH@Z 1001bca8 f   qt-mt323:qt-mt323.dll
 0001:0001acae       ?setInsertionPolicy@QComboBox@@UAEXW4Policy@1@@Z 1001bcae f   qt-mt323:qt-mt323.dll
 0001:0001acb4       ?setItalic@QTextEdit@@UAEX_N@Z 1001bcb4 f   qt-mt323:qt-mt323.dll
 0001:0001acba       ?setLineEdit@QComboBox@@UAEXPAVQLineEdit@@@Z 1001bcba f   qt-mt323:qt-mt323.dll
 0001:0001acc0       ?setLinkUnderline@QTextEdit@@UAEX_N@Z 1001bcc0 f   qt-mt323:qt-mt323.dll
 0001:0001acc6       ?setListBox@QComboBox@@UAEXPAVQListBox@@@Z 1001bcc6 f   qt-mt323:qt-mt323.dll
 0001:0001accc       ?setMaxCount@QComboBox@@UAEXH@Z 1001bccc f   qt-mt323:qt-mt323.dll
 0001:0001acd2       ?setMaxValue@QTimeEdit@@UAEXABVQTime@@@Z 1001bcd2 f   qt-mt323:qt-mt323.dll
 0001:0001acd8       ?setMimeSourceFactory@QTextEdit@@UAEXPAVQMimeSourceFactory@@@Z 1001bcd8 f   qt-mt323:qt-mt323.dll
 0001:0001acde       ?setMinValue@QTimeEdit@@UAEXABVQTime@@@Z 1001bcde f   qt-mt323:qt-mt323.dll
 0001:0001ace4       ?setMinute@QTimeEdit@@MAEXH@Z 1001bce4 f   qt-mt323:qt-mt323.dll
 0001:0001acea       ?setModified@QTextEdit@@UAEX_N@Z 1001bcea f   qt-mt323:qt-mt323.dll
 0001:0001acf0       ?setOpaqueResize@QSplitter@@UAEX_N@Z 1001bcf0 f   qt-mt323:qt-mt323.dll
 0001:0001acf6       ?setOrientation@QSplitter@@UAEXW4Orientation@Qt@@@Z 1001bcf6 f   qt-mt323:qt-mt323.dll
 0001:0001acfc       ?setOverwriteMode@QTextEdit@@UAEX_N@Z 1001bcfc f   qt-mt323:qt-mt323.dll
 0001:0001ad02       ?setPalette@QComboBox@@UAEXABVQPalette@@@Z 1001bd02 f   qt-mt323:qt-mt323.dll
 0001:0001ad08       ?setPalette@QTextEdit@@UAEXABVQPalette@@@Z 1001bd08 f   qt-mt323:qt-mt323.dll
 0001:0001ad0e       ?setPaper@QTextEdit@@UAEXABVQBrush@@@Z 1001bd0e f   qt-mt323:qt-mt323.dll
 0001:0001ad14       ?setParagType@QTextEdit@@UAEXW4DisplayMode@QStyleSheetItem@@W4ListStyle@3@@Z 1001bd14 f   qt-mt323:qt-mt323.dll
 0001:0001ad1a       ?setParagraphBackgroundColor@QTextEdit@@UAEXHABVQColor@@@Z 1001bd1a f   qt-mt323:qt-mt323.dll
 0001:0001ad20       ?setPointSize@QTextEdit@@UAEXH@Z 1001bd20 f   qt-mt323:qt-mt323.dll
 0001:0001ad26       ?setRange@QTimeEdit@@UAEXABVQTime@@0@Z 1001bd26 f   qt-mt323:qt-mt323.dll
 0001:0001ad2c       ?setReadOnly@QTextEdit@@UAEX_N@Z 1001bd2c f   qt-mt323:qt-mt323.dll
 0001:0001ad32       ?setResizeMode@QSplitter@@UAEXPAVQWidget@@W4ResizeMode@1@@Z 1001bd32 f   qt-mt323:qt-mt323.dll
 0001:0001ad38       ?setRowMode@QListBox@@UAEXH@Z 1001bd38 f   qt-mt323:qt-mt323.dll
 0001:0001ad3e       ?setRowMode@QListBox@@UAEXW4LayoutMode@1@@Z 1001bd3e f   qt-mt323:qt-mt323.dll
 0001:0001ad44       ?setRubberband@QSplitter@@MAEXH@Z 1001bd44 f   qt-mt323:qt-mt323.dll
 0001:0001ad4a       ?setSecond@QTimeEdit@@MAEXH@Z 1001bd4a f   qt-mt323:qt-mt323.dll
 0001:0001ad50       ?setSelected@QListBox@@UAEXPAVQListBoxItem@@_N@Z 1001bd50 f   qt-mt323:qt-mt323.dll
 0001:0001ad56       ?setSelection@QTextEdit@@UAEXHHHHH@Z 1001bd56 f   qt-mt323:qt-mt323.dll
 0001:0001ad5c       ?setSelectionAttributes@QTextEdit@@UAEXHABVQColor@@_N@Z 1001bd5c f   qt-mt323:qt-mt323.dll
 0001:0001ad62       ?setSelectionMode@QListBox@@UAEXW4SelectionMode@1@@Z 1001bd62 f   qt-mt323:qt-mt323.dll
 0001:0001ad68       ?setSeparator@QTimeEdit@@UAEXABVQString@@@Z 1001bd68 f   qt-mt323:qt-mt323.dll
 0001:0001ad6e       ?setSizeLimit@QComboBox@@UAEXH@Z 1001bd6e f   qt-mt323:qt-mt323.dll
 0001:0001ad74       ?setStyleSheet@QTextEdit@@UAEXPAVQStyleSheet@@@Z 1001bd74 f   qt-mt323:qt-mt323.dll
 0001:0001ad7a       ?setTabStopWidth@QTextEdit@@UAEXH@Z 1001bd7a f   qt-mt323:qt-mt323.dll
 0001:0001ad80       ?setText@QTextEdit@@UAEXABVQString@@0@Z 1001bd80 f   qt-mt323:qt-mt323.dll
 0001:0001ad86       ?setTextFormat@QTextEdit@@UAEXW4TextFormat@Qt@@@Z 1001bd86 f   qt-mt323:qt-mt323.dll
 0001:0001ad8c       ?setTime@QTimeEdit@@UAEXABVQTime@@@Z 1001bd8c f   qt-mt323:qt-mt323.dll
 0001:0001ad92       ?setTopItem@QListBox@@UAEXH@Z 1001bd92 f   qt-mt323:qt-mt323.dll
 0001:0001ad98       ?setUnderline@QTextEdit@@UAEX_N@Z 1001bd98 f   qt-mt323:qt-mt323.dll
 0001:0001ad9e       ?setUndoDepth@QTextEdit@@UAEXH@Z 1001bd9e f   qt-mt323:qt-mt323.dll
 0001:0001ada4       ?setUndoRedoEnabled@QTextEdit@@UAEX_N@Z 1001bda4 f   qt-mt323:qt-mt323.dll
 0001:0001adaa       ?setValidator@QComboBox@@UAEXPBVQValidator@@@Z 1001bdaa f   qt-mt323:qt-mt323.dll
 0001:0001adb0       ?setVariableHeight@QListBox@@UAEX_N@Z 1001bdb0 f   qt-mt323:qt-mt323.dll
 0001:0001adb6       ?setVariableWidth@QListBox@@UAEX_N@Z 1001bdb6 f   qt-mt323:qt-mt323.dll
 0001:0001adbc       ?setVerticalAlignment@QTextEdit@@UAEXW4VerticalAlignment@1@@Z 1001bdbc f   qt-mt323:qt-mt323.dll
 0001:0001adc2       ?setWordWrap@QTextEdit@@UAEXW4WordWrap@1@@Z 1001bdc2 f   qt-mt323:qt-mt323.dll
 0001:0001adc8       ?setWrapColumnOrWidth@QTextEdit@@UAEXH@Z 1001bdc8 f   qt-mt323:qt-mt323.dll
 0001:0001adce       ?setWrapPolicy@QTextEdit@@UAEXW4WrapPolicy@1@@Z 1001bdce f   qt-mt323:qt-mt323.dll
 0001:0001add4       ?show@QScrollView@@UAEXXZ  1001bdd4 f   qt-mt323:qt-mt323.dll
 0001:0001adda       ?show@QWidgetStack@@UAEXXZ 1001bdda f   qt-mt323:qt-mt323.dll
 0001:0001ade0       ?showEvent@QListBox@@MAEXPAVQShowEvent@@@Z 1001bde0 f   qt-mt323:qt-mt323.dll
 0001:0001ade6       ?sizeHint@QComboBox@@UBE?AVQSize@@XZ 1001bde6 f   qt-mt323:qt-mt323.dll
 0001:0001adec       ?sizeHint@QListBox@@UBE?AVQSize@@XZ 1001bdec f   qt-mt323:qt-mt323.dll
 0001:0001adf2       ?sizeHint@QSplitter@@UBE?AVQSize@@XZ 1001bdf2 f   qt-mt323:qt-mt323.dll
 0001:0001adf8       ?sizeHint@QTextEdit@@UBE?AVQSize@@XZ 1001bdf8 f   qt-mt323:qt-mt323.dll
 0001:0001adfe       ?sizeHint@QTimeEdit@@UBE?AVQSize@@XZ 1001bdfe f   qt-mt323:qt-mt323.dll
 0001:0001ae04       ?sizeHint@QWidgetStack@@UBE?AVQSize@@XZ 1001be04 f   qt-mt323:qt-mt323.dll
 0001:0001ae0a       ?stepDown@QTimeEdit@@MAEXXZ 1001be0a f   qt-mt323:qt-mt323.dll
 0001:0001ae10       ?stepUp@QTimeEdit@@MAEXXZ  1001be10 f   qt-mt323:qt-mt323.dll
 0001:0001ae16       ?styleChange@QComboBox@@MAEXAAVQStyle@@@Z 1001be16 f   qt-mt323:qt-mt323.dll
 0001:0001ae1c       ?styleChange@QScrollView@@UAEXAAVQStyle@@@Z 1001be1c f   qt-mt323:qt-mt323.dll
 0001:0001ae22       ?styleChange@QSplitter@@MAEXAAVQStyle@@@Z 1001be22 f   qt-mt323:qt-mt323.dll
 0001:0001ae28       ?sync@QTextEdit@@UAEXXZ    1001be28 f   qt-mt323:qt-mt323.dll
 0001:0001ae2e       ?timerEvent@QTimeEdit@@MAEXPAVQTimerEvent@@@Z 1001be2e f   qt-mt323:qt-mt323.dll
 0001:0001ae34       ?undo@QTextEdit@@UAEXXZ    1001be34 f   qt-mt323:qt-mt323.dll
 0001:0001ae3a       ?updateMask@QComboBox@@MAEXXZ 1001be3a f   qt-mt323:qt-mt323.dll
 0001:0001ae40       ?viewportPaintEvent@QListBox@@UAEXPAVQPaintEvent@@@Z 1001be40 f   qt-mt323:qt-mt323.dll
 0001:0001ae46       ?viewportResizeEvent@QScrollView@@MAEXPAVQResizeEvent@@@Z 1001be46 f   qt-mt323:qt-mt323.dll
 0001:0001ae4c       ?viewportResizeEvent@QTextEdit@@MAEXPAVQResizeEvent@@@Z 1001be4c f   qt-mt323:qt-mt323.dll
 0001:0001ae52       ?wheelEvent@QComboBox@@MAEXPAVQWheelEvent@@@Z 1001be52 f   qt-mt323:qt-mt323.dll
 0001:0001ae58       ?windowActivationChange@QListBox@@MAEX_N@Z 1001be58 f   qt-mt323:qt-mt323.dll
 0001:0001ae5e       ?windowActivationChange@QTextEdit@@MAEX_N@Z 1001be5e f   qt-mt323:qt-mt323.dll
 0001:0001ae64       ?zoomIn@QTextEdit@@UAEXH@Z 1001be64 f   qt-mt323:qt-mt323.dll
 0001:0001ae6a       ?zoomIn@QTextEdit@@UAEXXZ  1001be6a f   qt-mt323:qt-mt323.dll
 0001:0001ae70       ?zoomOut@QTextEdit@@UAEXH@Z 1001be70 f   qt-mt323:qt-mt323.dll
 0001:0001ae76       ?zoomOut@QTextEdit@@UAEXXZ 1001be76 f   qt-mt323:qt-mt323.dll
 0001:0001ae7c       ?zoomTo@QTextEdit@@UAEXH@Z 1001be7c f   qt-mt323:qt-mt323.dll
 0001:0001ae82       ?className@CAlm_sys_select@@UBEPBDXZ 1001be82 f   alm_sys_select:alm_sys_select.dll
 0001:0001ae88       ?metaObject@CAlm_sys_select@@UBEPAVQMetaObject@@XZ 1001be88 f   alm_sys_select:alm_sys_select.dll
 0001:0001ae8e       ?qt_cast@CAlm_sys_select@@UAEPAXPBD@Z 1001be8e f   alm_sys_select:alm_sys_select.dll
 0001:0001ae94       ?qt_emit@CAlm_sys_select@@UAE_NHPAUQUObject@@@Z 1001be94 f   alm_sys_select:alm_sys_select.dll
 0001:0001ae9a       ?qt_invoke@CAlm_sys_select@@UAE_NHPAUQUObject@@@Z 1001be9a f   alm_sys_select:alm_sys_select.dll
 0001:0001aea0       ?qt_property@CAlm_sys_select@@UAE_NHHPAVQVariant@@@Z 1001bea0 f   alm_sys_select:alm_sys_select.dll
 0001:0001aea6       ??0config_mb4@@QAE@IPAVQWidget@@PBD@Z 1001bea6 f   cfg_widgets001:config_mb4impl.obj
 0001:0001af05       ??1config_mb4@@UAE@XZ      1001bf05 f   cfg_widgets001:config_mb4impl.obj
 0001:0001af18       ??_Econfig_mb4@@WCI@AEPAXI@Z 1001bf18 f i cfg_widgets001:config_mb4impl.obj
 0001:0001af20       ??_Econfig_mb4@@UAEPAXI@Z  1001bf20 f i cfg_widgets001:config_mb4impl.obj
 0001:0001af20       ??_Gconfig_mb4@@UAEPAXI@Z  1001bf20 f i cfg_widgets001:config_mb4impl.obj
 0001:0001af3f       ?CreatePanel@config_mb4@@AAEXI@Z 1001bf3f f   cfg_widgets001:config_mb4impl.obj
 0001:0001b39c       ?buttonClicked@config_mb4@@QAEXH@Z 1001c39c f   cfg_widgets001:config_mb4impl.obj
 0001:0001b3b5       ?closeEvent@config_mb4@@EAEXPAVQCloseEvent@@@Z 1001c3b5 f   cfg_widgets001:config_mb4impl.obj
 0001:0001b3cc       ?metaObject@config_mb4@@UBEPAVQMetaObject@@XZ 1001c3cc f i cfg_widgets001:config_mb4impl.obj
 0001:0001b3d1       ?setIcon@config_mb4@@QAEXW4Icon@1@@Z 1001c3d1 f   cfg_widgets001:config_mb4impl.obj
 0001:0001b4d2       ?setIconPixmap@config_mb4@@QAEXABVQPixmap@@@Z 1001c4d2 f   cfg_widgets001:config_mb4impl.obj
 0001:0001b51c       ?setText@config_mb4@@QAEXVQString@@@Z 1001c51c f   cfg_widgets001:config_mb4impl.obj
 0001:0001b553       ?loadState@cfg_Settings@@SA?AVQString@@ABV2@@Z 1001c553 f   cfg_widgets001:cfg_Settings.obj
 0001:0001b5e5       ?loadState@cfg_Settings@@SAXAAVQPoint@@AAVQSize@@AA_NABVQString@@@Z 1001c5e5 f   cfg_widgets001:cfg_Settings.obj
 0001:0001b6de       ?loadState@cfg_Settings@@SAXQAVQListView@@ABVQString@@@Z 1001c6de f   cfg_widgets001:cfg_Settings.obj
 0001:0001b7db       ?loadState@cfg_Settings@@SAXQAVQSplitter@@ABVQString@@@Z 1001c7db f   cfg_widgets001:cfg_Settings.obj
 0001:0001b8d9       ?saveState@cfg_Settings@@SAXABVQPoint@@ABVQSize@@AB_NABVQString@@@Z 1001c8d9 f   cfg_widgets001:cfg_Settings.obj
 0001:0001b9f3       ?saveState@cfg_Settings@@SAXABVQString@@0@Z 1001c9f3 f   cfg_widgets001:cfg_Settings.obj
 0001:0001ba6f       ?saveState@cfg_Settings@@SAXQBVQListView@@ABVQString@@@Z 1001ca6f f   cfg_widgets001:cfg_Settings.obj
 0001:0001bb47       ?saveState@cfg_Settings@@SAXQBVQSplitter@@ABVQString@@@Z 1001cb47 f   cfg_widgets001:cfg_Settings.obj
 0001:0001bc24       ??0cfg_ListView@@QAE@ABV0@@Z 1001cc24 f i cfg_widgets001:cfg_ListView.obj
 0001:0001bc6e       ??0cfg_ListView@@QAE@PAVQWidget@@PBD@Z 1001cc6e f   cfg_widgets001:cfg_ListView.obj
 0001:0001bd2c       ??1cfg_ListView@@UAE@XZ    1001cd2c f   cfg_widgets001:cfg_ListView.obj
 0001:0001bd82       ??4cfg_ListView@@QAEAAV0@ABV0@@Z 1001cd82 f i cfg_widgets001:cfg_ListView.obj
 0001:0001bdd7       ??_Ecfg_ListView@@UAEPAXI@Z 1001cdd7 f i cfg_widgets001:cfg_ListView.obj
 0001:0001be24       ??_Ecfg_ListView@@WCI@AEPAXI@Z 1001ce24 f i cfg_widgets001:cfg_ListView.obj
 0001:0001be2c       ??_Fcfg_ListView@@QAEXXZ   1001ce2c f i cfg_widgets001:cfg_ListView.obj
 0001:0001be36       ?clearUndo@cfg_ListView@@AAEXXZ 1001ce36 f   cfg_widgets001:cfg_ListView.obj
 0001:0001be74       ?clipBoardDataChanged@cfg_ListView@@IAEXXZ 1001ce74 f   cfg_widgets001:cfg_ListView.obj
 0001:0001bec8       ?copyToClipboard@cfg_ListView@@QAEXXZ 1001cec8 f   cfg_widgets001:cfg_ListView.obj
 0001:0001bff7       ?deleteItems@cfg_ListView@@QAEXXZ 1001cff7 f   cfg_widgets001:cfg_ListView.obj
 0001:0001c0e2       ?insertData@cfg_ListView@@QAEXXZ 1001d0e2 f   cfg_widgets001:cfg_ListView.obj
 0001:0001c27d       ?metaObject@cfg_ListView@@UBEPAVQMetaObject@@XZ 1001d27d f i cfg_widgets001:cfg_ListView.obj
 0001:0001c282       ?newItem@cfg_ListView@@MAEPAVQListViewItem@@PAVQListView@@PAV2@@Z 1001d282 f   cfg_widgets001:cfg_ListView.obj
 0001:0001c2c5       ?replaceData@cfg_ListView@@QAEXXZ 1001d2c5 f   cfg_widgets001:cfg_ListView.obj
 0001:0001c603       ?undoPaste@cfg_ListView@@QAEXXZ 1001d603 f   cfg_widgets001:cfg_ListView.obj
 0001:0001c66e       ?updateEntry@cfg_ListView@@AAEPAVQListViewItem@@QAV2@ABVQString@@_N@Z 1001d66e f   cfg_widgets001:cfg_ListView.obj
 0001:0001c7aa       ?validateRow@cfg_ListView@@MAEHPAVQListViewItem@@@Z 1001d7aa f   cfg_widgets001:cfg_ListView.obj
 0001:0001c7bc       ??0cfg_Table@@QAE@ABV0@@Z  1001d7bc f i cfg_widgets001:cfg_Table.obj
 0001:0001c7ee       ??0cfg_Table@@QAE@PAVQWidget@@PBD@Z 1001d7ee f   cfg_widgets001:cfg_Table.obj
 0001:0001c848       ??1cfg_Table@@UAE@XZ       1001d848 f i cfg_widgets001:cfg_Table.obj
 0001:0001c84e       ??4cfg_Table@@QAEAAV0@ABV0@@Z 1001d84e f i cfg_widgets001:cfg_Table.obj
 0001:0001c873       ??_EQStringList@@QAEPAXI@Z 1001d873 f i cfg_widgets001:cfg_Table.obj
 0001:0001c8bf       ??_Ecfg_Table@@UAEPAXI@Z   1001d8bf f i cfg_widgets001:cfg_Table.obj
 0001:0001c90d       ??_Ecfg_Table@@WCI@AEPAXI@Z 1001d90d f i cfg_widgets001:cfg_Table.obj
 0001:0001c915       ??_Fcfg_Table@@QAEXXZ      1001d915 f i cfg_widgets001:cfg_Table.obj
 0001:0001c91f       ?clipBoardDataChanged@cfg_Table@@IAEXXZ 1001d91f f   cfg_widgets001:cfg_Table.obj
 0001:0001c973       ?copyToClipboard@cfg_Table@@QAEXXZ 1001d973 f   cfg_widgets001:cfg_Table.obj
 0001:0001ca82       ?deleteItems@cfg_Table@@QAEXXZ 1001da82 f   cfg_widgets001:cfg_Table.obj
 0001:0001cb0e       ?fillUndoBuffer@cfg_Table@@AAEXXZ 1001db0e f   cfg_widgets001:cfg_Table.obj
 0001:0001cc83       ?metaObject@cfg_Table@@UBEPAVQMetaObject@@XZ 1001dc83 f i cfg_widgets001:cfg_Table.obj
 0001:0001cc88       ?pasteClipboard@cfg_Table@@QAEXXZ 1001dc88 f   cfg_widgets001:cfg_Table.obj
 0001:0001d07b       ?qObject@cfg_Table@@QAEPAVQObject@@XZ 1001e07b f i cfg_widgets001:cfg_Table.obj
 0001:0001d07b       ?qObject@cfg_ListView@@QAEPAVQObject@@XZ 1001e07b f i cfg_widgets001:cfg_ListView.obj
 0001:0001d07e       ?undoPaste@cfg_Table@@QAEXXZ 1001e07e f   cfg_widgets001:cfg_Table.obj
 0001:0001d1b0       ?validateRow@cfg_Table@@MAEHH@Z 1001e1b0 f   cfg_widgets001:cfg_Table.obj
 0001:0001d1c2       ?className@config_mb4@@UBEPBDXZ 1001e1c2 f   cfg_widgets001:moc_config_mb4impl.obj
 0001:0001d1c8       ?qt_cast@config_mb4@@UAEPAXPBD@Z 1001e1c8 f   cfg_widgets001:moc_config_mb4impl.obj
 0001:0001d1f6       ?qt_emit@multiInputBase@@UAE_NHPAUQUObject@@@Z 1001e1f6 f   moc_multiinput.obj
 0001:0001d1f6       ?qt_emit@config_mb4@@UAE_NHPAUQUObject@@@Z 1001e1f6 f   cfg_widgets001:moc_config_mb4impl.obj
 0001:0001d1f6       ?qt_emit@CheckContDialogBase@@UAE_NHPAUQUObject@@@Z 1001e1f6 f   moc_checkcontributiondialog.obj
 0001:0001d1f6       ?qt_emit@singleInputBase@@UAE_NHPAUQUObject@@@Z 1001e1f6 f   moc_singleinput.obj
 0001:0001d1f6       ?qt_emit@LatchAckDialogBase@@UAE_NHPAUQUObject@@@Z 1001e1f6 f   moc_latchackdialog.obj
 0001:0001d1f6       ?qt_emit@template_dialogBase@@UAE_NHPAUQUObject@@@Z 1001e1f6 f   moc_template_dialog.obj
 0001:0001d200       ?qt_invoke@config_mb4@@UAE_NHPAUQUObject@@@Z 1001e200 f   cfg_widgets001:moc_config_mb4impl.obj
 0001:0001d235       ?qt_property@template_dialogBase@@UAE_NHHPAVQVariant@@@Z 1001e235 f   moc_template_dialog.obj
 0001:0001d235       ?qt_property@multiInputBase@@UAE_NHHPAVQVariant@@@Z 1001e235 f   moc_multiinput.obj
 0001:0001d235       ?qt_property@LatchAckDialogBase@@UAE_NHHPAVQVariant@@@Z 1001e235 f   moc_latchackdialog.obj
 0001:0001d235       ?qt_property@singleInputBase@@UAE_NHHPAVQVariant@@@Z 1001e235 f   moc_singleinput.obj
 0001:0001d235       ?qt_property@CheckContDialogBase@@UAE_NHHPAVQVariant@@@Z 1001e235 f   moc_checkcontributiondialog.obj
 0001:0001d235       ?qt_property@config_mb4@@UAE_NHHPAVQVariant@@@Z 1001e235 f   cfg_widgets001:moc_config_mb4impl.obj
 0001:0001d23f       ?staticMetaObject@config_mb4@@SAPAVQMetaObject@@XZ 1001e23f f   cfg_widgets001:moc_config_mb4impl.obj
 0001:0001d2b8       ?className@cfg_ListView@@UBEPBDXZ 1001e2b8 f   cfg_widgets001:moc_cfg_ListView.obj
 0001:0001d2be       ?clipboardDataValid@cfg_ListView@@IAEX_N@Z 1001e2be f   cfg_widgets001:moc_cfg_ListView.obj
 0001:0001d2de       ?dataPasted@cfg_ListView@@IAEXXZ 1001e2de f   cfg_widgets001:moc_cfg_ListView.obj
 0001:0001d2f3       ?qt_cast@cfg_ListView@@UAEPAXPBD@Z 1001e2f3 f   cfg_widgets001:moc_cfg_ListView.obj
 0001:0001d321       ?qt_emit@cfg_ListView@@UAE_NHPAUQUObject@@@Z 1001e321 f   cfg_widgets001:moc_cfg_ListView.obj
 0001:0001d365       ?qt_invoke@cfg_ListView@@UAE_NHPAUQUObject@@@Z 1001e365 f   cfg_widgets001:moc_cfg_ListView.obj
 0001:0001d3c9       ?qt_property@cfg_ListView@@UAE_NHHPAVQVariant@@@Z 1001e3c9 f   cfg_widgets001:moc_cfg_ListView.obj
 0001:0001d3d3       ?staticMetaObject@cfg_ListView@@SAPAVQMetaObject@@XZ 1001e3d3 f   cfg_widgets001:moc_cfg_ListView.obj
 0001:0001d452       ?tr@cfg_ListView@@SA?AVQString@@PBD0@Z 1001e452 f   cfg_widgets001:moc_cfg_ListView.obj
 0001:0001d495       ?trUtf8@cfg_ListView@@SA?AVQString@@PBD0@Z 1001e495 f   cfg_widgets001:moc_cfg_ListView.obj
 0001:0001d4d8       ?className@cfg_Table@@UBEPBDXZ 1001e4d8 f   cfg_widgets001:moc_cfg_Table.obj
 0001:0001d4de       ?clipboardDataValid@cfg_Table@@IAEX_N@Z 1001e4de f   cfg_widgets001:moc_cfg_Table.obj
 0001:0001d4fe       ?dataPasted@cfg_Table@@IAEXXZ 1001e4fe f   cfg_widgets001:moc_cfg_Table.obj
 0001:0001d513       ?qt_cast@cfg_Table@@UAEPAXPBD@Z 1001e513 f   cfg_widgets001:moc_cfg_Table.obj
 0001:0001d541       ?qt_emit@cfg_Table@@UAE_NHPAUQUObject@@@Z 1001e541 f   cfg_widgets001:moc_cfg_Table.obj
 0001:0001d585       ?qt_invoke@cfg_Table@@UAE_NHPAUQUObject@@@Z 1001e585 f   cfg_widgets001:moc_cfg_Table.obj
 0001:0001d5df       ?qt_property@cfg_Table@@UAE_NHHPAVQVariant@@@Z 1001e5df f   cfg_widgets001:moc_cfg_Table.obj
 0001:0001d5e9       ?staticMetaObject@cfg_Table@@SAPAVQMetaObject@@XZ 1001e5e9 f   cfg_widgets001:moc_cfg_Table.obj
 0001:0001d668       ?tr@cfg_Table@@SA?AVQString@@PBD0@Z 1001e668 f   cfg_widgets001:moc_cfg_Table.obj
 0001:0001d6ab       ?trUtf8@cfg_Table@@SA?AVQString@@PBD0@Z 1001e6ab f   cfg_widgets001:moc_cfg_Table.obj
 0001:0001d6ee       ??2@YAPAXI@Z               1001e6ee f   MSVCRT:MSVCR120.dll
 0001:0001d6f4       ??3@YAXPAX@Z               1001e6f4 f   MSVCRT:MSVCR120.dll
 0001:0001d6fa       ___atonexitinit            1001e6fa f   MSVCRT:atonexit.obj
 0001:0001d736       __onexit                   1001e736 f   MSVCRT:atonexit.obj
 0001:0001d7df       _atexit                    1001e7df f   MSVCRT:atonexit.obj
 0001:0001d7f4       @__security_check_cookie@4 1001e7f4 f   MSVCRT:secchk.obj
 0001:0001d804       __CxxThrowException@8      1001e804 f   MSVCRT:MSVCR120.dll
 0001:0001d80a       __EH_epilog3               1001e80a f   MSVCRT:ehprolg3.obj
 0001:0001d81e       __EH_epilog3_GS            1001e81e f   MSVCRT:ehprolg3.obj
 0001:0001d82d       __EH_prolog3               1001e82d f   MSVCRT:ehprolg3.obj
 0001:0001d860       __EH_prolog3_GS            1001e860 f   MSVCRT:ehprolg3.obj
 0001:0001d896       __EH_prolog3_catch         1001e896 f   MSVCRT:ehprolg3.obj
 0001:0001d8cc       ___CxxFrameHandler3        1001e8cc f   MSVCRT:MSVCR120.dll
 0001:0001d8d2       ___RTDynamicCast           1001e8d2 f   MSVCRT:MSVCR120.dll
 0001:0001d8d8       ??_Etype_info@@UAEPAXI@Z   1001e8d8 f i MSVCRT:ti_inst.obj
 0001:0001d930       __purecall                 1001e930 f   MSVCRT:MSVCR120.dll
 0001:0001d936       ??_L@YGXPAXIHP6EX0@Z1@Z    1001e936 f   MSVCRT:ehvecctr.obj
 0001:0001d998       ??_M@YGXPAXIHP6EX0@Z@Z     1001e998 f   MSVCRT:ehvecdtr.obj
 0001:0001da07       ?__ArrayUnwind@@YGXPAXIHP6EX0@Z@Z 1001ea07 f   MSVCRT:ehvecdtr.obj
 0001:0001dab1       __CRT_INIT@12              1001eab1 f   MSVCRT:crtdll.obj
 0001:0001dca8       __DllMainCRTStartup@12     1001eca8 f   MSVCRT:crtdll.obj
 0001:0001ddfe       __lock                     1001edfe f   MSVCRT:MSVCR120.dll
 0001:0001de04       __unlock                   1001ee04 f   MSVCRT:MSVCR120.dll
 0001:0001de0a       ___dllonexit               1001ee0a f   MSVCRT:MSVCR120.dll
 0001:0001de10       __SEH_prolog4              1001ee10 f   MSVCRT:sehprolg4.obj
 0001:0001de55       __SEH_epilog4              1001ee55 f   MSVCRT:sehprolg4.obj
 0001:0001de69       __except_handler4          1001ee69 f   MSVCRT:chandler4gs.obj
 0001:0001de8c       ___raise_securityfailure   1001ee8c f   MSVCRT:gs_report.obj
 0001:0001dec9       ___report_gsfailure        1001eec9 f   MSVCRT:gs_report.obj
 0001:0001dfc4       ??1type_info@@UAE@XZ       1001efc4 f   MSVCRT:MSVCR120.dll
 0001:0001dfca       ?terminate@@YAXXZ          1001efca f   MSVCRT:MSVCR120.dll
 0001:0001dfd0       ___CppXcptFilter           1001efd0 f   MSVCRT:MSVCR120.dll
 0001:0001dfd6       __amsg_exit                1001efd6 f   MSVCRT:MSVCR120.dll
 0001:0001dfe0       __FindPESection            1001efe0 f   MSVCRT:pesect.obj
 0001:0001e030       __IsNonwritableInCurrentImage 1001f030 f   MSVCRT:pesect.obj
 0001:0001e0f0       __ValidateImageBase        1001f0f0 f   MSVCRT:pesect.obj
 0001:0001e121       ___security_init_cookie    1001f121 f   MSVCRT:gs_support.obj
 0001:0001e1bd       _DllMain@12                1001f1bd f   MSVCRT:dllmain.obj
 0001:0001e1df       __RTC_Initialize           1001f1df f   MSVCRT:initsect.obj
 0001:0001e1ff       __RTC_Terminate            1001f1ff f   MSVCRT:initsect.obj
 0001:0001e220       __initterm                 1001f220 f   MSVCRT:MSVCR120.dll
 0001:0001e226       __initterm_e               1001f226 f   MSVCRT:MSVCR120.dll
 0001:0001e22c       ___clean_type_info_names   1001f22c f   MSVCRT:tncleanup.obj
 0001:0001e238       __except_handler4_common   1001f238 f   MSVCRT:MSVCR120.dll
 0001:0001e23e       __crt_debugger_hook        1001f23e f   MSVCRT:MSVCR120.dll
 0001:0001e244       ___crtUnhandledException   1001f244 f   MSVCRT:MSVCR120.dll
 0001:0001e24a       ___crtTerminateProcess     1001f24a f   MSVCRT:MSVCR120.dll
 0001:0001e250       ___clean_type_info_names_internal 1001f250 f   MSVCRT:MSVCR120.dll
 0001:0001e256       ?activateNextCell@QTable@@MAEXXZ 1001f256 f   qt-mt323:qt-mt323.dll
 0001:0001e25c       ?addSelection@QTable@@UAEHABVQTableSelection@@@Z 1001f25c f   qt-mt323:qt-mt323.dll
 0001:0001e262       ?adjustColumn@QTable@@UAEXH@Z 1001f262 f   qt-mt323:qt-mt323.dll
 0001:0001e268       ?adjustRow@QTable@@UAEXH@Z 1001f268 f   qt-mt323:qt-mt323.dll
 0001:0001e26e       ?beginEdit@QTable@@MAEPAVQWidget@@HH_N@Z 1001f26e f   qt-mt323:qt-mt323.dll
 0001:0001e274       ?cellGeometry@QTable@@UBE?AVQRect@@HH@Z 1001f274 f   qt-mt323:qt-mt323.dll
 0001:0001e27a       ?cellRect@QTable@@UBE?AVQRect@@HH@Z 1001f27a f   qt-mt323:qt-mt323.dll
 0001:0001e280       ?cellWidget@QTable@@UBEPAVQWidget@@HH@Z 1001f280 f   qt-mt323:qt-mt323.dll
 0001:0001e286       ?clearCell@QTable@@UAEXHH@Z 1001f286 f   qt-mt323:qt-mt323.dll
 0001:0001e28c       ?clearCellWidget@QTable@@UAEXHH@Z 1001f28c f   qt-mt323:qt-mt323.dll
 0001:0001e292       ?columnAt@QTable@@UBEHH@Z  1001f292 f   qt-mt323:qt-mt323.dll
 0001:0001e298       ?columnClicked@QTable@@MAEXH@Z 1001f298 f   qt-mt323:qt-mt323.dll
 0001:0001e29e       ?columnIndexChanged@QTable@@MAEXHHH@Z 1001f29e f   qt-mt323:qt-mt323.dll
 0001:0001e2a4       ?columnPos@QTable@@UBEHH@Z 1001f2a4 f   qt-mt323:qt-mt323.dll
 0001:0001e2aa       ?columnWidth@QTable@@UBEHH@Z 1001f2aa f   qt-mt323:qt-mt323.dll
 0001:0001e2b0       ?columnWidthChanged@QTable@@MAEXH@Z 1001f2b0 f   qt-mt323:qt-mt323.dll
 0001:0001e2b6       ?contentsContextMenuEvent@QTable@@MAEXPAVQContextMenuEvent@@@Z 1001f2b6 f   qt-mt323:qt-mt323.dll
 0001:0001e2bc       ?contentsDragEnterEvent@QTable@@MAEXPAVQDragEnterEvent@@@Z 1001f2bc f   qt-mt323:qt-mt323.dll
 0001:0001e2c2       ?contentsDragLeaveEvent@QTable@@MAEXPAVQDragLeaveEvent@@@Z 1001f2c2 f   qt-mt323:qt-mt323.dll
 0001:0001e2c8       ?contentsDragMoveEvent@QTable@@MAEXPAVQDragMoveEvent@@@Z 1001f2c8 f   qt-mt323:qt-mt323.dll
 0001:0001e2ce       ?contentsDropEvent@QTable@@MAEXPAVQDropEvent@@@Z 1001f2ce f   qt-mt323:qt-mt323.dll
 0001:0001e2d4       ?contentsMouseDoubleClickEvent@QTable@@MAEXPAVQMouseEvent@@@Z 1001f2d4 f   qt-mt323:qt-mt323.dll
 0001:0001e2da       ?contentsMouseMoveEvent@QTable@@MAEXPAVQMouseEvent@@@Z 1001f2da f   qt-mt323:qt-mt323.dll
 0001:0001e2e0       ?contentsMousePressEvent@QTable@@MAEXPAVQMouseEvent@@@Z 1001f2e0 f   qt-mt323:qt-mt323.dll
 0001:0001e2e6       ?contentsMouseReleaseEvent@QTable@@MAEXPAVQMouseEvent@@@Z 1001f2e6 f   qt-mt323:qt-mt323.dll
 0001:0001e2ec       ?createEditor@QTable@@MBEPAVQWidget@@HH_N@Z 1001f2ec f   qt-mt323:qt-mt323.dll
 0001:0001e2f2       ?currentSelection@QTable@@UBEHXZ 1001f2f2 f   qt-mt323:qt-mt323.dll
 0001:0001e2f8       ?dragObject@QTable@@MAEPAVQDragObject@@XZ 1001f2f8 f   qt-mt323:qt-mt323.dll
 0001:0001e2fe       ?drawContents@QTable@@EAEXPAVQPainter@@@Z 1001f2fe f   qt-mt323:qt-mt323.dll
 0001:0001e304       ?drawContents@QTable@@MAEXPAVQPainter@@HHHH@Z 1001f304 f   qt-mt323:qt-mt323.dll
 0001:0001e30a       ?editCell@QTable@@UAEXHH_N@Z 1001f30a f   qt-mt323:qt-mt323.dll
 0001:0001e310       ?endEdit@QTable@@MAEXHH_N0@Z 1001f310 f   qt-mt323:qt-mt323.dll
 0001:0001e316       ?eventFilter@QTable@@UAE_NPAVQObject@@PAVQEvent@@@Z 1001f316 f   qt-mt323:qt-mt323.dll
 0001:0001e31c       ?focusInEvent@QTable@@MAEXPAVQFocusEvent@@@Z 1001f31c f   qt-mt323:qt-mt323.dll
 0001:0001e322       ?focusOutEvent@QTable@@MAEXPAVQFocusEvent@@@Z 1001f322 f   qt-mt323:qt-mt323.dll
 0001:0001e328       ?hideColumn@QTable@@UAEXH@Z 1001f328 f   qt-mt323:qt-mt323.dll
 0001:0001e32e       ?hideRow@QTable@@UAEXH@Z   1001f32e f   qt-mt323:qt-mt323.dll
 0001:0001e334       ?insertColumns@QTable@@UAEXHH@Z 1001f334 f   qt-mt323:qt-mt323.dll
 0001:0001e33a       ?insertRows@QTable@@UAEXHH@Z 1001f33a f   qt-mt323:qt-mt323.dll
 0001:0001e340       ?insertWidget@QTable@@MAEXHHPAVQWidget@@@Z 1001f340 f   qt-mt323:qt-mt323.dll
 0001:0001e346       ?item@QTable@@UBEPAVQTableItem@@HH@Z 1001f346 f   qt-mt323:qt-mt323.dll
 0001:0001e34c       ?keyPressEvent@QTable@@MAEXPAVQKeyEvent@@@Z 1001f34c f   qt-mt323:qt-mt323.dll
 0001:0001e352       ?numCols@QTable@@UBEHXZ    1001f352 f   qt-mt323:qt-mt323.dll
 0001:0001e358       ?numRows@QTable@@UBEHXZ    1001f358 f   qt-mt323:qt-mt323.dll
 0001:0001e35e       ?paintCell@QTable@@UAEXPAVQPainter@@HHABVQRect@@_N@Z 1001f35e f   qt-mt323:qt-mt323.dll
 0001:0001e364       ?paintCell@QTable@@UAEXPAVQPainter@@HHABVQRect@@_NABVQColorGroup@@@Z 1001f364 f   qt-mt323:qt-mt323.dll
 0001:0001e36a       ?paintEmptyArea@QTable@@MAEXPAVQPainter@@HHHH@Z 1001f36a f   qt-mt323:qt-mt323.dll
 0001:0001e370       ?paintEvent@QTable@@MAEXPAVQPaintEvent@@@Z 1001f370 f   qt-mt323:qt-mt323.dll
 0001:0001e376       ?paintFocus@QTable@@UAEXPAVQPainter@@ABVQRect@@@Z 1001f376 f   qt-mt323:qt-mt323.dll
 0001:0001e37c       ?pixmap@QTable@@UBE?AVQPixmap@@HH@Z 1001f37c f   qt-mt323:qt-mt323.dll
 0001:0001e382       ?removeColumn@QTable@@UAEXH@Z 1001f382 f   qt-mt323:qt-mt323.dll
 0001:0001e388       ?removeColumns@QTable@@UAEXABV?$QMemArray@H@@@Z 1001f388 f   qt-mt323:qt-mt323.dll
 0001:0001e38e       ?removeRow@QTable@@UAEXH@Z 1001f38e f   qt-mt323:qt-mt323.dll
 0001:0001e394       ?removeRows@QTable@@UAEXABV?$QMemArray@H@@@Z 1001f394 f   qt-mt323:qt-mt323.dll
 0001:0001e39a       ?removeSelection@QTable@@UAEXABVQTableSelection@@@Z 1001f39a f   qt-mt323:qt-mt323.dll
 0001:0001e3a0       ?removeSelection@QTable@@UAEXH@Z 1001f3a0 f   qt-mt323:qt-mt323.dll
 0001:0001e3a6       ?resizeData@QTable@@MAEXH@Z 1001f3a6 f   qt-mt323:qt-mt323.dll
 0001:0001e3ac       ?resizeEvent@QScrollView@@MAEXPAVQResizeEvent@@@Z 1001f3ac f   qt-mt323:qt-mt323.dll
 0001:0001e3b2       ?rowAt@QTable@@UBEHH@Z     1001f3b2 f   qt-mt323:qt-mt323.dll
 0001:0001e3b8       ?rowHeight@QTable@@UBEHH@Z 1001f3b8 f   qt-mt323:qt-mt323.dll
 0001:0001e3be       ?rowHeightChanged@QTable@@MAEXH@Z 1001f3be f   qt-mt323:qt-mt323.dll
 0001:0001e3c4       ?rowIndexChanged@QTable@@MAEXHHH@Z 1001f3c4 f   qt-mt323:qt-mt323.dll
 0001:0001e3ca       ?rowPos@QTable@@UBEHH@Z    1001f3ca f   qt-mt323:qt-mt323.dll
 0001:0001e3d0       ?setCellContentFromEditor@QTable@@MAEXHH@Z 1001f3d0 f   qt-mt323:qt-mt323.dll
 0001:0001e3d6       ?setCellWidget@QTable@@UAEXHHPAVQWidget@@@Z 1001f3d6 f   qt-mt323:qt-mt323.dll
 0001:0001e3dc       ?setColumnMovingEnabled@QTable@@UAEX_N@Z 1001f3dc f   qt-mt323:qt-mt323.dll
 0001:0001e3e2       ?setColumnReadOnly@QTable@@UAEXH_N@Z 1001f3e2 f   qt-mt323:qt-mt323.dll
 0001:0001e3e8       ?setColumnStretchable@QTable@@UAEXH_N@Z 1001f3e8 f   qt-mt323:qt-mt323.dll
 0001:0001e3ee       ?setColumnWidth@QTable@@UAEXHH@Z 1001f3ee f   qt-mt323:qt-mt323.dll
 0001:0001e3f4       ?setCurrentCell@QTable@@UAEXHH@Z 1001f3f4 f   qt-mt323:qt-mt323.dll
 0001:0001e3fa       ?setDragEnabled@QTable@@UAEX_N@Z 1001f3fa f   qt-mt323:qt-mt323.dll
 0001:0001e400       ?setEnabled@QTable@@UAEX_N@Z 1001f400 f   qt-mt323:qt-mt323.dll
 0001:0001e406       ?setFocusStyle@QTable@@UAEXW4FocusStyle@1@@Z 1001f406 f   qt-mt323:qt-mt323.dll
 0001:0001e40c       ?setItem@QTable@@UAEXHHPAVQTableItem@@@Z 1001f40c f   qt-mt323:qt-mt323.dll
 0001:0001e412       ?setLeftMargin@QTable@@UAEXH@Z 1001f412 f   qt-mt323:qt-mt323.dll
 0001:0001e418       ?setNumCols@QTable@@UAEXH@Z 1001f418 f   qt-mt323:qt-mt323.dll
 0001:0001e41e       ?setNumRows@QTable@@UAEXH@Z 1001f41e f   qt-mt323:qt-mt323.dll
 0001:0001e424       ?setPixmap@QTable@@UAEXHHABVQPixmap@@@Z 1001f424 f   qt-mt323:qt-mt323.dll
 0001:0001e42a       ?setReadOnly@QTable@@UAEX_N@Z 1001f42a f   qt-mt323:qt-mt323.dll
 0001:0001e430       ?setRowHeight@QTable@@UAEXHH@Z 1001f430 f   qt-mt323:qt-mt323.dll
 0001:0001e436       ?setRowMovingEnabled@QTable@@UAEX_N@Z 1001f436 f   qt-mt323:qt-mt323.dll
 0001:0001e43c       ?setRowReadOnly@QTable@@UAEXH_N@Z 1001f43c f   qt-mt323:qt-mt323.dll
 0001:0001e442       ?setRowStretchable@QTable@@UAEXH_N@Z 1001f442 f   qt-mt323:qt-mt323.dll
 0001:0001e448       ?setSelectionMode@QTable@@UAEXW4SelectionMode@1@@Z 1001f448 f   qt-mt323:qt-mt323.dll
 0001:0001e44e       ?setShowGrid@QTable@@UAEX_N@Z 1001f44e f   qt-mt323:qt-mt323.dll
 0001:0001e454       ?setSorting@QTable@@UAEX_N@Z 1001f454 f   qt-mt323:qt-mt323.dll
 0001:0001e45a       ?setText@QTable@@UAEXHHABVQString@@@Z 1001f45a f   qt-mt323:qt-mt323.dll
 0001:0001e460       ?setTopMargin@QTable@@UAEXH@Z 1001f460 f   qt-mt323:qt-mt323.dll
 0001:0001e466       ?showColumn@QTable@@UAEXH@Z 1001f466 f   qt-mt323:qt-mt323.dll
 0001:0001e46c       ?showEvent@QTable@@MAEXPAVQShowEvent@@@Z 1001f46c f   qt-mt323:qt-mt323.dll
 0001:0001e472       ?showRow@QTable@@UAEXH@Z   1001f472 f   qt-mt323:qt-mt323.dll
 0001:0001e478       ?sizeHint@QTable@@UBE?AVQSize@@XZ 1001f478 f   qt-mt323:qt-mt323.dll
 0001:0001e47e       ?sortColumn@QTable@@UAEXH_N0@Z 1001f47e f   qt-mt323:qt-mt323.dll
 0001:0001e484       ?startDrag@QTable@@MAEXXZ  1001f484 f   qt-mt323:qt-mt323.dll
 0001:0001e48a       ?swapCells@QTable@@UAEXHHHH@Z 1001f48a f   qt-mt323:qt-mt323.dll
 0001:0001e490       ?swapColumns@QTable@@UAEXHH_N@Z 1001f490 f   qt-mt323:qt-mt323.dll
 0001:0001e496       ?swapRows@QTable@@UAEXHH_N@Z 1001f496 f   qt-mt323:qt-mt323.dll
 0001:0001e49c       ?takeItem@QTable@@UAEXPAVQTableItem@@@Z 1001f49c f   qt-mt323:qt-mt323.dll
 0001:0001e4a2       ?text@QTable@@UBE?AVQString@@HH@Z 1001f4a2 f   qt-mt323:qt-mt323.dll
 0001:0001e4a8       ?viewportResizeEvent@QTable@@MAEXPAVQResizeEvent@@@Z 1001f4a8 f   qt-mt323:qt-mt323.dll
 0001:0001e4ae       ?windowActivationChange@QTable@@MAEX_N@Z 1001f4ae f   qt-mt323:qt-mt323.dll
 0001:0001e4b4       _IsProcessorFeaturePresent@4 1001f4b4 f   kernel32:KERNEL32.dll
 0002:00000000       __imp__DisableThreadLibraryCalls@4 10024000     kernel32:KERNEL32.dll
 0002:00000004       __imp__GetCurrentThreadId@0 10024004     kernel32:KERNEL32.dll
 0002:00000008       __imp__GetCurrentProcessId@0 10024008     kernel32:KERNEL32.dll
 0002:0000000c       __imp__QueryPerformanceCounter@4 1002400c     kernel32:KERNEL32.dll
 0002:00000010       __imp__IsProcessorFeaturePresent@4 10024010     kernel32:KERNEL32.dll
 0002:00000014       __imp__IsDebuggerPresent@0 10024014     kernel32:KERNEL32.dll
 0002:00000018       __imp__DecodePointer@4     10024018     kernel32:KERNEL32.dll
 0002:0000001c       __imp__EncodePointer@4     1002401c     kernel32:KERNEL32.dll
 0002:00000020       __imp__GetPrivateProfileStringA@24 10024020     kernel32:KERNEL32.dll
 0002:00000024       __imp__GetSystemTimeAsFileTime@4 10024024     kernel32:KERNEL32.dll
 0002:00000028       \177KERNEL32_NULL_THUNK_DATA 10024028     kernel32:KERNEL32.dll
 0002:0000002c       __imp_?_Xbad_alloc@std@@YAXXZ 1002402c     msvcprt:MSVCP120.dll
 0002:00000030       __imp_?_Xlength_error@std@@YAXPBD@Z 10024030     msvcprt:MSVCP120.dll
 0002:00000034       \177MSVCP120_NULL_THUNK_DATA 10024034     msvcprt:MSVCP120.dll
 0002:00000038       __imp___except_handler4_common 10024038     MSVCRT:MSVCR120.dll
 0002:0000003c       __imp___initterm_e         1002403c     MSVCRT:MSVCR120.dll
 0002:00000040       __imp___initterm           10024040     MSVCRT:MSVCR120.dll
 0002:00000044       __imp___malloc_crt         10024044     MSVCRT:MSVCR120.dll
 0002:00000048       __imp__free                10024048     MSVCRT:MSVCR120.dll
 0002:0000004c       __imp___amsg_exit          1002404c     MSVCRT:MSVCR120.dll
 0002:00000050       __imp____CppXcptFilter     10024050     MSVCRT:MSVCR120.dll
 0002:00000054       __imp_?terminate@@YAXXZ    10024054     MSVCRT:MSVCR120.dll
 0002:00000058       __imp_??1type_info@@UAE@XZ 10024058     MSVCRT:MSVCR120.dll
 0002:0000005c       __imp___onexit             1002405c     MSVCRT:MSVCR120.dll
 0002:00000060       __imp___crt_debugger_hook  10024060     MSVCRT:MSVCR120.dll
 0002:00000064       __imp___calloc_crt         10024064     MSVCRT:MSVCR120.dll
 0002:00000068       __imp___unlock             10024068     MSVCRT:MSVCR120.dll
 0002:0000006c       __imp___lock               1002406c     MSVCRT:MSVCR120.dll
 0002:00000070       __imp___purecall           10024070     MSVCRT:MSVCR120.dll
 0002:00000074       __imp__sprintf             10024074     MSVCRT:MSVCR120.dll
 0002:00000078       __imp__atoi                10024078     MSVCRT:MSVCR120.dll
 0002:0000007c       __imp____RTDynamicCast     1002407c     MSVCRT:MSVCR120.dll
 0002:00000080       __imp____CxxFrameHandler3  10024080     MSVCRT:MSVCR120.dll
 0002:00000084       __imp___CxxThrowException@8 10024084     MSVCRT:MSVCR120.dll
 0002:00000088       __imp_??3@YAXPAX@Z         10024088     MSVCRT:MSVCR120.dll
 0002:0000008c       __imp_??2@YAPAXI@Z         1002408c     MSVCRT:MSVCR120.dll
 0002:00000090       __imp____crtUnhandledException 10024090     MSVCRT:MSVCR120.dll
 0002:00000094       __imp____dllonexit         10024094     MSVCRT:MSVCR120.dll
 0002:00000098       __imp____clean_type_info_names_internal 10024098     MSVCRT:MSVCR120.dll
 0002:0000009c       __imp____crtTerminateProcess 1002409c     MSVCRT:MSVCR120.dll
 0002:000000a0       \177MSVCR120_NULL_THUNK_DATA 100240a0     MSVCRT:MSVCR120.dll
 0002:000000a4       __imp_?metaObject@CAlm_sys_select@@UBEPAVQMetaObject@@XZ 100240a4     alm_sys_select:alm_sys_select.dll
 0002:000000a8       __imp_?qt_property@CAlm_sys_select@@UAE_NHHPAVQVariant@@@Z 100240a8     alm_sys_select:alm_sys_select.dll
 0002:000000ac       __imp_?qt_invoke@CAlm_sys_select@@UAE_NHPAUQUObject@@@Z 100240ac     alm_sys_select:alm_sys_select.dll
 0002:000000b0       __imp_?qt_emit@CAlm_sys_select@@UAE_NHPAUQUObject@@@Z 100240b0     alm_sys_select:alm_sys_select.dll
 0002:000000b4       __imp_?qt_cast@CAlm_sys_select@@UAEPAXPBD@Z 100240b4     alm_sys_select:alm_sys_select.dll
 0002:000000b8       __imp_?getSystemName@CAlm_sys_select@@QAE?AVQString@@XZ 100240b8     alm_sys_select:alm_sys_select.dll
 0002:000000bc       __imp_?className@CAlm_sys_select@@UBEPBDXZ 100240bc     alm_sys_select:alm_sys_select.dll
 0002:000000c0       __imp_??1CAlm_sys_select@@UAE@XZ 100240c0     alm_sys_select:alm_sys_select.dll
 0002:000000c4       __imp_??0CAlm_sys_select@@QAE@PAVQWidget@@PBD@Z 100240c4     alm_sys_select:alm_sys_select.dll
 0002:000000c8       __imp_?setSystemNames@CAlm_sys_select@@QAE_NVQString@@@Z 100240c8     alm_sys_select:alm_sys_select.dll
 0002:000000cc       \177alm_sys_select_NULL_THUNK_DATA 100240cc     alm_sys_select:alm_sys_select.dll
 0002:000000d0       __imp_?fnConfig_icons@@YAPAPBDPBD@Z 100240d0     config_icons:config_icons.dll
 0002:000000d4       \177config_icons_NULL_THUNK_DATA 100240d4     config_icons:config_icons.dll
 0002:000000d8       __imp_??1QGList@@MAE@XZ    100240d8     qt-mt323:qt-mt323.dll
 0002:000000dc       __imp_?append@QGList@@IAEXPAX@Z 100240dc     qt-mt323:qt-mt323.dll
 0002:000000e0       __imp_?remove@QGList@@IAE_NPAX@Z 100240e0     qt-mt323:qt-mt323.dll
 0002:000000e4       __imp_?clear@QGList@@MAEXXZ 100240e4     qt-mt323:qt-mt323.dll
 0002:000000e8       __imp_?first@QGList@@IAEPAXXZ 100240e8     qt-mt323:qt-mt323.dll
 0002:000000ec       __imp_?blockSignals@QObject@@QAEX_N@Z 100240ec     qt-mt323:qt-mt323.dll
 0002:000000f0       __imp_?connect@QObject@@SA_NPBV1@PBD01@Z 100240f0     qt-mt323:qt-mt323.dll
 0002:000000f4       __imp_??0QStringList@@QAE@XZ 100240f4     qt-mt323:qt-mt323.dll
 0002:000000f8       __imp_?sort@QStringList@@QAEXXZ 100240f8     qt-mt323:qt-mt323.dll
 0002:000000fc       __imp_?split@QStringList@@SA?AV1@ABVQString@@0_N@Z 100240fc     qt-mt323:qt-mt323.dll
 0002:00000100       __imp_?join@QStringList@@QBE?AVQString@@ABV2@@Z 10024100     qt-mt323:qt-mt323.dll
 0002:00000104       __imp_??1QStringList@@QAE@XZ 10024104     qt-mt323:qt-mt323.dll
 0002:00000108       __imp_??0QColor@@QAE@PBD@Z 10024108     qt-mt323:qt-mt323.dll
 0002:0000010c       __imp_??0QColor@@QAE@ABV0@@Z 1002410c     qt-mt323:qt-mt323.dll
 0002:00000110       __imp_??0QColorGroup@@QAE@ABV0@@Z 10024110     qt-mt323:qt-mt323.dll
 0002:00000114       __imp_??1QColorGroup@@QAE@XZ 10024114     qt-mt323:qt-mt323.dll
 0002:00000118       __imp_?color@QColorGroup@@QBEABVQColor@@W4ColorRole@1@@Z 10024118     qt-mt323:qt-mt323.dll
 0002:0000011c       __imp_?setColor@QColorGroup@@QAEXW4ColorRole@1@ABVQColor@@@Z 1002411c     qt-mt323:qt-mt323.dll
 0002:00000120       __imp_??0QWidget@@QAE@PAV0@PBDI@Z 10024120     qt-mt323:qt-mt323.dll
 0002:00000124       __imp_??1QWidget@@UAE@XZ   10024124     qt-mt323:qt-mt323.dll
 0002:00000128       __imp_?setName@QWidget@@UAEXPBD@Z 10024128     qt-mt323:qt-mt323.dll
 0002:0000012c       __imp_?setDisabled@QWidget@@QAEX_N@Z 1002412c     qt-mt323:qt-mt323.dll
 0002:00000130       __imp_?rect@QWidget@@QBE?AVQRect@@XZ 10024130     qt-mt323:qt-mt323.dll
 0002:00000134       __imp_?setCaption@QWidget@@UAEXABVQString@@@Z 10024134     qt-mt323:qt-mt323.dll
 0002:00000138       __imp_?setFocusPolicy@QWidget@@UAEXW4FocusPolicy@1@@Z 10024138     qt-mt323:qt-mt323.dll
 0002:0000013c       __imp_?exec@QDialog@@QAEHXZ 1002413c     qt-mt323:qt-mt323.dll
 0002:00000140       __imp_?information@QMessageBox@@SAHPAVQWidget@@ABVQString@@1111HH@Z 10024140     qt-mt323:qt-mt323.dll
 0002:00000144       __imp_?question@QMessageBox@@SAHPAVQWidget@@ABVQString@@1HHH@Z 10024144     qt-mt323:qt-mt323.dll
 0002:00000148       __imp_?warning@QMessageBox@@SAHPAVQWidget@@ABVQString@@1111HH@Z 10024148     qt-mt323:qt-mt323.dll
 0002:0000014c       __imp_?critical@QMessageBox@@SAHPAVQWidget@@ABVQString@@1111HH@Z 1002414c     qt-mt323:qt-mt323.dll
 0002:00000150       __imp_??0QPixmap@@QAE@QAPBD@Z 10024150     qt-mt323:qt-mt323.dll
 0002:00000154       __imp_??1QPixmap@@UAE@XZ   10024154     qt-mt323:qt-mt323.dll
 0002:00000158       __imp_??0QIconSet@@QAE@ABVQPixmap@@W4Size@0@@Z 10024158     qt-mt323:qt-mt323.dll
 0002:0000015c       __imp_??1QIconSet@@UAE@XZ  1002415c     qt-mt323:qt-mt323.dll
 0002:00000160       __imp_??0QKeySequence@@QAE@H@Z 10024160     qt-mt323:qt-mt323.dll
 0002:00000164       __imp_??0QAction@@QAE@ABVQString@@ABVQIconSet@@0VQKeySequence@@PAVQObject@@PBD_N@Z 10024164     qt-mt323:qt-mt323.dll
 0002:00000168       __imp_??0QAction@@QAE@ABVQString@@0VQKeySequence@@PAVQObject@@PBD_N@Z 10024168     qt-mt323:qt-mt323.dll
 0002:0000016c       __imp_??1QAction@@UAE@XZ   1002416c     qt-mt323:qt-mt323.dll
 0002:00000170       __imp_??0QDockWindow@@QAE@W4Place@0@PAVQWidget@@PBDI@Z 10024170     qt-mt323:qt-mt323.dll
 0002:00000174       __imp_??1QDockWindow@@UAE@XZ 10024174     qt-mt323:qt-mt323.dll
 0002:00000178       __imp_??1?$QPtrList@VQDockWindow@@@@UAE@XZ 10024178     qt-mt323:qt-mt323.dll
 0002:0000017c       __imp_??0QToolBar@@QAE@PAVQMainWindow@@PBD@Z 1002417c     qt-mt323:qt-mt323.dll
 0002:00000180       __imp_??1QToolBar@@UAE@XZ  10024180     qt-mt323:qt-mt323.dll
 0002:00000184       __imp_??0QFile@@QAE@ABVQString@@@Z 10024184     qt-mt323:qt-mt323.dll
 0002:00000188       __imp_??1QFile@@UAE@XZ     10024188     qt-mt323:qt-mt323.dll
 0002:0000018c       __imp_?exists@QFile@@QBE_NXZ 1002418c     qt-mt323:qt-mt323.dll
 0002:00000190       __imp_?remove@QFile@@QAE_NXZ 10024190     qt-mt323:qt-mt323.dll
 0002:00000194       __imp_?open@QFile@@UAE_NH@Z 10024194     qt-mt323:qt-mt323.dll
 0002:00000198       __imp_?close@QFile@@UAEXXZ 10024198     qt-mt323:qt-mt323.dll
 0002:0000019c       __imp_??0QListViewItem@@QAE@PAVQListView@@VQString@@1111111@Z 1002419c     qt-mt323:qt-mt323.dll
 0002:000001a0       __imp_??1QListViewItem@@UAE@XZ 100241a0     qt-mt323:qt-mt323.dll
 0002:000001a4       __imp_?text@QListViewItem@@UBE?AVQString@@H@Z 100241a4     qt-mt323:qt-mt323.dll
 0002:000001a8       __imp_?paintCell@QListViewItem@@UAEXPAVQPainter@@ABVQColorGroup@@HHH@Z 100241a8     qt-mt323:qt-mt323.dll
 0002:000001ac       __imp_?repaint@QListViewItem@@QBEXXZ 100241ac     qt-mt323:qt-mt323.dll
 0002:000001b0       __imp_?setVisible@QListViewItem@@QAEX_N@Z 100241b0     qt-mt323:qt-mt323.dll
 0002:000001b4       __imp_?setRenameEnabled@QListViewItem@@UAEXH_N@Z 100241b4     qt-mt323:qt-mt323.dll
 0002:000001b8       __imp_??0QListView@@QAE@PAVQWidget@@PBDI@Z 100241b8     qt-mt323:qt-mt323.dll
 0002:000001bc       __imp_??1QListView@@UAE@XZ 100241bc     qt-mt323:qt-mt323.dll
 0002:000001c0       __imp_?ensureItemVisible@QListView@@QAEXPBVQListViewItem@@@Z 100241c0     qt-mt323:qt-mt323.dll
 0002:000001c4       __imp_?setSelectionMode@QListView@@QAEXW4SelectionMode@1@@Z 100241c4     qt-mt323:qt-mt323.dll
 0002:000001c8       __imp_?selectedItem@QListView@@QBEPAVQListViewItem@@XZ 100241c8     qt-mt323:qt-mt323.dll
 0002:000001cc       __imp_?currentItem@QListView@@QBEPAVQListViewItem@@XZ 100241cc     qt-mt323:qt-mt323.dll
 0002:000001d0       __imp_?firstChild@QListView@@QBEPAVQListViewItem@@XZ 100241d0     qt-mt323:qt-mt323.dll
 0002:000001d4       __imp_?childCount@QListView@@QBEHXZ 100241d4     qt-mt323:qt-mt323.dll
 0002:000001d8       __imp_?sortColumn@QListView@@QBEHXZ 100241d8     qt-mt323:qt-mt323.dll
 0002:000001dc       __imp_?setSortColumn@QListView@@QAEXH@Z 100241dc     qt-mt323:qt-mt323.dll
 0002:000001e0       __imp_?sortOrder@QListView@@QBE?AW4SortOrder@Qt@@XZ 100241e0     qt-mt323:qt-mt323.dll
 0002:000001e4       __imp_?setSortOrder@QListView@@QAEXW4SortOrder@Qt@@@Z 100241e4     qt-mt323:qt-mt323.dll
 0002:000001e8       __imp_?findItem@QListView@@QBEPAVQListViewItem@@ABVQString@@HI@Z 100241e8     qt-mt323:qt-mt323.dll
 0002:000001ec       __imp_?keyPressEvent@QListView@@MAEXPAVQKeyEvent@@@Z 100241ec     qt-mt323:qt-mt323.dll
 0002:000001f0       __imp_??0QListViewItemIterator@@QAE@XZ 100241f0     qt-mt323:qt-mt323.dll
 0002:000001f4       __imp_??0QListViewItemIterator@@QAE@PAVQListView@@@Z 100241f4     qt-mt323:qt-mt323.dll
 0002:000001f8       __imp_??0QListViewItemIterator@@QAE@PAVQListView@@H@Z 100241f8     qt-mt323:qt-mt323.dll
 0002:000001fc       __imp_??4QListViewItemIterator@@QAEAAV0@ABV0@@Z 100241fc     qt-mt323:qt-mt323.dll
 0002:00000200       __imp_??1QListViewItemIterator@@QAE@XZ 10024200     qt-mt323:qt-mt323.dll
 0002:00000204       __imp_??EQListViewItemIterator@@QAEAAV0@XZ 10024204     qt-mt323:qt-mt323.dll
 0002:00000208       __imp_??EQListViewItemIterator@@QAE?BV0@H@Z 10024208     qt-mt323:qt-mt323.dll
 0002:0000020c       __imp_??DQListViewItemIterator@@QAEPAVQListViewItem@@XZ 1002420c     qt-mt323:qt-mt323.dll
 0002:00000210       __imp_?current@QListViewItemIterator@@QBEPAVQListViewItem@@XZ 10024210     qt-mt323:qt-mt323.dll
 0002:00000214       __imp_?secsTo@QTime@@QBEHABV1@@Z 10024214     qt-mt323:qt-mt323.dll
 0002:00000218       __imp_?msecsTo@QTime@@QBEHABV1@@Z 10024218     qt-mt323:qt-mt323.dll
 0002:0000021c       __imp_?currentTime@QTime@@SA?AV1@XZ 1002421c     qt-mt323:qt-mt323.dll
 0002:00000220       __imp_??8QDateTime@@QBE_NABV0@@Z 10024220     qt-mt323:qt-mt323.dll
 0002:00000224       __imp_??0QFileInfo@@QAE@XZ 10024224     qt-mt323:qt-mt323.dll
 0002:00000228       __imp_??1QFileInfo@@QAE@XZ 10024228     qt-mt323:qt-mt323.dll
 0002:0000022c       __imp_?setFile@QFileInfo@@QAEXABVQString@@@Z 1002422c     qt-mt323:qt-mt323.dll
 0002:00000230       __imp_?exists@QFileInfo@@QBE_NXZ 10024230     qt-mt323:qt-mt323.dll
 0002:00000234       __imp_?lastModified@QFileInfo@@QBE?AVQDateTime@@XZ 10024234     qt-mt323:qt-mt323.dll
 0002:00000238       __imp_??0QDir@@QAE@XZ      10024238     qt-mt323:qt-mt323.dll
 0002:0000023c       __imp_??1QDir@@UAE@XZ      1002423c     qt-mt323:qt-mt323.dll
 0002:00000240       __imp_?setPath@QDir@@UAEXABVQString@@@Z 10024240     qt-mt323:qt-mt323.dll
 0002:00000244       __imp_?mkdir@QDir@@UBE_NABVQString@@_N@Z 10024244     qt-mt323:qt-mt323.dll
 0002:00000248       __imp_?exists@QDir@@UBE_NXZ 10024248     qt-mt323:qt-mt323.dll
 0002:0000024c       __imp_??0QPushButton@@QAE@PAVQWidget@@PBD@Z 1002424c     qt-mt323:qt-mt323.dll
 0002:00000250       __imp_??1QPushButton@@UAE@XZ 10024250     qt-mt323:qt-mt323.dll
 0002:00000254       __imp_?insertStringList@QComboBox@@QAEXABVQStringList@@H@Z 10024254     qt-mt323:qt-mt323.dll
 0002:00000258       __imp_?clear@QComboBox@@QAEXXZ 10024258     qt-mt323:qt-mt323.dll
 0002:0000025c       __imp_??0QLineEdit@@QAE@PAVQWidget@@PBD@Z 1002425c     qt-mt323:qt-mt323.dll
 0002:00000260       __imp_??1QLineEdit@@UAE@XZ 10024260     qt-mt323:qt-mt323.dll
 0002:00000264       __imp_?text@QLineEdit@@QBE?AVQString@@XZ 10024264     qt-mt323:qt-mt323.dll
 0002:00000268       __imp_?end@QLineEdit@@QAEX_N@Z 10024268     qt-mt323:qt-mt323.dll
 0002:0000026c       __imp_?getText@QInputDialog@@SA?AVQString@@ABV2@0W4EchoMode@QLineEdit@@0PA_NPAVQWidget@@PBD@Z 1002426c     qt-mt323:qt-mt323.dll
 0002:00000270       __imp_?getItem@QInputDialog@@SA?AVQString@@ABV2@0ABVQStringList@@H_NPA_NPAVQWidget@@PBD@Z 10024270     qt-mt323:qt-mt323.dll
 0002:00000274       __imp_??0QTabWidget@@QAE@PAVQWidget@@PBDI@Z 10024274     qt-mt323:qt-mt323.dll
 0002:00000278       __imp_??1QTabWidget@@UAE@XZ 10024278     qt-mt323:qt-mt323.dll
 0002:0000027c       __imp_??1QLayoutItem@@UAE@XZ 1002427c     qt-mt323:qt-mt323.dll
 0002:00000280       __imp_??0QSpacerItem@@QAE@HHW4SizeType@QSizePolicy@@0@Z 10024280     qt-mt323:qt-mt323.dll
 0002:00000284       __imp_?add@QLayout@@QAEXPAVQWidget@@@Z 10024284     qt-mt323:qt-mt323.dll
 0002:00000288       __imp_??0QHBoxLayout@@QAE@PAVQLayout@@HPBD@Z 10024288     qt-mt323:qt-mt323.dll
 0002:0000028c       __imp_??1QHBoxLayout@@UAE@XZ 1002428c     qt-mt323:qt-mt323.dll
 0002:00000290       __imp_??0QVBoxLayout@@QAE@PAVQWidget@@HHPBD@Z 10024290     qt-mt323:qt-mt323.dll
 0002:00000294       __imp_??1QVBoxLayout@@UAE@XZ 10024294     qt-mt323:qt-mt323.dll
 0002:00000298       __imp_??0QRegExp@@QAE@ABVQString@@_N1@Z 10024298     qt-mt323:qt-mt323.dll
 0002:0000029c       __imp_??1QRegExp@@QAE@XZ   1002429c     qt-mt323:qt-mt323.dll
 0002:000002a0       __imp_?setChecked@QCheckBox@@QAEX_N@Z 100242a0     qt-mt323:qt-mt323.dll
 0002:000002a4       __imp_?value@QSpinBox@@QBEHXZ 100242a4     qt-mt323:qt-mt323.dll
 0002:000002a8       __imp_??0QLabel@@QAE@PAVQWidget@@PBDI@Z 100242a8     qt-mt323:qt-mt323.dll
 0002:000002ac       __imp_??1QLabel@@UAE@XZ    100242ac     qt-mt323:qt-mt323.dll
 0002:000002b0       __imp_??0QPopupMenu@@QAE@PAVQWidget@@PBD@Z 100242b0     qt-mt323:qt-mt323.dll
 0002:000002b4       __imp_??1QPopupMenu@@UAE@XZ 100242b4     qt-mt323:qt-mt323.dll
 0002:000002b8       __imp_?exec@QPopupMenu@@QAEHABVQPoint@@H@Z 100242b8     qt-mt323:qt-mt323.dll
 0002:000002bc       __imp_??0QGuardedPtrPrivate@@QAE@PAVQObject@@@Z 100242bc     qt-mt323:qt-mt323.dll
 0002:000002c0       __imp_??1QGuardedPtrPrivate@@UAE@XZ 100242c0     qt-mt323:qt-mt323.dll
 0002:000002c4       __imp_?reconnect@QGuardedPtrPrivate@@QAEXPAVQObject@@@Z 100242c4     qt-mt323:qt-mt323.dll
 0002:000002c8       __imp_?acceptDrop@QListViewItem@@UBE_NPBVQMimeSource@@@Z 100242c8     qt-mt323:qt-mt323.dll
 0002:000002cc       __imp_?activate@QListViewItem@@MAEXXZ 100242cc     qt-mt323:qt-mt323.dll
 0002:000002d0       __imp_?activateItemAt@QPopupMenu@@UAEXH@Z 100242d0     qt-mt323:qt-mt323.dll
 0002:000002d4       __imp_?addChild@QScrollView@@UAEXPAVQWidget@@HH@Z 100242d4     qt-mt323:qt-mt323.dll
 0002:000002d8       __imp_?addColumn@QListView@@UAEHABVQIconSet@@ABVQString@@H@Z 100242d8     qt-mt323:qt-mt323.dll
 0002:000002dc       __imp_?addColumn@QListView@@UAEHABVQString@@H@Z 100242dc     qt-mt323:qt-mt323.dll
 0002:000002e0       __imp_?addItem@QBoxLayout@@UAEXPAVQLayoutItem@@@Z 100242e0     qt-mt323:qt-mt323.dll
 0002:000002e4       __imp_?addTab@QTabWidget@@UAEXPAVQWidget@@ABVQIconSet@@ABVQString@@@Z 100242e4     qt-mt323:qt-mt323.dll
 0002:000002e8       __imp_?addTab@QTabWidget@@UAEXPAVQWidget@@ABVQString@@@Z 100242e8     qt-mt323:qt-mt323.dll
 0002:000002ec       __imp_?addTab@QTabWidget@@UAEXPAVQWidget@@PAVQTab@@@Z 100242ec     qt-mt323:qt-mt323.dll
 0002:000002f0       __imp_?addTo@QAction@@UAE_NPAVQWidget@@@Z 100242f0     qt-mt323:qt-mt323.dll
 0002:000002f4       __imp_?addedTo@QAction@@MAEXHPAVQPopupMenu@@@Z 100242f4     qt-mt323:qt-mt323.dll
 0002:000002f8       __imp_?addedTo@QAction@@MAEXPAVQWidget@@0@Z 100242f8     qt-mt323:qt-mt323.dll
 0002:000002fc       __imp_?adjustSize@QWidget@@UAEXXZ 100242fc     qt-mt323:qt-mt323.dll
 0002:00000300       __imp_?cancelRename@QListViewItem@@MAEXH@Z 10024300     qt-mt323:qt-mt323.dll
 0002:00000304       __imp_?checkConnectArgs@QObject@@MAE_NPBDPBV1@0@Z 10024304     qt-mt323:qt-mt323.dll
 0002:00000308       __imp_?childEvent@QLayout@@MAEXPAVQChildEvent@@@Z 10024308     qt-mt323:qt-mt323.dll
 0002:0000030c       __imp_?childEvent@QObject@@MAEXPAVQChildEvent@@@Z 1002430c     qt-mt323:qt-mt323.dll
 0002:00000310       __imp_?className@QAction@@UBEPBDXZ 10024310     qt-mt323:qt-mt323.dll
 0002:00000314       __imp_?className@QDockWindow@@UBEPBDXZ 10024314     qt-mt323:qt-mt323.dll
 0002:00000318       __imp_?className@QGuardedPtrPrivate@@UBEPBDXZ 10024318     qt-mt323:qt-mt323.dll
 0002:0000031c       __imp_?className@QHBoxLayout@@UBEPBDXZ 1002431c     qt-mt323:qt-mt323.dll
 0002:00000320       __imp_?className@QLabel@@UBEPBDXZ 10024320     qt-mt323:qt-mt323.dll
 0002:00000324       __imp_?className@QLineEdit@@UBEPBDXZ 10024324     qt-mt323:qt-mt323.dll
 0002:00000328       __imp_?className@QListView@@UBEPBDXZ 10024328     qt-mt323:qt-mt323.dll
 0002:0000032c       __imp_?className@QPopupMenu@@UBEPBDXZ 1002432c     qt-mt323:qt-mt323.dll
 0002:00000330       __imp_?className@QPushButton@@UBEPBDXZ 10024330     qt-mt323:qt-mt323.dll
 0002:00000334       __imp_?className@QTabWidget@@UBEPBDXZ 10024334     qt-mt323:qt-mt323.dll
 0002:00000338       __imp_?className@QToolBar@@UBEPBDXZ 10024338     qt-mt323:qt-mt323.dll
 0002:0000033c       __imp_?className@QVBoxLayout@@UBEPBDXZ 1002433c     qt-mt323:qt-mt323.dll
 0002:00000340       __imp_?className@QWidget@@UBEPBDXZ 10024340     qt-mt323:qt-mt323.dll
 0002:00000344       __imp_?clear@?$QPtrList@VQDockWindow@@@@UAEXXZ 10024344     qt-mt323:qt-mt323.dll
 0002:00000348       __imp_?clear@QLineEdit@@UAEXXZ 10024348     qt-mt323:qt-mt323.dll
 0002:0000034c       __imp_?clear@QListView@@UAEXXZ 1002434c     qt-mt323:qt-mt323.dll
 0002:00000350       __imp_?clear@QToolBar@@UAEXXZ 10024350     qt-mt323:qt-mt323.dll
 0002:00000354       __imp_?clearSelection@QListView@@UAEXXZ 10024354     qt-mt323:qt-mt323.dll
 0002:00000358       __imp_?clearValidator@QLineEdit@@UAEXXZ 10024358     qt-mt323:qt-mt323.dll
 0002:0000035c       __imp_?close@QWidget@@UAE_N_N@Z 1002435c     qt-mt323:qt-mt323.dll
 0002:00000360       __imp_?closeEvent@QPopupMenu@@MAEXPAVQCloseEvent@@@Z 10024360     qt-mt323:qt-mt323.dll
 0002:00000364       __imp_?closeEvent@QWidget@@MAEXPAVQCloseEvent@@@Z 10024364     qt-mt323:qt-mt323.dll
 0002:00000368       __imp_?cmd@QPaintDevice@@MAE_NHPAVQPainter@@PATQPDevCmdParam@@@Z 10024368     qt-mt323:qt-mt323.dll
 0002:0000036c       __imp_?compare@QListViewItem@@UBEHPAV1@H_N@Z 1002436c     qt-mt323:qt-mt323.dll
 0002:00000370       __imp_?compareItems@QGList@@MAEHPAX0@Z 10024370     qt-mt323:qt-mt323.dll
 0002:00000374       __imp_?connectNotify@QObject@@MAEXPBD@Z 10024374     qt-mt323:qt-mt323.dll
 0002:00000378       __imp_?contentsContextMenuEvent@QListView@@MAEXPAVQContextMenuEvent@@@Z 10024378     qt-mt323:qt-mt323.dll
 0002:0000037c       __imp_?contentsDragEnterEvent@QListView@@MAEXPAVQDragEnterEvent@@@Z 1002437c     qt-mt323:qt-mt323.dll
 0002:00000380       __imp_?contentsDragLeaveEvent@QListView@@MAEXPAVQDragLeaveEvent@@@Z 10024380     qt-mt323:qt-mt323.dll
 0002:00000384       __imp_?contentsDragMoveEvent@QListView@@MAEXPAVQDragMoveEvent@@@Z 10024384     qt-mt323:qt-mt323.dll
 0002:00000388       __imp_?contentsDropEvent@QListView@@MAEXPAVQDropEvent@@@Z 10024388     qt-mt323:qt-mt323.dll
 0002:0000038c       __imp_?contentsMouseDoubleClickEvent@QListView@@MAEXPAVQMouseEvent@@@Z 1002438c     qt-mt323:qt-mt323.dll
 0002:00000390       __imp_?contentsMouseMoveEvent@QListView@@MAEXPAVQMouseEvent@@@Z 10024390     qt-mt323:qt-mt323.dll
 0002:00000394       __imp_?contentsMousePressEvent@QListView@@MAEXPAVQMouseEvent@@@Z 10024394     qt-mt323:qt-mt323.dll
 0002:00000398       __imp_?contentsMouseReleaseEvent@QListView@@MAEXPAVQMouseEvent@@@Z 10024398     qt-mt323:qt-mt323.dll
 0002:0000039c       __imp_?contentsWheelEvent@QScrollView@@MAEXPAVQWheelEvent@@@Z 1002439c     qt-mt323:qt-mt323.dll
 0002:000003a0       __imp_?contextMenuEvent@QDockWindow@@MAEXPAVQContextMenuEvent@@@Z 100243a0     qt-mt323:qt-mt323.dll
 0002:000003a4       __imp_?contextMenuEvent@QLineEdit@@MAEXPAVQContextMenuEvent@@@Z 100243a4     qt-mt323:qt-mt323.dll
 0002:000003a8       __imp_?contextMenuEvent@QScrollView@@MAEXPAVQContextMenuEvent@@@Z 100243a8     qt-mt323:qt-mt323.dll
 0002:000003ac       __imp_?contextMenuEvent@QWidget@@MAEXPAVQContextMenuEvent@@@Z 100243ac     qt-mt323:qt-mt323.dll
 0002:000003b0       __imp_?copy@QLineEdit@@UBEXXZ 100243b0     qt-mt323:qt-mt323.dll
 0002:000003b4       __imp_?count@?$QPtrList@VQDockWindow@@@@UBEIXZ 100243b4     qt-mt323:qt-mt323.dll
 0002:000003b8       __imp_?create@QWidget@@MAEXPAUHWND__@@_N1@Z 100243b8     qt-mt323:qt-mt323.dll
 0002:000003bc       __imp_?createPopupMenu@QLineEdit@@MAEPAVQPopupMenu@@XZ 100243bc     qt-mt323:qt-mt323.dll
 0002:000003c0       __imp_?customEvent@QObject@@MAEXPAVQCustomEvent@@@Z 100243c0     qt-mt323:qt-mt323.dll
 0002:000003c4       __imp_?customWhatsThis@QPopupMenu@@UBE_NXZ 100243c4     qt-mt323:qt-mt323.dll
 0002:000003c8       __imp_?customWhatsThis@QWidget@@UBE_NXZ 100243c8     qt-mt323:qt-mt323.dll
 0002:000003cc       __imp_?cut@QLineEdit@@UAEXXZ 100243cc     qt-mt323:qt-mt323.dll
 0002:000003d0       __imp_?deleteItem@?$QPtrList@VQDockWindow@@@@EAEXPAX@Z 100243d0     qt-mt323:qt-mt323.dll
 0002:000003d4       __imp_?deselect@QLineEdit@@UAEXXZ 100243d4     qt-mt323:qt-mt323.dll
 0002:000003d8       __imp_?destroy@QWidget@@MAEX_N0@Z 100243d8     qt-mt323:qt-mt323.dll
 0002:000003dc       __imp_?disconnectNotify@QObject@@MAEXPBD@Z 100243dc     qt-mt323:qt-mt323.dll
 0002:000003e0       __imp_?dock@QDockWindow@@UAEXXZ 100243e0     qt-mt323:qt-mt323.dll
 0002:000003e4       __imp_?dragEnterEvent@QLineEdit@@MAEXPAVQDragEnterEvent@@@Z 100243e4     qt-mt323:qt-mt323.dll
 0002:000003e8       __imp_?dragEnterEvent@QWidget@@MAEXPAVQDragEnterEvent@@@Z 100243e8     qt-mt323:qt-mt323.dll
 0002:000003ec       __imp_?dragEntered@QListViewItem@@MAEXXZ 100243ec     qt-mt323:qt-mt323.dll
 0002:000003f0       __imp_?dragLeaveEvent@QLineEdit@@MAEXPAVQDragLeaveEvent@@@Z 100243f0     qt-mt323:qt-mt323.dll
 0002:000003f4       __imp_?dragLeaveEvent@QWidget@@MAEXPAVQDragLeaveEvent@@@Z 100243f4     qt-mt323:qt-mt323.dll
 0002:000003f8       __imp_?dragLeft@QListViewItem@@MAEXXZ 100243f8     qt-mt323:qt-mt323.dll
 0002:000003fc       __imp_?dragMoveEvent@QLineEdit@@MAEXPAVQDragMoveEvent@@@Z 100243fc     qt-mt323:qt-mt323.dll
 0002:00000400       __imp_?dragMoveEvent@QWidget@@MAEXPAVQDragMoveEvent@@@Z 10024400     qt-mt323:qt-mt323.dll
 0002:00000404       __imp_?dragObject@QListView@@MAEPAVQDragObject@@XZ 10024404     qt-mt323:qt-mt323.dll
 0002:00000408       __imp_?drawButton@QPushButton@@MAEXPAVQPainter@@@Z 10024408     qt-mt323:qt-mt323.dll
 0002:0000040c       __imp_?drawButtonLabel@QPushButton@@MAEXPAVQPainter@@@Z 1002440c     qt-mt323:qt-mt323.dll
 0002:00000410       __imp_?drawContents@QDockWindow@@MAEXPAVQPainter@@@Z 10024410     qt-mt323:qt-mt323.dll
 0002:00000414       __imp_?drawContents@QFrame@@MAEXPAVQPainter@@@Z 10024414     qt-mt323:qt-mt323.dll
 0002:00000418       __imp_?drawContents@QLabel@@MAEXPAVQPainter@@@Z 10024418     qt-mt323:qt-mt323.dll
 0002:0000041c       __imp_?drawContents@QLineEdit@@MAEXPAVQPainter@@@Z 1002441c     qt-mt323:qt-mt323.dll
 0002:00000420       __imp_?drawContents@QPopupMenu@@MAEXPAVQPainter@@@Z 10024420     qt-mt323:qt-mt323.dll
 0002:00000424       __imp_?drawContents@QScrollView@@EAEXPAVQPainter@@@Z 10024424     qt-mt323:qt-mt323.dll
 0002:00000428       __imp_?drawContents@QScrollView@@MAEXPAVQPainter@@HHHH@Z 10024428     qt-mt323:qt-mt323.dll
 0002:0000042c       __imp_?drawContentsOffset@QListView@@MAEXPAVQPainter@@HHHHHH@Z 1002442c     qt-mt323:qt-mt323.dll
 0002:00000430       __imp_?drawFrame@QDockWindow@@MAEXPAVQPainter@@@Z 10024430     qt-mt323:qt-mt323.dll
 0002:00000434       __imp_?drawFrame@QFrame@@MAEXPAVQPainter@@@Z 10024434     qt-mt323:qt-mt323.dll
 0002:00000438       __imp_?dropEvent@QLineEdit@@MAEXPAVQDropEvent@@@Z 10024438     qt-mt323:qt-mt323.dll
 0002:0000043c       __imp_?dropEvent@QWidget@@MAEXPAVQDropEvent@@@Z 1002443c     qt-mt323:qt-mt323.dll
 0002:00000440       __imp_?dropped@QListViewItem@@MAEXPAVQDropEvent@@@Z 10024440     qt-mt323:qt-mt323.dll
 0002:00000444       __imp_?enabledChange@QButton@@MAEX_N@Z 10024444     qt-mt323:qt-mt323.dll
 0002:00000448       __imp_?enabledChange@QPopupMenu@@MAEX_N@Z 10024448     qt-mt323:qt-mt323.dll
 0002:0000044c       __imp_?enabledChange@QWidget@@MAEX_N@Z 1002444c     qt-mt323:qt-mt323.dll
 0002:00000450       __imp_?enforceSortOrder@QListViewItem@@MBEXXZ 10024450     qt-mt323:qt-mt323.dll
 0002:00000454       __imp_?enterEvent@QWidget@@MAEXPAVQEvent@@@Z 10024454     qt-mt323:qt-mt323.dll
 0002:00000458       __imp_?event@QDockWindow@@MAE_NPAVQEvent@@@Z 10024458     qt-mt323:qt-mt323.dll
 0002:0000045c       __imp_?event@QLineEdit@@MAE_NPAVQEvent@@@Z 1002445c     qt-mt323:qt-mt323.dll
 0002:00000460       __imp_?event@QObject@@UAE_NPAVQEvent@@@Z 10024460     qt-mt323:qt-mt323.dll
 0002:00000464       __imp_?event@QToolBar@@UAE_NPAVQEvent@@@Z 10024464     qt-mt323:qt-mt323.dll
 0002:00000468       __imp_?event@QWidget@@MAE_NPAVQEvent@@@Z 10024468     qt-mt323:qt-mt323.dll
 0002:0000046c       __imp_?eventFilter@QDockWindow@@UAE_NPAVQObject@@PAVQEvent@@@Z 1002446c     qt-mt323:qt-mt323.dll
 0002:00000470       __imp_?eventFilter@QLayout@@MAE_NPAVQObject@@PAVQEvent@@@Z 10024470     qt-mt323:qt-mt323.dll
 0002:00000474       __imp_?eventFilter@QListView@@UAE_NPAVQObject@@PAVQEvent@@@Z 10024474     qt-mt323:qt-mt323.dll
 0002:00000478       __imp_?eventFilter@QObject@@UAE_NPAV1@PAVQEvent@@@Z 10024478     qt-mt323:qt-mt323.dll
 0002:0000047c       __imp_?eventFilter@QTabWidget@@MAE_NPAVQObject@@PAVQEvent@@@Z 1002447c     qt-mt323:qt-mt323.dll
 0002:00000480       __imp_?expanding@QBoxLayout@@UBE?AW4ExpandData@QSizePolicy@@XZ 10024480     qt-mt323:qt-mt323.dll
 0002:00000484       __imp_?expanding@QSpacerItem@@UBE?AW4ExpandData@QSizePolicy@@XZ 10024484     qt-mt323:qt-mt323.dll
 0002:00000488       __imp_?focusInEvent@QLineEdit@@MAEXPAVQFocusEvent@@@Z 10024488     qt-mt323:qt-mt323.dll
 0002:0000048c       __imp_?focusInEvent@QListView@@MAEXPAVQFocusEvent@@@Z 1002448c     qt-mt323:qt-mt323.dll
 0002:00000490       __imp_?focusInEvent@QPopupMenu@@MAEXPAVQFocusEvent@@@Z 10024490     qt-mt323:qt-mt323.dll
 0002:00000494       __imp_?focusInEvent@QPushButton@@MAEXPAVQFocusEvent@@@Z 10024494     qt-mt323:qt-mt323.dll
 0002:00000498       __imp_?focusInEvent@QWidget@@MAEXPAVQFocusEvent@@@Z 10024498     qt-mt323:qt-mt323.dll
 0002:0000049c       __imp_?focusNextPrevChild@QPopupMenu@@MAE_N_N@Z 1002449c     qt-mt323:qt-mt323.dll
 0002:000004a0       __imp_?focusNextPrevChild@QScrollView@@MAE_N_N@Z 100244a0     qt-mt323:qt-mt323.dll
 0002:000004a4       __imp_?focusNextPrevChild@QWidget@@MAE_N_N@Z 100244a4     qt-mt323:qt-mt323.dll
 0002:000004a8       __imp_?focusOutEvent@QLineEdit@@MAEXPAVQFocusEvent@@@Z 100244a8     qt-mt323:qt-mt323.dll
 0002:000004ac       __imp_?focusOutEvent@QListView@@MAEXPAVQFocusEvent@@@Z 100244ac     qt-mt323:qt-mt323.dll
 0002:000004b0       __imp_?focusOutEvent@QPopupMenu@@MAEXPAVQFocusEvent@@@Z 100244b0     qt-mt323:qt-mt323.dll
 0002:000004b4       __imp_?focusOutEvent@QPushButton@@MAEXPAVQFocusEvent@@@Z 100244b4     qt-mt323:qt-mt323.dll
 0002:000004b8       __imp_?focusOutEvent@QWidget@@MAEXPAVQFocusEvent@@@Z 100244b8     qt-mt323:qt-mt323.dll
 0002:000004bc       __imp_?fontChange@QLabel@@MAEXABVQFont@@@Z 100244bc     qt-mt323:qt-mt323.dll
 0002:000004c0       __imp_?fontChange@QScrollView@@MAEXABVQFont@@@Z 100244c0     qt-mt323:qt-mt323.dll
 0002:000004c4       __imp_?fontChange@QWidget@@MAEXABVQFont@@@Z 100244c4     qt-mt323:qt-mt323.dll
 0002:000004c8       __imp_?fontInf@QPaintDevice@@MBEHPAVQFont@@H@Z 100244c8     qt-mt323:qt-mt323.dll
 0002:000004cc       __imp_?fontMet@QPaintDevice@@MBEHPAVQFont@@HPBDH@Z 100244cc     qt-mt323:qt-mt323.dll
 0002:000004d0       __imp_?frameChanged@QFrame@@MAEXXZ 100244d0     qt-mt323:qt-mt323.dll
 0002:000004d4       __imp_?frameChanged@QHBox@@MAEXXZ 100244d4     qt-mt323:qt-mt323.dll
 0002:000004d8       __imp_?frameChanged@QPopupMenu@@EAEXXZ 100244d8     qt-mt323:qt-mt323.dll
 0002:000004dc       __imp_?frameChanged@QScrollView@@MAEXXZ 100244dc     qt-mt323:qt-mt323.dll
 0002:000004e0       __imp_?geometry@QLayout@@UBE?AVQRect@@XZ 100244e0     qt-mt323:qt-mt323.dll
 0002:000004e4       __imp_?geometry@QSpacerItem@@UBE?AVQRect@@XZ 100244e4     qt-mt323:qt-mt323.dll
 0002:000004e8       __imp_?handle@QPaintDevice@@UBEPAUHDC__@@XZ 100244e8     qt-mt323:qt-mt323.dll
 0002:000004ec       __imp_?hasHeightForWidth@QBoxLayout@@UBE_NXZ 100244ec     qt-mt323:qt-mt323.dll
 0002:000004f0       __imp_?hasHeightForWidth@QLayoutItem@@UBE_NXZ 100244f0     qt-mt323:qt-mt323.dll
 0002:000004f4       __imp_?heightForWidth@QBoxLayout@@UBEHH@Z 100244f4     qt-mt323:qt-mt323.dll
 0002:000004f8       __imp_?heightForWidth@QLabel@@UBEHH@Z 100244f8     qt-mt323:qt-mt323.dll
 0002:000004fc       __imp_?heightForWidth@QLayoutItem@@UBEHH@Z 100244fc     qt-mt323:qt-mt323.dll
 0002:00000500       __imp_?heightForWidth@QWidget@@UBEHH@Z 10024500     qt-mt323:qt-mt323.dll
 0002:00000504       __imp_?hide@QPopupMenu@@UAEXXZ 10024504     qt-mt323:qt-mt323.dll
 0002:00000508       __imp_?hide@QToolBar@@UAEXXZ 10024508     qt-mt323:qt-mt323.dll
 0002:0000050c       __imp_?hide@QWidget@@UAEXXZ 1002450c     qt-mt323:qt-mt323.dll
 0002:00000510       __imp_?hideEvent@QDockWindow@@MAEXPAVQHideEvent@@@Z 10024510     qt-mt323:qt-mt323.dll
 0002:00000514       __imp_?hideEvent@QWidget@@MAEXPAVQHideEvent@@@Z 10024514     qt-mt323:qt-mt323.dll
 0002:00000518       __imp_?hitButton@QButton@@MBE_NABVQPoint@@@Z 10024518     qt-mt323:qt-mt323.dll
 0002:0000051c       __imp_?imComposeEvent@QLineEdit@@MAEXPAVQIMEvent@@@Z 1002451c     qt-mt323:qt-mt323.dll
 0002:00000520       __imp_?imComposeEvent@QWidget@@MAEXPAVQIMEvent@@@Z 10024520     qt-mt323:qt-mt323.dll
 0002:00000524       __imp_?imEndEvent@QLineEdit@@MAEXPAVQIMEvent@@@Z 10024524     qt-mt323:qt-mt323.dll
 0002:00000528       __imp_?imEndEvent@QWidget@@MAEXPAVQIMEvent@@@Z 10024528     qt-mt323:qt-mt323.dll
 0002:0000052c       __imp_?imStartEvent@QLineEdit@@MAEXPAVQIMEvent@@@Z 1002452c     qt-mt323:qt-mt323.dll
 0002:00000530       __imp_?imStartEvent@QWidget@@MAEXPAVQIMEvent@@@Z 10024530     qt-mt323:qt-mt323.dll
 0002:00000534       __imp_?insert@QLineEdit@@UAEXABVQString@@@Z 10024534     qt-mt323:qt-mt323.dll
 0002:00000538       __imp_?insertChild@QObject@@UAEXPAV1@@Z 10024538     qt-mt323:qt-mt323.dll
 0002:0000053c       __imp_?insertItem@QListView@@UAEXPAVQListViewItem@@@Z 1002453c     qt-mt323:qt-mt323.dll
 0002:00000540       __imp_?insertItem@QListViewItem@@UAEXPAV1@@Z 10024540     qt-mt323:qt-mt323.dll
 0002:00000544       __imp_?insertTab@QTabWidget@@UAEXPAVQWidget@@ABVQIconSet@@ABVQString@@H@Z 10024544     qt-mt323:qt-mt323.dll
 0002:00000548       __imp_?insertTab@QTabWidget@@UAEXPAVQWidget@@ABVQString@@H@Z 10024548     qt-mt323:qt-mt323.dll
 0002:0000054c       __imp_?insertTab@QTabWidget@@UAEXPAVQWidget@@PAVQTab@@H@Z 1002454c     qt-mt323:qt-mt323.dll
 0002:00000550       __imp_?invalidate@QBoxLayout@@UAEXXZ 10024550     qt-mt323:qt-mt323.dll
 0002:00000554       __imp_?invalidate@QLayoutItem@@UAEXXZ 10024554     qt-mt323:qt-mt323.dll
 0002:00000558       __imp_?invalidateHeight@QListViewItem@@UAEXXZ 10024558     qt-mt323:qt-mt323.dll
 0002:0000055c       __imp_?invertSelection@QListView@@UAEXXZ 1002455c     qt-mt323:qt-mt323.dll
 0002:00000560       __imp_?isEmpty@QLayout@@UBE_NXZ 10024560     qt-mt323:qt-mt323.dll
 0002:00000564       __imp_?isEmpty@QSpacerItem@@UBE_NXZ 10024564     qt-mt323:qt-mt323.dll
 0002:00000568       __imp_?iterator@QBoxLayout@@UAE?AVQLayoutIterator@@XZ 10024568     qt-mt323:qt-mt323.dll
 0002:0000056c       __imp_?iterator@QLayoutItem@@UAE?AVQLayoutIterator@@XZ 1002456c     qt-mt323:qt-mt323.dll
 0002:00000570       __imp_?key@QListViewItem@@UBE?AVQString@@H_N@Z 10024570     qt-mt323:qt-mt323.dll
 0002:00000574       __imp_?keyPressEvent@QButton@@MAEXPAVQKeyEvent@@@Z 10024574     qt-mt323:qt-mt323.dll
 0002:00000578       __imp_?keyPressEvent@QLineEdit@@MAEXPAVQKeyEvent@@@Z 10024578     qt-mt323:qt-mt323.dll
 0002:0000057c       __imp_?keyPressEvent@QPopupMenu@@MAEXPAVQKeyEvent@@@Z 1002457c     qt-mt323:qt-mt323.dll
 0002:00000580       __imp_?keyPressEvent@QWidget@@MAEXPAVQKeyEvent@@@Z 10024580     qt-mt323:qt-mt323.dll
 0002:00000584       __imp_?keyReleaseEvent@QButton@@MAEXPAVQKeyEvent@@@Z 10024584     qt-mt323:qt-mt323.dll
 0002:00000588       __imp_?keyReleaseEvent@QWidget@@MAEXPAVQKeyEvent@@@Z 10024588     qt-mt323:qt-mt323.dll
 0002:0000058c       __imp_?layout@QLayout@@UAEPAV1@XZ 1002458c     qt-mt323:qt-mt323.dll
 0002:00000590       __imp_?layout@QLayoutItem@@UAEPAVQLayout@@XZ 10024590     qt-mt323:qt-mt323.dll
 0002:00000594       __imp_?leaveEvent@QPopupMenu@@MAEXPAVQEvent@@@Z 10024594     qt-mt323:qt-mt323.dll
 0002:00000598       __imp_?leaveEvent@QWidget@@MAEXPAVQEvent@@@Z 10024598     qt-mt323:qt-mt323.dll
 0002:0000059c       __imp_?maximumSize@QBoxLayout@@UBE?AVQSize@@XZ 1002459c     qt-mt323:qt-mt323.dll
 0002:000005a0       __imp_?maximumSize@QSpacerItem@@UBE?AVQSize@@XZ 100245a0     qt-mt323:qt-mt323.dll
 0002:000005a4       __imp_?menuContentsChanged@QPopupMenu@@EAEXXZ 100245a4     qt-mt323:qt-mt323.dll
 0002:000005a8       __imp_?menuDelPopup@QPopupMenu@@EAEXPAV1@@Z 100245a8     qt-mt323:qt-mt323.dll
 0002:000005ac       __imp_?menuInsPopup@QPopupMenu@@EAEXPAV1@@Z 100245ac     qt-mt323:qt-mt323.dll
 0002:000005b0       __imp_?menuStateChanged@QPopupMenu@@EAEXXZ 100245b0     qt-mt323:qt-mt323.dll
 0002:000005b4       __imp_?metaObject@QAction@@UBEPAVQMetaObject@@XZ 100245b4     qt-mt323:qt-mt323.dll
 0002:000005b8       __imp_?metaObject@QDockWindow@@UBEPAVQMetaObject@@XZ 100245b8     qt-mt323:qt-mt323.dll
 0002:000005bc       __imp_?metaObject@QGuardedPtrPrivate@@UBEPAVQMetaObject@@XZ 100245bc     qt-mt323:qt-mt323.dll
 0002:000005c0       __imp_?metaObject@QHBoxLayout@@UBEPAVQMetaObject@@XZ 100245c0     qt-mt323:qt-mt323.dll
 0002:000005c4       __imp_?metaObject@QLabel@@UBEPAVQMetaObject@@XZ 100245c4     qt-mt323:qt-mt323.dll
 0002:000005c8       __imp_?metaObject@QLineEdit@@UBEPAVQMetaObject@@XZ 100245c8     qt-mt323:qt-mt323.dll
 0002:000005cc       __imp_?metaObject@QListView@@UBEPAVQMetaObject@@XZ 100245cc     qt-mt323:qt-mt323.dll
 0002:000005d0       __imp_?metaObject@QPopupMenu@@UBEPAVQMetaObject@@XZ 100245d0     qt-mt323:qt-mt323.dll
 0002:000005d4       __imp_?metaObject@QPushButton@@UBEPAVQMetaObject@@XZ 100245d4     qt-mt323:qt-mt323.dll
 0002:000005d8       __imp_?metaObject@QTabWidget@@UBEPAVQMetaObject@@XZ 100245d8     qt-mt323:qt-mt323.dll
 0002:000005dc       __imp_?metaObject@QToolBar@@UBEPAVQMetaObject@@XZ 100245dc     qt-mt323:qt-mt323.dll
 0002:000005e0       __imp_?metaObject@QVBoxLayout@@UBEPAVQMetaObject@@XZ 100245e0     qt-mt323:qt-mt323.dll
 0002:000005e4       __imp_?metaObject@QWidget@@UBEPAVQMetaObject@@XZ 100245e4     qt-mt323:qt-mt323.dll
 0002:000005e8       __imp_?metric@QWidget@@MBEHH@Z 100245e8     qt-mt323:qt-mt323.dll
 0002:000005ec       __imp_?minimumSize@QBoxLayout@@UBE?AVQSize@@XZ 100245ec     qt-mt323:qt-mt323.dll
 0002:000005f0       __imp_?minimumSize@QSpacerItem@@UBE?AVQSize@@XZ 100245f0     qt-mt323:qt-mt323.dll
 0002:000005f4       __imp_?minimumSizeHint@QDockWindow@@UBE?AVQSize@@XZ 100245f4     qt-mt323:qt-mt323.dll
 0002:000005f8       __imp_?minimumSizeHint@QLabel@@UBE?AVQSize@@XZ 100245f8     qt-mt323:qt-mt323.dll
 0002:000005fc       __imp_?minimumSizeHint@QLineEdit@@UBE?AVQSize@@XZ 100245fc     qt-mt323:qt-mt323.dll
 0002:00000600       __imp_?minimumSizeHint@QListView@@UBE?AVQSize@@XZ 10024600     qt-mt323:qt-mt323.dll
 0002:00000604       __imp_?minimumSizeHint@QTabWidget@@UBE?AVQSize@@XZ 10024604     qt-mt323:qt-mt323.dll
 0002:00000608       __imp_?minimumSizeHint@QToolBar@@UBE?AVQSize@@XZ 10024608     qt-mt323:qt-mt323.dll
 0002:0000060c       __imp_?minimumSizeHint@QWidget@@UBE?AVQSize@@XZ 1002460c     qt-mt323:qt-mt323.dll
 0002:00000610       __imp_?mouseDoubleClickEvent@QLineEdit@@MAEXPAVQMouseEvent@@@Z 10024610     qt-mt323:qt-mt323.dll
 0002:00000614       __imp_?mouseDoubleClickEvent@QScrollView@@MAEXPAVQMouseEvent@@@Z 10024614     qt-mt323:qt-mt323.dll
 0002:00000618       __imp_?mouseDoubleClickEvent@QWidget@@MAEXPAVQMouseEvent@@@Z 10024618     qt-mt323:qt-mt323.dll
 0002:0000061c       __imp_?mouseMoveEvent@QButton@@MAEXPAVQMouseEvent@@@Z 1002461c     qt-mt323:qt-mt323.dll
 0002:00000620       __imp_?mouseMoveEvent@QLineEdit@@MAEXPAVQMouseEvent@@@Z 10024620     qt-mt323:qt-mt323.dll
 0002:00000624       __imp_?mouseMoveEvent@QPopupMenu@@MAEXPAVQMouseEvent@@@Z 10024624     qt-mt323:qt-mt323.dll
 0002:00000628       __imp_?mouseMoveEvent@QScrollView@@MAEXPAVQMouseEvent@@@Z 10024628     qt-mt323:qt-mt323.dll
 0002:0000062c       __imp_?mouseMoveEvent@QWidget@@MAEXPAVQMouseEvent@@@Z 1002462c     qt-mt323:qt-mt323.dll
 0002:00000630       __imp_?mousePressEvent@QButton@@MAEXPAVQMouseEvent@@@Z 10024630     qt-mt323:qt-mt323.dll
 0002:00000634       __imp_?mousePressEvent@QLineEdit@@MAEXPAVQMouseEvent@@@Z 10024634     qt-mt323:qt-mt323.dll
 0002:00000638       __imp_?mousePressEvent@QPopupMenu@@MAEXPAVQMouseEvent@@@Z 10024638     qt-mt323:qt-mt323.dll
 0002:0000063c       __imp_?mousePressEvent@QScrollView@@MAEXPAVQMouseEvent@@@Z 1002463c     qt-mt323:qt-mt323.dll
 0002:00000640       __imp_?mousePressEvent@QWidget@@MAEXPAVQMouseEvent@@@Z 10024640     qt-mt323:qt-mt323.dll
 0002:00000644       __imp_?mouseReleaseEvent@QButton@@MAEXPAVQMouseEvent@@@Z 10024644     qt-mt323:qt-mt323.dll
 0002:00000648       __imp_?mouseReleaseEvent@QLineEdit@@MAEXPAVQMouseEvent@@@Z 10024648     qt-mt323:qt-mt323.dll
 0002:0000064c       __imp_?mouseReleaseEvent@QPopupMenu@@MAEXPAVQMouseEvent@@@Z 1002464c     qt-mt323:qt-mt323.dll
 0002:00000650       __imp_?mouseReleaseEvent@QScrollView@@MAEXPAVQMouseEvent@@@Z 10024650     qt-mt323:qt-mt323.dll
 0002:00000654       __imp_?mouseReleaseEvent@QWidget@@MAEXPAVQMouseEvent@@@Z 10024654     qt-mt323:qt-mt323.dll
 0002:00000658       __imp_?move@QPushButton@@UAEXHH@Z 10024658     qt-mt323:qt-mt323.dll
 0002:0000065c       __imp_?move@QWidget@@UAEXHH@Z 1002465c     qt-mt323:qt-mt323.dll
 0002:00000660       __imp_?moveChild@QScrollView@@UAEXPAVQWidget@@HH@Z 10024660     qt-mt323:qt-mt323.dll
 0002:00000664       __imp_?moveEvent@QWidget@@MAEXPAVQMoveEvent@@@Z 10024664     qt-mt323:qt-mt323.dll
 0002:00000668       __imp_?newItem@QPtrCollection@@MAEPAXPAX@Z 10024668     qt-mt323:qt-mt323.dll
 0002:0000066c       __imp_?okRename@QListViewItem@@MAEXH@Z 1002466c     qt-mt323:qt-mt323.dll
 0002:00000670       __imp_?paintBranches@QListViewItem@@UAEXPAVQPainter@@ABVQColorGroup@@HHH@Z 10024670     qt-mt323:qt-mt323.dll
 0002:00000674       __imp_?paintEmptyArea@QListView@@MAEXPAVQPainter@@ABVQRect@@@Z 10024674     qt-mt323:qt-mt323.dll
 0002:00000678       __imp_?paintEvent@QButton@@MAEXPAVQPaintEvent@@@Z 10024678     qt-mt323:qt-mt323.dll
 0002:0000067c       __imp_?paintEvent@QFrame@@MAEXPAVQPaintEvent@@@Z 1002467c     qt-mt323:qt-mt323.dll
 0002:00000680       __imp_?paintEvent@QPopupMenu@@MAEXPAVQPaintEvent@@@Z 10024680     qt-mt323:qt-mt323.dll
 0002:00000684       __imp_?paintEvent@QWidget@@MAEXPAVQPaintEvent@@@Z 10024684     qt-mt323:qt-mt323.dll
 0002:00000688       __imp_?paintFocus@QListViewItem@@UAEXPAVQPainter@@ABVQColorGroup@@ABVQRect@@@Z 10024688     qt-mt323:qt-mt323.dll
 0002:0000068c       __imp_?paletteChange@QWidget@@MAEXABVQPalette@@@Z 1002468c     qt-mt323:qt-mt323.dll
 0002:00000690       __imp_?paste@QLineEdit@@UAEXXZ 10024690     qt-mt323:qt-mt323.dll
 0002:00000694       __imp_?pixmap@QListViewItem@@UBEPBVQPixmap@@H@Z 10024694     qt-mt323:qt-mt323.dll
 0002:00000698       __imp_?polish@QWidget@@UAEXXZ 10024698     qt-mt323:qt-mt323.dll
 0002:0000069c       __imp_?property@QObject@@UBE?AVQVariant@@PBD@Z 1002469c     qt-mt323:qt-mt323.dll
 0002:000006a0       __imp_?qt_cast@QAction@@UAEPAXPBD@Z 100246a0     qt-mt323:qt-mt323.dll
 0002:000006a4       __imp_?qt_cast@QDockWindow@@UAEPAXPBD@Z 100246a4     qt-mt323:qt-mt323.dll
 0002:000006a8       __imp_?qt_cast@QGuardedPtrPrivate@@UAEPAXPBD@Z 100246a8     qt-mt323:qt-mt323.dll
 0002:000006ac       __imp_?qt_cast@QHBoxLayout@@UAEPAXPBD@Z 100246ac     qt-mt323:qt-mt323.dll
 0002:000006b0       __imp_?qt_cast@QLabel@@UAEPAXPBD@Z 100246b0     qt-mt323:qt-mt323.dll
 0002:000006b4       __imp_?qt_cast@QLineEdit@@UAEPAXPBD@Z 100246b4     qt-mt323:qt-mt323.dll
 0002:000006b8       __imp_?qt_cast@QListView@@UAEPAXPBD@Z 100246b8     qt-mt323:qt-mt323.dll
 0002:000006bc       __imp_?qt_cast@QPopupMenu@@UAEPAXPBD@Z 100246bc     qt-mt323:qt-mt323.dll
 0002:000006c0       __imp_?qt_cast@QPushButton@@UAEPAXPBD@Z 100246c0     qt-mt323:qt-mt323.dll
 0002:000006c4       __imp_?qt_cast@QTabWidget@@UAEPAXPBD@Z 100246c4     qt-mt323:qt-mt323.dll
 0002:000006c8       __imp_?qt_cast@QToolBar@@UAEPAXPBD@Z 100246c8     qt-mt323:qt-mt323.dll
 0002:000006cc       __imp_?qt_cast@QVBoxLayout@@UAEPAXPBD@Z 100246cc     qt-mt323:qt-mt323.dll
 0002:000006d0       __imp_?qt_cast@QWidget@@UAEPAXPBD@Z 100246d0     qt-mt323:qt-mt323.dll
 0002:000006d4       __imp_?qt_emit@QAction@@UAE_NHPAUQUObject@@@Z 100246d4     qt-mt323:qt-mt323.dll
 0002:000006d8       __imp_?qt_emit@QDockWindow@@UAE_NHPAUQUObject@@@Z 100246d8     qt-mt323:qt-mt323.dll
 0002:000006dc       __imp_?qt_emit@QGuardedPtrPrivate@@UAE_NHPAUQUObject@@@Z 100246dc     qt-mt323:qt-mt323.dll
 0002:000006e0       __imp_?qt_emit@QHBoxLayout@@UAE_NHPAUQUObject@@@Z 100246e0     qt-mt323:qt-mt323.dll
 0002:000006e4       __imp_?qt_emit@QLabel@@UAE_NHPAUQUObject@@@Z 100246e4     qt-mt323:qt-mt323.dll
 0002:000006e8       __imp_?qt_emit@QLineEdit@@UAE_NHPAUQUObject@@@Z 100246e8     qt-mt323:qt-mt323.dll
 0002:000006ec       __imp_?qt_emit@QListView@@UAE_NHPAUQUObject@@@Z 100246ec     qt-mt323:qt-mt323.dll
 0002:000006f0       __imp_?qt_emit@QPopupMenu@@UAE_NHPAUQUObject@@@Z 100246f0     qt-mt323:qt-mt323.dll
 0002:000006f4       __imp_?qt_emit@QPushButton@@UAE_NHPAUQUObject@@@Z 100246f4     qt-mt323:qt-mt323.dll
 0002:000006f8       __imp_?qt_emit@QTabWidget@@UAE_NHPAUQUObject@@@Z 100246f8     qt-mt323:qt-mt323.dll
 0002:000006fc       __imp_?qt_emit@QToolBar@@UAE_NHPAUQUObject@@@Z 100246fc     qt-mt323:qt-mt323.dll
 0002:00000700       __imp_?qt_emit@QVBoxLayout@@UAE_NHPAUQUObject@@@Z 10024700     qt-mt323:qt-mt323.dll
 0002:00000704       __imp_?qt_emit@QWidget@@UAE_NHPAUQUObject@@@Z 10024704     qt-mt323:qt-mt323.dll
 0002:00000708       __imp_?qt_invoke@QAction@@UAE_NHPAUQUObject@@@Z 10024708     qt-mt323:qt-mt323.dll
 0002:0000070c       __imp_?qt_invoke@QDockWindow@@UAE_NHPAUQUObject@@@Z 1002470c     qt-mt323:qt-mt323.dll
 0002:00000710       __imp_?qt_invoke@QGuardedPtrPrivate@@UAE_NHPAUQUObject@@@Z 10024710     qt-mt323:qt-mt323.dll
 0002:00000714       __imp_?qt_invoke@QHBoxLayout@@UAE_NHPAUQUObject@@@Z 10024714     qt-mt323:qt-mt323.dll
 0002:00000718       __imp_?qt_invoke@QLabel@@UAE_NHPAUQUObject@@@Z 10024718     qt-mt323:qt-mt323.dll
 0002:0000071c       __imp_?qt_invoke@QLineEdit@@UAE_NHPAUQUObject@@@Z 1002471c     qt-mt323:qt-mt323.dll
 0002:00000720       __imp_?qt_invoke@QListView@@UAE_NHPAUQUObject@@@Z 10024720     qt-mt323:qt-mt323.dll
 0002:00000724       __imp_?qt_invoke@QPopupMenu@@UAE_NHPAUQUObject@@@Z 10024724     qt-mt323:qt-mt323.dll
 0002:00000728       __imp_?qt_invoke@QPushButton@@UAE_NHPAUQUObject@@@Z 10024728     qt-mt323:qt-mt323.dll
 0002:0000072c       __imp_?qt_invoke@QTabWidget@@UAE_NHPAUQUObject@@@Z 1002472c     qt-mt323:qt-mt323.dll
 0002:00000730       __imp_?qt_invoke@QToolBar@@UAE_NHPAUQUObject@@@Z 10024730     qt-mt323:qt-mt323.dll
 0002:00000734       __imp_?qt_invoke@QVBoxLayout@@UAE_NHPAUQUObject@@@Z 10024734     qt-mt323:qt-mt323.dll
 0002:00000738       __imp_?qt_invoke@QWidget@@UAE_NHPAUQUObject@@@Z 10024738     qt-mt323:qt-mt323.dll
 0002:0000073c       __imp_?qt_property@QAction@@UAE_NHHPAVQVariant@@@Z 1002473c     qt-mt323:qt-mt323.dll
 0002:00000740       __imp_?qt_property@QDockWindow@@UAE_NHHPAVQVariant@@@Z 10024740     qt-mt323:qt-mt323.dll
 0002:00000744       __imp_?qt_property@QGuardedPtrPrivate@@UAE_NHHPAVQVariant@@@Z 10024744     qt-mt323:qt-mt323.dll
 0002:00000748       __imp_?qt_property@QHBoxLayout@@UAE_NHHPAVQVariant@@@Z 10024748     qt-mt323:qt-mt323.dll
 0002:0000074c       __imp_?qt_property@QLabel@@UAE_NHHPAVQVariant@@@Z 1002474c     qt-mt323:qt-mt323.dll
 0002:00000750       __imp_?qt_property@QLineEdit@@UAE_NHHPAVQVariant@@@Z 10024750     qt-mt323:qt-mt323.dll
 0002:00000754       __imp_?qt_property@QListView@@UAE_NHHPAVQVariant@@@Z 10024754     qt-mt323:qt-mt323.dll
 0002:00000758       __imp_?qt_property@QPopupMenu@@UAE_NHHPAVQVariant@@@Z 10024758     qt-mt323:qt-mt323.dll
 0002:0000075c       __imp_?qt_property@QPushButton@@UAE_NHHPAVQVariant@@@Z 1002475c     qt-mt323:qt-mt323.dll
 0002:00000760       __imp_?qt_property@QTabWidget@@UAE_NHHPAVQVariant@@@Z 10024760     qt-mt323:qt-mt323.dll
 0002:00000764       __imp_?qt_property@QToolBar@@UAE_NHHPAVQVariant@@@Z 10024764     qt-mt323:qt-mt323.dll
 0002:00000768       __imp_?qt_property@QVBoxLayout@@UAE_NHHPAVQVariant@@@Z 10024768     qt-mt323:qt-mt323.dll
 0002:0000076c       __imp_?qt_property@QWidget@@UAE_NHHPAVQVariant@@@Z 1002476c     qt-mt323:qt-mt323.dll
 0002:00000770       __imp_?read@QGList@@MAEAAVQDataStream@@AAV2@AAPAX@Z 10024770     qt-mt323:qt-mt323.dll
 0002:00000774       __imp_?redo@QLineEdit@@UAEXXZ 10024774     qt-mt323:qt-mt323.dll
 0002:00000778       __imp_?removeChild@QObject@@UAEXPAV1@@Z 10024778     qt-mt323:qt-mt323.dll
 0002:0000077c       __imp_?removeChild@QScrollView@@UAEXPAVQObject@@@Z 1002477c     qt-mt323:qt-mt323.dll
 0002:00000780       __imp_?removeColumn@QListView@@UAEXH@Z 10024780     qt-mt323:qt-mt323.dll
 0002:00000784       __imp_?removeFrom@QAction@@UAE_NPAVQWidget@@@Z 10024784     qt-mt323:qt-mt323.dll
 0002:00000788       __imp_?removeItem@QListView@@UAEXPAVQListViewItem@@@Z 10024788     qt-mt323:qt-mt323.dll
 0002:0000078c       __imp_?removeItem@QListViewItem@@UAEXPAV1@@Z 1002478c     qt-mt323:qt-mt323.dll
 0002:00000790       __imp_?removePage@QTabWidget@@UAEXPAVQWidget@@@Z 10024790     qt-mt323:qt-mt323.dll
 0002:00000794       __imp_?reparent@QWidget@@UAEXPAV1@IABVQPoint@@_N@Z 10024794     qt-mt323:qt-mt323.dll
 0002:00000798       __imp_?resize@QPushButton@@UAEXHH@Z 10024798     qt-mt323:qt-mt323.dll
 0002:0000079c       __imp_?resize@QScrollView@@UAEXHH@Z 1002479c     qt-mt323:qt-mt323.dll
 0002:000007a0       __imp_?resize@QWidget@@UAEXHH@Z 100247a0     qt-mt323:qt-mt323.dll
 0002:000007a4       __imp_?resizeContents@QScrollView@@UAEXHH@Z 100247a4     qt-mt323:qt-mt323.dll
 0002:000007a8       __imp_?resizeEvent@QDockWindow@@MAEXPAVQResizeEvent@@@Z 100247a8     qt-mt323:qt-mt323.dll
 0002:000007ac       __imp_?resizeEvent@QFrame@@MAEXPAVQResizeEvent@@@Z 100247ac     qt-mt323:qt-mt323.dll
 0002:000007b0       __imp_?resizeEvent@QLabel@@MAEXPAVQResizeEvent@@@Z 100247b0     qt-mt323:qt-mt323.dll
 0002:000007b4       __imp_?resizeEvent@QLineEdit@@MAEXPAVQResizeEvent@@@Z 100247b4     qt-mt323:qt-mt323.dll
 0002:000007b8       __imp_?resizeEvent@QListView@@MAEXPAVQResizeEvent@@@Z 100247b8     qt-mt323:qt-mt323.dll
 0002:000007bc       __imp_?resizeEvent@QPushButton@@MAEXPAVQResizeEvent@@@Z 100247bc     qt-mt323:qt-mt323.dll
 0002:000007c0       __imp_?resizeEvent@QTabWidget@@MAEXPAVQResizeEvent@@@Z 100247c0     qt-mt323:qt-mt323.dll
 0002:000007c4       __imp_?resizeEvent@QToolBar@@MAEXPAVQResizeEvent@@@Z 100247c4     qt-mt323:qt-mt323.dll
 0002:000007c8       __imp_?resizeEvent@QWidget@@MAEXPAVQResizeEvent@@@Z 100247c8     qt-mt323:qt-mt323.dll
 0002:000007cc       __imp_?resolution@QPaintDevice@@UBEHXZ 100247cc     qt-mt323:qt-mt323.dll
 0002:000007d0       __imp_?rtti@QListViewItem@@UBEHXZ 100247d0     qt-mt323:qt-mt323.dll
 0002:000007d4       __imp_?selectAll@QLineEdit@@UAEXXZ 100247d4     qt-mt323:qt-mt323.dll
 0002:000007d8       __imp_?selectAll@QListView@@UAEX_N@Z 100247d8     qt-mt323:qt-mt323.dll
 0002:000007dc       __imp_?setAccel@QAction@@UAEXABVQKeySequence@@@Z 100247dc     qt-mt323:qt-mt323.dll
 0002:000007e0       __imp_?setAccel@QButton@@UAEXABVQKeySequence@@@Z 100247e0     qt-mt323:qt-mt323.dll
 0002:000007e4       __imp_?setAcceptDrops@QWidget@@UAEX_N@Z 100247e4     qt-mt323:qt-mt323.dll
 0002:000007e8       __imp_?setActiveItem@QPopupMenu@@UAEXH@Z 100247e8     qt-mt323:qt-mt323.dll
 0002:000007ec       __imp_?setActiveWindow@QWidget@@UAEXXZ 100247ec     qt-mt323:qt-mt323.dll
 0002:000007f0       __imp_?setAlignment@QLabel@@UAEXH@Z 100247f0     qt-mt323:qt-mt323.dll
 0002:000007f4       __imp_?setAlignment@QLayoutItem@@UAEXH@Z 100247f4     qt-mt323:qt-mt323.dll
 0002:000007f8       __imp_?setAlignment@QLineEdit@@UAEXH@Z 100247f8     qt-mt323:qt-mt323.dll
 0002:000007fc       __imp_?setAllColumnsShowFocus@QListView@@UAEX_N@Z 100247fc     qt-mt323:qt-mt323.dll
 0002:00000800       __imp_?setAutoAdd@QLayout@@UAEX_N@Z 10024800     qt-mt323:qt-mt323.dll
 0002:00000804       __imp_?setAutoDefault@QPushButton@@UAEX_N@Z 10024804     qt-mt323:qt-mt323.dll
 0002:00000808       __imp_?setAutoMask@QWidget@@UAEX_N@Z 10024808     qt-mt323:qt-mt323.dll
 0002:0000080c       __imp_?setAutoRepeat@QButton@@UAEX_N@Z 1002480c     qt-mt323:qt-mt323.dll
 0002:00000810       __imp_?setAutoResize@QLabel@@UAEX_N@Z 10024810     qt-mt323:qt-mt323.dll
 0002:00000814       __imp_?setBackgroundColor@QWidget@@UAEXABVQColor@@@Z 10024814     qt-mt323:qt-mt323.dll
 0002:00000818       __imp_?setBackgroundMode@QWidget@@UAEXW4BackgroundMode@Qt@@@Z 10024818     qt-mt323:qt-mt323.dll
 0002:0000081c       __imp_?setBackgroundOrigin@QWidget@@UAEXW4BackgroundOrigin@1@@Z 1002481c     qt-mt323:qt-mt323.dll
 0002:00000820       __imp_?setBackgroundPixmap@QWidget@@UAEXABVQPixmap@@@Z 10024820     qt-mt323:qt-mt323.dll
 0002:00000824       __imp_?setBuddy@QLabel@@UAEXPAVQWidget@@@Z 10024824     qt-mt323:qt-mt323.dll
 0002:00000828       __imp_?setCaption@QDockWindow@@UAEXABVQString@@@Z 10024828     qt-mt323:qt-mt323.dll
 0002:0000082c       __imp_?setCheckable@QPopupMenu@@UAEX_N@Z 1002482c     qt-mt323:qt-mt323.dll
 0002:00000830       __imp_?setCloseMode@QDockWindow@@UAEXH@Z 10024830     qt-mt323:qt-mt323.dll
 0002:00000834       __imp_?setColumnAlignment@QListView@@UAEXHH@Z 10024834     qt-mt323:qt-mt323.dll
 0002:00000838       __imp_?setColumnText@QListView@@UAEXHABVQIconSet@@ABVQString@@@Z 10024838     qt-mt323:qt-mt323.dll
 0002:0000083c       __imp_?setColumnText@QListView@@UAEXHABVQString@@@Z 1002483c     qt-mt323:qt-mt323.dll
 0002:00000840       __imp_?setColumnWidth@QListView@@UAEXHH@Z 10024840     qt-mt323:qt-mt323.dll
 0002:00000844       __imp_?setColumnWidthMode@QListView@@UAEXHW4WidthMode@1@@Z 10024844     qt-mt323:qt-mt323.dll
 0002:00000848       __imp_?setContentsPos@QListView@@UAEXHH@Z 10024848     qt-mt323:qt-mt323.dll
 0002:0000084c       __imp_?setCornerWidget@QScrollView@@UAEXPAVQWidget@@@Z 1002484c     qt-mt323:qt-mt323.dll
 0002:00000850       __imp_?setCurrentItem@QListView@@UAEXPAVQListViewItem@@@Z 10024850     qt-mt323:qt-mt323.dll
 0002:00000854       __imp_?setCursor@QWidget@@UAEXABVQCursor@@@Z 10024854     qt-mt323:qt-mt323.dll
 0002:00000858       __imp_?setCursorPosition@QLineEdit@@UAEXH@Z 10024858     qt-mt323:qt-mt323.dll
 0002:0000085c       __imp_?setDefault@QPushButton@@UAEX_N@Z 1002485c     qt-mt323:qt-mt323.dll
 0002:00000860       __imp_?setDefaultRenameAction@QListView@@UAEXW4RenameAction@1@@Z 10024860     qt-mt323:qt-mt323.dll
 0002:00000864       __imp_?setDown@QButton@@UAEX_N@Z 10024864     qt-mt323:qt-mt323.dll
 0002:00000868       __imp_?setDragAutoScroll@QScrollView@@UAEX_N@Z 10024868     qt-mt323:qt-mt323.dll
 0002:0000086c       __imp_?setDragEnabled@QLineEdit@@UAEX_N@Z 1002486c     qt-mt323:qt-mt323.dll
 0002:00000870       __imp_?setDragEnabled@QListViewItem@@UAEX_N@Z 10024870     qt-mt323:qt-mt323.dll
 0002:00000874       __imp_?setDropEnabled@QListViewItem@@UAEX_N@Z 10024874     qt-mt323:qt-mt323.dll
 0002:00000878       __imp_?setEchoMode@QLineEdit@@UAEXW4EchoMode@1@@Z 10024878     qt-mt323:qt-mt323.dll
 0002:0000087c       __imp_?setEnabled@QAction@@UAEX_N@Z 1002487c     qt-mt323:qt-mt323.dll
 0002:00000880       __imp_?setEnabled@QListViewItem@@UAEX_N@Z 10024880     qt-mt323:qt-mt323.dll
 0002:00000884       __imp_?setEnabled@QScrollView@@UAEX_N@Z 10024884     qt-mt323:qt-mt323.dll
 0002:00000888       __imp_?setEnabled@QWidget@@UAEX_N@Z 10024888     qt-mt323:qt-mt323.dll
 0002:0000088c       __imp_?setEraseColor@QWidget@@UAEXABVQColor@@@Z 1002488c     qt-mt323:qt-mt323.dll
 0002:00000890       __imp_?setErasePixmap@QWidget@@UAEXABVQPixmap@@@Z 10024890     qt-mt323:qt-mt323.dll
 0002:00000894       __imp_?setExpandable@QListViewItem@@UAEX_N@Z 10024894     qt-mt323:qt-mt323.dll
 0002:00000898       __imp_?setFirstItemActive@QPopupMenu@@EAEXXZ 10024898     qt-mt323:qt-mt323.dll
 0002:0000089c       __imp_?setFixedExtentHeight@QDockWindow@@UAEXH@Z 1002489c     qt-mt323:qt-mt323.dll
 0002:000008a0       __imp_?setFixedExtentWidth@QDockWindow@@UAEXH@Z 100248a0     qt-mt323:qt-mt323.dll
 0002:000008a4       __imp_?setFocus@QWidget@@UAEXXZ 100248a4     qt-mt323:qt-mt323.dll
 0002:000008a8       __imp_?setFocusProxy@QWidget@@UAEXPAV1@@Z 100248a8     qt-mt323:qt-mt323.dll
 0002:000008ac       __imp_?setFont@QLabel@@UAEXABVQFont@@@Z 100248ac     qt-mt323:qt-mt323.dll
 0002:000008b0       __imp_?setFont@QLineEdit@@UAEXABVQFont@@@Z 100248b0     qt-mt323:qt-mt323.dll
 0002:000008b4       __imp_?setFont@QListView@@UAEXABVQFont@@@Z 100248b4     qt-mt323:qt-mt323.dll
 0002:000008b8       __imp_?setFont@QPopupMenu@@UAEXABVQFont@@@Z 100248b8     qt-mt323:qt-mt323.dll
 0002:000008bc       __imp_?setFont@QWidget@@UAEXABVQFont@@@Z 100248bc     qt-mt323:qt-mt323.dll
 0002:000008c0       __imp_?setFrame@QLineEdit@@UAEX_N@Z 100248c0     qt-mt323:qt-mt323.dll
 0002:000008c4       __imp_?setFrameRect@QFrame@@UAEXABVQRect@@@Z 100248c4     qt-mt323:qt-mt323.dll
 0002:000008c8       __imp_?setFrameStyle@QFrame@@UAEXH@Z 100248c8     qt-mt323:qt-mt323.dll
 0002:000008cc       __imp_?setGeometry@QBoxLayout@@UAEXABVQRect@@@Z 100248cc     qt-mt323:qt-mt323.dll
 0002:000008d0       __imp_?setGeometry@QPushButton@@UAEXABVQRect@@@Z 100248d0     qt-mt323:qt-mt323.dll
 0002:000008d4       __imp_?setGeometry@QPushButton@@UAEXHHHH@Z 100248d4     qt-mt323:qt-mt323.dll
 0002:000008d8       __imp_?setGeometry@QSpacerItem@@UAEXABVQRect@@@Z 100248d8     qt-mt323:qt-mt323.dll
 0002:000008dc       __imp_?setGeometry@QWidget@@UAEXABVQRect@@@Z 100248dc     qt-mt323:qt-mt323.dll
 0002:000008e0       __imp_?setGeometry@QWidget@@UAEXHHHH@Z 100248e0     qt-mt323:qt-mt323.dll
 0002:000008e4       __imp_?setGroup@QButton@@EAEXPAVQButtonGroup@@@Z 100248e4     qt-mt323:qt-mt323.dll
 0002:000008e8       __imp_?setHBarGeometry@QScrollView@@MAEXAAVQScrollBar@@HHHH@Z 100248e8     qt-mt323:qt-mt323.dll
 0002:000008ec       __imp_?setHScrollBarMode@QScrollView@@UAEXW4ScrollBarMode@1@@Z 100248ec     qt-mt323:qt-mt323.dll
 0002:000008f0       __imp_?setHeight@QListViewItem@@MAEXH@Z 100248f0     qt-mt323:qt-mt323.dll
 0002:000008f4       __imp_?setHorizontallyStretchable@QDockWindow@@UAEX_N@Z 100248f4     qt-mt323:qt-mt323.dll
 0002:000008f8       __imp_?setIcon@QWidget@@UAEXABVQPixmap@@@Z 100248f8     qt-mt323:qt-mt323.dll
 0002:000008fc       __imp_?setIconSet@QAction@@UAEXABVQIconSet@@@Z 100248fc     qt-mt323:qt-mt323.dll
 0002:00000900       __imp_?setIconText@QWidget@@UAEXABVQString@@@Z 10024900     qt-mt323:qt-mt323.dll
 0002:00000904       __imp_?setId@QMenuData@@UAEXHH@Z 10024904     qt-mt323:qt-mt323.dll
 0002:00000908       __imp_?setIsMenuButton@QPushButton@@UAEX_N@Z 10024908     qt-mt323:qt-mt323.dll
 0002:0000090c       __imp_?setItemMargin@QListView@@UAEXH@Z 1002490c     qt-mt323:qt-mt323.dll
 0002:00000910       __imp_?setKeyCompression@QWidget@@MAEX_N@Z 10024910     qt-mt323:qt-mt323.dll
 0002:00000914       __imp_?setLabel@QToolBar@@UAEXABVQString@@@Z 10024914     qt-mt323:qt-mt323.dll
 0002:00000918       __imp_?setLineWidth@QFrame@@UAEXH@Z 10024918     qt-mt323:qt-mt323.dll
 0002:0000091c       __imp_?setMargin@QFrame@@UAEXH@Z 1002491c     qt-mt323:qt-mt323.dll
 0002:00000920       __imp_?setMargin@QLayout@@UAEXH@Z 10024920     qt-mt323:qt-mt323.dll
 0002:00000924       __imp_?setMargins@QScrollView@@MAEXHHHH@Z 10024924     qt-mt323:qt-mt323.dll
 0002:00000928       __imp_?setMask@QWidget@@UAEXABVQBitmap@@@Z 10024928     qt-mt323:qt-mt323.dll
 0002:0000092c       __imp_?setMask@QWidget@@UAEXABVQRegion@@@Z 1002492c     qt-mt323:qt-mt323.dll
 0002:00000930       __imp_?setMaxLength@QLineEdit@@UAEXH@Z 10024930     qt-mt323:qt-mt323.dll
 0002:00000934       __imp_?setMaximumSize@QWidget@@UAEXHH@Z 10024934     qt-mt323:qt-mt323.dll
 0002:00000938       __imp_?setMenuBar@QLayout@@UAEXPAVQMenuBar@@@Z 10024938     qt-mt323:qt-mt323.dll
 0002:0000093c       __imp_?setMenuText@QAction@@UAEXABVQString@@@Z 1002493c     qt-mt323:qt-mt323.dll
 0002:00000940       __imp_?setMicroFocusHint@QWidget@@MAEXHHHH_NPAVQFont@@@Z 10024940     qt-mt323:qt-mt323.dll
 0002:00000944       __imp_?setMidLineWidth@QFrame@@UAEXH@Z 10024944     qt-mt323:qt-mt323.dll
 0002:00000948       __imp_?setMinimumSize@QToolBar@@UAEXHH@Z 10024948     qt-mt323:qt-mt323.dll
 0002:0000094c       __imp_?setMinimumSize@QWidget@@UAEXHH@Z 1002494c     qt-mt323:qt-mt323.dll
 0002:00000950       __imp_?setMouseTracking@QWidget@@UAEX_N@Z 10024950     qt-mt323:qt-mt323.dll
 0002:00000954       __imp_?setMovie@QLabel@@UAEXABVQMovie@@@Z 10024954     qt-mt323:qt-mt323.dll
 0002:00000958       __imp_?setMovingEnabled@QDockWindow@@UAEX_N@Z 10024958     qt-mt323:qt-mt323.dll
 0002:0000095c       __imp_?setMultiLinesEnabled@QListViewItem@@UAEX_N@Z 1002495c     qt-mt323:qt-mt323.dll
 0002:00000960       __imp_?setMultiSelection@QListView@@UAEX_N@Z 10024960     qt-mt323:qt-mt323.dll
 0002:00000964       __imp_?setName@QObject@@UAEXPBD@Z 10024964     qt-mt323:qt-mt323.dll
 0002:00000968       __imp_?setNewLine@QDockWindow@@UAEX_N@Z 10024968     qt-mt323:qt-mt323.dll
 0002:0000096c       __imp_?setNum@QLabel@@UAEXH@Z 1002496c     qt-mt323:qt-mt323.dll
 0002:00000970       __imp_?setNum@QLabel@@UAEXN@Z 10024970     qt-mt323:qt-mt323.dll
 0002:00000974       __imp_?setOffset@QDockWindow@@UAEXH@Z 10024974     qt-mt323:qt-mt323.dll
 0002:00000978       __imp_?setOn@QAction@@UAEX_N@Z 10024978     qt-mt323:qt-mt323.dll
 0002:0000097c       __imp_?setOn@QPushButton@@UAEX_N@Z 1002497c     qt-mt323:qt-mt323.dll
 0002:00000980       __imp_?setOpaqueMoving@QDockWindow@@UAEX_N@Z 10024980     qt-mt323:qt-mt323.dll
 0002:00000984       __imp_?setOpen@QListView@@UAEXPAVQListViewItem@@_N@Z 10024984     qt-mt323:qt-mt323.dll
 0002:00000988       __imp_?setOpen@QListViewItem@@UAEX_N@Z 10024988     qt-mt323:qt-mt323.dll
 0002:0000098c       __imp_?setOrientation@QDockWindow@@UAEXW4Orientation@Qt@@@Z 1002498c     qt-mt323:qt-mt323.dll
 0002:00000990       __imp_?setOrientation@QToolBar@@UAEXW4Orientation@Qt@@@Z 10024990     qt-mt323:qt-mt323.dll
 0002:00000994       __imp_?setPalette@QLineEdit@@UAEXABVQPalette@@@Z 10024994     qt-mt323:qt-mt323.dll
 0002:00000998       __imp_?setPalette@QListView@@UAEXABVQPalette@@@Z 10024998     qt-mt323:qt-mt323.dll
 0002:0000099c       __imp_?setPalette@QWidget@@UAEXABVQPalette@@@Z 1002499c     qt-mt323:qt-mt323.dll
 0002:000009a0       __imp_?setPaletteBackgroundColor@QWidget@@UAEXABVQColor@@@Z 100249a0     qt-mt323:qt-mt323.dll
 0002:000009a4       __imp_?setPaletteBackgroundPixmap@QWidget@@UAEXABVQPixmap@@@Z 100249a4     qt-mt323:qt-mt323.dll
 0002:000009a8       __imp_?setPicture@QLabel@@UAEXABVQPicture@@@Z 100249a8     qt-mt323:qt-mt323.dll
 0002:000009ac       __imp_?setPixmap@QButton@@UAEXABVQPixmap@@@Z 100249ac     qt-mt323:qt-mt323.dll
 0002:000009b0       __imp_?setPixmap@QLabel@@UAEXABVQPixmap@@@Z 100249b0     qt-mt323:qt-mt323.dll
 0002:000009b4       __imp_?setPixmap@QListViewItem@@UAEXHABVQPixmap@@@Z 100249b4     qt-mt323:qt-mt323.dll
 0002:000009b8       __imp_?setProperty@QObject@@UAE_NPBDABVQVariant@@@Z 100249b8     qt-mt323:qt-mt323.dll
 0002:000009bc       __imp_?setReadOnly@QLineEdit@@UAEX_N@Z 100249bc     qt-mt323:qt-mt323.dll
 0002:000009c0       __imp_?setResizeEnabled@QDockWindow@@UAEX_N@Z 100249c0     qt-mt323:qt-mt323.dll
 0002:000009c4       __imp_?setResizeMode@QListView@@UAEXW4ResizeMode@1@@Z 100249c4     qt-mt323:qt-mt323.dll
 0002:000009c8       __imp_?setResizePolicy@QScrollView@@UAEXW4ResizePolicy@1@@Z 100249c8     qt-mt323:qt-mt323.dll
 0002:000009cc       __imp_?setResolution@QPaintDevice@@UAEXH@Z 100249cc     qt-mt323:qt-mt323.dll
 0002:000009d0       __imp_?setRootIsDecorated@QListView@@UAEX_N@Z 100249d0     qt-mt323:qt-mt323.dll
 0002:000009d4       __imp_?setSelectable@QListViewItem@@UAEX_N@Z 100249d4     qt-mt323:qt-mt323.dll
 0002:000009d8       __imp_?setSelected@QListView@@UAEXPAVQListViewItem@@_N@Z 100249d8     qt-mt323:qt-mt323.dll
 0002:000009dc       __imp_?setSelected@QListViewItem@@UAEX_N@Z 100249dc     qt-mt323:qt-mt323.dll
 0002:000009e0       __imp_?setSelection@QLineEdit@@UAEXHH@Z 100249e0     qt-mt323:qt-mt323.dll
 0002:000009e4       __imp_?setShowSortIndicator@QListView@@UAEX_N@Z 100249e4     qt-mt323:qt-mt323.dll
 0002:000009e8       __imp_?setShowToolTips@QListView@@UAEX_N@Z 100249e8     qt-mt323:qt-mt323.dll
 0002:000009ec       __imp_?setSizeIncrement@QWidget@@UAEXHH@Z 100249ec     qt-mt323:qt-mt323.dll
 0002:000009f0       __imp_?setSizePolicy@QWidget@@UAEXVQSizePolicy@@@Z 100249f0     qt-mt323:qt-mt323.dll
 0002:000009f4       __imp_?setSorting@QListView@@UAEXH_N@Z 100249f4     qt-mt323:qt-mt323.dll
 0002:000009f8       __imp_?setSpacing@QLayout@@UAEXH@Z 100249f8     qt-mt323:qt-mt323.dll
 0002:000009fc       __imp_?setState@QButton@@MAEXW4ToggleState@1@@Z 100249fc     qt-mt323:qt-mt323.dll
 0002:00000a00       __imp_?setStatusTip@QAction@@UAEXABVQString@@@Z 10024a00     qt-mt323:qt-mt323.dll
 0002:00000a04       __imp_?setStretchableWidget@QToolBar@@UAEXPAVQWidget@@@Z 10024a04     qt-mt323:qt-mt323.dll
 0002:00000a08       __imp_?setText@QAction@@UAEXABVQString@@@Z 10024a08     qt-mt323:qt-mt323.dll
 0002:00000a0c       __imp_?setText@QButton@@UAEXABVQString@@@Z 10024a0c     qt-mt323:qt-mt323.dll
 0002:00000a10       __imp_?setText@QLabel@@UAEXABVQString@@@Z 10024a10     qt-mt323:qt-mt323.dll
 0002:00000a14       __imp_?setText@QLineEdit@@UAEXABVQString@@@Z 10024a14     qt-mt323:qt-mt323.dll
 0002:00000a18       __imp_?setText@QListViewItem@@UAEXHABVQString@@@Z 10024a18     qt-mt323:qt-mt323.dll
 0002:00000a1c       __imp_?setToggleAction@QAction@@UAEX_N@Z 10024a1c     qt-mt323:qt-mt323.dll
 0002:00000a20       __imp_?setToggleType@QButton@@MAEXW4ToggleType@1@@Z 10024a20     qt-mt323:qt-mt323.dll
 0002:00000a24       __imp_?setToolTip@QAction@@UAEXABVQString@@@Z 10024a24     qt-mt323:qt-mt323.dll
 0002:00000a28       __imp_?setTreeStepSize@QListView@@UAEXH@Z 10024a28     qt-mt323:qt-mt323.dll
 0002:00000a2c       __imp_?setUpdatesEnabled@QWidget@@UAEX_N@Z 10024a2c     qt-mt323:qt-mt323.dll
 0002:00000a30       __imp_?setVBarGeometry@QScrollView@@MAEXAAVQScrollBar@@HHHH@Z 10024a30     qt-mt323:qt-mt323.dll
 0002:00000a34       __imp_?setVScrollBarMode@QScrollView@@UAEXW4ScrollBarMode@1@@Z 10024a34     qt-mt323:qt-mt323.dll
 0002:00000a38       __imp_?setValidator@QLineEdit@@UAEXPBVQValidator@@@Z 10024a38     qt-mt323:qt-mt323.dll
 0002:00000a3c       __imp_?setVerticallyStretchable@QDockWindow@@UAEX_N@Z 10024a3c     qt-mt323:qt-mt323.dll
 0002:00000a40       __imp_?setWFlags@QWidget@@MAEXI@Z 10024a40     qt-mt323:qt-mt323.dll
 0002:00000a44       __imp_?setWState@QWidget@@MAEXI@Z 10024a44     qt-mt323:qt-mt323.dll
 0002:00000a48       __imp_?setWhatsThis@QAction@@UAEXABVQString@@@Z 10024a48     qt-mt323:qt-mt323.dll
 0002:00000a4c       __imp_?setWidget@QDockWindow@@UAEXPAVQWidget@@@Z 10024a4c     qt-mt323:qt-mt323.dll
 0002:00000a50       __imp_?setup@QListViewItem@@UAEXXZ 10024a50     qt-mt323:qt-mt323.dll
 0002:00000a54       __imp_?show@QListView@@UAEXXZ 10024a54     qt-mt323:qt-mt323.dll
 0002:00000a58       __imp_?show@QPopupMenu@@UAEXXZ 10024a58     qt-mt323:qt-mt323.dll
 0002:00000a5c       __imp_?show@QToolBar@@UAEXXZ 10024a5c     qt-mt323:qt-mt323.dll
 0002:00000a60       __imp_?show@QWidget@@UAEXXZ 10024a60     qt-mt323:qt-mt323.dll
 0002:00000a64       __imp_?showEvent@QDockWindow@@MAEXPAVQShowEvent@@@Z 10024a64     qt-mt323:qt-mt323.dll
 0002:00000a68       __imp_?showEvent@QListView@@MAEXPAVQShowEvent@@@Z 10024a68     qt-mt323:qt-mt323.dll
 0002:00000a6c       __imp_?showEvent@QTabWidget@@MAEXPAVQShowEvent@@@Z 10024a6c     qt-mt323:qt-mt323.dll
 0002:00000a70       __imp_?showEvent@QWidget@@MAEXPAVQShowEvent@@@Z 10024a70     qt-mt323:qt-mt323.dll
 0002:00000a74       __imp_?showMaximized@QWidget@@UAEXXZ 10024a74     qt-mt323:qt-mt323.dll
 0002:00000a78       __imp_?showMinimized@QWidget@@UAEXXZ 10024a78     qt-mt323:qt-mt323.dll
 0002:00000a7c       __imp_?showNormal@QWidget@@UAEXXZ 10024a7c     qt-mt323:qt-mt323.dll
 0002:00000a80       __imp_?showPage@QTabWidget@@UAEXPAVQWidget@@@Z 10024a80     qt-mt323:qt-mt323.dll
 0002:00000a84       __imp_??6QTextStream@@QAEAAV0@ABVQString@@@Z 10024a84     qt-mt323:qt-mt323.dll
 0002:00000a88       __imp_?sizeHint@QHBox@@UBE?AVQSize@@XZ 10024a88     qt-mt323:qt-mt323.dll
 0002:00000a8c       __imp_?sizeHint@QLabel@@UBE?AVQSize@@XZ 10024a8c     qt-mt323:qt-mt323.dll
 0002:00000a90       __imp_?sizeHint@QLineEdit@@UBE?AVQSize@@XZ 10024a90     qt-mt323:qt-mt323.dll
 0002:00000a94       __imp_?sizeHint@QListView@@UBE?AVQSize@@XZ 10024a94     qt-mt323:qt-mt323.dll
 0002:00000a98       __imp_?sizeHint@QPopupMenu@@UBE?AVQSize@@XZ 10024a98     qt-mt323:qt-mt323.dll
 0002:00000a9c       __imp_?sizeHint@QPushButton@@UBE?AVQSize@@XZ 10024a9c     qt-mt323:qt-mt323.dll
 0002:00000aa0       __imp_?sizeHint@QSpacerItem@@UBE?AVQSize@@XZ 10024aa0     qt-mt323:qt-mt323.dll
 0002:00000aa4       __imp_?sizeHint@QTabWidget@@UBE?AVQSize@@XZ 10024aa4     qt-mt323:qt-mt323.dll
 0002:00000aa8       __imp_?sizeHint@QWidget@@UBE?AVQSize@@XZ 10024aa8     qt-mt323:qt-mt323.dll
 0002:00000aac       __imp_?sizePolicy@QWidget@@UBE?AVQSizePolicy@@XZ 10024aac     qt-mt323:qt-mt323.dll
 0002:00000ab0       __imp_?sort@QListView@@UAEXXZ 10024ab0     qt-mt323:qt-mt323.dll
 0002:00000ab4       __imp_?sort@QListViewItem@@UAEXXZ 10024ab4     qt-mt323:qt-mt323.dll
 0002:00000ab8       __imp_?sortChildItems@QListViewItem@@UAEXH_N@Z 10024ab8     qt-mt323:qt-mt323.dll
 0002:00000abc       __imp_?spacerItem@QLayoutItem@@UAEPAVQSpacerItem@@XZ 10024abc     qt-mt323:qt-mt323.dll
 0002:00000ac0       __imp_?spacerItem@QSpacerItem@@UAEPAV1@XZ 10024ac0     qt-mt323:qt-mt323.dll
 0002:00000ac4       __imp_?startDrag@QListView@@MAEXXZ 10024ac4     qt-mt323:qt-mt323.dll
 0002:00000ac8       __imp_?startRename@QListViewItem@@UAEXH@Z 10024ac8     qt-mt323:qt-mt323.dll
 0002:00000acc       __imp_?styleChange@QFrame@@MAEXAAVQStyle@@@Z 10024acc     qt-mt323:qt-mt323.dll
 0002:00000ad0       __imp_?styleChange@QListView@@MAEXAAVQStyle@@@Z 10024ad0     qt-mt323:qt-mt323.dll
 0002:00000ad4       __imp_?styleChange@QPopupMenu@@MAEXAAVQStyle@@@Z 10024ad4     qt-mt323:qt-mt323.dll
 0002:00000ad8       __imp_?styleChange@QTabWidget@@MAEXAAVQStyle@@@Z 10024ad8     qt-mt323:qt-mt323.dll
 0002:00000adc       __imp_?styleChange@QToolBar@@MAEXAAVQStyle@@@Z 10024adc     qt-mt323:qt-mt323.dll
 0002:00000ae0       __imp_?styleChange@QWidget@@MAEXAAVQStyle@@@Z 10024ae0     qt-mt323:qt-mt323.dll
 0002:00000ae4       __imp_?tabletEvent@QWidget@@MAEXPAVQTabletEvent@@@Z 10024ae4     qt-mt323:qt-mt323.dll
 0002:00000ae8       __imp_?takeItem@QListView@@UAEXPAVQListViewItem@@@Z 10024ae8     qt-mt323:qt-mt323.dll
 0002:00000aec       __imp_?takeItem@QListViewItem@@UAEXPAV1@@Z 10024aec     qt-mt323:qt-mt323.dll
 0002:00000af0       __imp_?timerEvent@QObject@@MAEXPAVQTimerEvent@@@Z 10024af0     qt-mt323:qt-mt323.dll
 0002:00000af4       __imp_?timerEvent@QPopupMenu@@MAEXPAVQTimerEvent@@@Z 10024af4     qt-mt323:qt-mt323.dll
 0002:00000af8       __imp_?undo@QLineEdit@@UAEXXZ 10024af8     qt-mt323:qt-mt323.dll
 0002:00000afc       __imp_?undock@QDockWindow@@UAEXPAVQWidget@@@Z 10024afc     qt-mt323:qt-mt323.dll
 0002:00000b00       __imp_?undock@QDockWindow@@UAEXXZ 10024b00     qt-mt323:qt-mt323.dll
 0002:00000b04       __imp_?unsetCursor@QWidget@@UAEXXZ 10024b04     qt-mt323:qt-mt323.dll
 0002:00000b08       __imp_?updateItem@QPopupMenu@@UAEXH@Z 10024b08     qt-mt323:qt-mt323.dll
 0002:00000b0c       __imp_?updateMask@QPushButton@@MAEXXZ 10024b0c     qt-mt323:qt-mt323.dll
 0002:00000b10       __imp_?updateMask@QTabWidget@@MAEXXZ 10024b10     qt-mt323:qt-mt323.dll
 0002:00000b14       __imp_?updateMask@QWidget@@MAEXXZ 10024b14     qt-mt323:qt-mt323.dll
 0002:00000b18       __imp_?viewportContextMenuEvent@QScrollView@@MAEXPAVQContextMenuEvent@@@Z 10024b18     qt-mt323:qt-mt323.dll
 0002:00000b1c       __imp_?viewportDragEnterEvent@QScrollView@@MAEXPAVQDragEnterEvent@@@Z 10024b1c     qt-mt323:qt-mt323.dll
 0002:00000b20       __imp_?viewportDragLeaveEvent@QScrollView@@MAEXPAVQDragLeaveEvent@@@Z 10024b20     qt-mt323:qt-mt323.dll
 0002:00000b24       __imp_?viewportDragMoveEvent@QScrollView@@MAEXPAVQDragMoveEvent@@@Z 10024b24     qt-mt323:qt-mt323.dll
 0002:00000b28       __imp_?viewportDropEvent@QScrollView@@MAEXPAVQDropEvent@@@Z 10024b28     qt-mt323:qt-mt323.dll
 0002:00000b2c       __imp_?viewportMouseDoubleClickEvent@QScrollView@@MAEXPAVQMouseEvent@@@Z 10024b2c     qt-mt323:qt-mt323.dll
 0002:00000b30       __imp_?viewportMouseMoveEvent@QScrollView@@MAEXPAVQMouseEvent@@@Z 10024b30     qt-mt323:qt-mt323.dll
 0002:00000b34       __imp_?viewportMousePressEvent@QScrollView@@MAEXPAVQMouseEvent@@@Z 10024b34     qt-mt323:qt-mt323.dll
 0002:00000b38       __imp_?viewportMouseReleaseEvent@QScrollView@@MAEXPAVQMouseEvent@@@Z 10024b38     qt-mt323:qt-mt323.dll
 0002:00000b3c       __imp_?viewportPaintEvent@QScrollView@@MAEXPAVQPaintEvent@@@Z 10024b3c     qt-mt323:qt-mt323.dll
 0002:00000b40       __imp_?viewportResizeEvent@QListView@@MAEXPAVQResizeEvent@@@Z 10024b40     qt-mt323:qt-mt323.dll
 0002:00000b44       __imp_?viewportWheelEvent@QScrollView@@MAEXPAVQWheelEvent@@@Z 10024b44     qt-mt323:qt-mt323.dll
 0002:00000b48       __imp_?wheelEvent@QScrollView@@MAEXPAVQWheelEvent@@@Z 10024b48     qt-mt323:qt-mt323.dll
 0002:00000b4c       __imp_?wheelEvent@QWidget@@MAEXPAVQWheelEvent@@@Z 10024b4c     qt-mt323:qt-mt323.dll
 0002:00000b50       __imp_?widget@QLayoutItem@@UAEPAVQWidget@@XZ 10024b50     qt-mt323:qt-mt323.dll
 0002:00000b54       __imp_?width@QListViewItem@@UBEHABVQFontMetrics@@PBVQListView@@H@Z 10024b54     qt-mt323:qt-mt323.dll
 0002:00000b58       __imp_?winEvent@QWidget@@MAE_NPAUtagMSG@@@Z 10024b58     qt-mt323:qt-mt323.dll
 0002:00000b5c       __imp_?windowActivationChange@QLineEdit@@MAEX_N@Z 10024b5c     qt-mt323:qt-mt323.dll
 0002:00000b60       __imp_?windowActivationChange@QListView@@MAEX_N@Z 10024b60     qt-mt323:qt-mt323.dll
 0002:00000b64       __imp_?windowActivationChange@QWidget@@MAEX_N@Z 10024b64     qt-mt323:qt-mt323.dll
 0002:00000b68       __imp_?write@QGList@@MBEAAVQDataStream@@AAV2@PAX@Z 10024b68     qt-mt323:qt-mt323.dll
 0002:00000b6c       __imp_?null@QString@@2V1@A 10024b6c     qt-mt323:qt-mt323.dll
 0002:00000b70       __imp_??_7?$QPtrList@VQDockWindow@@@@6B@ 10024b70     qt-mt323:qt-mt323.dll
 0002:00000b74       __imp_?section@QString@@QBE?AV1@PBDHHH@Z 10024b74     qt-mt323:qt-mt323.dll
 0002:00000b78       __imp_??0?$QMap@VQString@@H@@QAE@XZ 10024b78     qt-mt323:qt-mt323.dll
 0002:00000b7c       __imp_??1?$QMap@VQString@@H@@QAE@XZ 10024b7c     qt-mt323:qt-mt323.dll
 0002:00000b80       __imp_?begin@?$QMap@VQString@@H@@QAE?AV?$QMapIterator@VQString@@H@@XZ 10024b80     qt-mt323:qt-mt323.dll
 0002:00000b84       __imp_?end@?$QMap@VQString@@H@@QAE?AV?$QMapIterator@VQString@@H@@XZ 10024b84     qt-mt323:qt-mt323.dll
 0002:00000b88       __imp_??A?$QMap@VQString@@H@@QAEAAHABVQString@@@Z 10024b88     qt-mt323:qt-mt323.dll
 0002:00000b8c       __imp_?clear@?$QMap@VQString@@H@@QAEXXZ 10024b8c     qt-mt323:qt-mt323.dll
 0002:00000b90       __imp_?find@?$QMap@VQString@@H@@QAE?AV?$QMapIterator@VQString@@H@@ABVQString@@@Z 10024b90     qt-mt323:qt-mt323.dll
 0002:00000b94       __imp_?accept@QDialog@@MAEXXZ 10024b94     qt-mt323:qt-mt323.dll
 0002:00000b98       __imp_?warning@QMessageBox@@SAHPAVQWidget@@ABVQString@@1HHH@Z 10024b98     qt-mt323:qt-mt323.dll
 0002:00000b9c       __imp_?closeEvent@QDialog@@MAEXPAVQCloseEvent@@@Z 10024b9c     qt-mt323:qt-mt323.dll
 0002:00000ba0       __imp_?contextMenuEvent@QDialog@@MAEXPAVQContextMenuEvent@@@Z 10024ba0     qt-mt323:qt-mt323.dll
 0002:00000ba4       __imp_?truncate@QString@@QAEXI@Z 10024ba4     qt-mt323:qt-mt323.dll
 0002:00000ba8       __imp_?eventFilter@QDialog@@MAE_NPAVQObject@@PAVQEvent@@@Z 10024ba8     qt-mt323:qt-mt323.dll
 0002:00000bac       __imp_?hide@QDialog@@UAEXXZ 10024bac     qt-mt323:qt-mt323.dll
 0002:00000bb0       __imp_?keyPressEvent@QDialog@@MAEXPAVQKeyEvent@@@Z 10024bb0     qt-mt323:qt-mt323.dll
 0002:00000bb4       __imp_?minimumSizeHint@QDialog@@UBE?AVQSize@@XZ 10024bb4     qt-mt323:qt-mt323.dll
 0002:00000bb8       __imp_?move@QDialog@@UAEXHH@Z 10024bb8     qt-mt323:qt-mt323.dll
 0002:00000bbc       __imp_?reject@QDialog@@MAEXXZ 10024bbc     qt-mt323:qt-mt323.dll
 0002:00000bc0       __imp_?resize@QDialog@@UAEXHH@Z 10024bc0     qt-mt323:qt-mt323.dll
 0002:00000bc4       __imp_?resizeEvent@QDialog@@MAEXPAVQResizeEvent@@@Z 10024bc4     qt-mt323:qt-mt323.dll
 0002:00000bc8       __imp_?setGeometry@QDialog@@UAEXABVQRect@@@Z 10024bc8     qt-mt323:qt-mt323.dll
 0002:00000bcc       __imp_?setGeometry@QDialog@@UAEXHHHH@Z 10024bcc     qt-mt323:qt-mt323.dll
 0002:00000bd0       __imp_?show@QDialog@@UAEXXZ 10024bd0     qt-mt323:qt-mt323.dll
 0002:00000bd4       __imp_?sizeHint@QDialog@@UBE?AVQSize@@XZ 10024bd4     qt-mt323:qt-mt323.dll
 0002:00000bd8       __imp_??0QString@@QAE@VQChar@@@Z 10024bd8     qt-mt323:qt-mt323.dll
 0002:00000bdc       __imp_?section@QString@@QBE?AV1@DHHH@Z 10024bdc     qt-mt323:qt-mt323.dll
 0002:00000be0       __imp_?replace@QString@@QAEAAV1@DABV1@@Z 10024be0     qt-mt323:qt-mt323.dll
 0002:00000be4       __imp_?setNum@QString@@QAEAAV1@_JH@Z 10024be4     qt-mt323:qt-mt323.dll
 0002:00000be8       __imp_?first@?$QValueList@VQString@@@@QAEAAVQString@@XZ 10024be8     qt-mt323:qt-mt323.dll
 0002:00000bec       __imp_?rebalance@QMapPrivateBase@@QAEXPAUQMapNodeBase@@AAPAU2@@Z 10024bec     qt-mt323:qt-mt323.dll
 0002:00000bf0       __imp_?removeAndRebalance@QMapPrivateBase@@QAEPAUQMapNodeBase@@PAU2@AAPAU2@11@Z 10024bf0     qt-mt323:qt-mt323.dll
 0002:00000bf4       __imp_?child@QObject@@QAEPAV1@PBD0_N@Z 10024bf4     qt-mt323:qt-mt323.dll
 0002:00000bf8       __imp_??0QStringList@@QAE@ABV0@@Z 10024bf8     qt-mt323:qt-mt323.dll
 0002:00000bfc       __imp_??0QBrush@@QAE@ABVQColor@@W4BrushStyle@Qt@@@Z 10024bfc     qt-mt323:qt-mt323.dll
 0002:00000c00       __imp_??1QBrush@@QAE@XZ    10024c00     qt-mt323:qt-mt323.dll
 0002:00000c04       __imp_?setColor@QBrush@@QAEXABVQColor@@@Z 10024c04     qt-mt323:qt-mt323.dll
 0002:00000c08       __imp_?unsetPalette@QWidget@@QAEXXZ 10024c08     qt-mt323:qt-mt323.dll
 0002:00000c0c       __imp_?setPaletteForegroundColor@QWidget@@QAEXABVQColor@@@Z 10024c0c     qt-mt323:qt-mt323.dll
 0002:00000c10       __imp_?count@QComboBox@@QBEHXZ 10024c10     qt-mt323:qt-mt323.dll
 0002:00000c14       __imp_?insertItem@QComboBox@@QAEXABVQString@@H@Z 10024c14     qt-mt323:qt-mt323.dll
 0002:00000c18       __imp_?currentItem@QComboBox@@QBEHXZ 10024c18     qt-mt323:qt-mt323.dll
 0002:00000c1c       __imp_?currentText@QComboBox@@QBE?AVQString@@XZ 10024c1c     qt-mt323:qt-mt323.dll
 0002:00000c20       __imp_?listBox@QComboBox@@QBEPAVQListBox@@XZ 10024c20     qt-mt323:qt-mt323.dll
 0002:00000c24       __imp_?clearEdit@QComboBox@@QAEXXZ 10024c24     qt-mt323:qt-mt323.dll
 0002:00000c28       __imp_?count@QListBox@@QBEIXZ 10024c28     qt-mt323:qt-mt323.dll
 0002:00000c2c       __imp_?item@QListBox@@QBEPAVQListBoxItem@@H@Z 10024c2c     qt-mt323:qt-mt323.dll
 0002:00000c30       __imp_?findItem@QListBox@@QBEPAVQListBoxItem@@ABVQString@@I@Z 10024c30     qt-mt323:qt-mt323.dll
 0002:00000c34       __imp_?clear@QListBox@@QAEXXZ 10024c34     qt-mt323:qt-mt323.dll
 0002:00000c38       __imp_?listBox@QListBoxItem@@QBEPAVQListBox@@XZ 10024c38     qt-mt323:qt-mt323.dll
 0002:00000c3c       __imp_??0QListBoxText@@QAE@PAVQListBox@@ABVQString@@@Z 10024c3c     qt-mt323:qt-mt323.dll
 0002:00000c40       __imp_??1QListBoxText@@UAE@XZ 10024c40     qt-mt323:qt-mt323.dll
 0002:00000c44       __imp_?paint@QListBoxText@@MAEXPAVQPainter@@@Z 10024c44     qt-mt323:qt-mt323.dll
 0002:00000c48       __imp_?toString@QTime@@QBE?AVQString@@ABV2@@Z 10024c48     qt-mt323:qt-mt323.dll
 0002:00000c4c       __imp_?fromString@QTime@@SA?AV1@ABVQString@@W4DateFormat@Qt@@@Z 10024c4c     qt-mt323:qt-mt323.dll
 0002:00000c50       __imp_??9QDateTime@@QBE_NABV0@@Z 10024c50     qt-mt323:qt-mt323.dll
 0002:00000c54       __imp_?time@QTimeEdit@@QBE?AVQTime@@XZ 10024c54     qt-mt323:qt-mt323.dll
 0002:00000c58       __imp_?raiseWidget@QWidgetStack@@QAEXH@Z 10024c58     qt-mt323:qt-mt323.dll
 0002:00000c5c       __imp_?label@QHeader@@QBE?AVQString@@H@Z 10024c5c     qt-mt323:qt-mt323.dll
 0002:00000c60       __imp_?count@QHeader@@QBEHXZ 10024c60     qt-mt323:qt-mt323.dll
 0002:00000c64       __imp_?verticalHeader@QTable@@QBEPAVQHeader@@XZ 10024c64     qt-mt323:qt-mt323.dll
 0002:00000c68       __imp_?setRowLabels@QTable@@QAEXABVQStringList@@@Z 10024c68     qt-mt323:qt-mt323.dll
 0002:00000c6c       __imp_?text@QLabel@@QBE?AVQString@@XZ 10024c6c     qt-mt323:qt-mt323.dll
 0002:00000c70       __imp_??0QDir@@QAE@ABVQString@@0HH@Z 10024c70     qt-mt323:qt-mt323.dll
 0002:00000c74       __imp_?setNameFilter@QDir@@UAEXABVQString@@@Z 10024c74     qt-mt323:qt-mt323.dll
 0002:00000c78       __imp_?entryList@QDir@@UBE?AVQStringList@@HH@Z 10024c78     qt-mt323:qt-mt323.dll
 0002:00000c7c       __imp_??0QDoubleValidator@@QAE@NNHPAVQObject@@PBD@Z 10024c7c     qt-mt323:qt-mt323.dll
 0002:00000c80       __imp_??1QDoubleValidator@@UAE@XZ 10024c80     qt-mt323:qt-mt323.dll
 0002:00000c84       __imp_?text@QTextEdit@@QBE?AVQString@@XZ 10024c84     qt-mt323:qt-mt323.dll
 0002:00000c88       __imp_?setText@QTextEdit@@QAEXABVQString@@@Z 10024c88     qt-mt323:qt-mt323.dll
 0002:00000c8c       __imp_??0QPen@@QAE@ABVQColor@@IW4PenStyle@Qt@@@Z 10024c8c     qt-mt323:qt-mt323.dll
 0002:00000c90       __imp_??1QPen@@QAE@XZ      10024c90     qt-mt323:qt-mt323.dll
 0002:00000c94       __imp_?setColor@QPen@@QAEXABVQColor@@@Z 10024c94     qt-mt323:qt-mt323.dll
 0002:00000c98       __imp_?setPen@QPainter@@QAEXABVQPen@@@Z 10024c98     qt-mt323:qt-mt323.dll
 0002:00000c9c       __imp_?fillRect@QPainter@@QAEXHHHHABVQBrush@@@Z 10024c9c     qt-mt323:qt-mt323.dll
 0002:00000ca0       __imp_?className@QDoubleValidator@@UBEPBDXZ 10024ca0     qt-mt323:qt-mt323.dll
 0002:00000ca4       __imp_?fixup@QValidator@@UBEXAAVQString@@@Z 10024ca4     qt-mt323:qt-mt323.dll
 0002:00000ca8       __imp_?height@QListBoxText@@UBEHPBVQListBox@@@Z 10024ca8     qt-mt323:qt-mt323.dll
 0002:00000cac       __imp_?metaObject@QDoubleValidator@@UBEPAVQMetaObject@@XZ 10024cac     qt-mt323:qt-mt323.dll
 0002:00000cb0       __imp_?pixmap@QListBoxItem@@UBEPBVQPixmap@@XZ 10024cb0     qt-mt323:qt-mt323.dll
 0002:00000cb4       __imp_?qt_cast@QDoubleValidator@@UAEPAXPBD@Z 10024cb4     qt-mt323:qt-mt323.dll
 0002:00000cb8       __imp_?qt_emit@QDoubleValidator@@UAE_NHPAUQUObject@@@Z 10024cb8     qt-mt323:qt-mt323.dll
 0002:00000cbc       __imp_?qt_invoke@QDoubleValidator@@UAE_NHPAUQUObject@@@Z 10024cbc     qt-mt323:qt-mt323.dll
 0002:00000cc0       __imp_?qt_property@QDoubleValidator@@UAE_NHHPAVQVariant@@@Z 10024cc0     qt-mt323:qt-mt323.dll
 0002:00000cc4       __imp_?rtti@QListBoxText@@UBEHXZ 10024cc4     qt-mt323:qt-mt323.dll
 0002:00000cc8       __imp_?setRange@QDoubleValidator@@UAEXNNH@Z 10024cc8     qt-mt323:qt-mt323.dll
 0002:00000ccc       __imp_?setText@QListBoxItem@@MAEXABVQString@@@Z 10024ccc     qt-mt323:qt-mt323.dll
 0002:00000cd0       __imp_?text@QListBoxItem@@UBE?AVQString@@XZ 10024cd0     qt-mt323:qt-mt323.dll
 0002:00000cd4       __imp_?validate@QDoubleValidator@@UBE?AW4State@QValidator@@AAVQString@@AAH@Z 10024cd4     qt-mt323:qt-mt323.dll
 0002:00000cd8       __imp_?width@QListBoxText@@UBEHPBVQListBox@@@Z 10024cd8     qt-mt323:qt-mt323.dll
 0002:00000cdc       __imp_?null@QChar@@2V1@A   10024cdc     qt-mt323:qt-mt323.dll
 0002:00000ce0       __imp_?yellow@Qt@@2AAVQColor@@A 10024ce0     qt-mt323:qt-mt323.dll
 0002:00000ce4       __imp_?upper@QString@@QBE?AV1@XZ 10024ce4     qt-mt323:qt-mt323.dll
 0002:00000ce8       __imp_?setNum@QString@@QAEAAV1@_KH@Z 10024ce8     qt-mt323:qt-mt323.dll
 0002:00000cec       __imp_?begin@?$QValueList@VQString@@@@QBE?AV?$QValueListConstIterator@VQString@@@@XZ 10024cec     qt-mt323:qt-mt323.dll
 0002:00000cf0       __imp_?end@?$QValueList@VQString@@@@QBE?AV?$QValueListConstIterator@VQString@@@@XZ 10024cf0     qt-mt323:qt-mt323.dll
 0002:00000cf4       __imp_??4QStringList@@QAEAAV0@ABV0@@Z 10024cf4     qt-mt323:qt-mt323.dll
 0002:00000cf8       __imp_?look_string@QGDict@@QAEPAXABVQString@@PAXH@Z 10024cf8     qt-mt323:qt-mt323.dll
 0002:00000cfc       __imp_??0QGDict@@IAE@IW4KeyType@0@_N1@Z 10024cfc     qt-mt323:qt-mt323.dll
 0002:00000d00       __imp_??1QGDict@@MAE@XZ    10024d00     qt-mt323:qt-mt323.dll
 0002:00000d04       __imp_?clear@QGDict@@MAEXXZ 10024d04     qt-mt323:qt-mt323.dll
 0002:00000d08       __imp_?read@QGDict@@MAEAAVQDataStream@@AAV2@AAPAX@Z 10024d08     qt-mt323:qt-mt323.dll
 0002:00000d0c       __imp_?write@QGDict@@MBEAAVQDataStream@@AAV2@PAX@Z 10024d0c     qt-mt323:qt-mt323.dll
 0002:00000d10       __imp_??0QPixmap@@QAE@XZ   10024d10     qt-mt323:qt-mt323.dll
 0002:00000d14       __imp_??0QDialog@@QAE@PAVQWidget@@PBD_NI@Z 10024d14     qt-mt323:qt-mt323.dll
 0002:00000d18       __imp_??1QDialog@@UAE@XZ   10024d18     qt-mt323:qt-mt323.dll
 0002:00000d1c       __imp_?resize@QDialog@@QAEXABVQSize@@@Z 10024d1c     qt-mt323:qt-mt323.dll
 0002:00000d20       __imp_?setSizeGripEnabled@QDialog@@QAEX_N@Z 10024d20     qt-mt323:qt-mt323.dll
 0002:00000d24       __imp_?setFrameShape@QFrame@@QAEXW4Shape@1@@Z 10024d24     qt-mt323:qt-mt323.dll
 0002:00000d28       __imp_?setFrameShadow@QFrame@@QAEXW4Shadow@1@@Z 10024d28     qt-mt323:qt-mt323.dll
 0002:00000d2c       __imp_?addWidget@QBoxLayout@@QAEXPAVQWidget@@HH@Z 10024d2c     qt-mt323:qt-mt323.dll
 0002:00000d30       __imp_?addLayout@QBoxLayout@@QAEXPAVQLayout@@H@Z 10024d30     qt-mt323:qt-mt323.dll
 0002:00000d34       __imp_??0QHBoxLayout@@QAE@PAVQWidget@@HHPBD@Z 10024d34     qt-mt323:qt-mt323.dll
 0002:00000d38       __imp_?add@QToolTip@@SAXPAVQWidget@@ABVQString@@@Z 10024d38     qt-mt323:qt-mt323.dll
 0002:00000d3c       __imp_?add@QWhatsThis@@SAXPAVQWidget@@ABVQString@@@Z 10024d3c     qt-mt323:qt-mt323.dll
 0002:00000d40       __imp_?pos@QWidget@@QBE?AVQPoint@@XZ 10024d40     qt-mt323:qt-mt323.dll
 0002:00000d44       __imp_?isMaximized@QWidget@@QBE_NXZ 10024d44     qt-mt323:qt-mt323.dll
 0002:00000d48       __imp_?move@QDialog@@QAEXABVQPoint@@@Z 10024d48     qt-mt323:qt-mt323.dll
 0002:00000d4c       __imp_??6?$QValueList@VQString@@@@QAEAAV0@ABVQString@@@Z 10024d4c     qt-mt323:qt-mt323.dll
 0002:00000d50       __imp_?setTabOrder@QWidget@@SAXPAV1@0@Z 10024d50     qt-mt323:qt-mt323.dll
 0002:00000d54       __imp_??0QKeySequence@@QAE@ABVQString@@@Z 10024d54     qt-mt323:qt-mt323.dll
 0002:00000d58       __imp_??1QKeySequence@@QAE@XZ 10024d58     qt-mt323:qt-mt323.dll
 0002:00000d5c       __imp_??1QButton@@UAE@XZ   10024d5c     qt-mt323:qt-mt323.dll
 0002:00000d60       __imp_??0QCheckBox@@QAE@PAVQWidget@@PBD@Z 10024d60     qt-mt323:qt-mt323.dll
 0002:00000d64       __imp_??0QSpinBox@@QAE@PAVQWidget@@PBD@Z 10024d64     qt-mt323:qt-mt323.dll
 0002:00000d68       __imp_??1QSpinBox@@UAE@XZ  10024d68     qt-mt323:qt-mt323.dll
 0002:00000d6c       __imp_?setMaxValue@QSpinBox@@QAEXH@Z 10024d6c     qt-mt323:qt-mt323.dll
 0002:00000d70       __imp_??0QButtonGroup@@QAE@PAVQWidget@@PBD@Z 10024d70     qt-mt323:qt-mt323.dll
 0002:00000d74       __imp_??1QButtonGroup@@UAE@XZ 10024d74     qt-mt323:qt-mt323.dll
 0002:00000d78       __imp_??0QRadioButton@@QAE@PAVQWidget@@PBD@Z 10024d78     qt-mt323:qt-mt323.dll
 0002:00000d7c       __imp_??0QGridLayout@@QAE@PAVQWidget@@HHHHPBD@Z 10024d7c     qt-mt323:qt-mt323.dll
 0002:00000d80       __imp_??0QGridLayout@@QAE@PAVQLayout@@HHHPBD@Z 10024d80     qt-mt323:qt-mt323.dll
 0002:00000d84       __imp_??1QGridLayout@@UAE@XZ 10024d84     qt-mt323:qt-mt323.dll
 0002:00000d88       __imp_?addItem@QGridLayout@@QAEXPAVQLayoutItem@@HH@Z 10024d88     qt-mt323:qt-mt323.dll
 0002:00000d8c       __imp_?addWidget@QGridLayout@@QAEXPAVQWidget@@HHH@Z 10024d8c     qt-mt323:qt-mt323.dll
 0002:00000d90       __imp_?addMultiCellWidget@QGridLayout@@QAEXPAVQWidget@@HHHHH@Z 10024d90     qt-mt323:qt-mt323.dll
 0002:00000d94       __imp_?addMultiCellLayout@QGridLayout@@QAEXPAVQLayout@@HHHHH@Z 10024d94     qt-mt323:qt-mt323.dll
 0002:00000d98       __imp_?addItem@QGridLayout@@UAEXPAVQLayoutItem@@@Z 10024d98     qt-mt323:qt-mt323.dll
 0002:00000d9c       __imp_?childEvent@QGroupBox@@MAEXPAVQChildEvent@@@Z 10024d9c     qt-mt323:qt-mt323.dll
 0002:00000da0       __imp_?className@QButtonGroup@@UBEPBDXZ 10024da0     qt-mt323:qt-mt323.dll
 0002:00000da4       __imp_?className@QCheckBox@@UBEPBDXZ 10024da4     qt-mt323:qt-mt323.dll
 0002:00000da8       __imp_?className@QGridLayout@@UBEPBDXZ 10024da8     qt-mt323:qt-mt323.dll
 0002:00000dac       __imp_?className@QRadioButton@@UBEPBDXZ 10024dac     qt-mt323:qt-mt323.dll
 0002:00000db0       __imp_?className@QSpinBox@@UBEPBDXZ 10024db0     qt-mt323:qt-mt323.dll
 0002:00000db4       __imp_?cleanText@QSpinBox@@UBE?AVQString@@XZ 10024db4     qt-mt323:qt-mt323.dll
 0002:00000db8       __imp_?drawButton@QCheckBox@@MAEXPAVQPainter@@@Z 10024db8     qt-mt323:qt-mt323.dll
 0002:00000dbc       __imp_?drawButton@QRadioButton@@MAEXPAVQPainter@@@Z 10024dbc     qt-mt323:qt-mt323.dll
 0002:00000dc0       __imp_?drawButtonLabel@QCheckBox@@MAEXPAVQPainter@@@Z 10024dc0     qt-mt323:qt-mt323.dll
 0002:00000dc4       __imp_?drawButtonLabel@QRadioButton@@MAEXPAVQPainter@@@Z 10024dc4     qt-mt323:qt-mt323.dll
 0002:00000dc8       __imp_?event@QButtonGroup@@MAE_NPAVQEvent@@@Z 10024dc8     qt-mt323:qt-mt323.dll
 0002:00000dcc       __imp_?eventFilter@QSpinBox@@MAE_NPAVQObject@@PAVQEvent@@@Z 10024dcc     qt-mt323:qt-mt323.dll
 0002:00000dd0       __imp_?expanding@QGridLayout@@UBE?AW4ExpandData@QSizePolicy@@XZ 10024dd0     qt-mt323:qt-mt323.dll
 0002:00000dd4       __imp_?focusInEvent@QButton@@MAEXPAVQFocusEvent@@@Z 10024dd4     qt-mt323:qt-mt323.dll
 0002:00000dd8       __imp_?focusInEvent@QGroupBox@@MAEXPAVQFocusEvent@@@Z 10024dd8     qt-mt323:qt-mt323.dll
 0002:00000ddc       __imp_?focusOutEvent@QButton@@MAEXPAVQFocusEvent@@@Z 10024ddc     qt-mt323:qt-mt323.dll
 0002:00000de0       __imp_?fontChange@QGroupBox@@MAEXABVQFont@@@Z 10024de0     qt-mt323:qt-mt323.dll
 0002:00000de4       __imp_?hasHeightForWidth@QGridLayout@@UBE_NXZ 10024de4     qt-mt323:qt-mt323.dll
 0002:00000de8       __imp_?heightForWidth@QGridLayout@@UBEHH@Z 10024de8     qt-mt323:qt-mt323.dll
 0002:00000dec       __imp_?hitButton@QCheckBox@@MBE_NABVQPoint@@@Z 10024dec     qt-mt323:qt-mt323.dll
 0002:00000df0       __imp_?hitButton@QRadioButton@@MBE_NABVQPoint@@@Z 10024df0     qt-mt323:qt-mt323.dll
 0002:00000df4       __imp_?interpretText@QSpinBox@@MAEXXZ 10024df4     qt-mt323:qt-mt323.dll
 0002:00000df8       __imp_?invalidate@QGridLayout@@UAEXXZ 10024df8     qt-mt323:qt-mt323.dll
 0002:00000dfc       __imp_?iterator@QGridLayout@@UAE?AVQLayoutIterator@@XZ 10024dfc     qt-mt323:qt-mt323.dll
 0002:00000e00       __imp_?leaveEvent@QSpinBox@@MAEXPAVQEvent@@@Z 10024e00     qt-mt323:qt-mt323.dll
 0002:00000e04       __imp_?mapTextToValue@QSpinBox@@MAEHPA_N@Z 10024e04     qt-mt323:qt-mt323.dll
 0002:00000e08       __imp_?mapValueToText@QSpinBox@@MAE?AVQString@@H@Z 10024e08     qt-mt323:qt-mt323.dll
 0002:00000e0c       __imp_?maximumSize@QGridLayout@@UBE?AVQSize@@XZ 10024e0c     qt-mt323:qt-mt323.dll
 0002:00000e10       __imp_?metaObject@QButtonGroup@@UBEPAVQMetaObject@@XZ 10024e10     qt-mt323:qt-mt323.dll
 0002:00000e14       __imp_?metaObject@QCheckBox@@UBEPAVQMetaObject@@XZ 10024e14     qt-mt323:qt-mt323.dll
 0002:00000e18       __imp_?metaObject@QGridLayout@@UBEPAVQMetaObject@@XZ 10024e18     qt-mt323:qt-mt323.dll
 0002:00000e1c       __imp_?metaObject@QRadioButton@@UBEPAVQMetaObject@@XZ 10024e1c     qt-mt323:qt-mt323.dll
 0002:00000e20       __imp_?metaObject@QSpinBox@@UBEPAVQMetaObject@@XZ 10024e20     qt-mt323:qt-mt323.dll
 0002:00000e24       __imp_?minimumSize@QGridLayout@@UBE?AVQSize@@XZ 10024e24     qt-mt323:qt-mt323.dll
 0002:00000e28       __imp_?minimumSizeHint@QSpinBox@@UBE?AVQSize@@XZ 10024e28     qt-mt323:qt-mt323.dll
 0002:00000e2c       __imp_?moveFocus@QButtonGroup@@UAEXH@Z 10024e2c     qt-mt323:qt-mt323.dll
 0002:00000e30       __imp_?paintEvent@QGroupBox@@MAEXPAVQPaintEvent@@@Z 10024e30     qt-mt323:qt-mt323.dll
 0002:00000e34       __imp_?prefix@QSpinBox@@UBE?AVQString@@XZ 10024e34     qt-mt323:qt-mt323.dll
 0002:00000e38       __imp_?qt_cast@QButtonGroup@@UAEPAXPBD@Z 10024e38     qt-mt323:qt-mt323.dll
 0002:00000e3c       __imp_?qt_cast@QCheckBox@@UAEPAXPBD@Z 10024e3c     qt-mt323:qt-mt323.dll
 0002:00000e40       __imp_?qt_cast@QGridLayout@@UAEPAXPBD@Z 10024e40     qt-mt323:qt-mt323.dll
 0002:00000e44       __imp_?qt_cast@QRadioButton@@UAEPAXPBD@Z 10024e44     qt-mt323:qt-mt323.dll
 0002:00000e48       __imp_?qt_cast@QSpinBox@@UAEPAXPBD@Z 10024e48     qt-mt323:qt-mt323.dll
 0002:00000e4c       __imp_?qt_emit@QButtonGroup@@UAE_NHPAUQUObject@@@Z 10024e4c     qt-mt323:qt-mt323.dll
 0002:00000e50       __imp_?qt_emit@QCheckBox@@UAE_NHPAUQUObject@@@Z 10024e50     qt-mt323:qt-mt323.dll
 0002:00000e54       __imp_?qt_emit@QGridLayout@@UAE_NHPAUQUObject@@@Z 10024e54     qt-mt323:qt-mt323.dll
 0002:00000e58       __imp_?qt_emit@QRadioButton@@UAE_NHPAUQUObject@@@Z 10024e58     qt-mt323:qt-mt323.dll
 0002:00000e5c       __imp_?qt_emit@QSpinBox@@UAE_NHPAUQUObject@@@Z 10024e5c     qt-mt323:qt-mt323.dll
 0002:00000e60       __imp_?qt_invoke@QButtonGroup@@UAE_NHPAUQUObject@@@Z 10024e60     qt-mt323:qt-mt323.dll
 0002:00000e64       __imp_?qt_invoke@QCheckBox@@UAE_NHPAUQUObject@@@Z 10024e64     qt-mt323:qt-mt323.dll
 0002:00000e68       __imp_?qt_invoke@QGridLayout@@UAE_NHPAUQUObject@@@Z 10024e68     qt-mt323:qt-mt323.dll
 0002:00000e6c       __imp_?qt_invoke@QRadioButton@@UAE_NHPAUQUObject@@@Z 10024e6c     qt-mt323:qt-mt323.dll
 0002:00000e70       __imp_?qt_invoke@QSpinBox@@UAE_NHPAUQUObject@@@Z 10024e70     qt-mt323:qt-mt323.dll
 0002:00000e74       __imp_?qt_property@QButtonGroup@@UAE_NHHPAVQVariant@@@Z 10024e74     qt-mt323:qt-mt323.dll
 0002:00000e78       __imp_?qt_property@QCheckBox@@UAE_NHHPAVQVariant@@@Z 10024e78     qt-mt323:qt-mt323.dll
 0002:00000e7c       __imp_?qt_property@QGridLayout@@UAE_NHHPAVQVariant@@@Z 10024e7c     qt-mt323:qt-mt323.dll
 0002:00000e80       __imp_?qt_property@QRadioButton@@UAE_NHHPAVQVariant@@@Z 10024e80     qt-mt323:qt-mt323.dll
 0002:00000e84       __imp_?qt_property@QSpinBox@@UAE_NHHPAVQVariant@@@Z 10024e84     qt-mt323:qt-mt323.dll
 0002:00000e88       __imp_?rangeChange@QSpinBox@@MAEXXZ 10024e88     qt-mt323:qt-mt323.dll
 0002:00000e8c       __imp_?resizeEvent@QCheckBox@@MAEXPAVQResizeEvent@@@Z 10024e8c     qt-mt323:qt-mt323.dll
 0002:00000e90       __imp_?resizeEvent@QGroupBox@@MAEXPAVQResizeEvent@@@Z 10024e90     qt-mt323:qt-mt323.dll
 0002:00000e94       __imp_?resizeEvent@QRadioButton@@MAEXPAVQResizeEvent@@@Z 10024e94     qt-mt323:qt-mt323.dll
 0002:00000e98       __imp_?resizeEvent@QSpinBox@@MAEXPAVQResizeEvent@@@Z 10024e98     qt-mt323:qt-mt323.dll
 0002:00000e9c       __imp_?selectAll@QSpinBox@@UAEXXZ 10024e9c     qt-mt323:qt-mt323.dll
 0002:00000ea0       __imp_?setAlignment@QGroupBox@@UAEXH@Z 10024ea0     qt-mt323:qt-mt323.dll
 0002:00000ea4       __imp_?setButton@QButtonGroup@@UAEXH@Z 10024ea4     qt-mt323:qt-mt323.dll
 0002:00000ea8       __imp_?setButtonSymbols@QSpinBox@@UAEXW4ButtonSymbols@1@@Z 10024ea8     qt-mt323:qt-mt323.dll
 0002:00000eac       __imp_?setChecked@QRadioButton@@UAEX_N@Z 10024eac     qt-mt323:qt-mt323.dll
 0002:00000eb0       __imp_?setColStretch@QGridLayout@@UAEXHH@Z 10024eb0     qt-mt323:qt-mt323.dll
 0002:00000eb4       __imp_?setColumnLayout@QGroupBox@@UAEXHW4Orientation@Qt@@@Z 10024eb4     qt-mt323:qt-mt323.dll
 0002:00000eb8       __imp_?setEnabled@QGroupBox@@UAEX_N@Z 10024eb8     qt-mt323:qt-mt323.dll
 0002:00000ebc       __imp_?setEnabled@QSpinBox@@UAEX_N@Z 10024ebc     qt-mt323:qt-mt323.dll
 0002:00000ec0       __imp_?setExclusive@QButtonGroup@@UAEX_N@Z 10024ec0     qt-mt323:qt-mt323.dll
 0002:00000ec4       __imp_?setGeometry@QGridLayout@@UAEXABVQRect@@@Z 10024ec4     qt-mt323:qt-mt323.dll
 0002:00000ec8       __imp_?setPrefix@QSpinBox@@UAEXABVQString@@@Z 10024ec8     qt-mt323:qt-mt323.dll
 0002:00000ecc       __imp_?setRadioButtonExclusive@QButtonGroup@@UAEX_N@Z 10024ecc     qt-mt323:qt-mt323.dll
 0002:00000ed0       __imp_?setRowStretch@QGridLayout@@UAEXHH@Z 10024ed0     qt-mt323:qt-mt323.dll
 0002:00000ed4       __imp_?setSpecialValueText@QSpinBox@@UAEXABVQString@@@Z 10024ed4     qt-mt323:qt-mt323.dll
 0002:00000ed8       __imp_?setSuffix@QSpinBox@@UAEXABVQString@@@Z 10024ed8     qt-mt323:qt-mt323.dll
 0002:00000edc       __imp_?setTitle@QGroupBox@@UAEXABVQString@@@Z 10024edc     qt-mt323:qt-mt323.dll
 0002:00000ee0       __imp_?setValidator@QSpinBox@@UAEXPBVQValidator@@@Z 10024ee0     qt-mt323:qt-mt323.dll
 0002:00000ee4       __imp_?setValue@QSpinBox@@UAEXH@Z 10024ee4     qt-mt323:qt-mt323.dll
 0002:00000ee8       __imp_?setWrapping@QSpinBox@@UAEX_N@Z 10024ee8     qt-mt323:qt-mt323.dll
 0002:00000eec       __imp_?sizeHint@QCheckBox@@UBE?AVQSize@@XZ 10024eec     qt-mt323:qt-mt323.dll
 0002:00000ef0       __imp_?sizeHint@QGridLayout@@UBE?AVQSize@@XZ 10024ef0     qt-mt323:qt-mt323.dll
 0002:00000ef4       __imp_?sizeHint@QGroupBox@@UBE?AVQSize@@XZ 10024ef4     qt-mt323:qt-mt323.dll
 0002:00000ef8       __imp_?sizeHint@QRadioButton@@UBE?AVQSize@@XZ 10024ef8     qt-mt323:qt-mt323.dll
 0002:00000efc       __imp_?sizeHint@QSpinBox@@UBE?AVQSize@@XZ 10024efc     qt-mt323:qt-mt323.dll
 0002:00000f00       __imp_?stepChange@QRangeControl@@MAEXXZ 10024f00     qt-mt323:qt-mt323.dll
 0002:00000f04       __imp_?stepDown@QSpinBox@@UAEXXZ 10024f04     qt-mt323:qt-mt323.dll
 0002:00000f08       __imp_?stepUp@QSpinBox@@UAEXXZ 10024f08     qt-mt323:qt-mt323.dll
 0002:00000f0c       __imp_?styleChange@QSpinBox@@MAEXAAVQStyle@@@Z 10024f0c     qt-mt323:qt-mt323.dll
 0002:00000f10       __imp_?suffix@QSpinBox@@UBE?AVQString@@XZ 10024f10     qt-mt323:qt-mt323.dll
 0002:00000f14       __imp_?updateDisplay@QSpinBox@@MAEXXZ 10024f14     qt-mt323:qt-mt323.dll
 0002:00000f18       __imp_?updateMask@QCheckBox@@MAEXXZ 10024f18     qt-mt323:qt-mt323.dll
 0002:00000f1c       __imp_?updateMask@QRadioButton@@MAEXXZ 10024f1c     qt-mt323:qt-mt323.dll
 0002:00000f20       __imp_?valueChange@QSpinBox@@MAEXXZ 10024f20     qt-mt323:qt-mt323.dll
 0002:00000f24       __imp_?wheelEvent@QSpinBox@@MAEXPAVQWheelEvent@@@Z 10024f24     qt-mt323:qt-mt323.dll
 0002:00000f28       __imp_?deleteSelf@QStringData@@QAEXXZ 10024f28     qt-mt323:qt-mt323.dll
 0002:00000f2c       __imp_?rightJustify@QString@@QBE?AV1@IVQChar@@_N@Z 10024f2c     qt-mt323:qt-mt323.dll
 0002:00000f30       __imp_?insert@QString@@QAEAAV1@IABV1@@Z 10024f30     qt-mt323:qt-mt323.dll
 0002:00000f34       __imp_?number@QString@@SA?AV1@HH@Z 10024f34     qt-mt323:qt-mt323.dll
 0002:00000f38       __imp_?setLength@QString@@QAEXI@Z 10024f38     qt-mt323:qt-mt323.dll
 0002:00000f3c       __imp_?makeSharedNull@QString@@CAPAUQStringData@@XZ 10024f3c     qt-mt323:qt-mt323.dll
 0002:00000f40       __imp_?unicode@QCharRef@@QBEGXZ 10024f40     qt-mt323:qt-mt323.dll
 0002:00000f44       __imp_?next@QGList@@IAEPAXXZ 10024f44     qt-mt323:qt-mt323.dll
 0002:00000f48       __imp_??0QGListIterator@@IAE@ABVQGList@@@Z 10024f48     qt-mt323:qt-mt323.dll
 0002:00000f4c       __imp_??1QGListIterator@@IAE@XZ 10024f4c     qt-mt323:qt-mt323.dll
 0002:00000f50       __imp_??EQGListIterator@@IAEPAXXZ 10024f50     qt-mt323:qt-mt323.dll
 0002:00000f54       __imp_?shared_null@QString@@0PAUQStringData@@A 10024f54     qt-mt323:qt-mt323.dll
 0002:00000f58       __imp_?qWarning@@YAXPBDZZ  10024f58     qt-mt323:qt-mt323.dll
 0002:00000f5c       __imp_?setResizeMode@QLayout@@QAEXW4ResizeMode@1@@Z 10024f5c     qt-mt323:qt-mt323.dll
 0002:00000f60       __imp_?addLayout@QGridLayout@@QAEXPAVQLayout@@HH@Z 10024f60     qt-mt323:qt-mt323.dll
 0002:00000f64       __imp_?qstrcmp@@YAHPBD0@Z  10024f64     qt-mt323:qt-mt323.dll
 0002:00000f68       __imp_?fromLatin1@QString@@SA?AV1@PBDH@Z 10024f68     qt-mt323:qt-mt323.dll
 0002:00000f6c       __imp_?fromUtf8@QString@@SA?AV1@PBDH@Z 10024f6c     qt-mt323:qt-mt323.dll
 0002:00000f70       __imp_?receivers@QObject@@IBEPAVQConnectionList@@H@Z 10024f70     qt-mt323:qt-mt323.dll
 0002:00000f74       __imp_?activate_signal@QObject@@IAEXPAVQConnectionList@@PAUQUObject@@@Z 10024f74     qt-mt323:qt-mt323.dll
 0002:00000f78       __imp_?staticMetaObject@QWidget@@SAPAVQMetaObject@@XZ 10024f78     qt-mt323:qt-mt323.dll
 0002:00000f7c       __imp_?new_metaobject@QMetaObject@@SAPAV1@PBDPAV1@QBUQMetaData@@H2HQBVQMetaProperty@@HQBUQMetaEnum@@HQBUQClassInfo@@H@Z 10024f7c     qt-mt323:qt-mt323.dll
 0002:00000f80       __imp_??0QMetaObjectCleanUp@@QAE@PBDP6APAVQMetaObject@@XZ@Z 10024f80     qt-mt323:qt-mt323.dll
 0002:00000f84       __imp_??1QMetaObjectCleanUp@@QAE@XZ 10024f84     qt-mt323:qt-mt323.dll
 0002:00000f88       __imp_?setMetaObject@QMetaObjectCleanUp@@QAEXAAPAVQMetaObject@@@Z 10024f88     qt-mt323:qt-mt323.dll
 0002:00000f8c       __imp_?translate@QApplication@@QBE?AVQString@@PBD00W4Encoding@1@@Z 10024f8c     qt-mt323:qt-mt323.dll
 0002:00000f90       __imp_??0QUObject@@QAE@XZ  10024f90     qt-mt323:qt-mt323.dll
 0002:00000f94       __imp_??1QUObject@@QAE@XZ  10024f94     qt-mt323:qt-mt323.dll
 0002:00000f98       __imp_?set@QUType_QString@@QAEXPAUQUObject@@ABVQString@@@Z 10024f98     qt-mt323:qt-mt323.dll
 0002:00000f9c       __imp_?qApp@@3PAVQApplication@@A 10024f9c     qt-mt323:qt-mt323.dll
 0002:00000fa0       __imp_?static_QUType_ptr@@3UQUType_ptr@@A 10024fa0     qt-mt323:qt-mt323.dll
 0002:00000fa4       __imp_?static_QUType_int@@3UQUType_int@@A 10024fa4     qt-mt323:qt-mt323.dll
 0002:00000fa8       __imp_?static_QUType_QString@@3UQUType_QString@@A 10024fa8     qt-mt323:qt-mt323.dll
 0002:00000fac       __imp_?static_QUType_varptr@@3UQUType_varptr@@A 10024fac     qt-mt323:qt-mt323.dll
 0002:00000fb0       __imp_?qt_cast@QDialog@@UAEPAXPBD@Z 10024fb0     qt-mt323:qt-mt323.dll
 0002:00000fb4       __imp_?qt_invoke@QDialog@@UAE_NHPAUQUObject@@@Z 10024fb4     qt-mt323:qt-mt323.dll
 0002:00000fb8       __imp_?qt_emit@QDialog@@UAE_NHPAUQUObject@@@Z 10024fb8     qt-mt323:qt-mt323.dll
 0002:00000fbc       __imp_?qt_property@QDialog@@UAE_NHHPAVQVariant@@@Z 10024fbc     qt-mt323:qt-mt323.dll
 0002:00000fc0       __imp_?staticMetaObject@QDialog@@SAPAVQMetaObject@@XZ 10024fc0     qt-mt323:qt-mt323.dll
 0002:00000fc4       __imp_?activate_signal@QObject@@IAEXH@Z 10024fc4     qt-mt323:qt-mt323.dll
 0002:00000fc8       __imp_?activate_signal@QObject@@IAEXHVQString@@@Z 10024fc8     qt-mt323:qt-mt323.dll
 0002:00000fcc       __imp_?set@QUType_ptr@@QAEXPAUQUObject@@PBX@Z 10024fcc     qt-mt323:qt-mt323.dll
 0002:00000fd0       __imp_?setMinimumSize@QWidget@@QAEXABVQSize@@@Z 10024fd0     qt-mt323:qt-mt323.dll
 0002:00000fd4       __imp_?setMaximumSize@QWidget@@QAEXABVQSize@@@Z 10024fd4     qt-mt323:qt-mt323.dll
 0002:00000fd8       __imp_?resize@QWidget@@QAEXABVQSize@@@Z 10024fd8     qt-mt323:qt-mt323.dll
 0002:00000fdc       __imp_?setIndent@QLabel@@QAEXH@Z 10024fdc     qt-mt323:qt-mt323.dll
 0002:00000fe0       __imp_??0QSplitter@@QAE@PAVQWidget@@PBD@Z 10024fe0     qt-mt323:qt-mt323.dll
 0002:00000fe4       __imp_??1QSplitter@@UAE@XZ 10024fe4     qt-mt323:qt-mt323.dll
 0002:00000fe8       __imp_??0QGroupBox@@QAE@PAVQWidget@@PBD@Z 10024fe8     qt-mt323:qt-mt323.dll
 0002:00000fec       __imp_??1QGroupBox@@UAE@XZ 10024fec     qt-mt323:qt-mt323.dll
 0002:00000ff0       __imp_??0QComboBox@@QAE@_NPAVQWidget@@PBD@Z 10024ff0     qt-mt323:qt-mt323.dll
 0002:00000ff4       __imp_??1QComboBox@@UAE@XZ 10024ff4     qt-mt323:qt-mt323.dll
 0002:00000ff8       __imp_?setDuplicatesEnabled@QComboBox@@QAEX_N@Z 10024ff8     qt-mt323:qt-mt323.dll
 0002:00000ffc       __imp_??0QWidgetStack@@QAE@PAVQWidget@@PBD@Z 10024ffc     qt-mt323:qt-mt323.dll
 0002:00001000       __imp_??1QWidgetStack@@UAE@XZ 10025000     qt-mt323:qt-mt323.dll
 0002:00001004       __imp_?addWidget@QWidgetStack@@QAEHPAVQWidget@@H@Z 10025004     qt-mt323:qt-mt323.dll
 0002:00001008       __imp_??0QListBox@@QAE@PAVQWidget@@PBDI@Z 10025008     qt-mt323:qt-mt323.dll
 0002:0000100c       __imp_??1QListBox@@UAE@XZ  1002500c     qt-mt323:qt-mt323.dll
 0002:00001010       __imp_??0QTimeEdit@@QAE@PAVQWidget@@PBD@Z 10025010     qt-mt323:qt-mt323.dll
 0002:00001014       __imp_??1QTimeEdit@@UAE@XZ 10025014     qt-mt323:qt-mt323.dll
 0002:00001018       __imp_?setDisplay@QTimeEdit@@QAEXI@Z 10025018     qt-mt323:qt-mt323.dll
 0002:0000101c       __imp_??0QTextEdit@@QAE@PAVQWidget@@PBD@Z 1002501c     qt-mt323:qt-mt323.dll
 0002:00001020       __imp_??1QTextEdit@@UAE@XZ 10025020     qt-mt323:qt-mt323.dll
 0002:00001024       __imp_?setAutoFormatting@QTextEdit@@QAEXI@Z 10025024     qt-mt323:qt-mt323.dll
 0002:00001028       __imp_??0QVBoxLayout@@QAE@PAVQLayout@@HPBD@Z 10025028     qt-mt323:qt-mt323.dll
 0002:0000102c       __imp_?addNumber@QTimeEdit@@MAEXHH@Z 1002502c     qt-mt323:qt-mt323.dll
 0002:00001030       __imp_?append@QTextEdit@@UAEXABVQString@@@Z 10025030     qt-mt323:qt-mt323.dll
 0002:00001034       __imp_?childEvent@QSplitter@@MAEXPAVQChildEvent@@@Z 10025034     qt-mt323:qt-mt323.dll
 0002:00001038       __imp_?childEvent@QWidgetStack@@MAEXPAVQChildEvent@@@Z 10025038     qt-mt323:qt-mt323.dll
 0002:0000103c       __imp_?className@QComboBox@@UBEPBDXZ 1002503c     qt-mt323:qt-mt323.dll
 0002:00001040       __imp_?className@QGroupBox@@UBEPBDXZ 10025040     qt-mt323:qt-mt323.dll
 0002:00001044       __imp_?className@QListBox@@UBEPBDXZ 10025044     qt-mt323:qt-mt323.dll
 0002:00001048       __imp_?className@QSplitter@@UBEPBDXZ 10025048     qt-mt323:qt-mt323.dll
 0002:0000104c       __imp_?className@QTextEdit@@UBEPBDXZ 1002504c     qt-mt323:qt-mt323.dll
 0002:00001050       __imp_?className@QTimeEdit@@UBEPBDXZ 10025050     qt-mt323:qt-mt323.dll
 0002:00001054       __imp_?className@QWidgetStack@@UBEPBDXZ 10025054     qt-mt323:qt-mt323.dll
 0002:00001058       __imp_?clear@QTextEdit@@UAEXXZ 10025058     qt-mt323:qt-mt323.dll
 0002:0000105c       __imp_?clearParagraphBackground@QTextEdit@@UAEXH@Z 1002505c     qt-mt323:qt-mt323.dll
 0002:00001060       __imp_?clearSelection@QListBox@@UAEXXZ 10025060     qt-mt323:qt-mt323.dll
 0002:00001064       __imp_?contentsContextMenuEvent@QListBox@@MAEXPAVQContextMenuEvent@@@Z 10025064     qt-mt323:qt-mt323.dll
 0002:00001068       __imp_?contentsContextMenuEvent@QTextEdit@@MAEXPAVQContextMenuEvent@@@Z 10025068     qt-mt323:qt-mt323.dll
 0002:0000106c       __imp_?contentsDragEnterEvent@QScrollView@@MAEXPAVQDragEnterEvent@@@Z 1002506c     qt-mt323:qt-mt323.dll
 0002:00001070       __imp_?contentsDragEnterEvent@QTextEdit@@MAEXPAVQDragEnterEvent@@@Z 10025070     qt-mt323:qt-mt323.dll
 0002:00001074       __imp_?contentsDragLeaveEvent@QScrollView@@MAEXPAVQDragLeaveEvent@@@Z 10025074     qt-mt323:qt-mt323.dll
 0002:00001078       __imp_?contentsDragLeaveEvent@QTextEdit@@MAEXPAVQDragLeaveEvent@@@Z 10025078     qt-mt323:qt-mt323.dll
 0002:0000107c       __imp_?contentsDragMoveEvent@QScrollView@@MAEXPAVQDragMoveEvent@@@Z 1002507c     qt-mt323:qt-mt323.dll
 0002:00001080       __imp_?contentsDragMoveEvent@QTextEdit@@MAEXPAVQDragMoveEvent@@@Z 10025080     qt-mt323:qt-mt323.dll
 0002:00001084       __imp_?contentsDropEvent@QScrollView@@MAEXPAVQDropEvent@@@Z 10025084     qt-mt323:qt-mt323.dll
 0002:00001088       __imp_?contentsDropEvent@QTextEdit@@MAEXPAVQDropEvent@@@Z 10025088     qt-mt323:qt-mt323.dll
 0002:0000108c       __imp_?contentsMouseDoubleClickEvent@QScrollView@@MAEXPAVQMouseEvent@@@Z 1002508c     qt-mt323:qt-mt323.dll
 0002:00001090       __imp_?contentsMouseDoubleClickEvent@QTextEdit@@MAEXPAVQMouseEvent@@@Z 10025090     qt-mt323:qt-mt323.dll
 0002:00001094       __imp_?contentsMouseMoveEvent@QScrollView@@MAEXPAVQMouseEvent@@@Z 10025094     qt-mt323:qt-mt323.dll
 0002:00001098       __imp_?contentsMouseMoveEvent@QTextEdit@@MAEXPAVQMouseEvent@@@Z 10025098     qt-mt323:qt-mt323.dll
 0002:0000109c       __imp_?contentsMousePressEvent@QScrollView@@MAEXPAVQMouseEvent@@@Z 1002509c     qt-mt323:qt-mt323.dll
 0002:000010a0       __imp_?contentsMousePressEvent@QTextEdit@@MAEXPAVQMouseEvent@@@Z 100250a0     qt-mt323:qt-mt323.dll
 0002:000010a4       __imp_?contentsMouseReleaseEvent@QScrollView@@MAEXPAVQMouseEvent@@@Z 100250a4     qt-mt323:qt-mt323.dll
 0002:000010a8       __imp_?contentsMouseReleaseEvent@QTextEdit@@MAEXPAVQMouseEvent@@@Z 100250a8     qt-mt323:qt-mt323.dll
 0002:000010ac       __imp_?contentsWheelEvent@QTextEdit@@MAEXPAVQWheelEvent@@@Z 100250ac     qt-mt323:qt-mt323.dll
 0002:000010b0       __imp_?copy@QTextEdit@@UAEXXZ 100250b0     qt-mt323:qt-mt323.dll
 0002:000010b4       __imp_?createPopupMenu@QTextEdit@@MAEPAVQPopupMenu@@ABVQPoint@@@Z 100250b4     qt-mt323:qt-mt323.dll
 0002:000010b8       __imp_?createPopupMenu@QTextEdit@@MAEPAVQPopupMenu@@XZ 100250b8     qt-mt323:qt-mt323.dll
 0002:000010bc       __imp_?cut@QTextEdit@@UAEXXZ 100250bc     qt-mt323:qt-mt323.dll
 0002:000010c0       __imp_?del@QTextEdit@@UAEXXZ 100250c0     qt-mt323:qt-mt323.dll
 0002:000010c4       __imp_?doChangeInterval@QTextEdit@@MAEXXZ 100250c4     qt-mt323:qt-mt323.dll
 0002:000010c8       __imp_?doKeyboardAction@QTextEdit@@UAEXW4KeyboardAction@1@@Z 100250c8     qt-mt323:qt-mt323.dll
 0002:000010cc       __imp_?drawContents@QTextEdit@@EAEXPAVQPainter@@@Z 100250cc     qt-mt323:qt-mt323.dll
 0002:000010d0       __imp_?drawContents@QTextEdit@@MAEXPAVQPainter@@HHHH@Z 100250d0     qt-mt323:qt-mt323.dll
 0002:000010d4       __imp_?drawContentsOffset@QScrollView@@MAEXPAVQPainter@@HHHHHH@Z 100250d4     qt-mt323:qt-mt323.dll
 0002:000010d8       __imp_?drawSplitter@QSplitter@@MAEXPAVQPainter@@HHHH@Z 100250d8     qt-mt323:qt-mt323.dll
 0002:000010dc       __imp_?emitHighlighted@QTextEdit@@EAEXABVQString@@@Z 100250dc     qt-mt323:qt-mt323.dll
 0002:000010e0       __imp_?emitLinkClicked@QTextEdit@@EAEXABVQString@@@Z 100250e0     qt-mt323:qt-mt323.dll
 0002:000010e4       __imp_?ensureCurrentVisible@QListBox@@UAEXXZ 100250e4     qt-mt323:qt-mt323.dll
 0002:000010e8       __imp_?ensureCursorVisible@QTextEdit@@UAEXXZ 100250e8     qt-mt323:qt-mt323.dll
 0002:000010ec       __imp_?event@QGroupBox@@MAE_NPAVQEvent@@@Z 100250ec     qt-mt323:qt-mt323.dll
 0002:000010f0       __imp_?event@QSplitter@@MAE_NPAVQEvent@@@Z 100250f0     qt-mt323:qt-mt323.dll
 0002:000010f4       __imp_?event@QTextEdit@@MAE_NPAVQEvent@@@Z 100250f4     qt-mt323:qt-mt323.dll
 0002:000010f8       __imp_?event@QTimeEdit@@MAE_NPAVQEvent@@@Z 100250f8     qt-mt323:qt-mt323.dll
 0002:000010fc       __imp_?eventFilter@QComboBox@@UAE_NPAVQObject@@PAVQEvent@@@Z 100250fc     qt-mt323:qt-mt323.dll
 0002:00001100       __imp_?eventFilter@QListBox@@MAE_NPAVQObject@@PAVQEvent@@@Z 10025100     qt-mt323:qt-mt323.dll
 0002:00001104       __imp_?eventFilter@QTextEdit@@UAE_NPAVQObject@@PAVQEvent@@@Z 10025104     qt-mt323:qt-mt323.dll
 0002:00001108       __imp_?find@QTextEdit@@UAE_NABVQString@@_N11PAH2@Z 10025108     qt-mt323:qt-mt323.dll
 0002:0000110c       __imp_?focusInEvent@QComboBox@@MAEXPAVQFocusEvent@@@Z 1002510c     qt-mt323:qt-mt323.dll
 0002:00001110       __imp_?focusInEvent@QListBox@@MAEXPAVQFocusEvent@@@Z 10025110     qt-mt323:qt-mt323.dll
 0002:00001114       __imp_?focusNextPrevChild@QTextEdit@@MAE_N_N@Z 10025114     qt-mt323:qt-mt323.dll
 0002:00001118       __imp_?focusOutEvent@QComboBox@@MAEXPAVQFocusEvent@@@Z 10025118     qt-mt323:qt-mt323.dll
 0002:0000111c       __imp_?focusOutEvent@QListBox@@MAEXPAVQFocusEvent@@@Z 1002511c     qt-mt323:qt-mt323.dll
 0002:00001120       __imp_?frameChanged@QWidgetStack@@MAEXXZ 10025120     qt-mt323:qt-mt323.dll
 0002:00001124       __imp_?getFormat@QTextEdit@@UAE_NHHPAVQFont@@PAVQColor@@PAW4VerticalAlignment@1@@Z 10025124     qt-mt323:qt-mt323.dll
 0002:00001128       __imp_?getParagraphFormat@QTextEdit@@UAE_NHPAVQFont@@PAVQColor@@PAW4VerticalAlignment@1@PAHPAW4DisplayMode@QStyleSheetItem@@PAW4ListStyle@6@3@Z 10025128     qt-mt323:qt-mt323.dll
 0002:0000112c       __imp_?heightForWidth@QTextEdit@@UBEHH@Z 1002512c     qt-mt323:qt-mt323.dll
 0002:00001130       __imp_?imComposeEvent@QTextEdit@@MAEXPAVQIMEvent@@@Z 10025130     qt-mt323:qt-mt323.dll
 0002:00001134       __imp_?imEndEvent@QTextEdit@@MAEXPAVQIMEvent@@@Z 10025134     qt-mt323:qt-mt323.dll
 0002:00001138       __imp_?imStartEvent@QTextEdit@@MAEXPAVQIMEvent@@@Z 10025138     qt-mt323:qt-mt323.dll
 0002:0000113c       __imp_?indent@QTextEdit@@UAEXXZ 1002513c     qt-mt323:qt-mt323.dll
 0002:00001140       __imp_?insert@QTextEdit@@UAEXABVQString@@_N11@Z 10025140     qt-mt323:qt-mt323.dll
 0002:00001144       __imp_?insertAt@QTextEdit@@UAEXABVQString@@HH@Z 10025144     qt-mt323:qt-mt323.dll
 0002:00001148       __imp_?insertParagraph@QTextEdit@@UAEXABVQString@@H@Z 10025148     qt-mt323:qt-mt323.dll
 0002:0000114c       __imp_?invertSelection@QListBox@@UAEXXZ 1002514c     qt-mt323:qt-mt323.dll
 0002:00001150       __imp_?keyPressEvent@QComboBox@@MAEXPAVQKeyEvent@@@Z 10025150     qt-mt323:qt-mt323.dll
 0002:00001154       __imp_?keyPressEvent@QListBox@@MAEXPAVQKeyEvent@@@Z 10025154     qt-mt323:qt-mt323.dll
 0002:00001158       __imp_?keyPressEvent@QTextEdit@@MAEXPAVQKeyEvent@@@Z 10025158     qt-mt323:qt-mt323.dll
 0002:0000115c       __imp_?linksEnabled@QTextEdit@@EBE_NXZ 1002515c     qt-mt323:qt-mt323.dll
 0002:00001160       __imp_?metaObject@QComboBox@@UBEPAVQMetaObject@@XZ 10025160     qt-mt323:qt-mt323.dll
 0002:00001164       __imp_?metaObject@QGroupBox@@UBEPAVQMetaObject@@XZ 10025164     qt-mt323:qt-mt323.dll
 0002:00001168       __imp_?metaObject@QListBox@@UBEPAVQMetaObject@@XZ 10025168     qt-mt323:qt-mt323.dll
 0002:0000116c       __imp_?metaObject@QSplitter@@UBEPAVQMetaObject@@XZ 1002516c     qt-mt323:qt-mt323.dll
 0002:00001170       __imp_?metaObject@QTextEdit@@UBEPAVQMetaObject@@XZ 10025170     qt-mt323:qt-mt323.dll
 0002:00001174       __imp_?metaObject@QTimeEdit@@UBEPAVQMetaObject@@XZ 10025174     qt-mt323:qt-mt323.dll
 0002:00001178       __imp_?metaObject@QWidgetStack@@UBEPAVQMetaObject@@XZ 10025178     qt-mt323:qt-mt323.dll
 0002:0000117c       __imp_?minimumSizeHint@QListBox@@UBE?AVQSize@@XZ 1002517c     qt-mt323:qt-mt323.dll
 0002:00001180       __imp_?minimumSizeHint@QScrollView@@UBE?AVQSize@@XZ 10025180     qt-mt323:qt-mt323.dll
 0002:00001184       __imp_?minimumSizeHint@QSplitter@@UBE?AVQSize@@XZ 10025184     qt-mt323:qt-mt323.dll
 0002:00001188       __imp_?minimumSizeHint@QTimeEdit@@UBE?AVQSize@@XZ 10025188     qt-mt323:qt-mt323.dll
 0002:0000118c       __imp_?minimumSizeHint@QWidgetStack@@UBE?AVQSize@@XZ 1002518c     qt-mt323:qt-mt323.dll
 0002:00001190       __imp_?mouseDoubleClickEvent@QComboBox@@MAEXPAVQMouseEvent@@@Z 10025190     qt-mt323:qt-mt323.dll
 0002:00001194       __imp_?mouseDoubleClickEvent@QListBox@@MAEXPAVQMouseEvent@@@Z 10025194     qt-mt323:qt-mt323.dll
 0002:00001198       __imp_?mouseMoveEvent@QComboBox@@MAEXPAVQMouseEvent@@@Z 10025198     qt-mt323:qt-mt323.dll
 0002:0000119c       __imp_?mouseMoveEvent@QListBox@@MAEXPAVQMouseEvent@@@Z 1002519c     qt-mt323:qt-mt323.dll
 0002:000011a0       __imp_?mousePressEvent@QComboBox@@MAEXPAVQMouseEvent@@@Z 100251a0     qt-mt323:qt-mt323.dll
 0002:000011a4       __imp_?mousePressEvent@QListBox@@MAEXPAVQMouseEvent@@@Z 100251a4     qt-mt323:qt-mt323.dll
 0002:000011a8       __imp_?mouseReleaseEvent@QComboBox@@MAEXPAVQMouseEvent@@@Z 100251a8     qt-mt323:qt-mt323.dll
 0002:000011ac       __imp_?mouseReleaseEvent@QListBox@@MAEXPAVQMouseEvent@@@Z 100251ac     qt-mt323:qt-mt323.dll
 0002:000011b0       __imp_?moveCursor@QTextEdit@@UAEXW4CursorAction@1@_N@Z 100251b0     qt-mt323:qt-mt323.dll
 0002:000011b4       __imp_?outOfRange@QTimeEdit@@MBE_NHHH@Z 100251b4     qt-mt323:qt-mt323.dll
 0002:000011b8       __imp_?paintCell@QListBox@@MAEXPAVQPainter@@HH@Z 100251b8     qt-mt323:qt-mt323.dll
 0002:000011bc       __imp_?paintEvent@QComboBox@@MAEXPAVQPaintEvent@@@Z 100251bc     qt-mt323:qt-mt323.dll
 0002:000011c0       __imp_?paste@QTextEdit@@UAEXXZ 100251c0     qt-mt323:qt-mt323.dll
 0002:000011c4       __imp_?pasteSubType@QTextEdit@@UAEXABVQCString@@@Z 100251c4     qt-mt323:qt-mt323.dll
 0002:000011c8       __imp_?placeCursor@QTextEdit@@UAEXABVQPoint@@PAVQTextCursor@@@Z 100251c8     qt-mt323:qt-mt323.dll
 0002:000011cc       __imp_?polish@QTextEdit@@UAEXXZ 100251cc     qt-mt323:qt-mt323.dll
 0002:000011d0       __imp_?popup@QComboBox@@UAEXXZ 100251d0     qt-mt323:qt-mt323.dll
 0002:000011d4       __imp_?qt_cast@QComboBox@@UAEPAXPBD@Z 100251d4     qt-mt323:qt-mt323.dll
 0002:000011d8       __imp_?qt_cast@QGroupBox@@UAEPAXPBD@Z 100251d8     qt-mt323:qt-mt323.dll
 0002:000011dc       __imp_?qt_cast@QListBox@@UAEPAXPBD@Z 100251dc     qt-mt323:qt-mt323.dll
 0002:000011e0       __imp_?qt_cast@QSplitter@@UAEPAXPBD@Z 100251e0     qt-mt323:qt-mt323.dll
 0002:000011e4       __imp_?qt_cast@QTextEdit@@UAEPAXPBD@Z 100251e4     qt-mt323:qt-mt323.dll
 0002:000011e8       __imp_?qt_cast@QTimeEdit@@UAEPAXPBD@Z 100251e8     qt-mt323:qt-mt323.dll
 0002:000011ec       __imp_?qt_cast@QWidgetStack@@UAEPAXPBD@Z 100251ec     qt-mt323:qt-mt323.dll
 0002:000011f0       __imp_?qt_emit@QComboBox@@UAE_NHPAUQUObject@@@Z 100251f0     qt-mt323:qt-mt323.dll
 0002:000011f4       __imp_?qt_emit@QGroupBox@@UAE_NHPAUQUObject@@@Z 100251f4     qt-mt323:qt-mt323.dll
 0002:000011f8       __imp_?qt_emit@QListBox@@UAE_NHPAUQUObject@@@Z 100251f8     qt-mt323:qt-mt323.dll
 0002:000011fc       __imp_?qt_emit@QSplitter@@UAE_NHPAUQUObject@@@Z 100251fc     qt-mt323:qt-mt323.dll
 0002:00001200       __imp_?qt_emit@QTextEdit@@UAE_NHPAUQUObject@@@Z 10025200     qt-mt323:qt-mt323.dll
 0002:00001204       __imp_?qt_emit@QTimeEdit@@UAE_NHPAUQUObject@@@Z 10025204     qt-mt323:qt-mt323.dll
 0002:00001208       __imp_?qt_emit@QWidgetStack@@UAE_NHPAUQUObject@@@Z 10025208     qt-mt323:qt-mt323.dll
 0002:0000120c       __imp_?qt_invoke@QComboBox@@UAE_NHPAUQUObject@@@Z 1002520c     qt-mt323:qt-mt323.dll
 0002:00001210       __imp_?qt_invoke@QGroupBox@@UAE_NHPAUQUObject@@@Z 10025210     qt-mt323:qt-mt323.dll
 0002:00001214       __imp_?qt_invoke@QListBox@@UAE_NHPAUQUObject@@@Z 10025214     qt-mt323:qt-mt323.dll
 0002:00001218       __imp_?qt_invoke@QSplitter@@UAE_NHPAUQUObject@@@Z 10025218     qt-mt323:qt-mt323.dll
 0002:0000121c       __imp_?qt_invoke@QTextEdit@@UAE_NHPAUQUObject@@@Z 1002521c     qt-mt323:qt-mt323.dll
 0002:00001220       __imp_?qt_invoke@QTimeEdit@@UAE_NHPAUQUObject@@@Z 10025220     qt-mt323:qt-mt323.dll
 0002:00001224       __imp_?qt_invoke@QWidgetStack@@UAE_NHPAUQUObject@@@Z 10025224     qt-mt323:qt-mt323.dll
 0002:00001228       __imp_?qt_property@QComboBox@@UAE_NHHPAVQVariant@@@Z 10025228     qt-mt323:qt-mt323.dll
 0002:0000122c       __imp_?qt_property@QGroupBox@@UAE_NHHPAVQVariant@@@Z 1002522c     qt-mt323:qt-mt323.dll
 0002:00001230       __imp_?qt_property@QListBox@@UAE_NHHPAVQVariant@@@Z 10025230     qt-mt323:qt-mt323.dll
 0002:00001234       __imp_?qt_property@QSplitter@@UAE_NHHPAVQVariant@@@Z 10025234     qt-mt323:qt-mt323.dll
 0002:00001238       __imp_?qt_property@QTextEdit@@UAE_NHHPAVQVariant@@@Z 10025238     qt-mt323:qt-mt323.dll
 0002:0000123c       __imp_?qt_property@QTimeEdit@@UAE_NHHPAVQVariant@@@Z 1002523c     qt-mt323:qt-mt323.dll
 0002:00001240       __imp_?qt_property@QWidgetStack@@UAE_NHHPAVQVariant@@@Z 10025240     qt-mt323:qt-mt323.dll
 0002:00001244       __imp_?redo@QTextEdit@@UAEXXZ 10025244     qt-mt323:qt-mt323.dll
 0002:00001248       __imp_?removeLastNumber@QTimeEdit@@MAEXH@Z 10025248     qt-mt323:qt-mt323.dll
 0002:0000124c       __imp_?removeParagraph@QTextEdit@@UAEXH@Z 1002524c     qt-mt323:qt-mt323.dll
 0002:00001250       __imp_?removeSelectedText@QTextEdit@@UAEXH@Z 10025250     qt-mt323:qt-mt323.dll
 0002:00001254       __imp_?removeSelection@QTextEdit@@UAEXH@Z 10025254     qt-mt323:qt-mt323.dll
 0002:00001258       __imp_?resetFormat@QTextEdit@@UAEXXZ 10025258     qt-mt323:qt-mt323.dll
 0002:0000125c       __imp_?resizeEvent@QComboBox@@MAEXPAVQResizeEvent@@@Z 1002525c     qt-mt323:qt-mt323.dll
 0002:00001260       __imp_?resizeEvent@QListBox@@MAEXPAVQResizeEvent@@@Z 10025260     qt-mt323:qt-mt323.dll
 0002:00001264       __imp_?resizeEvent@QSplitter@@MAEXPAVQResizeEvent@@@Z 10025264     qt-mt323:qt-mt323.dll
 0002:00001268       __imp_?resizeEvent@QTextEdit@@MAEXPAVQResizeEvent@@@Z 10025268     qt-mt323:qt-mt323.dll
 0002:0000126c       __imp_?resizeEvent@QTimeEdit@@MAEXPAVQResizeEvent@@@Z 1002526c     qt-mt323:qt-mt323.dll
 0002:00001270       __imp_?resizeEvent@QWidgetStack@@MAEXPAVQResizeEvent@@@Z 10025270     qt-mt323:qt-mt323.dll
 0002:00001274       __imp_?scrollToAnchor@QTextEdit@@UAEXABVQString@@@Z 10025274     qt-mt323:qt-mt323.dll
 0002:00001278       __imp_?scrollToBottom@QTextEdit@@UAEXXZ 10025278     qt-mt323:qt-mt323.dll
 0002:0000127c       __imp_?sectionFormattedText@QTimeEdit@@MAE?AVQString@@H@Z 1002527c     qt-mt323:qt-mt323.dll
 0002:00001280       __imp_?selectAll@QListBox@@UAEX_N@Z 10025280     qt-mt323:qt-mt323.dll
 0002:00001284       __imp_?selectAll@QTextEdit@@UAEX_N@Z 10025284     qt-mt323:qt-mt323.dll
 0002:00001288       __imp_?setAlignment@QTextEdit@@UAEXH@Z 10025288     qt-mt323:qt-mt323.dll
 0002:0000128c       __imp_?setAutoAdvance@QTimeEdit@@UAEX_N@Z 1002528c     qt-mt323:qt-mt323.dll
 0002:00001290       __imp_?setAutoCompletion@QComboBox@@UAEX_N@Z 10025290     qt-mt323:qt-mt323.dll
 0002:00001294       __imp_?setAutoResize@QComboBox@@UAEX_N@Z 10025294     qt-mt323:qt-mt323.dll
 0002:00001298       __imp_?setBold@QTextEdit@@UAEX_N@Z 10025298     qt-mt323:qt-mt323.dll
 0002:0000129c       __imp_?setBottomItem@QListBox@@UAEXH@Z 1002529c     qt-mt323:qt-mt323.dll
 0002:000012a0       __imp_?setChildGeometries@QWidgetStack@@MAEXXZ 100252a0     qt-mt323:qt-mt323.dll
 0002:000012a4       __imp_?setColor@QTextEdit@@UAEXABVQColor@@@Z 100252a4     qt-mt323:qt-mt323.dll
 0002:000012a8       __imp_?setColumnMode@QListBox@@UAEXH@Z 100252a8     qt-mt323:qt-mt323.dll
 0002:000012ac       __imp_?setColumnMode@QListBox@@UAEXW4LayoutMode@1@@Z 100252ac     qt-mt323:qt-mt323.dll
 0002:000012b0       __imp_?setContentsPos@QScrollView@@UAEXHH@Z 100252b0     qt-mt323:qt-mt323.dll
 0002:000012b4       __imp_?setCurrentFont@QTextEdit@@UAEXABVQFont@@@Z 100252b4     qt-mt323:qt-mt323.dll
 0002:000012b8       __imp_?setCurrentItem@QComboBox@@UAEXH@Z 100252b8     qt-mt323:qt-mt323.dll
 0002:000012bc       __imp_?setCurrentItem@QListBox@@UAEXH@Z 100252bc     qt-mt323:qt-mt323.dll
 0002:000012c0       __imp_?setCurrentItem@QListBox@@UAEXPAVQListBoxItem@@@Z 100252c0     qt-mt323:qt-mt323.dll
 0002:000012c4       __imp_?setCurrentText@QComboBox@@UAEXABVQString@@@Z 100252c4     qt-mt323:qt-mt323.dll
 0002:000012c8       __imp_?setCursorPosition@QTextEdit@@UAEXHH@Z 100252c8     qt-mt323:qt-mt323.dll
 0002:000012cc       __imp_?setEditText@QComboBox@@UAEXABVQString@@@Z 100252cc     qt-mt323:qt-mt323.dll
 0002:000012d0       __imp_?setEnabled@QComboBox@@UAEX_N@Z 100252d0     qt-mt323:qt-mt323.dll
 0002:000012d4       __imp_?setEnabled@QTextEdit@@UAEX_N@Z 100252d4     qt-mt323:qt-mt323.dll
 0002:000012d8       __imp_?setFamily@QTextEdit@@UAEXABVQString@@@Z 100252d8     qt-mt323:qt-mt323.dll
 0002:000012dc       __imp_?setFocusSection@QTimeEdit@@MAE_NH@Z 100252dc     qt-mt323:qt-mt323.dll
 0002:000012e0       __imp_?setFont@QComboBox@@UAEXABVQFont@@@Z 100252e0     qt-mt323:qt-mt323.dll
 0002:000012e4       __imp_?setFont@QListBox@@UAEXABVQFont@@@Z 100252e4     qt-mt323:qt-mt323.dll
 0002:000012e8       __imp_?setFont@QTextEdit@@UAEXABVQFont@@@Z 100252e8     qt-mt323:qt-mt323.dll
 0002:000012ec       __imp_?setFormat@QTextEdit@@UAEXPAVQTextFormat@@H@Z 100252ec     qt-mt323:qt-mt323.dll
 0002:000012f0       __imp_?setFrameRect@QWidgetStack@@UAEXABVQRect@@@Z 100252f0     qt-mt323:qt-mt323.dll
 0002:000012f4       __imp_?setHour@QTimeEdit@@MAEXH@Z 100252f4     qt-mt323:qt-mt323.dll
 0002:000012f8       __imp_?setInsertionPolicy@QComboBox@@UAEXW4Policy@1@@Z 100252f8     qt-mt323:qt-mt323.dll
 0002:000012fc       __imp_?setItalic@QTextEdit@@UAEX_N@Z 100252fc     qt-mt323:qt-mt323.dll
 0002:00001300       __imp_?setLineEdit@QComboBox@@UAEXPAVQLineEdit@@@Z 10025300     qt-mt323:qt-mt323.dll
 0002:00001304       __imp_?setLinkUnderline@QTextEdit@@UAEX_N@Z 10025304     qt-mt323:qt-mt323.dll
 0002:00001308       __imp_?setListBox@QComboBox@@UAEXPAVQListBox@@@Z 10025308     qt-mt323:qt-mt323.dll
 0002:0000130c       __imp_?setMaxCount@QComboBox@@UAEXH@Z 1002530c     qt-mt323:qt-mt323.dll
 0002:00001310       __imp_?setMaxValue@QTimeEdit@@UAEXABVQTime@@@Z 10025310     qt-mt323:qt-mt323.dll
 0002:00001314       __imp_?setMimeSourceFactory@QTextEdit@@UAEXPAVQMimeSourceFactory@@@Z 10025314     qt-mt323:qt-mt323.dll
 0002:00001318       __imp_?setMinValue@QTimeEdit@@UAEXABVQTime@@@Z 10025318     qt-mt323:qt-mt323.dll
 0002:0000131c       __imp_?setMinute@QTimeEdit@@MAEXH@Z 1002531c     qt-mt323:qt-mt323.dll
 0002:00001320       __imp_?setModified@QTextEdit@@UAEX_N@Z 10025320     qt-mt323:qt-mt323.dll
 0002:00001324       __imp_?setOpaqueResize@QSplitter@@UAEX_N@Z 10025324     qt-mt323:qt-mt323.dll
 0002:00001328       __imp_?setOrientation@QSplitter@@UAEXW4Orientation@Qt@@@Z 10025328     qt-mt323:qt-mt323.dll
 0002:0000132c       __imp_?setOverwriteMode@QTextEdit@@UAEX_N@Z 1002532c     qt-mt323:qt-mt323.dll
 0002:00001330       __imp_?setPalette@QComboBox@@UAEXABVQPalette@@@Z 10025330     qt-mt323:qt-mt323.dll
 0002:00001334       __imp_?setPalette@QTextEdit@@UAEXABVQPalette@@@Z 10025334     qt-mt323:qt-mt323.dll
 0002:00001338       __imp_?setPaper@QTextEdit@@UAEXABVQBrush@@@Z 10025338     qt-mt323:qt-mt323.dll
 0002:0000133c       __imp_?setParagType@QTextEdit@@UAEXW4DisplayMode@QStyleSheetItem@@W4ListStyle@3@@Z 1002533c     qt-mt323:qt-mt323.dll
 0002:00001340       __imp_?setParagraphBackgroundColor@QTextEdit@@UAEXHABVQColor@@@Z 10025340     qt-mt323:qt-mt323.dll
 0002:00001344       __imp_?setPointSize@QTextEdit@@UAEXH@Z 10025344     qt-mt323:qt-mt323.dll
 0002:00001348       __imp_?setRange@QTimeEdit@@UAEXABVQTime@@0@Z 10025348     qt-mt323:qt-mt323.dll
 0002:0000134c       __imp_?setReadOnly@QTextEdit@@UAEX_N@Z 1002534c     qt-mt323:qt-mt323.dll
 0002:00001350       __imp_?setResizeMode@QSplitter@@UAEXPAVQWidget@@W4ResizeMode@1@@Z 10025350     qt-mt323:qt-mt323.dll
 0002:00001354       __imp_?setRowMode@QListBox@@UAEXH@Z 10025354     qt-mt323:qt-mt323.dll
 0002:00001358       __imp_?setRowMode@QListBox@@UAEXW4LayoutMode@1@@Z 10025358     qt-mt323:qt-mt323.dll
 0002:0000135c       __imp_?setRubberband@QSplitter@@MAEXH@Z 1002535c     qt-mt323:qt-mt323.dll
 0002:00001360       __imp_?setSecond@QTimeEdit@@MAEXH@Z 10025360     qt-mt323:qt-mt323.dll
 0002:00001364       __imp_?setSelected@QListBox@@UAEXPAVQListBoxItem@@_N@Z 10025364     qt-mt323:qt-mt323.dll
 0002:00001368       __imp_?setSelection@QTextEdit@@UAEXHHHHH@Z 10025368     qt-mt323:qt-mt323.dll
 0002:0000136c       __imp_?setSelectionAttributes@QTextEdit@@UAEXHABVQColor@@_N@Z 1002536c     qt-mt323:qt-mt323.dll
 0002:00001370       __imp_?setSelectionMode@QListBox@@UAEXW4SelectionMode@1@@Z 10025370     qt-mt323:qt-mt323.dll
 0002:00001374       __imp_?setSeparator@QTimeEdit@@UAEXABVQString@@@Z 10025374     qt-mt323:qt-mt323.dll
 0002:00001378       __imp_?setSizeLimit@QComboBox@@UAEXH@Z 10025378     qt-mt323:qt-mt323.dll
 0002:0000137c       __imp_?setStyleSheet@QTextEdit@@UAEXPAVQStyleSheet@@@Z 1002537c     qt-mt323:qt-mt323.dll
 0002:00001380       __imp_?setTabStopWidth@QTextEdit@@UAEXH@Z 10025380     qt-mt323:qt-mt323.dll
 0002:00001384       __imp_?setText@QTextEdit@@UAEXABVQString@@0@Z 10025384     qt-mt323:qt-mt323.dll
 0002:00001388       __imp_?setTextFormat@QTextEdit@@UAEXW4TextFormat@Qt@@@Z 10025388     qt-mt323:qt-mt323.dll
 0002:0000138c       __imp_?setTime@QTimeEdit@@UAEXABVQTime@@@Z 1002538c     qt-mt323:qt-mt323.dll
 0002:00001390       __imp_?setTopItem@QListBox@@UAEXH@Z 10025390     qt-mt323:qt-mt323.dll
 0002:00001394       __imp_?setUnderline@QTextEdit@@UAEX_N@Z 10025394     qt-mt323:qt-mt323.dll
 0002:00001398       __imp_?setUndoDepth@QTextEdit@@UAEXH@Z 10025398     qt-mt323:qt-mt323.dll
 0002:0000139c       __imp_?setUndoRedoEnabled@QTextEdit@@UAEX_N@Z 1002539c     qt-mt323:qt-mt323.dll
 0002:000013a0       __imp_?setValidator@QComboBox@@UAEXPBVQValidator@@@Z 100253a0     qt-mt323:qt-mt323.dll
 0002:000013a4       __imp_?setVariableHeight@QListBox@@UAEX_N@Z 100253a4     qt-mt323:qt-mt323.dll
 0002:000013a8       __imp_?setVariableWidth@QListBox@@UAEX_N@Z 100253a8     qt-mt323:qt-mt323.dll
 0002:000013ac       __imp_?setVerticalAlignment@QTextEdit@@UAEXW4VerticalAlignment@1@@Z 100253ac     qt-mt323:qt-mt323.dll
 0002:000013b0       __imp_?setWordWrap@QTextEdit@@UAEXW4WordWrap@1@@Z 100253b0     qt-mt323:qt-mt323.dll
 0002:000013b4       __imp_?setWrapColumnOrWidth@QTextEdit@@UAEXH@Z 100253b4     qt-mt323:qt-mt323.dll
 0002:000013b8       __imp_?setWrapPolicy@QTextEdit@@UAEXW4WrapPolicy@1@@Z 100253b8     qt-mt323:qt-mt323.dll
 0002:000013bc       __imp_?show@QScrollView@@UAEXXZ 100253bc     qt-mt323:qt-mt323.dll
 0002:000013c0       __imp_?show@QWidgetStack@@UAEXXZ 100253c0     qt-mt323:qt-mt323.dll
 0002:000013c4       __imp_?showEvent@QListBox@@MAEXPAVQShowEvent@@@Z 100253c4     qt-mt323:qt-mt323.dll
 0002:000013c8       __imp_?sizeHint@QComboBox@@UBE?AVQSize@@XZ 100253c8     qt-mt323:qt-mt323.dll
 0002:000013cc       __imp_?sizeHint@QListBox@@UBE?AVQSize@@XZ 100253cc     qt-mt323:qt-mt323.dll
 0002:000013d0       __imp_?sizeHint@QSplitter@@UBE?AVQSize@@XZ 100253d0     qt-mt323:qt-mt323.dll
 0002:000013d4       __imp_?sizeHint@QTextEdit@@UBE?AVQSize@@XZ 100253d4     qt-mt323:qt-mt323.dll
 0002:000013d8       __imp_?sizeHint@QTimeEdit@@UBE?AVQSize@@XZ 100253d8     qt-mt323:qt-mt323.dll
 0002:000013dc       __imp_?sizeHint@QWidgetStack@@UBE?AVQSize@@XZ 100253dc     qt-mt323:qt-mt323.dll
 0002:000013e0       __imp_?stepDown@QTimeEdit@@MAEXXZ 100253e0     qt-mt323:qt-mt323.dll
 0002:000013e4       __imp_?stepUp@QTimeEdit@@MAEXXZ 100253e4     qt-mt323:qt-mt323.dll
 0002:000013e8       __imp_?styleChange@QComboBox@@MAEXAAVQStyle@@@Z 100253e8     qt-mt323:qt-mt323.dll
 0002:000013ec       __imp_?styleChange@QScrollView@@UAEXAAVQStyle@@@Z 100253ec     qt-mt323:qt-mt323.dll
 0002:000013f0       __imp_?styleChange@QSplitter@@MAEXAAVQStyle@@@Z 100253f0     qt-mt323:qt-mt323.dll
 0002:000013f4       __imp_?sync@QTextEdit@@UAEXXZ 100253f4     qt-mt323:qt-mt323.dll
 0002:000013f8       __imp_?timerEvent@QTimeEdit@@MAEXPAVQTimerEvent@@@Z 100253f8     qt-mt323:qt-mt323.dll
 0002:000013fc       __imp_?undo@QTextEdit@@UAEXXZ 100253fc     qt-mt323:qt-mt323.dll
 0002:00001400       __imp_?updateMask@QComboBox@@MAEXXZ 10025400     qt-mt323:qt-mt323.dll
 0002:00001404       __imp_?viewportPaintEvent@QListBox@@UAEXPAVQPaintEvent@@@Z 10025404     qt-mt323:qt-mt323.dll
 0002:00001408       __imp_?viewportResizeEvent@QScrollView@@MAEXPAVQResizeEvent@@@Z 10025408     qt-mt323:qt-mt323.dll
 0002:0000140c       __imp_?viewportResizeEvent@QTextEdit@@MAEXPAVQResizeEvent@@@Z 1002540c     qt-mt323:qt-mt323.dll
 0002:00001410       __imp_?wheelEvent@QComboBox@@MAEXPAVQWheelEvent@@@Z 10025410     qt-mt323:qt-mt323.dll
 0002:00001414       __imp_?windowActivationChange@QListBox@@MAEX_N@Z 10025414     qt-mt323:qt-mt323.dll
 0002:00001418       __imp_?windowActivationChange@QTextEdit@@MAEX_N@Z 10025418     qt-mt323:qt-mt323.dll
 0002:0000141c       __imp_?zoomIn@QTextEdit@@UAEXH@Z 1002541c     qt-mt323:qt-mt323.dll
 0002:00001420       __imp_?zoomIn@QTextEdit@@UAEXXZ 10025420     qt-mt323:qt-mt323.dll
 0002:00001424       __imp_?zoomOut@QTextEdit@@UAEXH@Z 10025424     qt-mt323:qt-mt323.dll
 0002:00001428       __imp_?zoomOut@QTextEdit@@UAEXXZ 10025428     qt-mt323:qt-mt323.dll
 0002:0000142c       __imp_?zoomTo@QTextEdit@@UAEXH@Z 1002542c     qt-mt323:qt-mt323.dll
 0002:00001430       __imp_??0QGList@@IAE@XZ    10025430     qt-mt323:qt-mt323.dll
 0002:00001434       __imp_?detachInternal@?$QValueList@VQString@@@@AAEXXZ 10025434     qt-mt323:qt-mt323.dll
 0002:00001438       __imp_?contains@?$QValueList@VQString@@@@QBEIABVQString@@@Z 10025438     qt-mt323:qt-mt323.dll
 0002:0000143c       __imp_?findIndex@?$QValueList@VQString@@@@QBEHABVQString@@@Z 1002543c     qt-mt323:qt-mt323.dll
 0002:00001440       __imp_?find@?$QValueList@VQString@@@@QAE?AV?$QValueListIterator@VQString@@@@ABVQString@@@Z 10025440     qt-mt323:qt-mt323.dll
 0002:00001444       __imp_??A?$QValueList@VQString@@@@QAEAAVQString@@I@Z 10025444     qt-mt323:qt-mt323.dll
 0002:00001448       __imp_?remove@?$QValueList@VQString@@@@QAE?AV?$QValueListIterator@VQString@@@@V2@@Z 10025448     qt-mt323:qt-mt323.dll
 0002:0000144c       __imp_?append@?$QValueList@VQString@@@@QAE?AV?$QValueListIterator@VQString@@@@ABVQString@@@Z 1002544c     qt-mt323:qt-mt323.dll
 0002:00001450       __imp_?clear@?$QValueList@VQString@@@@QAEXXZ 10025450     qt-mt323:qt-mt323.dll
 0002:00001454       __imp_?remove@?$QValueList@VQString@@@@QAEIABVQString@@@Z 10025454     qt-mt323:qt-mt323.dll
 0002:00001458       __imp_?begin@?$QValueList@VQString@@@@QAE?AV?$QValueListIterator@VQString@@@@XZ 10025458     qt-mt323:qt-mt323.dll
 0002:0000145c       __imp_?sizeHint@QBoxLayout@@UBE?AVQSize@@XZ 1002545c     qt-mt323:qt-mt323.dll
 0002:00001460       __imp_?readLine@QTextStream@@QAE?AVQString@@XZ 10025460     qt-mt323:qt-mt323.dll
 0002:00001464       __imp_??4QString@@QAEAAV0@PBD@Z 10025464     qt-mt323:qt-mt323.dll
 0002:00001468       __imp_??4QString@@QAEAAV0@ABV0@@Z 10025468     qt-mt323:qt-mt323.dll
 0002:0000146c       __imp_??6QTextStream@@QAEAAV0@PBD@Z 1002546c     qt-mt323:qt-mt323.dll
 0002:00001470       __imp_?atEnd@QTextStream@@QBE_NXZ 10025470     qt-mt323:qt-mt323.dll
 0002:00001474       __imp_??1QTextStream@@UAE@XZ 10025474     qt-mt323:qt-mt323.dll
 0002:00001478       __imp_??0QTextStream@@QAE@PAVQIODevice@@@Z 10025478     qt-mt323:qt-mt323.dll
 0002:0000147c       __imp_?reset@QIODevice@@QAE_NXZ 1002547c     qt-mt323:qt-mt323.dll
 0002:00001480       __imp_??H@YA?BVQString@@PBDABV0@@Z 10025480     qt-mt323:qt-mt323.dll
 0002:00001484       __imp_??H@YA?BVQString@@ABV0@PBD@Z 10025484     qt-mt323:qt-mt323.dll
 0002:00001488       __imp_??H@YA?BVQString@@ABV0@0@Z 10025488     qt-mt323:qt-mt323.dll
 0002:0000148c       __imp_??8@YA_NABVQString@@PBD@Z 1002548c     qt-mt323:qt-mt323.dll
 0002:00001490       __imp_??9@YA_NABVQString@@PBD@Z 10025490     qt-mt323:qt-mt323.dll
 0002:00001494       __imp_??8@YA_NABVQString@@0@Z 10025494     qt-mt323:qt-mt323.dll
 0002:00001498       __imp_??M@YA_NABVQString@@0@Z 10025498     qt-mt323:qt-mt323.dll
 0002:0000149c       __imp_??9@YA_NABVQString@@0@Z 1002549c     qt-mt323:qt-mt323.dll
 0002:000014a0       __imp_?endsWith@QString@@QBE_NABV1@@Z 100254a0     qt-mt323:qt-mt323.dll
 0002:000014a4       __imp_?startsWith@QString@@QBE_NABV1@@Z 100254a4     qt-mt323:qt-mt323.dll
 0002:000014a8       __imp_?latin1@QString@@QBEPBDXZ 100254a8     qt-mt323:qt-mt323.dll
 0002:000014ac       __imp_?fromAscii@QString@@SA?AV1@PBDH@Z 100254ac     qt-mt323:qt-mt323.dll
 0002:000014b0       __imp_?ascii@QString@@QBEPBDXZ 100254b0     qt-mt323:qt-mt323.dll
 0002:000014b4       __imp_??YQString@@QAEAAV0@PBD@Z 100254b4     qt-mt323:qt-mt323.dll
 0002:000014b8       __imp_??YQString@@QAEAAV0@ABV0@@Z 100254b8     qt-mt323:qt-mt323.dll
 0002:000014bc       __imp_?toInt@QString@@QBEHPA_NH@Z 100254bc     qt-mt323:qt-mt323.dll
 0002:000014c0       __imp_?remove@QString@@QAEAAV1@II@Z 100254c0     qt-mt323:qt-mt323.dll
 0002:000014c4       __imp_?stripWhiteSpace@QString@@QBE?AV1@XZ 100254c4     qt-mt323:qt-mt323.dll
 0002:000014c8       __imp_?left@QString@@QBE?AV1@I@Z 100254c8     qt-mt323:qt-mt323.dll
 0002:000014cc       __imp_?contains@QString@@QBEHABVQRegExp@@@Z 100254cc     qt-mt323:qt-mt323.dll
 0002:000014d0       __imp_?find@QString@@QBEHABV1@H_N@Z 100254d0     qt-mt323:qt-mt323.dll
 0002:000014d4       __imp_?sprintf@QString@@QAAAAV1@PBDZZ 100254d4     qt-mt323:qt-mt323.dll
 0002:000014d8       __imp_?arg@QString@@QBE?AV1@ABV1@H@Z 100254d8     qt-mt323:qt-mt323.dll
 0002:000014dc       __imp_?arg@QString@@QBE?AV1@IHH@Z 100254dc     qt-mt323:qt-mt323.dll
 0002:000014e0       __imp_?sizeHint@QDockWindow@@UBE?AVQSize@@XZ 100254e0     qt-mt323:qt-mt323.dll
 0002:000014e4       __imp_?arg@QString@@QBE?AV1@HHH@Z 100254e4     qt-mt323:qt-mt323.dll
 0002:000014e8       __imp_?number@QString@@SA?AV1@IH@Z 100254e8     qt-mt323:qt-mt323.dll
 0002:000014ec       __imp_?style@QApplication@@SAAAVQStyle@@XZ 100254ec     qt-mt323:qt-mt323.dll
 0002:000014f0       __imp_??0QLabel@@QAE@ABVQString@@PAVQWidget@@PBDI@Z 100254f0     qt-mt323:qt-mt323.dll
 0002:000014f4       __imp_??0?$QValueList@H@@QAE@XZ 100254f4     qt-mt323:qt-mt323.dll
 0002:000014f8       __imp_??1?$QValueList@H@@QAE@XZ 100254f8     qt-mt323:qt-mt323.dll
 0002:000014fc       __imp_?begin@?$QValueList@H@@QAE?AV?$QValueListIterator@H@@XZ 100254fc     qt-mt323:qt-mt323.dll
 0002:00001500       __imp_?append@?$QValueList@H@@QAE?AV?$QValueListIterator@H@@ABH@Z 10025500     qt-mt323:qt-mt323.dll
 0002:00001504       __imp_?detachInternal@?$QValueList@H@@AAEXXZ 10025504     qt-mt323:qt-mt323.dll
 0002:00001508       __imp_?split@QStringList@@SA?AV1@ABVQChar@@ABVQString@@_N@Z 10025508     qt-mt323:qt-mt323.dll
 0002:0000150c       __imp_??0QSettings@@QAE@W4Format@0@@Z 1002550c     qt-mt323:qt-mt323.dll
 0002:00001510       __imp_??1QSettings@@QAE@XZ 10025510     qt-mt323:qt-mt323.dll
 0002:00001514       __imp_?writeEntry@QSettings@@QAE_NABVQString@@0@Z 10025514     qt-mt323:qt-mt323.dll
 0002:00001518       __imp_?readEntry@QSettings@@QAE?AVQString@@ABV2@0PA_N@Z 10025518     qt-mt323:qt-mt323.dll
 0002:0000151c       __imp_?sizes@QSplitter@@QBE?AV?$QValueList@H@@XZ 1002551c     qt-mt323:qt-mt323.dll
 0002:00001520       __imp_?setSizes@QSplitter@@QAEXV?$QValueList@H@@@Z 10025520     qt-mt323:qt-mt323.dll
 0002:00001524       __imp_?columnWidth@QListView@@QBEHH@Z 10025524     qt-mt323:qt-mt323.dll
 0002:00001528       __imp_?columns@QListView@@QBEHXZ 10025528     qt-mt323:qt-mt323.dll
 0002:0000152c       __imp_?remove@QString@@QAEAAV1@D@Z 1002552c     qt-mt323:qt-mt323.dll
 0002:00001530       __imp_??YQString@@QAEAAV0@D@Z 10025530     qt-mt323:qt-mt323.dll
 0002:00001534       __imp_?clipboard@QApplication@@SAPAVQClipboard@@XZ 10025534     qt-mt323:qt-mt323.dll
 0002:00001538       __imp_?text@QClipboard@@QBE?AVQString@@XZ 10025538     qt-mt323:qt-mt323.dll
 0002:0000153c       __imp_?setText@QClipboard@@QAEXABVQString@@@Z 1002553c     qt-mt323:qt-mt323.dll
 0002:00001540       __imp_??4QFrame@@QAEAAV0@ABV0@@Z 10025540     qt-mt323:qt-mt323.dll
 0002:00001544       __imp_??0QListViewItem@@QAE@PAVQListView@@PAV0@@Z 10025544     qt-mt323:qt-mt323.dll
 0002:00001548       __imp_??0QListView@@QAE@ABV0@@Z 10025548     qt-mt323:qt-mt323.dll
 0002:0000154c       __imp_??0QTable@@QAE@PAVQWidget@@PBD@Z 1002554c     qt-mt323:qt-mt323.dll
 0002:00001550       __imp_??1QTable@@UAE@XZ    10025550     qt-mt323:qt-mt323.dll
 0002:00001554       __imp_?numSelections@QTable@@QBEHXZ 10025554     qt-mt323:qt-mt323.dll
 0002:00001558       __imp_?selection@QTable@@QBE?AVQTableSelection@@H@Z 10025558     qt-mt323:qt-mt323.dll
 0002:0000155c       __imp_??0QTable@@QAE@ABV0@@Z 1002555c     qt-mt323:qt-mt323.dll
 0002:00001560       __imp_??4QTable@@QAEAAV0@ABV0@@Z 10025560     qt-mt323:qt-mt323.dll
 0002:00001564       __imp_?activateNextCell@QTable@@MAEXXZ 10025564     qt-mt323:qt-mt323.dll
 0002:00001568       __imp_?addSelection@QTable@@UAEHABVQTableSelection@@@Z 10025568     qt-mt323:qt-mt323.dll
 0002:0000156c       __imp_?adjustColumn@QTable@@UAEXH@Z 1002556c     qt-mt323:qt-mt323.dll
 0002:00001570       __imp_?adjustRow@QTable@@UAEXH@Z 10025570     qt-mt323:qt-mt323.dll
 0002:00001574       __imp_?beginEdit@QTable@@MAEPAVQWidget@@HH_N@Z 10025574     qt-mt323:qt-mt323.dll
 0002:00001578       __imp_?cellGeometry@QTable@@UBE?AVQRect@@HH@Z 10025578     qt-mt323:qt-mt323.dll
 0002:0000157c       __imp_?cellRect@QTable@@UBE?AVQRect@@HH@Z 1002557c     qt-mt323:qt-mt323.dll
 0002:00001580       __imp_?cellWidget@QTable@@UBEPAVQWidget@@HH@Z 10025580     qt-mt323:qt-mt323.dll
 0002:00001584       __imp_?clearCell@QTable@@UAEXHH@Z 10025584     qt-mt323:qt-mt323.dll
 0002:00001588       __imp_?clearCellWidget@QTable@@UAEXHH@Z 10025588     qt-mt323:qt-mt323.dll
 0002:0000158c       __imp_?columnAt@QTable@@UBEHH@Z 1002558c     qt-mt323:qt-mt323.dll
 0002:00001590       __imp_?columnClicked@QTable@@MAEXH@Z 10025590     qt-mt323:qt-mt323.dll
 0002:00001594       __imp_?columnIndexChanged@QTable@@MAEXHHH@Z 10025594     qt-mt323:qt-mt323.dll
 0002:00001598       __imp_?columnPos@QTable@@UBEHH@Z 10025598     qt-mt323:qt-mt323.dll
 0002:0000159c       __imp_?columnWidth@QTable@@UBEHH@Z 1002559c     qt-mt323:qt-mt323.dll
 0002:000015a0       __imp_?columnWidthChanged@QTable@@MAEXH@Z 100255a0     qt-mt323:qt-mt323.dll
 0002:000015a4       __imp_?contentsContextMenuEvent@QTable@@MAEXPAVQContextMenuEvent@@@Z 100255a4     qt-mt323:qt-mt323.dll
 0002:000015a8       __imp_?contentsDragEnterEvent@QTable@@MAEXPAVQDragEnterEvent@@@Z 100255a8     qt-mt323:qt-mt323.dll
 0002:000015ac       __imp_?contentsDragLeaveEvent@QTable@@MAEXPAVQDragLeaveEvent@@@Z 100255ac     qt-mt323:qt-mt323.dll
 0002:000015b0       __imp_?contentsDragMoveEvent@QTable@@MAEXPAVQDragMoveEvent@@@Z 100255b0     qt-mt323:qt-mt323.dll
 0002:000015b4       __imp_?contentsDropEvent@QTable@@MAEXPAVQDropEvent@@@Z 100255b4     qt-mt323:qt-mt323.dll
 0002:000015b8       __imp_?contentsMouseDoubleClickEvent@QTable@@MAEXPAVQMouseEvent@@@Z 100255b8     qt-mt323:qt-mt323.dll
 0002:000015bc       __imp_?contentsMouseMoveEvent@QTable@@MAEXPAVQMouseEvent@@@Z 100255bc     qt-mt323:qt-mt323.dll
 0002:000015c0       __imp_?contentsMousePressEvent@QTable@@MAEXPAVQMouseEvent@@@Z 100255c0     qt-mt323:qt-mt323.dll
 0002:000015c4       __imp_?contentsMouseReleaseEvent@QTable@@MAEXPAVQMouseEvent@@@Z 100255c4     qt-mt323:qt-mt323.dll
 0002:000015c8       __imp_?createEditor@QTable@@MBEPAVQWidget@@HH_N@Z 100255c8     qt-mt323:qt-mt323.dll
 0002:000015cc       __imp_?currentSelection@QTable@@UBEHXZ 100255cc     qt-mt323:qt-mt323.dll
 0002:000015d0       __imp_?dragObject@QTable@@MAEPAVQDragObject@@XZ 100255d0     qt-mt323:qt-mt323.dll
 0002:000015d4       __imp_?drawContents@QTable@@EAEXPAVQPainter@@@Z 100255d4     qt-mt323:qt-mt323.dll
 0002:000015d8       __imp_?drawContents@QTable@@MAEXPAVQPainter@@HHHH@Z 100255d8     qt-mt323:qt-mt323.dll
 0002:000015dc       __imp_?editCell@QTable@@UAEXHH_N@Z 100255dc     qt-mt323:qt-mt323.dll
 0002:000015e0       __imp_?endEdit@QTable@@MAEXHH_N0@Z 100255e0     qt-mt323:qt-mt323.dll
 0002:000015e4       __imp_?eventFilter@QTable@@UAE_NPAVQObject@@PAVQEvent@@@Z 100255e4     qt-mt323:qt-mt323.dll
 0002:000015e8       __imp_?focusInEvent@QTable@@MAEXPAVQFocusEvent@@@Z 100255e8     qt-mt323:qt-mt323.dll
 0002:000015ec       __imp_?focusOutEvent@QTable@@MAEXPAVQFocusEvent@@@Z 100255ec     qt-mt323:qt-mt323.dll
 0002:000015f0       __imp_?hideColumn@QTable@@UAEXH@Z 100255f0     qt-mt323:qt-mt323.dll
 0002:000015f4       __imp_?hideRow@QTable@@UAEXH@Z 100255f4     qt-mt323:qt-mt323.dll
 0002:000015f8       __imp_?insertColumns@QTable@@UAEXHH@Z 100255f8     qt-mt323:qt-mt323.dll
 0002:000015fc       __imp_?insertRows@QTable@@UAEXHH@Z 100255fc     qt-mt323:qt-mt323.dll
 0002:00001600       __imp_?insertWidget@QTable@@MAEXHHPAVQWidget@@@Z 10025600     qt-mt323:qt-mt323.dll
 0002:00001604       __imp_?item@QTable@@UBEPAVQTableItem@@HH@Z 10025604     qt-mt323:qt-mt323.dll
 0002:00001608       __imp_?keyPressEvent@QTable@@MAEXPAVQKeyEvent@@@Z 10025608     qt-mt323:qt-mt323.dll
 0002:0000160c       __imp_?numCols@QTable@@UBEHXZ 1002560c     qt-mt323:qt-mt323.dll
 0002:00001610       __imp_?numRows@QTable@@UBEHXZ 10025610     qt-mt323:qt-mt323.dll
 0002:00001614       __imp_?paintCell@QTable@@UAEXPAVQPainter@@HHABVQRect@@_N@Z 10025614     qt-mt323:qt-mt323.dll
 0002:00001618       __imp_?paintCell@QTable@@UAEXPAVQPainter@@HHABVQRect@@_NABVQColorGroup@@@Z 10025618     qt-mt323:qt-mt323.dll
 0002:0000161c       __imp_?paintEmptyArea@QTable@@MAEXPAVQPainter@@HHHH@Z 1002561c     qt-mt323:qt-mt323.dll
 0002:00001620       __imp_?paintEvent@QTable@@MAEXPAVQPaintEvent@@@Z 10025620     qt-mt323:qt-mt323.dll
 0002:00001624       __imp_?paintFocus@QTable@@UAEXPAVQPainter@@ABVQRect@@@Z 10025624     qt-mt323:qt-mt323.dll
 0002:00001628       __imp_?pixmap@QTable@@UBE?AVQPixmap@@HH@Z 10025628     qt-mt323:qt-mt323.dll
 0002:0000162c       __imp_?removeColumn@QTable@@UAEXH@Z 1002562c     qt-mt323:qt-mt323.dll
 0002:00001630       __imp_?removeColumns@QTable@@UAEXABV?$QMemArray@H@@@Z 10025630     qt-mt323:qt-mt323.dll
 0002:00001634       __imp_?removeRow@QTable@@UAEXH@Z 10025634     qt-mt323:qt-mt323.dll
 0002:00001638       __imp_?removeRows@QTable@@UAEXABV?$QMemArray@H@@@Z 10025638     qt-mt323:qt-mt323.dll
 0002:0000163c       __imp_?removeSelection@QTable@@UAEXABVQTableSelection@@@Z 1002563c     qt-mt323:qt-mt323.dll
 0002:00001640       __imp_?removeSelection@QTable@@UAEXH@Z 10025640     qt-mt323:qt-mt323.dll
 0002:00001644       __imp_?resizeData@QTable@@MAEXH@Z 10025644     qt-mt323:qt-mt323.dll
 0002:00001648       __imp_?resizeEvent@QScrollView@@MAEXPAVQResizeEvent@@@Z 10025648     qt-mt323:qt-mt323.dll
 0002:0000164c       __imp_?rowAt@QTable@@UBEHH@Z 1002564c     qt-mt323:qt-mt323.dll
 0002:00001650       __imp_?rowHeight@QTable@@UBEHH@Z 10025650     qt-mt323:qt-mt323.dll
 0002:00001654       __imp_?rowHeightChanged@QTable@@MAEXH@Z 10025654     qt-mt323:qt-mt323.dll
 0002:00001658       __imp_?rowIndexChanged@QTable@@MAEXHHH@Z 10025658     qt-mt323:qt-mt323.dll
 0002:0000165c       __imp_?rowPos@QTable@@UBEHH@Z 1002565c     qt-mt323:qt-mt323.dll
 0002:00001660       __imp_?setCellContentFromEditor@QTable@@MAEXHH@Z 10025660     qt-mt323:qt-mt323.dll
 0002:00001664       __imp_?setCellWidget@QTable@@UAEXHHPAVQWidget@@@Z 10025664     qt-mt323:qt-mt323.dll
 0002:00001668       __imp_?setColumnMovingEnabled@QTable@@UAEX_N@Z 10025668     qt-mt323:qt-mt323.dll
 0002:0000166c       __imp_?setColumnReadOnly@QTable@@UAEXH_N@Z 1002566c     qt-mt323:qt-mt323.dll
 0002:00001670       __imp_?setColumnStretchable@QTable@@UAEXH_N@Z 10025670     qt-mt323:qt-mt323.dll
 0002:00001674       __imp_?setColumnWidth@QTable@@UAEXHH@Z 10025674     qt-mt323:qt-mt323.dll
 0002:00001678       __imp_?setCurrentCell@QTable@@UAEXHH@Z 10025678     qt-mt323:qt-mt323.dll
 0002:0000167c       __imp_?setDragEnabled@QTable@@UAEX_N@Z 1002567c     qt-mt323:qt-mt323.dll
 0002:00001680       __imp_?setEnabled@QTable@@UAEX_N@Z 10025680     qt-mt323:qt-mt323.dll
 0002:00001684       __imp_?setFocusStyle@QTable@@UAEXW4FocusStyle@1@@Z 10025684     qt-mt323:qt-mt323.dll
 0002:00001688       __imp_?setItem@QTable@@UAEXHHPAVQTableItem@@@Z 10025688     qt-mt323:qt-mt323.dll
 0002:0000168c       __imp_?setLeftMargin@QTable@@UAEXH@Z 1002568c     qt-mt323:qt-mt323.dll
 0002:00001690       __imp_?setNumCols@QTable@@UAEXH@Z 10025690     qt-mt323:qt-mt323.dll
 0002:00001694       __imp_?setNumRows@QTable@@UAEXH@Z 10025694     qt-mt323:qt-mt323.dll
 0002:00001698       __imp_?setPixmap@QTable@@UAEXHHABVQPixmap@@@Z 10025698     qt-mt323:qt-mt323.dll
 0002:0000169c       __imp_?setReadOnly@QTable@@UAEX_N@Z 1002569c     qt-mt323:qt-mt323.dll
 0002:000016a0       __imp_?setRowHeight@QTable@@UAEXHH@Z 100256a0     qt-mt323:qt-mt323.dll
 0002:000016a4       __imp_?setRowMovingEnabled@QTable@@UAEX_N@Z 100256a4     qt-mt323:qt-mt323.dll
 0002:000016a8       __imp_?setRowReadOnly@QTable@@UAEXH_N@Z 100256a8     qt-mt323:qt-mt323.dll
 0002:000016ac       __imp_?setRowStretchable@QTable@@UAEXH_N@Z 100256ac     qt-mt323:qt-mt323.dll
 0002:000016b0       __imp_?setSelectionMode@QTable@@UAEXW4SelectionMode@1@@Z 100256b0     qt-mt323:qt-mt323.dll
 0002:000016b4       __imp_?setShowGrid@QTable@@UAEX_N@Z 100256b4     qt-mt323:qt-mt323.dll
 0002:000016b8       __imp_?setSorting@QTable@@UAEX_N@Z 100256b8     qt-mt323:qt-mt323.dll
 0002:000016bc       __imp_?setText@QTable@@UAEXHHABVQString@@@Z 100256bc     qt-mt323:qt-mt323.dll
 0002:000016c0       __imp_?setTopMargin@QTable@@UAEXH@Z 100256c0     qt-mt323:qt-mt323.dll
 0002:000016c4       __imp_?showColumn@QTable@@UAEXH@Z 100256c4     qt-mt323:qt-mt323.dll
 0002:000016c8       __imp_?showEvent@QTable@@MAEXPAVQShowEvent@@@Z 100256c8     qt-mt323:qt-mt323.dll
 0002:000016cc       __imp_?showRow@QTable@@UAEXH@Z 100256cc     qt-mt323:qt-mt323.dll
 0002:000016d0       __imp_?sizeHint@QTable@@UBE?AVQSize@@XZ 100256d0     qt-mt323:qt-mt323.dll
 0002:000016d4       __imp_?sortColumn@QTable@@UAEXH_N0@Z 100256d4     qt-mt323:qt-mt323.dll
 0002:000016d8       __imp_?startDrag@QTable@@MAEXXZ 100256d8     qt-mt323:qt-mt323.dll
 0002:000016dc       __imp_?swapCells@QTable@@UAEXHHHH@Z 100256dc     qt-mt323:qt-mt323.dll
 0002:000016e0       __imp_?swapColumns@QTable@@UAEXHH_N@Z 100256e0     qt-mt323:qt-mt323.dll
 0002:000016e4       __imp_?swapRows@QTable@@UAEXHH_N@Z 100256e4     qt-mt323:qt-mt323.dll
 0002:000016e8       __imp_?takeItem@QTable@@UAEXPAVQTableItem@@@Z 100256e8     qt-mt323:qt-mt323.dll
 0002:000016ec       __imp_?text@QTable@@UBE?AVQString@@HH@Z 100256ec     qt-mt323:qt-mt323.dll
 0002:000016f0       __imp_?viewportResizeEvent@QTable@@MAEXPAVQResizeEvent@@@Z 100256f0     qt-mt323:qt-mt323.dll
 0002:000016f4       __imp_?windowActivationChange@QTable@@MAEX_N@Z 100256f4     qt-mt323:qt-mt323.dll
 0002:000016f8       __imp_?activate_signal_bool@QObject@@IAEXH_N@Z 100256f8     qt-mt323:qt-mt323.dll
 0002:000016fc       __imp_?staticMetaObject@QListView@@SAPAVQMetaObject@@XZ 100256fc     qt-mt323:qt-mt323.dll
 0002:00001700       __imp_?static_QUType_bool@@3UQUType_bool@@A 10025700     qt-mt323:qt-mt323.dll
 0002:00001704       __imp_?qt_cast@QTable@@UAEPAXPBD@Z 10025704     qt-mt323:qt-mt323.dll
 0002:00001708       __imp_?qt_invoke@QTable@@UAE_NHPAUQUObject@@@Z 10025708     qt-mt323:qt-mt323.dll
 0002:0000170c       __imp_?qt_emit@QTable@@UAE_NHPAUQUObject@@@Z 1002570c     qt-mt323:qt-mt323.dll
 0002:00001710       __imp_?qt_property@QTable@@UAE_NHHPAVQVariant@@@Z 10025710     qt-mt323:qt-mt323.dll
 0002:00001714       __imp_?staticMetaObject@QTable@@SAPAVQMetaObject@@XZ 10025714     qt-mt323:qt-mt323.dll
 0002:00001718       __imp_??1QString@@QAE@XZ   10025718     qt-mt323:qt-mt323.dll
 0002:0000171c       __imp_??0QString@@QAE@PBD@Z 1002571c     qt-mt323:qt-mt323.dll
 0002:00001720       __imp_??0QString@@QAE@ABV0@@Z 10025720     qt-mt323:qt-mt323.dll
 0002:00001724       __imp_??0QString@@QAE@XZ   10025724     qt-mt323:qt-mt323.dll
 0002:00001728       __imp_??M@YA_NABVQCString@@PBD@Z 10025728     qt-mt323:qt-mt323.dll
 0002:0000172c       __imp_??1QCString@@UAE@XZ  1002572c     qt-mt323:qt-mt323.dll
 0002:00001730       __imp_??0QCString@@QAE@H@Z 10025730     qt-mt323:qt-mt323.dll
 0002:00001734       __imp_?done@QDialog@@MAEXH@Z 10025734     qt-mt323:qt-mt323.dll
 0002:00001738       __imp_?qDebug@@YAXPBDZZ    10025738     qt-mt323:qt-mt323.dll
 0002:0000173c       \177qt-mt323_NULL_THUNK_DATA 1002573c     qt-mt323:qt-mt323.dll
 0002:00001740       ___xc_a                    10025740     MSVCRT:cinitexe.obj
 0002:00001798       ___xc_z                    10025798     MSVCRT:cinitexe.obj
 0002:0000179c       ___xi_a                    1002579c     MSVCRT:cinitexe.obj
 0002:000017a8       ___xi_z                    100257a8     MSVCRT:cinitexe.obj
 0002:000017b0       ??_C@_09DOGBNGMO@16?516?53?51?$AA@ 100257b0     alm_process.obj
 0002:000017bc       ??_C@_08OHPPFJCC@?5?7c?5None?$AA@ 100257bc     alm_process.obj
 0002:000017c8       ??_C@_0M@MHIBGGCN@?4?7c?5?$CD000000?$AA@ 100257c8     alm_process.obj
 0002:000017d4       ??_C@_0M@BMDODKEN@?$CL?7c?5?$CDFFFFFF?$AA@ 100257d4     alm_process.obj
 0002:000017e0       ??_C@_0BB@FHAPCDKO@?5?5?5?5?5?5?5?5?5?5?5?5?5?5?5?5?$AA@ 100257e0     alm_process.obj
 0002:000017f4       ??_C@_0BB@MGMPIHHJ@?5?4?4?4?4?4?4?4?4?5?5?5?5?5?5?5?$AA@ 100257f4     alm_process.obj
 0002:00001808       ??_C@_0BB@ILAANKMI@?5?5?4?4?$CL?$CL?$CL?$CL?4?4?4?4?5?5?5?5?$AA@ 10025808     alm_process.obj
 0002:0000181c       ??_C@_0BB@CLBDBFCC@?5?5?5?4?4?$CL?$CL?$CL?$CL?$CL?$CL?4?5?5?5?5?$AA@ 1002581c     alm_process.obj
 0002:00001830       ??_C@_0BB@MHBLIJND@?5?5?5?5?4?4?$CL?$CL?$CL?$CL?$CL?4?4?5?5?5?$AA@ 10025830     alm_process.obj
 0002:00001844       ??_C@_0BB@EFAPOMJD@?5?5?5?5?5?4?$CL?$CL?$CL?$CL?$CL?$CL?$CL?4?5?5?$AA@ 10025844     alm_process.obj
 0002:00001858       ??_C@_0BB@EPJBMBJJ@?5?5?5?5?5?4?$CL?$CL?$CL?$CL?$CL?$CL?$CL?4?4?5?$AA@ 10025858     alm_process.obj
 0002:0000186c       ??_C@_0BB@OGMMBMCF@?5?5?5?5?5?4?$CL?$CL?$CL?$CL?$CL?$CL?$CL?$CL?4?4?$AA@ 1002586c     alm_process.obj
 0002:00001880       ??_C@_09KDLGOOHH@16?516?54?51?$AA@ 10025880     alm_process.obj
 0002:0000188c       ??_C@_08CPDNICLA@?4?7c?5None?$AA@ 1002588c     alm_process.obj
 0002:00001898       ??_C@_0M@NOBBKPA@?$CL?7c?5?$CDFF0000?$AA@ 10025898     alm_process.obj
 0002:000018a4       ??_C@_0M@GOCNJDL@?$EA?7c?5?$CD000000?$AA@ 100258a4     alm_process.obj
 0002:000018b0       ??_C@_0BB@IENEBEAP@?4?4?4?4?$CL?$CL?4?4?4?4?4?$EA?4?4?4?4?$AA@ 100258b0     alm_process.obj
 0002:000018c4       ??_C@_0BB@MOKOMCHC@?4?4?4?4?4?$CL?$CL?4?4?4?4?$EA?$EA?4?4?4?$AA@ 100258c4     alm_process.obj
 0002:000018d8       ??_C@_0BB@HPCBFJBA@?4?4?4?4?4?4?$CL?$CL?4?4?4?4?4?$EA?4?4?$AA@ 100258d8     alm_process.obj
 0002:000018ec       ??_C@_0BB@HOKACJPM@?4?4?$EA?$EA?$EA?$EA?$CL?$CL?$EA?$EA?$EA?$EA?$EA?$EA?$EA?4?$AA@ 100258ec     alm_process.obj
 0002:00001900       ??_C@_0BB@NDGDCHPJ@?4?4?$EA?$EA?$EA?$EA?$EA?$CL?$CL?$EA?$EA?$EA?$EA?$EA?$EA?4?$AA@ 10025900     alm_process.obj
 0002:00001914       ??_C@_0BB@EEOBLABN@?4?4?4?4?4?4?4?$CL?$CL?4?4?4?4?$EA?4?4?$AA@ 10025914     alm_process.obj
 0002:00001928       ??_C@_0BB@CFCNFCAL@?4?4?4?4?4?4?4?4?$CL?$CL?4?$EA?$EA?4?4?4?$AA@ 10025928     alm_process.obj
 0002:0000193c       ??_C@_0BB@DCPJLCH@?4?4?4?4?4?4?4?4?$CL?$CL?4?$EA?4?4?4?4?$AA@ 1002593c     alm_process.obj
 0002:00001954       ??_SQWidget@@6BQObject@@@  10025954     alm_process.obj
 0002:00001b08       ??_SQWidget@@6BQPaintDevice@@@ 10025b08     alm_process.obj
 0002:00001b28       ??_C@_02GIPFHKNO@OK?$AA@   10025b28     alm_process.obj
 0002:00001b34       ??_SQAction@@6B@           10025b34     alm_process.obj
 0002:00001bc4       ??_SQDockWindow@@6BQObject@@@ 10025bc4     alm_process.obj
 0002:00001dd4       ??_SQDockWindow@@6BQPaintDevice@@@ 10025dd4     alm_process.obj
 0002:00001dfc       ??_SQToolBar@@6BQObject@@@ 10025dfc     alm_process.obj
 0002:00002018       ??_SQToolBar@@6BQPaintDevice@@@ 10026018     alm_process.obj
 0002:0000203c       ??_SQListViewItem@@6B@     1002603c     alm_process.obj
 0002:000020dc       ??_SQPushButton@@6BQObject@@@ 100260dc     alm_process.obj
 0002:000022cc       ??_SQPushButton@@6BQPaintDevice@@@ 100262cc     alm_process.obj
 0002:000022f4       ??_SQLineEdit@@6BQObject@@@ 100262f4     alm_process.obj
 0002:0000251c       ??_SQLineEdit@@6BQPaintDevice@@@ 1002651c     alm_process.obj
 0002:00002544       ??_SQTabWidget@@6BQObject@@@ 10026544     alm_process.obj
 0002:00002718       ??_SQTabWidget@@6BQPaintDevice@@@ 10026718     alm_process.obj
 0002:0000273c       ??_SQSpacerItem@@6B@       1002673c     alm_process.obj
 0002:00002784       ??_SQHBoxLayout@@6BQObject@@@ 10026784     alm_process.obj
 0002:000027ec       ??_SQHBoxLayout@@6BQLayoutItem@@@ 100267ec     alm_process.obj
 0002:00002834       ??_SQVBoxLayout@@6BQObject@@@ 10026834     alm_process.obj
 0002:0000289c       ??_SQVBoxLayout@@6BQLayoutItem@@@ 1002689c     alm_process.obj
 0002:000028e4       ??_SQLabel@@6BQObject@@@   100268e4     alm_process.obj
 0002:00002adc       ??_SQLabel@@6BQPaintDevice@@@ 10026adc     alm_process.obj
 0002:00002b04       ??_SCAlm_sys_select@@6BQObject@@@ 10026b04     alm_process.obj
 0002:00002cd8       ??_SCAlm_sys_select@@6BQPaintDevice@@@ 10026cd8     alm_process.obj
 0002:00002cfc       ??_7QDockWindowList@@6B@   10026cfc     alm_process.obj
 0002:00002d24       ??_SQPopupMenu@@6BQObject@@@ 10026d24     alm_process.obj
 0002:00002f04       ??_SQPopupMenu@@6BQPaintDevice@@@ 10026f04     alm_process.obj
 0002:00002f28       ??_SQPopupMenu@@6B@        10026f28     alm_process.obj
 0002:00002f4c       ??_7?$QPtrList@VQPopupMenu@@@@6B@ 10026f4c     alm_process.obj
 0002:00002f70       ??_7QPopupMenuList@@6B@    10026f70     alm_process.obj
 0002:00002f94       ??_SQGuardedPtrPrivate@@6B@ 10026f94     alm_process.obj
 0002:00002fe8       ??_7config_plugin_base@@6BQObject@@@ 10026fe8     alm_process.obj
 0002:000031c0       ??_7config_plugin_base@@6BQPaintDevice@@@ 100271c0     alm_process.obj
 0002:000031e0       ??_C@_0EB@GNDACMDJ@?$CC?5?9?5the?5author?5should?5have?5defin@ 100271e0     alm_process.obj
 0002:00003224       ??_C@_0CH@BDPDPLDP@This?5is?5the?5default?5?$CCAbout?$CC?5text@ 10027224     alm_process.obj
 0002:00003250       ??_7ProcessListView@@6BQObject@@@ 10027250     alm_process.obj
 0002:00003534       ??_7ProcessListView@@6BQPaintDevice@@@ 10027534     alm_process.obj
 0002:00003558       ??_7ProcessListViewItem@@6B@ 10027558     alm_process.obj
 0002:000035f4       ??_7alm_process@@6BQObject@@@ 100275f4     alm_process.obj
 0002:000037cc       ??_7alm_process@@6BQPaintDevice@@@ 100277cc     alm_process.obj
 0002:000037ec       ??_C@_00CNPNBAHC@?$AA@     100277ec     alm_process.obj
 0002:000037f0       ??_C@_08LPKBGJKD@?$CGProcess?$AA@ 100277f0     alm_process.obj
 0002:000037fc       ??_C@_07HFOCFOCN@?$CGGroups?$AA@ 100277fc     alm_process.obj
 0002:00003804       ??_C@_0BA@LJCCHABL@?1Processtoolbar?$AA@ 10027804     alm_process.obj
 0002:00003814       ??_C@_03CLCAEGCJ@new?$AA@  10027814     alm_process.obj
 0002:00003818       ??_C@_0N@NKBJBGFI@?$CGNew?5Process?$AA@ 10027818     alm_process.obj
 0002:00003828       ??_C@_07EJAINBEK@filenew?$AA@ 10027828     alm_process.obj
 0002:00003830       ??_C@_0M@LNCDACJN@New?5Process?$AA@ 10027830     alm_process.obj
 0002:0000383c       ??_C@_0O@LCGNKDDP@1newProcess?$CI?$CJ?$AA@ 1002783c     alm_process.obj
 0002:0000384c       ??_C@_0N@KCMOKDBB@2activated?$CI?$CJ?$AA@ 1002784c     alm_process.obj
 0002:0000385c       ??_C@_09KHIKJOBP@duplicate?$AA@ 1002785c     alm_process.obj
 0002:00003868       ??_C@_0BD@OJAAGCLD@?$CGDuplicate?5Process?$AA@ 10027868     alm_process.obj
 0002:0000387c       ??_C@_0BC@OPELBJJG@Duplicate?5Process?$AA@ 1002787c     alm_process.obj
 0002:00003890       ??_C@_0BE@BCIBCHEA@1duplicateProcess?$CI?$CJ?$AA@ 10027890     alm_process.obj
 0002:000038a4       ??_C@_08FJNLKCPH@template?$AA@ 100278a4     alm_process.obj
 0002:000038b0       ??_C@_0BN@BJCAMEGK@Copy?5Process?5Using?5?$CGTemplate?$AA@ 100278b0     alm_process.obj
 0002:000038d0       ??_C@_0BM@HEPBIJAG@Copy?5Process?5Using?5Template?$AA@ 100278d0     alm_process.obj
 0002:000038ec       ??_C@_0BM@JMIJJJKI@1copyProcessUsingTemplate?$CI?$CJ?$AA@ 100278ec     alm_process.obj
 0002:00003908       ??_C@_06FOBLBEIN@delete?$AA@ 10027908     alm_process.obj
 0002:00003910       ??_C@_0P@OIBFGOMC@Delete?5Process?$AA@ 10027910     alm_process.obj
 0002:00003920       ??_C@_0L@BPDPNFLB@filedelete?$AA@ 10027920     alm_process.obj
 0002:0000392c       ??_C@_0BB@JOLLKJBF@1deleteProcess?$CI?$CJ?$AA@ 1002792c     alm_process.obj
 0002:00003940       ??_C@_06LMEAOBLB@rename?$AA@ 10027940     alm_process.obj
 0002:00003948       ??_C@_0P@DIGMFBAF@Rename?5Process?$AA@ 10027948     alm_process.obj
 0002:00003958       ??_C@_0BD@MMOAOGPE@1startRenameProc?$CI?$CJ?$AA@ 10027958     alm_process.obj
 0002:0000396c       ??_C@_09HPFHHGGM@set?5Group?$AA@ 1002796c     alm_process.obj
 0002:00003978       ??_C@_09DAAKHFLM@Set?5Group?$AA@ 10027978     alm_process.obj
 0002:00003984       ??_C@_0BD@OHDNNPLB@1setProcessGroup?$CI?$CJ?$AA@ 10027984     alm_process.obj
 0002:00003998       ??_C@_0L@JFKABNAC@Clear?5Mask?$AA@ 10027998     alm_process.obj
 0002:000039a4       ??_C@_0L@FEGBDCAG@Clear?5mask?$AA@ 100279a4     alm_process.obj
 0002:000039b0       ??_C@_0N@HLPMFBAG@1clearMask?$CI?$CJ?$AA@ 100279b0     alm_process.obj
 0002:000039c0       ??_C@_08KEBPCDGL@set?5Mask?$AA@ 100279c0     alm_process.obj
 0002:000039cc       ??_C@_08CGOOKBMI@Set?5Mask?$AA@ 100279cc     alm_process.obj
 0002:000039d8       ??_C@_08OHCPIOMM@Set?5mask?$AA@ 100279d8     alm_process.obj
 0002:000039e4       ??_C@_0L@JIDFBFDN@1setMask?$CI?$CJ?$AA@ 100279e4     alm_process.obj
 0002:000039f0       ??_C@_0M@KOONPAKC@Latch?5?1?5Ack?$AA@ 100279f0     alm_process.obj
 0002:000039fc       ??_C@_0N@MJNHOEGH@?$CGLatch?5?1?5Ack?$AA@ 100279fc     alm_process.obj
 0002:00003a0c       ??_C@_0P@NCECDMPJ@1setLatchAck?$CI?$CJ?$AA@ 10027a0c     alm_process.obj
 0002:00003a1c       ??_C@_07LCCOIHHF@newGate?$AA@ 10027a1c     alm_process.obj
 0002:00003a24       ??_C@_0DC@JPDMEGPG@New?5?$CGGate?5?$CIlogic?5process?$CJ?5from?5s@ 10027a24     alm_process.obj
 0002:00003a58       ??_C@_0CK@JGKGCGHF@New?5logic?5process?5from?5selected?5@ 10027a58     alm_process.obj
 0002:00003a84       ??_C@_0L@DCGFOMOL@1newGate?$CI?$CJ?$AA@ 10027a84     alm_process.obj
 0002:00003a90       ??_C@_0BJ@BPMLIBBA@checkProcessContributors?$AA@ 10027a90     alm_process.obj
 0002:00003aac       ??_C@_0BN@MPJIHPNI@?$CGCheck?5Process?5contributions?$AA@ 10027aac     alm_process.obj
 0002:00003acc       ??_C@_0BM@DDNABMF@Check?5Process?5contributions?$AA@ 10027acc     alm_process.obj
 0002:00003ae8       ??_C@_0BM@BEDKJMKI@1checkProcessContributors?$CI?$CJ?$AA@ 10027ae8     alm_process.obj
 0002:00003b04       ??_C@_08LDJMEMHO@newGroup?$AA@ 10027b04     alm_process.obj
 0002:00003b10       ??_C@_0L@IKPBOEAJ@?$CGNew?5Group?$AA@ 10027b10     alm_process.obj
 0002:00003b1c       ??_C@_09GMNFHIAH@New?5Group?$AA@ 10027b1c     alm_process.obj
 0002:00003b28       ??_C@_0M@CDBAGPAE@1newGroup?$CI?$CJ?$AA@ 10027b28     alm_process.obj
 0002:00003b34       ??_C@_0M@PEIBNGOO@renameGroup?$AA@ 10027b34     alm_process.obj
 0002:00003b40       ??_C@_0O@ILNHLCNH@?$CGRename?5Group?$AA@ 10027b40     alm_process.obj
 0002:00003b50       ??_C@_0N@GALOLOPM@Rename?5Group?$AA@ 10027b50     alm_process.obj
 0002:00003b60       ??_C@_0P@KOGBNFKI@1renameGroup?$CI?$CJ?$AA@ 10027b60     alm_process.obj
 0002:00003b70       ??_C@_0M@CNEJDFMD@deleteGroup?$AA@ 10027b70     alm_process.obj
 0002:00003b7c       ??_C@_0O@MONBCGEB@?$CGDelete?5Group?$AA@ 10027b7c     alm_process.obj
 0002:00003b8c       ??_C@_0N@CFLICKGK@Delete?5Group?$AA@ 10027b8c     alm_process.obj
 0002:00003b9c       ??_C@_0P@LHEIOFEN@1deleteGroup?$CI?$CJ?$AA@ 10027b9c     alm_process.obj
 0002:00003bac       ??_C@_0N@CLADDHOI@?1procBrowser?$AA@ 10027bac     alm_process.obj
 0002:00003bbc       ??_C@_0N@OAECLGMI@Process?5List?$AA@ 10027bbc     alm_process.obj
 0002:00003bcc       ??_C@_0N@CDKMAAAD@SystemSelect?$AA@ 10027bcc     alm_process.obj
 0002:00003bdc       ??_C@_06IBDJIBGI@Filter?$AA@ 10027bdc     alm_process.obj
 0002:00003be4       ??_C@_0BP@KOKPNIGE@1filterChange?$CIconst?5QString?5?$CG?$CJ?$AA@ 10027be4     alm_process.obj
 0002:00003c04       ??_C@_0BO@JONBIMPD@2textChanged?$CIconst?5QString?5?$CG?$CJ?$AA@ 10027c04     alm_process.obj
 0002:00003c24       ??_C@_0BF@BGBIPDBD@Check?5Process?5Filter?$AA@ 10027c24     alm_process.obj
 0002:00003c3c       ??_C@_0L@OELOHDKG@2clicked?$CI?$CJ?$AA@ 10027c3c     alm_process.obj
 0002:00003c48       ??_C@_0N@GLLBIEJ@Clear?5Filter?$AA@ 10027c48     alm_process.obj
 0002:00003c58       ??_C@_0P@LGOHPIPB@1clearFilter?$CI?$CJ?$AA@ 10027c58     alm_process.obj
 0002:00003c68       ??_C@_04FABLJDN@Name?$AA@  10027c68     alm_process.obj
 0002:00003c70       ??_C@_05MBDCODDP@Group?$AA@ 10027c70     alm_process.obj
 0002:00003c78       ??_C@_04HOKIGJEB@Rule?$AA@ 10027c78     alm_process.obj
 0002:00003c80       ??_C@_05HNPPNPM@Valid?$AA@ 10027c80     alm_process.obj
 0002:00003c88       ??_C@_08LAIGBKAI@ProcList?$AA@ 10027c88     alm_process.obj
 0002:00003c94       ??_C@_0BH@JFMCCFME@Home?1Alarms?1Processes?1?$AA@ 10027c94     alm_process.obj
 0002:00003cac       ??_C@_0BP@KFJPMMLE@1selectSystem?$CIconst?5QString?5?$CG?$CJ?$AA@ 10027cac     alm_process.obj
 0002:00003ccc       ??_C@_0BN@DDAIKEMB@2sysChanged?$CIconst?5QString?5?$CG?$CJ?$AA@ 10027ccc     alm_process.obj
 0002:00003cec       ??_C@_0CL@OEEOKDOP@1sysCommand?$CIconst?5QString?$CG?0const@ 10027cec     alm_process.obj
 0002:00003d18       ??_C@_0CI@OBEELDED@2command?$CIconst?5QString?$CG?0const?5QS@ 10027d18     alm_process.obj
 0002:00003d40       ??_C@_0BB@JCJNHAIG@1selectProcess?$CI?$CJ?$AA@ 10027d40     alm_process.obj
 0002:00003d54       ??_C@_0BG@PJBIDJAL@2selectionChanged?5?$CI?5?$CJ?$AA@ 10027d54     alm_process.obj
 0002:00003d6c       ??_C@_0BN@MGBHIHMO@1startRename?$CIQListViewItem?$CK?$CJ?$AA@ 10027d6c     alm_process.obj
 0002:00003d8c       ??_C@_0BP@NMMLAJFB@2doubleClicked?$CIQListViewItem?$CK?$CJ?$AA@ 10027d8c     alm_process.obj
 0002:00003dac       ??_C@_0DD@MKHHBBMJ@1renameProcess?$CIQListViewItem?$CK?0in@ 10027dac     alm_process.obj
 0002:00003de0       ??_C@_0DC@BDFAIPOL@2itemRenamed?$CIQListViewItem?$CK?0?5int@ 10027de0     alm_process.obj
 0002:00003e14       ??_C@_0DM@DHGDAJI@1procListContextMenu?$CIQListViewIt@ 10027e14     alm_process.obj
 0002:00003e50       ??_C@_0DN@PPNHBGND@2contextMenuRequested?5?$CIQListView@ 10027e50     alm_process.obj
 0002:00003e90       ??_C@_0O@LNLOBKPN@1changeMask?$CI?$CJ?$AA@ 10027e90     alm_process.obj
 0002:00003ea0       ??_C@_0BC@MNPMPCIL@1addMultiInputs?$CI?$CJ?$AA@ 10027ea0     alm_process.obj
 0002:00003eb4       ??_C@_0BD@FNHANIGE@1addSingleInputs?$CI?$CJ?$AA@ 10027eb4     alm_process.obj
 0002:00003ec8       ??_C@_0BL@DGNHFPNJ@1updateProcList?$CIcProcess?$CK?$CJ?$AA@ 10027ec8     alm_process.obj
 0002:00003ee4       ??_C@_0BH@JBEBKACO@2updateProc?$CIcProcess?$CK?$CJ?$AA@ 10027ee4     alm_process.obj
 0002:00003efc       ??_C@_0N@LMCHKLFE@1markDirty?$CI?$CJ?$AA@ 10027efc     alm_process.obj
 0002:00003f0c       ??_C@_0BA@LHBDKNBL@2itemsChanged?$CI?$CJ?$AA@ 10027f0c     alm_process.obj
 0002:00003f1c       ??_C@_0BI@FGCBACNP@1selectProcess?$CIQString?$CJ?$AA@ 10027f1c     alm_process.obj
 0002:00003f34       ??_C@_0BE@GKHJAMLL@2navToProc?$CIQString?$CJ?$AA@ 10027f34     alm_process.obj
 0002:00003f48       ??_C@_0BO@FHNPPLIC@1navToOutput?$CIQString?0QString?$CJ?$AA@ 10027f48     alm_process.obj
 0002:00003f68       ??_C@_0BO@BDHONOJK@2navToOutput?$CIQString?0QString?$CJ?$AA@ 10027f68     alm_process.obj
 0002:00003f88       ??_C@_0CD@LBLGFIKA@1navToAck?$CIQString?0QString?0QStrin@ 10027f88     alm_process.obj
 0002:00003fac       ??_C@_0CD@DKGFGGLJ@2navToAck?$CIQString?0QString?0QStrin@ 10027fac     alm_process.obj
 0002:00003fd0       ??_C@_06BNCCALCL@unlock?$AA@ 10027fd0     alm_process.obj
 0002:00003fd8       ??_C@_08HNIAHLMM@download?$AA@ 10027fd8     alm_process.obj
 0002:00003fe4       ??_C@_0BD@DDFIPJEJ@File?5downloaded?5?9?5?$AA@ 10027fe4     alm_process.obj
 0002:00003ff8       ??_C@_07MPPKIBJA@Error?3?6?$AA@ 10027ff8     alm_process.obj
 0002:00004000       ??_C@_05NAOIJFC@Error?$AA@ 10028000     alm_process.obj
 0002:00004008       ??_C@_0N@LEBPCLIG@proc_def?4cfg?$AA@ 10028008     alm_process.obj
 0002:00004018       ??_C@_01KMDKNFGN@?1?$AA@   10028018     alm_process.obj
 0002:0000401c       ??_C@_0O@MIFBLPDN@config?1alarms?$AA@ 1002801c     alm_process.obj
 0002:0000402c       ??_C@_03GJCOJFLC@?4?6?6?$AA@ 1002802c     alm_process.obj
 0002:00004030       ??_C@_0BM@CGOIHJMM@Could?5not?5Create?5directory?6?$AA@ 10028030     alm_process.obj
 0002:0000404c       ??_C@_0BB@IMCDCEGC@Alarms?1Processes?$AA@ 1002804c     alm_process.obj
 0002:00004060       ??_C@_07GEICGNKI@?1inputs?$AA@ 10028060     alm_process.obj
 0002:00004068       ??_C@_08JBEPPOLH@?1outputs?$AA@ 10028068     alm_process.obj
 0002:00004074       ??_C@_04MKMCLCOO@lock?$AA@ 10028074     alm_process.obj
 0002:0000407c       ??_C@_0CC@OAGIAEAC@?6File?5will?5be?5available?5read?5onl@ 1002807c     alm_process.obj
 0002:000040a0       ??_C@_03NLJIHOMM@?5?9?5?$AA@ 100280a0     alm_process.obj
 0002:000040a4       ??_C@_06JGFHLLHI@Lock?3?5?$AA@ 100280a4     alm_process.obj
 0002:000040ac       ??_C@_04LADJNOK@Lock?$AA@  100280ac     alm_process.obj
 0002:000040b4       ??_C@_06KAOCKAGB@upload?$AA@ 100280b4     alm_process.obj
 0002:000040bc       ??_C@_05CCAMFJOL@clean?$AA@ 100280bc     alm_process.obj
 0002:000040c4       ??_C@_03DAPAKLGM@dir?$AA@  100280c4     alm_process.obj
 0002:000040c8       ??_C@_04EMJEACDL@?5on?5?$AA@ 100280c8     alm_process.obj
 0002:000040d0       ??_C@_09EGFBFPH@Response?5?$AA@ 100280d0     alm_process.obj
 0002:000040dc       ??_C@_02PEIOPPKO@?2S?$AA@  100280dc     alm_process.obj
 0002:000040e0       ??_C@_0L@CIKGEHEG@uploadFile?$AA@ 100280e0     alm_process.obj
 0002:000040ec       ??_C@_0BC@IKCJJGKO@Loading?5File?5?8?$CFs?8?$AA@ 100280ec     alm_process.obj
 0002:00004100       ??_C@_0BJ@LIHFCLLM@File?5?8?$CFs?8?5does?5not?5exist?$AA@ 10028100     alm_process.obj
 0002:0000411c       ??_C@_01OHGJGJJP@?$FL?$AA@ 1002811c     alm_process.obj
 0002:00004120       ??_C@_01LBDDMOBJ@?$FN?$AA@ 10028120     alm_process.obj
 0002:00004124       ??_C@_0BC@PFKPCFNA@Load?5took?5?$CFd?5?$CI?$CFd?$CJ?$AA@ 10028124     alm_process.obj
 0002:00004138       ??_C@_0P@DONMDJCG@Done?5processes?$AA@ 10028138     alm_process.obj
 0002:00004148       ??_C@_0BA@IIJGOFHP@CheckProcParams?$AA@ 10028148     alm_process.obj
 0002:00004158       ??_C@_01IHBHIGKO@?0?$AA@   10028158     alm_process.obj
 0002:0000415c       ??_C@_04LOAJBDKD@true?$AA@ 1002815c     alm_process.obj
 0002:00004164       ??_C@_0DK@JGPMEDKF@?$DM?$DMfiltered?5to?5contain?5processes?5@ 10028164     alm_process.obj
 0002:000041a0       ??_C@_0EI@JMGLIDIG@?$DM?$DMfiltered?5to?5contain?5?$CF1?$CF2proces@ 100281a0     alm_process.obj
 0002:000041e8       ??_C@_06LMKDOJKC@INPUT?5?$AA@ 100281e8     alm_process.obj
 0002:000041f0       ??_C@_0BB@DKKDBPNH@OR?5?$CIand?5others?$CJ?5?$AA@ 100281f0     alm_process.obj
 0002:00004204       ??_C@_0BI@JILPLIJE@?$CF1?0?$CF2?0?$CF3?0?$CF4?0?$CF5?0?$CF6?0?$CF7?0?$CF8?$AA@ 10028204     alm_process.obj
 0002:0000421c       ??_C@_05LAPONLG@false?$AA@ 1002821c     alm_process.obj
 0002:00004224       ??_C@_0BA@JJNKKKK@selectProcess?$CI?$CJ?$AA@ 10028224     alm_process.obj
 0002:00004234       ??_C@_0BD@NDLOCEBI@selectProcess?$CIlvi?$CJ?$AA@ 10028234     alm_process.obj
 0002:00004248       ??_C@_0BD@PJKDBEGH@Process?5unknown?5?9?5?$AA@ 10028248     alm_process.obj
 0002:0000425c       ??_C@_0CH@LJGBFMOH@Process?5does?5not?5match?5listbox?5n@ 1002825c     alm_process.obj
 0002:00004284       ??_C@_0CD@FHEDPDHI@addSingleInputs?5?9?5no?5item?5select@ 10028284     alm_process.obj
 0002:000042a8       ??_C@_02JODFHDIE@?$FN?6?$AA@ 100282a8     alm_process.obj
 0002:000042ac       ??_C@_01EEMJAFIK@?6?$AA@   100282ac     alm_process.obj
 0002:000042b0       ??_C@_0DE@PHFGCFLH@alm_process?3?3saveProcesses?5?9?5Fai@ 100282b0     alm_process.obj
 0002:000042e4       ??_C@_0DC@CMEBAJGG@alm_process?3?3saveProcesses?$CIQStri@ 100282e4     alm_process.obj
 0002:00004318       ??_C@_0M@GABNMAMI@New_Proc_?$CFd?$AA@ 10028318     alm_process.obj
 0002:00004324       ??_C@_0BB@GJLJOPMM@Enter?5new?5Group?3?$AA@ 10028324     alm_process.obj
 0002:00004338       ??_C@_0BH@HLILEENB@Select?5Group?5to?5rename?$AA@ 10028338     alm_process.obj
 0002:00004350       ??_C@_0CN@JCGAOAAK@?$CF1?5already?5exists?0?5so?5?$CF2?5will?5no@ 10028350     alm_process.obj
 0002:00004380       ??_C@_0EB@OGAHIMLP@Select?5Group?5to?5delete?5?6Note?5tha@ 10028380     alm_process.obj
 0002:000043c8       ??_7?$QPtrList@VQListViewItem@@@@6B@ 100283c8     alm_process.obj
 0002:000043e8       ??_C@_05NGADHBOM@copy_?$AA@ 100283e8     alm_process.obj
 0002:000043f0       ??_C@_04JBKCEBKE@_of_?$AA@ 100283f0     alm_process.obj
 0002:000043f8       ??_C@_0O@BBDBGNLN@copy_?$CFd_of_?$CFs?$AA@ 100283f8     alm_process.obj
 0002:0000440c       ??_7?$QPtrList@VcProcess@@@@6B@ 1002840c     alm_process.obj
 0002:0000442c       ??_C@_0P@GANAFAFM@delete?5Process?$AA@ 1002842c     alm_process.obj
 0002:00004440       ??_C@_0FB@KENIIKMP@?5is?5used?5by?5other?5processes?0?5the@ 10028440     alm_process.obj
 0002:00004494       ??_C@_08JNCEHING@Process?5?$AA@ 10028494     alm_process.obj
 0002:000044a0       ??_C@_0M@KHNBGJNJ@New_Proc_?$CF1?$AA@ 100284a0     alm_process.obj
 0002:000044ac       ??_C@_01IDAFKMJL@_?$AA@    100284ac     alm_process.obj
 0002:000044b0       ??_C@_07DFOMLOAJ@Overall?$AA@ 100284b0     alm_process.obj
 0002:000044b8       ??_C@_05MFIFJEGB@?$CF1_?$CF2?$AA@ 100284b8     alm_process.obj
 0002:000044c0       ??_C@_07OHPALPHI@Rule?$DN?$CF1?$AA@ 100284c0     alm_process.obj
 0002:000044c8       ??_C@_02PDPFNDMG@OR?$AA@   100284c8     alm_process.obj
 0002:000044cc       ??_C@_09HANKKAH@Inputs?$DN?$CF2?$AA@ 100284cc     alm_process.obj
 0002:000044d8       ??_C@_05CFEJGMAI@dirty?$AA@ 100284d8     alm_process.obj
 0002:000044e0       ??_C@_0BC@KDFFAOOB@?5does?5not?5exist?4?6?$AA@ 100284e0     alm_process.obj
 0002:000044f4       ??_C@_0BG@PPJMIOPN@Process?5Configuration?$AA@ 100284f4     alm_process.obj
 0002:0000450c       ??_C@_0DN@HFHIEKMJ@alm_process?3?3selectProcess?5We?5ne@ 1002850c     alm_process.obj
 0002:0000454c       ??_C@_01ICJEACDI@?$DL?$AA@ 1002854c     alm_process.obj
 0002:00004550       ??_C@_08NCKPMOJE@navigate?$AA@ 10028550     alm_process.obj
 0002:0000455c       ??_C@_0BJ@KIDLFDNB@?5is?5an?5input?5to?5updated?$DP?$AA@ 1002855c     alm_process.obj
 0002:00004578       ??_C@_0CA@LIDGNDCF@Do?5you?5want?5the?5processes?5that?5?$AA@ 10028578     alm_process.obj
 0002:00004598       ??_C@_0BE@JHGPLILP@Update?5dependencies?$AA@ 10028598     alm_process.obj
 0002:000045ac       ??_C@_0CB@OOJBAIIA@Select?5Group?5to?5add?5processes?5to@ 100285ac     alm_process.obj
 0002:000045d0       ??_C@_0BD@IEBIJKLG@Re?9group?5Processes?$AA@ 100285d0     alm_process.obj
 0002:000045e4       ??_C@_0BN@ECJGNIGM@Failed?5to?5load?5settings?5for?5?$AA@ 100285e4     alm_process.obj
 0002:00004604       ??_C@_0DC@CJKPNBGB@?$DMnobr?$DO?$DMh3?$DOAlarm?5Process?5configur@ 10028604     alm_process.obj
 0002:00004638       ??_C@_0CN@IJPOCBJI@?$DMp?$DOWritten?5by?5Mark?5Baldry?0?5Richa@ 10028638     alm_process.obj
 0002:00004668       ??_C@_0BK@JBBNBDIM@?$DMp?$DOProcess?5count?5?$DN?5?$CF1?$DM?1p?$DO?$AA@ 10028668     alm_process.obj
 0002:00004684       ??_C@_0CB@ECGBNAEE@Selected?5the?5following?5system?5?9?5@ 10028684     alm_process.obj
 0002:000046a8       ??_C@_0N@EHHLDFOB@checkoutFile?$AA@ 100286a8     alm_process.obj
 0002:000046b8       ??_C@_0BA@GNHMHBBC@syncDirDownload?$AA@ 100286b8     alm_process.obj
 0002:000046c8       ??_C@_09LBJJOLLJ@Not?5Valid?$AA@ 100286c8     alm_process.obj
 0002:000046d4       ??_C@_07GFDMEDFB@darkRed?$AA@ 100286d4     alm_process.obj
 0002:000046dc       ??_C@_06ENJNJKEL@yellow?$AA@ 100286dc     alm_process.obj
 0002:000046e4       ??_C@_03FAAAOPJM@red?$AA@  100286e4     alm_process.obj
 0002:000046e8       ??_C@_0BE@JONHPENG@map?1set?$DMT?$DO?5too?5long?$AA@ 100286e8     alm_process.obj
 0002:00004700       ??_7cAcqFileData@@6B@      10028700     cAcqFileData.obj
 0002:00004704       ??_C@_07LKBEKAPA@?$FLInput_?$AA@ 10028704     cAcqFileData.obj
 0002:0000470c       ??_C@_08IJKOBABM@?$FLSystem?$FN?$AA@ 1002870c     cAcqFileData.obj
 0002:00004718       ??_C@_01NEMOKFLO@?$DN?$AA@ 10028718     cAcqFileData.obj
 0002:0000471c       ??_C@_0L@FGNBINDG@ConfigTool?$AA@ 1002871c     cAcqFileData.obj
 0002:00004728       ??_C@_06NHPJKFDC@Module?$AA@ 10028728     cAcqFileData.obj
 0002:00004734       ??_7CheckContDialog@@6BQObject@@@ 10028734     checkContDialogImpl.obj
 0002:00004900       ??_7CheckContDialog@@6BQPaintDevice@@@ 10028900     checkContDialogImpl.obj
 0002:00004920       ??_C@_0DA@HMABIMNA@At?5least?5one?5of?5INPUT?5and?5OR?5has@ 10028920     checkContDialogImpl.obj
 0002:00004950       ??_C@_0CJ@LPKPHEBK@Min?5has?5to?5be?5smaller?5or?5equal?5t@ 10028950     checkContDialogImpl.obj
 0002:00004980       ??_C@_0EA@DDGHDOGI@At?5least?5one?5of?5the?5input?5filter@ 10028980     checkContDialogImpl.obj
 0002:000049c4       ??_SQDoubleValidator@@6B@  100289c4     cProc_dialog.obj
 0002:00004a24       ??_7cProc_dialog@@6BQObject@@@ 10028a24     cProc_dialog.obj
 0002:00004bdc       ??_7cProc_dialog@@6BQPaintDevice@@@ 10028bdc     cProc_dialog.obj
 0002:00004c00       ??_7ContributorListBoxItem@@6B@ 10028c00     cProc_dialog.obj
 0002:00004c20       ??_C@_07MNGBFJEN@Process?$AA@ 10028c20     cProc_dialog.obj
 0002:00004c28       ??_C@_07LGFKBKFE@Outputs?$AA@ 10028c28     cProc_dialog.obj
 0002:00004c30       ??_C@_06MJDIICIN@Editor?$AA@ 10028c30     cProc_dialog.obj
 0002:00004c38       ??_C@_0O@KMDMJMFD@OutputModules?$AA@ 10028c38     cProc_dialog.obj
 0002:00004c48       ??_C@_08CGIOBMAK@Splitter?$AA@ 10028c48     cProc_dialog.obj
 0002:00004c54       ??_C@_0BP@PPHEOGJF@1changeGroup?$CI?5const?5QString?5?$CG?$CJ?$AA@ 10028c54     cProc_dialog.obj
 0002:00004c74       ??_C@_0BN@KGNOJIAM@2activated?$CI?5const?5QString?5?$CG?$CJ?$AA@ 10028c74     cProc_dialog.obj
 0002:00004c94       ??_C@_0CC@DOKFEGLN@1changeFunction?$CI?5const?5QString?5?$CG@ 10028c94     cProc_dialog.obj
 0002:00004cb8       ??_C@_0CE@GMOKJLKI@1inputBlockChange?$CI?5const?5QString@ 10028cb8     cProc_dialog.obj
 0002:00004cdc       ??_C@_0CD@ODDJLMKG@1inputSlotChange?$CI?5const?5QString?5@ 10028cdc     cProc_dialog.obj
 0002:00004d00       ??_C@_0P@PEAEIDFL@1editAcqSlot?$CI?$CJ?$AA@ 10028d00     cProc_dialog.obj
 0002:00004d10       ??_C@_0CA@EEBMNIG@1enableTruthDeleteCol?$CIint?0?5int?$CJ?$AA@ 10028d10     cProc_dialog.obj
 0002:00004d30       ??_C@_0BK@KAFPHPPN@2currentChanged?$CIint?0?5int?$CJ?$AA@ 10028d30     cProc_dialog.obj
 0002:00004d4c       ??_C@_0BC@DAGBINKH@1addTruthColumn?$CI?$CJ?$AA@ 10028d4c     cProc_dialog.obj
 0002:00004d60       ??_C@_0BF@CKDGBOCD@1deleteTruthColumn?$CI?$CJ?$AA@ 10028d60     cProc_dialog.obj
 0002:00004d78       ??_C@_0BP@JHOEKBFE@1changeHoldoff?$CIconst?5QString?$CG?$CJ?$AA@ 10028d78     cProc_dialog.obj
 0002:00004d98       ??_C@_0BN@HELOKIBG@2textChanged?$CIconst?5QString?$CG?$CJ?$AA@ 10028d98     cProc_dialog.obj
 0002:00004db8       ??_C@_0BC@CBBIDEJG@1enableNavigate?$CI?$CJ?$AA@ 10028db8     cProc_dialog.obj
 0002:00004dcc       ??_C@_0BE@BLJBKCLJ@2selectionChanged?$CI?$CJ?$AA@ 10028dcc     cProc_dialog.obj
 0002:00004de0       ??_C@_0BE@FLLGEHBM@1navContributesTo?$CI?$CJ?$AA@ 10028de0     cProc_dialog.obj
 0002:00004df4       ??_C@_0BD@LPMMPJMP@1navOutputModule?$CI?$CJ?$AA@ 10028df4     cProc_dialog.obj
 0002:00004e08       ??_C@_0P@PJIGAHMH@1itemChanged?$CI?$CJ?$AA@ 10028e08     cProc_dialog.obj
 0002:00004e18       ??_C@_0M@LPGBGFJN@2clicked?5?$CI?$CJ?$AA@ 10028e18     cProc_dialog.obj
 0002:00004e24       ??_C@_0BA@INEKJJEF@2textChanged?5?$CI?$CJ?$AA@ 10028e24     cProc_dialog.obj
 0002:00004e34       ??_C@_0BG@PKKIMHDC@1itemChanged?$CIint?0int?$CJ?$AA@ 10028e34     cProc_dialog.obj
 0002:00004e4c       ??_C@_0BI@KMCDOINC@2valueChanged?5?$CIint?0int?$CJ?$AA@ 10028e4c     cProc_dialog.obj
 0002:00004e64       ??_C@_0BC@ELMOLHPA@1itemChanged?$CIint?$CJ?$AA@ 10028e64     cProc_dialog.obj
 0002:00004e78       ??_C@_0O@GBIKBCJG@2clicked?$CIint?$CJ?$AA@ 10028e78     cProc_dialog.obj
 0002:00004e88       ??_C@_0CA@PJAFEACO@1startTimeChanged?$CIconst?5QTime?$CG?$CJ?$AA@ 10028e88     cProc_dialog.obj
 0002:00004ea8       ??_C@_0BM@FDJFLCNI@2valueChanged?$CIconst?5QTime?$CG?$CJ?$AA@ 10028ea8     cProc_dialog.obj
 0002:00004ec4       ??_C@_0BO@POHJAMO@1endTimeChanged?$CIconst?5QTime?$CG?$CJ?$AA@ 10028ec4     cProc_dialog.obj
 0002:00004ee4       ??_C@_05OEOKGKGJ@?$DM?1h1?$DO?$AA@ 10028ee4     cProc_dialog.obj
 0002:00004eec       ??_C@_0BG@PNENNKKG@?$DMh1?$DOAlarms?5Process?5?9?5?$AA@ 10028eec     cProc_dialog.obj
 0002:00004f04       ??_C@_01DNKMNLPK@?$HM?$AA@ 10028f04     cProc_dialog.obj
 0002:00004f08       ??_C@_01HIHLOKLC@1?$AA@    10028f08     cProc_dialog.obj
 0002:00004f0c       ??_C@_01GBGANLPD@0?$AA@    10028f0c     cProc_dialog.obj
 0002:00004f10       ??_C@_01NBENCBCI@?$CK?$AA@ 10028f10     cProc_dialog.obj
 0002:00004f14       ??_C@_05FACKIIFD@day?$CFd?$AA@ 10028f14     cProc_dialog.obj
 0002:00004f1c       ??_C@_05MBCLKLL@hh?3mm?$AA@ 10028f1c     cProc_dialog.obj
 0002:00004f24       ??_C@_0N@GGGHIOIL@Unknown?5Slot?$AA@ 10028f24     cProc_dialog.obj
 0002:00004f34       ??_C@_0O@CKEKOOLH@Unknown?5block?$AA@ 10028f34     cProc_dialog.obj
 0002:00004f44       ??_C@_07GHLHIMDE@Slot?5?$CFd?$AA@ 10028f44     cProc_dialog.obj
 0002:00004f4c       ??_C@_01OGPIMHDM@?$DP?$AA@ 10028f4c     cProc_dialog.obj
 0002:00004f50       ??_C@_01CLKCMJKC@?5?$AA@   10028f50     cProc_dialog.obj
 0002:00004f54       ??_C@_03BDACDFHA@AND?$AA@  10028f54     cProc_dialog.obj
 0002:00004f58       ??_C@_03GBFNEA@NOT?$AA@    10028f58     cProc_dialog.obj
 0002:00004f5c       ??_C@_05PIANNGJP@Truth?$AA@ 10028f5c     cProc_dialog.obj
 0002:00004f64       ??_C@_05DCDOHKAB@Input?$AA@ 10028f64     cProc_dialog.obj
 0002:00004f6c       ??_C@_04OKOFBOPB@Time?$AA@ 10028f6c     cProc_dialog.obj
 0002:00004f74       ??_C@_07BCGHEHII@Holdoff?$AA@ 10028f74     cProc_dialog.obj
 0002:00004f7c       ??_C@_0BE@IPNEPNBD@No?5valid?5rule?5found?$AA@ 10028f7c     cProc_dialog.obj
 0002:00004f90       ??_C@_0CO@EOCPFADL@?$DMh1?$DOAlarms?5Process?5?9?5No?5Process?5@ 10028f90     cProc_dialog.obj
 0002:00004fc0       ??_C@_0DG@HDOJGDC@?$DMh1?$DOAlarms?5Process?5?9?5Multiple?5Pr@ 10028fc0     cProc_dialog.obj
 0002:00004ff8       ??_C@_0BA@LBOGFKMD@?5does?5not?5exist?$AA@ 10028ff8     cProc_dialog.obj
 0002:00005008       ??_C@_0DA@EOAFNEEI@cProc_dialog?3?3loadOutputModules?$CI@ 10029008     cProc_dialog.obj
 0002:00005038       ??_C@_0BA@FGFBJDIA@al_out_?$DP?$DP?$DP?$DP?4cfg?$AA@ 10029038     cProc_dialog.obj
 0002:00005048       ??_C@_06JIODDOFH@System?$AA@ 10029048     cProc_dialog.obj
 0002:00005050       ??_C@_0BA@DOMFHLGO@al_acq_?$DP?$DP?$DP?$DP?4cfg?$AA@ 10029050     cProc_dialog.obj
 0002:00005060       ??_C@_0DF@BHDIIGED@cProc_dialog?3?3inputBlockChange?5?9@ 10029060     cProc_dialog.obj
 0002:00005098       ??_C@_0DA@GLEIFAFB@cProc_dialog?3?3inputSlotChange?5?9?5@ 10029098     cProc_dialog.obj
 0002:000050c8       ??_C@_0DB@BHIKFBIN@cProc_dialog?3?3inputSlotChange?5?9?5@ 100290c8     cProc_dialog.obj
 0002:000050fc       ??_C@_07MFAOOMGP@darkred?$AA@ 100290fc     cProc_dialog.obj
 0002:00005104       ??_C@_05PMAELIEO@white?$AA@ 10029104     cProc_dialog.obj
 0002:00005110       __xmm@40ac200000000000c0ac200000000000 10029110     cProc_dialog.obj
 0002:00005124       ??_7cProcess@@6B@          10029124     cProcess.obj
 0002:00005128       ??_C@_04CDDMLLAK@0?400?$AA@ 10029128     cProcess.obj
 0002:00005134       ??_7?$QDict@VQString@@@@6B@ 10029134     cProcess.obj
 0002:00005150       ??_C@_05POAEJIHJ@INPUT?$AA@ 10029150     cProcess.obj
 0002:00005158       ??_C@_05DEDHDEOH@TRUTH?$AA@ 10029158     cProcess.obj
 0002:00005160       ??_C@_04OHBONDIN@TIME?$AA@ 10029160     cProcess.obj
 0002:00005168       ??_C@_07BGEMJJFK@HOLDOFF?$AA@ 10029168     cProcess.obj
 0002:00005170       ??_C@_0CP@PPCANOLK@cProcess?3?3LoadSettings?5?5?9?9?9?9?9?5?5R@ 10029170     cProcess.obj
 0002:000051a0       ??_C@_05JBBNGJKL@Latch?$AA@ 100291a0     cProcess.obj
 0002:000051a8       ??_C@_07PEMGOODH@AckOnce?$AA@ 100291a8     cProcess.obj
 0002:000051b0       ??_C@_09BFIAHDLF@Retrigger?$AA@ 100291b0     cProcess.obj
 0002:000051bc       ??_C@_04MKJKGABJ@Mask?$AA@ 100291bc     cProcess.obj
 0002:000051c4       ??_C@_06HDCHCENJ@Inputs?$AA@ 100291c4     cProcess.obj
 0002:000051cc       ??_C@_05MOFOMBOJ@Notes?$AA@ 100291cc     cProcess.obj
 0002:000051d4       ??_C@_0BJ@ENBEDJDG@IgnoreIntermediateStates?$AA@ 100291d4     cProcess.obj
 0002:000051f0       ??_C@_05FHMJPCKA@Start?$AA@ 100291f0     cProcess.obj
 0002:000051f8       ??_C@_03DBKJMAGF@End?$AA@  100291f8     cProcess.obj
 0002:000051fc       ??_C@_04EIAGBPOH@Days?$AA@ 100291fc     cProcess.obj
 0002:00005204       ??_C@_0L@GIEEPBHH@Table_?$CF04d?$AA@ 10029204     cProcess.obj
 0002:00005210       ??_C@_05KABNCBHK@?$CFd?0?$CFd?$AA@ 10029210     cProcess.obj
 0002:00005218       ??_C@_0CC@DKEMHJFC@?8?5already?5exists?0?5request?5refuse@ 10029218     cProcess.obj
 0002:0000523c       ??_C@_0BP@IDAMMJCE@cProcess?3?3setName?5?9?5new?5name?5?8?$AA@ 1002923c     cProcess.obj
 0002:00005260       ??_7multiInputBase@@6BQObject@@@ 10029260     multiinput.obj
 0002:00005424       ??_7multiInputBase@@6BQPaintDevice@@@ 10029424     multiinput.obj
 0002:0000544c       ??_SQListView@@6BQObject@@@ 1002944c     multiinput.obj
 0002:00005730       ??_SQListView@@6BQPaintDevice@@@ 10029730     multiinput.obj
 0002:00005750       ??_C@_0P@PLGFOCHP@multiInputBase?$AA@ 10029750     multiinput.obj
 0002:00005760       ??_C@_0BF@NDOEAAPL@multiInputBaseLayout?$AA@ 10029760     multiinput.obj
 0002:00005778       ??_C@_07JIAJFOLA@layout7?$AA@ 10029778     multiinput.obj
 0002:00005780       ??_C@_07KKDPDMDC@layout5?$AA@ 10029780     multiinput.obj
 0002:00005788       ??_C@_0L@KGLFILOJ@textLabel1?$AA@ 10029788     multiinput.obj
 0002:00005794       ??_C@_0M@KGIHAGOO@unusedProcs?$AA@ 10029794     multiinput.obj
 0002:000057a0       ??_C@_07OFHOKKPF@layout2?$AA@ 100297a0     multiinput.obj
 0002:000057a8       ??_C@_09KPPPMFPM@addButton?$AA@ 100297a8     multiinput.obj
 0002:000057b4       ??_C@_0N@OCENLIDK@removeButton?$AA@ 100297b4     multiinput.obj
 0002:000057c4       ??_C@_07IBBCGPPB@layout6?$AA@ 100297c4     multiinput.obj
 0002:000057cc       ??_C@_0N@HPEGIJEE@textLabel1_2?$AA@ 100297cc     multiinput.obj
 0002:000057dc       ??_C@_09OBFMKEPE@inputList?$AA@ 100297dc     multiinput.obj
 0002:000057e8       ??_C@_09FKDKBANL@layout6_2?$AA@ 100297e8     multiinput.obj
 0002:000057f4       ??_C@_0N@GGFNLIAF@textLabel1_3?$AA@ 100297f4     multiinput.obj
 0002:00005804       ??_C@_0L@FGIHNJBP@editFilter?$AA@ 10029804     multiinput.obj
 0002:00005810       ??_C@_08DKBDHOFF@buttonOk?$AA@ 10029810     multiinput.obj
 0002:0000581c       ??_C@_0N@OLKBNHFJ@buttonCancel?$AA@ 1002981c     multiinput.obj
 0002:0000582c       ??_C@_09DMINLBG@1accept?$CI?$CJ?$AA@ 1002982c     multiinput.obj
 0002:00005838       ??_C@_09OCDCAEKE@1reject?$CI?$CJ?$AA@ 10029838     multiinput.obj
 0002:00005844       ??_C@_0BA@MFJMDOMG@Input?5Selection?$AA@ 10029844     multiinput.obj
 0002:00005854       ??_C@_0BE@PEEHCFMB@Available?5Processes?$AA@ 10029854     multiinput.obj
 0002:00005868       ??_C@_0BM@NDKLOFPH@List?5of?5avaialble?5Processes?$AA@ 10029868     multiinput.obj
 0002:00005888       ??_C@_0EJ@CCCFOODE@List?5of?5available?5processes?5to?5b@ 10029888     multiinput.obj
 0002:000058d4       ??_C@_09ILJNJIDP@Add?5Input?$AA@ 100298d4     multiinput.obj
 0002:000058e0       ??_C@_0BM@FIKDIOLC@Add?5processes?5to?5input?5list?$AA@ 100298e0     multiinput.obj
 0002:00005900       ??_C@_0GA@JFNLIIFE@Add?5the?5selected?5process?5from?5th@ 10029900     multiinput.obj
 0002:00005960       ??_C@_0N@DKAMKNNM@Remove?5Input?$AA@ 10029960     multiinput.obj
 0002:00005970       ??_C@_0BH@PCANCIJ@Remove?5selected?5inputs?$AA@ 10029970     multiinput.obj
 0002:00005988       ??_C@_0DP@IJENMLNA@Remove?5the?5selected?5processes?5fr@ 10029988     multiinput.obj
 0002:000059c8       ??_C@_0BA@PJCMKCAG@Selected?5Inputs?$AA@ 100299c8     multiinput.obj
 0002:000059d8       ??_C@_0P@CEJPBMPO@Current?5Inputs?$AA@ 100299d8     multiinput.obj
 0002:000059e8       ??_C@_0CM@OFLDJJDO@The?5current?5inputs?5to?5the?5sleect@ 100299e8     multiinput.obj
 0002:00005a14       ??_C@_03DDKJIMDC@?$CGOK?$AA@ 10029a14     multiinput.obj
 0002:00005a18       ??_C@_07JLEKEEPN@?$CGCancel?$AA@ 10029a18     multiinput.obj
 0002:00005a24       ??_7MultiInputInvalidListViewItem@@6B@ 10029a24     multiinputimpl.obj
 0002:00005ac0       ??_7multiInput@@6BQObject@@@ 10029ac0     multiinputimpl.obj
 0002:00005c84       ??_7multiInput@@6BQPaintDevice@@@ 10029c84     multiinputimpl.obj
 0002:00005ca4       ??_C@_07EHMCOPMF@PosSize?$AA@ 10029ca4     multiinputimpl.obj
 0002:00005cac       ??_C@_0CC@MGGGJFCF@Home?1Alarms?1Processes?1MultiInput@ 10029cac     multiinputimpl.obj
 0002:00005cd0       ??_C@_0N@OEKHNLII@1enableAdd?$CI?$CJ?$AA@ 10029cd0     multiinputimpl.obj
 0002:00005ce0       ??_C@_0BO@JOANJKKM@1addProcesses?$CIQListViewItem?$CK?$CJ?$AA@ 10029ce0     multiinputimpl.obj
 0002:00005d00       ??_C@_0M@LOLGNNBG@UnusedProcs?$AA@ 10029d00     multiinputimpl.obj
 0002:00005d0c       ??_C@_0BA@NPNJLGPG@1enableRemove?$CI?$CJ?$AA@ 10029d0c     multiinputimpl.obj
 0002:00005d1c       ??_C@_0CB@NMNBBLLG@1removeProcesses?$CIQListViewItem?$CK?$CJ@ 10029d1c     multiinputimpl.obj
 0002:00005d40       ??_C@_09MPMOOAPN@UsedProcs?$AA@ 10029d40     multiinputimpl.obj
 0002:00005d4c       ??_C@_07CJMBKHEI@forward?$AA@ 10029d4c     multiinputimpl.obj
 0002:00005d54       ??_C@_0BA@KBIAHJHB@1addProcesses?$CI?$CJ?$AA@ 10029d54     multiinputimpl.obj
 0002:00005d64       ??_C@_04JFCNHLLM@back?$AA@ 10029d64     multiinputimpl.obj
 0002:00005d6c       ??_C@_0BD@OGKCFANJ@1removeProcesses?$CI?$CJ?$AA@ 10029d6c     multiinputimpl.obj
 0002:00005d80       ??_C@_06NJHBABOH@grey90?$AA@ 10029d80     multiinputimpl.obj
 0002:00005d88       ??_C@_06NCCNEGNK@grey60?$AA@ 10029d88     multiinputimpl.obj
 0002:00005d90       ??_C@_0CD@BFGBAEB@?5?5?5?514?5?5?5?514?5?5?5?5?5?5?5?54?5?5?5?5?5?5?5?5?5?5?5@ 10029d90     plugindesc.obj
 0002:00005db4       ??_C@_0M@EKMPMHDK@?4?5c?5?$CD040404?$AA@ 10029db4     plugindesc.obj
 0002:00005dc0       ??_C@_0M@NBLJLJNN@?$CD?5c?5?$CD808304?$AA@ 10029dc0     plugindesc.obj
 0002:00005dcc       ??_C@_0M@EAFJJBBG@a?5c?5?$CDbfc2bf?$AA@ 10029dcc     plugindesc.obj
 0002:00005dd8       ??_C@_08PBKCALNO@b?5c?5None?$AA@ 10029dd8     plugindesc.obj
 0002:00005de4       ??_C@_0P@HFKAALMG@?4?4?4?4?4?4?4?4?4?4?4?4?4?4?$AA@ 10029de4     plugindesc.obj
 0002:00005df4       ??_C@_0P@LGBCEGMD@?4?$CD?4aaaaaaaa?4a?4?$AA@ 10029df4     plugindesc.obj
 0002:00005e04       ??_C@_0P@MNNEIMDO@?4?$CD?4aaaaaaaa?4?4?4?$AA@ 10029e04     plugindesc.obj
 0002:00005e14       ??_C@_0P@MFAMBPGN@?4?$CD?4aaaaaaaa?4?$CD?4?$AA@ 10029e14     plugindesc.obj
 0002:00005e24       ??_C@_0P@HPMEFAGN@?4?$CD?$CD?4?4?4?4?4?4?4?4?$CD?$CD?4?$AA@ 10029e24     plugindesc.obj
 0002:00005e34       ??_C@_0P@JAJCNDBN@?4?$CD?$CD?$CD?$CD?$CD?$CD?$CD?$CD?$CD?$CD?$CD?$CD?4?$AA@ 10029e34     plugindesc.obj
 0002:00005e44       ??_C@_0P@INKOIILA@?4?$CD?$CD?4?4?4?4?4?4?4?4?4?$CD?4?$AA@ 10029e44     plugindesc.obj
 0002:00005e54       ??_C@_0P@KJADPPJB@?4?$CD?$CD?4?4?4?4?4?4aa?4?$CD?4?$AA@ 10029e54     plugindesc.obj
 0002:00005e64       ??_C@_0P@PKKONJFP@b?4?4?4?4?4?4?4?4?4?4?4?4?4?$AA@ 10029e64     plugindesc.obj
 0002:00005e78       ??_7config_plugin_desc_base@@6B@ 10029e78     plugindesc.obj
 0002:00005e8c       ??_7plugindesc@@6B@        10029e8c     plugindesc.obj
 0002:00005e9c       ??_C@_0BG@NGLOHLJB@Home?1Alarms?1Processes?$AA@ 10029e9c     plugindesc.obj
 0002:00005eb8       ??_7singleInputBase@@6BQObject@@@ 10029eb8     singleinput.obj
 0002:0000607c       ??_7singleInputBase@@6BQPaintDevice@@@ 1002a07c     singleinput.obj
 0002:0000609c       ??_C@_0BA@HCJCHJKC@singleInputBase?$AA@ 1002a09c     singleinput.obj
 0002:000060ac       ??_C@_0BG@COMHBHBK@singleInputBaseLayout?$AA@ 1002a0ac     singleinput.obj
 0002:000060c4       ??_C@_08HEFODFJH@layout14?$AA@ 1002a0c4     singleinput.obj
 0002:000060d0       ??_C@_0O@MABFEOEO@m_qEditFilter?$AA@ 1002a0d0     singleinput.obj
 0002:000060e0       ??_C@_0BD@KLFFIOHF@m_qPushClearFilter?$AA@ 1002a0e0     singleinput.obj
 0002:000060f4       ??_C@_07BPJBECHP@layout8?$AA@ 1002a0f4     singleinput.obj
 0002:000060fc       ??_C@_0M@CJICOIGM@singleInput?$AA@ 1002a0fc     singleinput.obj
 0002:00006108       ??_C@_0EM@NPMOKCGO@Select?5a?5process?0?5the?5?8OK?8?0?5pres@ 1002a108     singleinput.obj
 0002:00006158       ??_7singleInput@@6BQObject@@@ 1002a158     singleinputimpl.obj
 0002:0000631c       ??_7singleInput@@6BQPaintDevice@@@ 1002a31c     singleinputimpl.obj
 0002:0000633c       ??_C@_0CC@PGHNPCFG@1selectinChanged?$CIQListViewItem?5?$CK@ 1002a33c     singleinputimpl.obj
 0002:00006360       ??_C@_0CC@LCOLGNI@2selectionChanged?$CIQListViewItem?$CK@ 1002a360     singleinputimpl.obj
 0002:00006388       ??_7template_dialogBase@@6BQObject@@@ 1002a388     template_dialog.obj
 0002:0000654c       ??_7template_dialogBase@@6BQPaintDevice@@@ 1002a54c     template_dialog.obj
 0002:00006574       ??_SQCheckBox@@6BQObject@@@ 1002a574     template_dialog.obj
 0002:00006754       ??_SQCheckBox@@6BQPaintDevice@@@ 1002a754     template_dialog.obj
 0002:0000677c       ??_SQSpinBox@@6BQObject@@@ 1002a77c     template_dialog.obj
 0002:00006974       ??_SQSpinBox@@6BQPaintDevice@@@ 1002a974     template_dialog.obj
 0002:00006998       ??_SQSpinBox@@6B@          1002a998     template_dialog.obj
 0002:000069ac       ??_SQButtonGroup@@6BQObject@@@ 1002a9ac     template_dialog.obj
 0002:00006b9c       ??_SQButtonGroup@@6BQPaintDevice@@@ 1002ab9c     template_dialog.obj
 0002:00006bc4       ??_SQRadioButton@@6BQObject@@@ 1002abc4     template_dialog.obj
 0002:00006da8       ??_SQRadioButton@@6BQPaintDevice@@@ 1002ada8     template_dialog.obj
 0002:00006dcc       ??_SQGridLayout@@6BQObject@@@ 1002adcc     template_dialog.obj
 0002:00006e3c       ??_SQGridLayout@@6BQLayoutItem@@@ 1002ae3c     template_dialog.obj
 0002:00006e7c       ??_C@_0BE@BJLJGBCO@template_dialogBase?$AA@ 1002ae7c     template_dialog.obj
 0002:00006e90       ??_C@_0BK@CEJEBDAE@template_dialogBaseLayout?$AA@ 1002ae90     template_dialog.obj
 0002:00006eac       ??_C@_0P@GMJDGEMK@checkOverwrite?$AA@ 1002aeac     template_dialog.obj
 0002:00006ebc       ??_C@_0O@GDFADIKM@checkRelation?$AA@ 1002aebc     template_dialog.obj
 0002:00006ecc       ??_C@_0L@EJODNDNM@spinCopies?$AA@ 1002aecc     template_dialog.obj
 0002:00006ed8       ??_C@_0L@INJINICK@textLabel2?$AA@ 1002aed8     template_dialog.obj
 0002:00006ee4       ??_C@_0O@BIHHDGEO@editOldPrefix?$AA@ 1002aee4     template_dialog.obj
 0002:00006ef4       ??_C@_0N@IIAHHGMJ@buttonGroup6?$AA@ 1002aef4     template_dialog.obj
 0002:00006f04       ??_C@_0O@MCGPINBG@editNewSuffix?$AA@ 1002af04     template_dialog.obj
 0002:00006f14       ??_C@_0N@GNPDCGKK@textLabel2_2?$AA@ 1002af14     template_dialog.obj
 0002:00006f24       ??_C@_0P@MHFIBJB@textLabel2_2_2?$AA@ 1002af24     template_dialog.obj
 0002:00006f34       ??_C@_0O@KJCCNNOD@editNewPrefix?$AA@ 1002af34     template_dialog.obj
 0002:00006f44       ??_C@_0L@IGGLKAGG@groupNames?$AA@ 1002af44     template_dialog.obj
 0002:00006f50       ??_C@_0BA@MHIDFLAK@editInitialChar?$AA@ 1002af50     template_dialog.obj
 0002:00006f60       ??_C@_0M@JMIOKMHO@radioLetter?$AA@ 1002af60     template_dialog.obj
 0002:00006f6c       ??_C@_07KFAKJJKN@radioNo?$AA@ 1002af6c     template_dialog.obj
 0002:00006f74       ??_C@_07NOBKPBGG@spinPad?$AA@ 1002af74     template_dialog.obj
 0002:00006f7c       ??_C@_0BB@OFNACKOA@spinInitialCount?$AA@ 1002af7c     template_dialog.obj
 0002:00006f90       ??_C@_08CELLGALL@labelPad?$AA@ 1002af90     template_dialog.obj
 0002:00006f9c       ??_C@_08GJCAOGIA@radioNum?$AA@ 1002af9c     template_dialog.obj
 0002:00006fa8       ??_C@_0BB@FPKNHHCJ@m_pqLabelExample?$AA@ 1002afa8     template_dialog.obj
 0002:00006fbc       ??_C@_0BH@JJKKLBPN@m_pqLabelSelectedCount?$AA@ 1002afbc     template_dialog.obj
 0002:00006fd4       ??_C@_0BC@DLEJKFKG@1setEnabled?$CIbool?$CJ?$AA@ 1002afd4     template_dialog.obj
 0002:00006fe8       ??_C@_0P@POCECEMJ@2toggled?$CIbool?$CJ?$AA@ 1002afe8     template_dialog.obj
 0002:00006ff8       ??_C@_0BN@NDOBKDDK@Create?5copies?5using?5template?$AA@ 1002aff8     template_dialog.obj
 0002:00007018       ??_C@_0EC@FIFCGBGF@Replace?5any?5existing?5processes?5?9@ 1002b018     template_dialog.obj
 0002:0000705c       ??_C@_0DN@PKBBOCIP@Maintain?5Relationships?5?9?5new?5inp@ 1002b05c     template_dialog.obj
 0002:0000709c       ??_C@_0BB@EBBCCNHP@Number?5of?5copies?$AA@ 1002b09c     template_dialog.obj
 0002:000070b0       ??_C@_0BC@BIKPGDHG@Prefix?5to?5replace?$AA@ 1002b0b0     template_dialog.obj
 0002:000070c4       ??_C@_0L@MAHMGJEK@New?5Prefix?$AA@ 1002b0c4     template_dialog.obj
 0002:000070d0       ??_C@_0L@MDNJGBEK@First?5Part?$AA@ 1002b0d0     template_dialog.obj
 0002:000070dc       ??_C@_0L@FPGADHIC@Third?5Part?$AA@ 1002b0dc     template_dialog.obj
 0002:000070e8       ??_C@_0M@ENNNPKDI@Second?5Part?$AA@ 1002b0e8     template_dialog.obj
 0002:000070f4       ??_C@_01FHEEJDEE@A?$AA@    1002b0f4     template_dialog.obj
 0002:000070f8       ??_C@_0L@MDMDHMFH@Add?5Letter?$AA@ 1002b0f8     template_dialog.obj
 0002:00007104       ??_C@_0M@OOMKIHID@No?5Addition?$AA@ 1002b104     template_dialog.obj
 0002:00007110       ??_C@_0BB@DAPMDJLB@Leading?5zero?5pad?$AA@ 1002b110     template_dialog.obj
 0002:00007124       ??_C@_0L@IALFKLMJ@Add?5number?$AA@ 1002b124     template_dialog.obj
 0002:00007130       ??_C@_0BF@BOOGMGCH@prefix?9number?9suffix?$AA@ 1002b130     template_dialog.obj
 0002:00007148       ??_C@_0BD@FKECGGNI@Processes?5selected?$AA@ 1002b148     template_dialog.obj
 0002:0000715c       ??_C@_05HBFPNANJ@Alt?$CLO?$AA@ 1002b15c     template_dialog.obj
 0002:00007164       ??_C@_05NNOKJPNF@Alt?$CLC?$AA@ 1002b164     template_dialog.obj
 0002:00007170       ??_7template_dialog@@6BQObject@@@ 1002b170     template_dialogimpl.obj
 0002:00007334       ??_7template_dialog@@6BQPaintDevice@@@ 1002b334     template_dialogimpl.obj
 0002:00007354       ??_C@_0BA@LACDMGIG@1numCopies?$CIint?$CJ?$AA@ 1002b354     template_dialogimpl.obj
 0002:00007364       ??_C@_0BD@OIBDOPAP@2valueChanged?$CIint?$CJ?$AA@ 1002b364     template_dialogimpl.obj
 0002:00007378       ??_C@_0CD@DEENPFBA@1oldPrefixChanged?$CIconst?5QString?5@ 1002b378     template_dialogimpl.obj
 0002:0000739c       ??_C@_0P@POJJJFKD@1showExample?$CI?$CJ?$AA@ 1002b39c     template_dialogimpl.obj
 0002:000073ac       ??_C@_0BA@HHAILMBL@2clicked?$CI?5int?5?$CJ?$AA@ 1002b3ac     template_dialogimpl.obj
 0002:000073bc       ??_C@_0BH@NMJOCACL@?$CF1?5processes?5selected?4?$AA@ 1002b3bc     template_dialogimpl.obj
 0002:000073d4       ??_C@_0BG@GMFAIIIH@?8?$CF1?8?5will?5become?5?8?$CF2?8?$AA@ 1002b3d4     template_dialogimpl.obj
 0002:000073ec       ??_C@_0BI@PEBOJNMN@Creating?5new?5process?5?9?5?$AA@ 1002b3ec     template_dialogimpl.obj
 0002:00007408       ??_7CheckContDialogBase@@6BQObject@@@ 1002b408     checkcontributiondialog.obj
 0002:000075d4       ??_7CheckContDialogBase@@6BQPaintDevice@@@ 1002b5d4     checkcontributiondialog.obj
 0002:000075f4       ??_C@_0BE@JKLAPPCA@CheckContDialogBase?$AA@ 1002b5f4     checkcontributiondialog.obj
 0002:00007608       ??_C@_0BK@OONDABFG@CheckContDialogBaseLayout?$AA@ 1002b608     checkcontributiondialog.obj
 0002:00007624       ??_C@_0N@MHEGOAAO@buttonGroup1?$AA@ 1002b624     checkcontributiondialog.obj
 0002:00007634       ??_C@_08LGPHPIL@layout21?$AA@ 1002b634     checkcontributiondialog.obj
 0002:00007640       ??_C@_0M@LIKKEEOC@rbInputDiag?$AA@ 1002b640     checkcontributiondialog.obj
 0002:0000764c       ??_C@_08BCHEEOMK@layout20?$AA@ 1002b64c     checkcontributiondialog.obj
 0002:00007658       ??_C@_07LDCEANHD@layout4?$AA@ 1002b658     checkcontributiondialog.obj
 0002:00007660       ??_C@_07CAJNFAIO@cbEmpty?$AA@ 1002b660     checkcontributiondialog.obj
 0002:00007668       ??_C@_09PHCFMJDA@cbInvalid?$AA@ 1002b668     checkcontributiondialog.obj
 0002:00007674       ??_C@_0O@JAMJBENM@rbContribDiag?$AA@ 1002b674     checkcontributiondialog.obj
 0002:00007684       ??_C@_08NIOLHKJL@layout18?$AA@ 1002b684     checkcontributiondialog.obj
 0002:00007690       ??_C@_0O@IFEFGEIO@lbDescription?$AA@ 1002b690     checkcontributiondialog.obj
 0002:000076a0       ??_C@_08MBPAELNK@layout19?$AA@ 1002b6a0     checkcontributiondialog.obj
 0002:000076ac       ??_C@_08JCJMBNC@layout11?$AA@ 1002b6ac     checkcontributiondialog.obj
 0002:000076b8       ??_C@_05BFHEGHFJ@lbMax?$AA@ 1002b6b8     checkcontributiondialog.obj
 0002:000076c0       ??_C@_05OPFPPHJK@spMin?$AA@ 1002b6c0     checkcontributiondialog.obj
 0002:000076c8       ??_C@_04BAKPOLHO@cbOr?$AA@ 1002b6c8     checkcontributiondialog.obj
 0002:000076d0       ??_C@_05HPPIDDG@lbMin?$AA@ 1002b6d0     checkcontributiondialog.obj
 0002:000076d8       ??_C@_07KEJDPOFP@cbInput?$AA@ 1002b6d8     checkcontributiondialog.obj
 0002:000076e0       ??_C@_05PNNEBDPF@spMax?$AA@ 1002b6e0     checkcontributiondialog.obj
 0002:000076e8       ??_C@_07PMGFJLLE@layout3?$AA@ 1002b6e8     checkcontributiondialog.obj
 0002:000076f0       ??_C@_0BH@DBJFGGOK@1rbInputDiag_clicked?$CI?$CJ?$AA@ 1002b6f0     checkcontributiondialog.obj
 0002:00007708       ??_C@_0BJ@NCBKINAD@1rbContribDiag_clicked?$CI?$CJ?$AA@ 1002b708     checkcontributiondialog.obj
 0002:00007724       ??_C@_0BJ@OJCKBKKI@Contribution?5Diagnostics?$AA@ 1002b724     checkcontributiondialog.obj
 0002:00007740       ??_C@_0BE@KBEGAJPD@Diagnostics?5options?$AA@ 1002b740     checkcontributiondialog.obj
 0002:00007754       ??_C@_0BC@HFJHHLPL@Input?5diagnostics?$AA@ 1002b754     checkcontributiondialog.obj
 0002:00007768       ??_C@_0CA@HGEHLPND@Processes?5with?5empty?5input?5list?$AA@ 1002b768     checkcontributiondialog.obj
 0002:00007788       ??_C@_0BO@GEKNFKIO@Invalid?5process?5on?5input?5list?$AA@ 1002b788     checkcontributiondialog.obj
 0002:000077a8       ??_C@_0CJ@PFJBANDG@Filter?5on?5number?5of?5contribution@ 1002b7a8     checkcontributiondialog.obj
 0002:000077d8       ??_C@_0GK@DDCOBNEO@Check?5the?5process?5type?5you?5are?5i@ 1002b7d8     checkcontributiondialog.obj
 0002:00007844       ??_C@_04GFGPODON@Max?3?$AA@ 1002b844     checkcontributiondialog.obj
 0002:0000784c       ??_C@_0O@PFJDINFF@OR?5and?5others?$AA@ 1002b84c     checkcontributiondialog.obj
 0002:0000785c       ??_C@_04LIHABEMA@Min?3?$AA@ 1002b85c     checkcontributiondialog.obj
 0002:00007868       ??_C@_0EA@EDKDFOJE@CheckContDialogBase?3?3rbInputDiag@ 1002b868     checkcontributiondialog.obj
 0002:000078a8       ??_C@_0EC@LOEDLAPF@CheckContDialogBase?3?3rbContribDi@ 1002b8a8     checkcontributiondialog.obj
 0002:000078f0       ??_7LatchAckDialogBase@@6BQObject@@@ 1002b8f0     latchackdialog.obj
 0002:00007ab4       ??_7LatchAckDialogBase@@6BQPaintDevice@@@ 1002bab4     latchackdialog.obj
 0002:00007ad4       ??_C@_0BD@DMMGDBFM@LatchAckDialogBase?$AA@ 1002bad4     latchackdialog.obj
 0002:00007ae8       ??_C@_0BJ@FHLHEEME@LatchAckDialogBaseLayout?$AA@ 1002bae8     latchackdialog.obj
 0002:00007b04       ??_C@_07HLAONPF@cbLatch?$AA@ 1002bb04     latchackdialog.obj
 0002:00007b0c       ??_C@_09DKCLEPHJ@cbAckOnce?$AA@ 1002bb0c     latchackdialog.obj
 0002:00007b18       ??_C@_0P@MDFLJKJI@LatchAckDialog?$AA@ 1002bb18     latchackdialog.obj
 0002:00007b28       ??_C@_0O@FLKLBJJK@Ack?5Once?5Only?$AA@ 1002bb28     latchackdialog.obj
 0002:00007b38       ??_C@_0DA@KELFEDEP@Set?5Latch?5?1?5Ack?5Once?5for?5the?5sel@ 1002bb38     latchackdialog.obj
 0002:00007b6c       ??_7LatchAckDialog@@6BQObject@@@ 1002bb6c     latchackdialogimpl.obj
 0002:00007d30       ??_7LatchAckDialog@@6BQPaintDevice@@@ 1002bd30     latchackdialogimpl.obj
 0002:00007d50       ??_C@_0M@EKCLAHOC@alm_process?$AA@ 1002bd50     moc_alm_process.obj
 0002:00007d68       ??_C@_05JLNEMJLN@dummy?$AA@ 1002bd68     moc_alm_process.obj
 0002:00007d70       ??_C@_07FLKIBHAM@sFilter?$AA@ 1002bd70     moc_alm_process.obj
 0002:00007d84       ??_C@_0N@NHGOHCF@filterChange?$AA@ 1002bd84     moc_alm_process.obj
 0002:00007da0       ??_C@_0M@PACBOOEA@clearFilter?$AA@ 1002bda0     moc_alm_process.obj
 0002:00007db8       ??_C@_0BJ@ELGKFKKF@copyProcessUsingTemplate?$AA@ 1002bdb8     moc_alm_process.obj
 0002:00007de0       ??_C@_0L@PEGIFJLJ@changeMask?$AA@ 1002bde0     moc_alm_process.obj
 0002:00007df8       ??_C@_0O@BKNIGMGG@deleteProcess?$AA@ 1002bdf8     moc_alm_process.obj
 0002:00007e14       ??_C@_0BB@MKKMGLEA@duplicateProcess?$AA@ 1002be14     moc_alm_process.obj
 0002:00007e64       ??_C@_0L@GCGKOLNO@newProcess?$AA@ 1002be64     moc_alm_process.obj
 0002:00007e70       ??_C@_04MGCDEED@proc?$AA@  1002be70     moc_alm_process.obj
 0002:00007e78       ??_C@_08CLKECPOL@cProcess?$AA@ 1002be78     moc_alm_process.obj
 0002:00007e90       ??_C@_0P@FKGAKEMJ@updateProcList?$AA@ 1002be90     moc_alm_process.obj
 0002:00007eac       ??_C@_0BA@NKJEPPCI@addSingleInputs?$AA@ 1002beac     moc_alm_process.obj
 0002:00007ec8       ??_C@_0P@BBOPFDKJ@addMultiInputs?$AA@ 1002bec8     moc_alm_process.obj
 0002:00007ee4       ??_C@_0O@GHGODGGJ@selectProcess?$AA@ 1002bee4     moc_alm_process.obj
 0002:00007f00       ??_C@_09HIGIDEDO@markDirty?$AA@ 1002bf00     moc_alm_process.obj
 0002:00007f18       ??_C@_0L@PPKMKFDG@sysCommand?$AA@ 1002bf18     moc_alm_process.obj
 0002:00007f24       ??_C@_07ECHCKIDD@sSystem?$AA@ 1002bf24     moc_alm_process.obj
 0002:00007f38       ??_C@_0N@JNMAEFDJ@selectSystem?$AA@ 1002bf38     moc_alm_process.obj
 0002:00007f54       ??_C@_0BA@DJDDKEKN@setProcessGroup?$AA@ 1002bf54     moc_alm_process.obj
 0002:00007f70       ??_C@_09JMJFHHPF@clearMask?$AA@ 1002bf70     moc_alm_process.obj
 0002:00007f88       ??_C@_07CHIPCIL@setMask?$AA@ 1002bf88     moc_alm_process.obj
 0002:00007f9c       ??_C@_0M@PNANGIDH@setLatchAck?$AA@ 1002bf9c     moc_alm_process.obj
 0002:00007fb4       ??_C@_0BA@FMCGOADO@startRenameProc?$AA@ 1002bfb4     moc_alm_process.obj
 0002:00007fc4       ??_C@_04NHONDGDE@item?$AA@ 1002bfc4     moc_alm_process.obj
 0002:00007fcc       ??_C@_0O@LAFKAPIP@QListViewItem?$AA@ 1002bfcc     moc_alm_process.obj
 0002:00007fdc       ??_C@_03PCBNCGFH@pos?$AA@  1002bfdc     moc_alm_process.obj
 0002:00007fe0       ??_C@_01CAKFMAIO@?$AO?$AA@ 1002bfe0     moc_alm_process.obj
 0002:00007fe4       ??_C@_03HNOLNALI@col?$AA@  1002bfe4     moc_alm_process.obj
 0002:00007ff4       ??_C@_0BE@NOBPCBPN@procListContextMenu?$AA@ 1002bff4     moc_alm_process.obj
 0002:00008014       ??_C@_0M@EAABKIDO@startRename?$AA@ 1002c014     moc_alm_process.obj
 0002:00008020       ??_C@_03ELAIKMFE@lvi?$AA@  1002c020     moc_alm_process.obj
 0002:00008024       ??_C@_04KOJNECLL@iCol?$AA@ 1002c024     moc_alm_process.obj
 0002:0000802c       ??_C@_07KMMJHNPL@newName?$AA@ 1002c02c     moc_alm_process.obj
 0002:00008040       ??_C@_0O@DPBFMID@renameProcess?$AA@ 1002c040     moc_alm_process.obj
 0002:00008050       ??_C@_07NGIDDFG@sModule?$AA@ 1002c050     moc_alm_process.obj
 0002:00008058       ??_C@_07BDKJBEOJ@sEditor?$AA@ 1002c058     moc_alm_process.obj
 0002:0000806c       ??_C@_0M@JOJJPBPE@navToOutput?$AA@ 1002c06c     moc_alm_process.obj
 0002:00008078       ??_C@_05MFBAOMHM@sSlot?$AA@ 1002c078     moc_alm_process.obj
 0002:0000808c       ??_C@_08HNODKGGD@navToAck?$AA@ 1002c08c     moc_alm_process.obj
 0002:00008098       ??_C@_05DHPFDCJG@sProc?$AA@ 1002c098     moc_alm_process.obj
 0002:0000822c       ??_C@_07MBMLLJIG@dummy?$CI?$CJ?$AA@ 1002c22c     moc_alm_process.obj
 0002:00008234       ??_C@_0BN@BJBBIKGE@filterChange?$CIconst?5QString?$CG?$CJ?$AA@ 1002c234     moc_alm_process.obj
 0002:00008254       ??_C@_0O@MFNDPIOI@clearFilter?$CI?$CJ?$AA@ 1002c254     moc_alm_process.obj
 0002:00008264       ??_C@_0BL@CKNGDDJP@copyProcessUsingTemplate?$CI?$CJ?$AA@ 1002c264     moc_alm_process.obj
 0002:00008280       ??_C@_0N@FFKIIAHK@changeMask?$CI?$CJ?$AA@ 1002c280     moc_alm_process.obj
 0002:00008290       ??_C@_0BA@FLLHDDJ@deleteProcess?$CI?$CJ?$AA@ 1002c290     moc_alm_process.obj
 0002:000082a0       ??_C@_0BD@FIABLFMK@duplicateProcess?$CI?$CJ?$AA@ 1002c2a0     moc_alm_process.obj
 0002:000082b4       ??_C@_09FDIMKBKN@newGate?$CI?$CJ?$AA@ 1002c2b4     moc_alm_process.obj
 0002:000082c0       ??_C@_0O@MEHMOFFE@deleteGroup?$CI?$CJ?$AA@ 1002c2c0     moc_alm_process.obj
 0002:000082d0       ??_C@_0O@NNFFNFLB@renameGroup?$CI?$CJ?$AA@ 1002c2d0     moc_alm_process.obj
 0002:000082e0       ??_C@_0L@LMMOGCOM@newGroup?$CI?$CJ?$AA@ 1002c2e0     moc_alm_process.obj
 0002:000082ec       ??_C@_0N@FKHLDJLI@newProcess?$CI?$CJ?$AA@ 1002c2ec     moc_alm_process.obj
 0002:000082fc       ??_C@_0BK@PFAFFOG@updateProcList?$CIcProcess?$CK?$CJ?$AA@ 1002c2fc     moc_alm_process.obj
 0002:00008318       ??_C@_0BC@CEHBDAA@addSingleInputs?$CI?$CJ?$AA@ 1002c318     moc_alm_process.obj
 0002:0000832c       ??_C@_0BB@PPLPJOLC@addMultiInputs?$CI?$CJ?$AA@ 1002c32c     moc_alm_process.obj
 0002:00008340       ??_C@_0M@BCGJBPBD@markDirty?$CI?$CJ?$AA@ 1002c340     moc_alm_process.obj
 0002:0000834c       ??_C@_0CK@JKOBFOMF@sysCommand?$CIconst?5QString?$CG?0const?5@ 1002c34c     moc_alm_process.obj
 0002:00008378       ??_C@_0BN@PCNKHLKL@selectSystem?$CIconst?5QString?$CG?$CJ?$AA@ 1002c378     moc_alm_process.obj
 0002:00008398       ??_C@_0BC@LIAKBENF@setProcessGroup?$CI?$CJ?$AA@ 1002c398     moc_alm_process.obj
 0002:000083ac       ??_C@_0M@NFLCOFEB@clearMask?$CI?$CJ?$AA@ 1002c3ac     moc_alm_process.obj
 0002:000083b8       ??_C@_09PJNMFIHL@setMask?$CI?$CJ?$AA@ 1002c3b8     moc_alm_process.obj
 0002:000083c4       ??_C@_0O@KBHGDMOA@setLatchAck?$CI?$CJ?$AA@ 1002c3c4     moc_alm_process.obj
 0002:000083d4       ??_C@_0BC@JDNHCNJA@startRenameProc?$CI?$CJ?$AA@ 1002c3d4     moc_alm_process.obj
 0002:000083e8       ??_C@_0DG@LGNBMBGO@procListContextMenu?$CIQListViewIte@ 1002c3e8     moc_alm_process.obj
 0002:00008420       ??_C@_0BM@HOBMHNGL@startRename?$CIQListViewItem?$CK?$CJ?$AA@ 1002c420     moc_alm_process.obj
 0002:0000843c       ??_C@_0DB@FDEIOBNI@renameProcess?$CIQListViewItem?$CK?0int@ 1002c43c     moc_alm_process.obj
 0002:00008470       ??_C@_0BN@PBNLKHBP@navToOutput?$CIQString?0QString?$CJ?$AA@ 1002c470     moc_alm_process.obj
 0002:00008490       ??_C@_0CC@OGKPLIKI@navToAck?$CIQString?0QString?0QString@ 1002c490     moc_alm_process.obj
 0002:000084b4       ??_C@_0BH@IHNIAINL@selectProcess?$CIQString?$CJ?$AA@ 1002c4b4     moc_alm_process.obj
 0002:000084cc       ??_C@_0BL@KCGFDGJP@checkProcessContributors?$CI?$CJ?$AA@ 1002c4cc     moc_alm_process.obj
 0002:000084f4       ??_C@_07KMMNMMFF@command?$AA@ 1002c4f4     moc_alm_process.obj
 0002:00008508       ??_C@_0BJ@FEFNJDLM@command?$CIQString?0QString?$CJ?$AA@ 1002c508     moc_alm_process.obj
 0002:00008524       ??_C@_0BA@ILBFGNJI@CheckContDialog?$AA@ 1002c524     moc_checkContDialogImpl.obj
 0002:00008540       ??_C@_06MPKMECK@accept?$AA@ 1002c540     moc_checkContDialogImpl.obj
 0002:00008554       ??_C@_0BE@ENLIJCA@rbInputDiag_clicked?$AA@ 1002c554     moc_checkContDialogImpl.obj
 0002:00008574       ??_C@_0BG@MIJIDIOJ@rbContribDiag_clicked?$AA@ 1002c574     moc_checkContDialogImpl.obj
 0002:000085b0       ??_C@_08IBHKEOMI@accept?$CI?$CJ?$AA@ 1002c5b0     moc_checkContDialogImpl.obj
 0002:000085bc       ??_C@_0BG@HDPIJDEO@rbInputDiag_clicked?$CI?$CJ?$AA@ 1002c5bc     moc_checkContDialogImpl.obj
 0002:000085d4       ??_C@_0BI@NFKGLABA@rbContribDiag_clicked?$CI?$CJ?$AA@ 1002c5d4     moc_checkContDialogImpl.obj
 0002:00008610       ??_C@_0P@DMEOIADN@languageChange?$AA@ 1002c610     moc_checkcontributiondialog.obj
 0002:00008644       ??_C@_0BB@PFEIHPGD@languageChange?$CI?$CJ?$AA@ 1002c644     moc_checkcontributiondialog.obj
 0002:00008658       ??_C@_0N@PMBEOMHK@cProc_dialog?$AA@ 1002c658     moc_cProc_dialog.obj
 0002:00008674       ??_C@_0M@MNOHPNHB@editAcqSlot?$AA@ 1002c674     moc_cProc_dialog.obj
 0002:0000868c       ??_C@_05DAMMEJMI@sMask?$AA@ 1002c68c     moc_cProc_dialog.obj
 0002:000086ac       ??_C@_0O@JGCIAEFM@changeHoldoff?$AA@ 1002c6ac     moc_cProc_dialog.obj
 0002:000086c8       ??_C@_0BA@IHBFMKB@inputSlotChange?$AA@ 1002c6c8     moc_cProc_dialog.obj
 0002:000086d8       ??_C@_06OJMPLFM@sBlock?$AA@ 1002c6d8     moc_cProc_dialog.obj
 0002:000086ec       ??_C@_0BB@NKLFLKJD@inputBlockChange?$AA@ 1002c6ec     moc_cProc_dialog.obj
 0002:0000870c       ??_C@_0BF@OFJBBBKL@enableTruthDeleteCol?$AA@ 1002c70c     moc_cProc_dialog.obj
 0002:00008730       ??_C@_0BA@FKANCDKO@navOutputModule?$AA@ 1002c730     moc_cProc_dialog.obj
 0002:0000874c       ??_C@_0BB@DDEEIDDI@navContributesTo?$AA@ 1002c74c     moc_cProc_dialog.obj
 0002:0000876c       ??_C@_0P@CNHHEADI@enableNavigate?$AA@ 1002c76c     moc_cProc_dialog.obj
 0002:00008788       ??_C@_0BC@OMAIIPML@deleteTruthColumn?$AA@ 1002c788     moc_cProc_dialog.obj
 0002:0000879c       ??_C@_08GEBDPLAG@sNewRule?$AA@ 1002c79c     moc_cProc_dialog.obj
 0002:000087b4       ??_C@_0P@HGJECJFI@changeFunction?$AA@ 1002c7b4     moc_cProc_dialog.obj
 0002:000087c4       ??_C@_05BDFBMKBD@sText?$AA@ 1002c7c4     moc_cProc_dialog.obj
 0002:000087d8       ??_C@_0M@BHNKLCOO@changeGroup?$AA@ 1002c7d8     moc_cProc_dialog.obj
 0002:000087e4       ??_C@_02OHHJDGIP@ti?$AA@   1002c7e4     moc_cProc_dialog.obj
 0002:000087e8       ??_C@_01BHBACGJK@?$BL?$AA@ 1002c7e8     moc_cProc_dialog.obj
 0002:000087f8       ??_C@_0BB@LFHEKDLC@startTimeChanged?$AA@ 1002c7f8     moc_cProc_dialog.obj
 0002:00008818       ??_C@_0P@OFANFFHJ@endTimeChanged?$AA@ 1002c818     moc_cProc_dialog.obj
 0002:00008834       ??_C@_0M@PGFFFNDC@itemChanged?$AA@ 1002c834     moc_cProc_dialog.obj
 0002:00008840       ??_C@_01KBJDNOO@i?$AA@     1002c840     moc_cProc_dialog.obj
 0002:00008850       ??_C@_01EFFIKLCJ@n?$AA@    1002c850     moc_cProc_dialog.obj
 0002:0000886c       ??_C@_0P@JINDDJHA@addTruthColumn?$AA@ 1002c86c     moc_cProc_dialog.obj
 0002:00008964       ??_C@_0O@IHDAIDEC@editAcqSlot?$CI?$CJ?$AA@ 1002c964     moc_cProc_dialog.obj
 0002:00008974       ??_C@_0BB@DBMDNPGG@setMask?$CIQString?$CJ?$AA@ 1002c974     moc_cProc_dialog.obj
 0002:00008988       ??_C@_0BO@BJPMEKPB@changeHoldoff?$CIconst?5QString?$CG?$CJ?$AA@ 1002c988     moc_cProc_dialog.obj
 0002:000089a8       ??_C@_0CA@LFOLMFFA@inputSlotChange?$CIconst?5QString?$CG?$CJ?$AA@ 1002c9a8     moc_cProc_dialog.obj
 0002:000089c8       ??_C@_0CB@PPMKPEFP@inputBlockChange?$CIconst?5QString?$CG?$CJ@ 1002c9c8     moc_cProc_dialog.obj
 0002:000089ec       ??_C@_0BO@IANBOHHB@enableTruthDeleteCol?$CIint?0int?$CJ?$AA@ 1002c9ec     moc_cProc_dialog.obj
 0002:00008a0c       ??_C@_0BC@OAPLDCKL@navOutputModule?$CI?$CJ?$AA@ 1002ca0c     moc_cProc_dialog.obj
 0002:00008a20       ??_C@_0BD@BBDGNFJG@navContributesTo?$CI?$CJ?$AA@ 1002ca20     moc_cProc_dialog.obj
 0002:00008a34       ??_C@_0BB@BDFLFIKP@enableNavigate?$CI?$CJ?$AA@ 1002ca34     moc_cProc_dialog.obj
 0002:00008a48       ??_C@_0BE@CHBBPEIP@deleteTruthColumn?$CI?$CJ?$AA@ 1002ca48     moc_cProc_dialog.obj
 0002:00008a5c       ??_C@_0BP@BFMPIPNG@changeFunction?$CIconst?5QString?$CG?$CJ?$AA@ 1002ca5c     moc_cProc_dialog.obj
 0002:00008a7c       ??_C@_0BM@GGONCGIF@changeGroup?$CIconst?5QString?$CG?$CJ?$AA@ 1002ca7c     moc_cProc_dialog.obj
 0002:00008a98       ??_C@_0BP@FPDHAPKC@startTimeChanged?$CIconst?5QTime?$CG?$CJ?$AA@ 1002ca98     moc_cProc_dialog.obj
 0002:00008ab8       ??_C@_0BN@KJODMMFD@endTimeChanged?$CIconst?5QTime?$CG?$CJ?$AA@ 1002cab8     moc_cProc_dialog.obj
 0002:00008ad8       ??_C@_0O@IKLCAHNO@itemChanged?$CI?$CJ?$AA@ 1002cad8     moc_cProc_dialog.obj
 0002:00008ae8       ??_C@_0BB@HJINNLMJ@itemChanged?$CIint?$CJ?$AA@ 1002cae8     moc_cProc_dialog.obj
 0002:00008afc       ??_C@_0BF@CFMFAPBL@itemChanged?$CIint?0int?$CJ?$AA@ 1002cafc     moc_cProc_dialog.obj
 0002:00008b14       ??_C@_0BB@CCCOBJO@addTruthColumn?$CI?$CJ?$AA@ 1002cb14     moc_cProc_dialog.obj
 0002:00008b34       ??_C@_0L@EEOKDMMD@updateProc?$AA@ 1002cb34     moc_cProc_dialog.obj
 0002:00008b4c       ??_C@_0N@IBIICDGH@itemsChanged?$AA@ 1002cb4c     moc_cProc_dialog.obj
 0002:00008b68       ??_C@_09CIDKMNDE@navToProc?$AA@ 1002cb68     moc_cProc_dialog.obj
 0002:00008bc8       ??_C@_0BG@KFMJGMLH@updateProc?$CIcProcess?$CK?$CJ?$AA@ 1002cbc8     moc_cProc_dialog.obj
 0002:00008be0       ??_C@_0P@PKMDIFCJ@itemsChanged?$CI?$CJ?$AA@ 1002cbe0     moc_cProc_dialog.obj
 0002:00008bf0       ??_C@_0BD@IPFANDPL@navToProc?$CIQString?$CJ?$AA@ 1002cbf0     moc_cProc_dialog.obj
 0002:00008c34       ??_C@_0L@OPDIBLEB@multiInput?$AA@ 1002cc34     moc_multiinputimpl.obj
 0002:00008c4c       ??_C@_0N@OCECJHCC@enableRemove?$AA@ 1002cc4c     moc_multiinputimpl.obj
 0002:00008c68       ??_C@_09PMHBDKHJ@enableAdd?$AA@ 1002cc68     moc_multiinputimpl.obj
 0002:00008c80       ??_C@_0BA@MDHAJGMB@removeProcesses?$AA@ 1002cc80     moc_multiinputimpl.obj
 0002:00008ca8       ??_C@_0N@OJKMKJGF@addProcesses?$AA@ 1002cca8     moc_multiinputimpl.obj
 0002:00008d24       ??_C@_0P@LLMBCKDG@enableRemove?$CI?$CJ?$AA@ 1002cd24     moc_multiinputimpl.obj
 0002:00008d34       ??_C@_0M@EKOJGPMP@enableAdd?$CI?$CJ?$AA@ 1002cd34     moc_multiinputimpl.obj
 0002:00008d40       ??_C@_0BC@LJJFJLLN@removeProcesses?$CI?$CJ?$AA@ 1002cd40     moc_multiinputimpl.obj
 0002:00008d54       ??_C@_0CA@DIHJOGPC@removeProcesses?$CIQListViewItem?$CK?$CJ?$AA@ 1002cd54     moc_multiinputimpl.obj
 0002:00008d74       ??_C@_0P@MFJIOFLB@addProcesses?$CI?$CJ?$AA@ 1002cd74     moc_multiinputimpl.obj
 0002:00008d84       ??_C@_0BN@DIAJMGDB@addProcesses?$CIQListViewItem?$CK?$CJ?$AA@ 1002cd84     moc_multiinputimpl.obj
 0002:00008da4       ??_C@_0M@NJCDNHGL@proc_config?$AA@ 1002cda4     moc_proc_config.obj
 0002:00008dec       ??_C@_0BA@JKFOGPOI@selectinChanged?$AA@ 1002cdec     moc_singleinputimpl.obj
 0002:00008e38       ??_C@_0CA@EEHELOOI@selectinChanged?$CIQListViewItem?$CK?$CJ?$AA@ 1002ce38     moc_singleinputimpl.obj
 0002:00008e70       ??_C@_0BA@NNLMAKOH@template_dialog?$AA@ 1002ce70     moc_template_dialogimpl.obj
 0002:00008e8c       ??_C@_0BB@FFHBKFJN@oldPrefixChanged?$AA@ 1002ce8c     moc_template_dialogimpl.obj
 0002:00008ea0       ??_C@_06DJHIOBEC@iValue?$AA@ 1002cea0     moc_template_dialogimpl.obj
 0002:00008eb4       ??_C@_09FLDCDJGJ@numCopies?$AA@ 1002ceb4     moc_template_dialogimpl.obj
 0002:00008ecc       ??_C@_0M@KHEPNMPE@showExample?$AA@ 1002cecc     moc_template_dialogimpl.obj
 0002:00008efc       ??_C@_0CB@JDNODJAM@oldPrefixChanged?$CIconst?5QString?$CG?$CJ@ 1002cefc     moc_template_dialogimpl.obj
 0002:00008f20       ??_C@_0P@NEDLFKEG@numCopies?$CIint?$CJ?$AA@ 1002cf20     moc_template_dialogimpl.obj
 0002:00008f30       ??_C@_0O@INKNJFLK@showExample?$CI?$CJ?$AA@ 1002cf30     moc_template_dialogimpl.obj
 0002:00008f44       ??_7proc_config@@6BQObject@@@ 1002cf44     proc_config.obj
 0002:000090fc       ??_7proc_config@@6BQPaintDevice@@@ 1002d0fc     proc_config.obj
 0002:00009124       ??_SQSplitter@@6BQObject@@@ 1002d124     proc_config.obj
 0002:0000930c       ??_SQSplitter@@6BQPaintDevice@@@ 1002d30c     proc_config.obj
 0002:00009334       ??_SQGroupBox@@6BQObject@@@ 1002d334     proc_config.obj
 0002:00009514       ??_SQGroupBox@@6BQPaintDevice@@@ 1002d514     proc_config.obj
 0002:0000953c       ??_SQComboBox@@6BQObject@@@ 1002d53c     proc_config.obj
 0002:00009720       ??_SQComboBox@@6BQPaintDevice@@@ 1002d720     proc_config.obj
 0002:00009744       ??_SQWidgetStack@@6BQObject@@@ 1002d744     proc_config.obj
 0002:0000991c       ??_SQWidgetStack@@6BQPaintDevice@@@ 1002d91c     proc_config.obj
 0002:00009944       ??_SQListBox@@6BQObject@@@ 1002d944     proc_config.obj
 0002:00009bec       ??_SQListBox@@6BQPaintDevice@@@ 1002dbec     proc_config.obj
 0002:00009c14       ??_SQTimeEdit@@6BQObject@@@ 1002dc14     proc_config.obj
 0002:00009e08       ??_SQTimeEdit@@6BQPaintDevice@@@ 1002de08     proc_config.obj
 0002:00009e2c       ??_SQTextEdit@@6BQObject@@@ 1002de2c     proc_config.obj
 0002:0000a1a8       ??_SQTextEdit@@6BQPaintDevice@@@ 1002e1a8     proc_config.obj
 0002:0000a1c8       ??_C@_0BC@KHNEOCOP@proc_configLayout?$AA@ 1002e1c8     proc_config.obj
 0002:0000a1dc       ??_C@_09FMLOPOJA@labelProc?$AA@ 1002e1dc     proc_config.obj
 0002:0000a1e8       ??_C@_0N@LBCDIEML@textLabel3_6?$AA@ 1002e1e8     proc_config.obj
 0002:0000a1f8       ??_C@_0BF@CDEFDLNL@labelNumberProcesses?$AA@ 1002e1f8     proc_config.obj
 0002:0000a210       ??_C@_09GJPDGDGA@splitter1?$AA@ 1002e210     proc_config.obj
 0002:0000a21c       ??_C@_08BADCPAJD@layout10?$AA@ 1002e21c     proc_config.obj
 0002:0000a228       ??_C@_07GIKHDDO@layout9?$AA@ 1002e228     proc_config.obj
 0002:0000a230       ??_C@_07NLAIMGB@ackOnce?$AA@ 1002e230     proc_config.obj
 0002:0000a238       ??_C@_0M@KCMHHDFF@actionFrame?$AA@ 1002e238     proc_config.obj
 0002:0000a244       ??_C@_09EMGPFCAF@comboRule?$AA@ 1002e244     proc_config.obj
 0002:0000a250       ??_C@_09FJBGAOOL@maskFrame?$AA@ 1002e250     proc_config.obj
 0002:0000a25c       ??_C@_0O@CINAIGFO@m_pqLabelMask?$AA@ 1002e25c     proc_config.obj
 0002:0000a26c       ??_C@_08CEMPFAPK@layout42?$AA@ 1002e26c     proc_config.obj
 0002:0000a278       ??_C@_09FFPAFMBO@maskClear?$AA@ 1002e278     proc_config.obj
 0002:0000a284       ??_C@_0BA@NPHDNPKE@maskChangeInput?$AA@ 1002e284     proc_config.obj
 0002:0000a294       ??_C@_0L@BFCFJEIO@groupFrame?$AA@ 1002e294     proc_config.obj
 0002:0000a2a0       ??_C@_0L@LALBKBIN@comboGroup?$AA@ 1002e2a0     proc_config.obj
 0002:0000a2ac       ??_C@_05JGLBGMJN@latch?$AA@ 1002e2ac     proc_config.obj
 0002:0000a2b4       ??_C@_05IANLDAEP@stack?$AA@ 1002e2b4     proc_config.obj
 0002:0000a2bc       ??_C@_05NLIPEJCP@BLANK?$AA@ 1002e2bc     proc_config.obj
 0002:0000a2c4       ??_C@_0M@DDIOEJAF@INPUTLayout?$AA@ 1002e2c4     proc_config.obj
 0002:0000a2d0       ??_C@_08CCAEJCBB@layout12?$AA@ 1002e2d0     proc_config.obj
 0002:0000a2dc       ??_C@_09ONBMAFOK@groupBox4?$AA@ 1002e2dc     proc_config.obj
 0002:0000a2e8       ??_C@_07DPHPLNNF@inBlock?$AA@ 1002e2e8     proc_config.obj
 0002:0000a2f0       ??_C@_06EINIIKNC@inSlot?$AA@ 1002e2f0     proc_config.obj
 0002:0000a2f8       ??_C@_09IBLEODOA@editInput?$AA@ 1002e2f8     proc_config.obj
 0002:0000a304       ??_C@_09BIGHFPMF@ANDLayout?$AA@ 1002e304     proc_config.obj
 0002:0000a310       ??_C@_09EBKJEKOG@groupBox8?$AA@ 1002e310     proc_config.obj
 0002:0000a31c       ??_C@_09PDOEAIOI@andInputs?$AA@ 1002e31c     proc_config.obj
 0002:0000a328       ??_C@_09CFJAAIN@layout9_2?$AA@ 1002e328     proc_config.obj
 0002:0000a334       ??_C@_0M@HDMBPFGN@andAddInput?$AA@ 1002e334     proc_config.obj
 0002:0000a340       ??_C@_08MBDDGDGM@ORLayout?$AA@ 1002e340     proc_config.obj
 0002:0000a34c       ??_C@_09MGDBFGCJ@groupBox7?$AA@ 1002e34c     proc_config.obj
 0002:0000a358       ??_C@_08GFONDHJB@orInputs?$AA@ 1002e358     proc_config.obj
 0002:0000a364       ??_C@_0L@GNEBAGAL@layout10_2?$AA@ 1002e364     proc_config.obj
 0002:0000a370       ??_C@_0M@DGHBLOHC@RetriggerOr?$AA@ 1002e370     proc_config.obj
 0002:0000a37c       ??_C@_0BD@JCEDCKBO@IgnoreIntermediate?$AA@ 1002e37c     proc_config.obj
 0002:0000a390       ??_C@_0L@DLFKIMOG@orAddInput?$AA@ 1002e390     proc_config.obj
 0002:0000a39c       ??_C@_09ICKMCBCA@NOTLayout?$AA@ 1002e39c     proc_config.obj
 0002:0000a3a8       ??_C@_09NPCKGHGI@groupBox6?$AA@ 1002e3a8     proc_config.obj
 0002:0000a3b4       ??_C@_08OALINDBF@notInput?$AA@ 1002e3b4     proc_config.obj
 0002:0000a3c0       ??_C@_0P@FPKIEFPL@notChangeInput?$AA@ 1002e3c0     proc_config.obj
 0002:0000a3d0       ??_C@_0M@NPJDAIHI@TRUTHLayout?$AA@ 1002e3d0     proc_config.obj
 0002:0000a3dc       ??_C@_0L@JJLPODHL@groupBox10?$AA@ 1002e3dc     proc_config.obj
 0002:0000a3e8       ??_C@_05PPKBNDKJ@truth?$AA@ 1002e3e8     proc_config.obj
 0002:0000a3f0       ??_C@_08DNNEGBLL@layout43?$AA@ 1002e3f0     proc_config.obj
 0002:0000a3fc       ??_C@_0O@KJLPBFBG@truthAddInput?$AA@ 1002e3fc     proc_config.obj
 0002:0000a40c       ??_C@_0M@KFMALCEL@truthAddCol?$AA@ 1002e40c     proc_config.obj
 0002:0000a418       ??_C@_0P@NIOBGLFG@truthDeleteCol?$AA@ 1002e418     proc_config.obj
 0002:0000a428       ??_C@_0L@LOPNFEFG@TIMELayout?$AA@ 1002e428     proc_config.obj
 0002:0000a434       ??_C@_09FILCHLKH@groupBox9?$AA@ 1002e434     proc_config.obj
 0002:0000a440       ??_C@_08HHNKOBPJ@layout34?$AA@ 1002e440     proc_config.obj
 0002:0000a44c       ??_C@_08PCMHLDEH@dayGroup?$AA@ 1002e44c     proc_config.obj
 0002:0000a458       ??_C@_04ELIIBNGE@day1?$AA@ 1002e458     proc_config.obj
 0002:0000a460       ??_C@_04GAKFEOKH@day2?$AA@ 1002e460     proc_config.obj
 0002:0000a468       ??_C@_04HJLOHPOG@day3?$AA@ 1002e468     proc_config.obj
 0002:0000a470       ??_C@_04DGPPOJCB@day4?$AA@ 1002e470     proc_config.obj
 0002:0000a478       ??_C@_04CPOENIGA@day5?$AA@ 1002e478     proc_config.obj
 0002:0000a480       ??_C@_04EMJILKD@day6?$AA@  1002e480     proc_config.obj
 0002:0000a488       ??_C@_04FCJDCMCF@day0?$AA@ 1002e488     proc_config.obj
 0002:0000a490       ??_C@_08NKKNMEMC@layout28?$AA@ 1002e490     proc_config.obj
 0002:0000a49c       ??_C@_0M@GCBLFBJE@groupBox2_3?$AA@ 1002e49c     proc_config.obj
 0002:0000a4a8       ??_C@_09JIIDPPEA@timeStart?$AA@ 1002e4a8     proc_config.obj
 0002:0000a4b4       ??_C@_07KGEDLCPF@timeEnd?$AA@ 1002e4b4     proc_config.obj
 0002:0000a4bc       ??_C@_0L@JEIDOJGL@textLabel3?$AA@ 1002e4bc     proc_config.obj
 0002:0000a4c8       ??_C@_07OLBBCFNO@holdoff?$AA@ 1002e4c8     proc_config.obj
 0002:0000a4d0       ??_C@_0O@KCOKGCMA@holdoffLayout?$AA@ 1002e4d0     proc_config.obj
 0002:0000a4e0       ??_C@_0M@PEGCPHIC@groupBox6_2?$AA@ 1002e4e0     proc_config.obj
 0002:0000a4ec       ??_C@_0N@HNEEFJAJ@holdoffInput?$AA@ 1002e4ec     proc_config.obj
 0002:0000a4fc       ??_C@_0BD@OJJBKNJE@holdoffChangeInput?$AA@ 1002e4fc     proc_config.obj
 0002:0000a510       ??_C@_0BB@IAOPENMP@buttonGroup1_2_2?$AA@ 1002e510     proc_config.obj
 0002:0000a524       ??_C@_0N@CEEOGAA@holdoffDelay?$AA@ 1002e524     proc_config.obj
 0002:0000a534       ??_C@_09BCNCJHCI@textNotes?$AA@ 1002e534     proc_config.obj
 0002:0000a540       ??_C@_09LLEGKCGM@groupBox2?$AA@ 1002e540     proc_config.obj
 0002:0000a54c       ??_C@_0M@BOFNCGCE@listOutputs?$AA@ 1002e54c     proc_config.obj
 0002:0000a558       ??_C@_0BC@HHDIOFPI@editContributesTo?$AA@ 1002e558     proc_config.obj
 0002:0000a56c       ??_C@_0M@HLAAGANF@groupBox2_2?$AA@ 1002e56c     proc_config.obj
 0002:0000a578       ??_C@_0BC@IJHDPAHE@listOutputModules?$AA@ 1002e578     proc_config.obj
 0002:0000a58c       ??_C@_0M@HIOMEAJD@editOutputs?$AA@ 1002e58c     proc_config.obj
 0002:0000a598       ??_C@_05MLDKGAGH@Form1?$AA@ 1002e598     proc_config.obj
 0002:0000a5a0       ??_C@_0BG@CPLADPN@?$DMh1?$DOProcess?5Name?$DM?1h1?$DO?$AA@ 1002e5a0     proc_config.obj
 0002:0000a5b8       ??_C@_0BB@NLIHJNIO@Selected?5Process?$AA@ 1002e5b8     proc_config.obj
 0002:0000a5d0       ??_C@_0EC@LMIHMPFO@?$DMh3?$DOProcess?5Name?$DM?1h3?$DO?6This?5is?5th@ 1002e5d0     proc_config.obj
 0002:0000a614       ??_C@_0BE@GABKMIND@Number?5of?5Processes?$AA@ 1002e614     proc_config.obj
 0002:0000a628       ??_C@_0BB@GCGGELOL@Latch?5the?5output?$AA@ 1002e628     proc_config.obj
 0002:0000a640       ??_C@_0IE@EAPLGCHO@Setthe?5output?5to?5?8Latched?8?5when?5@ 1002e640     proc_config.obj
 0002:0000a6c4       ??_C@_06PMAGBHAK@Action?$AA@ 1002e6c4     proc_config.obj
 0002:0000a6cc       ??_C@_05HOPBAMFM@?9?5?9?5?9?$AA@ 1002e6cc     proc_config.obj
 0002:0000a6d4       ??_C@_0M@BALIMOBC@AND?5process?$AA@ 1002e6d4     proc_config.obj
 0002:0000a6e0       ??_C@_0L@EABCGMGB@OR?5process?$AA@ 1002e6e0     proc_config.obj
 0002:0000a6ec       ??_C@_0M@IEAMAPEL@NOT?5process?$AA@ 1002e6ec     proc_config.obj
 0002:0000a6f8       ??_C@_0BE@PHKKPELF@Truth?5Table?5process?$AA@ 1002e6f8     proc_config.obj
 0002:0000a70c       ??_C@_0M@JKFJIKKO@Time?5of?5Day?$AA@ 1002e70c     proc_config.obj
 0002:0000a718       ??_C@_0P@GEADBGLB@Current?5action?$AA@ 1002e718     proc_config.obj
 0002:0000a728       ??_C@_0CPD@HBNNHONO@?$DMh3?$DO?$DM?1h3?$DOEach?5process?5is?5an?5acti@ 1002e728     proc_config.obj
 0002:0000aa1c       ??_C@_0BC@MMEOIMLG@Mask?5this?5process?$AA@ 1002ea1c     proc_config.obj
 0002:0000aa30       ??_C@_0OH@DCBDNKLC@When?5the?5mask?5is?5active?5the?5curr@ 1002ea30     proc_config.obj
 0002:0000ab18       ??_C@_05MDNHABIA@Clear?$AA@ 1002eb18     proc_config.obj
 0002:0000ab20       ??_C@_06NJGOFONI@Change?$AA@ 1002eb20     proc_config.obj
 0002:0000ab28       ??_C@_0KB@KCMLMCAD@Each?5process?5can?5be?5in?5a?5group?0?5@ 1002eb28     proc_config.obj
 0002:0000abcc       ??_C@_0N@JJAFAHJK@Latch?5Output?$AA@ 1002ebcc     proc_config.obj
 0002:0000abdc       ??_C@_0BA@IKMBDNBG@Input?5selection?$AA@ 1002ebdc     proc_config.obj
 0002:0000abf0       ??_C@_0HO@HGBAJEPJ@Select?5which?5input?5block?0?5and?5wh@ 1002ebf0     proc_config.obj
 0002:0000ac70       ??_C@_06JNOLMJDJ@Block?3?$AA@ 1002ec70     proc_config.obj
 0002:0000ac78       ??_C@_05INPBEHOJ@Slot?3?$AA@ 1002ec78     proc_config.obj
 0002:0000ac80       ??_C@_0L@IAAPOKOA@Edit?5Input?$AA@ 1002ec80     proc_config.obj
 0002:0000ac8c       ??_C@_09GFDEPCFE@AND?5Input?$AA@ 1002ec8c     proc_config.obj
 0002:0000ac98       ??_C@_0DJ@ECFPBHME@Select?5which?5processes?5are?5input@ 1002ec98     proc_config.obj
 0002:0000acd4       ??_C@_0O@DLDEHNJE@Change?5Inputs?$AA@ 1002ecd4     proc_config.obj
 0002:0000ace4       ??_C@_08LMGAMOPN@OR?5Input?$AA@ 1002ece4     proc_config.obj
 0002:0000acf0       ??_C@_0BI@FPDFCDDF@Re?9trigger?5on?5new?5error?$AA@ 1002ecf0     proc_config.obj
 0002:0000ad08       ??_C@_0BJ@CLFBCKFF@Ignore?5latched?0?5ack?5etc?4?$AA@ 1002ed08     proc_config.obj
 0002:0000ad28       ??_C@_0GB@NIAACFLO@Ignore?5inputs?5that?5are?5latched?5o@ 1002ed28     proc_config.obj
 0002:0000ad8c       ??_C@_09PPPPIMLB@NOT?5Input?$AA@ 1002ed8c     proc_config.obj
 0002:0000ad98       ??_C@_0DI@JBOMGJAI@Select?5which?5process?5is?5an?5input@ 1002ed98     proc_config.obj
 0002:0000add0       ??_C@_0M@JHKAGLHE@Truth?5Table?$AA@ 1002edd0     proc_config.obj
 0002:0000addc       ??_C@_0BF@HPHOGOFD@Truth?5table?5settings?$AA@ 1002eddc     proc_config.obj
 0002:0000adf8       ??_C@_0BBN@MKDOFGCO@The?5current?5Truth?5Table?4?5If?5any?5@ 1002edf8     proc_config.obj
 0002:0000af18       ??_C@_0L@JEFIJIBL@Add?5Column?$AA@ 1002ef18     proc_config.obj
 0002:0000af24       ??_C@_0O@EOGFAJOA@Delete?5Column?$AA@ 1002ef24     proc_config.obj
 0002:0000af34       ??_C@_0BF@OBFOCLJP@Time?5Of?5Day?5Settings?$AA@ 1002ef34     proc_config.obj
 0002:0000af4c       ??_C@_0BF@HEJANCEB@Time?5of?5Day?5settings?$AA@ 1002ef4c     proc_config.obj
 0002:0000af68       ??_C@_0BBI@CJBLBOOO@The?5outputs?5of?5this?5process?5is?5?8@ 1002ef68     proc_config.obj
 0002:0000b080       ??_C@_06JLEDEDGH@Monday?$AA@ 1002f080     proc_config.obj
 0002:0000b088       ??_C@_07BAAGCFCM@Tuesday?$AA@ 1002f088     proc_config.obj
 0002:0000b090       ??_C@_09DLIGFAKA@Wednesday?$AA@ 1002f090     proc_config.obj
 0002:0000b09c       ??_C@_08HACCIKIA@Thursday?$AA@ 1002f09c     proc_config.obj
 0002:0000b0a8       ??_C@_06JECMNKMI@Friday?$AA@ 1002f0a8     proc_config.obj
 0002:0000b0b0       ??_C@_08INBOOONO@Saturday?$AA@ 1002f0b0     proc_config.obj
 0002:0000b0bc       ??_C@_06OOPIFAJ@Sunday?$AA@ 1002f0bc     proc_config.obj
 0002:0000b0c4       ??_C@_0O@BCNNLHIJ@Holdoff?5Input?$AA@ 1002f0c4     proc_config.obj
 0002:0000b0d4       ??_C@_0P@GDJFNNCA@Hold?5off?5input?$AA@ 1002f0d4     proc_config.obj
 0002:0000b0e4       ??_C@_0CD@MDDBCIDJ@Select?5the?5input?5for?5this?5proces@ 1002f0e4     proc_config.obj
 0002:0000b108       ??_C@_05ENDOMFAI@Delay?$AA@ 1002f108     proc_config.obj
 0002:0000b110       ??_C@_0BM@PHCLBDK@Delay?5before?5output?5changes?$AA@ 1002f110     proc_config.obj
 0002:0000b130       ??_C@_0FI@EMEPIKPI@Set?5the?5time?5period?5that?5the?5inp@ 1002f130     proc_config.obj
 0002:0000b188       ??_C@_06PMLBNKGE@Notes?3?$AA@ 1002f188     proc_config.obj
 0002:0000b190       ??_C@_0P@DAKNOGAM@Contributes?5To?$AA@ 1002f190     proc_config.obj
 0002:0000b1a0       ??_C@_0DB@GNLFIDPG@Current?5process?5is?5used?5by?5these@ 1002f1a0     proc_config.obj
 0002:0000b1d8       ??_C@_0COM@CCICCFHA@?$DMh3?$DO?$DM?1h3?$DOEach?5process?5is?5an?5acti@ 1002f1d8     proc_config.obj
 0002:0000b4c4       ??_C@_0N@HKALLKJF@Edit?5Process?$AA@ 1002f4c4     proc_config.obj
 0002:0000b4d4       ??_C@_0P@CCHNPFEA@Output?5Modules?$AA@ 1002f4d4     proc_config.obj
 0002:0000b4e4       ??_C@_0BJ@DEKFFENE@Output?5module?5navigation?$AA@ 1002f4e4     proc_config.obj
 0002:0000b500       ??_C@_0IH@EMCPJE@List?5of?5output?5modules?5that?5the?5@ 1002f500     proc_config.obj
 0002:0000b588       ??_C@_0N@BDAPJIM@Edit?5Outputs?$AA@ 1002f588     proc_config.obj
 0002:0000b59c       ??_7config_mb4@@6BQObject@@@ 1002f59c     cfg_widgets001:config_mb4impl.obj
 0002:0000b75c       ??_7config_mb4@@6BQPaintDevice@@@ 1002f75c     cfg_widgets001:config_mb4impl.obj
 0002:0000b77c       ??_C@_0BF@NKGLKMD@Set?5text?5in?5the?5code?$AA@ 1002f77c     cfg_widgets001:config_mb4impl.obj
 0002:0000b794       ??_C@_07GHFMDGIP@Button?5?$AA@ 1002f794     cfg_widgets001:config_mb4impl.obj
 0002:0000b79c       ??_C@_04ILFHLBJA@?$CGYes?$AA@ 1002f79c     cfg_widgets001:config_mb4impl.obj
 0002:0000b7a4       ??_C@_0M@CMBAIKAM@Yes?5to?5?$CGAll?$AA@ 1002f7a4     cfg_widgets001:config_mb4impl.obj
 0002:0000b7b0       ??_C@_03MDIDAHKD@?$CGNo?$AA@ 1002f7b0     cfg_widgets001:config_mb4impl.obj
 0002:0000b7b4       ??_C@_0BN@PFBFBCOO@Do?5you?5want?5to?5save?5the?5file?$AA@ 1002f7b4     cfg_widgets001:config_mb4impl.obj
 0002:0000b7d4       ??_C@_0BE@KGMONIMP@1buttonClicked?$CIint?$CJ?$AA@ 1002f7d4     cfg_widgets001:config_mb4impl.obj
 0002:0000b7e8       ??_C@_0BI@GGLIKMPP@CC_ConfigEdit?1Controls?1?$AA@ 1002f7e8     cfg_widgets001:cfg_Settings.obj
 0002:0000b800       ??_C@_02PIGFKFFE@?$CF1?$AA@ 1002f800     cfg_widgets001:cfg_Settings.obj
 0002:0000b804       ??_C@_03MMIELDNM@?0?$CF1?$AA@ 1002f804     cfg_widgets001:cfg_Settings.obj
 0002:0000b808       ??_C@_03FFMPJLOG@?$CF1?0?$AA@ 1002f808     cfg_widgets001:cfg_Settings.obj
 0002:0000b80c       ??_C@_0P@JHCMIKMI@?$CF1?0?$CF2?0?$CF3?0?$CF4?0?$CF5?$AA@ 1002f80c     cfg_widgets001:cfg_Settings.obj
 0002:0000b820       ??_7cfg_ListView@@6BQObject@@@ 1002f820     cfg_widgets001:cfg_ListView.obj
 0002:0000bb0c       ??_7cfg_ListView@@6BQPaintDevice@@@ 1002fb0c     cfg_widgets001:cfg_ListView.obj
 0002:0000bb2c       ??_C@_0BI@DKLEEDHJ@1clipBoardDataChanged?$CI?$CJ?$AA@ 1002fb2c     cfg_widgets001:cfg_ListView.obj
 0002:0000bb44       ??_C@_0BA@NOIFKKAG@2dataChanged?5?$CI?$CJ?$AA@ 1002fb44     cfg_widgets001:cfg_ListView.obj
 0002:0000bb54       ??_C@_01GPOEFGEJ@?7?$AA@   1002fb54     cfg_widgets001:cfg_ListView.obj
 0002:0000bb58       ??_C@_0EB@PMPDJKLD@int?5cfg_ListView?3?3validateRow?$CIiR@ 1002fb58     cfg_widgets001:cfg_ListView.obj
 0002:0000bb9c       ??_C@_0BD@BEIDFIOE@Creating?5new?5entry?$AA@ 1002fb9c     cfg_widgets001:cfg_ListView.obj
 0002:0000bbb0       ??_C@_0DO@OOICEDKL@int?5cfg_Table?3?3validateRow?$CIiRow?$CJ@ 1002fbb0     cfg_widgets001:cfg_ListView.obj
 0002:0000bbf0       ??_C@_0EN@NNOBKMDG@cfg_ListView?3?3updateEntry?5?9?5newI@ 1002fbf0     cfg_widgets001:cfg_ListView.obj
 0002:0000bc40       ??_C@_0FB@OICAKFGC@int?5cfg_ListView?3?3validateRow?$CIQL@ 1002fc40     cfg_widgets001:cfg_ListView.obj
 0002:0000bc98       ??_7cfg_Table@@6BQObject@@@ 1002fc98     cfg_widgets001:cfg_Table.obj
 0002:0000c03c       ??_7cfg_Table@@6BQPaintDevice@@@ 1003003c     cfg_widgets001:cfg_Table.obj
 0002:0000c060       ??_C@_0EG@JCAEPHHD@Selected?5Area?5does?5not?5match?4?6Do@ 10030060     cfg_widgets001:cfg_Table.obj
 0002:0000c0a8       ??_C@_0BB@LNOIOJNO@Database?5Edtitor?$AA@ 100300a8     cfg_widgets001:cfg_Table.obj
 0002:0000c0c0       ??_C@_0EE@IEHIFONC@int?5cfg_Table?3?3validateRow?$CIint?5i@ 100300c0     cfg_widgets001:cfg_Table.obj
 0002:0000c104       ??_C@_0L@HHCOLPHE@config_mb4?$AA@ 10030104     cfg_widgets001:moc_config_mb4impl.obj
 0002:0000c110       ??_C@_02EGCJHIOB@id?$AA@   10030110     cfg_widgets001:moc_config_mb4impl.obj
 0002:0000c120       ??_C@_0O@IABBPLOA@buttonClicked?$AA@ 10030120     cfg_widgets001:moc_config_mb4impl.obj
 0002:0000c13c       ??_C@_0BD@OMEOEKEF@buttonClicked?$CIint?$CJ?$AA@ 1003013c     cfg_widgets001:moc_config_mb4impl.obj
 0002:0000c150       ??_C@_0N@NAADDCIB@cfg_ListView?$AA@ 10030150     cfg_widgets001:moc_cfg_ListView.obj
 0002:0000c16c       ??_C@_0L@MLFJPJPC@insertData?$AA@ 1003016c     cfg_widgets001:moc_cfg_ListView.obj
 0002:0000c184       ??_C@_0M@MOKGOAHM@deleteItems?$AA@ 10030184     cfg_widgets001:moc_cfg_ListView.obj
 0002:0000c19c       ??_C@_0BA@FJBCKEJL@copyToClipboard?$AA@ 1003019c     cfg_widgets001:moc_cfg_ListView.obj
 0002:0000c1b8       ??_C@_09CLMPBHDI@undoPaste?$AA@ 100301b8     cfg_widgets001:moc_cfg_ListView.obj
 0002:0000c1d0       ??_C@_0M@NOBHHHJI@replaceData?$AA@ 100301d0     cfg_widgets001:moc_cfg_ListView.obj
 0002:0000c1e8       ??_C@_0BF@CDBOAHLL@clipBoardDataChanged?$AA@ 100301e8     cfg_widgets001:moc_cfg_ListView.obj
 0002:0000c248       ??_C@_0N@JAPDIKGN@insertData?$CI?$CJ?$AA@ 10030248     cfg_widgets001:moc_cfg_ListView.obj
 0002:0000c258       ??_C@_0O@FBJIJCJH@deleteItems?$CI?$CJ?$AA@ 10030258     cfg_widgets001:moc_cfg_ListView.obj
 0002:0000c268       ??_C@_0BC@DBBGOFIB@copyToClipboard?$CI?$CJ?$AA@ 10030268     cfg_widgets001:moc_cfg_ListView.obj
 0002:0000c27c       ??_C@_0M@OGFEJKEA@undoPaste?$CI?$CJ?$AA@ 1003027c     cfg_widgets001:moc_cfg_ListView.obj
 0002:0000c288       ??_C@_0O@FOBLCCJ@replaceData?$CI?$CJ?$AA@ 10030288     cfg_widgets001:moc_cfg_ListView.obj
 0002:0000c298       ??_C@_0BH@OLENEJHN@clipBoardDataChanged?$CI?$CJ?$AA@ 10030298     cfg_widgets001:moc_cfg_ListView.obj
 0002:0000c2bc       ??_C@_0L@OIBMJOP@dataPasted?$AA@ 100302bc     cfg_widgets001:moc_cfg_ListView.obj
 0002:0000c2d4       ??_C@_0BD@IALCIEJE@clipboardDataValid?$AA@ 100302d4     cfg_widgets001:moc_cfg_ListView.obj
 0002:0000c300       ??_C@_0N@EJEGBDAF@dataPasted?$CI?$CJ?$AA@ 10030300     cfg_widgets001:moc_cfg_ListView.obj
 0002:0000c310       ??_C@_0BJ@FABNKMFK@clipboardDataValid?$CIbool?$CJ?$AA@ 10030310     cfg_widgets001:moc_cfg_ListView.obj
 0002:0000c32c       ??_C@_09PNEKGGBK@cfg_Table?$AA@ 1003032c     cfg_widgets001:moc_cfg_Table.obj
 0002:0000c368       ??_C@_0P@FJGFLBMO@pasteClipboard?$AA@ 10030368     cfg_widgets001:moc_cfg_Table.obj
 0002:0000c3c0       ??_C@_0BB@JLAHKIAM@pasteClipboard?$CI?$CJ?$AA@ 100303c0     cfg_widgets001:moc_cfg_Table.obj
 0002:0000c408       ??_7type_info@@6B@         10030408     MSVCRT:ti_inst.obj
 0002:0000c40c       __pRawDllMain              1003040c     MSVCRT:crtdll.obj
 0002:0000c40c       __pDefaultRawDllMain       1003040c     MSVCRT:crtdll.obj
 0002:0000c418       __load_config_used         10030418     MSVCRT:loadcfg.obj
 0002:0000c460       ??_R4QWidget@@6BQObject@@@ 10030460     alm_process.obj
 0002:0000c474       ??_R3QWidget@@8            10030474     alm_process.obj
 0002:0000c484       ??_R2QWidget@@8            10030484     alm_process.obj
 0002:0000c498       ??_R1A@?0A@EA@QWidget@@8   10030498     alm_process.obj
 0002:0000c4b4       ??_R1A@?0A@EA@QObject@@8   100304b4     alm_process.obj
 0002:0000c4d0       ??_R3QObject@@8            100304d0     alm_process.obj
 0002:0000c4e0       ??_R2QObject@@8            100304e0     alm_process.obj
 0002:0000c4ec       ??_R13?0A@EA@Qt@@8         100304ec     alm_process.obj
 0002:0000c508       ??_R3Qt@@8                 10030508     alm_process.obj
 0002:0000c518       ??_R2Qt@@8                 10030518     alm_process.obj
 0002:0000c520       ??_R1A@?0A@EA@Qt@@8        10030520     alm_process.obj
 0002:0000c53c       ??_R1CI@?0A@EA@QPaintDevice@@8 1003053c     alm_process.obj
 0002:0000c558       ??_R3QPaintDevice@@8       10030558     alm_process.obj
 0002:0000c568       ??_R2QPaintDevice@@8       10030568     alm_process.obj
 0002:0000c570       ??_R1A@?0A@EA@QPaintDevice@@8 10030570     alm_process.obj
 0002:0000c58c       ??_R4QWidget@@6BQPaintDevice@@@ 1003058c     alm_process.obj
 0002:0000c5a0       ??_R3QShared@@8            100305a0     alm_process.obj
 0002:0000c5b0       ??_R2QShared@@8            100305b0     alm_process.obj
 0002:0000c5b8       ??_R1A@?0A@EA@QShared@@8   100305b8     alm_process.obj
 0002:0000c5d4       ??_R1A@?0A@EA@QGList@@8    100305d4     alm_process.obj
 0002:0000c5f0       ??_R3QGList@@8             100305f0     alm_process.obj
 0002:0000c600       ??_R2QGList@@8             10030600     alm_process.obj
 0002:0000c60c       ??_R1A@?0A@EA@QPtrCollection@@8 1003060c     alm_process.obj
 0002:0000c628       ??_R3QPtrCollection@@8     10030628     alm_process.obj
 0002:0000c638       ??_R2QPtrCollection@@8     10030638     alm_process.obj
 0002:0000c640       ??_R4QPushButton@@6BQObject@@@ 10030640     alm_process.obj
 0002:0000c654       ??_R3QPushButton@@8        10030654     alm_process.obj
 0002:0000c664       ??_R2QPushButton@@8        10030664     alm_process.obj
 0002:0000c680       ??_R1A@?0A@EA@QPushButton@@8 10030680     alm_process.obj
 0002:0000c69c       ??_R1A@?0A@EA@QButton@@8   1003069c     alm_process.obj
 0002:0000c6b8       ??_R3QButton@@8            100306b8     alm_process.obj
 0002:0000c6c8       ??_R2QButton@@8            100306c8     alm_process.obj
 0002:0000c6e0       ??_R4QPushButton@@6BQPaintDevice@@@ 100306e0     alm_process.obj
 0002:0000c6f4       ??_R4QLabel@@6BQObject@@@  100306f4     alm_process.obj
 0002:0000c708       ??_R3QLabel@@8             10030708     alm_process.obj
 0002:0000c718       ??_R2QLabel@@8             10030718     alm_process.obj
 0002:0000c734       ??_R1A@?0A@EA@QLabel@@8    10030734     alm_process.obj
 0002:0000c750       ??_R1A@?0A@EA@QFrame@@8    10030750     alm_process.obj
 0002:0000c76c       ??_R3QFrame@@8             1003076c     alm_process.obj
 0002:0000c77c       ??_R2QFrame@@8             1003077c     alm_process.obj
 0002:0000c794       ??_R4QLabel@@6BQPaintDevice@@@ 10030794     alm_process.obj
 0002:0000c7a8       ??_R4QPopupMenu@@6BQObject@@@ 100307a8     alm_process.obj
 0002:0000c7bc       ??_R3QPopupMenu@@8         100307bc     alm_process.obj
 0002:0000c7cc       ??_R2QPopupMenu@@8         100307cc     alm_process.obj
 0002:0000c7ec       ??_R1A@?0A@EA@QPopupMenu@@8 100307ec     alm_process.obj
 0002:0000c808       ??_R1IM@?0A@EA@QMenuData@@8 10030808     alm_process.obj
 0002:0000c824       ??_R3QMenuData@@8          10030824     alm_process.obj
 0002:0000c834       ??_R2QMenuData@@8          10030834     alm_process.obj
 0002:0000c83c       ??_R1A@?0A@EA@QMenuData@@8 1003083c     alm_process.obj
 0002:0000c858       ??_R4QPopupMenu@@6BQPaintDevice@@@ 10030858     alm_process.obj
 0002:0000c86c       ??_R4QPopupMenu@@6B@       1003086c     alm_process.obj
 0002:0000c880       ??_R4QAction@@6B@          10030880     alm_process.obj
 0002:0000c894       ??_R3QAction@@8            10030894     alm_process.obj
 0002:0000c8a4       ??_R2QAction@@8            100308a4     alm_process.obj
 0002:0000c8b4       ??_R1A@?0A@EA@QAction@@8   100308b4     alm_process.obj
 0002:0000c8d0       ??_R4QHBoxLayout@@6BQObject@@@ 100308d0     alm_process.obj
 0002:0000c8e4       ??_R3QHBoxLayout@@8        100308e4     alm_process.obj
 0002:0000c8f4       ??_R2QHBoxLayout@@8        100308f4     alm_process.obj
 0002:0000c910       ??_R1A@?0A@EA@QHBoxLayout@@8 10030910     alm_process.obj
 0002:0000c92c       ??_R1A@?0A@EA@QBoxLayout@@8 1003092c     alm_process.obj
 0002:0000c948       ??_R3QBoxLayout@@8         10030948     alm_process.obj
 0002:0000c958       ??_R2QBoxLayout@@8         10030958     alm_process.obj
 0002:0000c970       ??_R1A@?0A@EA@QLayout@@8   10030970     alm_process.obj
 0002:0000c98c       ??_R3QLayout@@8            1003098c     alm_process.obj
 0002:0000c99c       ??_R2QLayout@@8            1003099c     alm_process.obj
 0002:0000c9b0       ??_R1CI@?0A@EA@QLayoutItem@@8 100309b0     alm_process.obj
 0002:0000c9cc       ??_R3QLayoutItem@@8        100309cc     alm_process.obj
 0002:0000c9dc       ??_R2QLayoutItem@@8        100309dc     alm_process.obj
 0002:0000c9e4       ??_R1A@?0A@EA@QLayoutItem@@8 100309e4     alm_process.obj
 0002:0000ca00       ??_R4QHBoxLayout@@6BQLayoutItem@@@ 10030a00     alm_process.obj
 0002:0000ca14       ??_R4QVBoxLayout@@6BQObject@@@ 10030a14     alm_process.obj
 0002:0000ca28       ??_R3QVBoxLayout@@8        10030a28     alm_process.obj
 0002:0000ca38       ??_R2QVBoxLayout@@8        10030a38     alm_process.obj
 0002:0000ca54       ??_R1A@?0A@EA@QVBoxLayout@@8 10030a54     alm_process.obj
 0002:0000ca70       ??_R4QVBoxLayout@@6BQLayoutItem@@@ 10030a70     alm_process.obj
 0002:0000ca84       ??_R4QToolBar@@6BQObject@@@ 10030a84     alm_process.obj
 0002:0000ca98       ??_R3QToolBar@@8           10030a98     alm_process.obj
 0002:0000caa8       ??_R2QToolBar@@8           10030aa8     alm_process.obj
 0002:0000cac8       ??_R1A@?0A@EA@QToolBar@@8  10030ac8     alm_process.obj
 0002:0000cae4       ??_R1A@?0A@EA@QDockWindow@@8 10030ae4     alm_process.obj
 0002:0000cb00       ??_R3QDockWindow@@8        10030b00     alm_process.obj
 0002:0000cb10       ??_R2QDockWindow@@8        10030b10     alm_process.obj
 0002:0000cb2c       ??_R4QToolBar@@6BQPaintDevice@@@ 10030b2c     alm_process.obj
 0002:0000cb40       ??_R4QDockWindow@@6BQObject@@@ 10030b40     alm_process.obj
 0002:0000cb54       ??_R4QDockWindow@@6BQPaintDevice@@@ 10030b54     alm_process.obj
 0002:0000cb68       ??_R4QLineEdit@@6BQObject@@@ 10030b68     alm_process.obj
 0002:0000cb7c       ??_R3QLineEdit@@8          10030b7c     alm_process.obj
 0002:0000cb8c       ??_R2QLineEdit@@8          10030b8c     alm_process.obj
 0002:0000cba8       ??_R1A@?0A@EA@QLineEdit@@8 10030ba8     alm_process.obj
 0002:0000cbc4       ??_R4QLineEdit@@6BQPaintDevice@@@ 10030bc4     alm_process.obj
 0002:0000cbd8       ??_R4QListViewItem@@6B@    10030bd8     alm_process.obj
 0002:0000cbec       ??_R3QListViewItem@@8      10030bec     alm_process.obj
 0002:0000cbfc       ??_R2QListViewItem@@8      10030bfc     alm_process.obj
 0002:0000cc08       ??_R1A@?0A@EA@QListViewItem@@8 10030c08     alm_process.obj
 0002:0000cc24       ??_R4QTabWidget@@6BQObject@@@ 10030c24     alm_process.obj
 0002:0000cc38       ??_R3QTabWidget@@8         10030c38     alm_process.obj
 0002:0000cc48       ??_R2QTabWidget@@8         10030c48     alm_process.obj
 0002:0000cc60       ??_R1A@?0A@EA@QTabWidget@@8 10030c60     alm_process.obj
 0002:0000cc7c       ??_R4QTabWidget@@6BQPaintDevice@@@ 10030c7c     alm_process.obj
 0002:0000cc90       ??_R4QSpacerItem@@6B@      10030c90     alm_process.obj
 0002:0000cca4       ??_R3QSpacerItem@@8        10030ca4     alm_process.obj
 0002:0000ccb4       ??_R2QSpacerItem@@8        10030cb4     alm_process.obj
 0002:0000ccc0       ??_R1A@?0A@EA@QSpacerItem@@8 10030cc0     alm_process.obj
 0002:0000ccdc       ??_R4?$QPtrList@VQListViewItem@@@@6B@ 10030cdc     alm_process.obj
 0002:0000ccf0       ??_R3?$QPtrList@VQListViewItem@@@@8 10030cf0     alm_process.obj
 0002:0000cd00       ??_R2?$QPtrList@VQListViewItem@@@@8 10030d00     alm_process.obj
 0002:0000cd10       ??_R1A@?0A@EA@?$QPtrList@VQListViewItem@@@@8 10030d10     alm_process.obj
 0002:0000cd2c       ??_R4CAlm_sys_select@@6BQObject@@@ 10030d2c     alm_process.obj
 0002:0000cd40       ??_R3CAlm_sys_select@@8    10030d40     alm_process.obj
 0002:0000cd50       ??_R2CAlm_sys_select@@8    10030d50     alm_process.obj
 0002:0000cd74       ??_R1A@?0A@EA@CAlm_sys_select@@8 10030d74     alm_process.obj
 0002:0000cd90       ??_R1A@?0A@EA@QVBox@@8     10030d90     alm_process.obj
 0002:0000cdac       ??_R3QVBox@@8              10030dac     alm_process.obj
 0002:0000cdbc       ??_R2QVBox@@8              10030dbc     alm_process.obj
 0002:0000cddc       ??_R1A@?0A@EA@QHBox@@8     10030ddc     alm_process.obj
 0002:0000cdf8       ??_R3QHBox@@8              10030df8     alm_process.obj
 0002:0000ce08       ??_R2QHBox@@8              10030e08     alm_process.obj
 0002:0000ce24       ??_R4CAlm_sys_select@@6BQPaintDevice@@@ 10030e24     alm_process.obj
 0002:0000ce38       ??_R4QDockWindowList@@6B@  10030e38     alm_process.obj
 0002:0000ce4c       ??_R3QDockWindowList@@8    10030e4c     alm_process.obj
 0002:0000ce5c       ??_R2QDockWindowList@@8    10030e5c     alm_process.obj
 0002:0000ce70       ??_R1A@?0A@EA@QDockWindowList@@8 10030e70     alm_process.obj
 0002:0000ce8c       ??_R1A@?0A@EA@?$QPtrList@VQDockWindow@@@@8 10030e8c     alm_process.obj
 0002:0000cea8       ??_R3?$QPtrList@VQDockWindow@@@@8 10030ea8     alm_process.obj
 0002:0000ceb8       ??_R2?$QPtrList@VQDockWindow@@@@8 10030eb8     alm_process.obj
 0002:0000cec8       ??_R4QPopupMenuList@@6B@   10030ec8     alm_process.obj
 0002:0000cedc       ??_R3QPopupMenuList@@8     10030edc     alm_process.obj
 0002:0000ceec       ??_R2QPopupMenuList@@8     10030eec     alm_process.obj
 0002:0000cf00       ??_R1A@?0A@EA@QPopupMenuList@@8 10030f00     alm_process.obj
 0002:0000cf1c       ??_R1A@?0A@EA@?$QPtrList@VQPopupMenu@@@@8 10030f1c     alm_process.obj
 0002:0000cf38       ??_R3?$QPtrList@VQPopupMenu@@@@8 10030f38     alm_process.obj
 0002:0000cf48       ??_R2?$QPtrList@VQPopupMenu@@@@8 10030f48     alm_process.obj
 0002:0000cf58       ??_R4?$QPtrList@VQPopupMenu@@@@6B@ 10030f58     alm_process.obj
 0002:0000cf6c       ??_R4QGuardedPtrPrivate@@6B@ 10030f6c     alm_process.obj
 0002:0000cf80       ??_R3QGuardedPtrPrivate@@8 10030f80     alm_process.obj
 0002:0000cf90       ??_R2QGuardedPtrPrivate@@8 10030f90     alm_process.obj
 0002:0000cfa4       ??_R1A@?0A@EA@QGuardedPtrPrivate@@8 10030fa4     alm_process.obj
 0002:0000cfc0       ??_R1CI@?0A@EA@QShared@@8  10030fc0     alm_process.obj
 0002:0000cfdc       ??_R4config_plugin_base@@6BQObject@@@ 10030fdc     alm_process.obj
 0002:0000cff0       ??_R3config_plugin_base@@8 10030ff0     alm_process.obj
 0002:0000d000       ??_R2config_plugin_base@@8 10031000     alm_process.obj
 0002:0000d018       ??_R1A@?0A@EA@config_plugin_base@@8 10031018     alm_process.obj
 0002:0000d034       ??_R4config_plugin_base@@6BQPaintDevice@@@ 10031034     alm_process.obj
 0002:0000d048       ??_R4ProcessListView@@6BQObject@@@ 10031048     alm_process.obj
 0002:0000d05c       ??_R3ProcessListView@@8    1003105c     alm_process.obj
 0002:0000d06c       ??_R2ProcessListView@@8    1003106c     alm_process.obj
 0002:0000d090       ??_R1A@?0A@EA@ProcessListView@@8 10031090     alm_process.obj
 0002:0000d0ac       ??_R1A@?0A@EA@QListView@@8 100310ac     alm_process.obj
 0002:0000d0c8       ??_R3QListView@@8          100310c8     alm_process.obj
 0002:0000d0d8       ??_R2QListView@@8          100310d8     alm_process.obj
 0002:0000d0f8       ??_R1A@?0A@EA@QScrollView@@8 100310f8     alm_process.obj
 0002:0000d114       ??_R3QScrollView@@8        10031114     alm_process.obj
 0002:0000d124       ??_R2QScrollView@@8        10031124     alm_process.obj
 0002:0000d140       ??_R4ProcessListView@@6BQPaintDevice@@@ 10031140     alm_process.obj
 0002:0000d154       ??_R4ProcessListViewItem@@6B@ 10031154     alm_process.obj
 0002:0000d168       ??_R3ProcessListViewItem@@8 10031168     alm_process.obj
 0002:0000d178       ??_R2ProcessListViewItem@@8 10031178     alm_process.obj
 0002:0000d188       ??_R1A@?0A@EA@ProcessListViewItem@@8 10031188     alm_process.obj
 0002:0000d1a4       ??_R4alm_process@@6BQObject@@@ 100311a4     alm_process.obj
 0002:0000d1b8       ??_R3alm_process@@8        100311b8     alm_process.obj
 0002:0000d1c8       ??_R2alm_process@@8        100311c8     alm_process.obj
 0002:0000d1e4       ??_R1A@?0A@EA@alm_process@@8 100311e4     alm_process.obj
 0002:0000d200       ??_R4alm_process@@6BQPaintDevice@@@ 10031200     alm_process.obj
 0002:0000d214       ??_R4?$QPtrList@VcProcess@@@@6B@ 10031214     alm_process.obj
 0002:0000d228       ??_R3?$QPtrList@VcProcess@@@@8 10031228     alm_process.obj
 0002:0000d238       ??_R2?$QPtrList@VcProcess@@@@8 10031238     alm_process.obj
 0002:0000d248       ??_R1A@?0A@EA@?$QPtrList@VcProcess@@@@8 10031248     alm_process.obj
 0002:0000d264       ??_R4cAcqFileData@@6B@     10031264     cAcqFileData.obj
 0002:0000d278       ??_R3cAcqFileData@@8       10031278     cAcqFileData.obj
 0002:0000d288       ??_R2cAcqFileData@@8       10031288     cAcqFileData.obj
 0002:0000d290       ??_R1A@?0A@EA@cAcqFileData@@8 10031290     cAcqFileData.obj
 0002:0000d2ac       ??_R4CheckContDialog@@6BQObject@@@ 100312ac     checkContDialogImpl.obj
 0002:0000d2c0       ??_R3CheckContDialog@@8    100312c0     checkContDialogImpl.obj
 0002:0000d2d0       ??_R2CheckContDialog@@8    100312d0     checkContDialogImpl.obj
 0002:0000d2f0       ??_R1A@?0A@EA@CheckContDialog@@8 100312f0     checkContDialogImpl.obj
 0002:0000d30c       ??_R1A@?0A@EA@CheckContDialogBase@@8 1003130c     checkContDialogImpl.obj
 0002:0000d328       ??_R3CheckContDialogBase@@8 10031328     checkContDialogImpl.obj
 0002:0000d338       ??_R2CheckContDialogBase@@8 10031338     checkContDialogImpl.obj
 0002:0000d354       ??_R1A@?0A@EA@QDialog@@8   10031354     checkContDialogImpl.obj
 0002:0000d370       ??_R3QDialog@@8            10031370     checkContDialogImpl.obj
 0002:0000d380       ??_R2QDialog@@8            10031380     checkContDialogImpl.obj
 0002:0000d398       ??_R4CheckContDialog@@6BQPaintDevice@@@ 10031398     checkContDialogImpl.obj
 0002:0000d3ac       ??_R4QDoubleValidator@@6B@ 100313ac     cProc_dialog.obj
 0002:0000d3c0       ??_R3QDoubleValidator@@8   100313c0     cProc_dialog.obj
 0002:0000d3d0       ??_R2QDoubleValidator@@8   100313d0     cProc_dialog.obj
 0002:0000d3e4       ??_R1A@?0A@EA@QDoubleValidator@@8 100313e4     cProc_dialog.obj
 0002:0000d400       ??_R1A@?0A@EA@QValidator@@8 10031400     cProc_dialog.obj
 0002:0000d41c       ??_R3QValidator@@8         1003141c     cProc_dialog.obj
 0002:0000d42c       ??_R2QValidator@@8         1003142c     cProc_dialog.obj
 0002:0000d43c       ??_R4cProc_dialog@@6BQObject@@@ 1003143c     cProc_dialog.obj
 0002:0000d450       ??_R3cProc_dialog@@8       10031450     cProc_dialog.obj
 0002:0000d460       ??_R2cProc_dialog@@8       10031460     cProc_dialog.obj
 0002:0000d47c       ??_R1A@?0A@EA@cProc_dialog@@8 1003147c     cProc_dialog.obj
 0002:0000d498       ??_R1A@?0A@EA@proc_config@@8 10031498     cProc_dialog.obj
 0002:0000d4b4       ??_R3proc_config@@8        100314b4     cProc_dialog.obj
 0002:0000d4c4       ??_R2proc_config@@8        100314c4     cProc_dialog.obj
 0002:0000d4dc       ??_R4cProc_dialog@@6BQPaintDevice@@@ 100314dc     cProc_dialog.obj
 0002:0000d4f0       ??_R4ContributorListBoxItem@@6B@ 100314f0     cProc_dialog.obj
 0002:0000d504       ??_R3ContributorListBoxItem@@8 10031504     cProc_dialog.obj
 0002:0000d514       ??_R2ContributorListBoxItem@@8 10031514     cProc_dialog.obj
 0002:0000d524       ??_R1A@?0A@EA@ContributorListBoxItem@@8 10031524     cProc_dialog.obj
 0002:0000d540       ??_R1A@?0A@EA@QListBoxText@@8 10031540     cProc_dialog.obj
 0002:0000d55c       ??_R3QListBoxText@@8       1003155c     cProc_dialog.obj
 0002:0000d56c       ??_R2QListBoxText@@8       1003156c     cProc_dialog.obj
 0002:0000d578       ??_R1A@?0A@EA@QListBoxItem@@8 10031578     cProc_dialog.obj
 0002:0000d594       ??_R3QListBoxItem@@8       10031594     cProc_dialog.obj
 0002:0000d5a4       ??_R2QListBoxItem@@8       100315a4     cProc_dialog.obj
 0002:0000d5ac       ??_R1A@?0A@EA@QGDict@@8    100315ac     cProcess.obj
 0002:0000d5c8       ??_R3QGDict@@8             100315c8     cProcess.obj
 0002:0000d5d8       ??_R2QGDict@@8             100315d8     cProcess.obj
 0002:0000d5e4       ??_R4cProcess@@6B@         100315e4     cProcess.obj
 0002:0000d5f8       ??_R3cProcess@@8           100315f8     cProcess.obj
 0002:0000d608       ??_R2cProcess@@8           10031608     cProcess.obj
 0002:0000d610       ??_R1A@?0A@EA@cProcess@@8  10031610     cProcess.obj
 0002:0000d62c       ??_R4?$QDict@VQString@@@@6B@ 1003162c     cProcess.obj
 0002:0000d640       ??_R3?$QDict@VQString@@@@8 10031640     cProcess.obj
 0002:0000d650       ??_R2?$QDict@VQString@@@@8 10031650     cProcess.obj
 0002:0000d660       ??_R1A@?0A@EA@?$QDict@VQString@@@@8 10031660     cProcess.obj
 0002:0000d67c       ??_R4QListView@@6BQObject@@@ 1003167c     multiinput.obj
 0002:0000d690       ??_R4QListView@@6BQPaintDevice@@@ 10031690     multiinput.obj
 0002:0000d6a4       ??_R4multiInputBase@@6BQObject@@@ 100316a4     multiinput.obj
 0002:0000d6b8       ??_R3multiInputBase@@8     100316b8     multiinput.obj
 0002:0000d6c8       ??_R2multiInputBase@@8     100316c8     multiinput.obj
 0002:0000d6e4       ??_R1A@?0A@EA@multiInputBase@@8 100316e4     multiinput.obj
 0002:0000d700       ??_R4multiInputBase@@6BQPaintDevice@@@ 10031700     multiinput.obj
 0002:0000d714       ??_R4MultiInputInvalidListViewItem@@6B@ 10031714     multiinputimpl.obj
 0002:0000d728       ??_R3MultiInputInvalidListViewItem@@8 10031728     multiinputimpl.obj
 0002:0000d738       ??_R2MultiInputInvalidListViewItem@@8 10031738     multiinputimpl.obj
 0002:0000d748       ??_R1A@?0A@EA@MultiInputInvalidListViewItem@@8 10031748     multiinputimpl.obj
 0002:0000d764       ??_R4multiInput@@6BQObject@@@ 10031764     multiinputimpl.obj
 0002:0000d778       ??_R3multiInput@@8         10031778     multiinputimpl.obj
 0002:0000d788       ??_R2multiInput@@8         10031788     multiinputimpl.obj
 0002:0000d7a8       ??_R1A@?0A@EA@multiInput@@8 100317a8     multiinputimpl.obj
 0002:0000d7c4       ??_R4multiInput@@6BQPaintDevice@@@ 100317c4     multiinputimpl.obj
 0002:0000d7d8       ??_R4config_plugin_desc_base@@6B@ 100317d8     plugindesc.obj
 0002:0000d7ec       ??_R3config_plugin_desc_base@@8 100317ec     plugindesc.obj
 0002:0000d7fc       ??_R2config_plugin_desc_base@@8 100317fc     plugindesc.obj
 0002:0000d804       ??_R1A@?0A@EA@config_plugin_desc_base@@8 10031804     plugindesc.obj
 0002:0000d820       ??_R4plugindesc@@6B@       10031820     plugindesc.obj
 0002:0000d834       ??_R3plugindesc@@8         10031834     plugindesc.obj
 0002:0000d844       ??_R2plugindesc@@8         10031844     plugindesc.obj
 0002:0000d850       ??_R1A@?0A@EA@plugindesc@@8 10031850     plugindesc.obj
 0002:0000d86c       ??_R4singleInputBase@@6BQObject@@@ 1003186c     singleinput.obj
 0002:0000d880       ??_R3singleInputBase@@8    10031880     singleinput.obj
 0002:0000d890       ??_R2singleInputBase@@8    10031890     singleinput.obj
 0002:0000d8ac       ??_R1A@?0A@EA@singleInputBase@@8 100318ac     singleinput.obj
 0002:0000d8c8       ??_R4singleInputBase@@6BQPaintDevice@@@ 100318c8     singleinput.obj
 0002:0000d8dc       ??_R4singleInput@@6BQObject@@@ 100318dc     singleinputimpl.obj
 0002:0000d8f0       ??_R3singleInput@@8        100318f0     singleinputimpl.obj
 0002:0000d900       ??_R2singleInput@@8        10031900     singleinputimpl.obj
 0002:0000d920       ??_R1A@?0A@EA@singleInput@@8 10031920     singleinputimpl.obj
 0002:0000d93c       ??_R4singleInput@@6BQPaintDevice@@@ 1003193c     singleinputimpl.obj
 0002:0000d950       ??_R4QGridLayout@@6BQObject@@@ 10031950     template_dialog.obj
 0002:0000d964       ??_R3QGridLayout@@8        10031964     template_dialog.obj
 0002:0000d974       ??_R2QGridLayout@@8        10031974     template_dialog.obj
 0002:0000d98c       ??_R1A@?0A@EA@QGridLayout@@8 1003198c     template_dialog.obj
 0002:0000d9a8       ??_R4QGridLayout@@6BQLayoutItem@@@ 100319a8     template_dialog.obj
 0002:0000d9bc       ??_R4QCheckBox@@6BQObject@@@ 100319bc     template_dialog.obj
 0002:0000d9d0       ??_R3QCheckBox@@8          100319d0     template_dialog.obj
 0002:0000d9e0       ??_R2QCheckBox@@8          100319e0     template_dialog.obj
 0002:0000d9fc       ??_R1A@?0A@EA@QCheckBox@@8 100319fc     template_dialog.obj
 0002:0000da18       ??_R4QCheckBox@@6BQPaintDevice@@@ 10031a18     template_dialog.obj
 0002:0000da2c       ??_R4QSpinBox@@6BQObject@@@ 10031a2c     template_dialog.obj
 0002:0000da40       ??_R3QSpinBox@@8           10031a40     template_dialog.obj
 0002:0000da50       ??_R2QSpinBox@@8           10031a50     template_dialog.obj
 0002:0000da6c       ??_R1A@?0A@EA@QSpinBox@@8  10031a6c     template_dialog.obj
 0002:0000da88       ??_R1GM@?0A@EA@QRangeControl@@8 10031a88     template_dialog.obj
 0002:0000daa4       ??_R3QRangeControl@@8      10031aa4     template_dialog.obj
 0002:0000dab4       ??_R2QRangeControl@@8      10031ab4     template_dialog.obj
 0002:0000dabc       ??_R1A@?0A@EA@QRangeControl@@8 10031abc     template_dialog.obj
 0002:0000dad8       ??_R4QSpinBox@@6BQPaintDevice@@@ 10031ad8     template_dialog.obj
 0002:0000daec       ??_R4QSpinBox@@6B@         10031aec     template_dialog.obj
 0002:0000db00       ??_R4QButtonGroup@@6BQObject@@@ 10031b00     template_dialog.obj
 0002:0000db14       ??_R3QButtonGroup@@8       10031b14     template_dialog.obj
 0002:0000db24       ??_R2QButtonGroup@@8       10031b24     template_dialog.obj
 0002:0000db44       ??_R1A@?0A@EA@QButtonGroup@@8 10031b44     template_dialog.obj
 0002:0000db60       ??_R1A@?0A@EA@QGroupBox@@8 10031b60     template_dialog.obj
 0002:0000db7c       ??_R3QGroupBox@@8          10031b7c     template_dialog.obj
 0002:0000db8c       ??_R2QGroupBox@@8          10031b8c     template_dialog.obj
 0002:0000dba8       ??_R4QButtonGroup@@6BQPaintDevice@@@ 10031ba8     template_dialog.obj
 0002:0000dbbc       ??_R4QRadioButton@@6BQObject@@@ 10031bbc     template_dialog.obj
 0002:0000dbd0       ??_R3QRadioButton@@8       10031bd0     template_dialog.obj
 0002:0000dbe0       ??_R2QRadioButton@@8       10031be0     template_dialog.obj
 0002:0000dbfc       ??_R1A@?0A@EA@QRadioButton@@8 10031bfc     template_dialog.obj
 0002:0000dc18       ??_R4QRadioButton@@6BQPaintDevice@@@ 10031c18     template_dialog.obj
 0002:0000dc2c       ??_R4template_dialogBase@@6BQObject@@@ 10031c2c     template_dialog.obj
 0002:0000dc40       ??_R3template_dialogBase@@8 10031c40     template_dialog.obj
 0002:0000dc50       ??_R2template_dialogBase@@8 10031c50     template_dialog.obj
 0002:0000dc6c       ??_R1A@?0A@EA@template_dialogBase@@8 10031c6c     template_dialog.obj
 0002:0000dc88       ??_R4template_dialogBase@@6BQPaintDevice@@@ 10031c88     template_dialog.obj
 0002:0000dc9c       ??_R4template_dialog@@6BQObject@@@ 10031c9c     template_dialogimpl.obj
 0002:0000dcb0       ??_R3template_dialog@@8    10031cb0     template_dialogimpl.obj
 0002:0000dcc0       ??_R2template_dialog@@8    10031cc0     template_dialogimpl.obj
 0002:0000dce0       ??_R1A@?0A@EA@template_dialog@@8 10031ce0     template_dialogimpl.obj
 0002:0000dcfc       ??_R4template_dialog@@6BQPaintDevice@@@ 10031cfc     template_dialogimpl.obj
 0002:0000dd10       ??_R4CheckContDialogBase@@6BQObject@@@ 10031d10     checkcontributiondialog.obj
 0002:0000dd24       ??_R4CheckContDialogBase@@6BQPaintDevice@@@ 10031d24     checkcontributiondialog.obj
 0002:0000dd38       ??_R4LatchAckDialogBase@@6BQObject@@@ 10031d38     latchackdialog.obj
 0002:0000dd4c       ??_R3LatchAckDialogBase@@8 10031d4c     latchackdialog.obj
 0002:0000dd5c       ??_R2LatchAckDialogBase@@8 10031d5c     latchackdialog.obj
 0002:0000dd78       ??_R1A@?0A@EA@LatchAckDialogBase@@8 10031d78     latchackdialog.obj
 0002:0000dd94       ??_R4LatchAckDialogBase@@6BQPaintDevice@@@ 10031d94     latchackdialog.obj
 0002:0000dda8       ??_R4LatchAckDialog@@6BQObject@@@ 10031da8     latchackdialogimpl.obj
 0002:0000ddbc       ??_R3LatchAckDialog@@8     10031dbc     latchackdialogimpl.obj
 0002:0000ddcc       ??_R2LatchAckDialog@@8     10031dcc     latchackdialogimpl.obj
 0002:0000ddec       ??_R1A@?0A@EA@LatchAckDialog@@8 10031dec     latchackdialogimpl.obj
 0002:0000de08       ??_R4LatchAckDialog@@6BQPaintDevice@@@ 10031e08     latchackdialogimpl.obj
 0002:0000de1c       ??_R4QSplitter@@6BQObject@@@ 10031e1c     proc_config.obj
 0002:0000de30       ??_R3QSplitter@@8          10031e30     proc_config.obj
 0002:0000de40       ??_R2QSplitter@@8          10031e40     proc_config.obj
 0002:0000de5c       ??_R1A@?0A@EA@QSplitter@@8 10031e5c     proc_config.obj
 0002:0000de78       ??_R4QSplitter@@6BQPaintDevice@@@ 10031e78     proc_config.obj
 0002:0000de8c       ??_R4QComboBox@@6BQObject@@@ 10031e8c     proc_config.obj
 0002:0000dea0       ??_R3QComboBox@@8          10031ea0     proc_config.obj
 0002:0000deb0       ??_R2QComboBox@@8          10031eb0     proc_config.obj
 0002:0000dec8       ??_R1A@?0A@EA@QComboBox@@8 10031ec8     proc_config.obj
 0002:0000dee4       ??_R4QComboBox@@6BQPaintDevice@@@ 10031ee4     proc_config.obj
 0002:0000def8       ??_R4QGroupBox@@6BQObject@@@ 10031ef8     proc_config.obj
 0002:0000df0c       ??_R4QGroupBox@@6BQPaintDevice@@@ 10031f0c     proc_config.obj
 0002:0000df20       ??_R4QWidgetStack@@6BQObject@@@ 10031f20     proc_config.obj
 0002:0000df34       ??_R3QWidgetStack@@8       10031f34     proc_config.obj
 0002:0000df44       ??_R2QWidgetStack@@8       10031f44     proc_config.obj
 0002:0000df60       ??_R1A@?0A@EA@QWidgetStack@@8 10031f60     proc_config.obj
 0002:0000df7c       ??_R4QWidgetStack@@6BQPaintDevice@@@ 10031f7c     proc_config.obj
 0002:0000df90       ??_R4QListBox@@6BQObject@@@ 10031f90     proc_config.obj
 0002:0000dfa4       ??_R3QListBox@@8           10031fa4     proc_config.obj
 0002:0000dfb4       ??_R2QListBox@@8           10031fb4     proc_config.obj
 0002:0000dfd4       ??_R1A@?0A@EA@QListBox@@8  10031fd4     proc_config.obj
 0002:0000dff0       ??_R4QListBox@@6BQPaintDevice@@@ 10031ff0     proc_config.obj
 0002:0000e004       ??_R4QTimeEdit@@6BQObject@@@ 10032004     proc_config.obj
 0002:0000e018       ??_R3QTimeEdit@@8          10032018     proc_config.obj
 0002:0000e028       ??_R2QTimeEdit@@8          10032028     proc_config.obj
 0002:0000e044       ??_R1A@?0A@EA@QTimeEdit@@8 10032044     proc_config.obj
 0002:0000e060       ??_R1A@?0A@EA@QDateTimeEditBase@@8 10032060     proc_config.obj
 0002:0000e07c       ??_R3QDateTimeEditBase@@8  1003207c     proc_config.obj
 0002:0000e08c       ??_R2QDateTimeEditBase@@8  1003208c     proc_config.obj
 0002:0000e0a4       ??_R4QTimeEdit@@6BQPaintDevice@@@ 100320a4     proc_config.obj
 0002:0000e0b8       ??_R4QTextEdit@@6BQObject@@@ 100320b8     proc_config.obj
 0002:0000e0cc       ??_R3QTextEdit@@8          100320cc     proc_config.obj
 0002:0000e0dc       ??_R2QTextEdit@@8          100320dc     proc_config.obj
 0002:0000e0fc       ??_R1A@?0A@EA@QTextEdit@@8 100320fc     proc_config.obj
 0002:0000e118       ??_R4QTextEdit@@6BQPaintDevice@@@ 10032118     proc_config.obj
 0002:0000e12c       ??_R4proc_config@@6BQObject@@@ 1003212c     proc_config.obj
 0002:0000e140       ??_R4proc_config@@6BQPaintDevice@@@ 10032140     proc_config.obj
 0002:0000e154       ??_R4config_mb4@@6BQObject@@@ 10032154     cfg_widgets001:config_mb4impl.obj
 0002:0000e168       ??_R3config_mb4@@8         10032168     cfg_widgets001:config_mb4impl.obj
 0002:0000e178       ??_R2config_mb4@@8         10032178     cfg_widgets001:config_mb4impl.obj
 0002:0000e194       ??_R1A@?0A@EA@config_mb4@@8 10032194     cfg_widgets001:config_mb4impl.obj
 0002:0000e1b0       ??_R4config_mb4@@6BQPaintDevice@@@ 100321b0     cfg_widgets001:config_mb4impl.obj
 0002:0000e1c4       ??_R4cfg_ListView@@6BQObject@@@ 100321c4     cfg_widgets001:cfg_ListView.obj
 0002:0000e1d8       ??_R3cfg_ListView@@8       100321d8     cfg_widgets001:cfg_ListView.obj
 0002:0000e1e8       ??_R2cfg_ListView@@8       100321e8     cfg_widgets001:cfg_ListView.obj
 0002:0000e20c       ??_R1A@?0A@EA@cfg_ListView@@8 1003220c     cfg_widgets001:cfg_ListView.obj
 0002:0000e228       ??_R4cfg_ListView@@6BQPaintDevice@@@ 10032228     cfg_widgets001:cfg_ListView.obj
 0002:0000e23c       ??_R4cfg_Table@@6BQObject@@@ 1003223c     cfg_widgets001:cfg_Table.obj
 0002:0000e250       ??_R3cfg_Table@@8          10032250     cfg_widgets001:cfg_Table.obj
 0002:0000e260       ??_R2cfg_Table@@8          10032260     cfg_widgets001:cfg_Table.obj
 0002:0000e284       ??_R1A@?0A@EA@cfg_Table@@8 10032284     cfg_widgets001:cfg_Table.obj
 0002:0000e2a0       ??_R1A@?0A@EA@QTable@@8    100322a0     cfg_widgets001:cfg_Table.obj
 0002:0000e2bc       ??_R3QTable@@8             100322bc     cfg_widgets001:cfg_Table.obj
 0002:0000e2cc       ??_R2QTable@@8             100322cc     cfg_widgets001:cfg_Table.obj
 0002:0000e2ec       ??_R4cfg_Table@@6BQPaintDevice@@@ 100322ec     cfg_widgets001:cfg_Table.obj
 0002:0000e300       ??_R4type_info@@6B@        10032300     MSVCRT:ti_inst.obj
 0002:0000e314       ??_R3type_info@@8          10032314     MSVCRT:ti_inst.obj
 0002:0000e324       ??_R2type_info@@8          10032324     MSVCRT:ti_inst.obj
 0002:0000e32c       ??_R1A@?0A@EA@type_info@@8 1003232c     MSVCRT:ti_inst.obj
 0002:0000e348       ___rtc_iaa                 10032348     MSVCRT:initsect.obj
 0002:0000e34c       ___rtc_izz                 1003234c     MSVCRT:initsect.obj
 0002:0000e350       ___rtc_taa                 10032350     MSVCRT:initsect.obj
 0002:0000e354       ___rtc_tzz                 10032354     MSVCRT:initsect.obj
 0002:00013130       __IMPORT_DESCRIPTOR_qt-mt323 10037130     qt-mt323:qt-mt323.dll
 0002:00013144       __IMPORT_DESCRIPTOR_alm_sys_select 10037144     alm_sys_select:alm_sys_select.dll
 0002:00013158       __IMPORT_DESCRIPTOR_config_icons 10037158     config_icons:config_icons.dll
 0002:0001316c       __IMPORT_DESCRIPTOR_KERNEL32 1003716c     kernel32:KERNEL32.dll
 0002:00013180       __IMPORT_DESCRIPTOR_MSVCP120 10037180     msvcprt:MSVCP120.dll
 0002:00013194       __IMPORT_DESCRIPTOR_MSVCR120 10037194     MSVCRT:MSVCR120.dll
 0002:000131a8       __NULL_IMPORT_DESCRIPTOR   100371a8     qt-mt323:qt-mt323.dll
 0003:000000a4       ?dialogSize@multiInput@@0VQSize@@A 100480a4     multiinputimpl.obj
 0003:000000fc       ?sm_bReplace@template_dialog@@0_NA 100480fc     template_dialogimpl.obj
 0003:000000fd       ?sm_bKeepRelations@template_dialog@@0_NA 100480fd     template_dialogimpl.obj
 0003:00000370       ___security_cookie         10048370     MSVCRT:gs_cookie.obj
 0003:00000374       ___security_cookie_complement 10048374     MSVCRT:gs_cookie.obj
 0003:00000378       ___native_dllmain_reason   10048378     MSVCRT:natstart.obj
 0003:0000037c       ??_R0?AVQListViewItem@@@8  1004837c     alm_process.obj
 0003:00000398       ??_R0?AVProcessListViewItem@@@8 10048398     alm_process.obj
 0003:000003bc       ??_R0?AVQWidget@@@8        100483bc     alm_process.obj
 0003:000003d4       ??_R0?AVQObject@@@8        100483d4     alm_process.obj
 0003:000003ec       ??_R0?AVQt@@@8             100483ec     alm_process.obj
 0003:00000400       ??_R0?AVQPaintDevice@@@8   10048400     alm_process.obj
 0003:0000041c       ??_R0?AUQShared@@@8        1004841c     alm_process.obj
 0003:00000434       ??_R0?AVQGList@@@8         10048434     alm_process.obj
 0003:0000044c       ??_R0?AVQPtrCollection@@@8 1004844c     alm_process.obj
 0003:0000046c       ??_R0?AVQPushButton@@@8    1004846c     alm_process.obj
 0003:00000488       ??_R0?AVQButton@@@8        10048488     alm_process.obj
 0003:000004a0       ??_R0?AVQLabel@@@8         100484a0     alm_process.obj
 0003:000004b8       ??_R0?AVQFrame@@@8         100484b8     alm_process.obj
 0003:000004d0       ??_R0?AVQPopupMenu@@@8     100484d0     alm_process.obj
 0003:000004ec       ??_R0?AVQMenuData@@@8      100484ec     alm_process.obj
 0003:00000504       ??_R0?AVQAction@@@8        10048504     alm_process.obj
 0003:0000051c       ??_R0?AVQHBoxLayout@@@8    1004851c     alm_process.obj
 0003:00000538       ??_R0?AVQBoxLayout@@@8     10048538     alm_process.obj
 0003:00000554       ??_R0?AVQLayout@@@8        10048554     alm_process.obj
 0003:0000056c       ??_R0?AVQLayoutItem@@@8    1004856c     alm_process.obj
 0003:00000588       ??_R0?AVQVBoxLayout@@@8    10048588     alm_process.obj
 0003:000005a4       ??_R0?AVQToolBar@@@8       100485a4     alm_process.obj
 0003:000005bc       ??_R0?AVQDockWindow@@@8    100485bc     alm_process.obj
 0003:000005d8       ??_R0?AVQLineEdit@@@8      100485d8     alm_process.obj
 0003:000005f0       ??_R0?AVQTabWidget@@@8     100485f0     alm_process.obj
 0003:0000060c       ??_R0?AVQSpacerItem@@@8    1004860c     alm_process.obj
 0003:00000628       ??_R0?AV?$QPtrList@VQListViewItem@@@@@8 10048628     alm_process.obj
 0003:00000654       ??_R0?AVCAlm_sys_select@@@8 10048654     alm_process.obj
 0003:00000674       ??_R0?AVQVBox@@@8          10048674     alm_process.obj
 0003:00000688       ??_R0?AVQHBox@@@8          10048688     alm_process.obj
 0003:0000069c       ??_R0?AVQDockWindowList@@@8 1004869c     alm_process.obj
 0003:000006bc       ??_R0?AV?$QPtrList@VQDockWindow@@@@@8 100486bc     alm_process.obj
 0003:000006e4       ??_R0?AVQPopupMenuList@@@8 100486e4     alm_process.obj
 0003:00000704       ??_R0?AV?$QPtrList@VQPopupMenu@@@@@8 10048704     alm_process.obj
 0003:0000072c       ??_R0?AVQGuardedPtrPrivate@@@8 1004872c     alm_process.obj
 0003:00000750       ??_R0?AVconfig_plugin_base@@@8 10048750     alm_process.obj
 0003:00000774       ??_R0?AVProcessListView@@@8 10048774     alm_process.obj
 0003:00000794       ??_R0?AVQListView@@@8      10048794     alm_process.obj
 0003:000007ac       ??_R0?AVQScrollView@@@8    100487ac     alm_process.obj
 0003:000007c8       ??_R0?AValm_process@@@8    100487c8     alm_process.obj
 0003:000007e4       ??_R0?AV?$QPtrList@VcProcess@@@@@8 100487e4     alm_process.obj
 0003:0000080c       ??_R0?AVcAcqFileData@@@8   1004880c     cAcqFileData.obj
 0003:00000828       ??_R0?AVCheckContDialog@@@8 10048828     checkContDialogImpl.obj
 0003:00000848       ??_R0?AVCheckContDialogBase@@@8 10048848     checkContDialogImpl.obj
 0003:0000086c       ??_R0?AVQDialog@@@8        1004886c     checkContDialogImpl.obj
 0003:00000884       ??_R0?AVQDoubleValidator@@@8 10048884     cProc_dialog.obj
 0003:000008a4       ??_R0?AVQValidator@@@8     100488a4     cProc_dialog.obj
 0003:000008c0       ??_R0?AVcProc_dialog@@@8   100488c0     cProc_dialog.obj
 0003:000008dc       ??_R0?AVproc_config@@@8    100488dc     cProc_dialog.obj
 0003:000008f8       ??_R0?AVContributorListBoxItem@@@8 100488f8     cProc_dialog.obj
 0003:00000920       ??_R0?AVQListBoxText@@@8   10048920     cProc_dialog.obj
 0003:0000093c       ??_R0?AVQListBoxItem@@@8   1004893c     cProc_dialog.obj
 0003:00000958       ??_R0?AVQGDict@@@8         10048958     cProcess.obj
 0003:00000970       ??_R0?AVcProcess@@@8       10048970     cProcess.obj
 0003:00000988       ??_R0?AV?$QDict@VQString@@@@@8 10048988     cProcess.obj
 0003:000009ac       ??_R0?AVmultiInputBase@@@8 100489ac     multiinput.obj
 0003:000009cc       ??_R0?AVMultiInputInvalidListViewItem@@@8 100489cc     multiinputimpl.obj
 0003:000009f8       ??_R0?AVmultiInput@@@8     100489f8     multiinputimpl.obj
 0003:00000a14       ??_R0?AVconfig_plugin_desc_base@@@8 10048a14     plugindesc.obj
 0003:00000a3c       ??_R0?AVplugindesc@@@8     10048a3c     plugindesc.obj
 0003:00000a58       ??_R0?AVsingleInputBase@@@8 10048a58     singleinput.obj
 0003:00000a78       ??_R0?AVsingleInput@@@8    10048a78     singleinputimpl.obj
 0003:00000a94       ??_R0?AVQGridLayout@@@8    10048a94     template_dialog.obj
 0003:00000ab0       ??_R0?AVQCheckBox@@@8      10048ab0     template_dialog.obj
 0003:00000ac8       ??_R0?AVQSpinBox@@@8       10048ac8     template_dialog.obj
 0003:00000ae0       ??_R0?AVQRangeControl@@@8  10048ae0     template_dialog.obj
 0003:00000afc       ??_R0?AVQButtonGroup@@@8   10048afc     template_dialog.obj
 0003:00000b18       ??_R0?AVQGroupBox@@@8      10048b18     template_dialog.obj
 0003:00000b30       ??_R0?AVQRadioButton@@@8   10048b30     template_dialog.obj
 0003:00000b4c       ??_R0?AVtemplate_dialogBase@@@8 10048b4c     template_dialog.obj
 0003:00000b70       ??_R0?AVtemplate_dialog@@@8 10048b70     template_dialogimpl.obj
 0003:00000b90       ??_R0?AVLatchAckDialogBase@@@8 10048b90     latchackdialog.obj
 0003:00000bb4       ??_R0?AVLatchAckDialog@@@8 10048bb4     latchackdialogimpl.obj
 0003:00000bd4       ??_R0?AVQSplitter@@@8      10048bd4     proc_config.obj
 0003:00000bec       ??_R0?AVQComboBox@@@8      10048bec     proc_config.obj
 0003:00000c04       ??_R0?AVQWidgetStack@@@8   10048c04     proc_config.obj
 0003:00000c20       ??_R0?AVQListBox@@@8       10048c20     proc_config.obj
 0003:00000c38       ??_R0?AVQTimeEdit@@@8      10048c38     proc_config.obj
 0003:00000c50       ??_R0?AVQDateTimeEditBase@@@8 10048c50     proc_config.obj
 0003:00000c70       ??_R0?AVQTextEdit@@@8      10048c70     proc_config.obj
 0003:00000c88       ??_R0?AVconfig_mb4@@@8     10048c88     cfg_widgets001:config_mb4impl.obj
 0003:00000ca4       ??_R0?AVcfg_ListView@@@8   10048ca4     cfg_widgets001:cfg_ListView.obj
 0003:00000cc0       ??_R0?AVcfg_Table@@@8      10048cc0     cfg_widgets001:cfg_Table.obj
 0003:00000cd8       ??_R0?AVQTable@@@8         10048cd8     cfg_widgets001:cfg_Table.obj
 0003:00000cf0       ??_R0?AVtype_info@@@8      10048cf0     MSVCRT:ti_inst.obj
 0003:00000d0c       ?ProcConfig@@3V?$map@VQString@@PAVcProcess@@U?$less@VQString@@@std@@V?$allocator@U?$pair@$$CBVQString@@PAVcProcess@@@std@@@4@@std@@A 10048d0c     alm_process.obj
 0003:00000d18       ?acqEditor@@3V?$QMap@HPAVcAcqFileData@@@@A 10048d18     cProc_dialog.obj
 0003:00000d20       ?procList@cProcess@@2VQStringList@@A 10048d20     cProcess.obj
 0003:00000d30       ?sm_sPrefix@template_dialog@@0VQString@@A 10048d30     template_dialogimpl.obj
 0003:00000d34       ?sm_sSuffix@template_dialog@@0VQString@@A 10048d34     template_dialogimpl.obj
 0003:00000d38       ?metaObj@alm_process@@0PAVQMetaObject@@A 10048d38     moc_alm_process.obj
 0003:00000d84       ?metaObj@CheckContDialog@@0PAVQMetaObject@@A 10048d84     moc_checkContDialogImpl.obj
 0003:00000d8c       ?metaObj@CheckContDialogBase@@0PAVQMetaObject@@A 10048d8c     moc_checkcontributiondialog.obj
 0003:00000d94       ?metaObj@cProc_dialog@@0PAVQMetaObject@@A 10048d94     moc_cProc_dialog.obj
 0003:00000dd0       ?metaObj@LatchAckDialogBase@@0PAVQMetaObject@@A 10048dd0     moc_latchackdialog.obj
 0003:00000dd8       ?metaObj@LatchAckDialog@@0PAVQMetaObject@@A 10048dd8     moc_latchackdialogimpl.obj
 0003:00000de0       ?metaObj@multiInputBase@@0PAVQMetaObject@@A 10048de0     moc_multiinput.obj
 0003:00000de8       ?metaObj@multiInput@@0PAVQMetaObject@@A 10048de8     moc_multiinputimpl.obj
 0003:00000e08       ?metaObj@proc_config@@0PAVQMetaObject@@A 10048e08     moc_proc_config.obj
 0003:00000e10       ?metaObj@singleInputBase@@0PAVQMetaObject@@A 10048e10     moc_singleinput.obj
 0003:00000e18       ?metaObj@singleInput@@0PAVQMetaObject@@A 10048e18     moc_singleinputimpl.obj
 0003:00000e28       ?metaObj@template_dialogBase@@0PAVQMetaObject@@A 10048e28     moc_template_dialog.obj
 0003:00000e30       ?metaObj@template_dialog@@0PAVQMetaObject@@A 10048e30     moc_template_dialogimpl.obj
 0003:00000e50       ?metaObj@config_mb4@@0PAVQMetaObject@@A 10048e50     cfg_widgets001:moc_config_mb4impl.obj
 0003:00000e5c       ?metaObj@cfg_ListView@@0PAVQMetaObject@@A 10048e5c     cfg_widgets001:moc_cfg_ListView.obj
 0003:00000e78       ?metaObj@cfg_Table@@0PAVQMetaObject@@A 10048e78     cfg_widgets001:moc_cfg_Table.obj
 0003:000011b8       ?__type_info_root_node@@3U__type_info_node@@A 100491b8     MSVCRT:tncleanup.obj
 0003:000011c0       ___native_startup_lock     100491c0     <common>
 0003:000011c4       ___native_startup_state    100491c4     <common>
 0003:000011c8       ___dyn_tls_init_callback   100491c8     <common>
 0003:000011cc       ___onexitend               100491cc     <common>
 0003:000011d0       ___onexitbegin             100491d0     <common>

 entry point at        0001:0001dca8

 Static symbols

 0001:00000000       ??__EProcConfig@@YAXXZ     10001000 f   alm_process.obj
 0001:0000001b       ??__EacqEditor@@YAXXZ      1000101b f   cProc_dialog.obj
 0001:00000031       ??__E?procList@cProcess@@2VQStringList@@A@@YAXXZ 10001031 f   cProcess.obj
 0001:00000048       ??__E?sm_sPrefix@template_dialog@@0VQString@@A@@YAXXZ 10001048 f   template_dialogimpl.obj
 0001:0000006c       ??__E?sm_sSuffix@template_dialog@@0VQString@@A@@YAXXZ 1000106c f   template_dialogimpl.obj
 0001:00000090       ??__EcleanUp_alm_process@@YAXXZ 10001090 f   moc_alm_process.obj
 0001:000000b1       ??__EcleanUp_CheckContDialog@@YAXXZ 100010b1 f   moc_checkContDialogImpl.obj
 0001:000000d2       ??__EcleanUp_CheckContDialogBase@@YAXXZ 100010d2 f   moc_checkcontributiondialog.obj
 0001:000000f3       ??__EcleanUp_cProc_dialog@@YAXXZ 100010f3 f   moc_cProc_dialog.obj
 0001:00000114       ??__EcleanUp_LatchAckDialogBase@@YAXXZ 10001114 f   moc_latchackdialog.obj
 0001:00000135       ??__EcleanUp_LatchAckDialog@@YAXXZ 10001135 f   moc_latchackdialogimpl.obj
 0001:00000156       ??__EcleanUp_multiInputBase@@YAXXZ 10001156 f   moc_multiinput.obj
 0001:00000177       ??__EcleanUp_multiInput@@YAXXZ 10001177 f   moc_multiinputimpl.obj
 0001:00000198       ??__EcleanUp_proc_config@@YAXXZ 10001198 f   moc_proc_config.obj
 0001:000001b9       ??__EcleanUp_singleInputBase@@YAXXZ 100011b9 f   moc_singleinput.obj
 0001:000001da       ??__EcleanUp_singleInput@@YAXXZ 100011da f   moc_singleinputimpl.obj
 0001:000001fb       ??__EcleanUp_template_dialogBase@@YAXXZ 100011fb f   moc_template_dialog.obj
 0001:0000021c       ??__EcleanUp_template_dialog@@YAXXZ 1000121c f   moc_template_dialogimpl.obj
 0001:0000023d       ??__EcleanUp_config_mb4@@YAXXZ 1000123d f   cfg_widgets001:moc_config_mb4impl.obj
 0001:0000025e       ??__EcleanUp_cfg_ListView@@YAXXZ 1000125e f   cfg_widgets001:moc_cfg_ListView.obj
 0001:0000027f       ??__EcleanUp_cfg_Table@@YAXXZ 1000127f f   cfg_widgets001:moc_cfg_Table.obj
 0001:0000030b       __catch$??$_Buynode@ABUpiecewise_construct_t@std@@V?$tuple@ABVQString@@@2@V?$tuple@$$$V@2@@?$_Tree_buy@U?$pair@$$CBVQString@@PAVcProcess@@@std@@V?$allocator@U?$pair@$$CBVQString@@PAVcProcess@@@std@@@2@@std@@QAEPAU?$_Tree_node@U?$pair@$$CBVQString@@PAVcProcess@@@std@@PAX@1@ABUpiecewise_construct_t@1@$$QAV?$tuple@ABVQString@@@1@$$QAV?$tuple@$$$V@1@@Z$0 1000130b f i alm_process.obj
 0001:0000030b       __catch$??$_Buynode@ABUpiecewise_construct_t@std@@V?$tuple@$$QAVQString@@@2@V?$tuple@$$$V@2@@?$_Tree_buy@U?$pair@$$CBVQString@@PAVcProcess@@@std@@V?$allocator@U?$pair@$$CBVQString@@PAVcProcess@@@std@@@2@@std@@QAEPAU?$_Tree_node@U?$pair@$$CBVQString@@PAVcProcess@@@std@@PAX@1@ABUpiecewise_construct_t@1@$$QAV?$tuple@$$QAVQString@@@1@$$QAV?$tuple@$$$V@1@@Z$0 1000130b f i alm_process.obj
 0001:00000356       __catch$??$_Buynode@U?$pair@VQString@@PAVcProcess@@@std@@@?$_Tree_buy@U?$pair@$$CBVQString@@PAVcProcess@@@std@@V?$allocator@U?$pair@$$CBVQString@@PAVcProcess@@@std@@@2@@std@@QAEPAU?$_Tree_node@U?$pair@$$CBVQString@@PAVcProcess@@@std@@PAX@1@$$QAU?$pair@VQString@@PAVcProcess@@@1@@Z$0 10001356 f i alm_process.obj
 0001:000005eb       __catch$??$_Insert_hint@AAU?$pair@$$CBVQString@@PAVcProcess@@@std@@PAU?$_Tree_node@U?$pair@$$CBVQString@@PAVcProcess@@@std@@PAX@2@@?$_Tree@V?$_Tmap_traits@VQString@@PAVcProcess@@U?$less@VQString@@@std@@V?$allocator@U?$pair@$$CBVQString@@PAVcProcess@@@std@@@4@$0A@@std@@@std@@IAE?AV?$_Tree_iterator@V?$_Tree_val@U?$_Tree_simple_types@U?$pair@$$CBVQString@@PAVcProcess@@@std@@@std@@@std@@@1@V?$_Tree_const_iterator@V?$_Tree_val@U?$_Tree_simple_types@U?$pair@$$CBVQString@@PAVcProcess@@@std@@@std@@@std@@@1@AAU?$pair@$$CBVQString@@PAVcProcess@@@1@PAU?$_Tree_node@U?$pair@$$CBVQString@@PAVcProcess@@@std@@PAX@1@@Z$0 100015eb f i alm_process.obj
 0001:000006e3       __catch$??$_Insert_nohint@AAU?$pair@$$CBVQString@@PAVcProcess@@@std@@PAU?$_Tree_node@U?$pair@$$CBVQString@@PAVcProcess@@@std@@PAX@2@@?$_Tree@V?$_Tmap_traits@VQString@@PAVcProcess@@U?$less@VQString@@@std@@V?$allocator@U?$pair@$$CBVQString@@PAVcProcess@@@std@@@4@$0A@@std@@@std@@IAE?AU?$pair@V?$_Tree_iterator@V?$_Tree_val@U?$_Tree_simple_types@U?$pair@$$CBVQString@@PAVcProcess@@@std@@@std@@@std@@@std@@_N@1@_NAAU?$pair@$$CBVQString@@PAVcProcess@@@1@PAU?$_Tree_node@U?$pair@$$CBVQString@@PAVcProcess@@@std@@PAX@1@@Z$0 100016e3 f i alm_process.obj
 0001:00013e52       $LN84                      10014e52     moc_alm_process.obj
 0001:0001481a       $LN59                      1001581a     moc_cProc_dialog.obj
 0001:0001da65       _pre_c_init                1001ea65 f   MSVCRT:crtdll.obj
 0001:0001dccb       ___DllMainCRTStartup       1001eccb f   MSVCRT:crtdll.obj
 0001:0001de10       $$000000                   1001ee10     MSVCRT:sehprolg4.obj
 0001:0001e4ba       __ehhandler$??$_Buynode@ABUpiecewise_construct_t@std@@V?$tuple@ABVQString@@@2@V?$tuple@$$$V@2@@?$_Tree_buy@U?$pair@$$CBVQString@@PAVcProcess@@@std@@V?$allocator@U?$pair@$$CBVQString@@PAVcProcess@@@std@@@2@@std@@QAEPAU?$_Tree_node@U?$pair@$$CBVQString@@PAVcProcess@@@std@@PAX@1@ABUpiecewise_construct_t@1@$$QAV?$tuple@ABVQString@@@1@$$QAV?$tuple@$$$V@1@@Z 1001f4ba f   alm_process.obj
 0001:0001e4ba       __ehhandler$??$_Buynode@ABUpiecewise_construct_t@std@@V?$tuple@$$QAVQString@@@2@V?$tuple@$$$V@2@@?$_Tree_buy@U?$pair@$$CBVQString@@PAVcProcess@@@std@@V?$allocator@U?$pair@$$CBVQString@@PAVcProcess@@@std@@@2@@std@@QAEPAU?$_Tree_node@U?$pair@$$CBVQString@@PAVcProcess@@@std@@PAX@1@ABUpiecewise_construct_t@1@$$QAV?$tuple@$$QAVQString@@@1@$$QAV?$tuple@$$$V@1@@Z 1001f4ba f   alm_process.obj
 0001:0001e4d5       __ehhandler$??$_Buynode@U?$pair@VQString@@PAVcProcess@@@std@@@?$_Tree_buy@U?$pair@$$CBVQString@@PAVcProcess@@@std@@V?$allocator@U?$pair@$$CBVQString@@PAVcProcess@@@std@@@2@@std@@QAEPAU?$_Tree_node@U?$pair@$$CBVQString@@PAVcProcess@@@std@@PAX@1@$$QAU?$pair@VQString@@PAVcProcess@@@1@@Z 1001f4d5 f   alm_process.obj
 0001:0001e4f0       __ehhandler$??$_Insert_hint@AAU?$pair@$$CBVQString@@PAVcProcess@@@std@@PAU?$_Tree_node@U?$pair@$$CBVQString@@PAVcProcess@@@std@@PAX@2@@?$_Tree@V?$_Tmap_traits@VQString@@PAVcProcess@@U?$less@VQString@@@std@@V?$allocator@U?$pair@$$CBVQString@@PAVcProcess@@@std@@@4@$0A@@std@@@std@@IAE?AV?$_Tree_iterator@V?$_Tree_val@U?$_Tree_simple_types@U?$pair@$$CBVQString@@PAVcProcess@@@std@@@std@@@std@@@1@V?$_Tree_const_iterator@V?$_Tree_val@U?$_Tree_simple_types@U?$pair@$$CBVQString@@PAVcProcess@@@std@@@std@@@std@@@1@AAU?$pair@$$CBVQString@@PAVcProcess@@@1@PAU?$_Tree_node@U?$pair@$$CBVQString@@PAVcProcess@@@std@@PAX@1@@Z 1001f4f0 f   alm_process.obj
 0001:0001e50b       __ehhandler$??$_Insert_nohint@AAU?$pair@$$CBVQString@@PAVcProcess@@@std@@PAU?$_Tree_node@U?$pair@$$CBVQString@@PAVcProcess@@@std@@PAX@2@@?$_Tree@V?$_Tmap_traits@VQString@@PAVcProcess@@U?$less@VQString@@@std@@V?$allocator@U?$pair@$$CBVQString@@PAVcProcess@@@std@@@4@$0A@@std@@@std@@IAE?AU?$pair@V?$_Tree_iterator@V?$_Tree_val@U?$_Tree_simple_types@U?$pair@$$CBVQString@@PAVcProcess@@@std@@@std@@@std@@@std@@_N@1@_NAAU?$pair@$$CBVQString@@PAVcProcess@@@1@PAU?$_Tree_node@U?$pair@$$CBVQString@@PAVcProcess@@@std@@PAX@1@@Z 1001f50b f   alm_process.obj
 0001:0001e526       __unwindfunclet$??$construct@U?$pair@$$CBVQString@@PAVcProcess@@@std@@ABUpiecewise_construct_t@2@V?$tuple@ABVQString@@@2@V?$tuple@$$$V@2@@?$allocator@U?$_Tree_node@U?$pair@$$CBVQString@@PAVcProcess@@@std@@PAX@std@@@std@@QAEXPAU?$pair@$$CBVQString@@PAVcProcess@@@1@ABUpiecewise_construct_t@1@$$QAV?$tuple@ABVQString@@@1@$$QAV?$tuple@$$$V@1@@Z$0 1001f526 f   alm_process.obj
 0001:0001e526       __unwindfunclet$??$construct@U?$pair@$$CBVQString@@PAVcProcess@@@std@@ABUpiecewise_construct_t@2@V?$tuple@$$QAVQString@@@2@V?$tuple@$$$V@2@@?$allocator@U?$_Tree_node@U?$pair@$$CBVQString@@PAVcProcess@@@std@@PAX@std@@@std@@QAEXPAU?$pair@$$CBVQString@@PAVcProcess@@@1@ABUpiecewise_construct_t@1@$$QAV?$tuple@$$QAVQString@@@1@$$QAV?$tuple@$$$V@1@@Z$0 1001f526 f   alm_process.obj
 0001:0001e526       __unwindfunclet$??$construct@U?$pair@$$CBVQString@@PAVcProcess@@@std@@U?$pair@VQString@@PAVcProcess@@@2@@?$allocator@U?$_Tree_node@U?$pair@$$CBVQString@@PAVcProcess@@@std@@PAX@std@@@std@@QAEXPAU?$pair@$$CBVQString@@PAVcProcess@@@1@$$QAU?$pair@VQString@@PAVcProcess@@@1@@Z$0 1001f526 f   alm_process.obj
 0001:0001e534       __ehhandler$??$construct@U?$pair@$$CBVQString@@PAVcProcess@@@std@@U?$pair@VQString@@PAVcProcess@@@2@@?$allocator@U?$_Tree_node@U?$pair@$$CBVQString@@PAVcProcess@@@std@@PAX@std@@@std@@QAEXPAU?$pair@$$CBVQString@@PAVcProcess@@@1@$$QAU?$pair@VQString@@PAVcProcess@@@1@@Z 1001f534 f   alm_process.obj
 0001:0001e534       __ehhandler$??$construct@U?$pair@$$CBVQString@@PAVcProcess@@@std@@ABUpiecewise_construct_t@2@V?$tuple@ABVQString@@@2@V?$tuple@$$$V@2@@?$allocator@U?$_Tree_node@U?$pair@$$CBVQString@@PAVcProcess@@@std@@PAX@std@@@std@@QAEXPAU?$pair@$$CBVQString@@PAVcProcess@@@1@ABUpiecewise_construct_t@1@$$QAV?$tuple@ABVQString@@@1@$$QAV?$tuple@$$$V@1@@Z 1001f534 f   alm_process.obj
 0001:0001e534       __ehhandler$??$construct@U?$pair@$$CBVQString@@PAVcProcess@@@std@@ABUpiecewise_construct_t@2@V?$tuple@$$QAVQString@@@2@V?$tuple@$$$V@2@@?$allocator@U?$_Tree_node@U?$pair@$$CBVQString@@PAVcProcess@@@std@@PAX@std@@@std@@QAEXPAU?$pair@$$CBVQString@@PAVcProcess@@@1@ABUpiecewise_construct_t@1@$$QAV?$tuple@$$QAVQString@@@1@$$QAV?$tuple@$$$V@1@@Z 1001f534 f   alm_process.obj
 0001:0001e54f       __unwindfunclet$??0ProcessListViewItem@@QAE@PAVQListView@@PAVcProcess@@@Z$0 1001f54f f   alm_process.obj
 0001:0001e558       __unwindfunclet$??0ProcessListViewItem@@QAE@PAVQListView@@PAVcProcess@@@Z$1 1001f558 f   alm_process.obj
 0001:0001e561       __unwindfunclet$??0ProcessListViewItem@@QAE@PAVQListView@@PAVcProcess@@@Z$2 1001f561 f   alm_process.obj
 0001:0001e56a       __unwindfunclet$??0ProcessListViewItem@@QAE@PAVQListView@@PAVcProcess@@@Z$3 1001f56a f   alm_process.obj
 0001:0001e573       __unwindfunclet$??0ProcessListViewItem@@QAE@PAVQListView@@PAVcProcess@@@Z$4 1001f573 f   alm_process.obj
 0001:0001e57c       __unwindfunclet$??0ProcessListViewItem@@QAE@PAVQListView@@PAVcProcess@@@Z$5 1001f57c f   alm_process.obj
 0001:0001e585       __unwindfunclet$??0ProcessListViewItem@@QAE@PAVQListView@@PAVcProcess@@@Z$6 1001f585 f   alm_process.obj
 0001:0001e58e       __unwindfunclet$??0ProcessListViewItem@@QAE@PAVQListView@@PAVcProcess@@@Z$8 1001f58e f   alm_process.obj
 0001:0001e597       __ehhandler$??0ProcessListViewItem@@QAE@PAVQListView@@PAVcProcess@@@Z 1001f597 f   alm_process.obj
 0001:0001e5b2       __unwindfunclet$??0alm_process@@QAE@ABVQString@@00@Z$0 1001f5b2 f   alm_process.obj
 0001:0001e5ba       __unwindfunclet$??0alm_process@@QAE@ABVQString@@00@Z$1 1001f5ba f   alm_process.obj
 0001:0001e5c6       __unwindfunclet$??0alm_process@@QAE@ABVQString@@00@Z$2 1001f5c6 f   alm_process.obj
 0001:0001e5d5       __unwindfunclet$??0alm_process@@QAE@ABVQString@@00@Z$3 1001f5d5 f   alm_process.obj
 0001:0001e5e4       __unwindfunclet$??0alm_process@@QAE@ABVQString@@00@Z$4 1001f5e4 f   alm_process.obj
 0001:0001e5f3       __unwindfunclet$??0alm_process@@QAE@ABVQString@@00@Z$5 1001f5f3 f   alm_process.obj
 0001:0001e602       __unwindfunclet$??0alm_process@@QAE@ABVQString@@00@Z$6 1001f602 f   alm_process.obj
 0001:0001e610       __unwindfunclet$??0alm_process@@QAE@ABVQString@@00@Z$7 1001f610 f   alm_process.obj
 0001:0001e61e       __unwindfunclet$??0alm_process@@QAE@ABVQString@@00@Z$8 1001f61e f   alm_process.obj
 0001:0001e62c       __unwindfunclet$??0alm_process@@QAE@ABVQString@@00@Z$9 1001f62c f   alm_process.obj
 0001:0001e63a       __unwindfunclet$??0alm_process@@QAE@ABVQString@@00@Z$10 1001f63a f   alm_process.obj
 0001:0001e649       __unwindfunclet$??0alm_process@@QAE@ABVQString@@00@Z$11 1001f649 f   alm_process.obj
 0001:0001e658       __unwindfunclet$??0alm_process@@QAE@ABVQString@@00@Z$12 1001f658 f   alm_process.obj
 0001:0001e667       __unwindfunclet$??0alm_process@@QAE@ABVQString@@00@Z$13 1001f667 f   alm_process.obj
 0001:0001e676       __unwindfunclet$??0alm_process@@QAE@ABVQString@@00@Z$14 1001f676 f   alm_process.obj
 0001:0001e685       __unwindfunclet$??0alm_process@@QAE@ABVQString@@00@Z$15 1001f685 f   alm_process.obj
 0001:0001e68f       __unwindfunclet$??0alm_process@@QAE@ABVQString@@00@Z$16 1001f68f f   alm_process.obj
 0001:0001e698       __unwindfunclet$??0alm_process@@QAE@ABVQString@@00@Z$17 1001f698 f   alm_process.obj
 0001:0001e6a2       __unwindfunclet$??0alm_process@@QAE@ABVQString@@00@Z$18 1001f6a2 f   alm_process.obj
 0001:0001e6ac       __unwindfunclet$??0alm_process@@QAE@ABVQString@@00@Z$19 1001f6ac f   alm_process.obj
 0001:0001e6b6       __unwindfunclet$??0alm_process@@QAE@ABVQString@@00@Z$20 1001f6b6 f   alm_process.obj
 0001:0001e6bf       __unwindfunclet$??0alm_process@@QAE@ABVQString@@00@Z$21 1001f6bf f   alm_process.obj
 0001:0001e6c9       __unwindfunclet$??0alm_process@@QAE@ABVQString@@00@Z$22 1001f6c9 f   alm_process.obj
 0001:0001e6e3       __unwindfunclet$??0alm_process@@QAE@ABVQString@@00@Z$23 1001f6e3 f   alm_process.obj
 0001:0001e6fd       __unwindfunclet$??0alm_process@@QAE@ABVQString@@00@Z$24 1001f6fd f   alm_process.obj
 0001:0001e717       __unwindfunclet$??0alm_process@@QAE@ABVQString@@00@Z$25 1001f717 f   alm_process.obj
 0001:0001e731       __unwindfunclet$??0alm_process@@QAE@ABVQString@@00@Z$27 1001f731 f   alm_process.obj
 0001:0001e73b       __unwindfunclet$??0alm_process@@QAE@ABVQString@@00@Z$28 1001f73b f   alm_process.obj
 0001:0001e755       __unwindfunclet$??0alm_process@@QAE@ABVQString@@00@Z$29 1001f755 f   alm_process.obj
 0001:0001e76f       __unwindfunclet$??0alm_process@@QAE@ABVQString@@00@Z$30 1001f76f f   alm_process.obj
 0001:0001e789       __unwindfunclet$??0alm_process@@QAE@ABVQString@@00@Z$31 1001f789 f   alm_process.obj
 0001:0001e7a8       __unwindfunclet$??0alm_process@@QAE@ABVQString@@00@Z$33 1001f7a8 f   alm_process.obj
 0001:0001e7b2       __unwindfunclet$??0alm_process@@QAE@ABVQString@@00@Z$34 1001f7b2 f   alm_process.obj
 0001:0001e7d1       __unwindfunclet$??0alm_process@@QAE@ABVQString@@00@Z$35 1001f7d1 f   alm_process.obj
 0001:0001e7f0       __unwindfunclet$??0alm_process@@QAE@ABVQString@@00@Z$36 1001f7f0 f   alm_process.obj
 0001:0001e80f       __unwindfunclet$??0alm_process@@QAE@ABVQString@@00@Z$37 1001f80f f   alm_process.obj
 0001:0001e82e       __unwindfunclet$??0alm_process@@QAE@ABVQString@@00@Z$39 1001f82e f   alm_process.obj
 0001:0001e838       __unwindfunclet$??0alm_process@@QAE@ABVQString@@00@Z$40 1001f838 f   alm_process.obj
 0001:0001e857       __unwindfunclet$??0alm_process@@QAE@ABVQString@@00@Z$41 1001f857 f   alm_process.obj
 0001:0001e876       __unwindfunclet$??0alm_process@@QAE@ABVQString@@00@Z$42 1001f876 f   alm_process.obj
 0001:0001e895       __unwindfunclet$??0alm_process@@QAE@ABVQString@@00@Z$43 1001f895 f   alm_process.obj
 0001:0001e8b4       __unwindfunclet$??0alm_process@@QAE@ABVQString@@00@Z$45 1001f8b4 f   alm_process.obj
 0001:0001e8be       __unwindfunclet$??0alm_process@@QAE@ABVQString@@00@Z$46 1001f8be f   alm_process.obj
 0001:0001e8dd       __unwindfunclet$??0alm_process@@QAE@ABVQString@@00@Z$47 1001f8dd f   alm_process.obj
 0001:0001e8fc       __unwindfunclet$??0alm_process@@QAE@ABVQString@@00@Z$48 1001f8fc f   alm_process.obj
 0001:0001e91b       __unwindfunclet$??0alm_process@@QAE@ABVQString@@00@Z$49 1001f91b f   alm_process.obj
 0001:0001e93a       __unwindfunclet$??0alm_process@@QAE@ABVQString@@00@Z$51 1001f93a f   alm_process.obj
 0001:0001e944       __unwindfunclet$??0alm_process@@QAE@ABVQString@@00@Z$52 1001f944 f   alm_process.obj
 0001:0001e963       __unwindfunclet$??0alm_process@@QAE@ABVQString@@00@Z$53 1001f963 f   alm_process.obj
 0001:0001e982       __unwindfunclet$??0alm_process@@QAE@ABVQString@@00@Z$54 1001f982 f   alm_process.obj
 0001:0001e9a1       __unwindfunclet$??0alm_process@@QAE@ABVQString@@00@Z$55 1001f9a1 f   alm_process.obj
 0001:0001e9c0       __unwindfunclet$??0alm_process@@QAE@ABVQString@@00@Z$57 1001f9c0 f   alm_process.obj
 0001:0001e9ca       __unwindfunclet$??0alm_process@@QAE@ABVQString@@00@Z$58 1001f9ca f   alm_process.obj
 0001:0001e9e9       __unwindfunclet$??0alm_process@@QAE@ABVQString@@00@Z$59 1001f9e9 f   alm_process.obj
 0001:0001ea08       __unwindfunclet$??0alm_process@@QAE@ABVQString@@00@Z$60 1001fa08 f   alm_process.obj
 0001:0001ea27       __unwindfunclet$??0alm_process@@QAE@ABVQString@@00@Z$61 1001fa27 f   alm_process.obj
 0001:0001ea46       __unwindfunclet$??0alm_process@@QAE@ABVQString@@00@Z$63 1001fa46 f   alm_process.obj
 0001:0001ea50       __unwindfunclet$??0alm_process@@QAE@ABVQString@@00@Z$64 1001fa50 f   alm_process.obj
 0001:0001ea6f       __unwindfunclet$??0alm_process@@QAE@ABVQString@@00@Z$65 1001fa6f f   alm_process.obj
 0001:0001ea8e       __unwindfunclet$??0alm_process@@QAE@ABVQString@@00@Z$66 1001fa8e f   alm_process.obj
 0001:0001eaad       __unwindfunclet$??0alm_process@@QAE@ABVQString@@00@Z$67 1001faad f   alm_process.obj
 0001:0001eacc       __unwindfunclet$??0alm_process@@QAE@ABVQString@@00@Z$69 1001facc f   alm_process.obj
 0001:0001ead6       __unwindfunclet$??0alm_process@@QAE@ABVQString@@00@Z$70 1001fad6 f   alm_process.obj
 0001:0001eaf0       __unwindfunclet$??0alm_process@@QAE@ABVQString@@00@Z$71 1001faf0 f   alm_process.obj
 0001:0001eb0a       __unwindfunclet$??0alm_process@@QAE@ABVQString@@00@Z$72 1001fb0a f   alm_process.obj
 0001:0001eb24       __unwindfunclet$??0alm_process@@QAE@ABVQString@@00@Z$73 1001fb24 f   alm_process.obj
 0001:0001eb3e       __unwindfunclet$??0alm_process@@QAE@ABVQString@@00@Z$75 1001fb3e f   alm_process.obj
 0001:0001eb48       __unwindfunclet$??0alm_process@@QAE@ABVQString@@00@Z$76 1001fb48 f   alm_process.obj
 0001:0001eb62       __unwindfunclet$??0alm_process@@QAE@ABVQString@@00@Z$77 1001fb62 f   alm_process.obj
 0001:0001eb7c       __unwindfunclet$??0alm_process@@QAE@ABVQString@@00@Z$78 1001fb7c f   alm_process.obj
 0001:0001eb96       __unwindfunclet$??0alm_process@@QAE@ABVQString@@00@Z$79 1001fb96 f   alm_process.obj
 0001:0001ebb5       __unwindfunclet$??0alm_process@@QAE@ABVQString@@00@Z$81 1001fbb5 f   alm_process.obj
 0001:0001ebbf       __unwindfunclet$??0alm_process@@QAE@ABVQString@@00@Z$82 1001fbbf f   alm_process.obj
 0001:0001ebde       __unwindfunclet$??0alm_process@@QAE@ABVQString@@00@Z$83 1001fbde f   alm_process.obj
 0001:0001ebfd       __unwindfunclet$??0alm_process@@QAE@ABVQString@@00@Z$84 1001fbfd f   alm_process.obj
 0001:0001ec1c       __unwindfunclet$??0alm_process@@QAE@ABVQString@@00@Z$85 1001fc1c f   alm_process.obj
 0001:0001ec3b       __unwindfunclet$??0alm_process@@QAE@ABVQString@@00@Z$87 1001fc3b f   alm_process.obj
 0001:0001ec45       __unwindfunclet$??0alm_process@@QAE@ABVQString@@00@Z$88 1001fc45 f   alm_process.obj
 0001:0001ec64       __unwindfunclet$??0alm_process@@QAE@ABVQString@@00@Z$89 1001fc64 f   alm_process.obj
 0001:0001ec83       __unwindfunclet$??0alm_process@@QAE@ABVQString@@00@Z$91 1001fc83 f   alm_process.obj
 0001:0001ec8d       __unwindfunclet$??0alm_process@@QAE@ABVQString@@00@Z$92 1001fc8d f   alm_process.obj
 0001:0001ecac       __unwindfunclet$??0alm_process@@QAE@ABVQString@@00@Z$93 1001fcac f   alm_process.obj
 0001:0001eccb       __unwindfunclet$??0alm_process@@QAE@ABVQString@@00@Z$95 1001fccb f   alm_process.obj
 0001:0001ecd5       __unwindfunclet$??0alm_process@@QAE@ABVQString@@00@Z$96 1001fcd5 f   alm_process.obj
 0001:0001ecf4       __unwindfunclet$??0alm_process@@QAE@ABVQString@@00@Z$97 1001fcf4 f   alm_process.obj
 0001:0001ed13       __unwindfunclet$??0alm_process@@QAE@ABVQString@@00@Z$99 1001fd13 f   alm_process.obj
 0001:0001ed1d       __unwindfunclet$??0alm_process@@QAE@ABVQString@@00@Z$100 1001fd1d f   alm_process.obj
 0001:0001ed26       __unwindfunclet$??0alm_process@@QAE@ABVQString@@00@Z$101 1001fd26 f   alm_process.obj
 0001:0001ed30       __unwindfunclet$??0alm_process@@QAE@ABVQString@@00@Z$102 1001fd30 f   alm_process.obj
 0001:0001ed3a       __unwindfunclet$??0alm_process@@QAE@ABVQString@@00@Z$103 1001fd3a f   alm_process.obj
 0001:0001ed43       __unwindfunclet$??0alm_process@@QAE@ABVQString@@00@Z$104 1001fd43 f   alm_process.obj
 0001:0001ed4d       __unwindfunclet$??0alm_process@@QAE@ABVQString@@00@Z$105 1001fd4d f   alm_process.obj
 0001:0001ed57       __unwindfunclet$??0alm_process@@QAE@ABVQString@@00@Z$106 1001fd57 f   alm_process.obj
 0001:0001ed61       __unwindfunclet$??0alm_process@@QAE@ABVQString@@00@Z$107 1001fd61 f   alm_process.obj
 0001:0001ed6b       __unwindfunclet$??0alm_process@@QAE@ABVQString@@00@Z$108 1001fd6b f   alm_process.obj
 0001:0001ed74       __unwindfunclet$??0alm_process@@QAE@ABVQString@@00@Z$109 1001fd74 f   alm_process.obj
 0001:0001ed7e       __unwindfunclet$??0alm_process@@QAE@ABVQString@@00@Z$110 1001fd7e f   alm_process.obj
 0001:0001ed88       __unwindfunclet$??0alm_process@@QAE@ABVQString@@00@Z$111 1001fd88 f   alm_process.obj
 0001:0001ed92       __unwindfunclet$??0alm_process@@QAE@ABVQString@@00@Z$112 1001fd92 f   alm_process.obj
 0001:0001ed9b       __unwindfunclet$??0alm_process@@QAE@ABVQString@@00@Z$113 1001fd9b f   alm_process.obj
 0001:0001eda5       __unwindfunclet$??0alm_process@@QAE@ABVQString@@00@Z$114 1001fda5 f   alm_process.obj
 0001:0001edae       __unwindfunclet$??0alm_process@@QAE@ABVQString@@00@Z$115 1001fdae f   alm_process.obj
 0001:0001edb8       __unwindfunclet$??0alm_process@@QAE@ABVQString@@00@Z$116 1001fdb8 f   alm_process.obj
 0001:0001edc1       __unwindfunclet$??0alm_process@@QAE@ABVQString@@00@Z$117 1001fdc1 f   alm_process.obj
 0001:0001edca       __unwindfunclet$??0alm_process@@QAE@ABVQString@@00@Z$118 1001fdca f   alm_process.obj
 0001:0001edd3       __unwindfunclet$??0alm_process@@QAE@ABVQString@@00@Z$119 1001fdd3 f   alm_process.obj
 0001:0001eddc       __unwindfunclet$??0alm_process@@QAE@ABVQString@@00@Z$120 1001fddc f   alm_process.obj
 0001:0001ede5       __unwindfunclet$??0alm_process@@QAE@ABVQString@@00@Z$121 1001fde5 f   alm_process.obj
 0001:0001edee       __ehhandler$??0alm_process@@QAE@ABVQString@@00@Z 1001fdee f   alm_process.obj
 0001:0001ee09       __unwindfunclet$??0config_plugin_base@@QAE@ABVQString@@00@Z$0 1001fe09 f   alm_process.obj
 0001:0001ee12       __unwindfunclet$??0config_plugin_base@@QAE@ABVQString@@00@Z$1 1001fe12 f   alm_process.obj
 0001:0001ee1e       __unwindfunclet$??0config_plugin_base@@QAE@ABVQString@@00@Z$2 1001fe1e f   alm_process.obj
 0001:0001ee2a       __unwindfunclet$??0config_plugin_base@@QAE@ABVQString@@00@Z$3 1001fe2a f   alm_process.obj
 0001:0001ee36       __ehhandler$??0config_plugin_base@@QAE@ABVQString@@00@Z 1001fe36 f   alm_process.obj
 0001:0001ee51       __unwindfunclet$??1?$QPtrList@VcProcess@@@@UAE@XZ$0 1001fe51 f   alm_process.obj
 0001:0001ee51       __unwindfunclet$??1?$QPtrList@VQPopupMenu@@@@UAE@XZ$0 1001fe51 f   alm_process.obj
 0001:0001ee51       __unwindfunclet$??1?$QPtrList@VQListViewItem@@@@UAE@XZ$0 1001fe51 f   alm_process.obj
 0001:0001ee5a       __ehhandler$??1?$QPtrList@VQPopupMenu@@@@UAE@XZ 1001fe5a f   alm_process.obj
 0001:0001ee5a       __ehhandler$??1?$QPtrList@VQListViewItem@@@@UAE@XZ 1001fe5a f   alm_process.obj
 0001:0001ee5a       __ehhandler$??1?$QPtrList@VcProcess@@@@UAE@XZ 1001fe5a f   alm_process.obj
 0001:0001ee75       __unwindfunclet$??1QDockWindowList@@UAE@XZ$0 1001fe75 f   alm_process.obj
 0001:0001ee7e       __unwindfunclet$??1QDockWindowList@@UAE@XZ$1 1001fe7e f   alm_process.obj
 0001:0001ee87       __ehhandler$??1QDockWindowList@@UAE@XZ 1001fe87 f   alm_process.obj
 0001:0001eea2       __unwindfunclet$??1QPopupMenuList@@UAE@XZ$0 1001fea2 f   alm_process.obj
 0001:0001eeaa       __ehhandler$??1QPopupMenuList@@UAE@XZ 1001feaa f   alm_process.obj
 0001:0001eec5       __unwindfunclet$??1alm_process@@UAE@XZ$0 1001fec5 f   alm_process.obj
 0001:0001eecd       __unwindfunclet$??1alm_process@@UAE@XZ$1 1001fecd f   alm_process.obj
 0001:0001eed9       __unwindfunclet$??1alm_process@@UAE@XZ$2 1001fed9 f   alm_process.obj
 0001:0001eee8       __unwindfunclet$??1alm_process@@UAE@XZ$3 1001fee8 f   alm_process.obj
 0001:0001eef7       __unwindfunclet$??1alm_process@@UAE@XZ$4 1001fef7 f   alm_process.obj
 0001:0001ef06       __unwindfunclet$??1alm_process@@UAE@XZ$5 1001ff06 f   alm_process.obj
 0001:0001ef15       __unwindfunclet$??1alm_process@@UAE@XZ$6 1001ff15 f   alm_process.obj
 0001:0001ef23       __unwindfunclet$??1alm_process@@UAE@XZ$7 1001ff23 f   alm_process.obj
 0001:0001ef31       __unwindfunclet$??1alm_process@@UAE@XZ$8 1001ff31 f   alm_process.obj
 0001:0001ef3f       __unwindfunclet$??1alm_process@@UAE@XZ$9 1001ff3f f   alm_process.obj
 0001:0001ef4d       __unwindfunclet$??1alm_process@@UAE@XZ$10 1001ff4d f   alm_process.obj
 0001:0001ef5c       __unwindfunclet$??1alm_process@@UAE@XZ$11 1001ff5c f   alm_process.obj
 0001:0001ef6b       __unwindfunclet$??1alm_process@@UAE@XZ$12 1001ff6b f   alm_process.obj
 0001:0001ef7a       __unwindfunclet$??1alm_process@@UAE@XZ$13 1001ff7a f   alm_process.obj
 0001:0001ef89       __unwindfunclet$??1alm_process@@UAE@XZ$14 1001ff89 f   alm_process.obj
 0001:0001ef98       __unwindfunclet$??1alm_process@@UAE@XZ$15 1001ff98 f   alm_process.obj
 0001:0001efa1       __unwindfunclet$??1alm_process@@UAE@XZ$16 1001ffa1 f   alm_process.obj
 0001:0001efaa       __ehhandler$??1alm_process@@UAE@XZ 1001ffaa f   alm_process.obj
 0001:0001efc5       __unwindfunclet$??1config_plugin_base@@UAE@XZ$0 1001ffc5 f   alm_process.obj
 0001:0001efce       __unwindfunclet$??1config_plugin_base@@UAE@XZ$1 1001ffce f   alm_process.obj
 0001:0001efda       __unwindfunclet$??1config_plugin_base@@UAE@XZ$2 1001ffda f   alm_process.obj
 0001:0001efe6       __ehhandler$??1config_plugin_base@@UAE@XZ 1001ffe6 f   alm_process.obj
 0001:0001f001       __unwindfunclet$?about@alm_process@@EAE?AVQString@@XZ$0 10020001 f   alm_process.obj
 0001:0001f01b       __unwindfunclet$?about@alm_process@@EAE?AVQString@@XZ$1 1002001b f   alm_process.obj
 0001:0001f024       __unwindfunclet$?about@alm_process@@EAE?AVQString@@XZ$2 10020024 f   alm_process.obj
 0001:0001f02d       __ehhandler$?about@alm_process@@EAE?AVQString@@XZ 1002002d f   alm_process.obj
 0001:0001f048       __unwindfunclet$?about@config_plugin_base@@UAE?AVQString@@XZ$0 10020048 f   alm_process.obj
 0001:0001f051       __unwindfunclet$?about@config_plugin_base@@UAE?AVQString@@XZ$1 10020051 f   alm_process.obj
 0001:0001f06b       __ehhandler$?about@config_plugin_base@@UAE?AVQString@@XZ 1002006b f   alm_process.obj
 0001:0001f086       __unwindfunclet$?activate@alm_process@@UAEX_N@Z$0 10020086 f   alm_process.obj
 0001:0001f08f       __unwindfunclet$?activate@alm_process@@UAEX_N@Z$3 1002008f f   alm_process.obj
 0001:0001f098       __unwindfunclet$?activate@alm_process@@UAEX_N@Z$4 10020098 f   alm_process.obj
 0001:0001f0a1       __unwindfunclet$?activate@alm_process@@UAEX_N@Z$5 100200a1 f   alm_process.obj
 0001:0001f0aa       __unwindfunclet$?activate@alm_process@@UAEX_N@Z$6 100200aa f   alm_process.obj
 0001:0001f0b3       __unwindfunclet$?activate@alm_process@@UAEX_N@Z$7 100200b3 f   alm_process.obj
 0001:0001f0bc       __ehhandler$?activate@alm_process@@UAEX_N@Z 100200bc f   alm_process.obj
 0001:0001f0d7       __unwindfunclet$?apply@alm_process@@EAEXXZ$0 100200d7 f   alm_process.obj
 0001:0001f0e0       __unwindfunclet$?apply@alm_process@@EAEXXZ$1 100200e0 f   alm_process.obj
 0001:0001f0e9       __unwindfunclet$?apply@alm_process@@EAEXXZ$2 100200e9 f   alm_process.obj
 0001:0001f0f2       __unwindfunclet$?apply@alm_process@@EAEXXZ$3 100200f2 f   alm_process.obj
 0001:0001f0fb       __unwindfunclet$?apply@alm_process@@EAEXXZ$5 100200fb f   alm_process.obj
 0001:0001f104       __ehhandler$?apply@alm_process@@EAEXXZ 10020104 f   alm_process.obj
 0001:0001f11f       __unwindfunclet$?checkProcessContributors@alm_process@@AAEXXZ$0 1002011f f   alm_process.obj
 0001:0001f128       __unwindfunclet$?checkProcessContributors@alm_process@@AAEXXZ$1 10020128 f   alm_process.obj
 0001:0001f131       __unwindfunclet$?checkProcessContributors@alm_process@@AAEXXZ$2 10020131 f   alm_process.obj
 0001:0001f13a       __unwindfunclet$?checkProcessContributors@alm_process@@AAEXXZ$3 1002013a f   alm_process.obj
 0001:0001f145       __unwindfunclet$?checkProcessContributors@alm_process@@AAEXXZ$4 10020145 f   alm_process.obj
 0001:0001f14e       __unwindfunclet$?checkProcessContributors@alm_process@@AAEXXZ$5 1002014e f   alm_process.obj
 0001:0001f157       __unwindfunclet$?checkProcessContributors@alm_process@@AAEXXZ$6 10020157 f   alm_process.obj
 0001:0001f160       __unwindfunclet$?checkProcessContributors@alm_process@@AAEXXZ$7 10020160 f   alm_process.obj
 0001:0001f169       __unwindfunclet$?checkProcessContributors@alm_process@@AAEXXZ$8 10020169 f   alm_process.obj
 0001:0001f172       __unwindfunclet$?checkProcessContributors@alm_process@@AAEXXZ$9 10020172 f   alm_process.obj
 0001:0001f17b       __unwindfunclet$?checkProcessContributors@alm_process@@AAEXXZ$10 1002017b f   alm_process.obj
 0001:0001f184       __unwindfunclet$?checkProcessContributors@alm_process@@AAEXXZ$11 10020184 f   alm_process.obj
 0001:0001f18d       __unwindfunclet$?checkProcessContributors@alm_process@@AAEXXZ$12 1002018d f   alm_process.obj
 0001:0001f196       __unwindfunclet$?checkProcessContributors@alm_process@@AAEXXZ$13 10020196 f   alm_process.obj
 0001:0001f19f       __unwindfunclet$?checkProcessContributors@alm_process@@AAEXXZ$14 1002019f f   alm_process.obj
 0001:0001f1a8       __unwindfunclet$?checkProcessContributors@alm_process@@AAEXXZ$15 100201a8 f   alm_process.obj
 0001:0001f1c2       __unwindfunclet$?checkProcessContributors@alm_process@@AAEXXZ$16 100201c2 f   alm_process.obj
 0001:0001f1cb       __unwindfunclet$?checkProcessContributors@alm_process@@AAEXXZ$17 100201cb f   alm_process.obj
 0001:0001f1d4       __unwindfunclet$?checkProcessContributors@alm_process@@AAEXXZ$18 100201d4 f   alm_process.obj
 0001:0001f1dd       __unwindfunclet$?checkProcessContributors@alm_process@@AAEXXZ$19 100201dd f   alm_process.obj
 0001:0001f1e6       __unwindfunclet$?checkProcessContributors@alm_process@@AAEXXZ$20 100201e6 f   alm_process.obj
 0001:0001f1ef       __unwindfunclet$?checkProcessContributors@alm_process@@AAEXXZ$21 100201ef f   alm_process.obj
 0001:0001f1f8       __unwindfunclet$?checkProcessContributors@alm_process@@AAEXXZ$22 100201f8 f   alm_process.obj
 0001:0001f201       __unwindfunclet$?checkProcessContributors@alm_process@@AAEXXZ$23 10020201 f   alm_process.obj
 0001:0001f20a       __unwindfunclet$?checkProcessContributors@alm_process@@AAEXXZ$24 1002020a f   alm_process.obj
 0001:0001f213       __unwindfunclet$?checkProcessContributors@alm_process@@AAEXXZ$25 10020213 f   alm_process.obj
 0001:0001f21c       __unwindfunclet$?checkProcessContributors@alm_process@@AAEXXZ$26 1002021c f   alm_process.obj
 0001:0001f225       __unwindfunclet$?checkProcessContributors@alm_process@@AAEXXZ$27 10020225 f   alm_process.obj
 0001:0001f22e       __unwindfunclet$?checkProcessContributors@alm_process@@AAEXXZ$28 1002022e f   alm_process.obj
 0001:0001f237       __unwindfunclet$?checkProcessContributors@alm_process@@AAEXXZ$29 10020237 f   alm_process.obj
 0001:0001f240       __unwindfunclet$?checkProcessContributors@alm_process@@AAEXXZ$30 10020240 f   alm_process.obj
 0001:0001f249       __unwindfunclet$?checkProcessContributors@alm_process@@AAEXXZ$31 10020249 f   alm_process.obj
 0001:0001f252       __unwindfunclet$?checkProcessContributors@alm_process@@AAEXXZ$32 10020252 f   alm_process.obj
 0001:0001f25b       __unwindfunclet$?checkProcessContributors@alm_process@@AAEXXZ$33 1002025b f   alm_process.obj
 0001:0001f264       __unwindfunclet$?checkProcessContributors@alm_process@@AAEXXZ$34 10020264 f   alm_process.obj
 0001:0001f26d       __unwindfunclet$?checkProcessContributors@alm_process@@AAEXXZ$35 1002026d f   alm_process.obj
 0001:0001f276       __unwindfunclet$?checkProcessContributors@alm_process@@AAEXXZ$36 10020276 f   alm_process.obj
 0001:0001f27f       __unwindfunclet$?checkProcessContributors@alm_process@@AAEXXZ$37 1002027f f   alm_process.obj
 0001:0001f28b       __unwindfunclet$?checkProcessContributors@alm_process@@AAEXXZ$38 1002028b f   alm_process.obj
 0001:0001f294       __unwindfunclet$?checkProcessContributors@alm_process@@AAEXXZ$39 10020294 f   alm_process.obj
 0001:0001f29d       __ehhandler$?checkProcessContributors@alm_process@@AAEXXZ 1002029d f   alm_process.obj
 0001:0001f2bb       __unwindfunclet$?checkReferences@alm_process@@AAEXXZ$0 100202bb f   alm_process.obj
 0001:0001f2c4       __unwindfunclet$?checkReferences@alm_process@@AAEXXZ$1 100202c4 f   alm_process.obj
 0001:0001f2cd       __ehhandler$?checkReferences@alm_process@@AAEXXZ 100202cd f   alm_process.obj
 0001:0001f2e8       __unwindfunclet$?clearMask@alm_process@@AAEXXZ$0 100202e8 f   alm_process.obj
 0001:0001f2f0       __unwindfunclet$?clearMask@alm_process@@AAEXXZ$1 100202f0 f   alm_process.obj
 0001:0001f2f9       __unwindfunclet$?clearMask@alm_process@@AAEXXZ$2 100202f9 f   alm_process.obj
 0001:0001f302       __unwindfunclet$?clearMask@alm_process@@AAEXXZ$3 10020302 f   alm_process.obj
 0001:0001f30b       __ehhandler$?clearMask@alm_process@@AAEXXZ 1002030b f   alm_process.obj
 0001:0001f326       __unwindfunclet$?closeEvent@alm_process@@UAEXPAVQCloseEvent@@@Z$0 10020326 f   alm_process.obj
 0001:0001f32f       __ehhandler$?closeEvent@alm_process@@UAEXPAVQCloseEvent@@@Z 1002032f f   alm_process.obj
 0001:0001f34a       __unwindfunclet$?copyProcessUsingTemplate@alm_process@@AAEXXZ$0 1002034a f   alm_process.obj
 0001:0001f352       __unwindfunclet$?copyProcessUsingTemplate@alm_process@@AAEXXZ$1 10020352 f   alm_process.obj
 0001:0001f35b       __unwindfunclet$?copyProcessUsingTemplate@alm_process@@AAEXXZ$2 1002035b f   alm_process.obj
 0001:0001f364       __unwindfunclet$?copyProcessUsingTemplate@alm_process@@AAEXXZ$3 10020364 f   alm_process.obj
 0001:0001f36d       __unwindfunclet$?copyProcessUsingTemplate@alm_process@@AAEXXZ$4 1002036d f   alm_process.obj
 0001:0001f377       __ehhandler$?copyProcessUsingTemplate@alm_process@@AAEXXZ 10020377 f   alm_process.obj
 0001:0001f392       __unwindfunclet$?deleteGroup@alm_process@@AAEXXZ$0 10020392 f   alm_process.obj
 0001:0001f39b       __unwindfunclet$?deleteGroup@alm_process@@AAEXXZ$1 1002039b f   alm_process.obj
 0001:0001f3a4       __unwindfunclet$?deleteGroup@alm_process@@AAEXXZ$2 100203a4 f   alm_process.obj
 0001:0001f3ad       __unwindfunclet$?deleteGroup@alm_process@@AAEXXZ$3 100203ad f   alm_process.obj
 0001:0001f3b6       __ehhandler$?deleteGroup@alm_process@@AAEXXZ 100203b6 f   alm_process.obj
 0001:0001f3d1       __unwindfunclet$?deleteProcess@alm_process@@AAEXXZ$0 100203d1 f   alm_process.obj
 0001:0001f3d9       __unwindfunclet$?deleteProcess@alm_process@@AAEXXZ$1 100203d9 f   alm_process.obj
 0001:0001f3e2       __unwindfunclet$?deleteProcess@alm_process@@AAEXXZ$2 100203e2 f   alm_process.obj
 0001:0001f3ea       __unwindfunclet$?deleteProcess@alm_process@@AAEXXZ$3 100203ea f   alm_process.obj
 0001:0001f3f3       __unwindfunclet$?deleteProcess@alm_process@@AAEXXZ$4 100203f3 f   alm_process.obj
 0001:0001f3fc       __unwindfunclet$?deleteProcess@alm_process@@AAEXXZ$5 100203fc f   alm_process.obj
 0001:0001f407       __unwindfunclet$?deleteProcess@alm_process@@AAEXXZ$6 10020407 f   alm_process.obj
 0001:0001f410       __unwindfunclet$?deleteProcess@alm_process@@AAEXXZ$7 10020410 f   alm_process.obj
 0001:0001f419       __ehhandler$?deleteProcess@alm_process@@AAEXXZ 10020419 f   alm_process.obj
 0001:0001f437       __unwindfunclet$?duplicateProcess@alm_process@@AAEXXZ$0 10020437 f   alm_process.obj
 0001:0001f43f       __unwindfunclet$?duplicateProcess@alm_process@@AAEXXZ$1 1002043f f   alm_process.obj
 0001:0001f448       __unwindfunclet$?duplicateProcess@alm_process@@AAEXXZ$2 10020448 f   alm_process.obj
 0001:0001f451       __unwindfunclet$?duplicateProcess@alm_process@@AAEXXZ$3 10020451 f   alm_process.obj
 0001:0001f45a       __unwindfunclet$?duplicateProcess@alm_process@@AAEXXZ$4 1002045a f   alm_process.obj
 0001:0001f463       __unwindfunclet$?duplicateProcess@alm_process@@AAEXXZ$11 10020463 f   alm_process.obj
 0001:0001f46c       __unwindfunclet$?duplicateProcess@alm_process@@AAEXXZ$5 1002046c f   alm_process.obj
 0001:0001f475       __unwindfunclet$?duplicateProcess@alm_process@@AAEXXZ$6 10020475 f   alm_process.obj
 0001:0001f47f       __unwindfunclet$?duplicateProcess@alm_process@@AAEXXZ$7 1002047f f   alm_process.obj
 0001:0001f488       __unwindfunclet$?duplicateProcess@alm_process@@AAEXXZ$8 10020488 f   alm_process.obj
 0001:0001f490       __unwindfunclet$?duplicateProcess@alm_process@@AAEXXZ$9 10020490 f   alm_process.obj
 0001:0001f49a       __ehhandler$?duplicateProcess@alm_process@@AAEXXZ 1002049a f   alm_process.obj
 0001:0001f4b5       __unwindfunclet$?loadProcesses@alm_process@@AAE_NVQString@@@Z$0 100204b5 f   alm_process.obj
 0001:0001f4be       __unwindfunclet$?loadProcesses@alm_process@@AAE_NVQString@@@Z$1 100204be f   alm_process.obj
 0001:0001f4c7       __unwindfunclet$?loadProcesses@alm_process@@AAE_NVQString@@@Z$2 100204c7 f   alm_process.obj
 0001:0001f4d0       __unwindfunclet$?loadProcesses@alm_process@@AAE_NVQString@@@Z$3 100204d0 f   alm_process.obj
 0001:0001f4dc       __unwindfunclet$?loadProcesses@alm_process@@AAE_NVQString@@@Z$4 100204dc f   alm_process.obj
 0001:0001f4e5       __unwindfunclet$?loadProcesses@alm_process@@AAE_NVQString@@@Z$5 100204e5 f   alm_process.obj
 0001:0001f4ee       __unwindfunclet$?loadProcesses@alm_process@@AAE_NVQString@@@Z$6 100204ee f   alm_process.obj
 0001:0001f4f7       __unwindfunclet$?loadProcesses@alm_process@@AAE_NVQString@@@Z$7 100204f7 f   alm_process.obj
 0001:0001f500       __unwindfunclet$?loadProcesses@alm_process@@AAE_NVQString@@@Z$8 10020500 f   alm_process.obj
 0001:0001f50c       __unwindfunclet$?loadProcesses@alm_process@@AAE_NVQString@@@Z$9 1002050c f   alm_process.obj
 0001:0001f515       __unwindfunclet$?loadProcesses@alm_process@@AAE_NVQString@@@Z$10 10020515 f   alm_process.obj
 0001:0001f51e       __unwindfunclet$?loadProcesses@alm_process@@AAE_NVQString@@@Z$11 1002051e f   alm_process.obj
 0001:0001f527       __unwindfunclet$?loadProcesses@alm_process@@AAE_NVQString@@@Z$12 10020527 f   alm_process.obj
 0001:0001f530       __unwindfunclet$?loadProcesses@alm_process@@AAE_NVQString@@@Z$13 10020530 f   alm_process.obj
 0001:0001f539       __unwindfunclet$?loadProcesses@alm_process@@AAE_NVQString@@@Z$14 10020539 f   alm_process.obj
 0001:0001f542       __unwindfunclet$?loadProcesses@alm_process@@AAE_NVQString@@@Z$15 10020542 f   alm_process.obj
 0001:0001f55c       __unwindfunclet$?loadProcesses@alm_process@@AAE_NVQString@@@Z$16 1002055c f   alm_process.obj
 0001:0001f576       __unwindfunclet$?loadProcesses@alm_process@@AAE_NVQString@@@Z$17 10020576 f   alm_process.obj
 0001:0001f57f       __unwindfunclet$?loadProcesses@alm_process@@AAE_NVQString@@@Z$18 1002057f f   alm_process.obj
 0001:0001f588       __unwindfunclet$?loadProcesses@alm_process@@AAE_NVQString@@@Z$19 10020588 f   alm_process.obj
 0001:0001f5a2       __unwindfunclet$?loadProcesses@alm_process@@AAE_NVQString@@@Z$20 100205a2 f   alm_process.obj
 0001:0001f5bc       __ehhandler$?loadProcesses@alm_process@@AAE_NVQString@@@Z 100205bc f   alm_process.obj
 0001:0001f5da       __unwindfunclet$?markDirty@alm_process@@AAEXXZ$0 100205da f   alm_process.obj
 0001:0001f5e3       __unwindfunclet$?markDirty@alm_process@@AAEXXZ$1 100205e3 f   alm_process.obj
 0001:0001f5ec       __unwindfunclet$?markDirty@alm_process@@AAEXXZ$2 100205ec f   alm_process.obj
 0001:0001f5f5       __unwindfunclet$?markDirty@alm_process@@AAEXXZ$3 100205f5 f   alm_process.obj
 0001:0001f5fe       __unwindfunclet$?markDirty@alm_process@@AAEXXZ$4 100205fe f   alm_process.obj
 0001:0001f607       __unwindfunclet$?markDirty@alm_process@@AAEXXZ$5 10020607 f   alm_process.obj
 0001:0001f610       __unwindfunclet$?markDirty@alm_process@@AAEXXZ$6 10020610 f   alm_process.obj
 0001:0001f619       __unwindfunclet$?markDirty@alm_process@@AAEXXZ$7 10020619 f   alm_process.obj
 0001:0001f622       __unwindfunclet$?markDirty@alm_process@@AAEXXZ$8 10020622 f   alm_process.obj
 0001:0001f62b       __unwindfunclet$?markDirty@alm_process@@AAEXXZ$9 1002062b f   alm_process.obj
 0001:0001f634       __unwindfunclet$?markDirty@alm_process@@AAEXXZ$10 10020634 f   alm_process.obj
 0001:0001f63d       __ehhandler$?markDirty@alm_process@@AAEXXZ 1002063d f   alm_process.obj
 0001:0001f658       __unwindfunclet$?menus@alm_process@@UAE?AVQPopupMenuList@@XZ$0 10020658 f   alm_process.obj
 0001:0001f671       __ehhandler$?menus@alm_process@@UAE?AVQPopupMenuList@@XZ 10020671 f   alm_process.obj
 0001:0001f68c       __unwindfunclet$?navToAck@alm_process@@AAEXVQString@@00@Z$0 1002068c f   alm_process.obj
 0001:0001f695       __unwindfunclet$?navToAck@alm_process@@AAEXVQString@@00@Z$1 10020695 f   alm_process.obj
 0001:0001f69e       __unwindfunclet$?navToAck@alm_process@@AAEXVQString@@00@Z$2 1002069e f   alm_process.obj
 0001:0001f6a7       __unwindfunclet$?navToAck@alm_process@@AAEXVQString@@00@Z$3 100206a7 f   alm_process.obj
 0001:0001f6b0       __unwindfunclet$?navToAck@alm_process@@AAEXVQString@@00@Z$4 100206b0 f   alm_process.obj
 0001:0001f6b9       __unwindfunclet$?navToAck@alm_process@@AAEXVQString@@00@Z$5 100206b9 f   alm_process.obj
 0001:0001f6c2       __unwindfunclet$?navToAck@alm_process@@AAEXVQString@@00@Z$6 100206c2 f   alm_process.obj
 0001:0001f6cb       __ehhandler$?navToAck@alm_process@@AAEXVQString@@00@Z 100206cb f   alm_process.obj
 0001:0001f6e6       __unwindfunclet$?navToOutput@alm_process@@AAEXVQString@@0@Z$0 100206e6 f   alm_process.obj
 0001:0001f6ef       __unwindfunclet$?navToOutput@alm_process@@AAEXVQString@@0@Z$1 100206ef f   alm_process.obj
 0001:0001f6f8       __unwindfunclet$?navToOutput@alm_process@@AAEXVQString@@0@Z$2 100206f8 f   alm_process.obj
 0001:0001f701       __unwindfunclet$?navToOutput@alm_process@@AAEXVQString@@0@Z$3 10020701 f   alm_process.obj
 0001:0001f70a       __unwindfunclet$?navToOutput@alm_process@@AAEXVQString@@0@Z$4 1002070a f   alm_process.obj
 0001:0001f713       __unwindfunclet$?navToOutput@alm_process@@AAEXVQString@@0@Z$5 10020713 f   alm_process.obj
 0001:0001f71c       __unwindfunclet$?navToOutput@alm_process@@AAEXVQString@@0@Z$6 1002071c f   alm_process.obj
 0001:0001f725       __ehhandler$?navToOutput@alm_process@@AAEXVQString@@0@Z 10020725 f   alm_process.obj
 0001:0001f740       __unwindfunclet$?navigate@alm_process@@UAEXABVQString@@0@Z$0 10020740 f   alm_process.obj
 0001:0001f75a       __unwindfunclet$?navigate@alm_process@@UAEXABVQString@@0@Z$1 1002075a f   alm_process.obj
 0001:0001f774       __ehhandler$?navigate@alm_process@@UAEXABVQString@@0@Z 10020774 f   alm_process.obj
 0001:0001f78f       __unwindfunclet$?newGate@alm_process@@AAEXXZ$0 1002078f f   alm_process.obj
 0001:0001f798       __unwindfunclet$?newGate@alm_process@@AAEXXZ$1 10020798 f   alm_process.obj
 0001:0001f7a1       __unwindfunclet$?newGate@alm_process@@AAEXXZ$2 100207a1 f   alm_process.obj
 0001:0001f7aa       __unwindfunclet$?newGate@alm_process@@AAEXXZ$4 100207aa f   alm_process.obj
 0001:0001f7b3       __unwindfunclet$?newGate@alm_process@@AAEXXZ$5 100207b3 f   alm_process.obj
 0001:0001f7bc       __unwindfunclet$?newGate@alm_process@@AAEXXZ$6 100207bc f   alm_process.obj
 0001:0001f7c5       __unwindfunclet$?newGate@alm_process@@AAEXXZ$7 100207c5 f   alm_process.obj
 0001:0001f7ce       __unwindfunclet$?newGate@alm_process@@AAEXXZ$8 100207ce f   alm_process.obj
 0001:0001f7d7       __unwindfunclet$?newGate@alm_process@@AAEXXZ$9 100207d7 f   alm_process.obj
 0001:0001f7e0       __unwindfunclet$?newGate@alm_process@@AAEXXZ$10 100207e0 f   alm_process.obj
 0001:0001f7e9       __unwindfunclet$?newGate@alm_process@@AAEXXZ$11 100207e9 f   alm_process.obj
 0001:0001f7f2       __unwindfunclet$?newGate@alm_process@@AAEXXZ$12 100207f2 f   alm_process.obj
 0001:0001f7fb       __unwindfunclet$?newGate@alm_process@@AAEXXZ$13 100207fb f   alm_process.obj
 0001:0001f804       __unwindfunclet$?newGate@alm_process@@AAEXXZ$14 10020804 f   alm_process.obj
 0001:0001f80d       __unwindfunclet$?newGate@alm_process@@AAEXXZ$15 1002080d f   alm_process.obj
 0001:0001f816       __unwindfunclet$?newGate@alm_process@@AAEXXZ$16 10020816 f   alm_process.obj
 0001:0001f81f       __unwindfunclet$?newGate@alm_process@@AAEXXZ$17 1002081f f   alm_process.obj
 0001:0001f828       __unwindfunclet$?newGate@alm_process@@AAEXXZ$18 10020828 f   alm_process.obj
 0001:0001f832       __unwindfunclet$?newGate@alm_process@@AAEXXZ$19 10020832 f   alm_process.obj
 0001:0001f83b       __unwindfunclet$?newGate@alm_process@@AAEXXZ$20 1002083b f   alm_process.obj
 0001:0001f844       __unwindfunclet$?newGate@alm_process@@AAEXXZ$21 10020844 f   alm_process.obj
 0001:0001f84d       __unwindfunclet$?newGate@alm_process@@AAEXXZ$22 1002084d f   alm_process.obj
 0001:0001f856       __unwindfunclet$?newGate@alm_process@@AAEXXZ$23 10020856 f   alm_process.obj
 0001:0001f85f       __unwindfunclet$?newGate@alm_process@@AAEXXZ$24 1002085f f   alm_process.obj
 0001:0001f868       __unwindfunclet$?newGate@alm_process@@AAEXXZ$25 10020868 f   alm_process.obj
 0001:0001f870       __unwindfunclet$?newGate@alm_process@@AAEXXZ$26 10020870 f   alm_process.obj
 0001:0001f87a       __ehhandler$?newGate@alm_process@@AAEXXZ 1002087a f   alm_process.obj
 0001:0001f895       __unwindfunclet$?newGroup@alm_process@@AAEXXZ$0 10020895 f   alm_process.obj
 0001:0001f89e       __unwindfunclet$?newGroup@alm_process@@AAEXXZ$1 1002089e f   alm_process.obj
 0001:0001f8a7       __unwindfunclet$?newGroup@alm_process@@AAEXXZ$2 100208a7 f   alm_process.obj
 0001:0001f8b0       __ehhandler$?newGroup@alm_process@@AAEXXZ 100208b0 f   alm_process.obj
 0001:0001f8cb       __unwindfunclet$?newProcess@alm_process@@AAEXVQString@@AAVQStringList@@@Z$0 100208cb f   alm_process.obj
 0001:0001f8d4       __unwindfunclet$?newProcess@alm_process@@AAEXVQString@@AAVQStringList@@@Z$1 100208d4 f   alm_process.obj
 0001:0001f8de       __unwindfunclet$?newProcess@alm_process@@AAEXVQString@@AAVQStringList@@@Z$2 100208de f   alm_process.obj
 0001:0001f8e7       __unwindfunclet$?newProcess@alm_process@@AAEXVQString@@AAVQStringList@@@Z$3 100208e7 f   alm_process.obj
 0001:0001f8f1       __unwindfunclet$?newProcess@alm_process@@AAEXVQString@@AAVQStringList@@@Z$4 100208f1 f   alm_process.obj
 0001:0001f8f9       __ehhandler$?newProcess@alm_process@@AAEXVQString@@AAVQStringList@@@Z 100208f9 f   alm_process.obj
 0001:0001f914       __unwindfunclet$?newProcess@alm_process@@AAEXXZ$0 10020914 f   alm_process.obj
 0001:0001f91d       __unwindfunclet$?newProcess@alm_process@@AAEXXZ$1 1002091d f   alm_process.obj
 0001:0001f927       __unwindfunclet$?newProcess@alm_process@@AAEXXZ$2 10020927 f   alm_process.obj
 0001:0001f92f       __unwindfunclet$?newProcess@alm_process@@AAEXXZ$3 1002092f f   alm_process.obj
 0001:0001f939       __ehhandler$?newProcess@alm_process@@AAEXXZ 10020939 f   alm_process.obj
 0001:0001f954       __unwindfunclet$?paintCell@ProcessListViewItem@@EAEXPAVQPainter@@ABVQColorGroup@@HHH@Z$0 10020954 f   alm_process.obj
 0001:0001f954       __unwindfunclet$?paintCell@MultiInputInvalidListViewItem@@EAEXPAVQPainter@@ABVQColorGroup@@HHH@Z$0 10020954 f   alm_process.obj
 0001:0001f95d       __ehhandler$?paintCell@MultiInputInvalidListViewItem@@EAEXPAVQPainter@@ABVQColorGroup@@HHH@Z 1002095d f   alm_process.obj
 0001:0001f95d       __ehhandler$?paintCell@ProcessListViewItem@@EAEXPAVQPainter@@ABVQColorGroup@@HHH@Z 1002095d f   alm_process.obj
 0001:0001f978       __unwindfunclet$?renameGroup@alm_process@@AAEXXZ$0 10020978 f   alm_process.obj
 0001:0001f981       __unwindfunclet$?renameGroup@alm_process@@AAEXXZ$1 10020981 f   alm_process.obj
 0001:0001f98a       __unwindfunclet$?renameGroup@alm_process@@AAEXXZ$2 1002098a f   alm_process.obj
 0001:0001f993       __unwindfunclet$?renameGroup@alm_process@@AAEXXZ$3 10020993 f   alm_process.obj
 0001:0001f99c       __unwindfunclet$?renameGroup@alm_process@@AAEXXZ$4 1002099c f   alm_process.obj
 0001:0001f9a5       __unwindfunclet$?renameGroup@alm_process@@AAEXXZ$5 100209a5 f   alm_process.obj
 0001:0001f9ae       __unwindfunclet$?renameGroup@alm_process@@AAEXXZ$6 100209ae f   alm_process.obj
 0001:0001f9b7       __unwindfunclet$?renameGroup@alm_process@@AAEXXZ$7 100209b7 f   alm_process.obj
 0001:0001f9c0       __unwindfunclet$?renameGroup@alm_process@@AAEXXZ$8 100209c0 f   alm_process.obj
 0001:0001f9c9       __unwindfunclet$?renameGroup@alm_process@@AAEXXZ$9 100209c9 f   alm_process.obj
 0001:0001f9d2       __unwindfunclet$?renameGroup@alm_process@@AAEXXZ$10 100209d2 f   alm_process.obj
 0001:0001f9db       __unwindfunclet$?renameGroup@alm_process@@AAEXXZ$11 100209db f   alm_process.obj
 0001:0001f9e4       __ehhandler$?renameGroup@alm_process@@AAEXXZ 100209e4 f   alm_process.obj
 0001:0001f9ff       __unwindfunclet$?renameProcess@alm_process@@AAEXPAVQListViewItem@@HABVQString@@@Z$0 100209ff f   alm_process.obj
 0001:0001fa08       __unwindfunclet$?renameProcess@alm_process@@AAEXPAVQListViewItem@@HABVQString@@@Z$1 10020a08 f   alm_process.obj
 0001:0001fa11       __unwindfunclet$?renameProcess@alm_process@@AAEXPAVQListViewItem@@HABVQString@@@Z$2 10020a11 f   alm_process.obj
 0001:0001fa19       __unwindfunclet$?renameProcess@alm_process@@AAEXPAVQListViewItem@@HABVQString@@@Z$3 10020a19 f   alm_process.obj
 0001:0001fa22       __unwindfunclet$?renameProcess@alm_process@@AAEXPAVQListViewItem@@HABVQString@@@Z$4 10020a22 f   alm_process.obj
 0001:0001fa2b       __unwindfunclet$?renameProcess@alm_process@@AAEXPAVQListViewItem@@HABVQString@@@Z$5 10020a2b f   alm_process.obj
 0001:0001fa34       __unwindfunclet$?renameProcess@alm_process@@AAEXPAVQListViewItem@@HABVQString@@@Z$6 10020a34 f   alm_process.obj
 0001:0001fa3d       __ehhandler$?renameProcess@alm_process@@AAEXPAVQListViewItem@@HABVQString@@@Z 10020a3d f   alm_process.obj
 0001:0001fa58       __unwindfunclet$?reply@alm_process@@UAEXPAVresponse@@@Z$0 10020a58 f   alm_process.obj
 0001:0001fa64       __unwindfunclet$?reply@alm_process@@UAEXPAVresponse@@@Z$1 10020a64 f   alm_process.obj
 0001:0001fa70       __unwindfunclet$?reply@alm_process@@UAEXPAVresponse@@@Z$2 10020a70 f   alm_process.obj
 0001:0001fa79       __unwindfunclet$?reply@alm_process@@UAEXPAVresponse@@@Z$30 10020a79 f   alm_process.obj
 0001:0001fa82       __unwindfunclet$?reply@alm_process@@UAEXPAVresponse@@@Z$31 10020a82 f   alm_process.obj
 0001:0001fa8b       __unwindfunclet$?reply@alm_process@@UAEXPAVresponse@@@Z$32 10020a8b f   alm_process.obj
 0001:0001fa94       __unwindfunclet$?reply@alm_process@@UAEXPAVresponse@@@Z$33 10020a94 f   alm_process.obj
 0001:0001faa0       __unwindfunclet$?reply@alm_process@@UAEXPAVresponse@@@Z$34 10020aa0 f   alm_process.obj
 0001:0001faa9       __unwindfunclet$?reply@alm_process@@UAEXPAVresponse@@@Z$36 10020aa9 f   alm_process.obj
 0001:0001fab5       __unwindfunclet$?reply@alm_process@@UAEXPAVresponse@@@Z$37 10020ab5 f   alm_process.obj
 0001:0001fabe       __unwindfunclet$?reply@alm_process@@UAEXPAVresponse@@@Z$38 10020abe f   alm_process.obj
 0001:0001fac7       __unwindfunclet$?reply@alm_process@@UAEXPAVresponse@@@Z$39 10020ac7 f   alm_process.obj
 0001:0001fad0       __unwindfunclet$?reply@alm_process@@UAEXPAVresponse@@@Z$40 10020ad0 f   alm_process.obj
 0001:0001fad9       __unwindfunclet$?reply@alm_process@@UAEXPAVresponse@@@Z$3 10020ad9 f   alm_process.obj
 0001:0001fae2       __unwindfunclet$?reply@alm_process@@UAEXPAVresponse@@@Z$4 10020ae2 f   alm_process.obj
 0001:0001faee       __unwindfunclet$?reply@alm_process@@UAEXPAVresponse@@@Z$5 10020aee f   alm_process.obj
 0001:0001fb08       __unwindfunclet$?reply@alm_process@@UAEXPAVresponse@@@Z$6 10020b08 f   alm_process.obj
 0001:0001fb25       __unwindfunclet$?reply@alm_process@@UAEXPAVresponse@@@Z$7 10020b25 f   alm_process.obj
 0001:0001fb3f       __unwindfunclet$?reply@alm_process@@UAEXPAVresponse@@@Z$8 10020b3f f   alm_process.obj
 0001:0001fb48       __unwindfunclet$?reply@alm_process@@UAEXPAVresponse@@@Z$9 10020b48 f   alm_process.obj
 0001:0001fb51       __unwindfunclet$?reply@alm_process@@UAEXPAVresponse@@@Z$10 10020b51 f   alm_process.obj
 0001:0001fb5a       __unwindfunclet$?reply@alm_process@@UAEXPAVresponse@@@Z$11 10020b5a f   alm_process.obj
 0001:0001fb66       __unwindfunclet$?reply@alm_process@@UAEXPAVresponse@@@Z$12 10020b66 f   alm_process.obj
 0001:0001fb6f       __unwindfunclet$?reply@alm_process@@UAEXPAVresponse@@@Z$13 10020b6f f   alm_process.obj
 0001:0001fb7b       __unwindfunclet$?reply@alm_process@@UAEXPAVresponse@@@Z$14 10020b7b f   alm_process.obj
 0001:0001fb84       __unwindfunclet$?reply@alm_process@@UAEXPAVresponse@@@Z$15 10020b84 f   alm_process.obj
 0001:0001fb90       __unwindfunclet$?reply@alm_process@@UAEXPAVresponse@@@Z$16 10020b90 f   alm_process.obj
 0001:0001fb99       __unwindfunclet$?reply@alm_process@@UAEXPAVresponse@@@Z$17 10020b99 f   alm_process.obj
 0001:0001fba2       __unwindfunclet$?reply@alm_process@@UAEXPAVresponse@@@Z$18 10020ba2 f   alm_process.obj
 0001:0001fbab       __unwindfunclet$?reply@alm_process@@UAEXPAVresponse@@@Z$19 10020bab f   alm_process.obj
 0001:0001fbb4       __unwindfunclet$?reply@alm_process@@UAEXPAVresponse@@@Z$20 10020bb4 f   alm_process.obj
 0001:0001fbbd       __unwindfunclet$?reply@alm_process@@UAEXPAVresponse@@@Z$21 10020bbd f   alm_process.obj
 0001:0001fbc6       __unwindfunclet$?reply@alm_process@@UAEXPAVresponse@@@Z$22 10020bc6 f   alm_process.obj
 0001:0001fbcf       __unwindfunclet$?reply@alm_process@@UAEXPAVresponse@@@Z$23 10020bcf f   alm_process.obj
 0001:0001fbd8       __unwindfunclet$?reply@alm_process@@UAEXPAVresponse@@@Z$24 10020bd8 f   alm_process.obj
 0001:0001fbe1       __unwindfunclet$?reply@alm_process@@UAEXPAVresponse@@@Z$25 10020be1 f   alm_process.obj
 0001:0001fbea       __unwindfunclet$?reply@alm_process@@UAEXPAVresponse@@@Z$26 10020bea f   alm_process.obj
 0001:0001fbf3       __unwindfunclet$?reply@alm_process@@UAEXPAVresponse@@@Z$27 10020bf3 f   alm_process.obj
 0001:0001fbfc       __unwindfunclet$?reply@alm_process@@UAEXPAVresponse@@@Z$28 10020bfc f   alm_process.obj
 0001:0001fc05       __unwindfunclet$?reply@alm_process@@UAEXPAVresponse@@@Z$42 10020c05 f   alm_process.obj
 0001:0001fc0e       __unwindfunclet$?reply@alm_process@@UAEXPAVresponse@@@Z$43 10020c0e f   alm_process.obj
 0001:0001fc17       __unwindfunclet$?reply@alm_process@@UAEXPAVresponse@@@Z$44 10020c17 f   alm_process.obj
 0001:0001fc20       __unwindfunclet$?reply@alm_process@@UAEXPAVresponse@@@Z$45 10020c20 f   alm_process.obj
 0001:0001fc29       __unwindfunclet$?reply@alm_process@@UAEXPAVresponse@@@Z$46 10020c29 f   alm_process.obj
 0001:0001fc32       __unwindfunclet$?reply@alm_process@@UAEXPAVresponse@@@Z$47 10020c32 f   alm_process.obj
 0001:0001fc3b       __unwindfunclet$?reply@alm_process@@UAEXPAVresponse@@@Z$50 10020c3b f   alm_process.obj
 0001:0001fc44       __unwindfunclet$?reply@alm_process@@UAEXPAVresponse@@@Z$51 10020c44 f   alm_process.obj
 0001:0001fc4d       __unwindfunclet$?reply@alm_process@@UAEXPAVresponse@@@Z$52 10020c4d f   alm_process.obj
 0001:0001fc56       __ehhandler$?reply@alm_process@@UAEXPAVresponse@@@Z 10020c56 f   alm_process.obj
 0001:0001fc74       __unwindfunclet$?saveProcesses@alm_process@@AAE_NVQString@@@Z$0 10020c74 f   alm_process.obj
 0001:0001fc7d       __unwindfunclet$?saveProcesses@alm_process@@AAE_NVQString@@@Z$1 10020c7d f   alm_process.obj
 0001:0001fc86       __unwindfunclet$?saveProcesses@alm_process@@AAE_NVQString@@@Z$2 10020c86 f   alm_process.obj
 0001:0001fc8f       __unwindfunclet$?saveProcesses@alm_process@@AAE_NVQString@@@Z$3 10020c8f f   alm_process.obj
 0001:0001fc98       __unwindfunclet$?saveProcesses@alm_process@@AAE_NVQString@@@Z$4 10020c98 f   alm_process.obj
 0001:0001fca4       __unwindfunclet$?saveProcesses@alm_process@@AAE_NVQString@@@Z$5 10020ca4 f   alm_process.obj
 0001:0001fcad       __unwindfunclet$?saveProcesses@alm_process@@AAE_NVQString@@@Z$6 10020cad f   alm_process.obj
 0001:0001fcb6       __unwindfunclet$?saveProcesses@alm_process@@AAE_NVQString@@@Z$7 10020cb6 f   alm_process.obj
 0001:0001fcbf       __unwindfunclet$?saveProcesses@alm_process@@AAE_NVQString@@@Z$8 10020cbf f   alm_process.obj
 0001:0001fcc8       __unwindfunclet$?saveProcesses@alm_process@@AAE_NVQString@@@Z$9 10020cc8 f   alm_process.obj
 0001:0001fcd1       __unwindfunclet$?saveProcesses@alm_process@@AAE_NVQString@@@Z$10 10020cd1 f   alm_process.obj
 0001:0001fcda       __unwindfunclet$?saveProcesses@alm_process@@AAE_NVQString@@@Z$11 10020cda f   alm_process.obj
 0001:0001fce3       __unwindfunclet$?saveProcesses@alm_process@@AAE_NVQString@@@Z$12 10020ce3 f   alm_process.obj
 0001:0001fcec       __ehhandler$?saveProcesses@alm_process@@AAE_NVQString@@@Z 10020cec f   alm_process.obj
 0001:0001fd0a       __unwindfunclet$?selectProcess@alm_process@@AAEXPAVQListViewItem@@@Z$0 10020d0a f   alm_process.obj
 0001:0001fd13       __unwindfunclet$?selectProcess@alm_process@@AAEXPAVQListViewItem@@@Z$1 10020d13 f   alm_process.obj
 0001:0001fd1c       __unwindfunclet$?selectProcess@alm_process@@AAEXPAVQListViewItem@@@Z$2 10020d1c f   alm_process.obj
 0001:0001fd25       __unwindfunclet$?selectProcess@alm_process@@AAEXPAVQListViewItem@@@Z$3 10020d25 f   alm_process.obj
 0001:0001fd2e       __unwindfunclet$?selectProcess@alm_process@@AAEXPAVQListViewItem@@@Z$4 10020d2e f   alm_process.obj
 0001:0001fd37       __unwindfunclet$?selectProcess@alm_process@@AAEXPAVQListViewItem@@@Z$5 10020d37 f   alm_process.obj
 0001:0001fd40       __unwindfunclet$?selectProcess@alm_process@@AAEXPAVQListViewItem@@@Z$16 10020d40 f   alm_process.obj
 0001:0001fd49       __unwindfunclet$?selectProcess@alm_process@@AAEXPAVQListViewItem@@@Z$17 10020d49 f   alm_process.obj
 0001:0001fd53       __unwindfunclet$?selectProcess@alm_process@@AAEXPAVQListViewItem@@@Z$18 10020d53 f   alm_process.obj
 0001:0001fd5c       __unwindfunclet$?selectProcess@alm_process@@AAEXPAVQListViewItem@@@Z$19 10020d5c f   alm_process.obj
 0001:0001fd65       __unwindfunclet$?selectProcess@alm_process@@AAEXPAVQListViewItem@@@Z$20 10020d65 f   alm_process.obj
 0001:0001fd6e       __unwindfunclet$?selectProcess@alm_process@@AAEXPAVQListViewItem@@@Z$21 10020d6e f   alm_process.obj
 0001:0001fd77       __unwindfunclet$?selectProcess@alm_process@@AAEXPAVQListViewItem@@@Z$22 10020d77 f   alm_process.obj
 0001:0001fd80       __unwindfunclet$?selectProcess@alm_process@@AAEXPAVQListViewItem@@@Z$23 10020d80 f   alm_process.obj
 0001:0001fd89       __unwindfunclet$?selectProcess@alm_process@@AAEXPAVQListViewItem@@@Z$24 10020d89 f   alm_process.obj
 0001:0001fd92       __unwindfunclet$?selectProcess@alm_process@@AAEXPAVQListViewItem@@@Z$6 10020d92 f   alm_process.obj
 0001:0001fd9b       __unwindfunclet$?selectProcess@alm_process@@AAEXPAVQListViewItem@@@Z$7 10020d9b f   alm_process.obj
 0001:0001fda5       __unwindfunclet$?selectProcess@alm_process@@AAEXPAVQListViewItem@@@Z$8 10020da5 f   alm_process.obj
 0001:0001fdae       __unwindfunclet$?selectProcess@alm_process@@AAEXPAVQListViewItem@@@Z$9 10020dae f   alm_process.obj
 0001:0001fdb7       __unwindfunclet$?selectProcess@alm_process@@AAEXPAVQListViewItem@@@Z$10 10020db7 f   alm_process.obj
 0001:0001fdc0       __unwindfunclet$?selectProcess@alm_process@@AAEXPAVQListViewItem@@@Z$11 10020dc0 f   alm_process.obj
 0001:0001fdc9       __unwindfunclet$?selectProcess@alm_process@@AAEXPAVQListViewItem@@@Z$12 10020dc9 f   alm_process.obj
 0001:0001fdd2       __unwindfunclet$?selectProcess@alm_process@@AAEXPAVQListViewItem@@@Z$13 10020dd2 f   alm_process.obj
 0001:0001fddb       __unwindfunclet$?selectProcess@alm_process@@AAEXPAVQListViewItem@@@Z$14 10020ddb f   alm_process.obj
 0001:0001fde4       __unwindfunclet$?selectProcess@alm_process@@AAEXPAVQListViewItem@@@Z$26 10020de4 f   alm_process.obj
 0001:0001fded       __unwindfunclet$?selectProcess@alm_process@@AAEXPAVQListViewItem@@@Z$27 10020ded f   alm_process.obj
 0001:0001fdf7       __unwindfunclet$?selectProcess@alm_process@@AAEXPAVQListViewItem@@@Z$28 10020df7 f   alm_process.obj
 0001:0001fe00       __unwindfunclet$?selectProcess@alm_process@@AAEXPAVQListViewItem@@@Z$29 10020e00 f   alm_process.obj
 0001:0001fe09       __unwindfunclet$?selectProcess@alm_process@@AAEXPAVQListViewItem@@@Z$30 10020e09 f   alm_process.obj
 0001:0001fe12       __unwindfunclet$?selectProcess@alm_process@@AAEXPAVQListViewItem@@@Z$31 10020e12 f   alm_process.obj
 0001:0001fe1b       __unwindfunclet$?selectProcess@alm_process@@AAEXPAVQListViewItem@@@Z$32 10020e1b f   alm_process.obj
 0001:0001fe24       __unwindfunclet$?selectProcess@alm_process@@AAEXPAVQListViewItem@@@Z$33 10020e24 f   alm_process.obj
 0001:0001fe2d       __unwindfunclet$?selectProcess@alm_process@@AAEXPAVQListViewItem@@@Z$34 10020e2d f   alm_process.obj
 0001:0001fe36       __unwindfunclet$?selectProcess@alm_process@@AAEXPAVQListViewItem@@@Z$36 10020e36 f   alm_process.obj
 0001:0001fe3f       __unwindfunclet$?selectProcess@alm_process@@AAEXPAVQListViewItem@@@Z$37 10020e3f f   alm_process.obj
 0001:0001fe48       __unwindfunclet$?selectProcess@alm_process@@AAEXPAVQListViewItem@@@Z$38 10020e48 f   alm_process.obj
 0001:0001fe51       __unwindfunclet$?selectProcess@alm_process@@AAEXPAVQListViewItem@@@Z$39 10020e51 f   alm_process.obj
 0001:0001fe5a       __unwindfunclet$?selectProcess@alm_process@@AAEXPAVQListViewItem@@@Z$40 10020e5a f   alm_process.obj
 0001:0001fe63       __ehhandler$?selectProcess@alm_process@@AAEXPAVQListViewItem@@@Z 10020e63 f   alm_process.obj
 0001:0001fe7e       __unwindfunclet$?selectProcess@alm_process@@AAEXVQString@@@Z$0 10020e7e f   alm_process.obj
 0001:0001fe87       __unwindfunclet$?selectProcess@alm_process@@AAEXVQString@@@Z$1 10020e87 f   alm_process.obj
 0001:0001fe90       __unwindfunclet$?selectProcess@alm_process@@AAEXVQString@@@Z$2 10020e90 f   alm_process.obj
 0001:0001fe99       __ehhandler$?selectProcess@alm_process@@AAEXVQString@@@Z 10020e99 f   alm_process.obj
 0001:0001feb7       __unwindfunclet$?selectSystem@alm_process@@AAEXABVQString@@@Z$0 10020eb7 f   alm_process.obj
 0001:0001fec0       __unwindfunclet$?selectSystem@alm_process@@AAEXABVQString@@@Z$1 10020ec0 f   alm_process.obj
 0001:0001fec9       __unwindfunclet$?selectSystem@alm_process@@AAEXABVQString@@@Z$2 10020ec9 f   alm_process.obj
 0001:0001fed2       __unwindfunclet$?selectSystem@alm_process@@AAEXABVQString@@@Z$3 10020ed2 f   alm_process.obj
 0001:0001fedb       __unwindfunclet$?selectSystem@alm_process@@AAEXABVQString@@@Z$4 10020edb f   alm_process.obj
 0001:0001fee4       __unwindfunclet$?selectSystem@alm_process@@AAEXABVQString@@@Z$6 10020ee4 f   alm_process.obj
 0001:0001feed       __unwindfunclet$?selectSystem@alm_process@@AAEXABVQString@@@Z$7 10020eed f   alm_process.obj
 0001:0001fef6       __unwindfunclet$?selectSystem@alm_process@@AAEXABVQString@@@Z$8 10020ef6 f   alm_process.obj
 0001:0001feff       __unwindfunclet$?selectSystem@alm_process@@AAEXABVQString@@@Z$9 10020eff f   alm_process.obj
 0001:0001ff08       __unwindfunclet$?selectSystem@alm_process@@AAEXABVQString@@@Z$10 10020f08 f   alm_process.obj
 0001:0001ff11       __unwindfunclet$?selectSystem@alm_process@@AAEXABVQString@@@Z$12 10020f11 f   alm_process.obj
 0001:0001ff1a       __unwindfunclet$?selectSystem@alm_process@@AAEXABVQString@@@Z$13 10020f1a f   alm_process.obj
 0001:0001ff23       __unwindfunclet$?selectSystem@alm_process@@AAEXABVQString@@@Z$14 10020f23 f   alm_process.obj
 0001:0001ff2c       __unwindfunclet$?selectSystem@alm_process@@AAEXABVQString@@@Z$15 10020f2c f   alm_process.obj
 0001:0001ff35       __unwindfunclet$?selectSystem@alm_process@@AAEXABVQString@@@Z$17 10020f35 f   alm_process.obj
 0001:0001ff3e       __unwindfunclet$?selectSystem@alm_process@@AAEXABVQString@@@Z$18 10020f3e f   alm_process.obj
 0001:0001ff47       __unwindfunclet$?selectSystem@alm_process@@AAEXABVQString@@@Z$19 10020f47 f   alm_process.obj
 0001:0001ff50       __unwindfunclet$?selectSystem@alm_process@@AAEXABVQString@@@Z$20 10020f50 f   alm_process.obj
 0001:0001ff59       __unwindfunclet$?selectSystem@alm_process@@AAEXABVQString@@@Z$21 10020f59 f   alm_process.obj
 0001:0001ff62       __unwindfunclet$?selectSystem@alm_process@@AAEXABVQString@@@Z$22 10020f62 f   alm_process.obj
 0001:0001ff6b       __unwindfunclet$?selectSystem@alm_process@@AAEXABVQString@@@Z$23 10020f6b f   alm_process.obj
 0001:0001ff74       __unwindfunclet$?selectSystem@alm_process@@AAEXABVQString@@@Z$24 10020f74 f   alm_process.obj
 0001:0001ff7d       __unwindfunclet$?selectSystem@alm_process@@AAEXABVQString@@@Z$26 10020f7d f   alm_process.obj
 0001:0001ff86       __unwindfunclet$?selectSystem@alm_process@@AAEXABVQString@@@Z$27 10020f86 f   alm_process.obj
 0001:0001ff8f       __unwindfunclet$?selectSystem@alm_process@@AAEXABVQString@@@Z$28 10020f8f f   alm_process.obj
 0001:0001ff98       __unwindfunclet$?selectSystem@alm_process@@AAEXABVQString@@@Z$29 10020f98 f   alm_process.obj
 0001:0001ffa1       __unwindfunclet$?selectSystem@alm_process@@AAEXABVQString@@@Z$31 10020fa1 f   alm_process.obj
 0001:0001ffaa       __unwindfunclet$?selectSystem@alm_process@@AAEXABVQString@@@Z$32 10020faa f   alm_process.obj
 0001:0001ffb3       __unwindfunclet$?selectSystem@alm_process@@AAEXABVQString@@@Z$33 10020fb3 f   alm_process.obj
 0001:0001ffbc       __unwindfunclet$?selectSystem@alm_process@@AAEXABVQString@@@Z$34 10020fbc f   alm_process.obj
 0001:0001ffc5       __unwindfunclet$?selectSystem@alm_process@@AAEXABVQString@@@Z$35 10020fc5 f   alm_process.obj
 0001:0001ffce       __unwindfunclet$?selectSystem@alm_process@@AAEXABVQString@@@Z$36 10020fce f   alm_process.obj
 0001:0001ffd7       __unwindfunclet$?selectSystem@alm_process@@AAEXABVQString@@@Z$37 10020fd7 f   alm_process.obj
 0001:0001ffe0       __unwindfunclet$?selectSystem@alm_process@@AAEXABVQString@@@Z$38 10020fe0 f   alm_process.obj
 0001:0001ffe9       __unwindfunclet$?selectSystem@alm_process@@AAEXABVQString@@@Z$40 10020fe9 f   alm_process.obj
 0001:0001fff2       __unwindfunclet$?selectSystem@alm_process@@AAEXABVQString@@@Z$41 10020ff2 f   alm_process.obj
 0001:0001fffb       __unwindfunclet$?selectSystem@alm_process@@AAEXABVQString@@@Z$42 10020ffb f   alm_process.obj
 0001:00020004       __unwindfunclet$?selectSystem@alm_process@@AAEXABVQString@@@Z$43 10021004 f   alm_process.obj
 0001:0002000d       __unwindfunclet$?selectSystem@alm_process@@AAEXABVQString@@@Z$45 1002100d f   alm_process.obj
 0001:00020016       __ehhandler$?selectSystem@alm_process@@AAEXABVQString@@@Z 10021016 f   alm_process.obj
 0001:00020031       __unwindfunclet$?setLatchAck@alm_process@@AAEXXZ$0 10021031 f   alm_process.obj
 0001:00020039       __unwindfunclet$?setLatchAck@alm_process@@AAEXXZ$1 10021039 f   alm_process.obj
 0001:00020042       __unwindfunclet$?setLatchAck@alm_process@@AAEXXZ$2 10021042 f   alm_process.obj
 0001:0002004c       __unwindfunclet$?setLatchAck@alm_process@@AAEXXZ$3 1002104c f   alm_process.obj
 0001:00020055       __ehhandler$?setLatchAck@alm_process@@AAEXXZ 10021055 f   alm_process.obj
 0001:00020070       __unwindfunclet$?setMask@alm_process@@AAEXXZ$0 10021070 f   alm_process.obj
 0001:00020078       __unwindfunclet$?setMask@alm_process@@AAEXXZ$1 10021078 f   alm_process.obj
 0001:00020081       __unwindfunclet$?setMask@alm_process@@AAEXXZ$2 10021081 f   alm_process.obj
 0001:0002008b       __unwindfunclet$?setMask@alm_process@@AAEXXZ$3 1002108b f   alm_process.obj
 0001:00020094       __unwindfunclet$?setMask@alm_process@@AAEXXZ$4 10021094 f   alm_process.obj
 0001:0002009d       __ehhandler$?setMask@alm_process@@AAEXXZ 1002109d f   alm_process.obj
 0001:000200b8       __unwindfunclet$?setProcessGroup@alm_process@@AAEXXZ$0 100210b8 f   alm_process.obj
 0001:000200c0       __unwindfunclet$?setProcessGroup@alm_process@@AAEXXZ$1 100210c0 f   alm_process.obj
 0001:000200c9       __unwindfunclet$?setProcessGroup@alm_process@@AAEXXZ$2 100210c9 f   alm_process.obj
 0001:000200d2       __unwindfunclet$?setProcessGroup@alm_process@@AAEXXZ$3 100210d2 f   alm_process.obj
 0001:000200db       __unwindfunclet$?setProcessGroup@alm_process@@AAEXXZ$4 100210db f   alm_process.obj
 0001:000200e4       __unwindfunclet$?setProcessGroup@alm_process@@AAEXXZ$5 100210e4 f   alm_process.obj
 0001:000200ed       __ehhandler$?setProcessGroup@alm_process@@AAEXXZ 100210ed f   alm_process.obj
 0001:00020108       __unwindfunclet$?sysCommand@alm_process@@AAEXABVQString@@0@Z$0 10021108 f   alm_process.obj
 0001:00020111       __ehhandler$?sysCommand@alm_process@@AAEXABVQString@@0@Z 10021111 f   alm_process.obj
 0001:0002012c       __unwindfunclet$?toolbars@alm_process@@UAE?AVQDockWindowList@@XZ$0 1002112c f   alm_process.obj
 0001:00020145       __ehhandler$?toolbars@alm_process@@UAE?AVQDockWindowList@@XZ 10021145 f   alm_process.obj
 0001:00020160       __unwindfunclet$?setText@config_mb4@@QAEXVQString@@@Z$0 10021160 f   alm_process.obj
 0001:00020160       __unwindfunclet$?updateProcList@alm_process@@AAEXPAVcProcess@@@Z$0 10021160 f   alm_process.obj
 0001:00020160       __unwindfunclet$?setOldPrefix@template_dialog@@QAEXVQString@@@Z$0 10021160 f   alm_process.obj
 0001:00020169       __ehhandler$?setOldPrefix@template_dialog@@QAEXVQString@@@Z 10021169 f   alm_process.obj
 0001:00020169       __ehhandler$?setText@config_mb4@@QAEXVQString@@@Z 10021169 f   alm_process.obj
 0001:00020169       __ehhandler$?updateProcList@alm_process@@AAEXPAVcProcess@@@Z 10021169 f   alm_process.obj
 0001:00020184       __unwindfunclet$??0cAcqFileData@@QAE@VQString@@@Z$0 10021184 f   cAcqFileData.obj
 0001:0002018d       __unwindfunclet$??0cAcqFileData@@QAE@VQString@@@Z$1 1002118d f   cAcqFileData.obj
 0001:00020199       __unwindfunclet$??0cAcqFileData@@QAE@VQString@@@Z$2 10021199 f   cAcqFileData.obj
 0001:000201a5       __unwindfunclet$??0cAcqFileData@@QAE@VQString@@@Z$3 100211a5 f   cAcqFileData.obj
 0001:000201b1       __unwindfunclet$??0cAcqFileData@@QAE@VQString@@@Z$4 100211b1 f   cAcqFileData.obj
 0001:000201bd       __unwindfunclet$??0cAcqFileData@@QAE@VQString@@@Z$5 100211bd f   cAcqFileData.obj
 0001:000201c9       __unwindfunclet$??0cAcqFileData@@QAE@VQString@@@Z$6 100211c9 f   cAcqFileData.obj
 0001:000201d5       __ehhandler$??0cAcqFileData@@QAE@VQString@@@Z 100211d5 f   cAcqFileData.obj
 0001:000201f0       __unwindfunclet$??1cAcqFileData@@UAE@XZ$0 100211f0 f   cAcqFileData.obj
 0001:000201fc       __unwindfunclet$??1cAcqFileData@@UAE@XZ$1 100211fc f   cAcqFileData.obj
 0001:00020208       __unwindfunclet$??1cAcqFileData@@UAE@XZ$2 10021208 f   cAcqFileData.obj
 0001:00020214       __unwindfunclet$??1cAcqFileData@@UAE@XZ$3 10021214 f   cAcqFileData.obj
 0001:00020220       __unwindfunclet$??1cAcqFileData@@UAE@XZ$4 10021220 f   cAcqFileData.obj
 0001:0002022c       __ehhandler$??1cAcqFileData@@UAE@XZ 1002122c f   cAcqFileData.obj
 0001:00020247       __unwindfunclet$?findSlot@cAcqFileData@@QAE?AVQString@@H@Z$0 10021247 f   cAcqFileData.obj
 0001:00020250       __unwindfunclet$?findSlot@cAcqFileData@@QAE?AVQString@@H@Z$1 10021250 f   cAcqFileData.obj
 0001:0002026a       __ehhandler$?findSlot@cAcqFileData@@QAE?AVQString@@H@Z 1002126a f   cAcqFileData.obj
 0001:00020285       __unwindfunclet$?findSlot@cAcqFileData@@QAEHVQString@@@Z$0 10021285 f   cAcqFileData.obj
 0001:00020285       __unwindfunclet$?setMask@cProc_dialog@@QAEXVQString@@@Z$0 10021285 f   cAcqFileData.obj
 0001:0002028e       __ehhandler$?setMask@cProc_dialog@@QAEXVQString@@@Z 1002128e f   cAcqFileData.obj
 0001:0002028e       __ehhandler$?findSlot@cAcqFileData@@QAEHVQString@@@Z 1002128e f   cAcqFileData.obj
 0001:000202a9       __unwindfunclet$?loadDetails@cAcqFileData@@QAE_NXZ$0 100212a9 f   cAcqFileData.obj
 0001:000202b2       __unwindfunclet$?loadDetails@cAcqFileData@@QAE_NXZ$1 100212b2 f   cAcqFileData.obj
 0001:000202be       __unwindfunclet$?loadDetails@cAcqFileData@@QAE_NXZ$2 100212be f   cAcqFileData.obj
 0001:000202ca       __unwindfunclet$?loadDetails@cAcqFileData@@QAE_NXZ$3 100212ca f   cAcqFileData.obj
 0001:000202d3       __unwindfunclet$?loadDetails@cAcqFileData@@QAE_NXZ$4 100212d3 f   cAcqFileData.obj
 0001:000202dc       __unwindfunclet$?loadDetails@cAcqFileData@@QAE_NXZ$5 100212dc f   cAcqFileData.obj
 0001:000202e5       __unwindfunclet$?loadDetails@cAcqFileData@@QAE_NXZ$6 100212e5 f   cAcqFileData.obj
 0001:000202ee       __unwindfunclet$?loadDetails@cAcqFileData@@QAE_NXZ$7 100212ee f   cAcqFileData.obj
 0001:00020308       __unwindfunclet$?loadDetails@cAcqFileData@@QAE_NXZ$8 10021308 f   cAcqFileData.obj
 0001:00020322       __unwindfunclet$?loadDetails@cAcqFileData@@QAE_NXZ$9 10021322 f   cAcqFileData.obj
 0001:0002032b       __unwindfunclet$?loadDetails@cAcqFileData@@QAE_NXZ$10 1002132b f   cAcqFileData.obj
 0001:00020334       __unwindfunclet$?loadDetails@cAcqFileData@@QAE_NXZ$11 10021334 f   cAcqFileData.obj
 0001:0002033d       __unwindfunclet$?loadDetails@cAcqFileData@@QAE_NXZ$12 1002133d f   cAcqFileData.obj
 0001:00020346       __unwindfunclet$?loadDetails@cAcqFileData@@QAE_NXZ$13 10021346 f   cAcqFileData.obj
 0001:0002034f       __unwindfunclet$?loadDetails@cAcqFileData@@QAE_NXZ$14 1002134f f   cAcqFileData.obj
 0001:00020358       __unwindfunclet$?loadDetails@cAcqFileData@@QAE_NXZ$15 10021358 f   cAcqFileData.obj
 0001:00020361       __unwindfunclet$?loadDetails@cAcqFileData@@QAE_NXZ$16 10021361 f   cAcqFileData.obj
 0001:0002036a       __ehhandler$?loadDetails@cAcqFileData@@QAE_NXZ 1002136a f   cAcqFileData.obj
 0001:00020388       __unwindfunclet$?accept@CheckContDialog@@UAEXXZ$0 10021388 f   checkContDialogImpl.obj
 0001:00020391       __unwindfunclet$?accept@CheckContDialog@@UAEXXZ$1 10021391 f   checkContDialogImpl.obj
 0001:0002039a       __ehhandler$?accept@CheckContDialog@@UAEXXZ 1002139a f   checkContDialogImpl.obj
 0001:000203b5       __unwindfunclet$??0cProc_dialog@@QAE@QAVQStringList@@PAVQWidget@@PBDI@Z$0 100213b5 f   cProc_dialog.obj
 0001:000203bd       __unwindfunclet$??0cProc_dialog@@QAE@QAVQStringList@@PAVQWidget@@PBDI@Z$1 100213bd f   cProc_dialog.obj
 0001:000203c7       __unwindfunclet$??0cProc_dialog@@QAE@QAVQStringList@@PAVQWidget@@PBDI@Z$2 100213c7 f   cProc_dialog.obj
 0001:000203d0       __unwindfunclet$??0cProc_dialog@@QAE@QAVQStringList@@PAVQWidget@@PBDI@Z$3 100213d0 f   cProc_dialog.obj
 0001:000203d9       __unwindfunclet$??0cProc_dialog@@QAE@QAVQStringList@@PAVQWidget@@PBDI@Z$4 100213d9 f   cProc_dialog.obj
 0001:000203e2       __unwindfunclet$??0cProc_dialog@@QAE@QAVQStringList@@PAVQWidget@@PBDI@Z$5 100213e2 f   cProc_dialog.obj
 0001:000203eb       __unwindfunclet$??0cProc_dialog@@QAE@QAVQStringList@@PAVQWidget@@PBDI@Z$6 100213eb f   cProc_dialog.obj
 0001:000203f4       __unwindfunclet$??0cProc_dialog@@QAE@QAVQStringList@@PAVQWidget@@PBDI@Z$7 100213f4 f   cProc_dialog.obj
 0001:000203fd       __unwindfunclet$??0cProc_dialog@@QAE@QAVQStringList@@PAVQWidget@@PBDI@Z$8 100213fd f   cProc_dialog.obj
 0001:00020406       __unwindfunclet$??0cProc_dialog@@QAE@QAVQStringList@@PAVQWidget@@PBDI@Z$9 10021406 f   cProc_dialog.obj
 0001:0002040f       __unwindfunclet$??0cProc_dialog@@QAE@QAVQStringList@@PAVQWidget@@PBDI@Z$10 1002140f f   cProc_dialog.obj
 0001:00020418       __unwindfunclet$??0cProc_dialog@@QAE@QAVQStringList@@PAVQWidget@@PBDI@Z$11 10021418 f   cProc_dialog.obj
 0001:00020421       __ehhandler$??0cProc_dialog@@QAE@QAVQStringList@@PAVQWidget@@PBDI@Z 10021421 f   cProc_dialog.obj
 0001:0002043c       __unwindfunclet$??1cProc_dialog@@UAE@XZ$0 1002143c f   cProc_dialog.obj
 0001:00020444       __unwindfunclet$??1cProc_dialog@@UAE@XZ$1 10021444 f   cProc_dialog.obj
 0001:0002044d       __unwindfunclet$??1cProc_dialog@@UAE@XZ$2 1002144d f   cProc_dialog.obj
 0001:00020456       __unwindfunclet$??1cProc_dialog@@UAE@XZ$3 10021456 f   cProc_dialog.obj
 0001:0002045f       __unwindfunclet$??1cProc_dialog@@UAE@XZ$4 1002145f f   cProc_dialog.obj
 0001:00020468       __unwindfunclet$??1cProc_dialog@@UAE@XZ$5 10021468 f   cProc_dialog.obj
 0001:00020471       __unwindfunclet$??1cProc_dialog@@UAE@XZ$6 10021471 f   cProc_dialog.obj
 0001:0002047a       __ehhandler$??1cProc_dialog@@UAE@XZ 1002147a f   cProc_dialog.obj
 0001:00020495       __unwindfunclet$?applyProc@cProc_dialog@@QAE_NXZ$0 10021495 f   cProc_dialog.obj
 0001:0002049e       __unwindfunclet$?applyProc@cProc_dialog@@QAE_NXZ$1 1002149e f   cProc_dialog.obj
 0001:000204a7       __unwindfunclet$?applyProc@cProc_dialog@@QAE_NXZ$2 100214a7 f   cProc_dialog.obj
 0001:000204b0       __unwindfunclet$?applyProc@cProc_dialog@@QAE_NXZ$3 100214b0 f   cProc_dialog.obj
 0001:000204b9       __unwindfunclet$?applyProc@cProc_dialog@@QAE_NXZ$15 100214b9 f   cProc_dialog.obj
 0001:000204c2       __unwindfunclet$?applyProc@cProc_dialog@@QAE_NXZ$16 100214c2 f   cProc_dialog.obj
 0001:000204cb       __unwindfunclet$?applyProc@cProc_dialog@@QAE_NXZ$10 100214cb f   cProc_dialog.obj
 0001:000204d4       __unwindfunclet$?applyProc@cProc_dialog@@QAE_NXZ$11 100214d4 f   cProc_dialog.obj
 0001:000204dd       __unwindfunclet$?applyProc@cProc_dialog@@QAE_NXZ$12 100214dd f   cProc_dialog.obj
 0001:000204e6       __unwindfunclet$?applyProc@cProc_dialog@@QAE_NXZ$13 100214e6 f   cProc_dialog.obj
 0001:000204ef       __unwindfunclet$?applyProc@cProc_dialog@@QAE_NXZ$14 100214ef f   cProc_dialog.obj
 0001:000204f8       __unwindfunclet$?applyProc@cProc_dialog@@QAE_NXZ$7 100214f8 f   cProc_dialog.obj
 0001:00020501       __unwindfunclet$?applyProc@cProc_dialog@@QAE_NXZ$8 10021501 f   cProc_dialog.obj
 0001:0002050a       __unwindfunclet$?applyProc@cProc_dialog@@QAE_NXZ$9 1002150a f   cProc_dialog.obj
 0001:00020513       __unwindfunclet$?applyProc@cProc_dialog@@QAE_NXZ$6 10021513 f   cProc_dialog.obj
 0001:0002051c       __unwindfunclet$?applyProc@cProc_dialog@@QAE_NXZ$5 1002151c f   cProc_dialog.obj
 0001:00020525       __unwindfunclet$?applyProc@cProc_dialog@@QAE_NXZ$4 10021525 f   cProc_dialog.obj
 0001:0002052e       __ehhandler$?applyProc@cProc_dialog@@QAE_NXZ 1002152e f   cProc_dialog.obj
 0001:00020549       __unwindfunclet$?changeFunction@cProc_dialog@@IAEXABVQString@@@Z$0 10021549 f   cProc_dialog.obj
 0001:00020552       __unwindfunclet$?changeFunction@cProc_dialog@@IAEXABVQString@@@Z$1 10021552 f   cProc_dialog.obj
 0001:0002055b       __ehhandler$?changeFunction@cProc_dialog@@IAEXABVQString@@@Z 1002155b f   cProc_dialog.obj
 0001:00020576       __unwindfunclet$?changeHoldoff@cProc_dialog@@IAEXABVQString@@@Z$0 10021576 f   cProc_dialog.obj
 0001:00020576       __unwindfunclet$?updateProcessCount@cProc_dialog@@QAEXH@Z$0 10021576 f   cProc_dialog.obj
 0001:0002057f       __ehhandler$?changeHoldoff@cProc_dialog@@IAEXABVQString@@@Z 1002157f f   cProc_dialog.obj
 0001:0002057f       __ehhandler$?updateProcessCount@cProc_dialog@@QAEXH@Z 1002157f f   cProc_dialog.obj
 0001:0002059a       __unwindfunclet$?clear@cProc_dialog@@QAEX_N@Z$0 1002159a f   cProc_dialog.obj
 0001:000205a3       __unwindfunclet$?clear@cProc_dialog@@QAEX_N@Z$1 100215a3 f   cProc_dialog.obj
 0001:000205ac       __unwindfunclet$?clear@cProc_dialog@@QAEX_N@Z$2 100215ac f   cProc_dialog.obj
 0001:000205b5       __ehhandler$?clear@cProc_dialog@@QAEX_N@Z 100215b5 f   cProc_dialog.obj
 0001:000205d0       __unwindfunclet$?editAcqSlot@cProc_dialog@@QAEXXZ$0 100215d0 f   cProc_dialog.obj
 0001:000205d9       __unwindfunclet$?editAcqSlot@cProc_dialog@@QAEXXZ$1 100215d9 f   cProc_dialog.obj
 0001:000205e2       __unwindfunclet$?editAcqSlot@cProc_dialog@@QAEXXZ$2 100215e2 f   cProc_dialog.obj
 0001:000205eb       __unwindfunclet$?editAcqSlot@cProc_dialog@@QAEXXZ$3 100215eb f   cProc_dialog.obj
 0001:000205f4       __ehhandler$?editAcqSlot@cProc_dialog@@QAEXXZ 100215f4 f   cProc_dialog.obj
 0001:0002060f       __unwindfunclet$?endTimeChanged@cProc_dialog@@IAEXABVQTime@@@Z$0 1002160f f   cProc_dialog.obj
 0001:0002060f       __unwindfunclet$?startTimeChanged@cProc_dialog@@IAEXABVQTime@@@Z$0 1002160f f   cProc_dialog.obj
 0001:00020618       __unwindfunclet$?startTimeChanged@cProc_dialog@@IAEXABVQTime@@@Z$1 10021618 f   cProc_dialog.obj
 0001:00020618       __unwindfunclet$?endTimeChanged@cProc_dialog@@IAEXABVQTime@@@Z$1 10021618 f   cProc_dialog.obj
 0001:00020621       __ehhandler$?endTimeChanged@cProc_dialog@@IAEXABVQTime@@@Z 10021621 f   cProc_dialog.obj
 0001:00020621       __ehhandler$?startTimeChanged@cProc_dialog@@IAEXABVQTime@@@Z 10021621 f   cProc_dialog.obj
 0001:0002063c       __unwindfunclet$?loadAcqFiles@cProc_dialog@@QAE_NVQString@@@Z$0 1002163c f   cProc_dialog.obj
 0001:00020645       __unwindfunclet$?loadAcqFiles@cProc_dialog@@QAE_NVQString@@@Z$1 10021645 f   cProc_dialog.obj
 0001:0002064e       __unwindfunclet$?loadAcqFiles@cProc_dialog@@QAE_NVQString@@@Z$2 1002164e f   cProc_dialog.obj
 0001:00020657       __unwindfunclet$?loadAcqFiles@cProc_dialog@@QAE_NVQString@@@Z$3 10021657 f   cProc_dialog.obj
 0001:00020660       __unwindfunclet$?loadAcqFiles@cProc_dialog@@QAE_NVQString@@@Z$4 10021660 f   cProc_dialog.obj
 0001:00020669       __unwindfunclet$?loadAcqFiles@cProc_dialog@@QAE_NVQString@@@Z$5 10021669 f   cProc_dialog.obj
 0001:00020672       __unwindfunclet$?loadAcqFiles@cProc_dialog@@QAE_NVQString@@@Z$6 10021672 f   cProc_dialog.obj
 0001:0002067b       __unwindfunclet$?loadAcqFiles@cProc_dialog@@QAE_NVQString@@@Z$7 1002167b f   cProc_dialog.obj
 0001:00020684       __unwindfunclet$?loadAcqFiles@cProc_dialog@@QAE_NVQString@@@Z$8 10021684 f   cProc_dialog.obj
 0001:0002068d       __unwindfunclet$?loadAcqFiles@cProc_dialog@@QAE_NVQString@@@Z$9 1002168d f   cProc_dialog.obj
 0001:00020696       __unwindfunclet$?loadAcqFiles@cProc_dialog@@QAE_NVQString@@@Z$10 10021696 f   cProc_dialog.obj
 0001:0002069f       __unwindfunclet$?loadAcqFiles@cProc_dialog@@QAE_NVQString@@@Z$11 1002169f f   cProc_dialog.obj
 0001:000206a9       __unwindfunclet$?loadAcqFiles@cProc_dialog@@QAE_NVQString@@@Z$13 100216a9 f   cProc_dialog.obj
 0001:000206b2       __unwindfunclet$?loadAcqFiles@cProc_dialog@@QAE_NVQString@@@Z$14 100216b2 f   cProc_dialog.obj
 0001:000206bc       __unwindfunclet$?loadAcqFiles@cProc_dialog@@QAE_NVQString@@@Z$16 100216bc f   cProc_dialog.obj
 0001:000206c5       __ehhandler$?loadAcqFiles@cProc_dialog@@QAE_NVQString@@@Z 100216c5 f   cProc_dialog.obj
 0001:000206e0       __unwindfunclet$?loadOutputModules@cProc_dialog@@QAE_NVQString@@@Z$0 100216e0 f   cProc_dialog.obj
 0001:000206e9       __unwindfunclet$?loadOutputModules@cProc_dialog@@QAE_NVQString@@@Z$1 100216e9 f   cProc_dialog.obj
 0001:000206f5       __unwindfunclet$?loadOutputModules@cProc_dialog@@QAE_NVQString@@@Z$2 100216f5 f   cProc_dialog.obj
 0001:00020701       __unwindfunclet$?loadOutputModules@cProc_dialog@@QAE_NVQString@@@Z$3 10021701 f   cProc_dialog.obj
 0001:0002070d       __unwindfunclet$?loadOutputModules@cProc_dialog@@QAE_NVQString@@@Z$4 1002170d f   cProc_dialog.obj
 0001:00020719       __unwindfunclet$?loadOutputModules@cProc_dialog@@QAE_NVQString@@@Z$5 10021719 f   cProc_dialog.obj
 0001:00020725       __unwindfunclet$?loadOutputModules@cProc_dialog@@QAE_NVQString@@@Z$6 10021725 f   cProc_dialog.obj
 0001:00020731       __unwindfunclet$?loadOutputModules@cProc_dialog@@QAE_NVQString@@@Z$7 10021731 f   cProc_dialog.obj
 0001:0002073d       __unwindfunclet$?loadOutputModules@cProc_dialog@@QAE_NVQString@@@Z$8 1002173d f   cProc_dialog.obj
 0001:00020749       __unwindfunclet$?loadOutputModules@cProc_dialog@@QAE_NVQString@@@Z$9 10021749 f   cProc_dialog.obj
 0001:00020755       __unwindfunclet$?loadOutputModules@cProc_dialog@@QAE_NVQString@@@Z$10 10021755 f   cProc_dialog.obj
 0001:00020762       __unwindfunclet$?loadOutputModules@cProc_dialog@@QAE_NVQString@@@Z$11 10021762 f   cProc_dialog.obj
 0001:0002076e       __unwindfunclet$?loadOutputModules@cProc_dialog@@QAE_NVQString@@@Z$12 1002176e f   cProc_dialog.obj
 0001:0002077a       __unwindfunclet$?loadOutputModules@cProc_dialog@@QAE_NVQString@@@Z$13 1002177a f   cProc_dialog.obj
 0001:00020786       __unwindfunclet$?loadOutputModules@cProc_dialog@@QAE_NVQString@@@Z$14 10021786 f   cProc_dialog.obj
 0001:00020792       __unwindfunclet$?loadOutputModules@cProc_dialog@@QAE_NVQString@@@Z$15 10021792 f   cProc_dialog.obj
 0001:0002079e       __unwindfunclet$?loadOutputModules@cProc_dialog@@QAE_NVQString@@@Z$16 1002179e f   cProc_dialog.obj
 0001:000207aa       __unwindfunclet$?loadOutputModules@cProc_dialog@@QAE_NVQString@@@Z$17 100217aa f   cProc_dialog.obj
 0001:000207b6       __ehhandler$?loadOutputModules@cProc_dialog@@QAE_NVQString@@@Z 100217b6 f   cProc_dialog.obj
 0001:000207de       __unwindfunclet$?navOutputModule@cProc_dialog@@IAEXXZ$0 100217de f   cProc_dialog.obj
 0001:000207e7       __ehhandler$?navOutputModule@cProc_dialog@@IAEXXZ 100217e7 f   cProc_dialog.obj
 0001:00020802       __unwindfunclet$?paint@ContributorListBoxItem@@EAEXPAVQPainter@@@Z$0 10021802 f   cProc_dialog.obj
 0001:0002080b       __unwindfunclet$?paint@ContributorListBoxItem@@EAEXPAVQPainter@@@Z$1 1002180b f   cProc_dialog.obj
 0001:00020814       __ehhandler$?paint@ContributorListBoxItem@@EAEXPAVQPainter@@@Z 10021814 f   cProc_dialog.obj
 0001:0002082f       __unwindfunclet$?reloadInputList@cProc_dialog@@QAEXXZ$0 1002182f f   cProc_dialog.obj
 0001:00020838       __unwindfunclet$?reloadInputList@cProc_dialog@@QAEXXZ$1 10021838 f   cProc_dialog.obj
 0001:00020841       __unwindfunclet$?reloadInputList@cProc_dialog@@QAEXXZ$2 10021841 f   cProc_dialog.obj
 0001:0002084a       __unwindfunclet$?reloadInputList@cProc_dialog@@QAEXXZ$3 1002184a f   cProc_dialog.obj
 0001:00020853       __ehhandler$?reloadInputList@cProc_dialog@@QAEXXZ 10021853 f   cProc_dialog.obj
 0001:0002086e       __unwindfunclet$?setProcess@cProc_dialog@@QAEXPAVcProcess@@_N@Z$0 1002186e f   cProc_dialog.obj
 0001:00020877       __unwindfunclet$?setProcess@cProc_dialog@@QAEXPAVcProcess@@_N@Z$1 10021877 f   cProc_dialog.obj
 0001:00020880       __unwindfunclet$?setProcess@cProc_dialog@@QAEXPAVcProcess@@_N@Z$2 10021880 f   cProc_dialog.obj
 0001:00020889       __unwindfunclet$?setProcess@cProc_dialog@@QAEXPAVcProcess@@_N@Z$3 10021889 f   cProc_dialog.obj
 0001:00020892       __unwindfunclet$?setProcess@cProc_dialog@@QAEXPAVcProcess@@_N@Z$4 10021892 f   cProc_dialog.obj
 0001:0002089b       __unwindfunclet$?setProcess@cProc_dialog@@QAEXPAVcProcess@@_N@Z$5 1002189b f   cProc_dialog.obj
 0001:000208a4       __ehhandler$?setProcess@cProc_dialog@@QAEXPAVcProcess@@_N@Z 100218a4 f   cProc_dialog.obj
 0001:000208bf       __unwindfunclet$?showAnd@cProc_dialog@@AAEXXZ$0 100218bf f   cProc_dialog.obj
 0001:000208bf       __unwindfunclet$?showOr@cProc_dialog@@AAEXXZ$0 100218bf f   cProc_dialog.obj
 0001:000208c9       __ehhandler$?showAnd@cProc_dialog@@AAEXXZ 100218c9 f   cProc_dialog.obj
 0001:000208c9       __ehhandler$?showOr@cProc_dialog@@AAEXXZ 100218c9 f   cProc_dialog.obj
 0001:000208e4       __unwindfunclet$?showInput@cProc_dialog@@AAEXXZ$0 100218e4 f   cProc_dialog.obj
 0001:000208ed       __unwindfunclet$?showInput@cProc_dialog@@AAEXXZ$1 100218ed f   cProc_dialog.obj
 0001:000208f6       __unwindfunclet$?showInput@cProc_dialog@@AAEXXZ$2 100218f6 f   cProc_dialog.obj
 0001:000208ff       __unwindfunclet$?showInput@cProc_dialog@@AAEXXZ$3 100218ff f   cProc_dialog.obj
 0001:00020908       __unwindfunclet$?showInput@cProc_dialog@@AAEXXZ$4 10021908 f   cProc_dialog.obj
 0001:00020911       __ehhandler$?showInput@cProc_dialog@@AAEXXZ 10021911 f   cProc_dialog.obj
 0001:0002092c       __unwindfunclet$?showTruth@cProc_dialog@@AAEXXZ$0 1002192c f   cProc_dialog.obj
 0001:00020946       __unwindfunclet$?showTruth@cProc_dialog@@AAEXXZ$1 10021946 f   cProc_dialog.obj
 0001:00020960       __unwindfunclet$?showTruth@cProc_dialog@@AAEXXZ$2 10021960 f   cProc_dialog.obj
 0001:00020969       __unwindfunclet$?showTruth@cProc_dialog@@AAEXXZ$3 10021969 f   cProc_dialog.obj
 0001:00020972       __ehhandler$?showTruth@cProc_dialog@@AAEXXZ 10021972 f   cProc_dialog.obj
 0001:0002098d       __unwindfunclet$??0cProcess@@QAE@ABVQString@@@Z$0 1002198d f   cProcess.obj
 0001:0002098d       __unwindfunclet$??1cProcess@@UAE@XZ$0 1002198d f   cProcess.obj
 0001:00020999       __unwindfunclet$??1cProcess@@UAE@XZ$1 10021999 f   cProcess.obj
 0001:00020999       __unwindfunclet$??0cProcess@@QAE@ABVQString@@@Z$1 10021999 f   cProcess.obj
 0001:000209a5       __unwindfunclet$??0cProcess@@QAE@ABVQString@@@Z$2 100219a5 f   cProcess.obj
 0001:000209a5       __unwindfunclet$??1cProcess@@UAE@XZ$2 100219a5 f   cProcess.obj
 0001:000209b1       __unwindfunclet$??0cProcess@@QAE@ABVQString@@@Z$3 100219b1 f   cProcess.obj
 0001:000209b1       __unwindfunclet$??1cProcess@@UAE@XZ$3 100219b1 f   cProcess.obj
 0001:000209bd       __unwindfunclet$??1cProcess@@UAE@XZ$4 100219bd f   cProcess.obj
 0001:000209bd       __unwindfunclet$??0cProcess@@QAE@ABVQString@@@Z$4 100219bd f   cProcess.obj
 0001:000209c9       __unwindfunclet$??0cProcess@@QAE@ABVQString@@@Z$5 100219c9 f   cProcess.obj
 0001:000209c9       __unwindfunclet$??1cProcess@@UAE@XZ$5 100219c9 f   cProcess.obj
 0001:000209d5       __unwindfunclet$??0cProcess@@QAE@ABVQString@@@Z$6 100219d5 f   cProcess.obj
 0001:000209d5       __unwindfunclet$??1cProcess@@UAE@XZ$6 100219d5 f   cProcess.obj
 0001:000209e1       __unwindfunclet$??1cProcess@@UAE@XZ$7 100219e1 f   cProcess.obj
 0001:000209e1       __unwindfunclet$??0cProcess@@QAE@ABVQString@@@Z$7 100219e1 f   cProcess.obj
 0001:000209ed       __unwindfunclet$??0cProcess@@QAE@ABVQString@@@Z$8 100219ed f   cProcess.obj
 0001:000209ed       __unwindfunclet$??1cProcess@@UAE@XZ$8 100219ed f   cProcess.obj
 0001:000209f9       __unwindfunclet$??0cProcess@@QAE@ABVQString@@@Z$9 100219f9 f   cProcess.obj
 0001:000209f9       __unwindfunclet$??1cProcess@@UAE@XZ$9 100219f9 f   cProcess.obj
 0001:00020a05       __unwindfunclet$??0cProcess@@QAE@ABVQString@@@Z$10 10021a05 f   cProcess.obj
 0001:00020a05       __unwindfunclet$??1cProcess@@UAE@XZ$10 10021a05 f   cProcess.obj
 0001:00020a11       __ehhandler$??0cProcess@@QAE@ABVQString@@@Z 10021a11 f   cProcess.obj
 0001:00020a11       __ehhandler$??1cProcess@@UAE@XZ 10021a11 f   cProcess.obj
 0001:00020a2c       __unwindfunclet$??1?$QDict@VQString@@@@UAE@XZ$0 10021a2c f   cProcess.obj
 0001:00020a35       __ehhandler$??1?$QDict@VQString@@@@UAE@XZ 10021a35 f   cProcess.obj
 0001:00020a50       __unwindfunclet$?FindEntry@cProcess@@AAE?AVQString@@AAV?$QDict@VQString@@@@ABV2@@Z$0 10021a50 f   cProcess.obj
 0001:00020a6a       __ehhandler$?FindEntry@cProcess@@AAE?AVQString@@AAV?$QDict@VQString@@@@ABV2@@Z 10021a6a f   cProcess.obj
 0001:00020a85       __unwindfunclet$?Index@cProcess@@AAEXABVQStringList@@AAV?$QDict@VQString@@@@@Z$0 10021a85 f   cProcess.obj
 0001:00020a8e       __unwindfunclet$?Index@cProcess@@AAEXABVQStringList@@AAV?$QDict@VQString@@@@@Z$1 10021a8e f   cProcess.obj
 0001:00020a97       __unwindfunclet$?Index@cProcess@@AAEXABVQStringList@@AAV?$QDict@VQString@@@@@Z$2 10021a97 f   cProcess.obj
 0001:00020aa0       __unwindfunclet$?Index@cProcess@@AAEXABVQStringList@@AAV?$QDict@VQString@@@@@Z$3 10021aa0 f   cProcess.obj
 0001:00020aaa       __ehhandler$?Index@cProcess@@AAEXABVQStringList@@AAV?$QDict@VQString@@@@@Z 10021aaa f   cProcess.obj
 0001:00020ac5       __unwindfunclet$?LoadSettings@cProcess@@QAE_NABVQStringList@@@Z$0 10021ac5 f   cProcess.obj
 0001:00020ace       __unwindfunclet$?LoadSettings@cProcess@@QAE_NABVQStringList@@@Z$1 10021ace f   cProcess.obj
 0001:00020ad6       __unwindfunclet$?LoadSettings@cProcess@@QAE_NABVQStringList@@@Z$2 10021ad6 f   cProcess.obj
 0001:00020adf       __unwindfunclet$?LoadSettings@cProcess@@QAE_NABVQStringList@@@Z$3 10021adf f   cProcess.obj
 0001:00020ae8       __unwindfunclet$?LoadSettings@cProcess@@QAE_NABVQStringList@@@Z$4 10021ae8 f   cProcess.obj
 0001:00020af1       __unwindfunclet$?LoadSettings@cProcess@@QAE_NABVQStringList@@@Z$5 10021af1 f   cProcess.obj
 0001:00020afa       __unwindfunclet$?LoadSettings@cProcess@@QAE_NABVQStringList@@@Z$6 10021afa f   cProcess.obj
 0001:00020b03       __unwindfunclet$?LoadSettings@cProcess@@QAE_NABVQStringList@@@Z$7 10021b03 f   cProcess.obj
 0001:00020b0c       __unwindfunclet$?LoadSettings@cProcess@@QAE_NABVQStringList@@@Z$8 10021b0c f   cProcess.obj
 0001:00020b15       __unwindfunclet$?LoadSettings@cProcess@@QAE_NABVQStringList@@@Z$9 10021b15 f   cProcess.obj
 0001:00020b1e       __unwindfunclet$?LoadSettings@cProcess@@QAE_NABVQStringList@@@Z$10 10021b1e f   cProcess.obj
 0001:00020b27       __unwindfunclet$?LoadSettings@cProcess@@QAE_NABVQStringList@@@Z$11 10021b27 f   cProcess.obj
 0001:00020b30       __unwindfunclet$?LoadSettings@cProcess@@QAE_NABVQStringList@@@Z$12 10021b30 f   cProcess.obj
 0001:00020b39       __unwindfunclet$?LoadSettings@cProcess@@QAE_NABVQStringList@@@Z$14 10021b39 f   cProcess.obj
 0001:00020b42       __unwindfunclet$?LoadSettings@cProcess@@QAE_NABVQStringList@@@Z$15 10021b42 f   cProcess.obj
 0001:00020b4b       __unwindfunclet$?LoadSettings@cProcess@@QAE_NABVQStringList@@@Z$16 10021b4b f   cProcess.obj
 0001:00020b54       __unwindfunclet$?LoadSettings@cProcess@@QAE_NABVQStringList@@@Z$17 10021b54 f   cProcess.obj
 0001:00020b5d       __unwindfunclet$?LoadSettings@cProcess@@QAE_NABVQStringList@@@Z$18 10021b5d f   cProcess.obj
 0001:00020b66       __unwindfunclet$?LoadSettings@cProcess@@QAE_NABVQStringList@@@Z$19 10021b66 f   cProcess.obj
 0001:00020b6f       __unwindfunclet$?LoadSettings@cProcess@@QAE_NABVQStringList@@@Z$20 10021b6f f   cProcess.obj
 0001:00020b78       __unwindfunclet$?LoadSettings@cProcess@@QAE_NABVQStringList@@@Z$21 10021b78 f   cProcess.obj
 0001:00020b81       __unwindfunclet$?LoadSettings@cProcess@@QAE_NABVQStringList@@@Z$22 10021b81 f   cProcess.obj
 0001:00020b8a       __unwindfunclet$?LoadSettings@cProcess@@QAE_NABVQStringList@@@Z$23 10021b8a f   cProcess.obj
 0001:00020b93       __unwindfunclet$?LoadSettings@cProcess@@QAE_NABVQStringList@@@Z$26 10021b93 f   cProcess.obj
 0001:00020b9c       __unwindfunclet$?LoadSettings@cProcess@@QAE_NABVQStringList@@@Z$27 10021b9c f   cProcess.obj
 0001:00020ba5       __unwindfunclet$?LoadSettings@cProcess@@QAE_NABVQStringList@@@Z$24 10021ba5 f   cProcess.obj
 0001:00020bae       __unwindfunclet$?LoadSettings@cProcess@@QAE_NABVQStringList@@@Z$25 10021bae f   cProcess.obj
 0001:00020bb7       __unwindfunclet$?LoadSettings@cProcess@@QAE_NABVQStringList@@@Z$28 10021bb7 f   cProcess.obj
 0001:00020bc0       __unwindfunclet$?LoadSettings@cProcess@@QAE_NABVQStringList@@@Z$29 10021bc0 f   cProcess.obj
 0001:00020bc9       __unwindfunclet$?LoadSettings@cProcess@@QAE_NABVQStringList@@@Z$32 10021bc9 f   cProcess.obj
 0001:00020bd2       __unwindfunclet$?LoadSettings@cProcess@@QAE_NABVQStringList@@@Z$33 10021bd2 f   cProcess.obj
 0001:00020bdb       __unwindfunclet$?LoadSettings@cProcess@@QAE_NABVQStringList@@@Z$34 10021bdb f   cProcess.obj
 0001:00020be4       __unwindfunclet$?LoadSettings@cProcess@@QAE_NABVQStringList@@@Z$35 10021be4 f   cProcess.obj
 0001:00020bed       __unwindfunclet$?LoadSettings@cProcess@@QAE_NABVQStringList@@@Z$36 10021bed f   cProcess.obj
 0001:00020bf6       __unwindfunclet$?LoadSettings@cProcess@@QAE_NABVQStringList@@@Z$37 10021bf6 f   cProcess.obj
 0001:00020bff       __unwindfunclet$?LoadSettings@cProcess@@QAE_NABVQStringList@@@Z$38 10021bff f   cProcess.obj
 0001:00020c08       __unwindfunclet$?LoadSettings@cProcess@@QAE_NABVQStringList@@@Z$39 10021c08 f   cProcess.obj
 0001:00020c11       __unwindfunclet$?LoadSettings@cProcess@@QAE_NABVQStringList@@@Z$40 10021c11 f   cProcess.obj
 0001:00020c1a       __unwindfunclet$?LoadSettings@cProcess@@QAE_NABVQStringList@@@Z$41 10021c1a f   cProcess.obj
 0001:00020c23       __unwindfunclet$?LoadSettings@cProcess@@QAE_NABVQStringList@@@Z$30 10021c23 f   cProcess.obj
 0001:00020c2c       __unwindfunclet$?LoadSettings@cProcess@@QAE_NABVQStringList@@@Z$31 10021c2c f   cProcess.obj
 0001:00020c35       __unwindfunclet$?LoadSettings@cProcess@@QAE_NABVQStringList@@@Z$13 10021c35 f   cProcess.obj
 0001:00020c3e       __ehhandler$?LoadSettings@cProcess@@QAE_NABVQStringList@@@Z 10021c3e f   cProcess.obj
 0001:00020c59       __unwindfunclet$?LoadTruth@cProcess@@AAEHAAV?$QDict@VQString@@@@@Z$0 10021c59 f   cProcess.obj
 0001:00020c62       __unwindfunclet$?LoadTruth@cProcess@@AAEHAAV?$QDict@VQString@@@@@Z$1 10021c62 f   cProcess.obj
 0001:00020c6b       __unwindfunclet$?LoadTruth@cProcess@@AAEHAAV?$QDict@VQString@@@@@Z$2 10021c6b f   cProcess.obj
 0001:00020c74       __unwindfunclet$?LoadTruth@cProcess@@AAEHAAV?$QDict@VQString@@@@@Z$3 10021c74 f   cProcess.obj
 0001:00020c7d       __ehhandler$?LoadTruth@cProcess@@AAEHAAV?$QDict@VQString@@@@@Z 10021c7d f   cProcess.obj
 0001:00020ca2       __unwindfunclet$?addEntry@cProcess@@AAEXAAVQStringList@@ABVQString@@1@Z$0 10021ca2 f   cProcess.obj
 0001:00020cab       __unwindfunclet$?addEntry@cProcess@@AAEXAAVQStringList@@ABVQString@@1@Z$1 10021cab f   cProcess.obj
 0001:00020cb4       __ehhandler$?addEntry@cProcess@@AAEXAAVQStringList@@ABVQString@@1@Z 10021cb4 f   cProcess.obj
 0001:00020ccf       __unwindfunclet$?countOutputs@cProcess@@AAEXABV?$map@VQString@@PAVcProcess@@U?$less@VQString@@@std@@V?$allocator@U?$pair@$$CBVQString@@PAVcProcess@@@std@@@4@@std@@@Z$1 10021ccf f   cProcess.obj
 0001:00020cd8       __unwindfunclet$?countOutputs@cProcess@@AAEXABV?$map@VQString@@PAVcProcess@@U?$less@VQString@@@std@@V?$allocator@U?$pair@$$CBVQString@@PAVcProcess@@@std@@@4@@std@@@Z$0 10021cd8 f   cProcess.obj
 0001:00020ce1       __ehhandler$?countOutputs@cProcess@@AAEXABV?$map@VQString@@PAVcProcess@@U?$less@VQString@@@std@@V?$allocator@U?$pair@$$CBVQString@@PAVcProcess@@@std@@@4@@std@@@Z 10021ce1 f   cProcess.obj
 0001:00020cfc       __unwindfunclet$?inputSlotChange@cProc_dialog@@IAEXABVQString@@@Z$0 10021cfc f   cProcess.obj
 0001:00020cfc       __unwindfunclet$?countProcessOutputs@cProcess@@SAXAAV?$map@VQString@@PAVcProcess@@U?$less@VQString@@@std@@V?$allocator@U?$pair@$$CBVQString@@PAVcProcess@@@std@@@4@@std@@@Z$0 10021cfc f   cProcess.obj
 0001:00020d05       __ehhandler$?countProcessOutputs@cProcess@@SAXAAV?$map@VQString@@PAVcProcess@@U?$less@VQString@@@std@@V?$allocator@U?$pair@$$CBVQString@@PAVcProcess@@@std@@@4@@std@@@Z 10021d05 f   cProcess.obj
 0001:00020d05       __ehhandler$?inputSlotChange@cProc_dialog@@IAEXABVQString@@@Z 10021d05 f   cProcess.obj
 0001:00020d20       __unwindfunclet$?saveSettings@cProcess@@QAE?AVQStringList@@XZ$0 10021d20 f   cProcess.obj
 0001:00020d2c       __unwindfunclet$?saveSettings@cProcess@@QAE?AVQStringList@@XZ$1 10021d2c f   cProcess.obj
 0001:00020d4f       __unwindfunclet$?saveSettings@cProcess@@QAE?AVQStringList@@XZ$2 10021d4f f   cProcess.obj
 0001:00020d5b       __unwindfunclet$?saveSettings@cProcess@@QAE?AVQStringList@@XZ$3 10021d5b f   cProcess.obj
 0001:00020d67       __unwindfunclet$?saveSettings@cProcess@@QAE?AVQStringList@@XZ$4 10021d67 f   cProcess.obj
 0001:00020d73       __unwindfunclet$?saveSettings@cProcess@@QAE?AVQStringList@@XZ$5 10021d73 f   cProcess.obj
 0001:00020d7f       __unwindfunclet$?saveSettings@cProcess@@QAE?AVQStringList@@XZ$6 10021d7f f   cProcess.obj
 0001:00020d8b       __unwindfunclet$?saveSettings@cProcess@@QAE?AVQStringList@@XZ$7 10021d8b f   cProcess.obj
 0001:00020d97       __unwindfunclet$?saveSettings@cProcess@@QAE?AVQStringList@@XZ$8 10021d97 f   cProcess.obj
 0001:00020da3       __unwindfunclet$?saveSettings@cProcess@@QAE?AVQStringList@@XZ$9 10021da3 f   cProcess.obj
 0001:00020daf       __unwindfunclet$?saveSettings@cProcess@@QAE?AVQStringList@@XZ$10 10021daf f   cProcess.obj
 0001:00020dbb       __unwindfunclet$?saveSettings@cProcess@@QAE?AVQStringList@@XZ$27 10021dbb f   cProcess.obj
 0001:00020dc7       __unwindfunclet$?saveSettings@cProcess@@QAE?AVQStringList@@XZ$28 10021dc7 f   cProcess.obj
 0001:00020dd3       __unwindfunclet$?saveSettings@cProcess@@QAE?AVQStringList@@XZ$23 10021dd3 f   cProcess.obj
 0001:00020ddf       __unwindfunclet$?saveSettings@cProcess@@QAE?AVQStringList@@XZ$24 10021ddf f   cProcess.obj
 0001:00020deb       __unwindfunclet$?saveSettings@cProcess@@QAE?AVQStringList@@XZ$25 10021deb f   cProcess.obj
 0001:00020df7       __unwindfunclet$?saveSettings@cProcess@@QAE?AVQStringList@@XZ$26 10021df7 f   cProcess.obj
 0001:00020e03       __unwindfunclet$?saveSettings@cProcess@@QAE?AVQStringList@@XZ$19 10021e03 f   cProcess.obj
 0001:00020e0f       __unwindfunclet$?saveSettings@cProcess@@QAE?AVQStringList@@XZ$20 10021e0f f   cProcess.obj
 0001:00020e1b       __unwindfunclet$?saveSettings@cProcess@@QAE?AVQStringList@@XZ$21 10021e1b f   cProcess.obj
 0001:00020e27       __unwindfunclet$?saveSettings@cProcess@@QAE?AVQStringList@@XZ$22 10021e27 f   cProcess.obj
 0001:00020e33       __unwindfunclet$?saveSettings@cProcess@@QAE?AVQStringList@@XZ$18 10021e33 f   cProcess.obj
 0001:00020e3f       __unwindfunclet$?saveSettings@cProcess@@QAE?AVQStringList@@XZ$13 10021e3f f   cProcess.obj
 0001:00020e4b       __unwindfunclet$?saveSettings@cProcess@@QAE?AVQStringList@@XZ$14 10021e4b f   cProcess.obj
 0001:00020e57       __unwindfunclet$?saveSettings@cProcess@@QAE?AVQStringList@@XZ$15 10021e57 f   cProcess.obj
 0001:00020e63       __unwindfunclet$?saveSettings@cProcess@@QAE?AVQStringList@@XZ$16 10021e63 f   cProcess.obj
 0001:00020e6f       __unwindfunclet$?saveSettings@cProcess@@QAE?AVQStringList@@XZ$17 10021e6f f   cProcess.obj
 0001:00020e7b       __unwindfunclet$?saveSettings@cProcess@@QAE?AVQStringList@@XZ$11 10021e7b f   cProcess.obj
 0001:00020e87       __unwindfunclet$?saveSettings@cProcess@@QAE?AVQStringList@@XZ$12 10021e87 f   cProcess.obj
 0001:00020e93       __unwindfunclet$?saveSettings@cProcess@@QAE?AVQStringList@@XZ$29 10021e93 f   cProcess.obj
 0001:00020e9f       __ehhandler$?saveSettings@cProcess@@QAE?AVQStringList@@XZ 10021e9f f   cProcess.obj
 0001:00020ec7       __unwindfunclet$?setName@cProcess@@QAE_NABVQString@@@Z$0 10021ec7 f   cProcess.obj
 0001:00020ed0       __unwindfunclet$?setName@cProcess@@QAE_NABVQString@@@Z$1 10021ed0 f   cProcess.obj
 0001:00020ed9       __ehhandler$?setName@cProcess@@QAE_NABVQString@@@Z 10021ed9 f   cProcess.obj
 0001:00020ef4       __unwindfunclet$??0multiInputBase@@QAE@PAVQWidget@@PBD_NI@Z$0 10021ef4 f   multiinput.obj
 0001:00020efd       __unwindfunclet$??0multiInputBase@@QAE@PAVQWidget@@PBD_NI@Z$1 10021efd f   multiinput.obj
 0001:00020f0c       __unwindfunclet$??0multiInputBase@@QAE@PAVQWidget@@PBD_NI@Z$2 10021f0c f   multiinput.obj
 0001:00020f16       __unwindfunclet$??0multiInputBase@@QAE@PAVQWidget@@PBD_NI@Z$3 10021f16 f   multiinput.obj
 0001:00020f20       __unwindfunclet$??0multiInputBase@@QAE@PAVQWidget@@PBD_NI@Z$4 10021f20 f   multiinput.obj
 0001:00020f2a       __unwindfunclet$??0multiInputBase@@QAE@PAVQWidget@@PBD_NI@Z$5 10021f2a f   multiinput.obj
 0001:00020f34       __unwindfunclet$??0multiInputBase@@QAE@PAVQWidget@@PBD_NI@Z$6 10021f34 f   multiinput.obj
 0001:00020f3e       __unwindfunclet$??0multiInputBase@@QAE@PAVQWidget@@PBD_NI@Z$7 10021f3e f   multiinput.obj
 0001:00020f48       __unwindfunclet$??0multiInputBase@@QAE@PAVQWidget@@PBD_NI@Z$8 10021f48 f   multiinput.obj
 0001:00020f52       __unwindfunclet$??0multiInputBase@@QAE@PAVQWidget@@PBD_NI@Z$9 10021f52 f   multiinput.obj
 0001:00020f5c       __unwindfunclet$??0multiInputBase@@QAE@PAVQWidget@@PBD_NI@Z$10 10021f5c f   multiinput.obj
 0001:00020f66       __unwindfunclet$??0multiInputBase@@QAE@PAVQWidget@@PBD_NI@Z$11 10021f66 f   multiinput.obj
 0001:00020f70       __unwindfunclet$??0multiInputBase@@QAE@PAVQWidget@@PBD_NI@Z$12 10021f70 f   multiinput.obj
 0001:00020f7a       __unwindfunclet$??0multiInputBase@@QAE@PAVQWidget@@PBD_NI@Z$13 10021f7a f   multiinput.obj
 0001:00020f84       __unwindfunclet$??0multiInputBase@@QAE@PAVQWidget@@PBD_NI@Z$14 10021f84 f   multiinput.obj
 0001:00020f8e       __unwindfunclet$??0multiInputBase@@QAE@PAVQWidget@@PBD_NI@Z$15 10021f8e f   multiinput.obj
 0001:00020f98       __unwindfunclet$??0multiInputBase@@QAE@PAVQWidget@@PBD_NI@Z$16 10021f98 f   multiinput.obj
 0001:00020fa2       __unwindfunclet$??0multiInputBase@@QAE@PAVQWidget@@PBD_NI@Z$17 10021fa2 f   multiinput.obj
 0001:00020fac       __unwindfunclet$??0multiInputBase@@QAE@PAVQWidget@@PBD_NI@Z$18 10021fac f   multiinput.obj
 0001:00020fb6       __unwindfunclet$??0multiInputBase@@QAE@PAVQWidget@@PBD_NI@Z$19 10021fb6 f   multiinput.obj
 0001:00020fc0       __unwindfunclet$??0multiInputBase@@QAE@PAVQWidget@@PBD_NI@Z$20 10021fc0 f   multiinput.obj
 0001:00020fca       __unwindfunclet$??0multiInputBase@@QAE@PAVQWidget@@PBD_NI@Z$21 10021fca f   multiinput.obj
 0001:00020fd4       __ehhandler$??0multiInputBase@@QAE@PAVQWidget@@PBD_NI@Z 10021fd4 f   multiinput.obj
 0001:00020fef       __unwindfunclet$??0config_mb4@@QAE@IPAVQWidget@@PBD@Z$0 10021fef f   multiinput.obj
 0001:00020fef       __unwindfunclet$??1multiInputBase@@UAE@XZ$0 10021fef f   multiinput.obj
 0001:00020ff8       __ehhandler$??1multiInputBase@@UAE@XZ 10021ff8 f   multiinput.obj
 0001:00020ff8       __ehhandler$??0config_mb4@@QAE@IPAVQWidget@@PBD@Z 10021ff8 f   multiinput.obj
 0001:00021013       __unwindfunclet$?languageChange@multiInputBase@@MAEXXZ$0 10022013 f   multiinput.obj
 0001:0002101c       __unwindfunclet$?languageChange@multiInputBase@@MAEXXZ$1 1002201c f   multiinput.obj
 0001:00021025       __unwindfunclet$?languageChange@multiInputBase@@MAEXXZ$2 10022025 f   multiinput.obj
 0001:0002102e       __unwindfunclet$?languageChange@multiInputBase@@MAEXXZ$3 1002202e f   multiinput.obj
 0001:00021037       __unwindfunclet$?languageChange@multiInputBase@@MAEXXZ$4 10022037 f   multiinput.obj
 0001:00021040       __unwindfunclet$?languageChange@multiInputBase@@MAEXXZ$5 10022040 f   multiinput.obj
 0001:00021049       __unwindfunclet$?languageChange@multiInputBase@@MAEXXZ$6 10022049 f   multiinput.obj
 0001:00021052       __unwindfunclet$?languageChange@multiInputBase@@MAEXXZ$7 10022052 f   multiinput.obj
 0001:0002105b       __unwindfunclet$?languageChange@multiInputBase@@MAEXXZ$8 1002205b f   multiinput.obj
 0001:00021064       __unwindfunclet$?languageChange@multiInputBase@@MAEXXZ$9 10022064 f   multiinput.obj
 0001:0002106d       __unwindfunclet$?languageChange@multiInputBase@@MAEXXZ$10 1002206d f   multiinput.obj
 0001:00021076       __unwindfunclet$?languageChange@multiInputBase@@MAEXXZ$11 10022076 f   multiinput.obj
 0001:0002107f       __unwindfunclet$?languageChange@multiInputBase@@MAEXXZ$12 1002207f f   multiinput.obj
 0001:00021088       __unwindfunclet$?languageChange@multiInputBase@@MAEXXZ$13 10022088 f   multiinput.obj
 0001:00021091       __unwindfunclet$?languageChange@multiInputBase@@MAEXXZ$14 10022091 f   multiinput.obj
 0001:0002109a       __unwindfunclet$?languageChange@multiInputBase@@MAEXXZ$15 1002209a f   multiinput.obj
 0001:000210a3       __ehhandler$?languageChange@multiInputBase@@MAEXXZ 100220a3 f   multiinput.obj
 0001:000210be       __unwindfunclet$??0MultiInputInvalidListViewItem@@QAE@PAVQListView@@ABVQString@@@Z$0 100220be f   multiinputimpl.obj
 0001:000210c7       __unwindfunclet$??0MultiInputInvalidListViewItem@@QAE@PAVQListView@@ABVQString@@@Z$1 100220c7 f   multiinputimpl.obj
 0001:000210d0       __unwindfunclet$??0MultiInputInvalidListViewItem@@QAE@PAVQListView@@ABVQString@@@Z$2 100220d0 f   multiinputimpl.obj
 0001:000210d9       __unwindfunclet$??0MultiInputInvalidListViewItem@@QAE@PAVQListView@@ABVQString@@@Z$3 100220d9 f   multiinputimpl.obj
 0001:000210e2       __unwindfunclet$??0MultiInputInvalidListViewItem@@QAE@PAVQListView@@ABVQString@@@Z$4 100220e2 f   multiinputimpl.obj
 0001:000210eb       __unwindfunclet$??0MultiInputInvalidListViewItem@@QAE@PAVQListView@@ABVQString@@@Z$5 100220eb f   multiinputimpl.obj
 0001:000210f4       __unwindfunclet$??0MultiInputInvalidListViewItem@@QAE@PAVQListView@@ABVQString@@@Z$6 100220f4 f   multiinputimpl.obj
 0001:000210fd       __ehhandler$??0MultiInputInvalidListViewItem@@QAE@PAVQListView@@ABVQString@@@Z 100220fd f   multiinputimpl.obj
 0001:00021118       __unwindfunclet$??0multiInput@@QAE@ABV?$map@VQString@@PAVcProcess@@U?$less@VQString@@@std@@V?$allocator@U?$pair@$$CBVQString@@PAVcProcess@@@std@@@4@@std@@QBVcProcess@@PAVQWidget@@PBD_NI@Z$0 10022118 f   multiinputimpl.obj
 0001:00021120       __unwindfunclet$??0multiInput@@QAE@ABV?$map@VQString@@PAVcProcess@@U?$less@VQString@@@std@@V?$allocator@U?$pair@$$CBVQString@@PAVcProcess@@@std@@@4@@std@@QBVcProcess@@PAVQWidget@@PBD_NI@Z$1 10022120 f   multiinputimpl.obj
 0001:00021129       __unwindfunclet$??0multiInput@@QAE@ABV?$map@VQString@@PAVcProcess@@U?$less@VQString@@@std@@V?$allocator@U?$pair@$$CBVQString@@PAVcProcess@@@std@@@4@@std@@QBVcProcess@@PAVQWidget@@PBD_NI@Z$2 10022129 f   multiinputimpl.obj
 0001:00021132       __unwindfunclet$??0multiInput@@QAE@ABV?$map@VQString@@PAVcProcess@@U?$less@VQString@@@std@@V?$allocator@U?$pair@$$CBVQString@@PAVcProcess@@@std@@@4@@std@@QBVcProcess@@PAVQWidget@@PBD_NI@Z$3 10022132 f   multiinputimpl.obj
 0001:0002113b       __unwindfunclet$??0multiInput@@QAE@ABV?$map@VQString@@PAVcProcess@@U?$less@VQString@@@std@@V?$allocator@U?$pair@$$CBVQString@@PAVcProcess@@@std@@@4@@std@@QBVcProcess@@PAVQWidget@@PBD_NI@Z$4 1002213b f   multiinputimpl.obj
 0001:00021144       __unwindfunclet$??0multiInput@@QAE@ABV?$map@VQString@@PAVcProcess@@U?$less@VQString@@@std@@V?$allocator@U?$pair@$$CBVQString@@PAVcProcess@@@std@@@4@@std@@QBVcProcess@@PAVQWidget@@PBD_NI@Z$5 10022144 f   multiinputimpl.obj
 0001:0002114d       __unwindfunclet$??0multiInput@@QAE@ABV?$map@VQString@@PAVcProcess@@U?$less@VQString@@@std@@V?$allocator@U?$pair@$$CBVQString@@PAVcProcess@@@std@@@4@@std@@QBVcProcess@@PAVQWidget@@PBD_NI@Z$6 1002214d f   multiinputimpl.obj
 0001:00021156       __unwindfunclet$??0multiInput@@QAE@ABV?$map@VQString@@PAVcProcess@@U?$less@VQString@@@std@@V?$allocator@U?$pair@$$CBVQString@@PAVcProcess@@@std@@@4@@std@@QBVcProcess@@PAVQWidget@@PBD_NI@Z$7 10022156 f   multiinputimpl.obj
 0001:0002115f       __unwindfunclet$??0multiInput@@QAE@ABV?$map@VQString@@PAVcProcess@@U?$less@VQString@@@std@@V?$allocator@U?$pair@$$CBVQString@@PAVcProcess@@@std@@@4@@std@@QBVcProcess@@PAVQWidget@@PBD_NI@Z$8 1002215f f   multiinputimpl.obj
 0001:00021168       __unwindfunclet$??0multiInput@@QAE@ABV?$map@VQString@@PAVcProcess@@U?$less@VQString@@@std@@V?$allocator@U?$pair@$$CBVQString@@PAVcProcess@@@std@@@4@@std@@QBVcProcess@@PAVQWidget@@PBD_NI@Z$9 10022168 f   multiinputimpl.obj
 0001:00021171       __unwindfunclet$??0multiInput@@QAE@ABV?$map@VQString@@PAVcProcess@@U?$less@VQString@@@std@@V?$allocator@U?$pair@$$CBVQString@@PAVcProcess@@@std@@@4@@std@@QBVcProcess@@PAVQWidget@@PBD_NI@Z$10 10022171 f   multiinputimpl.obj
 0001:0002117a       __unwindfunclet$??0multiInput@@QAE@ABV?$map@VQString@@PAVcProcess@@U?$less@VQString@@@std@@V?$allocator@U?$pair@$$CBVQString@@PAVcProcess@@@std@@@4@@std@@QBVcProcess@@PAVQWidget@@PBD_NI@Z$11 1002217a f   multiinputimpl.obj
 0001:00021183       __unwindfunclet$??0multiInput@@QAE@ABV?$map@VQString@@PAVcProcess@@U?$less@VQString@@@std@@V?$allocator@U?$pair@$$CBVQString@@PAVcProcess@@@std@@@4@@std@@QBVcProcess@@PAVQWidget@@PBD_NI@Z$12 10022183 f   multiinputimpl.obj
 0001:0002118c       __unwindfunclet$??0multiInput@@QAE@ABV?$map@VQString@@PAVcProcess@@U?$less@VQString@@@std@@V?$allocator@U?$pair@$$CBVQString@@PAVcProcess@@@std@@@4@@std@@QBVcProcess@@PAVQWidget@@PBD_NI@Z$13 1002218c f   multiinputimpl.obj
 0001:00021196       __unwindfunclet$??0multiInput@@QAE@ABV?$map@VQString@@PAVcProcess@@U?$less@VQString@@@std@@V?$allocator@U?$pair@$$CBVQString@@PAVcProcess@@@std@@@4@@std@@QBVcProcess@@PAVQWidget@@PBD_NI@Z$14 10022196 f   multiinputimpl.obj
 0001:0002119f       __unwindfunclet$??0multiInput@@QAE@ABV?$map@VQString@@PAVcProcess@@U?$less@VQString@@@std@@V?$allocator@U?$pair@$$CBVQString@@PAVcProcess@@@std@@@4@@std@@QBVcProcess@@PAVQWidget@@PBD_NI@Z$15 1002219f f   multiinputimpl.obj
 0001:000211a8       __unwindfunclet$??0multiInput@@QAE@ABV?$map@VQString@@PAVcProcess@@U?$less@VQString@@@std@@V?$allocator@U?$pair@$$CBVQString@@PAVcProcess@@@std@@@4@@std@@QBVcProcess@@PAVQWidget@@PBD_NI@Z$16 100221a8 f   multiinputimpl.obj
 0001:000211b1       __unwindfunclet$??0multiInput@@QAE@ABV?$map@VQString@@PAVcProcess@@U?$less@VQString@@@std@@V?$allocator@U?$pair@$$CBVQString@@PAVcProcess@@@std@@@4@@std@@QBVcProcess@@PAVQWidget@@PBD_NI@Z$17 100221b1 f   multiinputimpl.obj
 0001:000211ba       __unwindfunclet$??0multiInput@@QAE@ABV?$map@VQString@@PAVcProcess@@U?$less@VQString@@@std@@V?$allocator@U?$pair@$$CBVQString@@PAVcProcess@@@std@@@4@@std@@QBVcProcess@@PAVQWidget@@PBD_NI@Z$18 100221ba f   multiinputimpl.obj
 0001:000211c3       __unwindfunclet$??0multiInput@@QAE@ABV?$map@VQString@@PAVcProcess@@U?$less@VQString@@@std@@V?$allocator@U?$pair@$$CBVQString@@PAVcProcess@@@std@@@4@@std@@QBVcProcess@@PAVQWidget@@PBD_NI@Z$19 100221c3 f   multiinputimpl.obj
 0001:000211cc       __unwindfunclet$??0multiInput@@QAE@ABV?$map@VQString@@PAVcProcess@@U?$less@VQString@@@std@@V?$allocator@U?$pair@$$CBVQString@@PAVcProcess@@@std@@@4@@std@@QBVcProcess@@PAVQWidget@@PBD_NI@Z$20 100221cc f   multiinputimpl.obj
 0001:000211d5       __unwindfunclet$??0multiInput@@QAE@ABV?$map@VQString@@PAVcProcess@@U?$less@VQString@@@std@@V?$allocator@U?$pair@$$CBVQString@@PAVcProcess@@@std@@@4@@std@@QBVcProcess@@PAVQWidget@@PBD_NI@Z$22 100221d5 f   multiinputimpl.obj
 0001:000211de       __unwindfunclet$??0multiInput@@QAE@ABV?$map@VQString@@PAVcProcess@@U?$less@VQString@@@std@@V?$allocator@U?$pair@$$CBVQString@@PAVcProcess@@@std@@@4@@std@@QBVcProcess@@PAVQWidget@@PBD_NI@Z$23 100221de f   multiinputimpl.obj
 0001:000211e8       __ehhandler$??0multiInput@@QAE@ABV?$map@VQString@@PAVcProcess@@U?$less@VQString@@@std@@V?$allocator@U?$pair@$$CBVQString@@PAVcProcess@@@std@@@4@@std@@QBVcProcess@@PAVQWidget@@PBD_NI@Z 100221e8 f   multiinputimpl.obj
 0001:00021203       __unwindfunclet$??1multiInput@@UAE@XZ$0 10022203 f   multiinputimpl.obj
 0001:0002120b       __unwindfunclet$??1multiInput@@UAE@XZ$1 1002220b f   multiinputimpl.obj
 0001:00021214       __unwindfunclet$??1multiInput@@UAE@XZ$2 10022214 f   multiinputimpl.obj
 0001:0002121d       __unwindfunclet$??1multiInput@@UAE@XZ$3 1002221d f   multiinputimpl.obj
 0001:00021226       __unwindfunclet$??1multiInput@@UAE@XZ$4 10022226 f   multiinputimpl.obj
 0001:0002122f       __unwindfunclet$??1multiInput@@UAE@XZ$5 1002222f f   multiinputimpl.obj
 0001:00021238       __unwindfunclet$??1multiInput@@UAE@XZ$6 10022238 f   multiinputimpl.obj
 0001:00021241       __ehhandler$??1multiInput@@UAE@XZ 10022241 f   multiinputimpl.obj
 0001:0002125c       __unwindfunclet$?changeInputs@multiInput@@QAEXQAVcProcess@@@Z$0 1002225c f   multiinputimpl.obj
 0001:0002125c       __unwindfunclet$?changeInputs@singleInput@@QAE_NQAVcProcess@@@Z$0 1002225c f   multiinputimpl.obj
 0001:00021265       __ehhandler$?changeInputs@multiInput@@QAEXQAVcProcess@@@Z 10022265 f   multiinputimpl.obj
 0001:00021265       __ehhandler$?changeInputs@singleInput@@QAE_NQAVcProcess@@@Z 10022265 f   multiinputimpl.obj
 0001:00021280       __unwindfunclet$?countSelections@alm_process@@AAEHPAPAVQListViewItem@@@Z$0 10022280 f   multiinputimpl.obj
 0001:00021280       __unwindfunclet$?enableAdd@multiInput@@QAEXXZ$0 10022280 f   multiinputimpl.obj
 0001:00021280       __unwindfunclet$?enableRemove@multiInput@@QAEXXZ$0 10022280 f   multiinputimpl.obj
 0001:00021280       __unwindfunclet$?displayHome@ProcessListView@@AAEX_N@Z$0 10022280 f   multiinputimpl.obj
 0001:00021280       __unwindfunclet$?removeProcesses@multiInput@@QAEXPAVQListViewItem@@@Z$0 10022280 f   multiinputimpl.obj
 0001:00021280       __unwindfunclet$?displayEnd@ProcessListView@@AAEX_N@Z$0 10022280 f   multiinputimpl.obj
 0001:00021280       __unwindfunclet$?addProcesses@multiInput@@QAEXPAVQListViewItem@@@Z$0 10022280 f   multiinputimpl.obj
 0001:00021289       __ehhandler$?displayEnd@ProcessListView@@AAEX_N@Z 10022289 f   multiinputimpl.obj
 0001:00021289       __ehhandler$?countSelections@alm_process@@AAEHPAPAVQListViewItem@@@Z 10022289 f   multiinputimpl.obj
 0001:00021289       __ehhandler$?displayHome@ProcessListView@@AAEX_N@Z 10022289 f   multiinputimpl.obj
 0001:00021289       __ehhandler$?addProcesses@multiInput@@QAEXPAVQListViewItem@@@Z 10022289 f   multiinputimpl.obj
 0001:00021289       __ehhandler$?removeProcesses@multiInput@@QAEXPAVQListViewItem@@@Z 10022289 f   multiinputimpl.obj
 0001:00021289       __ehhandler$?enableRemove@multiInput@@QAEXXZ 10022289 f   multiinputimpl.obj
 0001:00021289       __ehhandler$?enableAdd@multiInput@@QAEXXZ 10022289 f   multiinputimpl.obj
 0001:000212a4       __unwindfunclet$?filterChange@multiInput@@QAEXABVQString@@@Z$0 100222a4 f   multiinputimpl.obj
 0001:000212ad       __unwindfunclet$?filterChange@multiInput@@QAEXABVQString@@@Z$1 100222ad f   multiinputimpl.obj
 0001:000212b6       __unwindfunclet$?filterChange@multiInput@@QAEXABVQString@@@Z$2 100222b6 f   multiinputimpl.obj
 0001:000212bf       __unwindfunclet$?filterChange@multiInput@@QAEXABVQString@@@Z$3 100222bf f   multiinputimpl.obj
 0001:000212c8       __unwindfunclet$?filterChange@multiInput@@QAEXABVQString@@@Z$4 100222c8 f   multiinputimpl.obj
 0001:000212d1       __unwindfunclet$?filterChange@multiInput@@QAEXABVQString@@@Z$5 100222d1 f   multiinputimpl.obj
 0001:000212da       __ehhandler$?filterChange@multiInput@@QAEXABVQString@@@Z 100222da f   multiinputimpl.obj
 0001:000212f5       __unwindfunclet$?keys@plugindesc@@UAE?AVQStringList@@ABVQString@@0@Z$0 100222f5 f   plugindesc.obj
 0001:0002130f       __unwindfunclet$?keys@plugindesc@@UAE?AVQStringList@@ABVQString@@0@Z$1 1002230f f   plugindesc.obj
 0001:00021318       __ehhandler$?keys@plugindesc@@UAE?AVQStringList@@ABVQString@@0@Z 10022318 f   plugindesc.obj
 0001:00021333       __unwindfunclet$??0singleInputBase@@QAE@PAVQWidget@@PBD_NI@Z$0 10022333 f   singleinput.obj
 0001:0002133c       __unwindfunclet$??0singleInputBase@@QAE@PAVQWidget@@PBD_NI@Z$1 1002233c f   singleinput.obj
 0001:00021346       __unwindfunclet$??0singleInputBase@@QAE@PAVQWidget@@PBD_NI@Z$2 10022346 f   singleinput.obj
 0001:00021350       __unwindfunclet$??0singleInputBase@@QAE@PAVQWidget@@PBD_NI@Z$3 10022350 f   singleinput.obj
 0001:0002135a       __unwindfunclet$??0singleInputBase@@QAE@PAVQWidget@@PBD_NI@Z$4 1002235a f   singleinput.obj
 0001:00021364       __unwindfunclet$??0singleInputBase@@QAE@PAVQWidget@@PBD_NI@Z$5 10022364 f   singleinput.obj
 0001:0002136e       __unwindfunclet$??0singleInputBase@@QAE@PAVQWidget@@PBD_NI@Z$6 1002236e f   singleinput.obj
 0001:00021378       __unwindfunclet$??0singleInputBase@@QAE@PAVQWidget@@PBD_NI@Z$7 10022378 f   singleinput.obj
 0001:00021382       __unwindfunclet$??0singleInputBase@@QAE@PAVQWidget@@PBD_NI@Z$8 10022382 f   singleinput.obj
 0001:0002138c       __unwindfunclet$??0singleInputBase@@QAE@PAVQWidget@@PBD_NI@Z$9 1002238c f   singleinput.obj
 0001:00021396       __unwindfunclet$??0singleInputBase@@QAE@PAVQWidget@@PBD_NI@Z$10 10022396 f   singleinput.obj
 0001:000213a0       __unwindfunclet$??0singleInputBase@@QAE@PAVQWidget@@PBD_NI@Z$11 100223a0 f   singleinput.obj
 0001:000213aa       __ehhandler$??0singleInputBase@@QAE@PAVQWidget@@PBD_NI@Z 100223aa f   singleinput.obj
 0001:000213c5       __unwindfunclet$?languageChange@singleInputBase@@MAEXXZ$0 100223c5 f   singleinput.obj
 0001:000213ce       __unwindfunclet$?languageChange@singleInputBase@@MAEXXZ$1 100223ce f   singleinput.obj
 0001:000213d7       __unwindfunclet$?languageChange@singleInputBase@@MAEXXZ$2 100223d7 f   singleinput.obj
 0001:000213e0       __unwindfunclet$?languageChange@singleInputBase@@MAEXXZ$3 100223e0 f   singleinput.obj
 0001:000213e9       __unwindfunclet$?languageChange@singleInputBase@@MAEXXZ$4 100223e9 f   singleinput.obj
 0001:000213f2       __unwindfunclet$?languageChange@singleInputBase@@MAEXXZ$5 100223f2 f   singleinput.obj
 0001:000213fb       __unwindfunclet$?languageChange@singleInputBase@@MAEXXZ$6 100223fb f   singleinput.obj
 0001:00021404       __ehhandler$?languageChange@singleInputBase@@MAEXXZ 10022404 f   singleinput.obj
 0001:0002141f       __unwindfunclet$??0singleInput@@QAE@ABV?$map@VQString@@PAVcProcess@@U?$less@VQString@@@std@@V?$allocator@U?$pair@$$CBVQString@@PAVcProcess@@@std@@@4@@std@@QBVcProcess@@W4ESingleType@0@PAVQWidget@@PBD_NI@Z$0 1002241f f   singleinputimpl.obj
 0001:00021427       __unwindfunclet$??0singleInput@@QAE@ABV?$map@VQString@@PAVcProcess@@U?$less@VQString@@@std@@V?$allocator@U?$pair@$$CBVQString@@PAVcProcess@@@std@@@4@@std@@QBVcProcess@@W4ESingleType@0@PAVQWidget@@PBD_NI@Z$1 10022427 f   singleinputimpl.obj
 0001:00021430       __unwindfunclet$??0singleInput@@QAE@ABV?$map@VQString@@PAVcProcess@@U?$less@VQString@@@std@@V?$allocator@U?$pair@$$CBVQString@@PAVcProcess@@@std@@@4@@std@@QBVcProcess@@W4ESingleType@0@PAVQWidget@@PBD_NI@Z$2 10022430 f   singleinputimpl.obj
 0001:00021439       __unwindfunclet$??0singleInput@@QAE@ABV?$map@VQString@@PAVcProcess@@U?$less@VQString@@@std@@V?$allocator@U?$pair@$$CBVQString@@PAVcProcess@@@std@@@4@@std@@QBVcProcess@@W4ESingleType@0@PAVQWidget@@PBD_NI@Z$12 10022439 f   singleinputimpl.obj
 0001:00021442       __unwindfunclet$??0singleInput@@QAE@ABV?$map@VQString@@PAVcProcess@@U?$less@VQString@@@std@@V?$allocator@U?$pair@$$CBVQString@@PAVcProcess@@@std@@@4@@std@@QBVcProcess@@W4ESingleType@0@PAVQWidget@@PBD_NI@Z$13 10022442 f   singleinputimpl.obj
 0001:0002144b       __unwindfunclet$??0singleInput@@QAE@ABV?$map@VQString@@PAVcProcess@@U?$less@VQString@@@std@@V?$allocator@U?$pair@$$CBVQString@@PAVcProcess@@@std@@@4@@std@@QBVcProcess@@W4ESingleType@0@PAVQWidget@@PBD_NI@Z$14 1002244b f   singleinputimpl.obj
 0001:00021455       __unwindfunclet$??0singleInput@@QAE@ABV?$map@VQString@@PAVcProcess@@U?$less@VQString@@@std@@V?$allocator@U?$pair@$$CBVQString@@PAVcProcess@@@std@@@4@@std@@QBVcProcess@@W4ESingleType@0@PAVQWidget@@PBD_NI@Z$15 10022455 f   singleinputimpl.obj
 0001:0002145e       __unwindfunclet$??0singleInput@@QAE@ABV?$map@VQString@@PAVcProcess@@U?$less@VQString@@@std@@V?$allocator@U?$pair@$$CBVQString@@PAVcProcess@@@std@@@4@@std@@QBVcProcess@@W4ESingleType@0@PAVQWidget@@PBD_NI@Z$16 1002245e f   singleinputimpl.obj
 0001:00021467       __unwindfunclet$??0singleInput@@QAE@ABV?$map@VQString@@PAVcProcess@@U?$less@VQString@@@std@@V?$allocator@U?$pair@$$CBVQString@@PAVcProcess@@@std@@@4@@std@@QBVcProcess@@W4ESingleType@0@PAVQWidget@@PBD_NI@Z$17 10022467 f   singleinputimpl.obj
 0001:00021470       __unwindfunclet$??0singleInput@@QAE@ABV?$map@VQString@@PAVcProcess@@U?$less@VQString@@@std@@V?$allocator@U?$pair@$$CBVQString@@PAVcProcess@@@std@@@4@@std@@QBVcProcess@@W4ESingleType@0@PAVQWidget@@PBD_NI@Z$18 10022470 f   singleinputimpl.obj
 0001:00021479       __unwindfunclet$??0singleInput@@QAE@ABV?$map@VQString@@PAVcProcess@@U?$less@VQString@@@std@@V?$allocator@U?$pair@$$CBVQString@@PAVcProcess@@@std@@@4@@std@@QBVcProcess@@W4ESingleType@0@PAVQWidget@@PBD_NI@Z$19 10022479 f   singleinputimpl.obj
 0001:00021482       __unwindfunclet$??0singleInput@@QAE@ABV?$map@VQString@@PAVcProcess@@U?$less@VQString@@@std@@V?$allocator@U?$pair@$$CBVQString@@PAVcProcess@@@std@@@4@@std@@QBVcProcess@@W4ESingleType@0@PAVQWidget@@PBD_NI@Z$20 10022482 f   singleinputimpl.obj
 0001:0002148b       __unwindfunclet$??0singleInput@@QAE@ABV?$map@VQString@@PAVcProcess@@U?$less@VQString@@@std@@V?$allocator@U?$pair@$$CBVQString@@PAVcProcess@@@std@@@4@@std@@QBVcProcess@@W4ESingleType@0@PAVQWidget@@PBD_NI@Z$21 1002248b f   singleinputimpl.obj
 0001:00021494       __unwindfunclet$??0singleInput@@QAE@ABV?$map@VQString@@PAVcProcess@@U?$less@VQString@@@std@@V?$allocator@U?$pair@$$CBVQString@@PAVcProcess@@@std@@@4@@std@@QBVcProcess@@W4ESingleType@0@PAVQWidget@@PBD_NI@Z$23 10022494 f   singleinputimpl.obj
 0001:0002149d       __unwindfunclet$??0singleInput@@QAE@ABV?$map@VQString@@PAVcProcess@@U?$less@VQString@@@std@@V?$allocator@U?$pair@$$CBVQString@@PAVcProcess@@@std@@@4@@std@@QBVcProcess@@W4ESingleType@0@PAVQWidget@@PBD_NI@Z$3 1002249d f   singleinputimpl.obj
 0001:000214a7       __unwindfunclet$??0singleInput@@QAE@ABV?$map@VQString@@PAVcProcess@@U?$less@VQString@@@std@@V?$allocator@U?$pair@$$CBVQString@@PAVcProcess@@@std@@@4@@std@@QBVcProcess@@W4ESingleType@0@PAVQWidget@@PBD_NI@Z$4 100224a7 f   singleinputimpl.obj
 0001:000214b0       __unwindfunclet$??0singleInput@@QAE@ABV?$map@VQString@@PAVcProcess@@U?$less@VQString@@@std@@V?$allocator@U?$pair@$$CBVQString@@PAVcProcess@@@std@@@4@@std@@QBVcProcess@@W4ESingleType@0@PAVQWidget@@PBD_NI@Z$5 100224b0 f   singleinputimpl.obj
 0001:000214b9       __unwindfunclet$??0singleInput@@QAE@ABV?$map@VQString@@PAVcProcess@@U?$less@VQString@@@std@@V?$allocator@U?$pair@$$CBVQString@@PAVcProcess@@@std@@@4@@std@@QBVcProcess@@W4ESingleType@0@PAVQWidget@@PBD_NI@Z$6 100224b9 f   singleinputimpl.obj
 0001:000214c2       __unwindfunclet$??0singleInput@@QAE@ABV?$map@VQString@@PAVcProcess@@U?$less@VQString@@@std@@V?$allocator@U?$pair@$$CBVQString@@PAVcProcess@@@std@@@4@@std@@QBVcProcess@@W4ESingleType@0@PAVQWidget@@PBD_NI@Z$7 100224c2 f   singleinputimpl.obj
 0001:000214cb       __unwindfunclet$??0singleInput@@QAE@ABV?$map@VQString@@PAVcProcess@@U?$less@VQString@@@std@@V?$allocator@U?$pair@$$CBVQString@@PAVcProcess@@@std@@@4@@std@@QBVcProcess@@W4ESingleType@0@PAVQWidget@@PBD_NI@Z$8 100224cb f   singleinputimpl.obj
 0001:000214d4       __unwindfunclet$??0singleInput@@QAE@ABV?$map@VQString@@PAVcProcess@@U?$less@VQString@@@std@@V?$allocator@U?$pair@$$CBVQString@@PAVcProcess@@@std@@@4@@std@@QBVcProcess@@W4ESingleType@0@PAVQWidget@@PBD_NI@Z$9 100224d4 f   singleinputimpl.obj
 0001:000214dd       __unwindfunclet$??0singleInput@@QAE@ABV?$map@VQString@@PAVcProcess@@U?$less@VQString@@@std@@V?$allocator@U?$pair@$$CBVQString@@PAVcProcess@@@std@@@4@@std@@QBVcProcess@@W4ESingleType@0@PAVQWidget@@PBD_NI@Z$10 100224dd f   singleinputimpl.obj
 0001:000214e6       __ehhandler$??0singleInput@@QAE@ABV?$map@VQString@@PAVcProcess@@U?$less@VQString@@@std@@V?$allocator@U?$pair@$$CBVQString@@PAVcProcess@@@std@@@4@@std@@QBVcProcess@@W4ESingleType@0@PAVQWidget@@PBD_NI@Z 100224e6 f   singleinputimpl.obj
 0001:00021501       __unwindfunclet$?filterChange@alm_process@@AAEXABVQString@@@Z$0 10022501 f   singleinputimpl.obj
 0001:00021501       __unwindfunclet$?filterChange@singleInput@@AAEXABVQString@@@Z$0 10022501 f   singleinputimpl.obj
 0001:0002150a       __unwindfunclet$?filterChange@singleInput@@AAEXABVQString@@@Z$1 1002250a f   singleinputimpl.obj
 0001:0002150a       __unwindfunclet$?filterChange@alm_process@@AAEXABVQString@@@Z$1 1002250a f   singleinputimpl.obj
 0001:00021513       __unwindfunclet$?filterChange@singleInput@@AAEXABVQString@@@Z$2 10022513 f   singleinputimpl.obj
 0001:00021513       __unwindfunclet$?filterChange@alm_process@@AAEXABVQString@@@Z$2 10022513 f   singleinputimpl.obj
 0001:0002151c       __unwindfunclet$?filterChange@singleInput@@AAEXABVQString@@@Z$3 1002251c f   singleinputimpl.obj
 0001:0002151c       __unwindfunclet$?filterChange@alm_process@@AAEXABVQString@@@Z$3 1002251c f   singleinputimpl.obj
 0001:00021525       __ehhandler$?filterChange@singleInput@@AAEXABVQString@@@Z 10022525 f   singleinputimpl.obj
 0001:00021525       __ehhandler$?filterChange@alm_process@@AAEXABVQString@@@Z 10022525 f   singleinputimpl.obj
 0001:00021540       __unwindfunclet$??0template_dialogBase@@QAE@PAVQWidget@@PBD_NI@Z$0 10022540 f   template_dialog.obj
 0001:00021549       __unwindfunclet$??0template_dialogBase@@QAE@PAVQWidget@@PBD_NI@Z$1 10022549 f   template_dialog.obj
 0001:00021553       __unwindfunclet$??0template_dialogBase@@QAE@PAVQWidget@@PBD_NI@Z$2 10022553 f   template_dialog.obj
 0001:0002155d       __unwindfunclet$??0template_dialogBase@@QAE@PAVQWidget@@PBD_NI@Z$3 1002255d f   template_dialog.obj
 0001:00021567       __unwindfunclet$??0template_dialogBase@@QAE@PAVQWidget@@PBD_NI@Z$4 10022567 f   template_dialog.obj
 0001:00021571       __unwindfunclet$??0template_dialogBase@@QAE@PAVQWidget@@PBD_NI@Z$5 10022571 f   template_dialog.obj
 0001:0002157b       __unwindfunclet$??0template_dialogBase@@QAE@PAVQWidget@@PBD_NI@Z$6 1002257b f   template_dialog.obj
 0001:00021585       __unwindfunclet$??0template_dialogBase@@QAE@PAVQWidget@@PBD_NI@Z$7 10022585 f   template_dialog.obj
 0001:0002158f       __unwindfunclet$??0template_dialogBase@@QAE@PAVQWidget@@PBD_NI@Z$8 1002258f f   template_dialog.obj
 0001:00021599       __unwindfunclet$??0template_dialogBase@@QAE@PAVQWidget@@PBD_NI@Z$9 10022599 f   template_dialog.obj
 0001:000215a3       __unwindfunclet$??0template_dialogBase@@QAE@PAVQWidget@@PBD_NI@Z$10 100225a3 f   template_dialog.obj
 0001:000215ad       __unwindfunclet$??0template_dialogBase@@QAE@PAVQWidget@@PBD_NI@Z$11 100225ad f   template_dialog.obj
 0001:000215b7       __unwindfunclet$??0template_dialogBase@@QAE@PAVQWidget@@PBD_NI@Z$12 100225b7 f   template_dialog.obj
 0001:000215c1       __unwindfunclet$??0template_dialogBase@@QAE@PAVQWidget@@PBD_NI@Z$13 100225c1 f   template_dialog.obj
 0001:000215cb       __unwindfunclet$??0template_dialogBase@@QAE@PAVQWidget@@PBD_NI@Z$14 100225cb f   template_dialog.obj
 0001:000215d5       __unwindfunclet$??0template_dialogBase@@QAE@PAVQWidget@@PBD_NI@Z$15 100225d5 f   template_dialog.obj
 0001:000215df       __unwindfunclet$??0template_dialogBase@@QAE@PAVQWidget@@PBD_NI@Z$16 100225df f   template_dialog.obj
 0001:000215e9       __unwindfunclet$??0template_dialogBase@@QAE@PAVQWidget@@PBD_NI@Z$17 100225e9 f   template_dialog.obj
 0001:000215f3       __unwindfunclet$??0template_dialogBase@@QAE@PAVQWidget@@PBD_NI@Z$18 100225f3 f   template_dialog.obj
 0001:000215fd       __unwindfunclet$??0template_dialogBase@@QAE@PAVQWidget@@PBD_NI@Z$19 100225fd f   template_dialog.obj
 0001:00021607       __unwindfunclet$??0template_dialogBase@@QAE@PAVQWidget@@PBD_NI@Z$20 10022607 f   template_dialog.obj
 0001:00021611       __unwindfunclet$??0template_dialogBase@@QAE@PAVQWidget@@PBD_NI@Z$21 10022611 f   template_dialog.obj
 0001:0002161b       __unwindfunclet$??0template_dialogBase@@QAE@PAVQWidget@@PBD_NI@Z$22 1002261b f   template_dialog.obj
 0001:00021625       __unwindfunclet$??0template_dialogBase@@QAE@PAVQWidget@@PBD_NI@Z$23 10022625 f   template_dialog.obj
 0001:0002162f       __unwindfunclet$??0template_dialogBase@@QAE@PAVQWidget@@PBD_NI@Z$24 1002262f f   template_dialog.obj
 0001:00021639       __unwindfunclet$??0template_dialogBase@@QAE@PAVQWidget@@PBD_NI@Z$25 10022639 f   template_dialog.obj
 0001:00021643       __unwindfunclet$??0template_dialogBase@@QAE@PAVQWidget@@PBD_NI@Z$26 10022643 f   template_dialog.obj
 0001:0002164d       __unwindfunclet$??0template_dialogBase@@QAE@PAVQWidget@@PBD_NI@Z$27 1002264d f   template_dialog.obj
 0001:00021657       __unwindfunclet$??0template_dialogBase@@QAE@PAVQWidget@@PBD_NI@Z$28 10022657 f   template_dialog.obj
 0001:00021661       __unwindfunclet$??0template_dialogBase@@QAE@PAVQWidget@@PBD_NI@Z$29 10022661 f   template_dialog.obj
 0001:0002166b       __unwindfunclet$??0template_dialogBase@@QAE@PAVQWidget@@PBD_NI@Z$30 1002266b f   template_dialog.obj
 0001:00021675       __unwindfunclet$??0template_dialogBase@@QAE@PAVQWidget@@PBD_NI@Z$31 10022675 f   template_dialog.obj
 0001:0002167f       __ehhandler$??0template_dialogBase@@QAE@PAVQWidget@@PBD_NI@Z 1002267f f   template_dialog.obj
 0001:0002169a       __unwindfunclet$?languageChange@template_dialogBase@@MAEXXZ$0 1002269a f   template_dialog.obj
 0001:000216a3       __unwindfunclet$?languageChange@template_dialogBase@@MAEXXZ$1 100226a3 f   template_dialog.obj
 0001:000216ac       __unwindfunclet$?languageChange@template_dialogBase@@MAEXXZ$2 100226ac f   template_dialog.obj
 0001:000216b5       __unwindfunclet$?languageChange@template_dialogBase@@MAEXXZ$3 100226b5 f   template_dialog.obj
 0001:000216be       __unwindfunclet$?languageChange@template_dialogBase@@MAEXXZ$4 100226be f   template_dialog.obj
 0001:000216c7       __unwindfunclet$?languageChange@template_dialogBase@@MAEXXZ$5 100226c7 f   template_dialog.obj
 0001:000216d0       __unwindfunclet$?languageChange@template_dialogBase@@MAEXXZ$6 100226d0 f   template_dialog.obj
 0001:000216d9       __unwindfunclet$?languageChange@template_dialogBase@@MAEXXZ$7 100226d9 f   template_dialog.obj
 0001:000216e2       __unwindfunclet$?languageChange@template_dialogBase@@MAEXXZ$8 100226e2 f   template_dialog.obj
 0001:000216eb       __unwindfunclet$?languageChange@template_dialogBase@@MAEXXZ$9 100226eb f   template_dialog.obj
 0001:000216f4       __unwindfunclet$?languageChange@template_dialogBase@@MAEXXZ$10 100226f4 f   template_dialog.obj
 0001:000216fd       __unwindfunclet$?languageChange@template_dialogBase@@MAEXXZ$11 100226fd f   template_dialog.obj
 0001:00021706       __unwindfunclet$?languageChange@template_dialogBase@@MAEXXZ$12 10022706 f   template_dialog.obj
 0001:0002170f       __unwindfunclet$?languageChange@template_dialogBase@@MAEXXZ$13 1002270f f   template_dialog.obj
 0001:00021718       __unwindfunclet$?languageChange@template_dialogBase@@MAEXXZ$14 10022718 f   template_dialog.obj
 0001:00021721       __unwindfunclet$?languageChange@template_dialogBase@@MAEXXZ$15 10022721 f   template_dialog.obj
 0001:0002172a       __unwindfunclet$?languageChange@template_dialogBase@@MAEXXZ$16 1002272a f   template_dialog.obj
 0001:00021733       __unwindfunclet$?languageChange@template_dialogBase@@MAEXXZ$17 10022733 f   template_dialog.obj
 0001:0002173c       __unwindfunclet$?languageChange@template_dialogBase@@MAEXXZ$18 1002273c f   template_dialog.obj
 0001:00021745       __unwindfunclet$?languageChange@template_dialogBase@@MAEXXZ$19 10022745 f   template_dialog.obj
 0001:0002174e       __unwindfunclet$?languageChange@template_dialogBase@@MAEXXZ$20 1002274e f   template_dialog.obj
 0001:00021757       __unwindfunclet$?languageChange@template_dialogBase@@MAEXXZ$21 10022757 f   template_dialog.obj
 0001:00021760       __ehhandler$?languageChange@template_dialogBase@@MAEXXZ 10022760 f   template_dialog.obj
 0001:0002177b       __unwindfunclet$??0template_dialog@@QAE@ABV?$QPtrList@VcProcess@@@@ABVQStringList@@PAVQWidget@@PBD_NI@Z$0 1002277b f   template_dialogimpl.obj
 0001:00021783       __unwindfunclet$??0template_dialog@@QAE@ABV?$QPtrList@VcProcess@@@@ABVQStringList@@PAVQWidget@@PBD_NI@Z$1 10022783 f   template_dialogimpl.obj
 0001:0002178c       __unwindfunclet$??0template_dialog@@QAE@ABV?$QPtrList@VcProcess@@@@ABVQStringList@@PAVQWidget@@PBD_NI@Z$2 1002278c f   template_dialogimpl.obj
 0001:00021794       __unwindfunclet$??0template_dialog@@QAE@ABV?$QPtrList@VcProcess@@@@ABVQStringList@@PAVQWidget@@PBD_NI@Z$3 10022794 f   template_dialogimpl.obj
 0001:0002179d       __ehhandler$??0template_dialog@@QAE@ABV?$QPtrList@VcProcess@@@@ABVQStringList@@PAVQWidget@@PBD_NI@Z 1002279d f   template_dialogimpl.obj
 0001:000217b8       __unwindfunclet$?copyProcesses@template_dialog@@QAEXAAV?$QPtrList@VcProcess@@@@AAV?$map@VQString@@PAVcProcess@@U?$less@VQString@@@std@@V?$allocator@U?$pair@$$CBVQString@@PAVcProcess@@@std@@@4@@std@@PAVQListView@@@Z$0 100227b8 f   template_dialogimpl.obj
 0001:000217c1       __unwindfunclet$?copyProcesses@template_dialog@@QAEXAAV?$QPtrList@VcProcess@@@@AAV?$map@VQString@@PAVcProcess@@U?$less@VQString@@@std@@V?$allocator@U?$pair@$$CBVQString@@PAVcProcess@@@std@@@4@@std@@PAVQListView@@@Z$1 100227c1 f   template_dialogimpl.obj
 0001:000217ca       __unwindfunclet$?copyProcesses@template_dialog@@QAEXAAV?$QPtrList@VcProcess@@@@AAV?$map@VQString@@PAVcProcess@@U?$less@VQString@@@std@@V?$allocator@U?$pair@$$CBVQString@@PAVcProcess@@@std@@@4@@std@@PAVQListView@@@Z$2 100227ca f   template_dialogimpl.obj
 0001:000217d3       __unwindfunclet$?copyProcesses@template_dialog@@QAEXAAV?$QPtrList@VcProcess@@@@AAV?$map@VQString@@PAVcProcess@@U?$less@VQString@@@std@@V?$allocator@U?$pair@$$CBVQString@@PAVcProcess@@@std@@@4@@std@@PAVQListView@@@Z$3 100227d3 f   template_dialogimpl.obj
 0001:000217dc       __unwindfunclet$?copyProcesses@template_dialog@@QAEXAAV?$QPtrList@VcProcess@@@@AAV?$map@VQString@@PAVcProcess@@U?$less@VQString@@@std@@V?$allocator@U?$pair@$$CBVQString@@PAVcProcess@@@std@@@4@@std@@PAVQListView@@@Z$4 100227dc f   template_dialogimpl.obj
 0001:000217e5       __unwindfunclet$?copyProcesses@template_dialog@@QAEXAAV?$QPtrList@VcProcess@@@@AAV?$map@VQString@@PAVcProcess@@U?$less@VQString@@@std@@V?$allocator@U?$pair@$$CBVQString@@PAVcProcess@@@std@@@4@@std@@PAVQListView@@@Z$5 100227e5 f   template_dialogimpl.obj
 0001:000217ee       __unwindfunclet$?copyProcesses@template_dialog@@QAEXAAV?$QPtrList@VcProcess@@@@AAV?$map@VQString@@PAVcProcess@@U?$less@VQString@@@std@@V?$allocator@U?$pair@$$CBVQString@@PAVcProcess@@@std@@@4@@std@@PAVQListView@@@Z$6 100227ee f   template_dialogimpl.obj
 0001:000217f7       __unwindfunclet$?copyProcesses@template_dialog@@QAEXAAV?$QPtrList@VcProcess@@@@AAV?$map@VQString@@PAVcProcess@@U?$less@VQString@@@std@@V?$allocator@U?$pair@$$CBVQString@@PAVcProcess@@@std@@@4@@std@@PAVQListView@@@Z$7 100227f7 f   template_dialogimpl.obj
 0001:00021801       __unwindfunclet$?copyProcesses@template_dialog@@QAEXAAV?$QPtrList@VcProcess@@@@AAV?$map@VQString@@PAVcProcess@@U?$less@VQString@@@std@@V?$allocator@U?$pair@$$CBVQString@@PAVcProcess@@@std@@@4@@std@@PAVQListView@@@Z$8 10022801 f   template_dialogimpl.obj
 0001:0002180a       __unwindfunclet$?copyProcesses@template_dialog@@QAEXAAV?$QPtrList@VcProcess@@@@AAV?$map@VQString@@PAVcProcess@@U?$less@VQString@@@std@@V?$allocator@U?$pair@$$CBVQString@@PAVcProcess@@@std@@@4@@std@@PAVQListView@@@Z$9 1002280a f   template_dialogimpl.obj
 0001:00021813       __unwindfunclet$?copyProcesses@template_dialog@@QAEXAAV?$QPtrList@VcProcess@@@@AAV?$map@VQString@@PAVcProcess@@U?$less@VQString@@@std@@V?$allocator@U?$pair@$$CBVQString@@PAVcProcess@@@std@@@4@@std@@PAVQListView@@@Z$10 10022813 f   template_dialogimpl.obj
 0001:0002181c       __unwindfunclet$?copyProcesses@template_dialog@@QAEXAAV?$QPtrList@VcProcess@@@@AAV?$map@VQString@@PAVcProcess@@U?$less@VQString@@@std@@V?$allocator@U?$pair@$$CBVQString@@PAVcProcess@@@std@@@4@@std@@PAVQListView@@@Z$11 1002281c f   template_dialogimpl.obj
 0001:00021824       __unwindfunclet$?copyProcesses@template_dialog@@QAEXAAV?$QPtrList@VcProcess@@@@AAV?$map@VQString@@PAVcProcess@@U?$less@VQString@@@std@@V?$allocator@U?$pair@$$CBVQString@@PAVcProcess@@@std@@@4@@std@@PAVQListView@@@Z$12 10022824 f   template_dialogimpl.obj
 0001:0002182e       __unwindfunclet$?copyProcesses@template_dialog@@QAEXAAV?$QPtrList@VcProcess@@@@AAV?$map@VQString@@PAVcProcess@@U?$less@VQString@@@std@@V?$allocator@U?$pair@$$CBVQString@@PAVcProcess@@@std@@@4@@std@@PAVQListView@@@Z$13 1002282e f   template_dialogimpl.obj
 0001:00021837       __unwindfunclet$?copyProcesses@template_dialog@@QAEXAAV?$QPtrList@VcProcess@@@@AAV?$map@VQString@@PAVcProcess@@U?$less@VQString@@@std@@V?$allocator@U?$pair@$$CBVQString@@PAVcProcess@@@std@@@4@@std@@PAVQListView@@@Z$14 10022837 f   template_dialogimpl.obj
 0001:00021840       __unwindfunclet$?copyProcesses@template_dialog@@QAEXAAV?$QPtrList@VcProcess@@@@AAV?$map@VQString@@PAVcProcess@@U?$less@VQString@@@std@@V?$allocator@U?$pair@$$CBVQString@@PAVcProcess@@@std@@@4@@std@@PAVQListView@@@Z$15 10022840 f   template_dialogimpl.obj
 0001:00021849       __ehhandler$?copyProcesses@template_dialog@@QAEXAAV?$QPtrList@VcProcess@@@@AAV?$map@VQString@@PAVcProcess@@U?$less@VQString@@@std@@V?$allocator@U?$pair@$$CBVQString@@PAVcProcess@@@std@@@4@@std@@PAVQListView@@@Z 10022849 f   template_dialogimpl.obj
 0001:00021864       __unwindfunclet$?getThisPrefix@template_dialog@@QAE?AVQString@@H@Z$0 10022864 f   template_dialogimpl.obj
 0001:0002187e       __unwindfunclet$?getThisPrefix@template_dialog@@QAE?AVQString@@H@Z$1 1002287e f   template_dialogimpl.obj
 0001:00021887       __unwindfunclet$?getThisPrefix@template_dialog@@QAE?AVQString@@H@Z$2 10022887 f   template_dialogimpl.obj
 0001:00021890       __unwindfunclet$?getThisPrefix@template_dialog@@QAE?AVQString@@H@Z$3 10022890 f   template_dialogimpl.obj
 0001:00021899       __unwindfunclet$?getThisPrefix@template_dialog@@QAE?AVQString@@H@Z$4 10022899 f   template_dialogimpl.obj
 0001:000218a2       __unwindfunclet$?getThisPrefix@template_dialog@@QAE?AVQString@@H@Z$5 100228a2 f   template_dialogimpl.obj
 0001:000218ab       __ehhandler$?getThisPrefix@template_dialog@@QAE?AVQString@@H@Z 100228ab f   template_dialogimpl.obj
 0001:000218c6       __unwindfunclet$?setSelectionData@template_dialog@@AAEXHQBVcProcess@@@Z$0 100228c6 f   template_dialogimpl.obj
 0001:000218cf       __unwindfunclet$?setSelectionData@template_dialog@@AAEXHQBVcProcess@@@Z$1 100228cf f   template_dialogimpl.obj
 0001:000218d8       __ehhandler$?setSelectionData@template_dialog@@AAEXHQBVcProcess@@@Z 100228d8 f   template_dialogimpl.obj
 0001:000218f3       __unwindfunclet$?showExample@template_dialog@@QAEXXZ$0 100228f3 f   template_dialogimpl.obj
 0001:000218fc       __unwindfunclet$?showExample@template_dialog@@QAEXXZ$1 100228fc f   template_dialogimpl.obj
 0001:00021905       __unwindfunclet$?showExample@template_dialog@@QAEXXZ$2 10022905 f   template_dialogimpl.obj
 0001:0002190e       __unwindfunclet$?showExample@template_dialog@@QAEXXZ$3 1002290e f   template_dialogimpl.obj
 0001:00021917       __unwindfunclet$?showExample@template_dialog@@QAEXXZ$4 10022917 f   template_dialogimpl.obj
 0001:00021920       __unwindfunclet$?showExample@template_dialog@@QAEXXZ$5 10022920 f   template_dialogimpl.obj
 0001:00021929       __unwindfunclet$?showExample@template_dialog@@QAEXXZ$6 10022929 f   template_dialogimpl.obj
 0001:00021932       __ehhandler$?showExample@template_dialog@@QAEXXZ 10022932 f   template_dialogimpl.obj
 0001:0002194d       __unwindfunclet$??0CheckContDialogBase@@QAE@PAVQWidget@@PBD_NI@Z$0 1002294d f   checkcontributiondialog.obj
 0001:00021956       __unwindfunclet$??0CheckContDialogBase@@QAE@PAVQWidget@@PBD_NI@Z$1 10022956 f   checkcontributiondialog.obj
 0001:00021960       __unwindfunclet$??0CheckContDialogBase@@QAE@PAVQWidget@@PBD_NI@Z$2 10022960 f   checkcontributiondialog.obj
 0001:0002196a       __unwindfunclet$??0CheckContDialogBase@@QAE@PAVQWidget@@PBD_NI@Z$3 1002296a f   checkcontributiondialog.obj
 0001:00021974       __unwindfunclet$??0CheckContDialogBase@@QAE@PAVQWidget@@PBD_NI@Z$4 10022974 f   checkcontributiondialog.obj
 0001:0002197e       __unwindfunclet$??0CheckContDialogBase@@QAE@PAVQWidget@@PBD_NI@Z$5 1002297e f   checkcontributiondialog.obj
 0001:00021988       __unwindfunclet$??0CheckContDialogBase@@QAE@PAVQWidget@@PBD_NI@Z$6 10022988 f   checkcontributiondialog.obj
 0001:00021992       __unwindfunclet$??0CheckContDialogBase@@QAE@PAVQWidget@@PBD_NI@Z$7 10022992 f   checkcontributiondialog.obj
 0001:0002199c       __unwindfunclet$??0CheckContDialogBase@@QAE@PAVQWidget@@PBD_NI@Z$8 1002299c f   checkcontributiondialog.obj
 0001:000219a6       __unwindfunclet$??0CheckContDialogBase@@QAE@PAVQWidget@@PBD_NI@Z$9 100229a6 f   checkcontributiondialog.obj
 0001:000219b0       __unwindfunclet$??0CheckContDialogBase@@QAE@PAVQWidget@@PBD_NI@Z$10 100229b0 f   checkcontributiondialog.obj
 0001:000219ba       __unwindfunclet$??0CheckContDialogBase@@QAE@PAVQWidget@@PBD_NI@Z$11 100229ba f   checkcontributiondialog.obj
 0001:000219c4       __unwindfunclet$??0CheckContDialogBase@@QAE@PAVQWidget@@PBD_NI@Z$12 100229c4 f   checkcontributiondialog.obj
 0001:000219ce       __unwindfunclet$??0CheckContDialogBase@@QAE@PAVQWidget@@PBD_NI@Z$13 100229ce f   checkcontributiondialog.obj
 0001:000219d8       __unwindfunclet$??0CheckContDialogBase@@QAE@PAVQWidget@@PBD_NI@Z$14 100229d8 f   checkcontributiondialog.obj
 0001:000219e2       __unwindfunclet$??0CheckContDialogBase@@QAE@PAVQWidget@@PBD_NI@Z$15 100229e2 f   checkcontributiondialog.obj
 0001:000219ec       __unwindfunclet$??0CheckContDialogBase@@QAE@PAVQWidget@@PBD_NI@Z$16 100229ec f   checkcontributiondialog.obj
 0001:000219f6       __unwindfunclet$??0CheckContDialogBase@@QAE@PAVQWidget@@PBD_NI@Z$17 100229f6 f   checkcontributiondialog.obj
 0001:00021a00       __unwindfunclet$??0CheckContDialogBase@@QAE@PAVQWidget@@PBD_NI@Z$18 10022a00 f   checkcontributiondialog.obj
 0001:00021a0a       __unwindfunclet$??0CheckContDialogBase@@QAE@PAVQWidget@@PBD_NI@Z$19 10022a0a f   checkcontributiondialog.obj
 0001:00021a14       __unwindfunclet$??0CheckContDialogBase@@QAE@PAVQWidget@@PBD_NI@Z$20 10022a14 f   checkcontributiondialog.obj
 0001:00021a1e       __unwindfunclet$??0CheckContDialogBase@@QAE@PAVQWidget@@PBD_NI@Z$21 10022a1e f   checkcontributiondialog.obj
 0001:00021a28       __unwindfunclet$??0CheckContDialogBase@@QAE@PAVQWidget@@PBD_NI@Z$22 10022a28 f   checkcontributiondialog.obj
 0001:00021a32       __unwindfunclet$??0CheckContDialogBase@@QAE@PAVQWidget@@PBD_NI@Z$23 10022a32 f   checkcontributiondialog.obj
 0001:00021a3c       __unwindfunclet$??0CheckContDialogBase@@QAE@PAVQWidget@@PBD_NI@Z$24 10022a3c f   checkcontributiondialog.obj
 0001:00021a46       __unwindfunclet$??0CheckContDialogBase@@QAE@PAVQWidget@@PBD_NI@Z$25 10022a46 f   checkcontributiondialog.obj
 0001:00021a50       __unwindfunclet$??0CheckContDialogBase@@QAE@PAVQWidget@@PBD_NI@Z$26 10022a50 f   checkcontributiondialog.obj
 0001:00021a5a       __unwindfunclet$??0CheckContDialogBase@@QAE@PAVQWidget@@PBD_NI@Z$27 10022a5a f   checkcontributiondialog.obj
 0001:00021a64       __unwindfunclet$??0CheckContDialogBase@@QAE@PAVQWidget@@PBD_NI@Z$28 10022a64 f   checkcontributiondialog.obj
 0001:00021a6e       __unwindfunclet$??0CheckContDialogBase@@QAE@PAVQWidget@@PBD_NI@Z$29 10022a6e f   checkcontributiondialog.obj
 0001:00021a78       __unwindfunclet$??0CheckContDialogBase@@QAE@PAVQWidget@@PBD_NI@Z$30 10022a78 f   checkcontributiondialog.obj
 0001:00021a82       __ehhandler$??0CheckContDialogBase@@QAE@PAVQWidget@@PBD_NI@Z 10022a82 f   checkcontributiondialog.obj
 0001:00021a9d       __unwindfunclet$?languageChange@CheckContDialogBase@@MAEXXZ$0 10022a9d f   checkcontributiondialog.obj
 0001:00021aa6       __unwindfunclet$?languageChange@CheckContDialogBase@@MAEXXZ$1 10022aa6 f   checkcontributiondialog.obj
 0001:00021aaf       __unwindfunclet$?languageChange@CheckContDialogBase@@MAEXXZ$2 10022aaf f   checkcontributiondialog.obj
 0001:00021ab8       __unwindfunclet$?languageChange@CheckContDialogBase@@MAEXXZ$3 10022ab8 f   checkcontributiondialog.obj
 0001:00021ac1       __unwindfunclet$?languageChange@CheckContDialogBase@@MAEXXZ$4 10022ac1 f   checkcontributiondialog.obj
 0001:00021aca       __unwindfunclet$?languageChange@CheckContDialogBase@@MAEXXZ$5 10022aca f   checkcontributiondialog.obj
 0001:00021ad3       __unwindfunclet$?languageChange@CheckContDialogBase@@MAEXXZ$6 10022ad3 f   checkcontributiondialog.obj
 0001:00021adc       __unwindfunclet$?languageChange@CheckContDialogBase@@MAEXXZ$7 10022adc f   checkcontributiondialog.obj
 0001:00021ae5       __unwindfunclet$?languageChange@CheckContDialogBase@@MAEXXZ$8 10022ae5 f   checkcontributiondialog.obj
 0001:00021aee       __unwindfunclet$?languageChange@CheckContDialogBase@@MAEXXZ$9 10022aee f   checkcontributiondialog.obj
 0001:00021af7       __unwindfunclet$?languageChange@CheckContDialogBase@@MAEXXZ$10 10022af7 f   checkcontributiondialog.obj
 0001:00021b00       __unwindfunclet$?languageChange@CheckContDialogBase@@MAEXXZ$11 10022b00 f   checkcontributiondialog.obj
 0001:00021b09       __unwindfunclet$?languageChange@CheckContDialogBase@@MAEXXZ$12 10022b09 f   checkcontributiondialog.obj
 0001:00021b12       __unwindfunclet$?languageChange@CheckContDialogBase@@MAEXXZ$13 10022b12 f   checkcontributiondialog.obj
 0001:00021b1b       __unwindfunclet$?languageChange@CheckContDialogBase@@MAEXXZ$14 10022b1b f   checkcontributiondialog.obj
 0001:00021b24       __unwindfunclet$?languageChange@CheckContDialogBase@@MAEXXZ$15 10022b24 f   checkcontributiondialog.obj
 0001:00021b2d       __unwindfunclet$?languageChange@CheckContDialogBase@@MAEXXZ$16 10022b2d f   checkcontributiondialog.obj
 0001:00021b36       __ehhandler$?languageChange@CheckContDialogBase@@MAEXXZ 10022b36 f   checkcontributiondialog.obj
 0001:00021b51       __unwindfunclet$??0LatchAckDialogBase@@QAE@PAVQWidget@@PBD_NI@Z$0 10022b51 f   latchackdialog.obj
 0001:00021b5a       __unwindfunclet$??0LatchAckDialogBase@@QAE@PAVQWidget@@PBD_NI@Z$1 10022b5a f   latchackdialog.obj
 0001:00021b64       __unwindfunclet$??0LatchAckDialogBase@@QAE@PAVQWidget@@PBD_NI@Z$2 10022b64 f   latchackdialog.obj
 0001:00021b6e       __unwindfunclet$??0LatchAckDialogBase@@QAE@PAVQWidget@@PBD_NI@Z$3 10022b6e f   latchackdialog.obj
 0001:00021b78       __unwindfunclet$??0LatchAckDialogBase@@QAE@PAVQWidget@@PBD_NI@Z$4 10022b78 f   latchackdialog.obj
 0001:00021b82       __unwindfunclet$??0LatchAckDialogBase@@QAE@PAVQWidget@@PBD_NI@Z$5 10022b82 f   latchackdialog.obj
 0001:00021b8c       __unwindfunclet$??0LatchAckDialogBase@@QAE@PAVQWidget@@PBD_NI@Z$6 10022b8c f   latchackdialog.obj
 0001:00021b96       __unwindfunclet$??0LatchAckDialogBase@@QAE@PAVQWidget@@PBD_NI@Z$7 10022b96 f   latchackdialog.obj
 0001:00021ba0       __unwindfunclet$??0LatchAckDialogBase@@QAE@PAVQWidget@@PBD_NI@Z$8 10022ba0 f   latchackdialog.obj
 0001:00021baa       __unwindfunclet$??0LatchAckDialogBase@@QAE@PAVQWidget@@PBD_NI@Z$9 10022baa f   latchackdialog.obj
 0001:00021bb4       __ehhandler$??0LatchAckDialogBase@@QAE@PAVQWidget@@PBD_NI@Z 10022bb4 f   latchackdialog.obj
 0001:00021bcf       __unwindfunclet$?languageChange@LatchAckDialogBase@@MAEXXZ$0 10022bcf f   latchackdialog.obj
 0001:00021bd8       __unwindfunclet$?languageChange@LatchAckDialogBase@@MAEXXZ$1 10022bd8 f   latchackdialog.obj
 0001:00021be1       __unwindfunclet$?languageChange@LatchAckDialogBase@@MAEXXZ$2 10022be1 f   latchackdialog.obj
 0001:00021bea       __unwindfunclet$?languageChange@LatchAckDialogBase@@MAEXXZ$3 10022bea f   latchackdialog.obj
 0001:00021bf3       __unwindfunclet$?languageChange@LatchAckDialogBase@@MAEXXZ$4 10022bf3 f   latchackdialog.obj
 0001:00021bfc       __unwindfunclet$?languageChange@LatchAckDialogBase@@MAEXXZ$5 10022bfc f   latchackdialog.obj
 0001:00021c05       __unwindfunclet$?languageChange@LatchAckDialogBase@@MAEXXZ$6 10022c05 f   latchackdialog.obj
 0001:00021c0e       __unwindfunclet$?languageChange@LatchAckDialogBase@@MAEXXZ$7 10022c0e f   latchackdialog.obj
 0001:00021c17       __unwindfunclet$?languageChange@LatchAckDialogBase@@MAEXXZ$8 10022c17 f   latchackdialog.obj
 0001:00021c20       __unwindfunclet$?languageChange@LatchAckDialogBase@@MAEXXZ$9 10022c20 f   latchackdialog.obj
 0001:00021c29       __ehhandler$?languageChange@LatchAckDialogBase@@MAEXXZ 10022c29 f   latchackdialog.obj
 0001:00021c44       __unwindfunclet$?qt_emit@alm_process@@UAE_NHPAUQUObject@@@Z$0 10022c44 f   moc_alm_process.obj
 0001:00021c4d       __ehhandler$?qt_emit@alm_process@@UAE_NHPAUQUObject@@@Z 10022c4d f   moc_alm_process.obj
 0001:00021c68       __unwindfunclet$?qt_invoke@alm_process@@UAE_NHPAUQUObject@@@Z$0 10022c68 f   moc_alm_process.obj
 0001:00021c71       __unwindfunclet$?qt_invoke@alm_process@@UAE_NHPAUQUObject@@@Z$2 10022c71 f   moc_alm_process.obj
 0001:00021c7a       __unwindfunclet$?qt_invoke@alm_process@@UAE_NHPAUQUObject@@@Z$3 10022c7a f   moc_alm_process.obj
 0001:00021c83       __ehhandler$?qt_invoke@alm_process@@UAE_NHPAUQUObject@@@Z 10022c83 f   moc_alm_process.obj
 0001:00021c9e       __unwindfunclet$?navToAck@cProc_dialog@@IAEXVQString@@00@Z$0 10022c9e f   moc_cProc_dialog.obj
 0001:00021ca7       __unwindfunclet$?navToAck@cProc_dialog@@IAEXVQString@@00@Z$1 10022ca7 f   moc_cProc_dialog.obj
 0001:00021cb0       __unwindfunclet$?navToAck@cProc_dialog@@IAEXVQString@@00@Z$2 10022cb0 f   moc_cProc_dialog.obj
 0001:00021cb9       __unwindfunclet$?navToAck@cProc_dialog@@IAEXVQString@@00@Z$3 10022cb9 f   moc_cProc_dialog.obj
 0001:00021ccd       __ehhandler$?navToAck@cProc_dialog@@IAEXVQString@@00@Z 10022ccd f   moc_cProc_dialog.obj
 0001:00021cf2       __unwindfunclet$?navToOutput@cProc_dialog@@IAEXVQString@@0@Z$0 10022cf2 f   moc_cProc_dialog.obj
 0001:00021cf2       __unwindfunclet$?command@alm_process@@IAEXVQString@@0@Z$0 10022cf2 f   moc_cProc_dialog.obj
 0001:00021cfb       __unwindfunclet$?navToOutput@cProc_dialog@@IAEXVQString@@0@Z$1 10022cfb f   moc_cProc_dialog.obj
 0001:00021cfb       __unwindfunclet$?command@alm_process@@IAEXVQString@@0@Z$1 10022cfb f   moc_cProc_dialog.obj
 0001:00021d04       __unwindfunclet$?navToOutput@cProc_dialog@@IAEXVQString@@0@Z$2 10022d04 f   moc_cProc_dialog.obj
 0001:00021d04       __unwindfunclet$?command@alm_process@@IAEXVQString@@0@Z$2 10022d04 f   moc_cProc_dialog.obj
 0001:00021d18       __ehhandler$?navToOutput@cProc_dialog@@IAEXVQString@@0@Z 10022d18 f   moc_cProc_dialog.obj
 0001:00021d18       __ehhandler$?command@alm_process@@IAEXVQString@@0@Z 10022d18 f   moc_cProc_dialog.obj
 0001:00021d3d       __unwindfunclet$?navToProc@cProc_dialog@@IAEXVQString@@@Z$0 10022d3d f   moc_cProc_dialog.obj
 0001:00021d46       __unwindfunclet$?navToProc@cProc_dialog@@IAEXVQString@@@Z$1 10022d46 f   moc_cProc_dialog.obj
 0001:00021d4f       __ehhandler$?navToProc@cProc_dialog@@IAEXVQString@@@Z 10022d4f f   moc_cProc_dialog.obj
 0001:00021d6a       __unwindfunclet$?qt_emit@cProc_dialog@@UAE_NHPAUQUObject@@@Z$3 10022d6a f   moc_cProc_dialog.obj
 0001:00021d73       __unwindfunclet$?qt_emit@cProc_dialog@@UAE_NHPAUQUObject@@@Z$4 10022d73 f   moc_cProc_dialog.obj
 0001:00021d7c       __unwindfunclet$?qt_emit@cProc_dialog@@UAE_NHPAUQUObject@@@Z$1 10022d7c f   moc_cProc_dialog.obj
 0001:00021d85       __ehhandler$?qt_emit@cProc_dialog@@UAE_NHPAUQUObject@@@Z 10022d85 f   moc_cProc_dialog.obj
 0001:00021da0       __unwindfunclet$?updateProc@cProc_dialog@@IAEXPAVcProcess@@@Z$0 10022da0 f   moc_cProc_dialog.obj
 0001:00021db4       __ehhandler$?updateProc@cProc_dialog@@IAEXPAVcProcess@@@Z 10022db4 f   moc_cProc_dialog.obj
 0001:00021dd9       __unwindfunclet$??0proc_config@@QAE@PAVQWidget@@PBDI@Z$0 10022dd9 f   proc_config.obj
 0001:00021de2       __unwindfunclet$??0proc_config@@QAE@PAVQWidget@@PBDI@Z$1 10022de2 f   proc_config.obj
 0001:00021df1       __unwindfunclet$??0proc_config@@QAE@PAVQWidget@@PBDI@Z$2 10022df1 f   proc_config.obj
 0001:00021e00       __unwindfunclet$??0proc_config@@QAE@PAVQWidget@@PBDI@Z$3 10022e00 f   proc_config.obj
 0001:00021e0a       __unwindfunclet$??0proc_config@@QAE@PAVQWidget@@PBDI@Z$4 10022e0a f   proc_config.obj
 0001:00021e14       __unwindfunclet$??0proc_config@@QAE@PAVQWidget@@PBDI@Z$5 10022e14 f   proc_config.obj
 0001:00021e1e       __unwindfunclet$??0proc_config@@QAE@PAVQWidget@@PBDI@Z$6 10022e1e f   proc_config.obj
 0001:00021e28       __unwindfunclet$??0proc_config@@QAE@PAVQWidget@@PBDI@Z$7 10022e28 f   proc_config.obj
 0001:00021e32       __unwindfunclet$??0proc_config@@QAE@PAVQWidget@@PBDI@Z$8 10022e32 f   proc_config.obj
 0001:00021e3c       __unwindfunclet$??0proc_config@@QAE@PAVQWidget@@PBDI@Z$9 10022e3c f   proc_config.obj
 0001:00021e46       __unwindfunclet$??0proc_config@@QAE@PAVQWidget@@PBDI@Z$10 10022e46 f   proc_config.obj
 0001:00021e50       __unwindfunclet$??0proc_config@@QAE@PAVQWidget@@PBDI@Z$11 10022e50 f   proc_config.obj
 0001:00021e5a       __unwindfunclet$??0proc_config@@QAE@PAVQWidget@@PBDI@Z$12 10022e5a f   proc_config.obj
 0001:00021e64       __unwindfunclet$??0proc_config@@QAE@PAVQWidget@@PBDI@Z$13 10022e64 f   proc_config.obj
 0001:00021e6e       __unwindfunclet$??0proc_config@@QAE@PAVQWidget@@PBDI@Z$14 10022e6e f   proc_config.obj
 0001:00021e78       __unwindfunclet$??0proc_config@@QAE@PAVQWidget@@PBDI@Z$15 10022e78 f   proc_config.obj
 0001:00021e82       __unwindfunclet$??0proc_config@@QAE@PAVQWidget@@PBDI@Z$16 10022e82 f   proc_config.obj
 0001:00021e8c       __unwindfunclet$??0proc_config@@QAE@PAVQWidget@@PBDI@Z$17 10022e8c f   proc_config.obj
 0001:00021e96       __unwindfunclet$??0proc_config@@QAE@PAVQWidget@@PBDI@Z$18 10022e96 f   proc_config.obj
 0001:00021ea0       __unwindfunclet$??0proc_config@@QAE@PAVQWidget@@PBDI@Z$19 10022ea0 f   proc_config.obj
 0001:00021eaa       __unwindfunclet$??0proc_config@@QAE@PAVQWidget@@PBDI@Z$20 10022eaa f   proc_config.obj
 0001:00021eb4       __unwindfunclet$??0proc_config@@QAE@PAVQWidget@@PBDI@Z$21 10022eb4 f   proc_config.obj
 0001:00021ebe       __unwindfunclet$??0proc_config@@QAE@PAVQWidget@@PBDI@Z$22 10022ebe f   proc_config.obj
 0001:00021ec8       __unwindfunclet$??0proc_config@@QAE@PAVQWidget@@PBDI@Z$23 10022ec8 f   proc_config.obj
 0001:00021ed2       __unwindfunclet$??0proc_config@@QAE@PAVQWidget@@PBDI@Z$24 10022ed2 f   proc_config.obj
 0001:00021edc       __unwindfunclet$??0proc_config@@QAE@PAVQWidget@@PBDI@Z$25 10022edc f   proc_config.obj
 0001:00021ee6       __unwindfunclet$??0proc_config@@QAE@PAVQWidget@@PBDI@Z$26 10022ee6 f   proc_config.obj
 0001:00021ef0       __unwindfunclet$??0proc_config@@QAE@PAVQWidget@@PBDI@Z$27 10022ef0 f   proc_config.obj
 0001:00021efa       __unwindfunclet$??0proc_config@@QAE@PAVQWidget@@PBDI@Z$28 10022efa f   proc_config.obj
 0001:00021f04       __unwindfunclet$??0proc_config@@QAE@PAVQWidget@@PBDI@Z$29 10022f04 f   proc_config.obj
 0001:00021f0e       __unwindfunclet$??0proc_config@@QAE@PAVQWidget@@PBDI@Z$30 10022f0e f   proc_config.obj
 0001:00021f18       __unwindfunclet$??0proc_config@@QAE@PAVQWidget@@PBDI@Z$31 10022f18 f   proc_config.obj
 0001:00021f22       __unwindfunclet$??0proc_config@@QAE@PAVQWidget@@PBDI@Z$32 10022f22 f   proc_config.obj
 0001:00021f2c       __unwindfunclet$??0proc_config@@QAE@PAVQWidget@@PBDI@Z$33 10022f2c f   proc_config.obj
 0001:00021f36       __unwindfunclet$??0proc_config@@QAE@PAVQWidget@@PBDI@Z$34 10022f36 f   proc_config.obj
 0001:00021f40       __unwindfunclet$??0proc_config@@QAE@PAVQWidget@@PBDI@Z$35 10022f40 f   proc_config.obj
 0001:00021f4a       __unwindfunclet$??0proc_config@@QAE@PAVQWidget@@PBDI@Z$36 10022f4a f   proc_config.obj
 0001:00021f54       __unwindfunclet$??0proc_config@@QAE@PAVQWidget@@PBDI@Z$37 10022f54 f   proc_config.obj
 0001:00021f5e       __unwindfunclet$??0proc_config@@QAE@PAVQWidget@@PBDI@Z$38 10022f5e f   proc_config.obj
 0001:00021f68       __unwindfunclet$??0proc_config@@QAE@PAVQWidget@@PBDI@Z$39 10022f68 f   proc_config.obj
 0001:00021f72       __unwindfunclet$??0proc_config@@QAE@PAVQWidget@@PBDI@Z$40 10022f72 f   proc_config.obj
 0001:00021f7c       __unwindfunclet$??0proc_config@@QAE@PAVQWidget@@PBDI@Z$41 10022f7c f   proc_config.obj
 0001:00021f86       __unwindfunclet$??0proc_config@@QAE@PAVQWidget@@PBDI@Z$42 10022f86 f   proc_config.obj
 0001:00021f90       __unwindfunclet$??0proc_config@@QAE@PAVQWidget@@PBDI@Z$43 10022f90 f   proc_config.obj
 0001:00021f9a       __unwindfunclet$??0proc_config@@QAE@PAVQWidget@@PBDI@Z$44 10022f9a f   proc_config.obj
 0001:00021fa4       __unwindfunclet$??0proc_config@@QAE@PAVQWidget@@PBDI@Z$45 10022fa4 f   proc_config.obj
 0001:00021fae       __unwindfunclet$??0proc_config@@QAE@PAVQWidget@@PBDI@Z$46 10022fae f   proc_config.obj
 0001:00021fb8       __unwindfunclet$??0proc_config@@QAE@PAVQWidget@@PBDI@Z$47 10022fb8 f   proc_config.obj
 0001:00021fc2       __unwindfunclet$??0proc_config@@QAE@PAVQWidget@@PBDI@Z$48 10022fc2 f   proc_config.obj
 0001:00021fcc       __unwindfunclet$??0proc_config@@QAE@PAVQWidget@@PBDI@Z$49 10022fcc f   proc_config.obj
 0001:00021fd6       __unwindfunclet$??0proc_config@@QAE@PAVQWidget@@PBDI@Z$50 10022fd6 f   proc_config.obj
 0001:00021fe0       __unwindfunclet$??0proc_config@@QAE@PAVQWidget@@PBDI@Z$51 10022fe0 f   proc_config.obj
 0001:00021fea       __unwindfunclet$??0proc_config@@QAE@PAVQWidget@@PBDI@Z$52 10022fea f   proc_config.obj
 0001:00021ff4       __unwindfunclet$??0proc_config@@QAE@PAVQWidget@@PBDI@Z$53 10022ff4 f   proc_config.obj
 0001:00021ffe       __unwindfunclet$??0proc_config@@QAE@PAVQWidget@@PBDI@Z$54 10022ffe f   proc_config.obj
 0001:00022008       __unwindfunclet$??0proc_config@@QAE@PAVQWidget@@PBDI@Z$55 10023008 f   proc_config.obj
 0001:00022012       __unwindfunclet$??0proc_config@@QAE@PAVQWidget@@PBDI@Z$56 10023012 f   proc_config.obj
 0001:0002201c       __unwindfunclet$??0proc_config@@QAE@PAVQWidget@@PBDI@Z$57 1002301c f   proc_config.obj
 0001:00022026       __unwindfunclet$??0proc_config@@QAE@PAVQWidget@@PBDI@Z$58 10023026 f   proc_config.obj
 0001:00022030       __unwindfunclet$??0proc_config@@QAE@PAVQWidget@@PBDI@Z$59 10023030 f   proc_config.obj
 0001:0002203a       __unwindfunclet$??0proc_config@@QAE@PAVQWidget@@PBDI@Z$60 1002303a f   proc_config.obj
 0001:00022044       __unwindfunclet$??0proc_config@@QAE@PAVQWidget@@PBDI@Z$61 10023044 f   proc_config.obj
 0001:0002204e       __unwindfunclet$??0proc_config@@QAE@PAVQWidget@@PBDI@Z$62 1002304e f   proc_config.obj
 0001:00022058       __unwindfunclet$??0proc_config@@QAE@PAVQWidget@@PBDI@Z$63 10023058 f   proc_config.obj
 0001:00022062       __unwindfunclet$??0proc_config@@QAE@PAVQWidget@@PBDI@Z$64 10023062 f   proc_config.obj
 0001:0002206c       __unwindfunclet$??0proc_config@@QAE@PAVQWidget@@PBDI@Z$65 1002306c f   proc_config.obj
 0001:00022076       __unwindfunclet$??0proc_config@@QAE@PAVQWidget@@PBDI@Z$66 10023076 f   proc_config.obj
 0001:00022080       __unwindfunclet$??0proc_config@@QAE@PAVQWidget@@PBDI@Z$67 10023080 f   proc_config.obj
 0001:0002208a       __unwindfunclet$??0proc_config@@QAE@PAVQWidget@@PBDI@Z$68 1002308a f   proc_config.obj
 0001:00022094       __unwindfunclet$??0proc_config@@QAE@PAVQWidget@@PBDI@Z$69 10023094 f   proc_config.obj
 0001:0002209e       __unwindfunclet$??0proc_config@@QAE@PAVQWidget@@PBDI@Z$70 1002309e f   proc_config.obj
 0001:000220a8       __unwindfunclet$??0proc_config@@QAE@PAVQWidget@@PBDI@Z$71 100230a8 f   proc_config.obj
 0001:000220b2       __unwindfunclet$??0proc_config@@QAE@PAVQWidget@@PBDI@Z$72 100230b2 f   proc_config.obj
 0001:000220bc       __unwindfunclet$??0proc_config@@QAE@PAVQWidget@@PBDI@Z$73 100230bc f   proc_config.obj
 0001:000220c6       __unwindfunclet$??0proc_config@@QAE@PAVQWidget@@PBDI@Z$74 100230c6 f   proc_config.obj
 0001:000220d0       __unwindfunclet$??0proc_config@@QAE@PAVQWidget@@PBDI@Z$75 100230d0 f   proc_config.obj
 0001:000220da       __unwindfunclet$??0proc_config@@QAE@PAVQWidget@@PBDI@Z$76 100230da f   proc_config.obj
 0001:000220e4       __unwindfunclet$??0proc_config@@QAE@PAVQWidget@@PBDI@Z$77 100230e4 f   proc_config.obj
 0001:000220ee       __unwindfunclet$??0proc_config@@QAE@PAVQWidget@@PBDI@Z$78 100230ee f   proc_config.obj
 0001:000220f8       __unwindfunclet$??0proc_config@@QAE@PAVQWidget@@PBDI@Z$79 100230f8 f   proc_config.obj
 0001:00022102       __unwindfunclet$??0proc_config@@QAE@PAVQWidget@@PBDI@Z$80 10023102 f   proc_config.obj
 0001:0002210c       __unwindfunclet$??0proc_config@@QAE@PAVQWidget@@PBDI@Z$81 1002310c f   proc_config.obj
 0001:00022116       __unwindfunclet$??0proc_config@@QAE@PAVQWidget@@PBDI@Z$82 10023116 f   proc_config.obj
 0001:00022120       __unwindfunclet$??0proc_config@@QAE@PAVQWidget@@PBDI@Z$83 10023120 f   proc_config.obj
 0001:0002212a       __unwindfunclet$??0proc_config@@QAE@PAVQWidget@@PBDI@Z$84 1002312a f   proc_config.obj
 0001:00022134       __unwindfunclet$??0proc_config@@QAE@PAVQWidget@@PBDI@Z$85 10023134 f   proc_config.obj
 0001:0002213e       __unwindfunclet$??0proc_config@@QAE@PAVQWidget@@PBDI@Z$86 1002313e f   proc_config.obj
 0001:00022148       __unwindfunclet$??0proc_config@@QAE@PAVQWidget@@PBDI@Z$87 10023148 f   proc_config.obj
 0001:00022152       __unwindfunclet$??0proc_config@@QAE@PAVQWidget@@PBDI@Z$88 10023152 f   proc_config.obj
 0001:0002215c       __unwindfunclet$??0proc_config@@QAE@PAVQWidget@@PBDI@Z$89 1002315c f   proc_config.obj
 0001:00022166       __unwindfunclet$??0proc_config@@QAE@PAVQWidget@@PBDI@Z$90 10023166 f   proc_config.obj
 0001:00022170       __unwindfunclet$??0proc_config@@QAE@PAVQWidget@@PBDI@Z$91 10023170 f   proc_config.obj
 0001:0002217a       __unwindfunclet$??0proc_config@@QAE@PAVQWidget@@PBDI@Z$92 1002317a f   proc_config.obj
 0001:00022184       __unwindfunclet$??0proc_config@@QAE@PAVQWidget@@PBDI@Z$93 10023184 f   proc_config.obj
 0001:0002218e       __unwindfunclet$??0proc_config@@QAE@PAVQWidget@@PBDI@Z$94 1002318e f   proc_config.obj
 0001:00022198       __unwindfunclet$??0proc_config@@QAE@PAVQWidget@@PBDI@Z$95 10023198 f   proc_config.obj
 0001:000221a2       __unwindfunclet$??0proc_config@@QAE@PAVQWidget@@PBDI@Z$96 100231a2 f   proc_config.obj
 0001:000221ac       __unwindfunclet$??0proc_config@@QAE@PAVQWidget@@PBDI@Z$97 100231ac f   proc_config.obj
 0001:000221b6       __unwindfunclet$??0proc_config@@QAE@PAVQWidget@@PBDI@Z$98 100231b6 f   proc_config.obj
 0001:000221c0       __unwindfunclet$??0proc_config@@QAE@PAVQWidget@@PBDI@Z$99 100231c0 f   proc_config.obj
 0001:000221ca       __unwindfunclet$??0proc_config@@QAE@PAVQWidget@@PBDI@Z$100 100231ca f   proc_config.obj
 0001:000221d4       __unwindfunclet$??0proc_config@@QAE@PAVQWidget@@PBDI@Z$101 100231d4 f   proc_config.obj
 0001:000221de       __unwindfunclet$??0proc_config@@QAE@PAVQWidget@@PBDI@Z$102 100231de f   proc_config.obj
 0001:000221e8       __unwindfunclet$??0proc_config@@QAE@PAVQWidget@@PBDI@Z$103 100231e8 f   proc_config.obj
 0001:000221f2       __unwindfunclet$??0proc_config@@QAE@PAVQWidget@@PBDI@Z$104 100231f2 f   proc_config.obj
 0001:000221fc       __unwindfunclet$??0proc_config@@QAE@PAVQWidget@@PBDI@Z$105 100231fc f   proc_config.obj
 0001:00022206       __unwindfunclet$??0proc_config@@QAE@PAVQWidget@@PBDI@Z$106 10023206 f   proc_config.obj
 0001:00022210       __unwindfunclet$??0proc_config@@QAE@PAVQWidget@@PBDI@Z$107 10023210 f   proc_config.obj
 0001:0002221a       __unwindfunclet$??0proc_config@@QAE@PAVQWidget@@PBDI@Z$108 1002321a f   proc_config.obj
 0001:00022224       __unwindfunclet$??0proc_config@@QAE@PAVQWidget@@PBDI@Z$109 10023224 f   proc_config.obj
 0001:0002222e       __unwindfunclet$??0proc_config@@QAE@PAVQWidget@@PBDI@Z$110 1002322e f   proc_config.obj
 0001:00022238       __unwindfunclet$??0proc_config@@QAE@PAVQWidget@@PBDI@Z$111 10023238 f   proc_config.obj
 0001:00022242       __unwindfunclet$??0proc_config@@QAE@PAVQWidget@@PBDI@Z$112 10023242 f   proc_config.obj
 0001:0002224c       __unwindfunclet$??0proc_config@@QAE@PAVQWidget@@PBDI@Z$113 1002324c f   proc_config.obj
 0001:00022256       __unwindfunclet$??0proc_config@@QAE@PAVQWidget@@PBDI@Z$114 10023256 f   proc_config.obj
 0001:00022260       __unwindfunclet$??0proc_config@@QAE@PAVQWidget@@PBDI@Z$115 10023260 f   proc_config.obj
 0001:0002226a       __unwindfunclet$??0proc_config@@QAE@PAVQWidget@@PBDI@Z$116 1002326a f   proc_config.obj
 0001:00022274       __unwindfunclet$??0proc_config@@QAE@PAVQWidget@@PBDI@Z$117 10023274 f   proc_config.obj
 0001:0002227e       __ehhandler$??0proc_config@@QAE@PAVQWidget@@PBDI@Z 1002327e f   proc_config.obj
 0001:00022299       __unwindfunclet$??1proc_config@@UAE@XZ$0 10023299 f   proc_config.obj
 0001:000222a2       __unwindfunclet$??1proc_config@@UAE@XZ$1 100232a2 f   proc_config.obj
 0001:000222b1       __ehhandler$??1proc_config@@UAE@XZ 100232b1 f   proc_config.obj
 0001:000222cc       __unwindfunclet$?languageChange@proc_config@@MAEXXZ$0 100232cc f   proc_config.obj
 0001:000222d5       __unwindfunclet$?languageChange@proc_config@@MAEXXZ$1 100232d5 f   proc_config.obj
 0001:000222de       __unwindfunclet$?languageChange@proc_config@@MAEXXZ$2 100232de f   proc_config.obj
 0001:000222e7       __unwindfunclet$?languageChange@proc_config@@MAEXXZ$3 100232e7 f   proc_config.obj
 0001:000222f0       __unwindfunclet$?languageChange@proc_config@@MAEXXZ$4 100232f0 f   proc_config.obj
 0001:000222f9       __unwindfunclet$?languageChange@proc_config@@MAEXXZ$5 100232f9 f   proc_config.obj
 0001:00022302       __unwindfunclet$?languageChange@proc_config@@MAEXXZ$6 10023302 f   proc_config.obj
 0001:0002230b       __unwindfunclet$?languageChange@proc_config@@MAEXXZ$7 1002330b f   proc_config.obj
 0001:00022314       __unwindfunclet$?languageChange@proc_config@@MAEXXZ$8 10023314 f   proc_config.obj
 0001:0002231d       __unwindfunclet$?languageChange@proc_config@@MAEXXZ$9 1002331d f   proc_config.obj
 0001:00022326       __unwindfunclet$?languageChange@proc_config@@MAEXXZ$10 10023326 f   proc_config.obj
 0001:0002232f       __unwindfunclet$?languageChange@proc_config@@MAEXXZ$11 1002332f f   proc_config.obj
 0001:00022338       __unwindfunclet$?languageChange@proc_config@@MAEXXZ$12 10023338 f   proc_config.obj
 0001:00022341       __unwindfunclet$?languageChange@proc_config@@MAEXXZ$13 10023341 f   proc_config.obj
 0001:0002234a       __unwindfunclet$?languageChange@proc_config@@MAEXXZ$14 1002334a f   proc_config.obj
 0001:00022353       __unwindfunclet$?languageChange@proc_config@@MAEXXZ$15 10023353 f   proc_config.obj
 0001:0002235c       __unwindfunclet$?languageChange@proc_config@@MAEXXZ$16 1002335c f   proc_config.obj
 0001:00022365       __unwindfunclet$?languageChange@proc_config@@MAEXXZ$17 10023365 f   proc_config.obj
 0001:0002236e       __unwindfunclet$?languageChange@proc_config@@MAEXXZ$18 1002336e f   proc_config.obj
 0001:00022377       __unwindfunclet$?languageChange@proc_config@@MAEXXZ$19 10023377 f   proc_config.obj
 0001:00022380       __unwindfunclet$?languageChange@proc_config@@MAEXXZ$20 10023380 f   proc_config.obj
 0001:00022389       __unwindfunclet$?languageChange@proc_config@@MAEXXZ$21 10023389 f   proc_config.obj
 0001:00022392       __unwindfunclet$?languageChange@proc_config@@MAEXXZ$22 10023392 f   proc_config.obj
 0001:0002239b       __unwindfunclet$?languageChange@proc_config@@MAEXXZ$23 1002339b f   proc_config.obj
 0001:000223a4       __unwindfunclet$?languageChange@proc_config@@MAEXXZ$24 100233a4 f   proc_config.obj
 0001:000223ad       __unwindfunclet$?languageChange@proc_config@@MAEXXZ$25 100233ad f   proc_config.obj
 0001:000223b6       __unwindfunclet$?languageChange@proc_config@@MAEXXZ$26 100233b6 f   proc_config.obj
 0001:000223bf       __unwindfunclet$?languageChange@proc_config@@MAEXXZ$27 100233bf f   proc_config.obj
 0001:000223c8       __unwindfunclet$?languageChange@proc_config@@MAEXXZ$28 100233c8 f   proc_config.obj
 0001:000223d1       __unwindfunclet$?languageChange@proc_config@@MAEXXZ$29 100233d1 f   proc_config.obj
 0001:000223da       __unwindfunclet$?languageChange@proc_config@@MAEXXZ$30 100233da f   proc_config.obj
 0001:000223e3       __unwindfunclet$?languageChange@proc_config@@MAEXXZ$31 100233e3 f   proc_config.obj
 0001:000223ec       __unwindfunclet$?languageChange@proc_config@@MAEXXZ$32 100233ec f   proc_config.obj
 0001:000223f5       __unwindfunclet$?languageChange@proc_config@@MAEXXZ$33 100233f5 f   proc_config.obj
 0001:000223fe       __unwindfunclet$?languageChange@proc_config@@MAEXXZ$34 100233fe f   proc_config.obj
 0001:00022407       __unwindfunclet$?languageChange@proc_config@@MAEXXZ$35 10023407 f   proc_config.obj
 0001:00022410       __unwindfunclet$?languageChange@proc_config@@MAEXXZ$36 10023410 f   proc_config.obj
 0001:00022419       __unwindfunclet$?languageChange@proc_config@@MAEXXZ$37 10023419 f   proc_config.obj
 0001:00022422       __unwindfunclet$?languageChange@proc_config@@MAEXXZ$38 10023422 f   proc_config.obj
 0001:0002242b       __unwindfunclet$?languageChange@proc_config@@MAEXXZ$39 1002342b f   proc_config.obj
 0001:00022434       __unwindfunclet$?languageChange@proc_config@@MAEXXZ$40 10023434 f   proc_config.obj
 0001:0002243d       __unwindfunclet$?languageChange@proc_config@@MAEXXZ$41 1002343d f   proc_config.obj
 0001:00022446       __unwindfunclet$?languageChange@proc_config@@MAEXXZ$42 10023446 f   proc_config.obj
 0001:0002244f       __unwindfunclet$?languageChange@proc_config@@MAEXXZ$43 1002344f f   proc_config.obj
 0001:00022458       __unwindfunclet$?languageChange@proc_config@@MAEXXZ$44 10023458 f   proc_config.obj
 0001:00022461       __unwindfunclet$?languageChange@proc_config@@MAEXXZ$45 10023461 f   proc_config.obj
 0001:0002246a       __unwindfunclet$?languageChange@proc_config@@MAEXXZ$46 1002346a f   proc_config.obj
 0001:00022473       __unwindfunclet$?languageChange@proc_config@@MAEXXZ$47 10023473 f   proc_config.obj
 0001:0002247c       __unwindfunclet$?languageChange@proc_config@@MAEXXZ$48 1002347c f   proc_config.obj
 0001:00022485       __unwindfunclet$?languageChange@proc_config@@MAEXXZ$49 10023485 f   proc_config.obj
 0001:0002248e       __unwindfunclet$?languageChange@proc_config@@MAEXXZ$50 1002348e f   proc_config.obj
 0001:00022497       __unwindfunclet$?languageChange@proc_config@@MAEXXZ$51 10023497 f   proc_config.obj
 0001:000224a0       __unwindfunclet$?languageChange@proc_config@@MAEXXZ$52 100234a0 f   proc_config.obj
 0001:000224a9       __unwindfunclet$?languageChange@proc_config@@MAEXXZ$53 100234a9 f   proc_config.obj
 0001:000224b2       __unwindfunclet$?languageChange@proc_config@@MAEXXZ$54 100234b2 f   proc_config.obj
 0001:000224bb       __unwindfunclet$?languageChange@proc_config@@MAEXXZ$55 100234bb f   proc_config.obj
 0001:000224c4       __unwindfunclet$?languageChange@proc_config@@MAEXXZ$56 100234c4 f   proc_config.obj
 0001:000224cd       __unwindfunclet$?languageChange@proc_config@@MAEXXZ$57 100234cd f   proc_config.obj
 0001:000224d6       __unwindfunclet$?languageChange@proc_config@@MAEXXZ$58 100234d6 f   proc_config.obj
 0001:000224df       __unwindfunclet$?languageChange@proc_config@@MAEXXZ$59 100234df f   proc_config.obj
 0001:000224e8       __unwindfunclet$?languageChange@proc_config@@MAEXXZ$60 100234e8 f   proc_config.obj
 0001:000224f1       __unwindfunclet$?languageChange@proc_config@@MAEXXZ$61 100234f1 f   proc_config.obj
 0001:000224fa       __unwindfunclet$?languageChange@proc_config@@MAEXXZ$62 100234fa f   proc_config.obj
 0001:00022503       __unwindfunclet$?languageChange@proc_config@@MAEXXZ$63 10023503 f   proc_config.obj
 0001:0002250c       __unwindfunclet$?languageChange@proc_config@@MAEXXZ$64 1002350c f   proc_config.obj
 0001:00022515       __unwindfunclet$?languageChange@proc_config@@MAEXXZ$65 10023515 f   proc_config.obj
 0001:0002251e       __unwindfunclet$?languageChange@proc_config@@MAEXXZ$66 1002351e f   proc_config.obj
 0001:00022527       __unwindfunclet$?languageChange@proc_config@@MAEXXZ$67 10023527 f   proc_config.obj
 0001:00022530       __unwindfunclet$?languageChange@proc_config@@MAEXXZ$68 10023530 f   proc_config.obj
 0001:00022539       __unwindfunclet$?languageChange@proc_config@@MAEXXZ$69 10023539 f   proc_config.obj
 0001:00022542       __unwindfunclet$?languageChange@proc_config@@MAEXXZ$70 10023542 f   proc_config.obj
 0001:0002254b       __unwindfunclet$?languageChange@proc_config@@MAEXXZ$71 1002354b f   proc_config.obj
 0001:00022554       __unwindfunclet$?languageChange@proc_config@@MAEXXZ$72 10023554 f   proc_config.obj
 0001:0002255d       __unwindfunclet$?languageChange@proc_config@@MAEXXZ$73 1002355d f   proc_config.obj
 0001:00022566       __unwindfunclet$?languageChange@proc_config@@MAEXXZ$74 10023566 f   proc_config.obj
 0001:0002256f       __unwindfunclet$?languageChange@proc_config@@MAEXXZ$75 1002356f f   proc_config.obj
 0001:00022578       __unwindfunclet$?languageChange@proc_config@@MAEXXZ$76 10023578 f   proc_config.obj
 0001:00022581       __unwindfunclet$?languageChange@proc_config@@MAEXXZ$77 10023581 f   proc_config.obj
 0001:0002258a       __unwindfunclet$?languageChange@proc_config@@MAEXXZ$78 1002358a f   proc_config.obj
 0001:00022593       __unwindfunclet$?languageChange@proc_config@@MAEXXZ$79 10023593 f   proc_config.obj
 0001:0002259c       __unwindfunclet$?languageChange@proc_config@@MAEXXZ$80 1002359c f   proc_config.obj
 0001:000225a5       __unwindfunclet$?languageChange@proc_config@@MAEXXZ$81 100235a5 f   proc_config.obj
 0001:000225ae       __unwindfunclet$?languageChange@proc_config@@MAEXXZ$82 100235ae f   proc_config.obj
 0001:000225b7       __unwindfunclet$?languageChange@proc_config@@MAEXXZ$83 100235b7 f   proc_config.obj
 0001:000225c0       __unwindfunclet$?languageChange@proc_config@@MAEXXZ$84 100235c0 f   proc_config.obj
 0001:000225c9       __unwindfunclet$?languageChange@proc_config@@MAEXXZ$85 100235c9 f   proc_config.obj
 0001:000225d2       __unwindfunclet$?languageChange@proc_config@@MAEXXZ$86 100235d2 f   proc_config.obj
 0001:000225db       __ehhandler$?languageChange@proc_config@@MAEXXZ 100235db f   proc_config.obj
 0001:000225f6       __unwindfunclet$?CreatePanel@config_mb4@@AAEXI@Z$0 100235f6 f   cfg_widgets001:config_mb4impl.obj
 0001:00022600       __unwindfunclet$?CreatePanel@config_mb4@@AAEXI@Z$1 10023600 f   cfg_widgets001:config_mb4impl.obj
 0001:0002261a       __unwindfunclet$?CreatePanel@config_mb4@@AAEXI@Z$2 1002361a f   cfg_widgets001:config_mb4impl.obj
 0001:00022624       __unwindfunclet$?CreatePanel@config_mb4@@AAEXI@Z$3 10023624 f   cfg_widgets001:config_mb4impl.obj
 0001:0002262e       __unwindfunclet$?CreatePanel@config_mb4@@AAEXI@Z$4 1002362e f   cfg_widgets001:config_mb4impl.obj
 0001:00022638       __unwindfunclet$?CreatePanel@config_mb4@@AAEXI@Z$5 10023638 f   cfg_widgets001:config_mb4impl.obj
 0001:00022642       __unwindfunclet$?CreatePanel@config_mb4@@AAEXI@Z$6 10023642 f   cfg_widgets001:config_mb4impl.obj
 0001:0002264c       __unwindfunclet$?CreatePanel@config_mb4@@AAEXI@Z$7 1002364c f   cfg_widgets001:config_mb4impl.obj
 0001:00022656       __unwindfunclet$?CreatePanel@config_mb4@@AAEXI@Z$8 10023656 f   cfg_widgets001:config_mb4impl.obj
 0001:0002265f       __unwindfunclet$?CreatePanel@config_mb4@@AAEXI@Z$9 1002365f f   cfg_widgets001:config_mb4impl.obj
 0001:00022668       __unwindfunclet$?CreatePanel@config_mb4@@AAEXI@Z$10 10023668 f   cfg_widgets001:config_mb4impl.obj
 0001:00022671       __unwindfunclet$?CreatePanel@config_mb4@@AAEXI@Z$14 10023671 f   cfg_widgets001:config_mb4impl.obj
 0001:0002267a       __unwindfunclet$?CreatePanel@config_mb4@@AAEXI@Z$13 1002367a f   cfg_widgets001:config_mb4impl.obj
 0001:00022683       __unwindfunclet$?CreatePanel@config_mb4@@AAEXI@Z$12 10023683 f   cfg_widgets001:config_mb4impl.obj
 0001:0002268c       __unwindfunclet$?CreatePanel@config_mb4@@AAEXI@Z$11 1002368c f   cfg_widgets001:config_mb4impl.obj
 0001:00022695       __unwindfunclet$?CreatePanel@config_mb4@@AAEXI@Z$15 10023695 f   cfg_widgets001:config_mb4impl.obj
 0001:0002269e       __ehhandler$?CreatePanel@config_mb4@@AAEXI@Z 1002369e f   cfg_widgets001:config_mb4impl.obj
 0001:000226b9       __unwindfunclet$?setIcon@config_mb4@@QAEXW4Icon@1@@Z$3 100236b9 f   cfg_widgets001:config_mb4impl.obj
 0001:000226c2       __unwindfunclet$?setIcon@config_mb4@@QAEXW4Icon@1@@Z$2 100236c2 f   cfg_widgets001:config_mb4impl.obj
 0001:000226cb       __unwindfunclet$?setIcon@config_mb4@@QAEXW4Icon@1@@Z$1 100236cb f   cfg_widgets001:config_mb4impl.obj
 0001:000226d4       __unwindfunclet$?setIcon@config_mb4@@QAEXW4Icon@1@@Z$0 100236d4 f   cfg_widgets001:config_mb4impl.obj
 0001:000226dd       __ehhandler$?setIcon@config_mb4@@QAEXW4Icon@1@@Z 100236dd f   cfg_widgets001:config_mb4impl.obj
 0001:000226fb       __unwindfunclet$?loadState@cfg_Settings@@SA?AVQString@@ABV2@@Z$0 100236fb f   cfg_widgets001:cfg_Settings.obj
 0001:00022704       __unwindfunclet$?loadState@cfg_Settings@@SA?AVQString@@ABV2@@Z$1 10023704 f   cfg_widgets001:cfg_Settings.obj
 0001:0002270d       __unwindfunclet$?loadState@cfg_Settings@@SA?AVQString@@ABV2@@Z$2 1002370d f   cfg_widgets001:cfg_Settings.obj
 0001:00022716       __unwindfunclet$?loadState@cfg_Settings@@SA?AVQString@@ABV2@@Z$3 10023716 f   cfg_widgets001:cfg_Settings.obj
 0001:00022730       __ehhandler$?loadState@cfg_Settings@@SA?AVQString@@ABV2@@Z 10023730 f   cfg_widgets001:cfg_Settings.obj
 0001:0002274b       __unwindfunclet$?loadState@cfg_Settings@@SAXAAVQPoint@@AAVQSize@@AA_NABVQString@@@Z$0 1002374b f   cfg_widgets001:cfg_Settings.obj
 0001:00022754       __unwindfunclet$?loadState@cfg_Settings@@SAXAAVQPoint@@AAVQSize@@AA_NABVQString@@@Z$1 10023754 f   cfg_widgets001:cfg_Settings.obj
 0001:0002275d       __ehhandler$?loadState@cfg_Settings@@SAXAAVQPoint@@AAVQSize@@AA_NABVQString@@@Z 1002375d f   cfg_widgets001:cfg_Settings.obj
 0001:00022778       __unwindfunclet$?loadState@cfg_Settings@@SAXQAVQListView@@ABVQString@@@Z$0 10023778 f   cfg_widgets001:cfg_Settings.obj
 0001:00022781       __unwindfunclet$?loadState@cfg_Settings@@SAXQAVQListView@@ABVQString@@@Z$1 10023781 f   cfg_widgets001:cfg_Settings.obj
 0001:0002278a       __ehhandler$?loadState@cfg_Settings@@SAXQAVQListView@@ABVQString@@@Z 1002378a f   cfg_widgets001:cfg_Settings.obj
 0001:000227a5       __unwindfunclet$?loadState@cfg_Settings@@SAXQAVQSplitter@@ABVQString@@@Z$0 100237a5 f   cfg_widgets001:cfg_Settings.obj
 0001:000227ae       __unwindfunclet$?loadState@cfg_Settings@@SAXQAVQSplitter@@ABVQString@@@Z$1 100237ae f   cfg_widgets001:cfg_Settings.obj
 0001:000227b7       __unwindfunclet$?loadState@cfg_Settings@@SAXQAVQSplitter@@ABVQString@@@Z$2 100237b7 f   cfg_widgets001:cfg_Settings.obj
 0001:000227c0       __ehhandler$?loadState@cfg_Settings@@SAXQAVQSplitter@@ABVQString@@@Z 100237c0 f   cfg_widgets001:cfg_Settings.obj
 0001:000227db       __unwindfunclet$?saveState@cfg_Settings@@SAXABVQPoint@@ABVQSize@@AB_NABVQString@@@Z$0 100237db f   cfg_widgets001:cfg_Settings.obj
 0001:000227e4       __unwindfunclet$?saveState@cfg_Settings@@SAXABVQPoint@@ABVQSize@@AB_NABVQString@@@Z$1 100237e4 f   cfg_widgets001:cfg_Settings.obj
 0001:000227ed       __unwindfunclet$?saveState@cfg_Settings@@SAXABVQPoint@@ABVQSize@@AB_NABVQString@@@Z$2 100237ed f   cfg_widgets001:cfg_Settings.obj
 0001:000227f6       __unwindfunclet$?saveState@cfg_Settings@@SAXABVQPoint@@ABVQSize@@AB_NABVQString@@@Z$3 100237f6 f   cfg_widgets001:cfg_Settings.obj
 0001:000227ff       __unwindfunclet$?saveState@cfg_Settings@@SAXABVQPoint@@ABVQSize@@AB_NABVQString@@@Z$4 100237ff f   cfg_widgets001:cfg_Settings.obj
 0001:00022808       __unwindfunclet$?saveState@cfg_Settings@@SAXABVQPoint@@ABVQSize@@AB_NABVQString@@@Z$5 10023808 f   cfg_widgets001:cfg_Settings.obj
 0001:00022811       __unwindfunclet$?saveState@cfg_Settings@@SAXABVQPoint@@ABVQSize@@AB_NABVQString@@@Z$6 10023811 f   cfg_widgets001:cfg_Settings.obj
 0001:0002281a       __ehhandler$?saveState@cfg_Settings@@SAXABVQPoint@@ABVQSize@@AB_NABVQString@@@Z 1002381a f   cfg_widgets001:cfg_Settings.obj
 0001:00022835       __unwindfunclet$?saveState@cfg_Settings@@SAXABVQString@@0@Z$0 10023835 f   cfg_widgets001:cfg_Settings.obj
 0001:0002283e       __unwindfunclet$?saveState@cfg_Settings@@SAXABVQString@@0@Z$1 1002383e f   cfg_widgets001:cfg_Settings.obj
 0001:00022847       __unwindfunclet$?saveState@cfg_Settings@@SAXABVQString@@0@Z$2 10023847 f   cfg_widgets001:cfg_Settings.obj
 0001:00022850       __ehhandler$?saveState@cfg_Settings@@SAXABVQString@@0@Z 10023850 f   cfg_widgets001:cfg_Settings.obj
 0001:0002286b       __unwindfunclet$?saveState@cfg_Settings@@SAXQBVQListView@@ABVQString@@@Z$0 1002386b f   cfg_widgets001:cfg_Settings.obj
 0001:00022874       __unwindfunclet$?saveState@cfg_Settings@@SAXQBVQListView@@ABVQString@@@Z$1 10023874 f   cfg_widgets001:cfg_Settings.obj
 0001:0002287d       __unwindfunclet$?saveState@cfg_Settings@@SAXQBVQListView@@ABVQString@@@Z$2 1002387d f   cfg_widgets001:cfg_Settings.obj
 0001:00022886       __unwindfunclet$?saveState@cfg_Settings@@SAXQBVQListView@@ABVQString@@@Z$3 10023886 f   cfg_widgets001:cfg_Settings.obj
 0001:0002288f       __ehhandler$?saveState@cfg_Settings@@SAXQBVQListView@@ABVQString@@@Z 1002388f f   cfg_widgets001:cfg_Settings.obj
 0001:000228aa       __unwindfunclet$?saveState@cfg_Settings@@SAXQBVQSplitter@@ABVQString@@@Z$0 100238aa f   cfg_widgets001:cfg_Settings.obj
 0001:000228b3       __unwindfunclet$?saveState@cfg_Settings@@SAXQBVQSplitter@@ABVQString@@@Z$1 100238b3 f   cfg_widgets001:cfg_Settings.obj
 0001:000228bc       __unwindfunclet$?saveState@cfg_Settings@@SAXQBVQSplitter@@ABVQString@@@Z$2 100238bc f   cfg_widgets001:cfg_Settings.obj
 0001:000228c5       __unwindfunclet$?saveState@cfg_Settings@@SAXQBVQSplitter@@ABVQString@@@Z$3 100238c5 f   cfg_widgets001:cfg_Settings.obj
 0001:000228ce       __ehhandler$?saveState@cfg_Settings@@SAXQBVQSplitter@@ABVQString@@@Z 100238ce f   cfg_widgets001:cfg_Settings.obj
 0001:000228e9       __unwindfunclet$??0cfg_ListView@@QAE@PAVQWidget@@PBD@Z$0 100238e9 f   cfg_widgets001:cfg_ListView.obj
 0001:000228f2       __unwindfunclet$??0cfg_ListView@@QAE@PAVQWidget@@PBD@Z$1 100238f2 f   cfg_widgets001:cfg_ListView.obj
 0001:000228fc       __unwindfunclet$??0cfg_ListView@@QAE@PAVQWidget@@PBD@Z$2 100238fc f   cfg_widgets001:cfg_ListView.obj
 0001:00022906       __ehhandler$??0cfg_ListView@@QAE@PAVQWidget@@PBD@Z 10023906 f   cfg_widgets001:cfg_ListView.obj
 0001:00022921       __unwindfunclet$??1cfg_ListView@@UAE@XZ$0 10023921 f   cfg_widgets001:cfg_ListView.obj
 0001:00022921       __unwindfunclet$??0ProcessListView@@QAE@PAVQWidget@@PBDI@Z$0 10023921 f   cfg_widgets001:cfg_ListView.obj
 0001:0002292a       __ehhandler$??1cfg_ListView@@UAE@XZ 1002392a f   cfg_widgets001:cfg_ListView.obj
 0001:0002292a       __ehhandler$??0ProcessListView@@QAE@PAVQWidget@@PBDI@Z 1002392a f   cfg_widgets001:cfg_ListView.obj
 0001:00022945       __unwindfunclet$?clipBoardDataChanged@cfg_Table@@IAEXXZ$0 10023945 f   cfg_widgets001:cfg_ListView.obj
 0001:00022945       __unwindfunclet$?clipBoardDataChanged@cfg_ListView@@IAEXXZ$0 10023945 f   cfg_widgets001:cfg_ListView.obj
 0001:00022945       __unwindfunclet$?showTime@cProc_dialog@@AAEXXZ$0 10023945 f   cfg_widgets001:cfg_ListView.obj
 0001:0002294e       __ehhandler$?clipBoardDataChanged@cfg_ListView@@IAEXXZ 1002394e f   cfg_widgets001:cfg_ListView.obj
 0001:0002294e       __ehhandler$?clipBoardDataChanged@cfg_Table@@IAEXXZ 1002394e f   cfg_widgets001:cfg_ListView.obj
 0001:0002294e       __ehhandler$?showTime@cProc_dialog@@AAEXXZ 1002394e f   cfg_widgets001:cfg_ListView.obj
 0001:00022969       __unwindfunclet$?copyToClipboard@cfg_ListView@@QAEXXZ$0 10023969 f   cfg_widgets001:cfg_ListView.obj
 0001:00022972       __unwindfunclet$?copyToClipboard@cfg_ListView@@QAEXXZ$1 10023972 f   cfg_widgets001:cfg_ListView.obj
 0001:0002297b       __unwindfunclet$?copyToClipboard@cfg_ListView@@QAEXXZ$2 1002397b f   cfg_widgets001:cfg_ListView.obj
 0001:00022984       __unwindfunclet$?copyToClipboard@cfg_ListView@@QAEXXZ$3 10023984 f   cfg_widgets001:cfg_ListView.obj
 0001:0002298d       __ehhandler$?copyToClipboard@cfg_ListView@@QAEXXZ 1002398d f   cfg_widgets001:cfg_ListView.obj
 0001:000229a8       __unwindfunclet$?deleteItems@cfg_ListView@@QAEXXZ$0 100239a8 f   cfg_widgets001:cfg_ListView.obj
 0001:000229b0       __unwindfunclet$?deleteItems@cfg_ListView@@QAEXXZ$1 100239b0 f   cfg_widgets001:cfg_ListView.obj
 0001:000229b9       __ehhandler$?deleteItems@cfg_ListView@@QAEXXZ 100239b9 f   cfg_widgets001:cfg_ListView.obj
 0001:000229d4       __unwindfunclet$?insertData@cfg_ListView@@QAEXXZ$0 100239d4 f   cfg_widgets001:cfg_ListView.obj
 0001:000229dd       __unwindfunclet$?insertData@cfg_ListView@@QAEXXZ$1 100239dd f   cfg_widgets001:cfg_ListView.obj
 0001:000229e6       __unwindfunclet$?insertData@cfg_ListView@@QAEXXZ$2 100239e6 f   cfg_widgets001:cfg_ListView.obj
 0001:000229ef       __unwindfunclet$?insertData@cfg_ListView@@QAEXXZ$3 100239ef f   cfg_widgets001:cfg_ListView.obj
 0001:000229f8       __ehhandler$?insertData@cfg_ListView@@QAEXXZ 100239f8 f   cfg_widgets001:cfg_ListView.obj
 0001:00022a13       __unwindfunclet$?newItem@cfg_ListView@@MAEPAVQListViewItem@@PAVQListView@@PAV2@@Z$0 10023a13 f   cfg_widgets001:cfg_ListView.obj
 0001:00022a13       __unwindfunclet$??4?$QGuardedPtr@VQPopupMenu@@@@QAEAAV0@PAVQPopupMenu@@@Z$0 10023a13 f   cfg_widgets001:cfg_ListView.obj
 0001:00022a13       __unwindfunclet$??4?$QGuardedPtr@VQDockWindow@@@@QAEAAV0@PAVQDockWindow@@@Z$0 10023a13 f   cfg_widgets001:cfg_ListView.obj
 0001:00022a13       __unwindfunclet$?changeMask@alm_process@@AAEXXZ$0 10023a13 f   cfg_widgets001:cfg_ListView.obj
 0001:00022a13       __unwindfunclet$?detachInternal@?$QMap@HPAVcAcqFileData@@@@AAEXXZ$0 10023a13 f   cfg_widgets001:cfg_ListView.obj
 0001:00022a13       __unwindfunclet$?addMultiInputs@alm_process@@AAEXXZ$0 10023a13 f   cfg_widgets001:cfg_ListView.obj
 0001:00022a13       __unwindfunclet$??0?$QGuardedPtr@VQPopupMenu@@@@QAE@XZ$0 10023a13 f   cfg_widgets001:cfg_ListView.obj
 0001:00022a13       __unwindfunclet$??0?$QGuardedPtr@VQDockWindow@@@@QAE@XZ$0 10023a13 f   cfg_widgets001:cfg_ListView.obj
 0001:00022a13       __unwindfunclet$?create@plugindesc@@UAEPAVconfig_plugin_base@@ABVQString@@00@Z$0 10023a13 f   cfg_widgets001:cfg_ListView.obj
 0001:00022a13       __unwindfunclet$?addSingleInputs@alm_process@@AAEXXZ$0 10023a13 f   cfg_widgets001:cfg_ListView.obj
 0001:00022a13       __unwindfunclet$??0?$QMap@HPAVcAcqFileData@@@@QAE@XZ$0 10023a13 f   cfg_widgets001:cfg_ListView.obj
 0001:00022a1d       __ehhandler$?detachInternal@?$QMap@HPAVcAcqFileData@@@@AAEXXZ 10023a1d f   cfg_widgets001:cfg_ListView.obj
 0001:00022a1d       __ehhandler$?addSingleInputs@alm_process@@AAEXXZ 10023a1d f   cfg_widgets001:cfg_ListView.obj
 0001:00022a1d       __ehhandler$??0?$QMap@HPAVcAcqFileData@@@@QAE@XZ 10023a1d f   cfg_widgets001:cfg_ListView.obj
 0001:00022a1d       __ehhandler$?addMultiInputs@alm_process@@AAEXXZ 10023a1d f   cfg_widgets001:cfg_ListView.obj
 0001:00022a1d       __ehhandler$??4?$QGuardedPtr@VQDockWindow@@@@QAEAAV0@PAVQDockWindow@@@Z 10023a1d f   cfg_widgets001:cfg_ListView.obj
 0001:00022a1d       __ehhandler$??0?$QGuardedPtr@VQPopupMenu@@@@QAE@XZ 10023a1d f   cfg_widgets001:cfg_ListView.obj
 0001:00022a1d       __ehhandler$?changeMask@alm_process@@AAEXXZ 10023a1d f   cfg_widgets001:cfg_ListView.obj
 0001:00022a1d       __ehhandler$?newItem@cfg_ListView@@MAEPAVQListViewItem@@PAVQListView@@PAV2@@Z 10023a1d f   cfg_widgets001:cfg_ListView.obj
 0001:00022a1d       __ehhandler$??0?$QGuardedPtr@VQDockWindow@@@@QAE@XZ 10023a1d f   cfg_widgets001:cfg_ListView.obj
 0001:00022a1d       __ehhandler$??4?$QGuardedPtr@VQPopupMenu@@@@QAEAAV0@PAVQPopupMenu@@@Z 10023a1d f   cfg_widgets001:cfg_ListView.obj
 0001:00022a1d       __ehhandler$?create@plugindesc@@UAEPAVconfig_plugin_base@@ABVQString@@00@Z 10023a1d f   cfg_widgets001:cfg_ListView.obj
 0001:00022a38       __unwindfunclet$?replaceData@cfg_ListView@@QAEXXZ$0 10023a38 f   cfg_widgets001:cfg_ListView.obj
 0001:00022a40       __unwindfunclet$?replaceData@cfg_ListView@@QAEXXZ$1 10023a40 f   cfg_widgets001:cfg_ListView.obj
 0001:00022a49       __unwindfunclet$?replaceData@cfg_ListView@@QAEXXZ$2 10023a49 f   cfg_widgets001:cfg_ListView.obj
 0001:00022a52       __unwindfunclet$?replaceData@cfg_ListView@@QAEXXZ$3 10023a52 f   cfg_widgets001:cfg_ListView.obj
 0001:00022a5b       __unwindfunclet$?replaceData@cfg_ListView@@QAEXXZ$4 10023a5b f   cfg_widgets001:cfg_ListView.obj
 0001:00022a64       __unwindfunclet$?replaceData@cfg_ListView@@QAEXXZ$5 10023a64 f   cfg_widgets001:cfg_ListView.obj
 0001:00022a6d       __ehhandler$?replaceData@cfg_ListView@@QAEXXZ 10023a6d f   cfg_widgets001:cfg_ListView.obj
 0001:00022a88       __unwindfunclet$?updateEntry@cfg_ListView@@AAEPAVQListViewItem@@QAV2@ABVQString@@_N@Z$0 10023a88 f   cfg_widgets001:cfg_ListView.obj
 0001:00022a91       __unwindfunclet$?updateEntry@cfg_ListView@@AAEPAVQListViewItem@@QAV2@ABVQString@@_N@Z$1 10023a91 f   cfg_widgets001:cfg_ListView.obj
 0001:00022a9a       __unwindfunclet$?updateEntry@cfg_ListView@@AAEPAVQListViewItem@@QAV2@ABVQString@@_N@Z$2 10023a9a f   cfg_widgets001:cfg_ListView.obj
 0001:00022aa3       __ehhandler$?updateEntry@cfg_ListView@@AAEPAVQListViewItem@@QAV2@ABVQString@@_N@Z 10023aa3 f   cfg_widgets001:cfg_ListView.obj
 0001:00022abe       __unwindfunclet$??0cfg_Table@@QAE@PAVQWidget@@PBD@Z$0 10023abe f   cfg_widgets001:cfg_Table.obj
 0001:00022ac7       __ehhandler$??0cfg_Table@@QAE@PAVQWidget@@PBD@Z 10023ac7 f   cfg_widgets001:cfg_Table.obj
 0001:00022ae2       __unwindfunclet$?copyToClipboard@cfg_Table@@QAEXXZ$0 10023ae2 f   cfg_widgets001:cfg_Table.obj
 0001:00022aeb       __unwindfunclet$?copyToClipboard@cfg_Table@@QAEXXZ$1 10023aeb f   cfg_widgets001:cfg_Table.obj
 0001:00022af4       __unwindfunclet$?copyToClipboard@cfg_Table@@QAEXXZ$2 10023af4 f   cfg_widgets001:cfg_Table.obj
 0001:00022afd       __ehhandler$?copyToClipboard@cfg_Table@@QAEXXZ 10023afd f   cfg_widgets001:cfg_Table.obj
 0001:00022b18       __unwindfunclet$?deleteItems@cfg_Table@@QAEXXZ$0 10023b18 f   cfg_widgets001:cfg_Table.obj
 0001:00022b21       __ehhandler$?deleteItems@cfg_Table@@QAEXXZ 10023b21 f   cfg_widgets001:cfg_Table.obj
 0001:00022b3c       __unwindfunclet$?fillUndoBuffer@cfg_Table@@AAEXXZ$0 10023b3c f   cfg_widgets001:cfg_Table.obj
 0001:00022b46       __unwindfunclet$?fillUndoBuffer@cfg_Table@@AAEXXZ$1 10023b46 f   cfg_widgets001:cfg_Table.obj
 0001:00022b4f       __unwindfunclet$?fillUndoBuffer@cfg_Table@@AAEXXZ$2 10023b4f f   cfg_widgets001:cfg_Table.obj
 0001:00022b58       __unwindfunclet$?fillUndoBuffer@cfg_Table@@AAEXXZ$3 10023b58 f   cfg_widgets001:cfg_Table.obj
 0001:00022b61       __ehhandler$?fillUndoBuffer@cfg_Table@@AAEXXZ 10023b61 f   cfg_widgets001:cfg_Table.obj
 0001:00022b7c       __unwindfunclet$?pasteClipboard@cfg_Table@@QAEXXZ$0 10023b7c f   cfg_widgets001:cfg_Table.obj
 0001:00022b85       __unwindfunclet$?pasteClipboard@cfg_Table@@QAEXXZ$1 10023b85 f   cfg_widgets001:cfg_Table.obj
 0001:00022b8e       __unwindfunclet$?pasteClipboard@cfg_Table@@QAEXXZ$2 10023b8e f   cfg_widgets001:cfg_Table.obj
 0001:00022b97       __unwindfunclet$?pasteClipboard@cfg_Table@@QAEXXZ$3 10023b97 f   cfg_widgets001:cfg_Table.obj
 0001:00022ba0       __unwindfunclet$?pasteClipboard@cfg_Table@@QAEXXZ$4 10023ba0 f   cfg_widgets001:cfg_Table.obj
 0001:00022ba9       __unwindfunclet$?pasteClipboard@cfg_Table@@QAEXXZ$5 10023ba9 f   cfg_widgets001:cfg_Table.obj
 0001:00022bb2       __unwindfunclet$?pasteClipboard@cfg_Table@@QAEXXZ$6 10023bb2 f   cfg_widgets001:cfg_Table.obj
 0001:00022bbb       __unwindfunclet$?pasteClipboard@cfg_Table@@QAEXXZ$7 10023bbb f   cfg_widgets001:cfg_Table.obj
 0001:00022bc4       __unwindfunclet$?pasteClipboard@cfg_Table@@QAEXXZ$8 10023bc4 f   cfg_widgets001:cfg_Table.obj
 0001:00022bcd       __unwindfunclet$?pasteClipboard@cfg_Table@@QAEXXZ$9 10023bcd f   cfg_widgets001:cfg_Table.obj
 0001:00022bd6       __unwindfunclet$?pasteClipboard@cfg_Table@@QAEXXZ$10 10023bd6 f   cfg_widgets001:cfg_Table.obj
 0001:00022bdf       __unwindfunclet$?pasteClipboard@cfg_Table@@QAEXXZ$11 10023bdf f   cfg_widgets001:cfg_Table.obj
 0001:00022be8       __unwindfunclet$?pasteClipboard@cfg_Table@@QAEXXZ$12 10023be8 f   cfg_widgets001:cfg_Table.obj
 0001:00022bf1       __unwindfunclet$?pasteClipboard@cfg_Table@@QAEXXZ$13 10023bf1 f   cfg_widgets001:cfg_Table.obj
 0001:00022bfa       __ehhandler$?pasteClipboard@cfg_Table@@QAEXXZ 10023bfa f   cfg_widgets001:cfg_Table.obj
 0001:00022c15       __unwindfunclet$?undoPaste@cfg_Table@@QAEXXZ$0 10023c15 f   cfg_widgets001:cfg_Table.obj
 0001:00022c1e       __unwindfunclet$?undoPaste@cfg_Table@@QAEXXZ$1 10023c1e f   cfg_widgets001:cfg_Table.obj
 0001:00022c27       __unwindfunclet$?undoPaste@cfg_Table@@QAEXXZ$2 10023c27 f   cfg_widgets001:cfg_Table.obj
 0001:00022c30       __ehhandler$?undoPaste@cfg_Table@@QAEXXZ 10023c30 f   cfg_widgets001:cfg_Table.obj
 0001:00022c4b       ??__FProcConfig@@YAXXZ     10023c4b f   alm_process.obj
 0001:00022c55       ??__FacqEditor@@YAXXZ      10023c55 f   cProc_dialog.obj
 0001:00022c70       ??__F?procList@cProcess@@2VQStringList@@A@@YAXXZ 10023c70 f   cProcess.obj
 0001:00022c7b       ??__F?sm_sPrefix@template_dialog@@0VQString@@A@@YAXXZ 10023c7b f   template_dialogimpl.obj
 0001:00022c9a       ??__F?sm_sSuffix@template_dialog@@0VQString@@A@@YAXXZ 10023c9a f   template_dialogimpl.obj
 0001:00022cb9       ??__FcleanUp_alm_process@@YAXXZ 10023cb9 f   moc_alm_process.obj
 0001:00022cc4       ??__FcleanUp_CheckContDialog@@YAXXZ 10023cc4 f   moc_checkContDialogImpl.obj
 0001:00022ccf       ??__FcleanUp_CheckContDialogBase@@YAXXZ 10023ccf f   moc_checkcontributiondialog.obj
 0001:00022cda       ??__FcleanUp_cProc_dialog@@YAXXZ 10023cda f   moc_cProc_dialog.obj
 0001:00022ce5       ??__FcleanUp_LatchAckDialogBase@@YAXXZ 10023ce5 f   moc_latchackdialog.obj
 0001:00022cf0       ??__FcleanUp_LatchAckDialog@@YAXXZ 10023cf0 f   moc_latchackdialogimpl.obj
 0001:00022cfb       ??__FcleanUp_multiInputBase@@YAXXZ 10023cfb f   moc_multiinput.obj
 0001:00022d06       ??__FcleanUp_multiInput@@YAXXZ 10023d06 f   moc_multiinputimpl.obj
 0001:00022d11       ??__FcleanUp_proc_config@@YAXXZ 10023d11 f   moc_proc_config.obj
 0001:00022d1c       ??__FcleanUp_singleInputBase@@YAXXZ 10023d1c f   moc_singleinput.obj
 0001:00022d27       ??__FcleanUp_singleInput@@YAXXZ 10023d27 f   moc_singleinputimpl.obj
 0001:00022d32       ??__FcleanUp_template_dialogBase@@YAXXZ 10023d32 f   moc_template_dialog.obj
 0001:00022d3d       ??__FcleanUp_template_dialog@@YAXXZ 10023d3d f   moc_template_dialogimpl.obj
 0001:00022d48       ??__FcleanUp_config_mb4@@YAXXZ 10023d48 f   cfg_widgets001:moc_config_mb4impl.obj
 0001:00022d53       ??__FcleanUp_cfg_ListView@@YAXXZ 10023d53 f   cfg_widgets001:moc_cfg_ListView.obj
 0001:00022d5e       ??__FcleanUp_cfg_Table@@YAXXZ 10023d5e f   cfg_widgets001:moc_cfg_Table.obj
 0002:00001744       _ProcConfig$initializer$   10025744     alm_process.obj
 0002:00001748       _acqEditor$initializer$    10025748     cProc_dialog.obj
 0002:0000174c       ?procList$initializer$@cProcess@@2P6AXXZA 1002574c     cProcess.obj
 0002:00001750       ?sm_sPrefix$initializer$@template_dialog@@0P6AXXZA 10025750     template_dialogimpl.obj
 0002:00001754       ?sm_sSuffix$initializer$@template_dialog@@0P6AXXZA 10025754     template_dialogimpl.obj
 0002:00001758       _cleanUp_alm_process$initializer$ 10025758     moc_alm_process.obj
 0002:0000175c       _cleanUp_CheckContDialog$initializer$ 1002575c     moc_checkContDialogImpl.obj
 0002:00001760       _cleanUp_CheckContDialogBase$initializer$ 10025760     moc_checkcontributiondialog.obj
 0002:00001764       _cleanUp_cProc_dialog$initializer$ 10025764     moc_cProc_dialog.obj
 0002:00001768       _cleanUp_LatchAckDialogBase$initializer$ 10025768     moc_latchackdialog.obj
 0002:0000176c       _cleanUp_LatchAckDialog$initializer$ 1002576c     moc_latchackdialogimpl.obj
 0002:00001770       _cleanUp_multiInputBase$initializer$ 10025770     moc_multiinput.obj
 0002:00001774       _cleanUp_multiInput$initializer$ 10025774     moc_multiinputimpl.obj
 0002:00001778       _cleanUp_proc_config$initializer$ 10025778     moc_proc_config.obj
 0002:0000177c       _cleanUp_singleInputBase$initializer$ 1002577c     moc_singleinput.obj
 0002:00001780       _cleanUp_singleInput$initializer$ 10025780     moc_singleinputimpl.obj
 0002:00001784       _cleanUp_template_dialogBase$initializer$ 10025784     moc_template_dialog.obj
 0002:00001788       _cleanUp_template_dialog$initializer$ 10025788     moc_template_dialogimpl.obj
 0002:0000178c       _cleanUp_config_mb4$initializer$ 1002578c     cfg_widgets001:moc_config_mb4impl.obj
 0002:00001790       _cleanUp_cfg_ListView$initializer$ 10025790     cfg_widgets001:moc_cfg_ListView.obj
 0002:00001794       _cleanUp_cfg_Table$initializer$ 10025794     cfg_widgets001:moc_cfg_Table.obj
 0002:000017a0       _pcinit                    100257a0     MSVCRT:crtdll.obj
 0002:000017a4       _pinit                     100257a4     MSVCRT:atonexit.obj
 0002:00007d5c       ?slot_0@?3??staticMetaObject@alm_process@@SAPAVQMetaObject@@XZ@4UQUMethod@@B 1002bd5c     moc_alm_process.obj
 0002:00007d78       ?slot_1@?3??staticMetaObject@alm_process@@SAPAVQMetaObject@@XZ@4UQUMethod@@B 1002bd78     moc_alm_process.obj
 0002:00007d94       ?slot_2@?3??staticMetaObject@alm_process@@SAPAVQMetaObject@@XZ@4UQUMethod@@B 1002bd94     moc_alm_process.obj
 0002:00007dac       ?slot_3@?3??staticMetaObject@alm_process@@SAPAVQMetaObject@@XZ@4UQUMethod@@B 1002bdac     moc_alm_process.obj
 0002:00007dd4       ?slot_4@?3??staticMetaObject@alm_process@@SAPAVQMetaObject@@XZ@4UQUMethod@@B 1002bdd4     moc_alm_process.obj
 0002:00007dec       ?slot_5@?3??staticMetaObject@alm_process@@SAPAVQMetaObject@@XZ@4UQUMethod@@B 1002bdec     moc_alm_process.obj
 0002:00007e08       ?slot_6@?3??staticMetaObject@alm_process@@SAPAVQMetaObject@@XZ@4UQUMethod@@B 1002be08     moc_alm_process.obj
 0002:00007e28       ?slot_7@?3??staticMetaObject@alm_process@@SAPAVQMetaObject@@XZ@4UQUMethod@@B 1002be28     moc_alm_process.obj
 0002:00007e34       ?slot_8@?3??staticMetaObject@alm_process@@SAPAVQMetaObject@@XZ@4UQUMethod@@B 1002be34     moc_alm_process.obj
 0002:00007e40       ?slot_9@?3??staticMetaObject@alm_process@@SAPAVQMetaObject@@XZ@4UQUMethod@@B 1002be40     moc_alm_process.obj
 0002:00007e4c       ?slot_10@?3??staticMetaObject@alm_process@@SAPAVQMetaObject@@XZ@4UQUMethod@@B 1002be4c     moc_alm_process.obj
 0002:00007e58       ?slot_11@?3??staticMetaObject@alm_process@@SAPAVQMetaObject@@XZ@4UQUMethod@@B 1002be58     moc_alm_process.obj
 0002:00007e84       ?slot_12@?3??staticMetaObject@alm_process@@SAPAVQMetaObject@@XZ@4UQUMethod@@B 1002be84     moc_alm_process.obj
 0002:00007ea0       ?slot_13@?3??staticMetaObject@alm_process@@SAPAVQMetaObject@@XZ@4UQUMethod@@B 1002bea0     moc_alm_process.obj
 0002:00007ebc       ?slot_14@?3??staticMetaObject@alm_process@@SAPAVQMetaObject@@XZ@4UQUMethod@@B 1002bebc     moc_alm_process.obj
 0002:00007ed8       ?slot_15@?3??staticMetaObject@alm_process@@SAPAVQMetaObject@@XZ@4UQUMethod@@B 1002bed8     moc_alm_process.obj
 0002:00007ef4       ?slot_16@?3??staticMetaObject@alm_process@@SAPAVQMetaObject@@XZ@4UQUMethod@@B 1002bef4     moc_alm_process.obj
 0002:00007f0c       ?slot_17@?3??staticMetaObject@alm_process@@SAPAVQMetaObject@@XZ@4UQUMethod@@B 1002bf0c     moc_alm_process.obj
 0002:00007f2c       ?slot_18@?3??staticMetaObject@alm_process@@SAPAVQMetaObject@@XZ@4UQUMethod@@B 1002bf2c     moc_alm_process.obj
 0002:00007f48       ?slot_19@?3??staticMetaObject@alm_process@@SAPAVQMetaObject@@XZ@4UQUMethod@@B 1002bf48     moc_alm_process.obj
 0002:00007f64       ?slot_20@?3??staticMetaObject@alm_process@@SAPAVQMetaObject@@XZ@4UQUMethod@@B 1002bf64     moc_alm_process.obj
 0002:00007f7c       ?slot_21@?3??staticMetaObject@alm_process@@SAPAVQMetaObject@@XZ@4UQUMethod@@B 1002bf7c     moc_alm_process.obj
 0002:00007f90       ?slot_22@?3??staticMetaObject@alm_process@@SAPAVQMetaObject@@XZ@4UQUMethod@@B 1002bf90     moc_alm_process.obj
 0002:00007fa8       ?slot_23@?3??staticMetaObject@alm_process@@SAPAVQMetaObject@@XZ@4UQUMethod@@B 1002bfa8     moc_alm_process.obj
 0002:00007fe8       ?slot_24@?3??staticMetaObject@alm_process@@SAPAVQMetaObject@@XZ@4UQUMethod@@B 1002bfe8     moc_alm_process.obj
 0002:00008008       ?slot_25@?3??staticMetaObject@alm_process@@SAPAVQMetaObject@@XZ@4UQUMethod@@B 1002c008     moc_alm_process.obj
 0002:00008034       ?slot_26@?3??staticMetaObject@alm_process@@SAPAVQMetaObject@@XZ@4UQUMethod@@B 1002c034     moc_alm_process.obj
 0002:00008060       ?slot_27@?3??staticMetaObject@alm_process@@SAPAVQMetaObject@@XZ@4UQUMethod@@B 1002c060     moc_alm_process.obj
 0002:00008080       ?slot_28@?3??staticMetaObject@alm_process@@SAPAVQMetaObject@@XZ@4UQUMethod@@B 1002c080     moc_alm_process.obj
 0002:000080a0       ?slot_29@?3??staticMetaObject@alm_process@@SAPAVQMetaObject@@XZ@4UQUMethod@@B 1002c0a0     moc_alm_process.obj
 0002:000080ac       ?slot_30@?3??staticMetaObject@alm_process@@SAPAVQMetaObject@@XZ@4UQUMethod@@B 1002c0ac     moc_alm_process.obj
 0002:000080b8       ?slot_tbl@?3??staticMetaObject@alm_process@@SAPAVQMetaObject@@XZ@4QBUQMetaData@@B 1002c0b8     moc_alm_process.obj
 0002:000084e8       ?signal_0@?3??staticMetaObject@alm_process@@SAPAVQMetaObject@@XZ@4UQUMethod@@B 1002c4e8     moc_alm_process.obj
 0002:000084fc       ?signal_tbl@?3??staticMetaObject@alm_process@@SAPAVQMetaObject@@XZ@4QBUQMetaData@@B 1002c4fc     moc_alm_process.obj
 0002:00008534       ?slot_0@?3??staticMetaObject@CheckContDialog@@SAPAVQMetaObject@@XZ@4UQUMethod@@B 1002c534     moc_checkContDialogImpl.obj
 0002:00008548       ?slot_1@?3??staticMetaObject@CheckContDialog@@SAPAVQMetaObject@@XZ@4UQUMethod@@B 1002c548     moc_checkContDialogImpl.obj
 0002:00008568       ?slot_2@?3??staticMetaObject@CheckContDialog@@SAPAVQMetaObject@@XZ@4UQUMethod@@B 1002c568     moc_checkContDialogImpl.obj
 0002:0000858c       ?slot_tbl@?3??staticMetaObject@CheckContDialog@@SAPAVQMetaObject@@XZ@4QBUQMetaData@@B 1002c58c     moc_checkContDialogImpl.obj
 0002:000085ec       ?slot_0@?3??staticMetaObject@CheckContDialogBase@@SAPAVQMetaObject@@XZ@4UQUMethod@@B 1002c5ec     moc_checkcontributiondialog.obj
 0002:000085f8       ?slot_1@?3??staticMetaObject@CheckContDialogBase@@SAPAVQMetaObject@@XZ@4UQUMethod@@B 1002c5f8     moc_checkcontributiondialog.obj
 0002:00008604       ?slot_2@?3??staticMetaObject@CheckContDialogBase@@SAPAVQMetaObject@@XZ@4UQUMethod@@B 1002c604     moc_checkcontributiondialog.obj
 0002:00008620       ?slot_tbl@?3??staticMetaObject@CheckContDialogBase@@SAPAVQMetaObject@@XZ@4QBUQMetaData@@B 1002c620     moc_checkcontributiondialog.obj
 0002:00008668       ?slot_0@?3??staticMetaObject@cProc_dialog@@SAPAVQMetaObject@@XZ@4UQUMethod@@B 1002c668     moc_cProc_dialog.obj
 0002:00008680       ?slot_1@?3??staticMetaObject@cProc_dialog@@SAPAVQMetaObject@@XZ@4UQUMethod@@B 1002c680     moc_cProc_dialog.obj
 0002:00008694       ?slot_2@?3??staticMetaObject@cProc_dialog@@SAPAVQMetaObject@@XZ@4UQUMethod@@B 1002c694     moc_cProc_dialog.obj
 0002:000086a0       ?slot_3@?3??staticMetaObject@cProc_dialog@@SAPAVQMetaObject@@XZ@4UQUMethod@@B 1002c6a0     moc_cProc_dialog.obj
 0002:000086bc       ?slot_4@?3??staticMetaObject@cProc_dialog@@SAPAVQMetaObject@@XZ@4UQUMethod@@B 1002c6bc     moc_cProc_dialog.obj
 0002:000086e0       ?slot_5@?3??staticMetaObject@cProc_dialog@@SAPAVQMetaObject@@XZ@4UQUMethod@@B 1002c6e0     moc_cProc_dialog.obj
 0002:00008700       ?slot_6@?3??staticMetaObject@cProc_dialog@@SAPAVQMetaObject@@XZ@4UQUMethod@@B 1002c700     moc_cProc_dialog.obj
 0002:00008724       ?slot_7@?3??staticMetaObject@cProc_dialog@@SAPAVQMetaObject@@XZ@4UQUMethod@@B 1002c724     moc_cProc_dialog.obj
 0002:00008740       ?slot_8@?3??staticMetaObject@cProc_dialog@@SAPAVQMetaObject@@XZ@4UQUMethod@@B 1002c740     moc_cProc_dialog.obj
 0002:00008760       ?slot_9@?3??staticMetaObject@cProc_dialog@@SAPAVQMetaObject@@XZ@4UQUMethod@@B 1002c760     moc_cProc_dialog.obj
 0002:0000877c       ?slot_10@?3??staticMetaObject@cProc_dialog@@SAPAVQMetaObject@@XZ@4UQUMethod@@B 1002c77c     moc_cProc_dialog.obj
 0002:000087a8       ?slot_11@?3??staticMetaObject@cProc_dialog@@SAPAVQMetaObject@@XZ@4UQUMethod@@B 1002c7a8     moc_cProc_dialog.obj
 0002:000087cc       ?slot_12@?3??staticMetaObject@cProc_dialog@@SAPAVQMetaObject@@XZ@4UQUMethod@@B 1002c7cc     moc_cProc_dialog.obj
 0002:000087ec       ?slot_13@?3??staticMetaObject@cProc_dialog@@SAPAVQMetaObject@@XZ@4UQUMethod@@B 1002c7ec     moc_cProc_dialog.obj
 0002:0000880c       ?slot_14@?3??staticMetaObject@cProc_dialog@@SAPAVQMetaObject@@XZ@4UQUMethod@@B 1002c80c     moc_cProc_dialog.obj
 0002:00008828       ?slot_15@?3??staticMetaObject@cProc_dialog@@SAPAVQMetaObject@@XZ@4UQUMethod@@B 1002c828     moc_cProc_dialog.obj
 0002:00008844       ?slot_16@?3??staticMetaObject@cProc_dialog@@SAPAVQMetaObject@@XZ@4UQUMethod@@B 1002c844     moc_cProc_dialog.obj
 0002:00008854       ?slot_17@?3??staticMetaObject@cProc_dialog@@SAPAVQMetaObject@@XZ@4UQUMethod@@B 1002c854     moc_cProc_dialog.obj
 0002:00008860       ?slot_18@?3??staticMetaObject@cProc_dialog@@SAPAVQMetaObject@@XZ@4UQUMethod@@B 1002c860     moc_cProc_dialog.obj
 0002:00008880       ?slot_tbl@?3??staticMetaObject@cProc_dialog@@SAPAVQMetaObject@@XZ@4QBUQMetaData@@B 1002c880     moc_cProc_dialog.obj
 0002:00008b28       ?signal_0@?3??staticMetaObject@cProc_dialog@@SAPAVQMetaObject@@XZ@4UQUMethod@@B 1002cb28     moc_cProc_dialog.obj
 0002:00008b40       ?signal_1@?3??staticMetaObject@cProc_dialog@@SAPAVQMetaObject@@XZ@4UQUMethod@@B 1002cb40     moc_cProc_dialog.obj
 0002:00008b5c       ?signal_2@?3??staticMetaObject@cProc_dialog@@SAPAVQMetaObject@@XZ@4UQUMethod@@B 1002cb5c     moc_cProc_dialog.obj
 0002:00008b74       ?signal_3@?3??staticMetaObject@cProc_dialog@@SAPAVQMetaObject@@XZ@4UQUMethod@@B 1002cb74     moc_cProc_dialog.obj
 0002:00008b80       ?signal_4@?3??staticMetaObject@cProc_dialog@@SAPAVQMetaObject@@XZ@4UQUMethod@@B 1002cb80     moc_cProc_dialog.obj
 0002:00008b8c       ?signal_tbl@?3??staticMetaObject@cProc_dialog@@SAPAVQMetaObject@@XZ@4QBUQMetaData@@B 1002cb8c     moc_cProc_dialog.obj
 0002:00008c04       ?slot_0@?3??staticMetaObject@LatchAckDialogBase@@SAPAVQMetaObject@@XZ@4UQUMethod@@B 1002cc04     moc_latchackdialog.obj
 0002:00008c10       ?slot_tbl@?3??staticMetaObject@LatchAckDialogBase@@SAPAVQMetaObject@@XZ@4QBUQMetaData@@B 1002cc10     moc_latchackdialog.obj
 0002:00008c1c       ?slot_0@?3??staticMetaObject@multiInputBase@@SAPAVQMetaObject@@XZ@4UQUMethod@@B 1002cc1c     moc_multiinput.obj
 0002:00008c28       ?slot_tbl@?3??staticMetaObject@multiInputBase@@SAPAVQMetaObject@@XZ@4QBUQMetaData@@B 1002cc28     moc_multiinput.obj
 0002:00008c40       ?slot_0@?3??staticMetaObject@multiInput@@SAPAVQMetaObject@@XZ@4UQUMethod@@B 1002cc40     moc_multiinputimpl.obj
 0002:00008c5c       ?slot_1@?3??staticMetaObject@multiInput@@SAPAVQMetaObject@@XZ@4UQUMethod@@B 1002cc5c     moc_multiinputimpl.obj
 0002:00008c74       ?slot_2@?3??staticMetaObject@multiInput@@SAPAVQMetaObject@@XZ@4UQUMethod@@B 1002cc74     moc_multiinputimpl.obj
 0002:00008c90       ?slot_3@?3??staticMetaObject@multiInput@@SAPAVQMetaObject@@XZ@4UQUMethod@@B 1002cc90     moc_multiinputimpl.obj
 0002:00008c9c       ?slot_4@?3??staticMetaObject@multiInput@@SAPAVQMetaObject@@XZ@4UQUMethod@@B 1002cc9c     moc_multiinputimpl.obj
 0002:00008cb8       ?slot_5@?3??staticMetaObject@multiInput@@SAPAVQMetaObject@@XZ@4UQUMethod@@B 1002ccb8     moc_multiinputimpl.obj
 0002:00008cc4       ?slot_6@?3??staticMetaObject@multiInput@@SAPAVQMetaObject@@XZ@4UQUMethod@@B 1002ccc4     moc_multiinputimpl.obj
 0002:00008cd0       ?slot_tbl@?3??staticMetaObject@multiInput@@SAPAVQMetaObject@@XZ@4QBUQMetaData@@B 1002ccd0     moc_multiinputimpl.obj
 0002:00008db0       ?slot_0@?3??staticMetaObject@proc_config@@SAPAVQMetaObject@@XZ@4UQUMethod@@B 1002cdb0     moc_proc_config.obj
 0002:00008dbc       ?slot_tbl@?3??staticMetaObject@proc_config@@SAPAVQMetaObject@@XZ@4QBUQMetaData@@B 1002cdbc     moc_proc_config.obj
 0002:00008dc8       ?slot_0@?3??staticMetaObject@singleInputBase@@SAPAVQMetaObject@@XZ@4UQUMethod@@B 1002cdc8     moc_singleinput.obj
 0002:00008dd4       ?slot_tbl@?3??staticMetaObject@singleInputBase@@SAPAVQMetaObject@@XZ@4QBUQMetaData@@B 1002cdd4     moc_singleinput.obj
 0002:00008de0       ?slot_0@?3??staticMetaObject@singleInput@@SAPAVQMetaObject@@XZ@4UQUMethod@@B 1002cde0     moc_singleinputimpl.obj
 0002:00008dfc       ?slot_1@?3??staticMetaObject@singleInput@@SAPAVQMetaObject@@XZ@4UQUMethod@@B 1002cdfc     moc_singleinputimpl.obj
 0002:00008e08       ?slot_2@?3??staticMetaObject@singleInput@@SAPAVQMetaObject@@XZ@4UQUMethod@@B 1002ce08     moc_singleinputimpl.obj
 0002:00008e14       ?slot_tbl@?3??staticMetaObject@singleInput@@SAPAVQMetaObject@@XZ@4QBUQMetaData@@B 1002ce14     moc_singleinputimpl.obj
 0002:00008e58       ?slot_0@?3??staticMetaObject@template_dialogBase@@SAPAVQMetaObject@@XZ@4UQUMethod@@B 1002ce58     moc_template_dialog.obj
 0002:00008e64       ?slot_tbl@?3??staticMetaObject@template_dialogBase@@SAPAVQMetaObject@@XZ@4QBUQMetaData@@B 1002ce64     moc_template_dialog.obj
 0002:00008e80       ?slot_0@?3??staticMetaObject@template_dialog@@SAPAVQMetaObject@@XZ@4UQUMethod@@B 1002ce80     moc_template_dialogimpl.obj
 0002:00008ea8       ?slot_1@?3??staticMetaObject@template_dialog@@SAPAVQMetaObject@@XZ@4UQUMethod@@B 1002cea8     moc_template_dialogimpl.obj
 0002:00008ec0       ?slot_2@?3??staticMetaObject@template_dialog@@SAPAVQMetaObject@@XZ@4UQUMethod@@B 1002cec0     moc_template_dialogimpl.obj
 0002:00008ed8       ?slot_tbl@?3??staticMetaObject@template_dialog@@SAPAVQMetaObject@@XZ@4QBUQMetaData@@B 1002ced8     moc_template_dialogimpl.obj
 0002:0000c114       ?slot_0@?3??staticMetaObject@config_mb4@@SAPAVQMetaObject@@XZ@4UQUMethod@@B 10030114     cfg_widgets001:moc_config_mb4impl.obj
 0002:0000c130       ?slot_tbl@?3??staticMetaObject@config_mb4@@SAPAVQMetaObject@@XZ@4QBUQMetaData@@B 10030130     cfg_widgets001:moc_config_mb4impl.obj
 0002:0000c160       ?slot_0@?3??staticMetaObject@cfg_ListView@@SAPAVQMetaObject@@XZ@4UQUMethod@@B 10030160     cfg_widgets001:moc_cfg_ListView.obj
 0002:0000c178       ?slot_1@?3??staticMetaObject@cfg_ListView@@SAPAVQMetaObject@@XZ@4UQUMethod@@B 10030178     cfg_widgets001:moc_cfg_ListView.obj
 0002:0000c190       ?slot_2@?3??staticMetaObject@cfg_ListView@@SAPAVQMetaObject@@XZ@4UQUMethod@@B 10030190     cfg_widgets001:moc_cfg_ListView.obj
 0002:0000c1ac       ?slot_3@?3??staticMetaObject@cfg_ListView@@SAPAVQMetaObject@@XZ@4UQUMethod@@B 100301ac     cfg_widgets001:moc_cfg_ListView.obj
 0002:0000c1c4       ?slot_4@?3??staticMetaObject@cfg_ListView@@SAPAVQMetaObject@@XZ@4UQUMethod@@B 100301c4     cfg_widgets001:moc_cfg_ListView.obj
 0002:0000c1dc       ?slot_5@?3??staticMetaObject@cfg_ListView@@SAPAVQMetaObject@@XZ@4UQUMethod@@B 100301dc     cfg_widgets001:moc_cfg_ListView.obj
 0002:0000c200       ?slot_tbl@?3??staticMetaObject@cfg_ListView@@SAPAVQMetaObject@@XZ@4QBUQMetaData@@B 10030200     cfg_widgets001:moc_cfg_ListView.obj
 0002:0000c2b0       ?signal_0@?3??staticMetaObject@cfg_ListView@@SAPAVQMetaObject@@XZ@4UQUMethod@@B 100302b0     cfg_widgets001:moc_cfg_ListView.obj
 0002:0000c2c8       ?signal_1@?3??staticMetaObject@cfg_ListView@@SAPAVQMetaObject@@XZ@4UQUMethod@@B 100302c8     cfg_widgets001:moc_cfg_ListView.obj
 0002:0000c2e8       ?signal_tbl@?3??staticMetaObject@cfg_ListView@@SAPAVQMetaObject@@XZ@4QBUQMetaData@@B 100302e8     cfg_widgets001:moc_cfg_ListView.obj
 0002:0000c338       ?slot_0@?3??staticMetaObject@cfg_Table@@SAPAVQMetaObject@@XZ@4UQUMethod@@B 10030338     cfg_widgets001:moc_cfg_Table.obj
 0002:0000c344       ?slot_1@?3??staticMetaObject@cfg_Table@@SAPAVQMetaObject@@XZ@4UQUMethod@@B 10030344     cfg_widgets001:moc_cfg_Table.obj
 0002:0000c350       ?slot_2@?3??staticMetaObject@cfg_Table@@SAPAVQMetaObject@@XZ@4UQUMethod@@B 10030350     cfg_widgets001:moc_cfg_Table.obj
 0002:0000c35c       ?slot_3@?3??staticMetaObject@cfg_Table@@SAPAVQMetaObject@@XZ@4UQUMethod@@B 1003035c     cfg_widgets001:moc_cfg_Table.obj
 0002:0000c378       ?slot_4@?3??staticMetaObject@cfg_Table@@SAPAVQMetaObject@@XZ@4UQUMethod@@B 10030378     cfg_widgets001:moc_cfg_Table.obj
 0002:0000c384       ?slot_tbl@?3??staticMetaObject@cfg_Table@@SAPAVQMetaObject@@XZ@4QBUQMetaData@@B 10030384     cfg_widgets001:moc_cfg_Table.obj
 0002:0000c3d4       ?signal_0@?3??staticMetaObject@cfg_Table@@SAPAVQMetaObject@@XZ@4UQUMethod@@B 100303d4     cfg_widgets001:moc_cfg_Table.obj
 0002:0000c3e0       ?signal_1@?3??staticMetaObject@cfg_Table@@SAPAVQMetaObject@@XZ@4UQUMethod@@B 100303e0     cfg_widgets001:moc_cfg_Table.obj
 0002:0000c3ec       ?signal_tbl@?3??staticMetaObject@cfg_Table@@SAPAVQMetaObject@@XZ@4QBUQMetaData@@B 100303ec     cfg_widgets001:moc_cfg_Table.obj
 0002:0000c410       _GS_ExceptionPointers      10030410     MSVCRT:gs_report.obj
 0002:0000e358       __unwindtable$??1QDockWindowList@@UAE@XZ 10032358     alm_process.obj
 0002:0000e368       __ehfuncinfo$??1QDockWindowList@@UAE@XZ 10032368     alm_process.obj
 0002:0000e38c       __unwindtable$??1QPopupMenuList@@UAE@XZ 1003238c     alm_process.obj
 0002:0000e394       __ehfuncinfo$??1QPopupMenuList@@UAE@XZ 10032394     alm_process.obj
 0002:0000e3b8       __unwindtable$??0config_plugin_base@@QAE@ABVQString@@00@Z 100323b8     alm_process.obj
 0002:0000e3d8       __ehfuncinfo$??0config_plugin_base@@QAE@ABVQString@@00@Z 100323d8     alm_process.obj
 0002:0000e3fc       __unwindtable$??1config_plugin_base@@UAE@XZ 100323fc     alm_process.obj
 0002:0000e414       __ehfuncinfo$??1config_plugin_base@@UAE@XZ 10032414     alm_process.obj
 0002:0000e438       __unwindtable$?about@config_plugin_base@@UAE?AVQString@@XZ 10032438     alm_process.obj
 0002:0000e448       __ehfuncinfo$?about@config_plugin_base@@UAE?AVQString@@XZ 10032448     alm_process.obj
 0002:0000e46c       __ehfuncinfo$??0ProcessListViewItem@@QAE@PAVQListView@@PAVcProcess@@@Z 1003246c     alm_process.obj
 0002:0000e490       __unwindtable$??0ProcessListViewItem@@QAE@PAVQListView@@PAVcProcess@@@Z 10032490     alm_process.obj
 0002:0000e4d0       __unwindtable$?paintCell@MultiInputInvalidListViewItem@@EAEXPAVQPainter@@ABVQColorGroup@@HHH@Z 100324d0     alm_process.obj
 0002:0000e4d0       __unwindtable$?paintCell@ProcessListViewItem@@EAEXPAVQPainter@@ABVQColorGroup@@HHH@Z 100324d0     alm_process.obj
 0002:0000e4d8       __ehfuncinfo$?paintCell@MultiInputInvalidListViewItem@@EAEXPAVQPainter@@ABVQColorGroup@@HHH@Z 100324d8     alm_process.obj
 0002:0000e4d8       __ehfuncinfo$?paintCell@ProcessListViewItem@@EAEXPAVQPainter@@ABVQColorGroup@@HHH@Z 100324d8     alm_process.obj
 0002:0000e4fc       __ehfuncinfo$??0alm_process@@QAE@ABVQString@@00@Z 100324fc     alm_process.obj
 0002:0000e520       __unwindtable$??0alm_process@@QAE@ABVQString@@00@Z 10032520     alm_process.obj
 0002:0000ea10       __ehfuncinfo$??1alm_process@@UAE@XZ 10032a10     alm_process.obj
 0002:0000ea34       __unwindtable$??1alm_process@@UAE@XZ 10032a34     alm_process.obj
 0002:0000eabc       __unwindtable$?toolbars@alm_process@@UAE?AVQDockWindowList@@XZ 10032abc     alm_process.obj
 0002:0000eac4       __ehfuncinfo$?toolbars@alm_process@@UAE?AVQDockWindowList@@XZ 10032ac4     alm_process.obj
 0002:0000eae8       __unwindtable$?menus@alm_process@@UAE?AVQPopupMenuList@@XZ 10032ae8     alm_process.obj
 0002:0000eaf0       __ehfuncinfo$?menus@alm_process@@UAE?AVQPopupMenuList@@XZ 10032af0     alm_process.obj
 0002:0000eb14       __ehfuncinfo$?reply@alm_process@@UAEXPAVresponse@@@Z 10032b14     alm_process.obj
 0002:0000eb38       __unwindtable$?reply@alm_process@@UAEXPAVresponse@@@Z 10032b38     alm_process.obj
 0002:0000ecb8       __unwindtable$?navigate@alm_process@@UAEXABVQString@@0@Z 10032cb8     alm_process.obj
 0002:0000ecc8       __ehfuncinfo$?navigate@alm_process@@UAEXABVQString@@0@Z 10032cc8     alm_process.obj
 0002:0000ecec       __ehfuncinfo$?activate@alm_process@@UAEX_N@Z 10032cec     alm_process.obj
 0002:0000ed10       __unwindtable$?activate@alm_process@@UAEX_N@Z 10032d10     alm_process.obj
 0002:0000ed40       __unwindtable$?closeEvent@alm_process@@UAEXPAVQCloseEvent@@@Z 10032d40     alm_process.obj
 0002:0000ed48       __ehfuncinfo$?closeEvent@alm_process@@UAEXPAVQCloseEvent@@@Z 10032d48     alm_process.obj
 0002:0000ed6c       __ehfuncinfo$?copyProcessUsingTemplate@alm_process@@AAEXXZ 10032d6c     alm_process.obj
 0002:0000ed90       __unwindtable$?copyProcessUsingTemplate@alm_process@@AAEXXZ 10032d90     alm_process.obj
 0002:0000edb8       __ehfuncinfo$?deleteProcess@alm_process@@AAEXXZ 10032db8     alm_process.obj
 0002:0000eddc       __unwindtable$?deleteProcess@alm_process@@AAEXXZ 10032ddc     alm_process.obj
 0002:0000ee1c       __ehfuncinfo$?duplicateProcess@alm_process@@AAEXXZ 10032e1c     alm_process.obj
 0002:0000ee40       __unwindtable$?duplicateProcess@alm_process@@AAEXXZ 10032e40     alm_process.obj
 0002:0000ee98       __ehfuncinfo$?newGate@alm_process@@AAEXXZ 10032e98     alm_process.obj
 0002:0000eebc       __unwindtable$?newGate@alm_process@@AAEXXZ 10032ebc     alm_process.obj
 0002:0000ef8c       __ehfuncinfo$?deleteGroup@alm_process@@AAEXXZ 10032f8c     alm_process.obj
 0002:0000efb0       __unwindtable$?deleteGroup@alm_process@@AAEXXZ 10032fb0     alm_process.obj
 0002:0000efe0       __ehfuncinfo$?renameGroup@alm_process@@AAEXXZ 10032fe0     alm_process.obj
 0002:0000f004       __unwindtable$?renameGroup@alm_process@@AAEXXZ 10033004     alm_process.obj
 0002:0000f064       __ehfuncinfo$?newGroup@alm_process@@AAEXXZ 10033064     alm_process.obj
 0002:0000f088       __unwindtable$?newGroup@alm_process@@AAEXXZ 10033088     alm_process.obj
 0002:0000f0b0       __unwindtable$?newProcess@alm_process@@AAEXXZ 100330b0     alm_process.obj
 0002:0000f0d0       __ehfuncinfo$?newProcess@alm_process@@AAEXXZ 100330d0     alm_process.obj
 0002:0000f0f4       __unwindtable$?updateProcList@alm_process@@AAEXPAVcProcess@@@Z 100330f4     alm_process.obj
 0002:0000f0f4       __unwindtable$?setOldPrefix@template_dialog@@QAEXVQString@@@Z 100330f4     alm_process.obj
 0002:0000f0f4       __unwindtable$?setText@config_mb4@@QAEXVQString@@@Z 100330f4     alm_process.obj
 0002:0000f0fc       __ehfuncinfo$?setText@config_mb4@@QAEXVQString@@@Z 100330fc     alm_process.obj
 0002:0000f0fc       __ehfuncinfo$?setOldPrefix@template_dialog@@QAEXVQString@@@Z 100330fc     alm_process.obj
 0002:0000f0fc       __ehfuncinfo$?updateProcList@alm_process@@AAEXPAVcProcess@@@Z 100330fc     alm_process.obj
 0002:0000f120       __ehfuncinfo$?markDirty@alm_process@@AAEXXZ 10033120     alm_process.obj
 0002:0000f144       __unwindtable$?markDirty@alm_process@@AAEXXZ 10033144     alm_process.obj
 0002:0000f19c       __ehfuncinfo$?newProcess@alm_process@@AAEXVQString@@AAVQStringList@@@Z 1003319c     alm_process.obj
 0002:0000f1c0       __unwindtable$?newProcess@alm_process@@AAEXVQString@@AAVQStringList@@@Z 100331c0     alm_process.obj
 0002:0000f1e8       __ehfuncinfo$?saveProcesses@alm_process@@AAE_NVQString@@@Z 100331e8     alm_process.obj
 0002:0000f20c       __unwindtable$?saveProcesses@alm_process@@AAE_NVQString@@@Z 1003320c     alm_process.obj
 0002:0000f27c       __ehfuncinfo$?loadProcesses@alm_process@@AAE_NVQString@@@Z 1003327c     alm_process.obj
 0002:0000f2a0       __unwindtable$?loadProcesses@alm_process@@AAE_NVQString@@@Z 100332a0     alm_process.obj
 0002:0000f350       __ehfuncinfo$?selectProcess@alm_process@@AAEXPAVQListViewItem@@@Z 10033350     alm_process.obj
 0002:0000f374       __unwindtable$?selectProcess@alm_process@@AAEXPAVQListViewItem@@@Z 10033374     alm_process.obj
 0002:0000f4a4       __unwindtable$?about@alm_process@@EAE?AVQString@@XZ 100334a4     alm_process.obj
 0002:0000f4bc       __ehfuncinfo$?about@alm_process@@EAE?AVQString@@XZ 100334bc     alm_process.obj
 0002:0000f4e0       __ehfuncinfo$?apply@alm_process@@EAEXXZ 100334e0     alm_process.obj
 0002:0000f504       __unwindtable$?apply@alm_process@@EAEXXZ 10033504     alm_process.obj
 0002:0000f52c       __unwindtable$?checkReferences@alm_process@@AAEXXZ 1003352c     alm_process.obj
 0002:0000f53c       __ehfuncinfo$?checkReferences@alm_process@@AAEXXZ 1003353c     alm_process.obj
 0002:0000f560       __unwindtable$?sysCommand@alm_process@@AAEXABVQString@@0@Z 10033560     alm_process.obj
 0002:0000f568       __ehfuncinfo$?sysCommand@alm_process@@AAEXABVQString@@0@Z 10033568     alm_process.obj
 0002:0000f58c       __ehfuncinfo$?selectSystem@alm_process@@AAEXABVQString@@@Z 1003358c     alm_process.obj
 0002:0000f5b0       __unwindtable$?selectSystem@alm_process@@AAEXABVQString@@@Z 100335b0     alm_process.obj
 0002:0000f6e8       __ehfuncinfo$?setProcessGroup@alm_process@@AAEXXZ 100336e8     alm_process.obj
 0002:0000f70c       __unwindtable$?setProcessGroup@alm_process@@AAEXXZ 1003370c     alm_process.obj
 0002:0000f74c       __unwindtable$?clearMask@alm_process@@AAEXXZ 1003374c     alm_process.obj
 0002:0000f76c       __ehfuncinfo$?clearMask@alm_process@@AAEXXZ 1003376c     alm_process.obj
 0002:0000f790       __ehfuncinfo$?setMask@alm_process@@AAEXXZ 10033790     alm_process.obj
 0002:0000f7b4       __unwindtable$?setMask@alm_process@@AAEXXZ 100337b4     alm_process.obj
 0002:0000f7dc       __unwindtable$?setLatchAck@alm_process@@AAEXXZ 100337dc     alm_process.obj
 0002:0000f7fc       __ehfuncinfo$?setLatchAck@alm_process@@AAEXXZ 100337fc     alm_process.obj
 0002:0000f820       __ehfuncinfo$?renameProcess@alm_process@@AAEXPAVQListViewItem@@HABVQString@@@Z 10033820     alm_process.obj
 0002:0000f844       __unwindtable$?renameProcess@alm_process@@AAEXPAVQListViewItem@@HABVQString@@@Z 10033844     alm_process.obj
 0002:0000f87c       __ehfuncinfo$?navToOutput@alm_process@@AAEXVQString@@0@Z 1003387c     alm_process.obj
 0002:0000f8a0       __unwindtable$?navToOutput@alm_process@@AAEXVQString@@0@Z 100338a0     alm_process.obj
 0002:0000f8d8       __ehfuncinfo$?navToAck@alm_process@@AAEXVQString@@00@Z 100338d8     alm_process.obj
 0002:0000f8fc       __unwindtable$?navToAck@alm_process@@AAEXVQString@@00@Z 100338fc     alm_process.obj
 0002:0000f934       __unwindtable$?selectProcess@alm_process@@AAEXVQString@@@Z 10033934     alm_process.obj
 0002:0000f94c       __ehfuncinfo$?selectProcess@alm_process@@AAEXVQString@@@Z 1003394c     alm_process.obj
 0002:0000f970       __ehfuncinfo$?checkProcessContributors@alm_process@@AAEXXZ 10033970     alm_process.obj
 0002:0000f994       __unwindtable$?checkProcessContributors@alm_process@@AAEXXZ 10033994     alm_process.obj
 0002:0000fafc       __unwindtable$??1?$QPtrList@VQListViewItem@@@@UAE@XZ 10033afc     alm_process.obj
 0002:0000fafc       __unwindtable$??1?$QPtrList@VQPopupMenu@@@@UAE@XZ 10033afc     alm_process.obj
 0002:0000fafc       __unwindtable$??1?$QPtrList@VcProcess@@@@UAE@XZ 10033afc     alm_process.obj
 0002:0000fb04       __ehfuncinfo$??1?$QPtrList@VQPopupMenu@@@@UAE@XZ 10033b04     alm_process.obj
 0002:0000fb04       __ehfuncinfo$??1?$QPtrList@VcProcess@@@@UAE@XZ 10033b04     alm_process.obj
 0002:0000fb04       __ehfuncinfo$??1?$QPtrList@VQListViewItem@@@@UAE@XZ 10033b04     alm_process.obj
 0002:0000fb28       __catchsym$??$_Buynode@U?$pair@VQString@@PAVcProcess@@@std@@@?$_Tree_buy@U?$pair@$$CBVQString@@PAVcProcess@@@std@@V?$allocator@U?$pair@$$CBVQString@@PAVcProcess@@@std@@@2@@std@@QAEPAU?$_Tree_node@U?$pair@$$CBVQString@@PAVcProcess@@@std@@PAX@1@$$QAU?$pair@VQString@@PAVcProcess@@@1@@Z$2 10033b28     alm_process.obj
 0002:0000fb38       __unwindtable$??$_Buynode@U?$pair@VQString@@PAVcProcess@@@std@@@?$_Tree_buy@U?$pair@$$CBVQString@@PAVcProcess@@@std@@V?$allocator@U?$pair@$$CBVQString@@PAVcProcess@@@std@@@2@@std@@QAEPAU?$_Tree_node@U?$pair@$$CBVQString@@PAVcProcess@@@std@@PAX@1@$$QAU?$pair@VQString@@PAVcProcess@@@1@@Z 10033b38     alm_process.obj
 0002:0000fb48       __tryblocktable$??$_Buynode@U?$pair@VQString@@PAVcProcess@@@std@@@?$_Tree_buy@U?$pair@$$CBVQString@@PAVcProcess@@@std@@V?$allocator@U?$pair@$$CBVQString@@PAVcProcess@@@std@@@2@@std@@QAEPAU?$_Tree_node@U?$pair@$$CBVQString@@PAVcProcess@@@std@@PAX@1@$$QAU?$pair@VQString@@PAVcProcess@@@1@@Z 10033b48     alm_process.obj
 0002:0000fb5c       __ehfuncinfo$??$_Buynode@U?$pair@VQString@@PAVcProcess@@@std@@@?$_Tree_buy@U?$pair@$$CBVQString@@PAVcProcess@@@std@@V?$allocator@U?$pair@$$CBVQString@@PAVcProcess@@@std@@@2@@std@@QAEPAU?$_Tree_node@U?$pair@$$CBVQString@@PAVcProcess@@@std@@PAX@1@$$QAU?$pair@VQString@@PAVcProcess@@@1@@Z 10033b5c     alm_process.obj
 0002:0000fb80       __catchsym$??$_Insert_nohint@AAU?$pair@$$CBVQString@@PAVcProcess@@@std@@PAU?$_Tree_node@U?$pair@$$CBVQString@@PAVcProcess@@@std@@PAX@2@@?$_Tree@V?$_Tmap_traits@VQString@@PAVcProcess@@U?$less@VQString@@@std@@V?$allocator@U?$pair@$$CBVQString@@PAVcProcess@@@std@@@4@$0A@@std@@@std@@IAE?AU?$pair@V?$_Tree_iterator@V?$_Tree_val@U?$_Tree_simple_types@U?$pair@$$CBVQString@@PAVcProcess@@@std@@@std@@@std@@@std@@_N@1@_NAAU?$pair@$$CBVQString@@PAVcProcess@@@1@PAU?$_Tree_node@U?$pair@$$CBVQString@@PAVcProcess@@@std@@PAX@1@@Z$4 10033b80     alm_process.obj
 0002:0000fb90       __unwindtable$??$_Insert_nohint@AAU?$pair@$$CBVQString@@PAVcProcess@@@std@@PAU?$_Tree_node@U?$pair@$$CBVQString@@PAVcProcess@@@std@@PAX@2@@?$_Tree@V?$_Tmap_traits@VQString@@PAVcProcess@@U?$less@VQString@@@std@@V?$allocator@U?$pair@$$CBVQString@@PAVcProcess@@@std@@@4@$0A@@std@@@std@@IAE?AU?$pair@V?$_Tree_iterator@V?$_Tree_val@U?$_Tree_simple_types@U?$pair@$$CBVQString@@PAVcProcess@@@std@@@std@@@std@@@std@@_N@1@_NAAU?$pair@$$CBVQString@@PAVcProcess@@@1@PAU?$_Tree_node@U?$pair@$$CBVQString@@PAVcProcess@@@std@@PAX@1@@Z 10033b90     alm_process.obj
 0002:0000fba0       __tryblocktable$??$_Insert_nohint@AAU?$pair@$$CBVQString@@PAVcProcess@@@std@@PAU?$_Tree_node@U?$pair@$$CBVQString@@PAVcProcess@@@std@@PAX@2@@?$_Tree@V?$_Tmap_traits@VQString@@PAVcProcess@@U?$less@VQString@@@std@@V?$allocator@U?$pair@$$CBVQString@@PAVcProcess@@@std@@@4@$0A@@std@@@std@@IAE?AU?$pair@V?$_Tree_iterator@V?$_Tree_val@U?$_Tree_simple_types@U?$pair@$$CBVQString@@PAVcProcess@@@std@@@std@@@std@@@std@@_N@1@_NAAU?$pair@$$CBVQString@@PAVcProcess@@@1@PAU?$_Tree_node@U?$pair@$$CBVQString@@PAVcProcess@@@std@@PAX@1@@Z 10033ba0     alm_process.obj
 0002:0000fbb4       __ehfuncinfo$??$_Insert_nohint@AAU?$pair@$$CBVQString@@PAVcProcess@@@std@@PAU?$_Tree_node@U?$pair@$$CBVQString@@PAVcProcess@@@std@@PAX@2@@?$_Tree@V?$_Tmap_traits@VQString@@PAVcProcess@@U?$less@VQString@@@std@@V?$allocator@U?$pair@$$CBVQString@@PAVcProcess@@@std@@@4@$0A@@std@@@std@@IAE?AU?$pair@V?$_Tree_iterator@V?$_Tree_val@U?$_Tree_simple_types@U?$pair@$$CBVQString@@PAVcProcess@@@std@@@std@@@std@@@std@@_N@1@_NAAU?$pair@$$CBVQString@@PAVcProcess@@@1@PAU?$_Tree_node@U?$pair@$$CBVQString@@PAVcProcess@@@std@@PAX@1@@Z 10033bb4     alm_process.obj
 0002:0000fbd8       __catchsym$??$_Insert_hint@AAU?$pair@$$CBVQString@@PAVcProcess@@@std@@PAU?$_Tree_node@U?$pair@$$CBVQString@@PAVcProcess@@@std@@PAX@2@@?$_Tree@V?$_Tmap_traits@VQString@@PAVcProcess@@U?$less@VQString@@@std@@V?$allocator@U?$pair@$$CBVQString@@PAVcProcess@@@std@@@4@$0A@@std@@@std@@IAE?AV?$_Tree_iterator@V?$_Tree_val@U?$_Tree_simple_types@U?$pair@$$CBVQString@@PAVcProcess@@@std@@@std@@@std@@@1@V?$_Tree_const_iterator@V?$_Tree_val@U?$_Tree_simple_types@U?$pair@$$CBVQString@@PAVcProcess@@@std@@@std@@@std@@@1@AAU?$pair@$$CBVQString@@PAVcProcess@@@1@PAU?$_Tree_node@U?$pair@$$CBVQString@@PAVcProcess@@@std@@PAX@1@@Z$3 10033bd8     alm_process.obj
 0002:0000fbe8       __unwindtable$??$_Insert_hint@AAU?$pair@$$CBVQString@@PAVcProcess@@@std@@PAU?$_Tree_node@U?$pair@$$CBVQString@@PAVcProcess@@@std@@PAX@2@@?$_Tree@V?$_Tmap_traits@VQString@@PAVcProcess@@U?$less@VQString@@@std@@V?$allocator@U?$pair@$$CBVQString@@PAVcProcess@@@std@@@4@$0A@@std@@@std@@IAE?AV?$_Tree_iterator@V?$_Tree_val@U?$_Tree_simple_types@U?$pair@$$CBVQString@@PAVcProcess@@@std@@@std@@@std@@@1@V?$_Tree_const_iterator@V?$_Tree_val@U?$_Tree_simple_types@U?$pair@$$CBVQString@@PAVcProcess@@@std@@@std@@@std@@@1@AAU?$pair@$$CBVQString@@PAVcProcess@@@1@PAU?$_Tree_node@U?$pair@$$CBVQString@@PAVcProcess@@@std@@PAX@1@@Z 10033be8     alm_process.obj
 0002:0000fbf8       __tryblocktable$??$_Insert_hint@AAU?$pair@$$CBVQString@@PAVcProcess@@@std@@PAU?$_Tree_node@U?$pair@$$CBVQString@@PAVcProcess@@@std@@PAX@2@@?$_Tree@V?$_Tmap_traits@VQString@@PAVcProcess@@U?$less@VQString@@@std@@V?$allocator@U?$pair@$$CBVQString@@PAVcProcess@@@std@@@4@$0A@@std@@@std@@IAE?AV?$_Tree_iterator@V?$_Tree_val@U?$_Tree_simple_types@U?$pair@$$CBVQString@@PAVcProcess@@@std@@@std@@@std@@@1@V?$_Tree_const_iterator@V?$_Tree_val@U?$_Tree_simple_types@U?$pair@$$CBVQString@@PAVcProcess@@@std@@@std@@@std@@@1@AAU?$pair@$$CBVQString@@PAVcProcess@@@1@PAU?$_Tree_node@U?$pair@$$CBVQString@@PAVcProcess@@@std@@PAX@1@@Z 10033bf8     alm_process.obj
 0002:0000fc0c       __ehfuncinfo$??$_Insert_hint@AAU?$pair@$$CBVQString@@PAVcProcess@@@std@@PAU?$_Tree_node@U?$pair@$$CBVQString@@PAVcProcess@@@std@@PAX@2@@?$_Tree@V?$_Tmap_traits@VQString@@PAVcProcess@@U?$less@VQString@@@std@@V?$allocator@U?$pair@$$CBVQString@@PAVcProcess@@@std@@@4@$0A@@std@@@std@@IAE?AV?$_Tree_iterator@V?$_Tree_val@U?$_Tree_simple_types@U?$pair@$$CBVQString@@PAVcProcess@@@std@@@std@@@std@@@1@V?$_Tree_const_iterator@V?$_Tree_val@U?$_Tree_simple_types@U?$pair@$$CBVQString@@PAVcProcess@@@std@@@std@@@std@@@1@AAU?$pair@$$CBVQString@@PAVcProcess@@@1@PAU?$_Tree_node@U?$pair@$$CBVQString@@PAVcProcess@@@std@@PAX@1@@Z 10033c0c     alm_process.obj
 0002:0000fc30       __catchsym$??$_Buynode@ABUpiecewise_construct_t@std@@V?$tuple@$$QAVQString@@@2@V?$tuple@$$$V@2@@?$_Tree_buy@U?$pair@$$CBVQString@@PAVcProcess@@@std@@V?$allocator@U?$pair@$$CBVQString@@PAVcProcess@@@std@@@2@@std@@QAEPAU?$_Tree_node@U?$pair@$$CBVQString@@PAVcProcess@@@std@@PAX@1@ABUpiecewise_construct_t@1@$$QAV?$tuple@$$QAVQString@@@1@$$QAV?$tuple@$$$V@1@@Z$2 10033c30     alm_process.obj
 0002:0000fc30       __catchsym$??$_Buynode@ABUpiecewise_construct_t@std@@V?$tuple@ABVQString@@@2@V?$tuple@$$$V@2@@?$_Tree_buy@U?$pair@$$CBVQString@@PAVcProcess@@@std@@V?$allocator@U?$pair@$$CBVQString@@PAVcProcess@@@std@@@2@@std@@QAEPAU?$_Tree_node@U?$pair@$$CBVQString@@PAVcProcess@@@std@@PAX@1@ABUpiecewise_construct_t@1@$$QAV?$tuple@ABVQString@@@1@$$QAV?$tuple@$$$V@1@@Z$2 10033c30     alm_process.obj
 0002:0000fc40       __unwindtable$??$_Buynode@ABUpiecewise_construct_t@std@@V?$tuple@$$QAVQString@@@2@V?$tuple@$$$V@2@@?$_Tree_buy@U?$pair@$$CBVQString@@PAVcProcess@@@std@@V?$allocator@U?$pair@$$CBVQString@@PAVcProcess@@@std@@@2@@std@@QAEPAU?$_Tree_node@U?$pair@$$CBVQString@@PAVcProcess@@@std@@PAX@1@ABUpiecewise_construct_t@1@$$QAV?$tuple@$$QAVQString@@@1@$$QAV?$tuple@$$$V@1@@Z 10033c40     alm_process.obj
 0002:0000fc40       __unwindtable$??$_Buynode@ABUpiecewise_construct_t@std@@V?$tuple@ABVQString@@@2@V?$tuple@$$$V@2@@?$_Tree_buy@U?$pair@$$CBVQString@@PAVcProcess@@@std@@V?$allocator@U?$pair@$$CBVQString@@PAVcProcess@@@std@@@2@@std@@QAEPAU?$_Tree_node@U?$pair@$$CBVQString@@PAVcProcess@@@std@@PAX@1@ABUpiecewise_construct_t@1@$$QAV?$tuple@ABVQString@@@1@$$QAV?$tuple@$$$V@1@@Z 10033c40     alm_process.obj
 0002:0000fc50       __tryblocktable$??$_Buynode@ABUpiecewise_construct_t@std@@V?$tuple@ABVQString@@@2@V?$tuple@$$$V@2@@?$_Tree_buy@U?$pair@$$CBVQString@@PAVcProcess@@@std@@V?$allocator@U?$pair@$$CBVQString@@PAVcProcess@@@std@@@2@@std@@QAEPAU?$_Tree_node@U?$pair@$$CBVQString@@PAVcProcess@@@std@@PAX@1@ABUpiecewise_construct_t@1@$$QAV?$tuple@ABVQString@@@1@$$QAV?$tuple@$$$V@1@@Z 10033c50     alm_process.obj
 0002:0000fc50       __tryblocktable$??$_Buynode@ABUpiecewise_construct_t@std@@V?$tuple@$$QAVQString@@@2@V?$tuple@$$$V@2@@?$_Tree_buy@U?$pair@$$CBVQString@@PAVcProcess@@@std@@V?$allocator@U?$pair@$$CBVQString@@PAVcProcess@@@std@@@2@@std@@QAEPAU?$_Tree_node@U?$pair@$$CBVQString@@PAVcProcess@@@std@@PAX@1@ABUpiecewise_construct_t@1@$$QAV?$tuple@$$QAVQString@@@1@$$QAV?$tuple@$$$V@1@@Z 10033c50     alm_process.obj
 0002:0000fc64       __ehfuncinfo$??$_Buynode@ABUpiecewise_construct_t@std@@V?$tuple@$$QAVQString@@@2@V?$tuple@$$$V@2@@?$_Tree_buy@U?$pair@$$CBVQString@@PAVcProcess@@@std@@V?$allocator@U?$pair@$$CBVQString@@PAVcProcess@@@std@@@2@@std@@QAEPAU?$_Tree_node@U?$pair@$$CBVQString@@PAVcProcess@@@std@@PAX@1@ABUpiecewise_construct_t@1@$$QAV?$tuple@$$QAVQString@@@1@$$QAV?$tuple@$$$V@1@@Z 10033c64     alm_process.obj
 0002:0000fc64       __ehfuncinfo$??$_Buynode@ABUpiecewise_construct_t@std@@V?$tuple@ABVQString@@@2@V?$tuple@$$$V@2@@?$_Tree_buy@U?$pair@$$CBVQString@@PAVcProcess@@@std@@V?$allocator@U?$pair@$$CBVQString@@PAVcProcess@@@std@@@2@@std@@QAEPAU?$_Tree_node@U?$pair@$$CBVQString@@PAVcProcess@@@std@@PAX@1@ABUpiecewise_construct_t@1@$$QAV?$tuple@ABVQString@@@1@$$QAV?$tuple@$$$V@1@@Z 10033c64     alm_process.obj
 0002:0000fc88       __unwindtable$??$construct@U?$pair@$$CBVQString@@PAVcProcess@@@std@@ABUpiecewise_construct_t@2@V?$tuple@ABVQString@@@2@V?$tuple@$$$V@2@@?$allocator@U?$_Tree_node@U?$pair@$$CBVQString@@PAVcProcess@@@std@@PAX@std@@@std@@QAEXPAU?$pair@$$CBVQString@@PAVcProcess@@@1@ABUpiecewise_construct_t@1@$$QAV?$tuple@ABVQString@@@1@$$QAV?$tuple@$$$V@1@@Z 10033c88     alm_process.obj
 0002:0000fc88       __unwindtable$??$construct@U?$pair@$$CBVQString@@PAVcProcess@@@std@@ABUpiecewise_construct_t@2@V?$tuple@$$QAVQString@@@2@V?$tuple@$$$V@2@@?$allocator@U?$_Tree_node@U?$pair@$$CBVQString@@PAVcProcess@@@std@@PAX@std@@@std@@QAEXPAU?$pair@$$CBVQString@@PAVcProcess@@@1@ABUpiecewise_construct_t@1@$$QAV?$tuple@$$QAVQString@@@1@$$QAV?$tuple@$$$V@1@@Z 10033c88     alm_process.obj
 0002:0000fc88       __unwindtable$??$construct@U?$pair@$$CBVQString@@PAVcProcess@@@std@@U?$pair@VQString@@PAVcProcess@@@2@@?$allocator@U?$_Tree_node@U?$pair@$$CBVQString@@PAVcProcess@@@std@@PAX@std@@@std@@QAEXPAU?$pair@$$CBVQString@@PAVcProcess@@@1@$$QAU?$pair@VQString@@PAVcProcess@@@1@@Z 10033c88     alm_process.obj
 0002:0000fc90       __ehfuncinfo$??$construct@U?$pair@$$CBVQString@@PAVcProcess@@@std@@U?$pair@VQString@@PAVcProcess@@@2@@?$allocator@U?$_Tree_node@U?$pair@$$CBVQString@@PAVcProcess@@@std@@PAX@std@@@std@@QAEXPAU?$pair@$$CBVQString@@PAVcProcess@@@1@$$QAU?$pair@VQString@@PAVcProcess@@@1@@Z 10033c90     alm_process.obj
 0002:0000fc90       __ehfuncinfo$??$construct@U?$pair@$$CBVQString@@PAVcProcess@@@std@@ABUpiecewise_construct_t@2@V?$tuple@$$QAVQString@@@2@V?$tuple@$$$V@2@@?$allocator@U?$_Tree_node@U?$pair@$$CBVQString@@PAVcProcess@@@std@@PAX@std@@@std@@QAEXPAU?$pair@$$CBVQString@@PAVcProcess@@@1@ABUpiecewise_construct_t@1@$$QAV?$tuple@$$QAVQString@@@1@$$QAV?$tuple@$$$V@1@@Z 10033c90     alm_process.obj
 0002:0000fc90       __ehfuncinfo$??$construct@U?$pair@$$CBVQString@@PAVcProcess@@@std@@ABUpiecewise_construct_t@2@V?$tuple@ABVQString@@@2@V?$tuple@$$$V@2@@?$allocator@U?$_Tree_node@U?$pair@$$CBVQString@@PAVcProcess@@@std@@PAX@std@@@std@@QAEXPAU?$pair@$$CBVQString@@PAVcProcess@@@1@ABUpiecewise_construct_t@1@$$QAV?$tuple@ABVQString@@@1@$$QAV?$tuple@$$$V@1@@Z 10033c90     alm_process.obj
 0002:0000fcb4       __unwindtable$?setMask@cProc_dialog@@QAEXVQString@@@Z 10033cb4     cAcqFileData.obj
 0002:0000fcb4       __unwindtable$?findSlot@cAcqFileData@@QAEHVQString@@@Z 10033cb4     cAcqFileData.obj
 0002:0000fcbc       __ehfuncinfo$?setMask@cProc_dialog@@QAEXVQString@@@Z 10033cbc     cAcqFileData.obj
 0002:0000fcbc       __ehfuncinfo$?findSlot@cAcqFileData@@QAEHVQString@@@Z 10033cbc     cAcqFileData.obj
 0002:0000fce0       __unwindtable$?findSlot@cAcqFileData@@QAE?AVQString@@H@Z 10033ce0     cAcqFileData.obj
 0002:0000fcf0       __ehfuncinfo$?findSlot@cAcqFileData@@QAE?AVQString@@H@Z 10033cf0     cAcqFileData.obj
 0002:0000fd14       __ehfuncinfo$?loadDetails@cAcqFileData@@QAE_NXZ 10033d14     cAcqFileData.obj
 0002:0000fd38       __unwindtable$?loadDetails@cAcqFileData@@QAE_NXZ 10033d38     cAcqFileData.obj
 0002:0000fdc0       __ehfuncinfo$??0cAcqFileData@@QAE@VQString@@@Z 10033dc0     cAcqFileData.obj
 0002:0000fde4       __unwindtable$??0cAcqFileData@@QAE@VQString@@@Z 10033de4     cAcqFileData.obj
 0002:0000fe1c       __ehfuncinfo$??1cAcqFileData@@UAE@XZ 10033e1c     cAcqFileData.obj
 0002:0000fe40       __unwindtable$??1cAcqFileData@@UAE@XZ 10033e40     cAcqFileData.obj
 0002:0000fe68       __unwindtable$?accept@CheckContDialog@@UAEXXZ 10033e68     checkContDialogImpl.obj
 0002:0000fe78       __ehfuncinfo$?accept@CheckContDialog@@UAEXXZ 10033e78     checkContDialogImpl.obj
 0002:0000fe9c       __ehfuncinfo$??0cProc_dialog@@QAE@QAVQStringList@@PAVQWidget@@PBDI@Z 10033e9c     cProc_dialog.obj
 0002:0000fec0       __unwindtable$??0cProc_dialog@@QAE@QAVQStringList@@PAVQWidget@@PBDI@Z 10033ec0     cProc_dialog.obj
 0002:0000ff20       __ehfuncinfo$??1cProc_dialog@@UAE@XZ 10033f20     cProc_dialog.obj
 0002:0000ff44       __unwindtable$??1cProc_dialog@@UAE@XZ 10033f44     cProc_dialog.obj
 0002:0000ff7c       __ehfuncinfo$?applyProc@cProc_dialog@@QAE_NXZ 10033f7c     cProc_dialog.obj
 0002:0000ffa0       __unwindtable$?applyProc@cProc_dialog@@QAE_NXZ 10033fa0     cProc_dialog.obj
 0002:00010028       __ehfuncinfo$?setProcess@cProc_dialog@@QAEXPAVcProcess@@_N@Z 10034028     cProc_dialog.obj
 0002:0001004c       __unwindtable$?setProcess@cProc_dialog@@QAEXPAVcProcess@@_N@Z 1003404c     cProc_dialog.obj
 0002:0001007c       __unwindtable$?reloadInputList@cProc_dialog@@QAEXXZ 1003407c     cProc_dialog.obj
 0002:0001009c       __ehfuncinfo$?reloadInputList@cProc_dialog@@QAEXXZ 1003409c     cProc_dialog.obj
 0002:000100c0       __unwindtable$?clear@cProc_dialog@@QAEX_N@Z 100340c0     cProc_dialog.obj
 0002:000100d8       __ehfuncinfo$?clear@cProc_dialog@@QAEX_N@Z 100340d8     cProc_dialog.obj
 0002:000100fc       __ehfuncinfo$?loadAcqFiles@cProc_dialog@@QAE_NVQString@@@Z 100340fc     cProc_dialog.obj
 0002:00010120       __unwindtable$?loadAcqFiles@cProc_dialog@@QAE_NVQString@@@Z 10034120     cProc_dialog.obj
 0002:000101a0       __ehfuncinfo$?loadOutputModules@cProc_dialog@@QAE_NVQString@@@Z 100341a0     cProc_dialog.obj
 0002:000101c4       __unwindtable$?loadOutputModules@cProc_dialog@@QAE_NVQString@@@Z 100341c4     cProc_dialog.obj
 0002:0001025c       __unwindtable$?editAcqSlot@cProc_dialog@@QAEXXZ 1003425c     cProc_dialog.obj
 0002:0001027c       __ehfuncinfo$?editAcqSlot@cProc_dialog@@QAEXXZ 1003427c     cProc_dialog.obj
 0002:000102a0       __unwindtable$?showTruth@cProc_dialog@@AAEXXZ 100342a0     cProc_dialog.obj
 0002:000102c0       __ehfuncinfo$?showTruth@cProc_dialog@@AAEXXZ 100342c0     cProc_dialog.obj
 0002:000102e4       __unwindtable$?showOr@cProc_dialog@@AAEXXZ 100342e4     cProc_dialog.obj
 0002:000102e4       __unwindtable$?showAnd@cProc_dialog@@AAEXXZ 100342e4     cProc_dialog.obj
 0002:000102ec       __ehfuncinfo$?showOr@cProc_dialog@@AAEXXZ 100342ec     cProc_dialog.obj
 0002:000102ec       __ehfuncinfo$?showAnd@cProc_dialog@@AAEXXZ 100342ec     cProc_dialog.obj
 0002:00010310       __ehfuncinfo$?showInput@cProc_dialog@@AAEXXZ 10034310     cProc_dialog.obj
 0002:00010334       __unwindtable$?showInput@cProc_dialog@@AAEXXZ 10034334     cProc_dialog.obj
 0002:0001035c       __unwindtable$?updateProcessCount@cProc_dialog@@QAEXH@Z 1003435c     cProc_dialog.obj
 0002:0001035c       __unwindtable$?changeHoldoff@cProc_dialog@@IAEXABVQString@@@Z 1003435c     cProc_dialog.obj
 0002:00010364       __ehfuncinfo$?updateProcessCount@cProc_dialog@@QAEXH@Z 10034364     cProc_dialog.obj
 0002:00010364       __ehfuncinfo$?changeHoldoff@cProc_dialog@@IAEXABVQString@@@Z 10034364     cProc_dialog.obj
 0002:00010388       __unwindtable$?navOutputModule@cProc_dialog@@IAEXXZ 10034388     cProc_dialog.obj
 0002:00010390       __ehfuncinfo$?navOutputModule@cProc_dialog@@IAEXXZ 10034390     cProc_dialog.obj
 0002:000103b4       __unwindtable$?changeFunction@cProc_dialog@@IAEXABVQString@@@Z 100343b4     cProc_dialog.obj
 0002:000103c4       __ehfuncinfo$?changeFunction@cProc_dialog@@IAEXABVQString@@@Z 100343c4     cProc_dialog.obj
 0002:000103e8       __unwindtable$?startTimeChanged@cProc_dialog@@IAEXABVQTime@@@Z 100343e8     cProc_dialog.obj
 0002:000103e8       __unwindtable$?endTimeChanged@cProc_dialog@@IAEXABVQTime@@@Z 100343e8     cProc_dialog.obj
 0002:000103f8       __ehfuncinfo$?startTimeChanged@cProc_dialog@@IAEXABVQTime@@@Z 100343f8     cProc_dialog.obj
 0002:000103f8       __ehfuncinfo$?endTimeChanged@cProc_dialog@@IAEXABVQTime@@@Z 100343f8     cProc_dialog.obj
 0002:0001041c       __unwindtable$?paint@ContributorListBoxItem@@EAEXPAVQPainter@@@Z 1003441c     cProc_dialog.obj
 0002:0001042c       __ehfuncinfo$?paint@ContributorListBoxItem@@EAEXPAVQPainter@@@Z 1003442c     cProc_dialog.obj
 0002:00010450       __ehfuncinfo$??0cProcess@@QAE@ABVQString@@@Z 10034450     cProcess.obj
 0002:00010450       __ehfuncinfo$??1cProcess@@UAE@XZ 10034450     cProcess.obj
 0002:00010474       __unwindtable$??0cProcess@@QAE@ABVQString@@@Z 10034474     cProcess.obj
 0002:00010474       __unwindtable$??1cProcess@@UAE@XZ 10034474     cProcess.obj
 0002:000104cc       __unwindtable$?setName@cProcess@@QAE_NABVQString@@@Z 100344cc     cProcess.obj
 0002:000104dc       __ehfuncinfo$?setName@cProcess@@QAE_NABVQString@@@Z 100344dc     cProcess.obj
 0002:00010500       __ehfuncinfo$?saveSettings@cProcess@@QAE?AVQStringList@@XZ 10034500     cProcess.obj
 0002:00010524       __unwindtable$?saveSettings@cProcess@@QAE?AVQStringList@@XZ 10034524     cProcess.obj
 0002:00010614       __ehfuncinfo$?LoadSettings@cProcess@@QAE_NABVQStringList@@@Z 10034614     cProcess.obj
 0002:00010638       __unwindtable$?LoadSettings@cProcess@@QAE_NABVQStringList@@@Z 10034638     cProcess.obj
 0002:00010790       __unwindtable$?inputSlotChange@cProc_dialog@@IAEXABVQString@@@Z 10034790     cProcess.obj
 0002:00010790       __unwindtable$?countProcessOutputs@cProcess@@SAXAAV?$map@VQString@@PAVcProcess@@U?$less@VQString@@@std@@V?$allocator@U?$pair@$$CBVQString@@PAVcProcess@@@std@@@4@@std@@@Z 10034790     cProcess.obj
 0002:00010798       __ehfuncinfo$?inputSlotChange@cProc_dialog@@IAEXABVQString@@@Z 10034798     cProcess.obj
 0002:00010798       __ehfuncinfo$?countProcessOutputs@cProcess@@SAXAAV?$map@VQString@@PAVcProcess@@U?$less@VQString@@@std@@V?$allocator@U?$pair@$$CBVQString@@PAVcProcess@@@std@@@4@@std@@@Z 10034798     cProcess.obj
 0002:000107bc       __unwindtable$?addEntry@cProcess@@AAEXAAVQStringList@@ABVQString@@1@Z 100347bc     cProcess.obj
 0002:000107cc       __ehfuncinfo$?addEntry@cProcess@@AAEXAAVQStringList@@ABVQString@@1@Z 100347cc     cProcess.obj
 0002:000107f0       __unwindtable$?LoadTruth@cProcess@@AAEHAAV?$QDict@VQString@@@@@Z 100347f0     cProcess.obj
 0002:00010810       __ehfuncinfo$?LoadTruth@cProcess@@AAEHAAV?$QDict@VQString@@@@@Z 10034810     cProcess.obj
 0002:00010834       __unwindtable$?FindEntry@cProcess@@AAE?AVQString@@AAV?$QDict@VQString@@@@ABV2@@Z 10034834     cProcess.obj
 0002:0001083c       __ehfuncinfo$?FindEntry@cProcess@@AAE?AVQString@@AAV?$QDict@VQString@@@@ABV2@@Z 1003483c     cProcess.obj
 0002:00010860       __ehfuncinfo$?Index@cProcess@@AAEXABVQStringList@@AAV?$QDict@VQString@@@@@Z 10034860     cProcess.obj
 0002:00010884       __unwindtable$?Index@cProcess@@AAEXABVQStringList@@AAV?$QDict@VQString@@@@@Z 10034884     cProcess.obj
 0002:000108ac       __unwindtable$?countOutputs@cProcess@@AAEXABV?$map@VQString@@PAVcProcess@@U?$less@VQString@@@std@@V?$allocator@U?$pair@$$CBVQString@@PAVcProcess@@@std@@@4@@std@@@Z 100348ac     cProcess.obj
 0002:000108bc       __ehfuncinfo$?countOutputs@cProcess@@AAEXABV?$map@VQString@@PAVcProcess@@U?$less@VQString@@@std@@V?$allocator@U?$pair@$$CBVQString@@PAVcProcess@@@std@@@4@@std@@@Z 100348bc     cProcess.obj
 0002:000108e0       __unwindtable$??1?$QDict@VQString@@@@UAE@XZ 100348e0     cProcess.obj
 0002:000108e8       __ehfuncinfo$??1?$QDict@VQString@@@@UAE@XZ 100348e8     cProcess.obj
 0002:0001090c       __ehfuncinfo$??0multiInputBase@@QAE@PAVQWidget@@PBD_NI@Z 1003490c     multiinput.obj
 0002:00010930       __unwindtable$??0multiInputBase@@QAE@PAVQWidget@@PBD_NI@Z 10034930     multiinput.obj
 0002:000109e0       __unwindtable$??0config_mb4@@QAE@IPAVQWidget@@PBD@Z 100349e0     multiinput.obj
 0002:000109e0       __unwindtable$??1multiInputBase@@UAE@XZ 100349e0     multiinput.obj
 0002:000109e8       __ehfuncinfo$??1multiInputBase@@UAE@XZ 100349e8     multiinput.obj
 0002:000109e8       __ehfuncinfo$??0config_mb4@@QAE@IPAVQWidget@@PBD@Z 100349e8     multiinput.obj
 0002:00010a0c       __ehfuncinfo$?languageChange@multiInputBase@@MAEXXZ 10034a0c     multiinput.obj
 0002:00010a30       __unwindtable$?languageChange@multiInputBase@@MAEXXZ 10034a30     multiinput.obj
 0002:00010ab0       __ehfuncinfo$??0MultiInputInvalidListViewItem@@QAE@PAVQListView@@ABVQString@@@Z 10034ab0     multiinputimpl.obj
 0002:00010ad4       __unwindtable$??0MultiInputInvalidListViewItem@@QAE@PAVQListView@@ABVQString@@@Z 10034ad4     multiinputimpl.obj
 0002:00010b0c       __ehfuncinfo$??0multiInput@@QAE@ABV?$map@VQString@@PAVcProcess@@U?$less@VQString@@@std@@V?$allocator@U?$pair@$$CBVQString@@PAVcProcess@@@std@@@4@@std@@QBVcProcess@@PAVQWidget@@PBD_NI@Z 10034b0c     multiinputimpl.obj
 0002:00010b30       __unwindtable$??0multiInput@@QAE@ABV?$map@VQString@@PAVcProcess@@U?$less@VQString@@@std@@V?$allocator@U?$pair@$$CBVQString@@PAVcProcess@@@std@@@4@@std@@QBVcProcess@@PAVQWidget@@PBD_NI@Z 10034b30     multiinputimpl.obj
 0002:00010be8       __ehfuncinfo$??1multiInput@@UAE@XZ 10034be8     multiinputimpl.obj
 0002:00010c0c       __unwindtable$??1multiInput@@UAE@XZ 10034c0c     multiinputimpl.obj
 0002:00010c44       __unwindtable$?changeInputs@singleInput@@QAE_NQAVcProcess@@@Z 10034c44     multiinputimpl.obj
 0002:00010c44       __unwindtable$?changeInputs@multiInput@@QAEXQAVcProcess@@@Z 10034c44     multiinputimpl.obj
 0002:00010c4c       __ehfuncinfo$?changeInputs@singleInput@@QAE_NQAVcProcess@@@Z 10034c4c     multiinputimpl.obj
 0002:00010c4c       __ehfuncinfo$?changeInputs@multiInput@@QAEXQAVcProcess@@@Z 10034c4c     multiinputimpl.obj
 0002:00010c70       __unwindtable$?countSelections@alm_process@@AAEHPAPAVQListViewItem@@@Z 10034c70     multiinputimpl.obj
 0002:00010c70       __unwindtable$?enableRemove@multiInput@@QAEXXZ 10034c70     multiinputimpl.obj
 0002:00010c70       __unwindtable$?displayEnd@ProcessListView@@AAEX_N@Z 10034c70     multiinputimpl.obj
 0002:00010c70       __unwindtable$?enableAdd@multiInput@@QAEXXZ 10034c70     multiinputimpl.obj
 0002:00010c70       __unwindtable$?removeProcesses@multiInput@@QAEXPAVQListViewItem@@@Z 10034c70     multiinputimpl.obj
 0002:00010c70       __unwindtable$?displayHome@ProcessListView@@AAEX_N@Z 10034c70     multiinputimpl.obj
 0002:00010c70       __unwindtable$?addProcesses@multiInput@@QAEXPAVQListViewItem@@@Z 10034c70     multiinputimpl.obj
 0002:00010c78       __ehfuncinfo$?addProcesses@multiInput@@QAEXPAVQListViewItem@@@Z 10034c78     multiinputimpl.obj
 0002:00010c78       __ehfuncinfo$?displayHome@ProcessListView@@AAEX_N@Z 10034c78     multiinputimpl.obj
 0002:00010c78       __ehfuncinfo$?displayEnd@ProcessListView@@AAEX_N@Z 10034c78     multiinputimpl.obj
 0002:00010c78       __ehfuncinfo$?enableAdd@multiInput@@QAEXXZ 10034c78     multiinputimpl.obj
 0002:00010c78       __ehfuncinfo$?enableRemove@multiInput@@QAEXXZ 10034c78     multiinputimpl.obj
 0002:00010c78       __ehfuncinfo$?countSelections@alm_process@@AAEHPAPAVQListViewItem@@@Z 10034c78     multiinputimpl.obj
 0002:00010c78       __ehfuncinfo$?removeProcesses@multiInput@@QAEXPAVQListViewItem@@@Z 10034c78     multiinputimpl.obj
 0002:00010c9c       __ehfuncinfo$?filterChange@multiInput@@QAEXABVQString@@@Z 10034c9c     multiinputimpl.obj
 0002:00010cc0       __unwindtable$?filterChange@multiInput@@QAEXABVQString@@@Z 10034cc0     multiinputimpl.obj
 0002:00010cf0       __unwindtable$?keys@plugindesc@@UAE?AVQStringList@@ABVQString@@0@Z 10034cf0     plugindesc.obj
 0002:00010d00       __ehfuncinfo$?keys@plugindesc@@UAE?AVQStringList@@ABVQString@@0@Z 10034d00     plugindesc.obj
 0002:00010d24       __ehfuncinfo$??0singleInputBase@@QAE@PAVQWidget@@PBD_NI@Z 10034d24     singleinput.obj
 0002:00010d48       __unwindtable$??0singleInputBase@@QAE@PAVQWidget@@PBD_NI@Z 10034d48     singleinput.obj
 0002:00010da8       __ehfuncinfo$?languageChange@singleInputBase@@MAEXXZ 10034da8     singleinput.obj
 0002:00010dcc       __unwindtable$?languageChange@singleInputBase@@MAEXXZ 10034dcc     singleinput.obj
 0002:00010e04       __ehfuncinfo$??0singleInput@@QAE@ABV?$map@VQString@@PAVcProcess@@U?$less@VQString@@@std@@V?$allocator@U?$pair@$$CBVQString@@PAVcProcess@@@std@@@4@@std@@QBVcProcess@@W4ESingleType@0@PAVQWidget@@PBD_NI@Z 10034e04     singleinputimpl.obj
 0002:00010e28       __unwindtable$??0singleInput@@QAE@ABV?$map@VQString@@PAVcProcess@@U?$less@VQString@@@std@@V?$allocator@U?$pair@$$CBVQString@@PAVcProcess@@@std@@@4@@std@@QBVcProcess@@W4ESingleType@0@PAVQWidget@@PBD_NI@Z 10034e28     singleinputimpl.obj
 0002:00010ed8       __unwindtable$?filterChange@singleInput@@AAEXABVQString@@@Z 10034ed8     singleinputimpl.obj
 0002:00010ed8       __unwindtable$?filterChange@alm_process@@AAEXABVQString@@@Z 10034ed8     singleinputimpl.obj
 0002:00010ef8       __ehfuncinfo$?filterChange@alm_process@@AAEXABVQString@@@Z 10034ef8     singleinputimpl.obj
 0002:00010ef8       __ehfuncinfo$?filterChange@singleInput@@AAEXABVQString@@@Z 10034ef8     singleinputimpl.obj
 0002:00010f1c       __ehfuncinfo$??0template_dialogBase@@QAE@PAVQWidget@@PBD_NI@Z 10034f1c     template_dialog.obj
 0002:00010f40       __unwindtable$??0template_dialogBase@@QAE@PAVQWidget@@PBD_NI@Z 10034f40     template_dialog.obj
 0002:00011040       __ehfuncinfo$?languageChange@template_dialogBase@@MAEXXZ 10035040     template_dialog.obj
 0002:00011064       __unwindtable$?languageChange@template_dialogBase@@MAEXXZ 10035064     template_dialog.obj
 0002:00011114       __unwindtable$??0template_dialog@@QAE@ABV?$QPtrList@VcProcess@@@@ABVQStringList@@PAVQWidget@@PBD_NI@Z 10035114     template_dialogimpl.obj
 0002:00011134       __ehfuncinfo$??0template_dialog@@QAE@ABV?$QPtrList@VcProcess@@@@ABVQStringList@@PAVQWidget@@PBD_NI@Z 10035134     template_dialogimpl.obj
 0002:00011158       __ehfuncinfo$?copyProcesses@template_dialog@@QAEXAAV?$QPtrList@VcProcess@@@@AAV?$map@VQString@@PAVcProcess@@U?$less@VQString@@@std@@V?$allocator@U?$pair@$$CBVQString@@PAVcProcess@@@std@@@4@@std@@PAVQListView@@@Z 10035158     template_dialogimpl.obj
 0002:0001117c       __unwindtable$?copyProcesses@template_dialog@@QAEXAAV?$QPtrList@VcProcess@@@@AAV?$map@VQString@@PAVcProcess@@U?$less@VQString@@@std@@V?$allocator@U?$pair@$$CBVQString@@PAVcProcess@@@std@@@4@@std@@PAVQListView@@@Z 1003517c     template_dialogimpl.obj
 0002:000111fc       __ehfuncinfo$?getThisPrefix@template_dialog@@QAE?AVQString@@H@Z 100351fc     template_dialogimpl.obj
 0002:00011220       __unwindtable$?getThisPrefix@template_dialog@@QAE?AVQString@@H@Z 10035220     template_dialogimpl.obj
 0002:00011250       __ehfuncinfo$?showExample@template_dialog@@QAEXXZ 10035250     template_dialogimpl.obj
 0002:00011274       __unwindtable$?showExample@template_dialog@@QAEXXZ 10035274     template_dialogimpl.obj
 0002:000112ac       __unwindtable$?setSelectionData@template_dialog@@AAEXHQBVcProcess@@@Z 100352ac     template_dialogimpl.obj
 0002:000112bc       __ehfuncinfo$?setSelectionData@template_dialog@@AAEXHQBVcProcess@@@Z 100352bc     template_dialogimpl.obj
 0002:000112e0       __ehfuncinfo$??0CheckContDialogBase@@QAE@PAVQWidget@@PBD_NI@Z 100352e0     checkcontributiondialog.obj
 0002:00011304       __unwindtable$??0CheckContDialogBase@@QAE@PAVQWidget@@PBD_NI@Z 10035304     checkcontributiondialog.obj
 0002:000113fc       __ehfuncinfo$?languageChange@CheckContDialogBase@@MAEXXZ 100353fc     checkcontributiondialog.obj
 0002:00011420       __unwindtable$?languageChange@CheckContDialogBase@@MAEXXZ 10035420     checkcontributiondialog.obj
 0002:000114a8       __ehfuncinfo$??0LatchAckDialogBase@@QAE@PAVQWidget@@PBD_NI@Z 100354a8     latchackdialog.obj
 0002:000114cc       __unwindtable$??0LatchAckDialogBase@@QAE@PAVQWidget@@PBD_NI@Z 100354cc     latchackdialog.obj
 0002:0001151c       __ehfuncinfo$?languageChange@LatchAckDialogBase@@MAEXXZ 1003551c     latchackdialog.obj
 0002:00011540       __unwindtable$?languageChange@LatchAckDialogBase@@MAEXXZ 10035540     latchackdialog.obj
 0002:00011590       __unwindtable$?qt_invoke@alm_process@@UAE_NHPAUQUObject@@@Z 10035590     moc_alm_process.obj
 0002:000115a8       __ehfuncinfo$?qt_invoke@alm_process@@UAE_NHPAUQUObject@@@Z 100355a8     moc_alm_process.obj
 0002:000115cc       __unwindtable$?qt_emit@alm_process@@UAE_NHPAUQUObject@@@Z 100355cc     moc_alm_process.obj
 0002:000115d4       __ehfuncinfo$?qt_emit@alm_process@@UAE_NHPAUQUObject@@@Z 100355d4     moc_alm_process.obj
 0002:000115f8       __unwindtable$?qt_emit@cProc_dialog@@UAE_NHPAUQUObject@@@Z 100355f8     moc_cProc_dialog.obj
 0002:00011610       __ehfuncinfo$?qt_emit@cProc_dialog@@UAE_NHPAUQUObject@@@Z 10035610     moc_cProc_dialog.obj
 0002:00011634       __unwindtable$?updateProc@cProc_dialog@@IAEXPAVcProcess@@@Z 10035634     moc_cProc_dialog.obj
 0002:0001163c       __ehfuncinfo$?updateProc@cProc_dialog@@IAEXPAVcProcess@@@Z 1003563c     moc_cProc_dialog.obj
 0002:00011660       __unwindtable$?navToProc@cProc_dialog@@IAEXVQString@@@Z 10035660     moc_cProc_dialog.obj
 0002:00011670       __ehfuncinfo$?navToProc@cProc_dialog@@IAEXVQString@@@Z 10035670     moc_cProc_dialog.obj
 0002:00011694       __unwindtable$?command@alm_process@@IAEXVQString@@0@Z 10035694     moc_cProc_dialog.obj
 0002:00011694       __unwindtable$?navToOutput@cProc_dialog@@IAEXVQString@@0@Z 10035694     moc_cProc_dialog.obj
 0002:000116ac       __ehfuncinfo$?command@alm_process@@IAEXVQString@@0@Z 100356ac     moc_cProc_dialog.obj
 0002:000116ac       __ehfuncinfo$?navToOutput@cProc_dialog@@IAEXVQString@@0@Z 100356ac     moc_cProc_dialog.obj
 0002:000116d0       __unwindtable$?navToAck@cProc_dialog@@IAEXVQString@@00@Z 100356d0     moc_cProc_dialog.obj
 0002:000116f0       __ehfuncinfo$?navToAck@cProc_dialog@@IAEXVQString@@00@Z 100356f0     moc_cProc_dialog.obj
 0002:00011714       __ehfuncinfo$??0proc_config@@QAE@PAVQWidget@@PBDI@Z 10035714     proc_config.obj
 0002:00011738       __unwindtable$??0proc_config@@QAE@PAVQWidget@@PBDI@Z 10035738     proc_config.obj
 0002:00011ae8       __unwindtable$??1proc_config@@UAE@XZ 10035ae8     proc_config.obj
 0002:00011af8       __ehfuncinfo$??1proc_config@@UAE@XZ 10035af8     proc_config.obj
 0002:00011b1c       __ehfuncinfo$?languageChange@proc_config@@MAEXXZ 10035b1c     proc_config.obj
 0002:00011b40       __unwindtable$?languageChange@proc_config@@MAEXXZ 10035b40     proc_config.obj
 0002:00011df8       __unwindtable$?setIcon@config_mb4@@QAEXW4Icon@1@@Z 10035df8     cfg_widgets001:config_mb4impl.obj
 0002:00011e18       __ehfuncinfo$?setIcon@config_mb4@@QAEXW4Icon@1@@Z 10035e18     cfg_widgets001:config_mb4impl.obj
 0002:00011e3c       __ehfuncinfo$?CreatePanel@config_mb4@@AAEXI@Z 10035e3c     cfg_widgets001:config_mb4impl.obj
 0002:00011e60       __unwindtable$?CreatePanel@config_mb4@@AAEXI@Z 10035e60     cfg_widgets001:config_mb4impl.obj
 0002:00011ee8       __unwindtable$?saveState@cfg_Settings@@SAXABVQString@@0@Z 10035ee8     cfg_widgets001:cfg_Settings.obj
 0002:00011f00       __ehfuncinfo$?saveState@cfg_Settings@@SAXABVQString@@0@Z 10035f00     cfg_widgets001:cfg_Settings.obj
 0002:00011f24       __ehfuncinfo$?saveState@cfg_Settings@@SAXQBVQListView@@ABVQString@@@Z 10035f24     cfg_widgets001:cfg_Settings.obj
 0002:00011f48       __unwindtable$?saveState@cfg_Settings@@SAXQBVQListView@@ABVQString@@@Z 10035f48     cfg_widgets001:cfg_Settings.obj
 0002:00011f70       __unwindtable$?saveState@cfg_Settings@@SAXQBVQSplitter@@ABVQString@@@Z 10035f70     cfg_widgets001:cfg_Settings.obj
 0002:00011f90       __ehfuncinfo$?saveState@cfg_Settings@@SAXQBVQSplitter@@ABVQString@@@Z 10035f90     cfg_widgets001:cfg_Settings.obj
 0002:00011fb4       __ehfuncinfo$?saveState@cfg_Settings@@SAXABVQPoint@@ABVQSize@@AB_NABVQString@@@Z 10035fb4     cfg_widgets001:cfg_Settings.obj
 0002:00011fd8       __unwindtable$?saveState@cfg_Settings@@SAXABVQPoint@@ABVQSize@@AB_NABVQString@@@Z 10035fd8     cfg_widgets001:cfg_Settings.obj
 0002:00012010       __unwindtable$?loadState@cfg_Settings@@SA?AVQString@@ABV2@@Z 10036010     cfg_widgets001:cfg_Settings.obj
 0002:00012030       __ehfuncinfo$?loadState@cfg_Settings@@SA?AVQString@@ABV2@@Z 10036030     cfg_widgets001:cfg_Settings.obj
 0002:00012054       __unwindtable$?loadState@cfg_Settings@@SAXQAVQListView@@ABVQString@@@Z 10036054     cfg_widgets001:cfg_Settings.obj
 0002:00012064       __ehfuncinfo$?loadState@cfg_Settings@@SAXQAVQListView@@ABVQString@@@Z 10036064     cfg_widgets001:cfg_Settings.obj
 0002:00012088       __unwindtable$?loadState@cfg_Settings@@SAXQAVQSplitter@@ABVQString@@@Z 10036088     cfg_widgets001:cfg_Settings.obj
 0002:000120a0       __ehfuncinfo$?loadState@cfg_Settings@@SAXQAVQSplitter@@ABVQString@@@Z 100360a0     cfg_widgets001:cfg_Settings.obj
 0002:000120c4       __unwindtable$?loadState@cfg_Settings@@SAXAAVQPoint@@AAVQSize@@AA_NABVQString@@@Z 100360c4     cfg_widgets001:cfg_Settings.obj
 0002:000120d4       __ehfuncinfo$?loadState@cfg_Settings@@SAXAAVQPoint@@AAVQSize@@AA_NABVQString@@@Z 100360d4     cfg_widgets001:cfg_Settings.obj
 0002:000120f8       __unwindtable$??0cfg_ListView@@QAE@PAVQWidget@@PBD@Z 100360f8     cfg_widgets001:cfg_ListView.obj
 0002:00012110       __ehfuncinfo$??0cfg_ListView@@QAE@PAVQWidget@@PBD@Z 10036110     cfg_widgets001:cfg_ListView.obj
 0002:00012134       __unwindtable$??0ProcessListView@@QAE@PAVQWidget@@PBDI@Z 10036134     cfg_widgets001:cfg_ListView.obj
 0002:00012134       __unwindtable$??1cfg_ListView@@UAE@XZ 10036134     cfg_widgets001:cfg_ListView.obj
 0002:0001213c       __ehfuncinfo$??1cfg_ListView@@UAE@XZ 1003613c     cfg_widgets001:cfg_ListView.obj
 0002:0001213c       __ehfuncinfo$??0ProcessListView@@QAE@PAVQWidget@@PBDI@Z 1003613c     cfg_widgets001:cfg_ListView.obj
 0002:00012160       __ehfuncinfo$?insertData@cfg_ListView@@QAEXXZ 10036160     cfg_widgets001:cfg_ListView.obj
 0002:00012184       __unwindtable$?insertData@cfg_ListView@@QAEXXZ 10036184     cfg_widgets001:cfg_ListView.obj
 0002:000121ac       __unwindtable$?deleteItems@cfg_ListView@@QAEXXZ 100361ac     cfg_widgets001:cfg_ListView.obj
 0002:000121bc       __ehfuncinfo$?deleteItems@cfg_ListView@@QAEXXZ 100361bc     cfg_widgets001:cfg_ListView.obj
 0002:000121e0       __unwindtable$?copyToClipboard@cfg_ListView@@QAEXXZ 100361e0     cfg_widgets001:cfg_ListView.obj
 0002:00012200       __ehfuncinfo$?copyToClipboard@cfg_ListView@@QAEXXZ 10036200     cfg_widgets001:cfg_ListView.obj
 0002:00012224       __ehfuncinfo$?replaceData@cfg_ListView@@QAEXXZ 10036224     cfg_widgets001:cfg_ListView.obj
 0002:00012248       __unwindtable$?replaceData@cfg_ListView@@QAEXXZ 10036248     cfg_widgets001:cfg_ListView.obj
 0002:00012280       __unwindtable$??0?$QMap@HPAVcAcqFileData@@@@QAE@XZ 10036280     cfg_widgets001:cfg_ListView.obj
 0002:00012280       __unwindtable$?create@plugindesc@@UAEPAVconfig_plugin_base@@ABVQString@@00@Z 10036280     cfg_widgets001:cfg_ListView.obj
 0002:00012280       __unwindtable$?addMultiInputs@alm_process@@AAEXXZ 10036280     cfg_widgets001:cfg_ListView.obj
 0002:00012280       __unwindtable$??4?$QGuardedPtr@VQPopupMenu@@@@QAEAAV0@PAVQPopupMenu@@@Z 10036280     cfg_widgets001:cfg_ListView.obj
 0002:00012280       __unwindtable$??0?$QGuardedPtr@VQDockWindow@@@@QAE@XZ 10036280     cfg_widgets001:cfg_ListView.obj
 0002:00012280       __unwindtable$?detachInternal@?$QMap@HPAVcAcqFileData@@@@AAEXXZ 10036280     cfg_widgets001:cfg_ListView.obj
 0002:00012280       __unwindtable$??0?$QGuardedPtr@VQPopupMenu@@@@QAE@XZ 10036280     cfg_widgets001:cfg_ListView.obj
 0002:00012280       __unwindtable$?newItem@cfg_ListView@@MAEPAVQListViewItem@@PAVQListView@@PAV2@@Z 10036280     cfg_widgets001:cfg_ListView.obj
 0002:00012280       __unwindtable$??4?$QGuardedPtr@VQDockWindow@@@@QAEAAV0@PAVQDockWindow@@@Z 10036280     cfg_widgets001:cfg_ListView.obj
 0002:00012280       __unwindtable$?addSingleInputs@alm_process@@AAEXXZ 10036280     cfg_widgets001:cfg_ListView.obj
 0002:00012280       __unwindtable$?changeMask@alm_process@@AAEXXZ 10036280     cfg_widgets001:cfg_ListView.obj
 0002:00012288       __ehfuncinfo$??0?$QMap@HPAVcAcqFileData@@@@QAE@XZ 10036288     cfg_widgets001:cfg_ListView.obj
 0002:00012288       __ehfuncinfo$??4?$QGuardedPtr@VQPopupMenu@@@@QAEAAV0@PAVQPopupMenu@@@Z 10036288     cfg_widgets001:cfg_ListView.obj
 0002:00012288       __ehfuncinfo$??4?$QGuardedPtr@VQDockWindow@@@@QAEAAV0@PAVQDockWindow@@@Z 10036288     cfg_widgets001:cfg_ListView.obj
 0002:00012288       __ehfuncinfo$?changeMask@alm_process@@AAEXXZ 10036288     cfg_widgets001:cfg_ListView.obj
 0002:00012288       __ehfuncinfo$?detachInternal@?$QMap@HPAVcAcqFileData@@@@AAEXXZ 10036288     cfg_widgets001:cfg_ListView.obj
 0002:00012288       __ehfuncinfo$?newItem@cfg_ListView@@MAEPAVQListViewItem@@PAVQListView@@PAV2@@Z 10036288     cfg_widgets001:cfg_ListView.obj
 0002:00012288       __ehfuncinfo$??0?$QGuardedPtr@VQPopupMenu@@@@QAE@XZ 10036288     cfg_widgets001:cfg_ListView.obj
 0002:00012288       __ehfuncinfo$??0?$QGuardedPtr@VQDockWindow@@@@QAE@XZ 10036288     cfg_widgets001:cfg_ListView.obj
 0002:00012288       __ehfuncinfo$?addSingleInputs@alm_process@@AAEXXZ 10036288     cfg_widgets001:cfg_ListView.obj
 0002:00012288       __ehfuncinfo$?addMultiInputs@alm_process@@AAEXXZ 10036288     cfg_widgets001:cfg_ListView.obj
 0002:00012288       __ehfuncinfo$?create@plugindesc@@UAEPAVconfig_plugin_base@@ABVQString@@00@Z 10036288     cfg_widgets001:cfg_ListView.obj
 0002:000122ac       __unwindtable$?showTime@cProc_dialog@@AAEXXZ 100362ac     cfg_widgets001:cfg_ListView.obj
 0002:000122ac       __unwindtable$?clipBoardDataChanged@cfg_Table@@IAEXXZ 100362ac     cfg_widgets001:cfg_ListView.obj
 0002:000122ac       __unwindtable$?clipBoardDataChanged@cfg_ListView@@IAEXXZ 100362ac     cfg_widgets001:cfg_ListView.obj
 0002:000122b4       __ehfuncinfo$?clipBoardDataChanged@cfg_ListView@@IAEXXZ 100362b4     cfg_widgets001:cfg_ListView.obj
 0002:000122b4       __ehfuncinfo$?clipBoardDataChanged@cfg_Table@@IAEXXZ 100362b4     cfg_widgets001:cfg_ListView.obj
 0002:000122b4       __ehfuncinfo$?showTime@cProc_dialog@@AAEXXZ 100362b4     cfg_widgets001:cfg_ListView.obj
 0002:000122d8       __unwindtable$?updateEntry@cfg_ListView@@AAEPAVQListViewItem@@QAV2@ABVQString@@_N@Z 100362d8     cfg_widgets001:cfg_ListView.obj
 0002:000122f8       __ehfuncinfo$?updateEntry@cfg_ListView@@AAEPAVQListViewItem@@QAV2@ABVQString@@_N@Z 100362f8     cfg_widgets001:cfg_ListView.obj
 0002:0001231c       __unwindtable$??0cfg_Table@@QAE@PAVQWidget@@PBD@Z 1003631c     cfg_widgets001:cfg_Table.obj
 0002:00012324       __ehfuncinfo$??0cfg_Table@@QAE@PAVQWidget@@PBD@Z 10036324     cfg_widgets001:cfg_Table.obj
 0002:00012348       __unwindtable$?deleteItems@cfg_Table@@QAEXXZ 10036348     cfg_widgets001:cfg_Table.obj
 0002:00012350       __ehfuncinfo$?deleteItems@cfg_Table@@QAEXXZ 10036350     cfg_widgets001:cfg_Table.obj
 0002:00012374       __unwindtable$?copyToClipboard@cfg_Table@@QAEXXZ 10036374     cfg_widgets001:cfg_Table.obj
 0002:0001238c       __ehfuncinfo$?copyToClipboard@cfg_Table@@QAEXXZ 1003638c     cfg_widgets001:cfg_Table.obj
 0002:000123b0       __unwindtable$?undoPaste@cfg_Table@@QAEXXZ 100363b0     cfg_widgets001:cfg_Table.obj
 0002:000123c8       __ehfuncinfo$?undoPaste@cfg_Table@@QAEXXZ 100363c8     cfg_widgets001:cfg_Table.obj
 0002:000123ec       __ehfuncinfo$?pasteClipboard@cfg_Table@@QAEXXZ 100363ec     cfg_widgets001:cfg_Table.obj
 0002:00012410       __unwindtable$?pasteClipboard@cfg_Table@@QAEXXZ 10036410     cfg_widgets001:cfg_Table.obj
 0002:00012480       __unwindtable$?fillUndoBuffer@cfg_Table@@AAEXXZ 10036480     cfg_widgets001:cfg_Table.obj
 0002:000124a0       __ehfuncinfo$?fillUndoBuffer@cfg_Table@@AAEXXZ 100364a0     cfg_widgets001:cfg_Table.obj
 0002:000124c8       __sehtable$__onexit        100364c8     MSVCRT:atonexit.obj
 0002:000124e8       __sehtable$??_L@YGXPAXIHP6EX0@Z1@Z 100364e8     MSVCRT:ehvecctr.obj
 0002:00012508       __sehtable$??_M@YGXPAXIHP6EX0@Z@Z 10036508     MSVCRT:ehvecdtr.obj
 0002:00012528       __sehtable$?__ArrayUnwind@@YGXPAXIHP6EX0@Z@Z 10036528     MSVCRT:ehvecdtr.obj
 0002:00012548       __sehtable$___DllMainCRTStartup 10036548     MSVCRT:crtdll.obj
 0002:00012570       __sehtable$__IsNonwritableInCurrentImage 10036570     MSVCRT:pesect.obj
 0002:00012590       .edata                     10036590     config_alm_process.exp
 0002:000125b8       rgpv                       100365b8     config_alm_process.exp
 0002:000126a8       rgszName                   100366a8     config_alm_process.exp
 0002:00012798       rgwOrd                     10036798     config_alm_process.exp
 0002:00012810       szName                     10036810     config_alm_process.exp
 0002:00012827       $N00001                    10036827     config_alm_process.exp
 0002:00012844       $N00002                    10036844     config_alm_process.exp
 0002:0001286b       $N00003                    1003686b     config_alm_process.exp
 0002:00012885       $N00004                    10036885     config_alm_process.exp
 0002:000128a9       $N00005                    100368a9     config_alm_process.exp
 0002:000128c1       $N00006                    100368c1     config_alm_process.exp
 0002:000128d6       $N00007                    100368d6     config_alm_process.exp
 0002:000128f7       $N00008                    100368f7     config_alm_process.exp
 0002:00012915       $N00009                    10036915     config_alm_process.exp
 0002:00012934       $N00010                    10036934     config_alm_process.exp
 0002:00012958       $N00011                    10036958     config_alm_process.exp
 0002:00012974       $N00012                    10036974     config_alm_process.exp
 0002:00012995       $N00013                    10036995     config_alm_process.exp
 0002:000129ae       $N00014                    100369ae     config_alm_process.exp
 0002:000129c4       $N00015                    100369c4     config_alm_process.exp
 0002:000129e6       $N00016                    100369e6     config_alm_process.exp
 0002:00012a05       $N00017                    10036a05     config_alm_process.exp
 0002:00012a25       $N00018                    10036a25     config_alm_process.exp
 0002:00012a50       $N00019                    10036a50     config_alm_process.exp
 0002:00012a78       $N00020                    10036a78     config_alm_process.exp
 0002:00012aa3       $N00021                    10036aa3     config_alm_process.exp
 0002:00012acb       $N00022                    10036acb     config_alm_process.exp
 0002:00012af1       $N00023                    10036af1     config_alm_process.exp
 0002:00012b14       $N00024                    10036b14     config_alm_process.exp
 0002:00012b35       $N00025                    10036b35     config_alm_process.exp
 0002:00012b53       $N00026                    10036b53     config_alm_process.exp
 0002:00012b75       $N00027                    10036b75     config_alm_process.exp
 0002:00012b94       $N00028                    10036b94     config_alm_process.exp
 0002:00012bb6       $N00029                    10036bb6     config_alm_process.exp
 0002:00012bd7       $N00030                    10036bd7     config_alm_process.exp
 0002:00012c01       $N00031                    10036c01     config_alm_process.exp
 0002:00012c28       $N00032                    10036c28     config_alm_process.exp
 0002:00012c58       $N00033                    10036c58     config_alm_process.exp
 0002:00012c85       $N00034                    10036c85     config_alm_process.exp
 0002:00012cc7       $N00035                    10036cc7     config_alm_process.exp
 0002:00012ce9       $N00036                    10036ce9     config_alm_process.exp
 0002:00012d12       $N00037                    10036d12     config_alm_process.exp
 0002:00012d38       $N00038                    10036d38     config_alm_process.exp
 0002:00012d5b       $N00039                    10036d5b     config_alm_process.exp
 0002:00012d7b       $N00040                    10036d7b     config_alm_process.exp
 0002:00012da8       $N00041                    10036da8     config_alm_process.exp
 0002:00012dd2       $N00042                    10036dd2     config_alm_process.exp
 0002:00012e01       $N00043                    10036e01     config_alm_process.exp
 0002:00012e2d       $N00044                    10036e2d     config_alm_process.exp
 0002:00012e5f       $N00045                    10036e5f     config_alm_process.exp
 0002:00012e8e       $N00046                    10036e8e     config_alm_process.exp
 0002:00012ed2       $N00047                    10036ed2     config_alm_process.exp
 0002:00012f13       $N00048                    10036f13     config_alm_process.exp
 0002:00012f35       $N00049                    10036f35     config_alm_process.exp
 0002:00012f6a       $N00050                    10036f6a     config_alm_process.exp
 0002:00012f9c       $N00051                    10036f9c     config_alm_process.exp
 0002:00012fc3       $N00052                    10036fc3     config_alm_process.exp
 0002:00012fe7       $N00053                    10036fe7     config_alm_process.exp
 0002:00013012       $N00054                    10037012     config_alm_process.exp
 0002:0001303a       $N00055                    1003703a     config_alm_process.exp
 0002:0001305a       $N00056                    1003705a     config_alm_process.exp
 0002:00013077       $N00057                    10037077     config_alm_process.exp
 0002:000130bd       $N00058                    100370bd     config_alm_process.exp
 0002:000130f1       $N00059                    100370f1     config_alm_process.exp
 0002:00013111       $N00060                    10037111     config_alm_process.exp
 0002:000220cc       .idata$6                   100460cc     qt-mt323:qt-mt323.dll
 0002:000222b2       .idata$6                   100462b2     alm_sys_select:alm_sys_select.dll
 0002:000222e6       .idata$6                   100462e6     config_icons:config_icons.dll
 0002:00022314       .idata$6                   10046314     kernel32:KERNEL32.dll
 0002:0002235c       .idata$6                   1004635c     msvcprt:MSVCP120.dll
 0002:000223e6       .idata$6                   100463e6     MSVCRT:MSVCR120.dll
 0003:00000000       _gate_xpm                  10048000     alm_process.obj
 0003:00000050       _checkCont_xpm             10048050     alm_process.obj
 0003:000000b0       _filesave                  100480b0     plugindesc.obj
 0003:00000100       ?param_slot_1@?3??staticMetaObject@alm_process@@SAPAVQMetaObject@@XZ@4QBUQUParameter@@B 10048100     moc_alm_process.obj
 0003:00000110       ?param_slot_12@?3??staticMetaObject@alm_process@@SAPAVQMetaObject@@XZ@4QBUQUParameter@@B 10048110     moc_alm_process.obj
 0003:00000120       ?param_slot_18@?3??staticMetaObject@alm_process@@SAPAVQMetaObject@@XZ@4QBUQUParameter@@B 10048120     moc_alm_process.obj
 0003:00000130       ?param_slot_24@?3??staticMetaObject@alm_process@@SAPAVQMetaObject@@XZ@4QBUQUParameter@@B 10048130     moc_alm_process.obj
 0003:00000160       ?param_slot_25@?3??staticMetaObject@alm_process@@SAPAVQMetaObject@@XZ@4QBUQUParameter@@B 10048160     moc_alm_process.obj
 0003:00000170       ?param_slot_26@?3??staticMetaObject@alm_process@@SAPAVQMetaObject@@XZ@4QBUQUParameter@@B 10048170     moc_alm_process.obj
 0003:000001a0       ?param_slot_27@?3??staticMetaObject@alm_process@@SAPAVQMetaObject@@XZ@4QBUQUParameter@@B 100481a0     moc_alm_process.obj
 0003:000001c0       ?param_slot_28@?3??staticMetaObject@alm_process@@SAPAVQMetaObject@@XZ@4QBUQUParameter@@B 100481c0     moc_alm_process.obj
 0003:000001f0       ?param_slot_29@?3??staticMetaObject@alm_process@@SAPAVQMetaObject@@XZ@4QBUQUParameter@@B 100481f0     moc_alm_process.obj
 0003:00000200       ?param_slot_2@?3??staticMetaObject@cProc_dialog@@SAPAVQMetaObject@@XZ@4QBUQUParameter@@B 10048200     moc_cProc_dialog.obj
 0003:00000210       ?param_slot_4@?3??staticMetaObject@cProc_dialog@@SAPAVQMetaObject@@XZ@4QBUQUParameter@@B 10048210     moc_cProc_dialog.obj
 0003:00000220       ?param_slot_5@?3??staticMetaObject@cProc_dialog@@SAPAVQMetaObject@@XZ@4QBUQUParameter@@B 10048220     moc_cProc_dialog.obj
 0003:00000230       ?param_slot_11@?3??staticMetaObject@cProc_dialog@@SAPAVQMetaObject@@XZ@4QBUQUParameter@@B 10048230     moc_cProc_dialog.obj
 0003:00000240       ?param_slot_12@?3??staticMetaObject@cProc_dialog@@SAPAVQMetaObject@@XZ@4QBUQUParameter@@B 10048240     moc_cProc_dialog.obj
 0003:00000250       ?param_slot_13@?3??staticMetaObject@cProc_dialog@@SAPAVQMetaObject@@XZ@4QBUQUParameter@@B 10048250     moc_cProc_dialog.obj
 0003:00000260       ?param_slot_14@?3??staticMetaObject@cProc_dialog@@SAPAVQMetaObject@@XZ@4QBUQUParameter@@B 10048260     moc_cProc_dialog.obj
 0003:00000270       ?param_slot_16@?3??staticMetaObject@cProc_dialog@@SAPAVQMetaObject@@XZ@4QBUQUParameter@@B 10048270     moc_cProc_dialog.obj
 0003:00000280       ?param_slot_17@?3??staticMetaObject@cProc_dialog@@SAPAVQMetaObject@@XZ@4QBUQUParameter@@B 10048280     moc_cProc_dialog.obj
 0003:000002a0       ?param_signal_0@?3??staticMetaObject@cProc_dialog@@SAPAVQMetaObject@@XZ@4QBUQUParameter@@B 100482a0     moc_cProc_dialog.obj
 0003:000002b0       ?param_signal_2@?3??staticMetaObject@cProc_dialog@@SAPAVQMetaObject@@XZ@4QBUQUParameter@@B 100482b0     moc_cProc_dialog.obj
 0003:000002c0       ?param_signal_3@?3??staticMetaObject@cProc_dialog@@SAPAVQMetaObject@@XZ@4QBUQUParameter@@B 100482c0     moc_cProc_dialog.obj
 0003:000002e0       ?param_signal_4@?3??staticMetaObject@cProc_dialog@@SAPAVQMetaObject@@XZ@4QBUQUParameter@@B 100482e0     moc_cProc_dialog.obj
 0003:00000310       ?param_slot_3@?3??staticMetaObject@multiInput@@SAPAVQMetaObject@@XZ@4QBUQUParameter@@B 10048310     moc_multiinputimpl.obj
 0003:00000320       ?param_slot_5@?3??staticMetaObject@multiInput@@SAPAVQMetaObject@@XZ@4QBUQUParameter@@B 10048320     moc_multiinputimpl.obj
 0003:00000330       ?param_slot_0@?3??staticMetaObject@singleInput@@SAPAVQMetaObject@@XZ@4QBUQUParameter@@B 10048330     moc_singleinputimpl.obj
 0003:00000340       ?param_slot_1@?3??staticMetaObject@singleInput@@SAPAVQMetaObject@@XZ@4QBUQUParameter@@B 10048340     moc_singleinputimpl.obj
 0003:00000350       ?param_slot_1@?3??staticMetaObject@template_dialog@@SAPAVQMetaObject@@XZ@4QBUQUParameter@@B 10048350     moc_template_dialogimpl.obj
 0003:00000360       ?param_slot_0@?3??staticMetaObject@config_mb4@@SAPAVQMetaObject@@XZ@4QBUQUParameter@@B 10048360     cfg_widgets001:moc_config_mb4impl.obj
 0003:00000d08       __Tuple_alloc              10048d08     alm_process.obj
 0003:00000d09       _ignore                    10048d09     alm_process.obj
 0003:00000d0a       _allocator_arg             10048d0a     alm_process.obj
 0003:00000d0b       _piecewise_construct       10048d0b     alm_process.obj
 0003:00000d14       __Tuple_alloc              10048d14     cProc_dialog.obj
 0003:00000d15       _ignore                    10048d15     cProc_dialog.obj
 0003:00000d16       _allocator_arg             10048d16     cProc_dialog.obj
 0003:00000d17       _piecewise_construct       10048d17     cProc_dialog.obj
 0003:00000d1c       __Tuple_alloc              10048d1c     cProcess.obj
 0003:00000d1d       _ignore                    10048d1d     cProcess.obj
 0003:00000d1e       _allocator_arg             10048d1e     cProcess.obj
 0003:00000d1f       _piecewise_construct       10048d1f     cProcess.obj
 0003:00000d24       __Tuple_alloc              10048d24     multiinputimpl.obj
 0003:00000d25       _ignore                    10048d25     multiinputimpl.obj
 0003:00000d26       _allocator_arg             10048d26     multiinputimpl.obj
 0003:00000d27       _piecewise_construct       10048d27     multiinputimpl.obj
 0003:00000d28       __Tuple_alloc              10048d28     singleinputimpl.obj
 0003:00000d29       _ignore                    10048d29     singleinputimpl.obj
 0003:00000d2a       _allocator_arg             10048d2a     singleinputimpl.obj
 0003:00000d2b       _piecewise_construct       10048d2b     singleinputimpl.obj
 0003:00000d2c       __Tuple_alloc              10048d2c     template_dialogimpl.obj
 0003:00000d2d       _ignore                    10048d2d     template_dialogimpl.obj
 0003:00000d2e       _allocator_arg             10048d2e     template_dialogimpl.obj
 0003:00000d2f       _piecewise_construct       10048d2f     template_dialogimpl.obj
 0003:00000d3c       _cleanUp_alm_process       10048d3c     moc_alm_process.obj
 0003:00000d40       ?$S1@?3??staticMetaObject@alm_process@@SAPAVQMetaObject@@XZ@4IA 10048d40     moc_alm_process.obj
 0003:00000d44       ?param_slot_17@?3??staticMetaObject@alm_process@@SAPAVQMetaObject@@XZ@4QBUQUParameter@@B 10048d44     moc_alm_process.obj
 0003:00000d64       ?param_signal_0@?3??staticMetaObject@alm_process@@SAPAVQMetaObject@@XZ@4QBUQUParameter@@B 10048d64     moc_alm_process.obj
 0003:00000d88       _cleanUp_CheckContDialog   10048d88     moc_checkContDialogImpl.obj
 0003:00000d90       _cleanUp_CheckContDialogBase 10048d90     moc_checkcontributiondialog.obj
 0003:00000d98       _cleanUp_cProc_dialog      10048d98     moc_cProc_dialog.obj
 0003:00000d9c       ?$S1@?3??staticMetaObject@cProc_dialog@@SAPAVQMetaObject@@XZ@4IA 10048d9c     moc_cProc_dialog.obj
 0003:00000da0       ?param_slot_3@?3??staticMetaObject@cProc_dialog@@SAPAVQMetaObject@@XZ@4QBUQUParameter@@B 10048da0     moc_cProc_dialog.obj
 0003:00000db0       ?param_slot_6@?3??staticMetaObject@cProc_dialog@@SAPAVQMetaObject@@XZ@4QBUQUParameter@@B 10048db0     moc_cProc_dialog.obj
 0003:00000dd4       _cleanUp_LatchAckDialogBase 10048dd4     moc_latchackdialog.obj
 0003:00000ddc       _cleanUp_LatchAckDialog    10048ddc     moc_latchackdialogimpl.obj
 0003:00000de4       _cleanUp_multiInputBase    10048de4     moc_multiinput.obj
 0003:00000dec       __Tuple_alloc              10048dec     moc_multiinputimpl.obj
 0003:00000ded       _ignore                    10048ded     moc_multiinputimpl.obj
 0003:00000dee       _allocator_arg             10048dee     moc_multiinputimpl.obj
 0003:00000def       _piecewise_construct       10048def     moc_multiinputimpl.obj
 0003:00000df0       _cleanUp_multiInput        10048df0     moc_multiinputimpl.obj
 0003:00000df4       ?$S1@?3??staticMetaObject@multiInput@@SAPAVQMetaObject@@XZ@4IA 10048df4     moc_multiinputimpl.obj
 0003:00000df8       ?param_slot_6@?3??staticMetaObject@multiInput@@SAPAVQMetaObject@@XZ@4QBUQUParameter@@B 10048df8     moc_multiinputimpl.obj
 0003:00000e0c       _cleanUp_proc_config       10048e0c     moc_proc_config.obj
 0003:00000e14       _cleanUp_singleInputBase   10048e14     moc_singleinput.obj
 0003:00000e1c       __Tuple_alloc              10048e1c     moc_singleinputimpl.obj
 0003:00000e1d       _ignore                    10048e1d     moc_singleinputimpl.obj
 0003:00000e1e       _allocator_arg             10048e1e     moc_singleinputimpl.obj
 0003:00000e1f       _piecewise_construct       10048e1f     moc_singleinputimpl.obj
 0003:00000e20       _cleanUp_singleInput       10048e20     moc_singleinputimpl.obj
 0003:00000e24       ?$S1@?3??staticMetaObject@singleInput@@SAPAVQMetaObject@@XZ@4IA 10048e24     moc_singleinputimpl.obj
 0003:00000e2c       _cleanUp_template_dialogBase 10048e2c     moc_template_dialog.obj
 0003:00000e34       __Tuple_alloc              10048e34     moc_template_dialogimpl.obj
 0003:00000e35       _ignore                    10048e35     moc_template_dialogimpl.obj
 0003:00000e36       _allocator_arg             10048e36     moc_template_dialogimpl.obj
 0003:00000e37       _piecewise_construct       10048e37     moc_template_dialogimpl.obj
 0003:00000e38       _cleanUp_template_dialog   10048e38     moc_template_dialogimpl.obj
 0003:00000e3c       ?param_slot_0@?3??staticMetaObject@template_dialog@@SAPAVQMetaObject@@XZ@4QBUQUParameter@@B 10048e3c     moc_template_dialogimpl.obj
 0003:00000e4c       ?$S1@?3??staticMetaObject@template_dialog@@SAPAVQMetaObject@@XZ@4IA 10048e4c     moc_template_dialogimpl.obj
 0003:00000e54       _cleanUp_config_mb4        10048e54     cfg_widgets001:moc_config_mb4impl.obj
 0003:00000e58       ?$S1@?3??staticMetaObject@config_mb4@@SAPAVQMetaObject@@XZ@4IA 10048e58     cfg_widgets001:moc_config_mb4impl.obj
 0003:00000e60       _cleanUp_cfg_ListView      10048e60     cfg_widgets001:moc_cfg_ListView.obj
 0003:00000e64       ?param_signal_1@?3??staticMetaObject@cfg_ListView@@SAPAVQMetaObject@@XZ@4QBUQUParameter@@B 10048e64     cfg_widgets001:moc_cfg_ListView.obj
 0003:00000e74       ?$S1@?3??staticMetaObject@cfg_ListView@@SAPAVQMetaObject@@XZ@4IA 10048e74     cfg_widgets001:moc_cfg_ListView.obj
 0003:00000e7c       _cleanUp_cfg_Table         10048e7c     cfg_widgets001:moc_cfg_Table.obj
 0003:00000e80       ?param_signal_1@?3??staticMetaObject@cfg_Table@@SAPAVQMetaObject@@XZ@4QBUQUParameter@@B 10048e80     cfg_widgets001:moc_cfg_Table.obj
 0003:00000e90       ?$S1@?3??staticMetaObject@cfg_Table@@SAPAVQMetaObject@@XZ@4IA 10048e90     cfg_widgets001:moc_cfg_Table.obj
 0003:00000e94       ___proc_attached           10048e94     MSVCRT:crtdll.obj
 0003:00000e98       _GS_ExceptionRecord        10048e98     MSVCRT:gs_report.obj
 0003:00000ee8       _GS_ContextRecord          10048ee8     MSVCRT:gs_report.obj
 0003:000011b4       _DebuggerWasPresent        100491b4     MSVCRT:gs_report.obj
 0004:000000a0       $R000000                   1004a0a0     version.res
 0004:00000548       $R0004A8                   1004a548     version.res
